 luafar3

 Timestamp is 58ab93ea (Tue Feb 21 04:12:10 2017)

 Preferred load address is 10000000

 Start         Length     Name                   Class
 0001:00000000 00000004H .CRT$XCA                CODE
 0001:00000004 00000004H .CRT$XCZ                CODE
 0001:00000008 00000004H .CRT$XIA                CODE
 0001:0000000c 0000000cH .CRT$XIC                CODE
 0001:00000018 00000004H .CRT$XIZ                CODE
 0001:0000001c 00000004H .CRT$XPA                CODE
 0001:00000020 0000000cH .CRT$XPX                CODE
 0001:0000002c 00000004H .CRT$XPXA               CODE
 0001:00000030 00000004H .CRT$XPZ                CODE
 0001:00000034 00000004H .CRT$XTA                CODE
 0001:00000038 00000008H .CRT$XTZ                CODE
 0001:00000040 00015440H .rdata                  CODE
 0001:0001547c 00000000H .rdata$r                CODE
 0001:00015480 0000000cH .rdata$sxdata           CODE
 0001:0001548c 0000028cH .rdata$zzzdbg           CODE
 0001:00015718 00000004H .rtc$IAA                CODE
 0001:0001571c 00000004H .rtc$IZZ                CODE
 0001:00015720 00000004H .rtc$TAA                CODE
 0001:00015724 0000000cH .rtc$TZZ                CODE
 0001:00015730 00039208H .text$mn                CODE
 0001:0004e938 000007c8H .xdata$x                CODE
 0001:0004f100 00000482H .edata                  CODE
 0002:00000000 00008530H .data                   DATA
 0002:00008530 00000000H .data$r                 DATA
 0002:00008530 00000abcH .bss                    DATA
 0003:00000000 00000360H .idata$5                DATA
 0003:00000360 00000004H .00cfg                  DATA
 0003:00000364 00000078H .idata$2                DATA
 0003:000003dc 00000014H .idata$3                DATA
 0003:000003f0 00000360H .idata$4                DATA
 0003:00000750 00000ec8H .idata$6                DATA
 0004:00000000 00000090H .gfids$x                DATA
 0004:00000090 00000014H .gfids$y                DATA
 0005:00000000 00000060H .rsrc$01                DATA
 0005:00000060 00000358H .rsrc$02                DATA

  Address         Publics by Value              Rva+Base       Lib:Object

 0000:00000000       ___guard_longjmp_count     00000000     <absolute>
 0000:00000000       ___guard_fids_count        00000000     <absolute>
 0000:00000000       __except_list              00000000     <absolute>
 0000:00000000       ___guard_longjmp_table     00000000     <absolute>
 0000:00000000       ___guard_iat_table         00000000     <absolute>
 0000:00000000       ___guard_iat_count         00000000     <absolute>
 0000:00000000       ___dynamic_value_reloc_table 00000000     <absolute>
 0000:00000000       ___guard_fids_table        00000000     <absolute>
 0000:00000003       ___safe_se_handler_count   00000003     <absolute>
 0000:00000100       ___guard_flags             00000100     <absolute>
 0000:00000000       ___ImageBase               10000000     <linker-defined>
 0001:00000000       ___xc_a                    10001000     LIBCMT:initializers.obj
 0001:00000004       ___xc_z                    10001004     LIBCMT:initializers.obj
 0001:00000008       ___xi_a                    10001008     LIBCMT:initializers.obj
 0001:0000000c       ___acrt_stdio_initializer  1000100c     libucrt:stdio_initializer.obj
 0001:00000010       ___acrt_multibyte_initializer 10001010     libucrt:multibyte_initializer.obj
 0001:00000014       ___acrt_tran_sse2_initializer 10001014     libucrt:sse2_initializer.obj
 0001:00000018       ___xi_z                    10001018     LIBCMT:initializers.obj
 0001:0000001c       ___xp_a                    1000101c     LIBCMT:initializers.obj
 0001:00000020       ___acrt_locale_terminator  10001020     libucrt:locale_initializer.obj
 0001:00000024       ___acrt_tmpfile_terminator 10001024     libucrt:tmpfile_initializer.obj
 0001:00000028       ___dcrt_console_output_terminator 10001028     libucrt:console_output_initializer.obj
 0001:0000002c       ___acrt_stdio_terminator   1000102c     libucrt:stdio_initializer.obj
 0001:00000030       ___xp_z                    10001030     LIBCMT:initializers.obj
 0001:00000034       ___xt_a                    10001034     LIBCMT:initializers.obj
 0001:00000038       ___xt_z                    10001038     LIBCMT:initializers.obj
 0001:00000040       _metatable_name            10001040     bit64.obj
 0001:00000138       ??_C@_04JAOJMBA@bnot?$AA@  10001138     bit64.obj
 0001:00000140       ??_C@_04BKGNPECA@band?$AA@ 10001140     bit64.obj
 0001:00000148       ??_C@_03BBBGIIAC@bor?$AA@  10001148     bit64.obj
 0001:0000014c       ??_C@_04CKCGDDNF@bxor?$AA@ 1000114c     bit64.obj
 0001:00000154       ??_C@_06ELFGPGBK@lshift?$AA@ 10001154     bit64.obj
 0001:0000015c       ??_C@_06HMLHBBIJ@rshift?$AA@ 1000115c     bit64.obj
 0001:00000164       ??_C@_07JILILBLL@arshift?$AA@ 10001164     bit64.obj
 0001:0000016c       ??_C@_03CLCAEGCJ@new?$AA@  1000116c     bit64.obj
 0001:00000170       ??_C@_03BDGOHNNK@add?$AA@  10001170     bit64.obj
 0001:00000174       ??_C@_03KCMAIMAP@sub?$AA@  10001174     bit64.obj
 0001:00000178       ??_C@_03IMIFIBCN@mul?$AA@  10001178     bit64.obj
 0001:0000017c       ??_C@_03FEJMGOGI@div?$AA@  1000117c     bit64.obj
 0001:00000180       ??_C@_03FFONCNID@mod?$AA@  10001180     bit64.obj
 0001:00000184       ??_C@_02HIIGGHJB@eq?$AA@   10001184     bit64.obj
 0001:00000188       ??_C@_02KCAKIFL@lt?$AA@    10001188     bit64.obj
 0001:0000018c       ??_C@_02FJPJILEL@le?$AA@   1000118c     bit64.obj
 0001:00000190       ??_C@_04GPMDFGEJ@type?$AA@ 10001190     bit64.obj
 0001:00000198       ??_C@_05MEHDOBFN@__add?$AA@ 10001198     bit64.obj
 0001:000001a0       ??_C@_05HFNNBAII@__sub?$AA@ 100011a0     bit64.obj
 0001:000001a8       ??_C@_05FLJIBNKK@__mul?$AA@ 100011a8     bit64.obj
 0001:000001b0       ??_C@_05IDIBPCOP@__div?$AA@ 100011b0     bit64.obj
 0001:000001b8       ??_C@_05ICPALBAE@__mod?$AA@ 100011b8     bit64.obj
 0001:000001c0       ??_C@_05MHFNBPAK@__unm?$AA@ 100011c0     bit64.obj
 0001:000001c8       ??_C@_04GIMIAOHA@__eq?$AA@ 100011c8     bit64.obj
 0001:000001d0       ??_C@_04BKGOMBLK@__lt?$AA@ 100011d0     bit64.obj
 0001:000001d8       ??_C@_04EJLHOCKK@__le?$AA@ 100011d8     bit64.obj
 0001:000001e0       ??_C@_0L@HDFPAPPH@__tostring?$AA@ 100011e0     bit64.obj
 0001:000001ec       ??_C@_09GPALILFO@bad?5int64?$AA@ 100011ec     bit64.obj
 0001:000001f8       ??_C@_05LLAMLEHD@?$CFI64d?$AA@ 100011f8     bit64.obj
 0001:00000200       ??_C@_05OALCLICP@bit64?$AA@ 10001200     bit64.obj
 0001:00000208       __real@433fffffffffffff    10001208     bit64.obj
 0001:000004f8       _COLLECTOR_FD              100014f8     exported.obj
 0001:0000050c       _COLLECTOR_OPI             1000150c     exported.obj
 0001:00000538       _COLLECTOR_PI              10001538     exported.obj
 0001:00000568       _KEY_OBJECT                10001568     exported.obj
 0001:00000af8       ??_C@_05GFCDIDHO@debug?$AA@ 10001af8     exported.obj
 0001:00000b00       ??_C@_09GPFEECNC@traceback?$AA@ 10001b00     exported.obj
 0001:00000b0c       ??_C@_06NKNNMLDJ@export?$AA@ 10001b0c     exported.obj
 0001:00000b14       ??_C@_07PCNKBAGB@OnError?$AA@ 10001b14     exported.obj
 0001:00000b1c       ??_C@_0N@NJMIGDDL@CreationTime?$AA@ 10001b1c     exported.obj
 0001:00000b2c       ??_C@_0P@MFHPCDDH@LastAccessTime?$AA@ 10001b2c     exported.obj
 0001:00000b3c       ??_C@_0O@FCFNCAHK@LastWriteTime?$AA@ 10001b3c     exported.obj
 0001:00000b4c       ??_C@_0L@FCILKIIG@ChangeTime?$AA@ 10001b4c     exported.obj
 0001:00000b58       ??_C@_08BHIEONMC@FileSize?$AA@ 10001b58     exported.obj
 0001:00000b64       ??_C@_0P@JBACEJLL@AllocationSize?$AA@ 10001b64     exported.obj
 0001:00000b74       ??_C@_05BOOEKJH@Flags?$AA@ 10001b74     exported.obj
 0001:00000b7c       ??_C@_0O@DLGJHFNH@NumberOfLinks?$AA@ 10001b7c     exported.obj
 0001:00000b8c       ??_C@_05MHNOECFO@CRC32?$AA@ 10001b8c     exported.obj
 0001:00000b94       ??_C@_08FDCJCDOL@FileName?$AA@ 10001b94     exported.obj
 0001:00000ba0       ??_C@_0BC@COCBGKAE@AlternateFileName?$AA@ 10001ba0     exported.obj
 0001:00000bb4       ??_C@_0M@OHKMKKDH@Description?$AA@ 10001bb4     exported.obj
 0001:00000bc0       ??_C@_05HDCNEILF@Owner?$AA@ 10001bc0     exported.obj
 0001:00000bc8       ??_C@_0BB@OKGMKOG@CustomColumnData?$AA@ 10001bc8     exported.obj
 0001:00000bdc       ??_C@_11LOCGONAA@?$AA?$AA@ 10001bdc     exported.obj
 0001:00000be0       ??_C@_08JNHPECBG@UserData?$AA@ 10001be0     exported.obj
 0001:00000bec       ??_C@_0M@DFMHDHBL@GetFindData?$AA@ 10001bec     exported.obj
 0001:00000bf8       ??_C@_08FFPEEIHA@GetFiles?$AA@ 10001bf8     exported.obj
 0001:00000c04       ??_C@_0BC@IECOKJFL@GetFiles?4DestPath?$AA@ 10001c04     exported.obj
 0001:00000c18       ??_C@_05LFOKGKBN@?$DMboot?$AA@ 10001c18     exported.obj
 0001:00000c20       ??_C@_15CBMDENPJ@?$AA?4?$AA?9?$AA?$AA@ 10001c20     exported.obj
 0001:00000c28       ??_C@_07KNEGBPNO@package?$AA@ 10001c28     exported.obj
 0001:00000c30       ??_C@_07GCEAJMEA@preload?$AA@ 10001c30     exported.obj
 0001:00000c38       ??_C@_19BCNABNAK@?$AA?4?$AAl?$AAu?$AAa?$AA?$AA@ 10001c38     exported.obj
 0001:00000c44       ??_C@_13BPINEIPE@?$AAr?$AA?$AA@ 10001c44     exported.obj
 0001:00000c48       ??_C@_1DC@PABHCCON@?$AAD?$AAe?$AAf?$AAa?$AAu?$AAl?$AAt?$AA?5?$AAs?$AAc?$AAr?$AAi?$AAp?$AAt?$AA?5?$AAn?$AAo?$AAt?$AA?5?$AAf?$AAo?$AAu?$AAn?$AAd?$AA?$AA@ 10001c48     exported.obj
 0001:00000c7c       ??_C@_03JEOKDCFP@far?$AA@  10001c7c     exported.obj
 0001:00000c80       ??_C@_0BE@HCPAIELH@ReloadDefaultScript?$AA@ 10001c80     exported.obj
 0001:00000c94       ??_C@_0L@OCPPMCCK@StructSize?$AA@ 10001c94     exported.obj
 0001:00000ca0       ??_C@_06LBMCOACO@Buffer?$AA@ 10001ca0     exported.obj
 0001:00000ca8       ??_C@_06EPIAKPGD@OpMode?$AA@ 10001ca8     exported.obj
 0001:00000cb0       ??_C@_07GDADDFBD@Analyse?$AA@ 10001cb0     exported.obj
 0001:00000cb8       ??_C@_0BB@CKIGBGLB@GetOpenPanelInfo?$AA@ 10001cb8     exported.obj
 0001:00000ccc       ??_C@_05ELNJBDOO@reuse?$AA@ 10001ccc     exported.obj
 0001:00000cd8       ??_C@_1EO@OOOCECGK@?$AAG?$AAe?$AAt?$AAO?$AAp?$AAe?$AAn?$AAP?$AAa?$AAn?$AAe?$AAl?$AAI?$AAn?$AAf?$AAo?$AA?5?$AAs?$AAh?$AAo?$AAu?$AAl?$AAd?$AA?5?$AAr?$AAe?$AAt?$AAu?$AAr?$AAn?$AA?5?$AAa@ 10001cd8     exported.obj
 0001:00000d28       ??_C@_08KDMNIFGM@FreeSize?$AA@ 10001d28     exported.obj
 0001:00000d34       ??_C@_08PAJOMFPO@HostFile?$AA@ 10001d34     exported.obj
 0001:00000d40       ??_C@_06IBPEEEAJ@CurDir?$AA@ 10001d40     exported.obj
 0001:00000d48       ??_C@_06PEPCFMNJ@Format?$AA@ 10001d48     exported.obj
 0001:00000d50       ??_C@_0L@CMHIOLLB@PanelTitle?$AA@ 10001d50     exported.obj
 0001:00000d5c       ??_C@_09PMEOAIAA@InfoLines?$AA@ 10001d5c     exported.obj
 0001:00000d68       ??_C@_0BA@BLCGOCOG@InfoLinesNumber?$AA@ 10001d68     exported.obj
 0001:00000d78       ??_C@_04OJAHODMC@Text?$AA@ 10001d78     exported.obj
 0001:00000d80       ??_C@_04DICKPMGH@Data?$AA@ 10001d80     exported.obj
 0001:00000d88       ??_C@_0L@FPEHOFAI@DescrFiles?$AA@ 10001d88     exported.obj
 0001:00000d94       ??_C@_0BA@BBOGKOKF@PanelModesArray?$AA@ 10001d94     exported.obj
 0001:00000da4       ??_C@_0BB@LFNABPEF@PanelModesNumber?$AA@ 10001da4     exported.obj
 0001:00000db8       ??_C@_0M@KDJPJFOF@ColumnTypes?$AA@ 10001db8     exported.obj
 0001:00000dc4       ??_C@_0N@ILFJPGHI@ColumnWidths?$AA@ 10001dc4     exported.obj
 0001:00000dd4       ??_C@_0BC@KELOOKNK@StatusColumnTypes?$AA@ 10001dd4     exported.obj
 0001:00000de8       ??_C@_0BD@DNDIPKDK@StatusColumnWidths?$AA@ 10001de8     exported.obj
 0001:00000dfc       ??_C@_0N@EHCEJHEE@ColumnTitles?$AA@ 10001dfc     exported.obj
 0001:00000e0c       ??_C@_0P@BEEDPJDK@StartPanelMode?$AA@ 10001e0c     exported.obj
 0001:00000e1c       ??_C@_0O@NIFKFGBJ@StartSortMode?$AA@ 10001e1c     exported.obj
 0001:00000e2c       ??_C@_0P@KMACBLNK@StartSortOrder?$AA@ 10001e2c     exported.obj
 0001:00000e3c       ??_C@_06ONGFDHIA@KeyBar?$AA@ 10001e3c     exported.obj
 0001:00000e44       ??_C@_0P@PKDBPEJI@VirtualKeyCode?$AA@ 10001e44     exported.obj
 0001:00000e54       ??_C@_0BA@MFFHAKP@ControlKeyState?$AA@ 10001e54     exported.obj
 0001:00000e64       ??_C@_08DGDJEKCP@LongText?$AA@ 10001e64     exported.obj
 0001:00000e70       ??_C@_0N@IHDKLODA@ShortcutData?$AA@ 10001e70     exported.obj
 0001:00000e80       ??_C@_05HIFJDKLD@array?$AA@ 10001e80     exported.obj
 0001:00000e88       ??_C@_01EFFIKLCJ@n?$AA@    10001e88     exported.obj
 0001:00000e8a       ??_C@_00CNPNBAHC@?$AA@     10001e8a     exported.obj
 0001:00000e8c       ??_C@_04DNCDCIAE@Open?$AA@ 10001e8c     exported.obj
 0001:00000e94       ??_C@_04OPJIDECA@hDlg?$AA@ 10001e94     exported.obj
 0001:00000e9c       ??_C@_06BNNOMDLO@Handle?$AA@ 10001e9c     exported.obj
 0001:00000ea4       ??_C@_05LNOAKADA@panel?$AA@ 10001ea4     exported.obj
 0001:00000eac       ??_C@_0L@JMPDJFBN@ClosePanel?$AA@ 10001eac     exported.obj
 0001:00000eb8       ??_C@_07MBOMJGGF@Compare?$AA@ 10001eb8     exported.obj
 0001:00000ec0       ??_C@_09NANCCILE@Configure?$AA@ 10001ec0     exported.obj
 0001:00000ecc       ??_C@_0M@MMKKMEFA@DeleteFiles?$AA@ 10001ecc     exported.obj
 0001:00000ed8       ??_C@_0O@GLLEDHJA@MakeDirectory?$AA@ 10001ed8     exported.obj
 0001:00000ee8       ??_C@_0BD@PJNONGDB@MakeDirectory?4Name?$AA@ 10001ee8     exported.obj
 0001:00000efc       ??_C@_0BC@COPMJGBI@ProcessPanelEvent?$AA@ 10001efc     exported.obj
 0001:00000f10       ??_C@_0BA@DPJAKFGC@ProcessHostFile?$AA@ 10001f10     exported.obj
 0001:00000f20       ??_C@_0BC@HOBKGBBM@ProcessPanelInput?$AA@ 10001f20     exported.obj
 0001:00000f34       ??_C@_08OBOOFGOD@PutFiles?$AA@ 10001f34     exported.obj
 0001:00000f40       ??_C@_0N@KCFEBPAO@SetDirectory?$AA@ 10001f40     exported.obj
 0001:00000f50       ??_C@_0M@PNOHHCCH@SetFindList?$AA@ 10001f50     exported.obj
 0001:00000f5c       ??_C@_07EACELFAO@ExitFAR?$AA@ 10001f5c     exported.obj
 0001:00000f64       ??_C@_0O@JHMGCIHI@FarTimerQueue?$AA@ 10001f64     exported.obj
 0001:00000f74       ??_C@_0O@OBCKADMD@GetPluginInfo?$AA@ 10001f74     exported.obj
 0001:00000f84       ??_C@_0O@GDMHGAFH@CommandPrefix?$AA@ 10001f84     exported.obj
 0001:00000f94       ??_C@_0O@PHBKMNMJ@DiskMenuGuids?$AA@ 10001f94     exported.obj
 0001:00000fa4       ??_C@_0BA@NLBDFPEO@DiskMenuStrings?$AA@ 10001fa4     exported.obj
 0001:00000fb4       ??_C@_0BA@FOMPNLJF@PluginMenuGuids?$AA@ 10001fb4     exported.obj
 0001:00000fc4       ??_C@_0BC@DJMJFBJC@PluginMenuStrings?$AA@ 10001fc4     exported.obj
 0001:00000fd8       ??_C@_0BC@ILBHAHCH@PluginConfigGuids?$AA@ 10001fd8     exported.obj
 0001:00000fec       ??_C@_0BE@GAFPNGIP@PluginConfigStrings?$AA@ 10001fec     exported.obj
 0001:00001000       ??_C@_0BD@DECJPBBK@ProcessEditorInput?$AA@ 10002000     exported.obj
 0001:00001014       ??_C@_0BD@GEMPAGBO@ProcessEditorEvent?$AA@ 10002014     exported.obj
 0001:00001028       ??_C@_04KOACHJEN@Type?$AA@ 10002028     exported.obj
 0001:00001030       ??_C@_0N@EKPHGDMI@StringNumber?$AA@ 10002030     exported.obj
 0001:00001040       ??_C@_07MOCFLHCN@FileEOL?$AA@ 10002040     exported.obj
 0001:00001048       ??_C@_08DOHJINHB@CodePage?$AA@ 10002048     exported.obj
 0001:00001054       ??_C@_0BD@GGKMLEJG@ProcessViewerEvent?$AA@ 10002054     exported.obj
 0001:00001068       ??_C@_0BD@FNHBEIC@ProcessDialogEvent?$AA@ 10002068     exported.obj
 0001:0000107c       ??_C@_06CPBJDKAC@Param2?$AA@ 1000207c     exported.obj
 0001:00001084       ??_C@_06EDEGJMB@Param1?$AA@ 10002084     exported.obj
 0001:0000108c       ??_C@_03MLMOILGK@Msg?$AA@  1000208c     exported.obj
 0001:00001090       ??_C@_0BE@LHJGGGHN@ProcessSynchroEvent?$AA@ 10002090     exported.obj
 0001:000010a4       ??_C@_0BB@PHIEFGHD@GetContentFields?$AA@ 100020a4     exported.obj
 0001:000010b8       ??_C@_0P@DPJDPMPI@GetContentData?$AA@ 100020b8     exported.obj
 0001:000010c8       ??_C@_0N@DDJEHLKE@?$DM_globalinfo?$AA@ 100020c8     exported.obj
 0001:000010d8       ??_C@_1CA@IBKDMBNJ@?$AA_?$AAg?$AAl?$AAo?$AAb?$AAa?$AAl?$AAi?$AAn?$AAf?$AAo?$AA?4?$AAl?$AAu?$AAa?$AA?$AA@ 100020d8     exported.obj
 0001:000010f8       ??_C@_0O@GJMOPLGM@GetGlobalInfo?$AA@ 100020f8     exported.obj
 0001:00001108       ??_C@_0O@CALOEOI@MinFarVersion?$AA@ 10002108     exported.obj
 0001:00001118       ??_C@_07NGFJPNPN@Version?$AA@ 10002118     exported.obj
 0001:00001120       ??_C@_04MJHIICBJ@Guid?$AA@ 10002120     exported.obj
 0001:00001128       ??_C@_05PABKJLOM@Title?$AA@ 10002128     exported.obj
 0001:00001130       ??_C@_06HHECMMLE@Author?$AA@ 10002130     exported.obj
 0001:00001138       ??_C@_0BE@DONMOPMJ@ProcessConsoleInput?$AA@ 10002138     exported.obj
 0001:00001150       __real@43e0000000000000    10002150     exported.obj
 0001:00001158       __real@bff0000000000000    10002158     exported.obj
 0001:000017f0       _Vals                      100027f0     flags.obj
 0001:00003028       ??_C@_0BI@IDKIJMME@FARMANAGERVERSION_MAJOR?$AA@ 10004028     flags.obj
 0001:00003040       ??_C@_0BI@DMLKEAFC@FARMANAGERVERSION_MINOR?$AA@ 10004040     flags.obj
 0001:00003058       ??_C@_0BL@NMALNAFP@FARMANAGERVERSION_REVISION?$AA@ 10004058     flags.obj
 0001:00003074       ??_C@_0BI@OLPFLLDD@FARMANAGERVERSION_BUILD?$AA@ 10004074     flags.obj
 0001:0000308c       ??_C@_0BI@MOOFLFPC@FARMANAGERVERSION_STAGE?$AA@ 1000408c     flags.obj
 0001:000030a4       ??_C@_0L@MIDBGFJO@CP_UNICODE?$AA@ 100040a4     flags.obj
 0001:000030b0       ??_C@_0O@MNMCMEJH@CP_REVERSEBOM?$AA@ 100040b0     flags.obj
 0001:000030c0       ??_C@_0L@JDNPCEDH@CP_DEFAULT?$AA@ 100040c0     flags.obj
 0001:000030cc       ??_C@_0M@OMCMFJHA@CP_REDETECT?$AA@ 100040cc     flags.obj
 0001:000030d8       ??_C@_09MNAPNKKC@INDEXMASK?$AA@ 100040d8     flags.obj
 0001:000030e4       ??_C@_09BLFIDJLF@COLORMASK?$AA@ 100040e4     flags.obj
 0001:000030f0       ??_C@_09ENNBLPJC@ALPHAMASK?$AA@ 100040f0     flags.obj
 0001:000030fc       ??_C@_0L@EHFOPLFD@PANEL_NONE?$AA@ 100040fc     flags.obj
 0001:00003108       ??_C@_0N@LPMKALBG@PANEL_ACTIVE?$AA@ 10004108     flags.obj
 0001:00003118       ??_C@_0O@HPKEABPN@PANEL_PASSIVE?$AA@ 10004118     flags.obj
 0001:00003128       ??_C@_0L@GOEBPENN@PANEL_STOP?$AA@ 10004128     flags.obj
 0001:00003134       ??_C@_0N@HLIFAAPJ@EEREDRAW_ALL?$AA@ 10004134     flags.obj
 0001:00003144       ??_C@_0P@NHNDIKJ@CURRENT_EDITOR?$AA@ 10004144     flags.obj
 0001:00003154       ??_C@_0BN@PPNDCHHA@EDITOR_COLOR_NORMAL_PRIORITY?$AA@ 10004154     flags.obj
 0001:00003174       ??_C@_07MGGAEAFF@DI_TEXT?$AA@ 10004174     flags.obj
 0001:0000317c       ??_C@_08HODBDEHE@DI_VTEXT?$AA@ 1000417c     flags.obj
 0001:00003188       ??_C@_0N@IGKKGFMF@DI_SINGLEBOX?$AA@ 10004188     flags.obj
 0001:00003198       ??_C@_0N@EDCLIEAE@DI_DOUBLEBOX?$AA@ 10004198     flags.obj
 0001:000031a8       ??_C@_07DOLIFAEF@DI_EDIT?$AA@ 100041a8     flags.obj
 0001:000031b0       ??_C@_0L@EOMEIIFM@DI_PSWEDIT?$AA@ 100041b0     flags.obj
 0001:000031bc       ??_C@_0L@MGOIMBKF@DI_FIXEDIT?$AA@ 100041bc     flags.obj
 0001:000031c8       ??_C@_09GGAEMAPJ@DI_BUTTON?$AA@ 100041c8     flags.obj
 0001:000031d4       ??_C@_0M@MHFHGPHJ@DI_CHECKBOX?$AA@ 100041d4     flags.obj
 0001:000031e0       ??_C@_0P@GIPCGMBE@DI_RADIOBUTTON?$AA@ 100041e0     flags.obj
 0001:000031f0       ??_C@_0M@MAKBFNGC@DI_COMBOBOX?$AA@ 100041f0     flags.obj
 0001:000031fc       ??_C@_0L@ONDMPPPO@DI_LISTBOX?$AA@ 100041fc     flags.obj
 0001:00003208       ??_C@_0P@GDJDPEIK@DI_USERCONTROL?$AA@ 10004208     flags.obj
 0001:00003218       ??_C@_08KAEGOLOB@DM_FIRST?$AA@ 10004218     flags.obj
 0001:00003224       ??_C@_08MJMBFJHA@DM_CLOSE?$AA@ 10004224     flags.obj
 0001:00003230       ??_C@_09KLJOCKAA@DM_ENABLE?$AA@ 10004230     flags.obj
 0001:0000323c       ??_C@_0BA@KAMJGFDG@DM_ENABLEREDRAW?$AA@ 1000423c     flags.obj
 0001:0000324c       ??_C@_0O@FKGMMKLP@DM_GETDLGDATA?$AA@ 1000424c     flags.obj
 0001:0000325c       ??_C@_0O@HEGKCPOI@DM_GETDLGITEM?$AA@ 1000425c     flags.obj
 0001:0000326c       ??_C@_0O@BEHCGMCL@DM_GETDLGRECT?$AA@ 1000426c     flags.obj
 0001:0000327c       ??_C@_0L@ELBDNLFO@DM_GETTEXT?$AA@ 1000427c     flags.obj
 0001:00003288       ??_C@_06IKGPEGEJ@DM_KEY?$AA@ 10004288     flags.obj
 0001:00003290       ??_C@_0O@DIPLLJEH@DM_MOVEDIALOG?$AA@ 10004290     flags.obj
 0001:000032a0       ??_C@_0O@EEEDHNPG@DM_SETDLGDATA?$AA@ 100042a0     flags.obj
 0001:000032b0       ??_C@_0O@GKEFJIKB@DM_SETDLGITEM?$AA@ 100042b0     flags.obj
 0001:000032c0       ??_C@_0M@GOFGHDFK@DM_SETFOCUS?$AA@ 100042c0     flags.obj
 0001:000032cc       ??_C@_09ILPFEDOM@DM_REDRAW?$AA@ 100042cc     flags.obj
 0001:000032d8       ??_C@_0L@LDOCOEIP@DM_SETTEXT?$AA@ 100042d8     flags.obj
 0001:000032e4       ??_C@_0BE@LABEAIPD@DM_SETMAXTEXTLENGTH?$AA@ 100042e4     flags.obj
 0001:000032f8       ??_C@_0O@BIFKIPIP@DM_SHOWDIALOG?$AA@ 100042f8     flags.obj
 0001:00003308       ??_C@_0M@JPHKGACH@DM_GETFOCUS?$AA@ 10004308     flags.obj
 0001:00003314       ??_C@_0BA@NLMONBKJ@DM_GETCURSORPOS?$AA@ 10004314     flags.obj
 0001:00003324       ??_C@_0BA@KPHABNOF@DM_SETCURSORPOS?$AA@ 10004324     flags.obj
 0001:00003334       ??_C@_0O@LGEKFPKK@DM_SETTEXTPTR?$AA@ 10004334     flags.obj
 0001:00003344       ??_C@_0M@NCOJHJKI@DM_SHOWITEM?$AA@ 10004344     flags.obj
 0001:00003350       ??_C@_0O@GKKCFHIM@DM_ADDHISTORY?$AA@ 10004350     flags.obj
 0001:00003360       ??_C@_0M@MCEMDFMD@DM_GETCHECK?$AA@ 10004360     flags.obj
 0001:0000336c       ??_C@_0M@DDGACGLO@DM_SETCHECK?$AA@ 1000436c     flags.obj
 0001:00003378       ??_C@_0N@MEGOPFGK@DM_SET3STATE?$AA@ 10004378     flags.obj
 0001:00003388       ??_C@_0M@GEPBDDNC@DM_LISTSORT?$AA@ 10004388     flags.obj
 0001:00003394       ??_C@_0P@NFJNHAKH@DM_LISTGETITEM?$AA@ 10004394     flags.obj
 0001:000033a4       ??_C@_0BB@EEIMACNO@DM_LISTGETCURPOS?$AA@ 100043a4     flags.obj
 0001:000033b8       ??_C@_0BB@GKMJCDEM@DM_LISTSETCURPOS?$AA@ 100043b8     flags.obj
 0001:000033cc       ??_C@_0O@NOPCAHGJ@DM_LISTDELETE?$AA@ 100043cc     flags.obj
 0001:000033dc       ??_C@_0L@BMEAECNG@DM_LISTADD?$AA@ 100043dc     flags.obj
 0001:000033e8       ??_C@_0O@HBHDMHP@DM_LISTADDSTR?$AA@ 100043e8     flags.obj
 0001:000033f8       ??_C@_0O@PDFCNPKN@DM_LISTUPDATE?$AA@ 100043f8     flags.obj
 0001:00003408       ??_C@_0O@GAAGMJJL@DM_LISTINSERT?$AA@ 10004408     flags.obj
 0001:00003418       ??_C@_0BC@MIFCLOBD@DM_LISTFINDSTRING?$AA@ 10004418     flags.obj
 0001:0000342c       ??_C@_0M@EEAEBLKC@DM_LISTINFO?$AA@ 1000442c     flags.obj
 0001:00003438       ??_C@_0P@PLJLJFPA@DM_LISTGETDATA?$AA@ 10004438     flags.obj
 0001:00003448       ??_C@_0P@DGKKKCB@DM_LISTSETDATA?$AA@ 10004448     flags.obj
 0001:00003458       ??_C@_0BB@CELMNLLN@DM_LISTSETTITLES?$AA@ 10004458     flags.obj
 0001:0000346c       ??_C@_0BB@KPJPKCP@DM_LISTGETTITLES?$AA@ 1000446c     flags.obj
 0001:00003480       ??_C@_0BA@ICDJCFLE@DM_RESIZEDIALOG?$AA@ 10004480     flags.obj
 0001:00003490       ??_C@_0BD@CNGGHGJF@DM_SETITEMPOSITION?$AA@ 10004490     flags.obj
 0001:000034a4       ??_C@_0BF@JMINBGBA@DM_GETDROPDOWNOPENED?$AA@ 100044a4     flags.obj
 0001:000034bc       ??_C@_0BF@LJIGJNAO@DM_SETDROPDOWNOPENED?$AA@ 100044bc     flags.obj
 0001:000034d4       ??_C@_0O@NPDKADMJ@DM_SETHISTORY?$AA@ 100044d4     flags.obj
 0001:000034e4       ??_C@_0BD@BPHAAEIM@DM_GETITEMPOSITION?$AA@ 100044e4     flags.obj
 0001:000034f8       ??_C@_0BC@BENFKLNH@DM_SETINPUTNOTIFY?$AA@ 100044f8     flags.obj
 0001:0000350c       ??_C@_0BH@CFMLLNNM@DM_SETMOUSEEVENTNOTIFY?$AA@ 1000450c     flags.obj
 0001:00003524       ??_C@_0BF@IAGIACOD@DM_EDITUNCHANGEDFLAG?$AA@ 10004524     flags.obj
 0001:0000353c       ??_C@_0P@OJKNHIPN@DM_GETITEMDATA?$AA@ 1000453c     flags.obj
 0001:0000354c       ??_C@_0P@OGLDKOHO@DM_SETITEMDATA?$AA@ 1000454c     flags.obj
 0001:0000355c       ??_C@_0L@KNFAKFKE@DM_LISTSET?$AA@ 1000455c     flags.obj
 0001:00003568       ??_C@_0BB@EPMFHAFO@DM_GETCURSORSIZE?$AA@ 10004568     flags.obj
 0001:0000357c       ??_C@_0BB@DANLMDCJ@DM_SETCURSORSIZE?$AA@ 1000457c     flags.obj
 0001:00003590       ??_C@_0BD@LAOOKGHD@DM_LISTGETDATASIZE?$AA@ 10004590     flags.obj
 0001:000035a4       ??_C@_0BA@BHGANJAP@DM_GETSELECTION?$AA@ 100045a4     flags.obj
 0001:000035b4       ??_C@_0BA@GDNOBFED@DM_SETSELECTION?$AA@ 100045b4     flags.obj
 0001:000035c4       ??_C@_0BD@FIHDGIGO@DM_GETEDITPOSITION?$AA@ 100045c4     flags.obj
 0001:000035d8       ??_C@_0BD@GKGFBKHH@DM_SETEDITPOSITION?$AA@ 100045d8     flags.obj
 0001:000035ec       ??_C@_0BE@MCECGHBC@DM_SETCOMBOBOXEVENT?$AA@ 100045ec     flags.obj
 0001:00003600       ??_C@_0BE@KGBLNJKA@DM_GETCOMBOBOXEVENT?$AA@ 10004600     flags.obj
 0001:00003614       ??_C@_0BD@CJEPBACF@DM_GETCONSTTEXTPTR?$AA@ 10004614     flags.obj
 0001:00003628       ??_C@_0BD@HOOHICEG@DM_GETDLGITEMSHORT?$AA@ 10004628     flags.obj
 0001:0000363c       ??_C@_0BD@EMPBPAFP@DM_SETDLGITEMSHORT?$AA@ 1000463c     flags.obj
 0001:00003650       ??_C@_0BB@GAPFMPKE@DM_GETDIALOGINFO?$AA@ 10004650     flags.obj
 0001:00003664       ??_C@_0BC@KJOLMFGG@DM_GETDIALOGTITLE?$AA@ 10004664     flags.obj
 0001:00003678       ??_C@_08COMJOMAC@DN_FIRST?$AA@ 10004678     flags.obj
 0001:00003684       ??_C@_0M@NNNAPNMA@DN_BTNCLICK?$AA@ 10004684     flags.obj
 0001:00003690       ??_C@_0BC@MJFJAANN@DN_CTLCOLORDIALOG?$AA@ 10004690     flags.obj
 0001:000036a4       ??_C@_0BD@HFGBIBBL@DN_CTLCOLORDLGITEM?$AA@ 100046a4     flags.obj
 0001:000036b8       ??_C@_0BD@JMFJPHPD@DN_CTLCOLORDLGLIST?$AA@ 100046b8     flags.obj
 0001:000036cc       ??_C@_0O@NKBDPILK@DN_DRAWDIALOG?$AA@ 100046cc     flags.obj
 0001:000036dc       ??_C@_0P@KGKEDPBI@DN_DRAWDLGITEM?$AA@ 100046dc     flags.obj
 0001:000036ec       ??_C@_0O@JMKNGFLE@DN_EDITCHANGE?$AA@ 100046ec     flags.obj
 0001:000036fc       ??_C@_0N@OCGKCPJF@DN_ENTERIDLE?$AA@ 100046fc     flags.obj
 0001:0000370c       ??_C@_0M@JHFIBKOO@DN_GOTFOCUS?$AA@ 1000470c     flags.obj
 0001:00003718       ??_C@_07NJJEMKPA@DN_HELP?$AA@ 10004718     flags.obj
 0001:00003720       ??_C@_09EDGJFAK@DN_HOTKEY?$AA@ 10004720     flags.obj
 0001:0000372c       ??_C@_0O@BJECHBCA@DN_INITDIALOG?$AA@ 1000472c     flags.obj
 0001:0000373c       ??_C@_0N@CHLLLNBO@DN_KILLFOCUS?$AA@ 1000473c     flags.obj
 0001:0000374c       ??_C@_0O@CLPABIGO@DN_LISTCHANGE?$AA@ 1000474c     flags.obj
 0001:0000375c       ??_C@_0L@MLMFBHN@DN_DRAGGED?$AA@ 1000475c     flags.obj
 0001:00003768       ??_C@_0BB@BOOOCAEG@DN_RESIZECONSOLE?$AA@ 10004768     flags.obj
 0001:0000377c       ??_C@_0BC@FHPPFLKG@DN_DRAWDIALOGDONE?$AA@ 1000477c     flags.obj
 0001:00003790       ??_C@_0O@EONPBNNP@DN_LISTHOTKEY?$AA@ 10004790     flags.obj
 0001:000037a0       ??_C@_08MDDLDGPO@DN_INPUT?$AA@ 100047a0     flags.obj
 0001:000037ac       ??_C@_0BA@FGOGLDBC@DN_CONTROLINPUT?$AA@ 100047ac     flags.obj
 0001:000037bc       ??_C@_08EHEOFOJD@DN_CLOSE?$AA@ 100047bc     flags.obj
 0001:000037c8       ??_C@_0M@POIFBPFN@DN_GETVALUE?$AA@ 100047c8     flags.obj
 0001:000037d4       ??_C@_0BC@MHCBFAAO@DN_DROPDOWNOPENED?$AA@ 100047d4     flags.obj
 0001:000037e8       ??_C@_0BD@NGEKAPIF@DN_DRAWDLGITEMDONE?$AA@ 100047e8     flags.obj
 0001:000037fc       ??_C@_07DIJJNCBA@DM_USER?$AA@ 100047fc     flags.obj
 0001:00003804       ??_C@_0BB@HLBBGMAN@BSTATE_UNCHECKED?$AA@ 10004804     flags.obj
 0001:00003818       ??_C@_0P@FALAMPGP@BSTATE_CHECKED?$AA@ 10004818     flags.obj
 0001:00003828       ??_C@_0O@KBIFGGHO@BSTATE_3STATE?$AA@ 10004828     flags.obj
 0001:00003838       ??_C@_0O@ILJOJGLD@BSTATE_TOGGLE?$AA@ 10004838     flags.obj
 0001:00003848       ??_C@_08PPADCPCM@CBET_KEY?$AA@ 10004848     flags.obj
 0001:00003854       ??_C@_0L@KHCLMGFJ@CBET_MOUSE?$AA@ 10004854     flags.obj
 0001:00003860       ??_C@_0BA@KNHGEBNE@PTYPE_FILEPANEL?$AA@ 10004860     flags.obj
 0001:00003870       ??_C@_0BA@LPPHNHIG@PTYPE_TREEPANEL?$AA@ 10004870     flags.obj
 0001:00003880       ??_C@_0BB@JBINOKAI@PTYPE_QVIEWPANEL?$AA@ 10004880     flags.obj
 0001:00003894       ??_C@_0BA@NKMDEBG@PTYPE_INFOPANEL?$AA@ 10004894     flags.obj
 0001:000038a4       ??_C@_0L@OPHJOKKE@SM_DEFAULT?$AA@ 100048a4     flags.obj
 0001:000038b0       ??_C@_0M@JGBFGGEA@SM_UNSORTED?$AA@ 100048b0     flags.obj
 0001:000038bc       ??_C@_07KIFHAGIL@SM_NAME?$AA@ 100048bc     flags.obj
 0001:000038c4       ??_C@_06GJJJNNFE@SM_EXT?$AA@ 100048c4     flags.obj
 0001:000038cc       ??_C@_08FICJBKFN@SM_MTIME?$AA@ 100048cc     flags.obj
 0001:000038d8       ??_C@_08GCCDHLCN@SM_CTIME?$AA@ 100048d8     flags.obj
 0001:000038e4       ??_C@_08CPOLNKCG@SM_ATIME?$AA@ 100048e4     flags.obj
 0001:000038f0       ??_C@_07OMPKMIKC@SM_SIZE?$AA@ 100048f0     flags.obj
 0001:000038f8       ??_C@_08BCBPOLMA@SM_DESCR?$AA@ 100048f8     flags.obj
 0001:00003904       ??_C@_08MEAGCMBB@SM_OWNER?$AA@ 10004904     flags.obj
 0001:00003910       ??_C@_0BC@NKDBNAHD@SM_COMPRESSEDSIZE?$AA@ 10004910     flags.obj
 0001:00003924       ??_C@_0M@PKNLKFI@SM_NUMLINKS?$AA@ 10004924     flags.obj
 0001:00003930       ??_C@_0O@CCKEKPHL@SM_NUMSTREAMS?$AA@ 10004930     flags.obj
 0001:00003940       ??_C@_0P@PKGMDPMD@SM_STREAMSSIZE?$AA@ 10004940     flags.obj
 0001:00003950       ??_C@_0M@OAFEBGNH@SM_FULLNAME?$AA@ 10004950     flags.obj
 0001:0000395c       ??_C@_09KFKGJDHC@SM_CHTIME?$AA@ 1000495c     flags.obj
 0001:00003968       ??_C@_08DOEDKINA@SM_COUNT?$AA@ 10004968     flags.obj
 0001:00003974       ??_C@_0P@FEMAMJLE@EEC_OPEN_ERROR?$AA@ 10004974     flags.obj
 0001:00003984       ??_C@_0N@GLMELIKF@EEC_MODIFIED?$AA@ 10004984     flags.obj
 0001:00003994       ??_C@_0BB@HALKEFOL@EEC_NOT_MODIFIED?$AA@ 10004994     flags.obj
 0001:000039a8       ??_C@_0BI@CNPFKHKO@EEC_LOADING_INTERRUPTED?$AA@ 100049a8     flags.obj
 0001:000039c0       ??_C@_0BK@PHBCABMB@ACTL_GETFARMANAGERVERSION?$AA@ 100049c0     flags.obj
 0001:000039dc       ??_C@_0N@DPABJDML@ACTL_WAITKEY?$AA@ 100049dc     flags.obj
 0001:000039ec       ??_C@_0O@CEHHJAFD@ACTL_GETCOLOR?$AA@ 100049ec     flags.obj
 0001:000039fc       ??_C@_0BD@OKPAACIK@ACTL_GETARRAYCOLOR?$AA@ 100049fc     flags.obj
 0001:00003a10       ??_C@_0BD@DIFEEKNN@ACTL_GETWINDOWINFO?$AA@ 10004a10     flags.obj
 0001:00003a24       ??_C@_0BE@PJBIPKOD@ACTL_GETWINDOWCOUNT?$AA@ 10004a24     flags.obj
 0001:00003a38       ??_C@_0BG@MNKPOEEN@ACTL_SETCURRENTWINDOW?$AA@ 10004a38     flags.obj
 0001:00003a50       ??_C@_0M@IHHFGPPA@ACTL_COMMIT?$AA@ 10004a50     flags.obj
 0001:00003a5c       ??_C@_0BA@CLHFKJJP@ACTL_GETFARHWND?$AA@ 10004a5c     flags.obj
 0001:00003a6c       ??_C@_0BD@JFOOLBPN@ACTL_SETARRAYCOLOR?$AA@ 10004a6c     flags.obj
 0001:00003a80       ??_C@_0P@JECKFIA@ACTL_REDRAWALL?$AA@ 10004a80     flags.obj
 0001:00003a90       ??_C@_0N@DHPLJLHO@ACTL_SYNCHRO?$AA@ 10004a90     flags.obj
 0001:00003aa0       ??_C@_0BG@IJPADENB@ACTL_SETPROGRESSSTATE?$AA@ 10004aa0     flags.obj
 0001:00003ab8       ??_C@_0BG@ICJFAPHK@ACTL_SETPROGRESSVALUE?$AA@ 10004ab8     flags.obj
 0001:00003ad0       ??_C@_09HNDBKLDC@ACTL_QUIT?$AA@ 10004ad0     flags.obj
 0001:00003adc       ??_C@_0BA@LJCPDIKK@ACTL_GETFARRECT?$AA@ 10004adc     flags.obj
 0001:00003aec       ??_C@_0BC@FELBEIDG@ACTL_GETCURSORPOS?$AA@ 10004aec     flags.obj
 0001:00003b00       ??_C@_0BC@CAAPIEHK@ACTL_SETCURSORPOS?$AA@ 10004b00     flags.obj
 0001:00003b14       ??_C@_0BE@NPJGMDBM@ACTL_PROGRESSNOTIFY?$AA@ 10004b14     flags.obj
 0001:00003b28       ??_C@_0BD@IPKOEBIA@ACTL_GETWINDOWTYPE?$AA@ 10004b28     flags.obj
 0001:00003b3c       ??_C@_09CEDFMINA@MSSC_POST?$AA@ 10004b3c     flags.obj
 0001:00003b48       ??_C@_0L@MOADGAEB@MSSC_CHECK?$AA@ 10004b48     flags.obj
 0001:00003b54       ??_C@_0BA@MMOAIEKP@MACROAREA_OTHER?$AA@ 10004b54     flags.obj
 0001:00003b64       ??_C@_0BA@DEBOOAEB@MACROAREA_SHELL?$AA@ 10004b64     flags.obj
 0001:00003b74       ??_C@_0BB@JIMPEHCD@MACROAREA_VIEWER?$AA@ 10004b74     flags.obj
 0001:00003b88       ??_C@_0BB@KILFBFJH@MACROAREA_EDITOR?$AA@ 10004b88     flags.obj
 0001:00003b9c       ??_C@_0BB@CADENPFI@MACROAREA_DIALOG?$AA@ 10004b9c     flags.obj
 0001:00003bb0       ??_C@_0BB@MLMLHIGE@MACROAREA_SEARCH?$AA@ 10004bb0     flags.obj
 0001:00003bc4       ??_C@_0BA@KKMKOLIK@MACROAREA_DISKS?$AA@ 10004bc4     flags.obj
 0001:00003bd4       ??_C@_0BD@IGOOIJP@MACROAREA_MAINMENU?$AA@ 10004bd4     flags.obj
 0001:00003be8       ??_C@_0P@LFLMAHBF@MACROAREA_MENU?$AA@ 10004be8     flags.obj
 0001:00003bf8       ??_C@_0P@DKPKIEO@MACROAREA_HELP?$AA@ 10004bf8     flags.obj
 0001:00003c08       ??_C@_0BE@MDJPICHC@MACROAREA_INFOPANEL?$AA@ 10004c08     flags.obj
 0001:00003c1c       ??_C@_0BF@NLJMHMPP@MACROAREA_QVIEWPANEL?$AA@ 10004c1c     flags.obj
 0001:00003c34       ??_C@_0BE@HBMEGBOC@MACROAREA_TREEPANEL?$AA@ 10004c34     flags.obj
 0001:00003c48       ??_C@_0BF@FCHKCGLL@MACROAREA_FINDFOLDER?$AA@ 10004c48     flags.obj
 0001:00003c60       ??_C@_0BD@JCFMJGDE@MACROAREA_USERMENU?$AA@ 10004c60     flags.obj
 0001:00003c74       ??_C@_0BO@OMLEPJPM@MACROAREA_SHELLAUTOCOMPLETION?$AA@ 10004c74     flags.obj
 0001:00003c94       ??_C@_0BP@OIHAIGBK@MACROAREA_DIALOGAUTOCOMPLETION?$AA@ 10004c94     flags.obj
 0001:00003cb4       ??_C@_0BB@JPEEDDOG@MACROAREA_COMMON?$AA@ 10004cb4     flags.obj
 0001:00003cc8       ??_C@_0BD@DIKEKAIJ@MACROSTATE_NOMACRO?$AA@ 10004cc8     flags.obj
 0001:00003cdc       ??_C@_0BF@PCDEFEGP@MACROSTATE_EXECUTING?$AA@ 10004cdc     flags.obj
 0001:00003cf4       ??_C@_0BM@EJOFDENO@MACROSTATE_EXECUTING_COMMON?$AA@ 10004cf4     flags.obj
 0001:00003d10       ??_C@_0BF@BGODKPBB@MACROSTATE_RECORDING?$AA@ 10004d10     flags.obj
 0001:00003d28       ??_C@_0BM@OICPADFE@MACROSTATE_RECORDING_COMMON?$AA@ 10004d28     flags.obj
 0001:00003d44       ??_C@_0N@CGFFMLBC@MPEC_SUCCESS?$AA@ 10004d44     flags.obj
 0001:00003d54       ??_C@_0L@FJDDLDNN@MPEC_ERROR?$AA@ 10004d54     flags.obj
 0001:00003d60       ??_C@_0N@IBOAADDD@FMVT_UNKNOWN?$AA@ 10004d60     flags.obj
 0001:00003d70       ??_C@_0N@BDMFKEKE@FMVT_INTEGER?$AA@ 10004d70     flags.obj
 0001:00003d80       ??_C@_0M@LFMLDDKI@FMVT_STRING?$AA@ 10004d80     flags.obj
 0001:00003d8c       ??_C@_0M@CKDAIOEN@FMVT_DOUBLE?$AA@ 10004d8c     flags.obj
 0001:00003d98       ??_C@_0N@MHKOBOGF@FMVT_BOOLEAN?$AA@ 10004d98     flags.obj
 0001:00003da8       ??_C@_0M@GKPDICDA@FMVT_BINARY?$AA@ 10004da8     flags.obj
 0001:00003db4       ??_C@_0N@FMHCFNDF@FMVT_POINTER?$AA@ 10004db4     flags.obj
 0001:00003dc4       ??_C@_08DDPDBBNO@FMVT_NIL?$AA@ 10004dc4     flags.obj
 0001:00003dd0       ??_C@_0L@DJIKMOJA@FMVT_ARRAY?$AA@ 10004dd0     flags.obj
 0001:00003ddc       ??_C@_0L@PMDDFEBD@FMVT_PANEL?$AA@ 10004ddc     flags.obj
 0001:00003de8       ??_C@_0O@DCGKMPOM@WTYPE_DESKTOP?$AA@ 10004de8     flags.obj
 0001:00003df8       ??_C@_0N@FNCFCPIG@WTYPE_PANELS?$AA@ 10004df8     flags.obj
 0001:00003e08       ??_C@_0N@EJKMDMBK@WTYPE_VIEWER?$AA@ 10004e08     flags.obj
 0001:00003e18       ??_C@_0N@HJNGGOKO@WTYPE_EDITOR?$AA@ 10004e18     flags.obj
 0001:00003e28       ??_C@_0N@PBFHKEGB@WTYPE_DIALOG?$AA@ 10004e28     flags.obj
 0001:00003e38       ??_C@_0M@OMKLELFA@WTYPE_VMENU?$AA@ 10004e38     flags.obj
 0001:00003e44       ??_C@_0L@BCEMNGOG@WTYPE_HELP?$AA@ 10004e44     flags.obj
 0001:00003e50       ??_C@_0P@MMIDEOJJ@WTYPE_COMBOBOX?$AA@ 10004e50     flags.obj
 0001:00003e60       ??_C@_0BA@IPEAOBGN@TBPS_NOPROGRESS?$AA@ 10004e60     flags.obj
 0001:00003e70       ??_C@_0BD@HMEHMDAL@TBPS_INDETERMINATE?$AA@ 10004e70     flags.obj
 0001:00003e84       ??_C@_0M@KHLNKPHE@TBPS_NORMAL?$AA@ 10004e84     flags.obj
 0001:00003e90       ??_C@_0L@DFDPCOFD@TBPS_ERROR?$AA@ 10004e90     flags.obj
 0001:00003e9c       ??_C@_0M@GHGAPHPP@TBPS_PAUSED?$AA@ 10004e9c     flags.obj
 0001:00003ea8       ??_C@_0O@MCNCFBLF@VSMT_VIEWMODE?$AA@ 10004ea8     flags.obj
 0001:00003eb8       ??_C@_09FLKONCNO@VSMT_WRAP?$AA@ 10004eb8     flags.obj
 0001:00003ec4       ??_C@_0O@INKALKJK@VSMT_WORDWRAP?$AA@ 10004ec4     flags.obj
 0001:00003ed4       ??_C@_08FNEFFFEL@VMT_TEXT?$AA@ 10004ed4     flags.obj
 0001:00003ee0       ??_C@_07FLIHDEDA@VMT_HEX?$AA@ 10004ee0     flags.obj
 0001:00003ee8       ??_C@_08BDDNDBMJ@VMT_DUMP?$AA@ 10004ee8     flags.obj
 0001:00003ef4       ??_C@_07OJCLGDHJ@VE_READ?$AA@ 10004ef4     flags.obj
 0001:00003efc       ??_C@_08JIBCCIDC@VE_CLOSE?$AA@ 10004efc     flags.obj
 0001:00003f08       ??_C@_0M@FEFKOOMJ@VE_GOTFOCUS?$AA@ 10004f08     flags.obj
 0001:00003f14       ??_C@_0N@ICHCAKIB@VE_KILLFOCUS?$AA@ 10004f14     flags.obj
 0001:00003f24       ??_C@_07BLBPFFLB@EE_READ?$AA@ 10004f24     flags.obj
 0001:00003f2c       ??_C@_07KJGPGPOC@EE_SAVE?$AA@ 10004f2c     flags.obj
 0001:00003f34       ??_C@_09NPOPIKMK@EE_REDRAW?$AA@ 10004f34     flags.obj
 0001:00003f40       ??_C@_08NFPFGIG@EE_CLOSE?$AA@ 10004f40     flags.obj
 0001:00003f4c       ??_C@_0M@CPNMNBMF@EE_GOTFOCUS?$AA@ 10004f4c     flags.obj
 0001:00003f58       ??_C@_0N@ILLPMAJF@EE_KILLFOCUS?$AA@ 10004f58     flags.obj
 0001:00003f68       ??_C@_09MIOGFFI@EE_CHANGE?$AA@ 10004f68     flags.obj
 0001:00003f74       ??_C@_0P@MBHAHBBG@DE_DLGPROCINIT?$AA@ 10004f74     flags.obj
 0001:00003f84       ??_C@_0BC@BMFEJAMO@DE_DEFDLGPROCINIT?$AA@ 10004f84     flags.obj
 0001:00003f98       ??_C@_0O@ICBCOJCG@DE_DLGPROCEND?$AA@ 10004f98     flags.obj
 0001:00003fa8       ??_C@_0BB@MNODJNPE@SE_COMMONSYNCHRO?$AA@ 10004fa8     flags.obj
 0001:00003fbc       ??_C@_0N@HKGMPMJE@ESPT_TABSIZE?$AA@ 10004fbc     flags.obj
 0001:00003fcc       ??_C@_0BA@GOKHPFCK@ESPT_EXPANDTABS?$AA@ 10004fcc     flags.obj
 0001:00003fdc       ??_C@_0BA@KOADDMLI@ESPT_AUTOINDENT?$AA@ 10004fdc     flags.obj
 0001:00003fec       ??_C@_0BF@LPNONOMF@ESPT_CURSORBEYONDEOL?$AA@ 10004fec     flags.obj
 0001:00004004       ??_C@_0BC@OECOCGLJ@ESPT_CHARCODEBASE?$AA@ 10005004     flags.obj
 0001:00004018       ??_C@_0O@PIAOJINE@ESPT_CODEPAGE?$AA@ 10005018     flags.obj
 0001:00004028       ??_C@_0BG@HAPABMJH@ESPT_SAVEFILEPOSITION?$AA@ 10005028     flags.obj
 0001:00004040       ??_C@_0O@KCPDJCKC@ESPT_LOCKMODE?$AA@ 10005040     flags.obj
 0001:00004050       ??_C@_0BA@EIGIAOHM@ESPT_SETWORDDIV?$AA@ 10005050     flags.obj
 0001:00004060       ??_C@_0BA@FGEHLJDF@ESPT_GETWORDDIV?$AA@ 10005060     flags.obj
 0001:00004070       ??_C@_0BE@MACJBCFP@ESPT_SHOWWHITESPACE?$AA@ 10005070     flags.obj
 0001:00004084       ??_C@_0M@FICNFPPA@ESPT_SETBOM?$AA@ 10005084     flags.obj
 0001:00004090       ??_C@_09FLEMPKKP@EUR_BEGIN?$AA@ 10005090     flags.obj
 0001:0000409c       ??_C@_07DDJDFJCN@EUR_END?$AA@ 1000509c     flags.obj
 0001:000040a4       ??_C@_08FCONALGE@EUR_UNDO?$AA@ 100050a4     flags.obj
 0001:000040b0       ??_C@_08DHMMFAHF@EUR_REDO?$AA@ 100050b0     flags.obj
 0001:000040bc       ??_C@_0O@PKOIFEBO@EXPAND_NOTABS?$AA@ 100050bc     flags.obj
 0001:000040cc       ??_C@_0P@MLHPCNDM@EXPAND_ALLTABS?$AA@ 100050cc     flags.obj
 0001:000040dc       ??_C@_0P@OONGIIBL@EXPAND_NEWTABS?$AA@ 100050dc     flags.obj
 0001:000040ec       ??_C@_0BD@DKHPEOHH@EOPT_EXPANDALLTABS?$AA@ 100050ec     flags.obj
 0001:00004100       ??_C@_0BG@BOINMDEK@EOPT_PERSISTENTBLOCKS?$AA@ 10005100     flags.obj
 0001:00004118       ??_C@_0BG@PIIHHCAN@EOPT_DELREMOVESBLOCKS?$AA@ 10005118     flags.obj
 0001:00004130       ??_C@_0BA@KPJEAKBD@EOPT_AUTOINDENT?$AA@ 10005130     flags.obj
 0001:00004140       ??_C@_0BG@MBPADLG@EOPT_SAVEFILEPOSITION?$AA@ 10005140     flags.obj
 0001:00004158       ??_C@_0BI@PFHCGCAI@EOPT_AUTODETECTCODEPAGE?$AA@ 10005158     flags.obj
 0001:00004170       ??_C@_0BF@IMCOEIAL@EOPT_CURSORBEYONDEOL?$AA@ 10005170     flags.obj
 0001:00004188       ??_C@_0BH@CJPAGGLC@EOPT_EXPANDONLYNEWTABS?$AA@ 10005188     flags.obj
 0001:000041a0       ??_C@_0BE@DDKCDJDC@EOPT_SHOWWHITESPACE?$AA@ 100051a0     flags.obj
 0001:000041b4       ??_C@_08HMMLONBH@EOPT_BOM?$AA@ 100051b4     flags.obj
 0001:000041c0       ??_C@_0BD@CLLAKGOA@EOPT_SHOWLINEBREAK?$AA@ 100051c0     flags.obj
 0001:000041d4       ??_C@_0BC@JCJEPKEC@EOPT_SHOWTITLEBAR?$AA@ 100051d4     flags.obj
 0001:000041e8       ??_C@_0BA@KPGMOBKI@EOPT_SHOWKEYBAR?$AA@ 100051e8     flags.obj
 0001:000041f8       ??_C@_0BD@EFCFEAD@EOPT_SHOWSCROLLBAR?$AA@ 100051f8     flags.obj
 0001:0000420c       ??_C@_0L@BJCBJJNB@BTYPE_NONE?$AA@ 1000520c     flags.obj
 0001:00004218       ??_C@_0N@OPHHGFPF@BTYPE_STREAM?$AA@ 10005218     flags.obj
 0001:00004228       ??_C@_0N@EMEGNPLI@BTYPE_COLUMN?$AA@ 10005228     flags.obj
 0001:00004238       ??_C@_0BB@BNPDAPGB@ECSTATE_MODIFIED?$AA@ 10005238     flags.obj
 0001:0000424c       ??_C@_0O@GBBGHDFM@ECSTATE_SAVED?$AA@ 1000524c     flags.obj
 0001:0000425c       ??_C@_0P@BECIAJAM@ECSTATE_LOCKED?$AA@ 1000525c     flags.obj
 0001:0000426c       ??_C@_0P@DOBJCNIG@ECTYPE_CHANGED?$AA@ 1000526c     flags.obj
 0001:0000427c       ??_C@_0N@MDEFMEEA@ECTYPE_ADDED?$AA@ 1000527c     flags.obj
 0001:0000428c       ??_C@_0P@NMOJJPOB@ECTYPE_DELETED?$AA@ 1000528c     flags.obj
 0001:0000429c       ??_C@_08HHHKLJPB@PLT_PATH?$AA@ 1000529c     flags.obj
 0001:000042a8       ??_C@_08KBAMIIFB@PFM_GUID?$AA@ 100052a8     flags.obj
 0001:000042b4       ??_C@_0P@KKEMMPNI@PFM_MODULENAME?$AA@ 100052b4     flags.obj
 0001:000042c4       ??_C@_09BOODOHKD@FFT_PANEL?$AA@ 100052c4     flags.obj
 0001:000042d0       ??_C@_0N@GMEDAGNH@FFT_FINDFILE?$AA@ 100052d0     flags.obj
 0001:000042e0       ??_C@_08KKCPIPGP@FFT_COPY?$AA@ 100052e0     flags.obj
 0001:000042ec       ??_C@_0L@EKPDMFDD@FFT_SELECT?$AA@ 100052ec     flags.obj
 0001:000042f8       ??_C@_0L@LGPEDLLD@FFT_CUSTOM?$AA@ 100052f8     flags.obj
 0001:00004304       ??_C@_0M@OIOMMFOE@FST_UNKNOWN?$AA@ 10005304     flags.obj
 0001:00004310       ??_C@_0L@GGGOEGKJ@FST_SUBKEY?$AA@ 10005310     flags.obj
 0001:0000431c       ??_C@_09LFEEAJIC@FST_QWORD?$AA@ 1000531c     flags.obj
 0001:00004328       ??_C@_0L@LPMPBKDL@FST_STRING?$AA@ 10005328     flags.obj
 0001:00004334       ??_C@_08EJJJCLIG@FST_DATA?$AA@ 10005334     flags.obj
 0001:00004340       ??_C@_09OBBBBFPE@FSSF_ROOT?$AA@ 10005340     flags.obj
 0001:0000434c       ??_C@_0BB@HDKCPBIO@FSSF_HISTORY_CMD?$AA@ 1000534c     flags.obj
 0001:00004360       ??_C@_0BE@BLPOFODL@FSSF_HISTORY_FOLDER?$AA@ 10005360     flags.obj
 0001:00004374       ??_C@_0BC@NJCJCCNH@FSSF_HISTORY_VIEW?$AA@ 10005374     flags.obj
 0001:00004388       ??_C@_0BC@CODELNPP@FSSF_HISTORY_EDIT?$AA@ 10005388     flags.obj
 0001:0000439c       ??_C@_0BG@IFGEMJIF@FSSF_HISTORY_EXTERNAL?$AA@ 1000539c     flags.obj
 0001:000043b4       ??_C@_0BG@DGAKDKFK@FSSF_FOLDERSHORTCUT_0?$AA@ 100053b4     flags.obj
 0001:000043cc       ??_C@_0BG@CPBBALBL@FSSF_FOLDERSHORTCUT_1?$AA@ 100053cc     flags.obj
 0001:000043e4       ??_C@_0BG@EDMFINI@FSSF_FOLDERSHORTCUT_2?$AA@ 100053e4     flags.obj
 0001:000043fc       ??_C@_0BG@BNCHGJJJ@FSSF_FOLDERSHORTCUT_3?$AA@ 100053fc     flags.obj
 0001:00004414       ??_C@_0BG@FCGGPPFO@FSSF_FOLDERSHORTCUT_4?$AA@ 10005414     flags.obj
 0001:0000442c       ??_C@_0BG@ELHNMOBP@FSSF_FOLDERSHORTCUT_5?$AA@ 1000542c     flags.obj
 0001:00004444       ??_C@_0BG@GAFAJNNM@FSSF_FOLDERSHORTCUT_6?$AA@ 10005444     flags.obj
 0001:0000445c       ??_C@_0BG@HJELKMJN@FSSF_FOLDERSHORTCUT_7?$AA@ 1000545c     flags.obj
 0001:00004474       ??_C@_0BG@PONDLAFC@FSSF_FOLDERSHORTCUT_8?$AA@ 10005474     flags.obj
 0001:0000448c       ??_C@_0BG@OHMIIBBD@FSSF_FOLDERSHORTCUT_9?$AA@ 1000548c     flags.obj
 0001:000044a4       ??_C@_0BD@PBIEGEHP@FSSF_CONFIRMATIONS?$AA@ 100054a4     flags.obj
 0001:000044b8       ??_C@_0M@PIGDMPJB@FSSF_SYSTEM?$AA@ 100054b8     flags.obj
 0001:000044c4       ??_C@_0L@LBFNJGFB@FSSF_PANEL?$AA@ 100054c4     flags.obj
 0001:000044d0       ??_C@_0M@KJLIHDEL@FSSF_EDITOR?$AA@ 100054d0     flags.obj
 0001:000044dc       ??_C@_0M@KEMGKEOF@FSSF_SCREEN?$AA@ 100054dc     flags.obj
 0001:000044e8       ??_C@_0M@CBDJLJIE@FSSF_DIALOG?$AA@ 100054e8     flags.obj
 0001:000044f4       ??_C@_0P@OCDADNBF@FSSF_INTERFACE?$AA@ 100054f4     flags.obj
 0001:00004504       ??_C@_0BB@GBBEBNKE@FSSF_PANELLAYOUT?$AA@ 10005504     flags.obj
 0001:00004518       ??_C@_0M@JCGHGLJF@PSL_ROAMING?$AA@ 10005518     flags.obj
 0001:00004524       ??_C@_09EDBNDHCM@PSL_LOCAL?$AA@ 10005524     flags.obj
 0001:00004530       ??_C@_07BPEFOPGM@FCT_ANY?$AA@ 10005530     flags.obj
 0001:00004538       ??_C@_0L@CDAEILNM@FCT_STREAM?$AA@ 10005538     flags.obj
 0001:00004544       ??_C@_0L@IADFDBJB@FCT_COLUMN?$AA@ 10005544     flags.obj
 0001:00004550       ??_C@_0O@KJFMBLFE@LINK_HARDLINK?$AA@ 10005550     flags.obj
 0001:00004560       ??_C@_0O@OOAFIIDA@LINK_JUNCTION?$AA@ 10005560     flags.obj
 0001:00004570       ??_C@_0O@FIAPLKLH@LINK_VOLMOUNT?$AA@ 10005570     flags.obj
 0001:00004580       ??_C@_0BB@JDBEPJDK@LINK_SYMLINKFILE?$AA@ 10005580     flags.obj
 0001:00004594       ??_C@_0BA@GFPIOFMG@LINK_SYMLINKDIR?$AA@ 10005594     flags.obj
 0001:000045a4       ??_C@_0N@PJENIJFN@LINK_SYMLINK?$AA@ 100055a4     flags.obj
 0001:000045b4       ??_C@_08HNOHKPBK@CPM_FULL?$AA@ 100055b4     flags.obj
 0001:000045c0       ??_C@_08LAEGFKJE@CPM_REAL?$AA@ 100055c0     flags.obj
 0001:000045cc       ??_C@_0L@NPJNPCJM@CPM_NATIVE?$AA@ 100055cc     flags.obj
 0001:000045d8       ??_C@_0L@NCFOENCC@VS_RELEASE?$AA@ 100055d8     flags.obj
 0001:000045e4       ??_C@_08BDGLHPMJ@VS_ALPHA?$AA@ 100055e4     flags.obj
 0001:000045f0       ??_C@_07OKFPMINB@VS_BETA?$AA@ 100055f0     flags.obj
 0001:000045f8       ??_C@_05MMFLPJEB@VS_RC?$AA@ 100055f8     flags.obj
 0001:00004600       ??_C@_0BC@OOKLINPG@OPEN_LEFTDISKMENU?$AA@ 10005600     flags.obj
 0001:00004614       ??_C@_0BB@CEFDHHLF@OPEN_PLUGINSMENU?$AA@ 10005614     flags.obj
 0001:00004628       ??_C@_0O@IEJHJCNB@OPEN_FINDLIST?$AA@ 10005628     flags.obj
 0001:00004638       ??_C@_0O@OGDCDPNG@OPEN_SHORTCUT?$AA@ 10005638     flags.obj
 0001:00004648       ??_C@_0BB@JHCCMIPF@OPEN_COMMANDLINE?$AA@ 10005648     flags.obj
 0001:0000465c       ??_C@_0M@DMJLHMGM@OPEN_EDITOR?$AA@ 1000565c     flags.obj
 0001:00004668       ??_C@_0M@MOBCONI@OPEN_VIEWER?$AA@ 10005668     flags.obj
 0001:00004674       ??_C@_0P@LCDNLGDE@OPEN_FILEPANEL?$AA@ 10005674     flags.obj
 0001:00004684       ??_C@_0M@LEBKLGKD@OPEN_DIALOG?$AA@ 10005684     flags.obj
 0001:00004690       ??_C@_0N@CBHPGAKB@OPEN_ANALYSE?$AA@ 10005690     flags.obj
 0001:000046a0       ??_C@_0BD@NFNGGFHI@OPEN_RIGHTDISKMENU?$AA@ 100056a0     flags.obj
 0001:000046b4       ??_C@_0P@FOKOAMLC@OPEN_FROMMACRO?$AA@ 100056b4     flags.obj
 0001:000046c4       ??_C@_0O@NEDDJIHC@OPEN_LUAMACRO?$AA@ 100056c4     flags.obj
 0001:000046d4       ??_C@_0P@GBMLNMMI@MCT_MACROPARSE?$AA@ 100056d4     flags.obj
 0001:000046e4       ??_C@_0P@GNPFPCF@MCT_LOADMACROS?$AA@ 100056e4     flags.obj
 0001:000046f4       ??_C@_0P@HMDDACMI@MCT_ENUMMACROS?$AA@ 100056f4     flags.obj
 0001:00004704       ??_C@_0BA@MOCJHMJK@MCT_WRITEMACROS?$AA@ 10005704     flags.obj
 0001:00004714       ??_C@_0N@IGJGAHKE@MCT_GETMACRO?$AA@ 10005714     flags.obj
 0001:00004724       ??_C@_0BC@NFGGBILF@MCT_RECORDEDMACRO?$AA@ 10005724     flags.obj
 0001:00004738       ??_C@_0N@OLCKOJMI@MCT_DELMACRO?$AA@ 10005738     flags.obj
 0001:00004748       ??_C@_0BC@NALHIHJ@MCT_RUNSTARTMACRO?$AA@ 10005748     flags.obj
 0001:0000475c       ??_C@_0P@HOMHAEFB@MCT_EXECSTRING?$AA@ 1000575c     flags.obj
 0001:0000476c       ??_C@_0O@CDBDPKIC@MCT_PANELSORT?$AA@ 1000576c     flags.obj
 0001:0000477c       ??_C@_0BH@PKKJIOHM@MCT_GETCUSTOMSORTMODES?$AA@ 1000577c     flags.obj
 0001:00004794       ??_C@_0N@FOPIOCHO@MCT_ADDMACRO?$AA@ 10005794     flags.obj
 0001:000047a4       ??_C@_0N@BHFJFHA@MCT_KEYMACRO?$AA@ 100057a4     flags.obj
 0001:000047b4       ??_C@_0BB@LPDAOGB@MCT_CANPANELSORT?$AA@ 100057b4     flags.obj
 0001:000047c8       ??_C@_0BC@IOECJI@MPRT_NORMALFINISH?$AA@ 100057c8     flags.obj
 0001:000047dc       ??_C@_0BB@PMCBIGCA@MPRT_ERRORFINISH?$AA@ 100057dc     flags.obj
 0001:000047f0       ??_C@_0BA@BCBAEEOI@MPRT_ERRORPARSE?$AA@ 100057f0     flags.obj
 0001:00004800       ??_C@_09EJDAADCN@MPRT_KEYS?$AA@ 10005800     flags.obj
 0001:0000480c       ??_C@_0L@GEHHCKFA@MPRT_PRINT?$AA@ 1000580c     flags.obj
 0001:00004818       ??_C@_0BA@OBIDLEIM@MPRT_PLUGINCALL?$AA@ 10005818     flags.obj
 0001:00004828       ??_C@_0BA@EJFFOAMM@MPRT_PLUGINMENU?$AA@ 10005828     flags.obj
 0001:00004838       ??_C@_0BC@LEDOPMKI@MPRT_PLUGINCONFIG?$AA@ 10005838     flags.obj
 0001:0000484c       ??_C@_0BD@HHINMPPI@MPRT_PLUGINCOMMAND?$AA@ 1000584c     flags.obj
 0001:00004860       ??_C@_0O@IEMNLPAB@MPRT_USERMENU?$AA@ 10005860     flags.obj
 0001:00004870       ??_C@_0BA@GEAFHJNF@MPRT_HASNOMACRO?$AA@ 10005870     flags.obj
 0001:00004880       ??_C@_0BC@PNCKAHJO@FE_CHANGEVIEWMODE?$AA@ 10005880     flags.obj
 0001:00004894       ??_C@_09DENIDBMJ@FE_REDRAW?$AA@ 10005894     flags.obj
 0001:000048a0       ??_C@_07CLNPDBLG@FE_IDLE?$AA@ 100058a0     flags.obj
 0001:000048a8       ??_C@_08DENCGKED@FE_CLOSE?$AA@ 100058a8     flags.obj
 0001:000048b4       ??_C@_08MOMCCKPB@FE_BREAK?$AA@ 100058b4     flags.obj
 0001:000048c0       ??_C@_0L@LELAIPLL@FE_COMMAND?$AA@ 100058c0     flags.obj
 0001:000048cc       ??_C@_0M@FIECADDF@FE_GOTFOCUS?$AA@ 100058cc     flags.obj
 0001:000048d8       ??_C@_0N@DGHFKMFL@FE_KILLFOCUS?$AA@ 100058d8     flags.obj
 0001:000048e8       ??_C@_0BE@PONEECEM@FE_CHANGESORTPARAMS?$AA@ 100058e8     flags.obj
 0001:000048fc       ??_C@_0M@HNDHDHHO@FCF_FG_4BIT?$AA@ 100058fc     flags.obj
 0001:00004908       ??_C@_0M@PJHNDJIE@FCF_BG_4BIT?$AA@ 10005908     flags.obj
 0001:00004914       ??_C@_0N@HMKJBHOA@FCF_4BITMASK?$AA@ 10005914     flags.obj
 0001:00004924       ??_C@_0BB@PJFLJJLD@FCF_RAWATTR_MASK?$AA@ 10005924     flags.obj
 0001:00004938       ??_C@_0BC@NKBLNNIA@FCF_EXTENDEDFLAGS?$AA@ 10005938     flags.obj
 0001:0000494c       ??_C@_0M@LFMGCKHG@FCF_FG_BOLD?$AA@ 1000594c     flags.obj
 0001:00004958       ??_C@_0O@FAPDECBF@FCF_FG_ITALIC?$AA@ 10005958     flags.obj
 0001:00004968       ??_C@_0BB@NPEFGEGA@FCF_FG_UNDERLINE?$AA@ 10005968     flags.obj
 0001:0000497c       ??_C@_0O@LGBGBIGB@FCF_STYLEMASK?$AA@ 1000597c     flags.obj
 0001:0000498c       ??_C@_08BKNBBLHK@FCF_NONE?$AA@ 1000598c     flags.obj
 0001:00004998       ??_C@_08FKIDFHCM@CDF_NONE?$AA@ 10005998     flags.obj
 0001:000049a4       ??_C@_0N@ELMEMNDH@FMSG_WARNING?$AA@ 100059a4     flags.obj
 0001:000049b4       ??_C@_0P@HHIGLJAP@FMSG_ERRORTYPE?$AA@ 100059b4     flags.obj
 0001:000049c4       ??_C@_0BE@FHOOILPH@FMSG_KEEPBACKGROUND?$AA@ 100059c4     flags.obj
 0001:000049d8       ??_C@_0P@KBEMNNEP@FMSG_LEFTALIGN?$AA@ 100059d8     flags.obj
 0001:000049e8       ??_C@_0O@FOIOKDHJ@FMSG_ALLINONE?$AA@ 100059e8     flags.obj
 0001:000049f8       ??_C@_0L@BGALGPOK@FMSG_MB_OK?$AA@ 100059f8     flags.obj
 0001:00004a04       ??_C@_0BB@JGAPGIEP@FMSG_MB_OKCANCEL?$AA@ 10005a04     flags.obj
 0001:00004a18       ??_C@_0BJ@BKJADAHA@FMSG_MB_ABORTRETRYIGNORE?$AA@ 10005a18     flags.obj
 0001:00004a34       ??_C@_0O@GPCAPHCL@FMSG_MB_YESNO?$AA@ 10005a34     flags.obj
 0001:00004a44       ??_C@_0BE@IBNOLCGP@FMSG_MB_YESNOCANCEL?$AA@ 10005a44     flags.obj
 0001:00004a58       ??_C@_0BE@OCLAIENB@FMSG_MB_RETRYCANCEL?$AA@ 10005a58     flags.obj
 0001:00004a6c       ??_C@_09NEGPLEAH@FMSG_NONE?$AA@ 10005a6c     flags.obj
 0001:00004a78       ??_C@_0N@DHJCDIKM@DIF_BOXCOLOR?$AA@ 10005a78     flags.obj
 0001:00004a88       ??_C@_09IAEPIICA@DIF_GROUP?$AA@ 10005a88     flags.obj
 0001:00004a94       ??_C@_0N@GCKJNBCM@DIF_LEFTTEXT?$AA@ 10005a94     flags.obj
 0001:00004aa4       ??_C@_0P@BGPBEDHH@DIF_MOVESELECT?$AA@ 10005aa4     flags.obj
 0001:00004ab4       ??_C@_0BC@PDKFKKEI@DIF_SHOWAMPERSAND?$AA@ 10005ab4     flags.obj
 0001:00004ac8       ??_C@_0BA@BLCOKAAO@DIF_CENTERGROUP?$AA@ 10005ac8     flags.obj
 0001:00004ad8       ??_C@_0P@MKFBJPOB@DIF_NOBRACKETS?$AA@ 10005ad8     flags.obj
 0001:00004ae8       ??_C@_0BF@JBCDBJCL@DIF_MANUALADDHISTORY?$AA@ 10005ae8     flags.obj
 0001:00004b00       ??_C@_0O@JKNMBNLA@DIF_SEPARATOR?$AA@ 10005b00     flags.obj
 0001:00004b10       ??_C@_0P@CGILDLOA@DIF_SEPARATOR2?$AA@ 10005b10     flags.obj
 0001:00004b20       ??_C@_0L@NBPFNGLB@DIF_EDITOR?$AA@ 10005b20     flags.obj
 0001:00004b2c       ??_C@_0BE@PFICAGJF@DIF_LISTNOAMPERSAND?$AA@ 10005b2c     flags.obj
 0001:00004b40       ??_C@_0O@FFJNBMAD@DIF_LISTNOBOX?$AA@ 10005b40     flags.obj
 0001:00004b50       ??_C@_0M@IPFBMFDN@DIF_HISTORY?$AA@ 10005b50     flags.obj
 0001:00004b5c       ??_C@_0P@EGFAEEDC@DIF_BTNNOCLOSE?$AA@ 10005b5c     flags.obj
 0001:00004b6c       ??_C@_0P@KOJCCCGB@DIF_CENTERTEXT?$AA@ 10005b6c     flags.obj
 0001:00004b7c       ??_C@_0BC@ODEMBOPK@DIF_SEPARATORUSER?$AA@ 10005b7c     flags.obj
 0001:00004b90       ??_C@_0O@IKJBMPOF@DIF_SETSHIELD?$AA@ 10005b90     flags.obj
 0001:00004ba0       ??_C@_0P@EEJEDBLH@DIF_EDITEXPAND?$AA@ 10005ba0     flags.obj
 0001:00004bb0       ??_C@_0BB@EIMEKEFP@DIF_DROPDOWNLIST?$AA@ 10005bb0     flags.obj
 0001:00004bc4       ??_C@_0BD@MNGIOLFF@DIF_USELASTHISTORY?$AA@ 10005bc4     flags.obj
 0001:00004bd8       ??_C@_0N@MOCGNIKC@DIF_MASKEDIT?$AA@ 10005bd8     flags.obj
 0001:00004be8       ??_C@_0BD@LPDHCLJI@DIF_LISTTRACKMOUSE?$AA@ 10005be8     flags.obj
 0001:00004bfc       ??_C@_0BK@LEFIBDOA@DIF_LISTTRACKMOUSEINFOCUS?$AA@ 10005bfc     flags.obj
 0001:00004c18       ??_C@_0BC@JNLDMGBD@DIF_SELECTONENTRY?$AA@ 10005c18     flags.obj
 0001:00004c2c       ??_C@_0L@KKNJDNBK@DIF_3STATE?$AA@ 10005c2c     flags.obj
 0001:00004c38       ??_C@_0N@GBGHICKO@DIF_EDITPATH?$AA@ 10005c38     flags.obj
 0001:00004c48       ??_C@_0BB@NPNALIGO@DIF_LISTWRAPMODE?$AA@ 10005c48     flags.obj
 0001:00004c5c       ??_C@_0BD@MFOKKGGF@DIF_NOAUTOCOMPLETE?$AA@ 10005c5c     flags.obj
 0001:00004c70       ??_C@_0BG@MONEJILE@DIF_LISTAUTOHIGHLIGHT?$AA@ 10005c70     flags.obj
 0001:00004c88       ??_C@_0BA@JNOKLHOL@DIF_LISTNOCLOSE?$AA@ 10005c88     flags.obj
 0001:00004c98       ??_C@_0BB@GMKDKOOP@DIF_EDITPATHEXEC?$AA@ 10005c98     flags.obj
 0001:00004cac       ??_C@_0L@EPNFOPAK@DIF_HIDDEN?$AA@ 10005cac     flags.obj
 0001:00004cb8       ??_C@_0N@KOGKCAKJ@DIF_READONLY?$AA@ 10005cb8     flags.obj
 0001:00004cc8       ??_C@_0M@NLLDINIM@DIF_NOFOCUS?$AA@ 10005cc8     flags.obj
 0001:00004cd4       ??_C@_0M@HCFLMDHK@DIF_DISABLE?$AA@ 10005cd4     flags.obj
 0001:00004ce0       ??_C@_0BC@CHAAKEJO@DIF_DEFAULTBUTTON?$AA@ 10005ce0     flags.obj
 0001:00004cf4       ??_C@_09LCJIOEMN@DIF_FOCUS?$AA@ 10005cf4     flags.obj
 0001:00004d00       ??_C@_0O@KJADCBBN@DIF_RIGHTTEXT?$AA@ 10005d00     flags.obj
 0001:00004d10       ??_C@_0N@LAEOODAD@DIF_WORDWRAP?$AA@ 10005d10     flags.obj
 0001:00004d20       ??_C@_08KFOHCPDE@DIF_NONE?$AA@ 10005d20     flags.obj
 0001:00004d2c       ??_C@_0N@EDHAFIIL@LIF_SELECTED?$AA@ 10005d2c     flags.obj
 0001:00004d3c       ??_C@_0M@BMGIEAIL@LIF_CHECKED?$AA@ 10005d3c     flags.obj
 0001:00004d48       ??_C@_0O@KJIFADIG@LIF_SEPARATOR?$AA@ 10005d48     flags.obj
 0001:00004d58       ??_C@_0M@HEFHLFIE@LIF_DISABLE?$AA@ 10005d58     flags.obj
 0001:00004d64       ??_C@_0L@PKDDGEEG@LIF_GRAYED?$AA@ 10005d64     flags.obj
 0001:00004d70       ??_C@_0L@PFBGAOEP@LIF_HIDDEN?$AA@ 10005d70     flags.obj
 0001:00004d7c       ??_C@_0BD@HEPCOIEH@LIF_DELETEUSERDATA?$AA@ 10005d7c     flags.obj
 0001:00004d90       ??_C@_08BODPINCM@LIF_NONE?$AA@ 10005d90     flags.obj
 0001:00004d9c       ??_C@_0BC@BGAENNBJ@LIFIND_EXACTMATCH?$AA@ 10005d9c     flags.obj
 0001:00004db0       ??_C@_0M@FPOGKIGO@LIFIND_NONE?$AA@ 10005db0     flags.obj
 0001:00004dbc       ??_C@_0BA@OOIEKCFB@LINFO_SHOWNOBOX?$AA@ 10005dbc     flags.obj
 0001:00004dcc       ??_C@_0BE@DECCEGNO@LINFO_AUTOHIGHLIGHT?$AA@ 10005dcc     flags.obj
 0001:00004de0       ??_C@_0BH@BADLEILJ@LINFO_REVERSEHIGHLIGHT?$AA@ 10005de0     flags.obj
 0001:00004df8       ??_C@_0P@KLBMHNCG@LINFO_WRAPMODE?$AA@ 10005df8     flags.obj
 0001:00004e08       ??_C@_0BE@OHJCOKAE@LINFO_SHOWAMPERSAND?$AA@ 10005e08     flags.obj
 0001:00004e1c       ??_C@_0L@EPACPANF@LINFO_NONE?$AA@ 10005e1c     flags.obj
 0001:00004e28       ??_C@_0N@OLGDMHKL@FDLG_WARNING?$AA@ 10005e28     flags.obj
 0001:00004e38       ??_C@_0BB@DKMEBDJJ@FDLG_SMALLDIALOG?$AA@ 10005e38     flags.obj
 0001:00004e4c       ??_C@_0BC@ONGLDAJN@FDLG_NODRAWSHADOW?$AA@ 10005e4c     flags.obj
 0001:00004e60       ??_C@_0BB@NPLEEAKK@FDLG_NODRAWPANEL?$AA@ 10005e60     flags.obj
 0001:00004e74       ??_C@_0BG@GHNOOENB@FDLG_KEEPCONSOLETITLE?$AA@ 10005e74     flags.obj
 0001:00004e8c       ??_C@_09NNFHCBNL@FDLG_NONE?$AA@ 10005e8c     flags.obj
 0001:00004e98       ??_C@_0N@JOOGIBAO@MIF_SELECTED?$AA@ 10005e98     flags.obj
 0001:00004ea8       ??_C@_0M@IHMNAMOE@MIF_CHECKED?$AA@ 10005ea8     flags.obj
 0001:00004eb4       ??_C@_0O@DEIKOCPA@MIF_SEPARATOR?$AA@ 10005eb4     flags.obj
 0001:00004ec4       ??_C@_0M@OPPCPJOL@MIF_DISABLE?$AA@ 10005ec4     flags.obj
 0001:00004ed0       ??_C@_0L@DLLNLLIG@MIF_GRAYED?$AA@ 10005ed0     flags.obj
 0001:00004edc       ??_C@_0L@DEJINBIP@MIF_HIDDEN?$AA@ 10005edc     flags.obj
 0001:00004ee8       ??_C@_08JEEJJGP@MIF_NONE?$AA@ 10005ee8     flags.obj
 0001:00004ef4       ??_C@_0BE@FALMPPJK@FMENU_SHOWAMPERSAND?$AA@ 10005ef4     flags.obj
 0001:00004f08       ??_C@_0P@HICDNKDJ@FMENU_WRAPMODE?$AA@ 10005f08     flags.obj
 0001:00004f18       ??_C@_0BE@IDAMFDEA@FMENU_AUTOHIGHLIGHT?$AA@ 10005f18     flags.obj
 0001:00004f2c       ??_C@_0BL@OKAIKPMN@FMENU_REVERSEAUTOHIGHLIGHT?$AA@ 10005f2c     flags.obj
 0001:00004f48       ??_C@_0BJ@FCEONOJC@FMENU_CHANGECONSOLETITLE?$AA@ 10005f48     flags.obj
 0001:00004f64       ??_C@_0L@DGFIEOMD@FMENU_NONE?$AA@ 10005f64     flags.obj
 0001:00004f70       ??_C@_0O@JEAJLDHC@PPIF_SELECTED?$AA@ 10005f70     flags.obj
 0001:00004f80       ??_C@_0BC@LPBDBIOM@PPIF_PROCESSDESCR?$AA@ 10005f80     flags.obj
 0001:00004f94       ??_C@_09OIFMMGNJ@PPIF_NONE?$AA@ 10005f94     flags.obj
 0001:00004fa0       ??_C@_0BC@BONLDOOD@PFLAGS_SHOWHIDDEN?$AA@ 10005fa0     flags.obj
 0001:00004fb4       ??_C@_0BB@BCAJEJEH@PFLAGS_HIGHLIGHT?$AA@ 10005fb4     flags.obj
 0001:00004fc8       ??_C@_0BI@BFAFODJ@PFLAGS_REVERSESORTORDER?$AA@ 10005fc8     flags.obj
 0001:00004fe0       ??_C@_0BF@KJNCJPKN@PFLAGS_USESORTGROUPS?$AA@ 10005fe0     flags.obj
 0001:00004ff8       ??_C@_0BF@LBBAIOCD@PFLAGS_SELECTEDFIRST?$AA@ 10005ff8     flags.obj
 0001:00005010       ??_C@_0BB@KDANIJNM@PFLAGS_REALNAMES?$AA@ 10006010     flags.obj
 0001:00005024       ??_C@_0BD@MOODMDAB@PFLAGS_NUMERICSORT?$AA@ 10006024     flags.obj
 0001:00005038       ??_C@_0BB@ILEHDKFJ@PFLAGS_PANELLEFT?$AA@ 10006038     flags.obj
 0001:0000504c       ??_C@_0BI@EHHAJLOH@PFLAGS_DIRECTORIESFIRST?$AA@ 1000604c     flags.obj
 0001:00005064       ??_C@_0BA@KJEPHDOM@PFLAGS_USECRC32?$AA@ 10006064     flags.obj
 0001:00005074       ??_C@_0BJ@HJFOABKG@PFLAGS_CASESENSITIVESORT?$AA@ 10006074     flags.obj
 0001:00005090       ??_C@_0O@DBPJGING@PFLAGS_PLUGIN?$AA@ 10006090     flags.obj
 0001:000050a0       ??_C@_0P@MLDEBNPK@PFLAGS_VISIBLE?$AA@ 100060a0     flags.obj
 0001:000050b0       ??_C@_0N@EOFAELOJ@PFLAGS_FOCUS?$AA@ 100060b0     flags.obj
 0001:000050c0       ??_C@_0BI@EOCCAHFA@PFLAGS_ALTERNATIVENAMES?$AA@ 100060c0     flags.obj
 0001:000050d8       ??_C@_0BA@GHMDCHHI@PFLAGS_SHORTCUT?$AA@ 100060d8     flags.obj
 0001:000050e8       ??_C@_0M@NEMAHHGP@PFLAGS_NONE?$AA@ 100060e8     flags.obj
 0001:000050f4       ??_C@_0M@IDNADAFL@VF_NONMODAL?$AA@ 100060f4     flags.obj
 0001:00005100       ??_C@_0BB@OCDDPIKL@VF_DELETEONCLOSE?$AA@ 10006100     flags.obj
 0001:00005114       ??_C@_0N@LDHALKKM@VF_ENABLE_F6?$AA@ 10006114     flags.obj
 0001:00005124       ??_C@_0BC@DLGKMECC@VF_DISABLEHISTORY?$AA@ 10006124     flags.obj
 0001:00005138       ??_C@_0BD@DHJCMLFI@VF_IMMEDIATERETURN?$AA@ 10006138     flags.obj
 0001:0000514c       ??_C@_0BJ@OGNFHEJG@VF_DELETEONLYFILEONCLOSE?$AA@ 1000614c     flags.obj
 0001:00005168       ??_C@_07CJJFHP@VF_NONE?$AA@ 10006168     flags.obj
 0001:00005170       ??_C@_0M@PIFGAPFH@EF_NONMODAL?$AA@ 10006170     flags.obj
 0001:0000517c       ??_C@_0N@DBHFPBEO@EF_CREATENEW?$AA@ 1000617c     flags.obj
 0001:0000518c       ??_C@_0N@LKLNHALI@EF_ENABLE_F6?$AA@ 1000618c     flags.obj
 0001:0000519c       ??_C@_0BC@PPEPEFFI@EF_DISABLEHISTORY?$AA@ 1000619c     flags.obj
 0001:000051b0       ??_C@_0BB@KGPIDKFC@EF_DELETEONCLOSE?$AA@ 100061b0     flags.obj
 0001:000051c4       ??_C@_0BD@IHIGHGPL@EF_IMMEDIATERETURN?$AA@ 100061c4     flags.obj
 0001:000051d8       ??_C@_0BJ@ILCPOFKL@EF_DELETEONLYFILEONCLOSE?$AA@ 100061d8     flags.obj
 0001:000051f4       ??_C@_09IJMPFPLB@EF_LOCKED?$AA@ 100061f4     flags.obj
 0001:00005200       ??_C@_0BC@GFHJGKD@EF_DISABLESAVEPOS?$AA@ 10006200     flags.obj
 0001:00005214       ??_C@_0BB@NILAHAFO@EF_OPENMODE_MASK?$AA@ 10006214     flags.obj
 0001:00005228       ??_C@_0BC@GAIDEJIA@EF_OPENMODE_QUERY?$AA@ 10006228     flags.obj
 0001:0000523c       ??_C@_0BG@BFKJJBAG@EF_OPENMODE_NEWIFOPEN?$AA@ 1000623c     flags.obj
 0001:00005254       ??_C@_0BI@KGOKGPEI@EF_OPENMODE_USEEXISTING?$AA@ 10006254     flags.obj
 0001:0000526c       ??_C@_0BI@EJBKKDJ@EF_OPENMODE_BREAKIFOPEN?$AA@ 1000626c     flags.obj
 0001:00005284       ??_C@_0BJ@MOLGCBMH@EF_OPENMODE_RELOADIFOPEN?$AA@ 10006284     flags.obj
 0001:000052a0       ??_C@_07MBPCONNA@EN_NONE?$AA@ 100062a0     flags.obj
 0001:000052a8       ??_C@_0BC@HHNGCBAM@FHELP_NOSHOWERROR?$AA@ 100062a8     flags.obj
 0001:000052bc       ??_C@_0P@GANNLHEJ@FHELP_SELFHELP?$AA@ 100062bc     flags.obj
 0001:000052cc       ??_C@_0O@FLGGLFLC@FHELP_FARHELP?$AA@ 100062cc     flags.obj
 0001:000052dc       ??_C@_0BB@KNKDPNI@FHELP_CUSTOMFILE?$AA@ 100062dc     flags.obj
 0001:000052f0       ??_C@_0BB@IHFFPJJA@FHELP_CUSTOMPATH?$AA@ 100062f0     flags.obj
 0001:00005304       ??_C@_0L@OOIMFPBD@FHELP_GUID?$AA@ 10006304     flags.obj
 0001:00005310       ??_C@_0BC@PNPOIHMG@FHELP_USECONTENTS?$AA@ 10006310     flags.obj
 0001:00005324       ??_C@_0L@MAGMKNFN@FHELP_NONE?$AA@ 10006324     flags.obj
 0001:00005330       ??_C@_0BE@GEGKIINM@KMFLAGS_SILENTCHECK?$AA@ 10006330     flags.obj
 0001:00005344       ??_C@_0BM@BBOPLPKC@KMFLAGS_NOSENDKEYSTOPLUGINS?$AA@ 10006344     flags.obj
 0001:00005360       ??_C@_0BF@PHHPAAOK@KMFLAGS_ENABLEOUTPUT?$AA@ 10006360     flags.obj
 0001:00005378       ??_C@_0BB@NCECNBPK@KMFLAGS_LANGMASK?$AA@ 10006378     flags.obj
 0001:0000538c       ??_C@_0M@HFBACHCP@KMFLAGS_LUA?$AA@ 1000638c     flags.obj
 0001:00005398       ??_C@_0BD@JHNPMIGP@KMFLAGS_MOONSCRIPT?$AA@ 10006398     flags.obj
 0001:000053ac       ??_C@_0N@GIJCDFJI@KMFLAGS_NONE?$AA@ 100063ac     flags.obj
 0001:000053bc       ??_C@_0O@GKOLBMFK@AKMFLAGS_NONE?$AA@ 100063bc     flags.obj
 0001:000053cc       ??_C@_0P@LMBMJIMF@FSETCLR_REDRAW?$AA@ 100063cc     flags.obj
 0001:000053dc       ??_C@_0N@LCOHPDHN@FSETCLR_NONE?$AA@ 100063dc     flags.obj
 0001:000053ec       ??_C@_0N@MLMCEKPH@WIF_MODIFIED?$AA@ 100063ec     flags.obj
 0001:000053fc       ??_C@_0M@ICPAPCOF@WIF_CURRENT?$AA@ 100063fc     flags.obj
 0001:00005408       ??_C@_09FPGEBDGO@WIF_MODAL?$AA@ 10006408     flags.obj
 0001:00005414       ??_C@_08DAKKFBIA@WIF_NONE?$AA@ 10006414     flags.obj
 0001:00005420       ??_C@_0BG@JMJAOELH@VOPT_SAVEFILEPOSITION?$AA@ 10006420     flags.obj
 0001:00005438       ??_C@_0BI@NCAHLEBN@VOPT_AUTODETECTCODEPAGE?$AA@ 10006438     flags.obj
 0001:00005450       ??_C@_0BC@FGLBHLDI@VOPT_SHOWTITLEBAR?$AA@ 10006450     flags.obj
 0001:00005464       ??_C@_0BA@GAIDGLME@VOPT_SHOWKEYBAR?$AA@ 10006464     flags.obj
 0001:00005474       ??_C@_0BD@LEEGOJKA@VOPT_SHOWSCROLLBAR?$AA@ 10006474     flags.obj
 0001:00005488       ??_C@_0P@NEIKPMJJ@VOPT_QUICKVIEW?$AA@ 10006488     flags.obj
 0001:00005498       ??_C@_09FIOJMNJ@VOPT_NONE?$AA@ 10006498     flags.obj
 0001:000054a4       ??_C@_0N@ILNDJNNO@VSMFL_REDRAW?$AA@ 100064a4     flags.obj
 0001:000054b4       ??_C@_0L@DLLCFLOD@VSMFL_NONE?$AA@ 100064b4     flags.obj
 0001:000054c0       ??_C@_0N@GHEHKHJN@VSP_NOREDRAW?$AA@ 100064c0     flags.obj
 0001:000054d0       ??_C@_0M@LHNGMHFO@VSP_PERCENT?$AA@ 100064d0     flags.obj
 0001:000054dc       ??_C@_0N@JGGGCNIP@VSP_RELATIVE?$AA@ 100064dc     flags.obj
 0001:000054ec       ??_C@_0BA@JKDMJLJG@VSP_NORETNEWPOS?$AA@ 100064ec     flags.obj
 0001:000054fc       ??_C@_08MOKEMBNE@VSP_NONE?$AA@ 100064fc     flags.obj
 0001:00005508       ??_C@_08FAPBJAKB@VMF_WRAP?$AA@ 10006508     flags.obj
 0001:00005514       ??_C@_0N@GHBDMLON@VMF_WORDWRAP?$AA@ 10006514     flags.obj
 0001:00005524       ??_C@_08KDJLELDJ@VMF_NONE?$AA@ 10006524     flags.obj
 0001:00005530       ??_C@_0BB@EDGIEBDF@ECF_TABMARKFIRST?$AA@ 10006530     flags.obj
 0001:00005544       ??_C@_0BD@DKGCCJNG@ECF_TABMARKCURRENT?$AA@ 10006544     flags.obj
 0001:00005558       ??_C@_0P@BAFEMBAJ@ECF_AUTODELETE?$AA@ 10006558     flags.obj
 0001:00005568       ??_C@_08CDFMCHLP@ECF_NONE?$AA@ 10006568     flags.obj
 0001:00005574       ??_C@_0BA@KNNLMGCA@FIB_ENABLEEMPTY?$AA@ 10006574     flags.obj
 0001:00005584       ??_C@_0N@DLDJCGJI@FIB_PASSWORD?$AA@ 10006584     flags.obj
 0001:00005594       ??_C@_0O@DOHEGELC@FIB_EXPANDENV?$AA@ 10006594     flags.obj
 0001:000055a4       ??_C@_0BF@CEMIHIOK@FIB_NOUSELASTHISTORY?$AA@ 100065a4     flags.obj
 0001:000055bc       ??_C@_0M@KJOJJDIM@FIB_BUTTONS?$AA@ 100065bc     flags.obj
 0001:000055c8       ??_C@_0BA@COBBDHNL@FIB_NOAMPERSAND?$AA@ 100065c8     flags.obj
 0001:000055d8       ??_C@_0N@LBOCEEGH@FIB_EDITPATH?$AA@ 100065d8     flags.obj
 0001:000055e8       ??_C@_0BB@DCODFLEL@FIB_EDITPATHEXEC?$AA@ 100065e8     flags.obj
 0001:000055fc       ??_C@_08HPFOCDKB@FIB_NONE?$AA@ 100065fc     flags.obj
 0001:00005608       ??_C@_0L@NMBLFMBN@FPF_LOADED?$AA@ 10006608     flags.obj
 0001:00005614       ??_C@_08GKECKCCJ@FPF_ANSI?$AA@ 10006614     flags.obj
 0001:00005620       ??_C@_08OIOFCNLC@FPF_NONE?$AA@ 10006620     flags.obj
 0001:0000562c       ??_C@_0L@HODJIPGA@PN_CMPNAME?$AA@ 1000662c     flags.obj
 0001:00005638       ??_C@_0P@KDEENAHJ@PN_CMPNAMELIST?$AA@ 10006638     flags.obj
 0001:00005648       ??_C@_0BA@BJCCEIOI@PN_GENERATENAME?$AA@ 10006648     flags.obj
 0001:00005658       ??_C@_0N@FEGPCCPJ@PN_CHECKMASK?$AA@ 10006658     flags.obj
 0001:00005668       ??_C@_0M@NOOLKEBH@PN_SKIPPATH?$AA@ 10006668     flags.obj
 0001:00005674       ??_C@_0BE@OPDBOAAE@PN_SHOWERRORMESSAGE?$AA@ 10006674     flags.obj
 0001:00005688       ??_C@_07PFKJNCJP@PN_NONE?$AA@ 10006688     flags.obj
 0001:00005690       ??_C@_0BG@GOMJDMCK@XLAT_SWITCHKEYBLAYOUT?$AA@ 10006690     flags.obj
 0001:000056a8       ??_C@_0BE@KOIJDNLA@XLAT_SWITCHKEYBBEEP?$AA@ 100066a8     flags.obj
 0001:000056bc       ??_C@_0BH@KBFAFPNA@XLAT_USEKEYBLAYOUTNAME?$AA@ 100066bc     flags.obj
 0001:000056d4       ??_C@_0BH@IANKLOAC@XLAT_CONVERTALLCMDLINE?$AA@ 100066d4     flags.obj
 0001:000056ec       ??_C@_09JCNLKBBK@XLAT_NONE?$AA@ 100066ec     flags.obj
 0001:000056f8       ??_C@_0N@PJEDCNNJ@FRS_RETUPDIR?$AA@ 100066f8     flags.obj
 0001:00005708       ??_C@_09GHEPLOHO@FRS_RECUR?$AA@ 10006708     flags.obj
 0001:00005714       ??_C@_0BA@JCPHOEAE@FRS_SCANSYMLINK?$AA@ 10006714     flags.obj
 0001:00005724       ??_C@_08JPCGJJKG@FRS_NONE?$AA@ 10006724     flags.obj
 0001:00005730       ??_C@_0P@LJPBHEIE@MLF_SHOWERRMSG?$AA@ 10006730     flags.obj
 0001:00005740       ??_C@_0BF@LMAGFLHF@MLF_DONOTUPDATEPANEL?$AA@ 10006740     flags.obj
 0001:00005758       ??_C@_0P@EPFBLPAE@MLF_HOLDTARGET?$AA@ 10006758     flags.obj
 0001:00005768       ??_C@_08EBKEJHAL@MLF_NONE?$AA@ 10006768     flags.obj
 0001:00005774       ??_C@_0M@JDMKDBDH@FFFS_COMMAS?$AA@ 10006774     flags.obj
 0001:00005780       ??_C@_0P@JPMLNBKL@FFFS_FLOATSIZE?$AA@ 10006780     flags.obj
 0001:00005790       ??_C@_0BE@NPKCCEJ@FFFS_SHOWBYTESINDEX?$AA@ 10006790     flags.obj
 0001:000057a4       ??_C@_0O@FPIOAIMC@FFFS_ECONOMIC?$AA@ 100067a4     flags.obj
 0001:000057b4       ??_C@_0O@HFIGPFIH@FFFS_THOUSAND?$AA@ 100067b4     flags.obj
 0001:000057c4       ??_C@_0BC@LLLANJJO@FFFS_MINSIZEINDEX?$AA@ 100067c4     flags.obj
 0001:000057d8       ??_C@_0BH@PEGBPJKE@FFFS_MINSIZEINDEX_MASK?$AA@ 100067d8     flags.obj
 0001:000057f0       ??_C@_09PBPAKNEI@FFFS_NONE?$AA@ 100067f0     flags.obj
 0001:000057fc       ??_C@_0L@NHEJGKCF@PF_PRELOAD?$AA@ 100067fc     flags.obj
 0001:00005808       ??_C@_0BB@GCINAIGN@PF_DISABLEPANELS?$AA@ 10006808     flags.obj
 0001:0000581c       ??_C@_09OENCMPGE@PF_EDITOR?$AA@ 1000681c     flags.obj
 0001:00005828       ??_C@_09NEKIJNNA@PF_VIEWER?$AA@ 10006828     flags.obj
 0001:00005834       ??_C@_0P@MBLBBCNK@PF_FULLCMDLINE?$AA@ 10006834     flags.obj
 0001:00005844       ??_C@_09GMFDAFKL@PF_DIALOG?$AA@ 10006844     flags.obj
 0001:00005850       ??_C@_07MGEGJMPI@PF_NONE?$AA@ 10006850     flags.obj
 0001:00005858       ??_C@_0BD@EGELEIIG@IPLFLAGS_SEPARATOR?$AA@ 10006858     flags.obj
 0001:0000586c       ??_C@_0O@JBNJFHHK@IPLFLAGS_NONE?$AA@ 1000686c     flags.obj
 0001:0000587c       ??_C@_0BD@KGHJOBGM@PMFLAGS_FULLSCREEN?$AA@ 1000687c     flags.obj
 0001:00005890       ??_C@_0BH@GDAAKEMH@PMFLAGS_DETAILEDSTATUS?$AA@ 10006890     flags.obj
 0001:000058a8       ??_C@_0BI@BMHIBDMH@PMFLAGS_ALIGNEXTENSIONS?$AA@ 100068a8     flags.obj
 0001:000058c0       ??_C@_0BH@KOFCBJBO@PMFLAGS_CASECONVERSION?$AA@ 100068c0     flags.obj
 0001:000058d8       ??_C@_0N@DLFMCMOB@PMFLAGS_NONE?$AA@ 100068d8     flags.obj
 0001:000058e8       ??_C@_0BD@PBMGDJEM@OPIF_DISABLEFILTER?$AA@ 100068e8     flags.obj
 0001:000058fc       ??_C@_0BH@FHBKALPD@OPIF_DISABLESORTGROUPS?$AA@ 100068fc     flags.obj
 0001:00005914       ??_C@_0BJ@NGLIANCL@OPIF_DISABLEHIGHLIGHTING?$AA@ 10006914     flags.obj
 0001:00005930       ??_C@_0N@JANKJMLP@OPIF_ADDDOTS?$AA@ 10006930     flags.obj
 0001:00005940       ??_C@_0BC@HOFHNJIG@OPIF_RAWSELECTION?$AA@ 10006940     flags.obj
 0001:00005954       ??_C@_0P@OFEDJCO@OPIF_REALNAMES?$AA@ 10006954     flags.obj
 0001:00005964       ??_C@_0BD@FPGMNAPD@OPIF_SHOWNAMESONLY?$AA@ 10006964     flags.obj
 0001:00005978       ??_C@_0BJ@NMIFAPJD@OPIF_SHOWRIGHTALIGNNAMES?$AA@ 10006978     flags.obj
 0001:00005994       ??_C@_0BG@HGPMKHIE@OPIF_SHOWPRESERVECASE?$AA@ 10006994     flags.obj
 0001:000059ac       ??_C@_0BE@GJEJHNKJ@OPIF_COMPAREFATTIME?$AA@ 100069ac     flags.obj
 0001:000059c0       ??_C@_0BB@PELHBPAM@OPIF_EXTERNALGET?$AA@ 100069c0     flags.obj
 0001:000059d4       ??_C@_0BB@CFFPNDFK@OPIF_EXTERNALPUT?$AA@ 100069d4     flags.obj
 0001:000059e8       ??_C@_0BE@LKEMICNM@OPIF_EXTERNALDELETE?$AA@ 100069e8     flags.obj
 0001:000059fc       ??_C@_0BD@JIMJPFEP@OPIF_EXTERNALMKDIR?$AA@ 100069fc     flags.obj
 0001:00005a10       ??_C@_0BJ@CALDMPLF@OPIF_USEATTRHIGHLIGHTING?$AA@ 10006a10     flags.obj
 0001:00005a2c       ??_C@_0O@JHHHMHIG@OPIF_USECRC32?$AA@ 10006a2c     flags.obj
 0001:00005a3c       ??_C@_0BB@PFDFAFHG@OPIF_USEFREESIZE?$AA@ 10006a3c     flags.obj
 0001:00005a50       ??_C@_0O@FJPLJDBC@OPIF_SHORTCUT?$AA@ 10006a50     flags.obj
 0001:00005a60       ??_C@_09DOPJBMLM@OPIF_NONE?$AA@ 10006a60     flags.obj
 0001:00005a6c       ??_C@_0L@GEHHKNBL@OPM_SILENT?$AA@ 10006a6c     flags.obj
 0001:00005a78       ??_C@_08EKEBOKEP@OPM_FIND?$AA@ 10006a78     flags.obj
 0001:00005a84       ??_C@_08EHBLNDLO@OPM_VIEW?$AA@ 10006a84     flags.obj
 0001:00005a90       ??_C@_08LAAGEMJG@OPM_EDIT?$AA@ 10006a90     flags.obj
 0001:00005a9c       ??_C@_0N@NDGKAFDM@OPM_TOPLEVEL?$AA@ 10006a9c     flags.obj
 0001:00005aac       ??_C@_09EBKAPHPA@OPM_DESCR?$AA@ 10006aac     flags.obj
 0001:00005ab8       ??_C@_0O@OPDAGBBE@OPM_QUICKVIEW?$AA@ 10006ab8     flags.obj
 0001:00005ac8       ??_C@_08LCEGJCAC@OPM_PGDN?$AA@ 10006ac8     flags.obj
 0001:00005ad4       ??_C@_0N@HKCLLJDG@OPM_COMMANDS?$AA@ 10006ad4     flags.obj
 0001:00005ae4       ??_C@_08EGEBMPBD@OPM_NONE?$AA@ 10006ae4     flags.obj
 0001:00005af0       ??_C@_0M@MIGJPBPE@FOSF_ACTIVE?$AA@ 10006af0     flags.obj
 0001:00005afc       ??_C@_09FMOOJHDF@FOSF_NONE?$AA@ 10006afc     flags.obj
 0001:00005b08       ??_C@_0O@PLFENGLI@PCIF_FROMMAIN?$AA@ 10006b08     flags.obj
 0001:00005b18       ??_C@_09HNBBLIGN@PCIF_NONE?$AA@ 10006b18     flags.obj
 0001:00005b24       ??_C@_0BA@MAEBFMHC@FOREGROUND_BLUE?$AA@ 10006b24     flags.obj
 0001:00005b34       ??_C@_0BB@PDFNMAI@FOREGROUND_GREEN?$AA@ 10006b34     flags.obj
 0001:00005b48       ??_C@_0P@PBJHCFGA@FOREGROUND_RED?$AA@ 10006b48     flags.obj
 0001:00005b58       ??_C@_0BF@OOGEJCC@FOREGROUND_INTENSITY?$AA@ 10006b58     flags.obj
 0001:00005b70       ??_C@_0BA@PIFINJCK@BACKGROUND_BLUE?$AA@ 10006b70     flags.obj
 0001:00005b80       ??_C@_0BB@GKLNBMEL@BACKGROUND_GREEN?$AA@ 10006b80     flags.obj
 0001:00005b94       ??_C@_0P@DANALJMC@BACKGROUND_RED?$AA@ 10006b94     flags.obj
 0001:00005ba4       ??_C@_0BF@NIGKKPCF@BACKGROUND_INTENSITY?$AA@ 10006ba4     flags.obj
 0001:00005bbc       ??_C@_0N@FEFOEFHG@CTRL_C_EVENT?$AA@ 10006bbc     flags.obj
 0001:00005bcc       ??_C@_0BB@ELEIIFAE@CTRL_BREAK_EVENT?$AA@ 10006bcc     flags.obj
 0001:00005be0       ??_C@_0BB@KMPDMOKK@CTRL_CLOSE_EVENT?$AA@ 10006be0     flags.obj
 0001:00005bf4       ??_C@_0BC@MCKCEPAL@CTRL_LOGOFF_EVENT?$AA@ 10006bf4     flags.obj
 0001:00005c08       ??_C@_0BE@BCNEFGKM@CTRL_SHUTDOWN_EVENT?$AA@ 10006c08     flags.obj
 0001:00005c1c       ??_C@_0BC@BBOPHMOM@ENABLE_LINE_INPUT?$AA@ 10006c1c     flags.obj
 0001:00005c30       ??_C@_0BC@JPFKLHOC@ENABLE_ECHO_INPUT?$AA@ 10006c30     flags.obj
 0001:00005c44       ??_C@_0BH@EHINFMOF@ENABLE_PROCESSED_INPUT?$AA@ 10006c44     flags.obj
 0001:00005c5c       ??_C@_0BE@BLAHACNB@ENABLE_WINDOW_INPUT?$AA@ 10006c5c     flags.obj
 0001:00005c70       ??_C@_0BD@BJECBJPO@ENABLE_MOUSE_INPUT?$AA@ 10006c70     flags.obj
 0001:00005c84       ??_C@_0BD@KJBPOMPN@ENABLE_INSERT_MODE?$AA@ 10006c84     flags.obj
 0001:00005c98       ??_C@_0BH@BJKMFKAO@ENABLE_QUICK_EDIT_MODE?$AA@ 10006c98     flags.obj
 0001:00005cb0       ??_C@_0BG@CBCHHIEH@ENABLE_EXTENDED_FLAGS?$AA@ 10006cb0     flags.obj
 0001:00005cc8       ??_C@_0BF@PEBFEBKN@ENABLE_AUTO_POSITION?$AA@ 10006cc8     flags.obj
 0001:00005ce0       ??_C@_0BI@MHKNPIFM@ENABLE_PROCESSED_OUTPUT?$AA@ 10006ce0     flags.obj
 0001:00005cf8       ??_C@_0BK@CDKLKCHJ@ENABLE_WRAP_AT_EOL_OUTPUT?$AA@ 10006cf8     flags.obj
 0001:00005d14       ??_C@_09JBABGNAE@KEY_EVENT?$AA@ 10006d14     flags.obj
 0001:00005d20       ??_C@_0M@CPILDGOO@MOUSE_EVENT?$AA@ 10006d20     flags.obj
 0001:00005d2c       ??_C@_0BJ@OHDOHJKG@WINDOW_BUFFER_SIZE_EVENT?$AA@ 10006d2c     flags.obj
 0001:00005d48       ??_C@_0L@MPODFLFH@MENU_EVENT?$AA@ 10006d48     flags.obj
 0001:00005d54       ??_C@_0M@LNGHCCGJ@FOCUS_EVENT?$AA@ 10006d54     flags.obj
 0001:00005d60       ??_C@_0M@MKBGBFGO@CAPSLOCK_ON?$AA@ 10006d60     flags.obj
 0001:00005d6c       ??_C@_0N@EMEOEKDA@ENHANCED_KEY?$AA@ 10006d6c     flags.obj
 0001:00005d7c       ??_C@_0BC@GDHABBAP@RIGHT_ALT_PRESSED?$AA@ 10006d7c     flags.obj
 0001:00005d90       ??_C@_0BB@MCADLJJO@LEFT_ALT_PRESSED?$AA@ 10006d90     flags.obj
 0001:00005da4       ??_C@_0BD@NEHHNAHO@RIGHT_CTRL_PRESSED?$AA@ 10006da4     flags.obj
 0001:00005db8       ??_C@_0BC@FDNOAAAE@LEFT_CTRL_PRESSED?$AA@ 10006db8     flags.obj
 0001:00005dcc       ??_C@_0O@OGDFJMBK@SHIFT_PRESSED?$AA@ 10006dcc     flags.obj
 0001:00005ddc       ??_C@_0L@IMGKKBIM@NUMLOCK_ON?$AA@ 10006ddc     flags.obj
 0001:00005de8       ??_C@_0O@LAHFNPLG@SCROLLLOCK_ON?$AA@ 10006de8     flags.obj
 0001:00005df8       ??_C@_0BN@HACKHGAB@FROM_LEFT_1ST_BUTTON_PRESSED?$AA@ 10006df8     flags.obj
 0001:00005e18       ??_C@_0BJ@JECFAJNJ@RIGHTMOST_BUTTON_PRESSED?$AA@ 10006e18     flags.obj
 0001:00005e34       ??_C@_0BN@BJCFPKCG@FROM_LEFT_2ND_BUTTON_PRESSED?$AA@ 10006e34     flags.obj
 0001:00005e54       ??_C@_0BN@PMJNFPGM@FROM_LEFT_3RD_BUTTON_PRESSED?$AA@ 10006e54     flags.obj
 0001:00005e74       ??_C@_0BN@CNMHAAPD@FROM_LEFT_4TH_BUTTON_PRESSED?$AA@ 10006e74     flags.obj
 0001:00005e94       ??_C@_0M@KKBDEELB@MOUSE_MOVED?$AA@ 10006e94     flags.obj
 0001:00005ea0       ??_C@_0N@EDCKBGJE@DOUBLE_CLICK?$AA@ 10006ea0     flags.obj
 0001:00005eb0       ??_C@_0O@GABDOPO@MOUSE_WHEELED?$AA@ 10006eb0     flags.obj
 0001:00005ec0       ??_C@_0BA@OOKCCMHH@KEY_WOW64_32KEY?$AA@ 10006ec0     flags.obj
 0001:00005ed0       ??_C@_0BA@DBCPEIGE@KEY_WOW64_64KEY?$AA@ 10006ed0     flags.obj
 0001:000080fc       ??_C@_06ICDCBJPI@Colors?$AA@ 100090fc     keysandcolors.obj
 0001:00008104       ??_C@_05GALAPKHH@Guids?$AA@ 10009104     keysandcolors.obj
 0001:000089a8       ??_C@_01EEMJAFIK@?6?$AA@   100099a8     lflua.obj
 0001:000089ac       ??_C@_0BB@BJDGDOHH@cannot?5?$CFs?5?$CFs?3?5?$CFs?$AA@ 100099ac     lflua.obj
 0001:000089c0       ??_C@_03PKPBNCAL@?o?$LL?$LP?$AA@ 100099c0     lflua.obj
 0001:000089c4       ??_C@_06CCPPALKB@?$DNstdin?$AA@ 100099c4     lflua.obj
 0001:000089cc       ??_C@_01EOFPKCAF@?$EA?$AA@ 100099cc     lflua.obj
 0001:000089d0       ??_C@_04PMOCAHAA@open?$AA@ 100099d0     lflua.obj
 0001:000089d8       ??_C@_15JJPIMNBO@?$AAr?$AAb?$AA?$AA@ 100099d8     lflua.obj
 0001:000089e0       ??_C@_06IEGCHAII@reopen?$AA@ 100099e0     lflua.obj
 0001:000089e8       ??_C@_04POLDLDMI@read?$AA@ 100099e8     lflua.obj
 0001:000089f0       ??_C@_02LOCGON@?$AA?$AA?$AA@ 100099f0     lflua.obj
 0001:00008dd0       _regex_methods             10009dd0     lregex.obj
 0001:00008e80       _regex_functions           10009e80     lregex.obj
 0001:00009330       ??_C@_04CKFJHKAP@find?$AA@ 1000a330     lregex.obj
 0001:00009338       ??_C@_04GOLEAPFD@gsub?$AA@ 1000a338     lregex.obj
 0001:00009340       ??_C@_05FNONLPDI@match?$AA@ 1000a340     lregex.obj
 0001:00009348       ??_C@_05GFGPIPHI@findW?$AA@ 1000a348     lregex.obj
 0001:00009350       ??_C@_05HPGHPNC@gsubW?$AA@ 1000a350     lregex.obj
 0001:00009358       ??_C@_06NNKFJOLC@matchW?$AA@ 1000a358     lregex.obj
 0001:00009360       ??_C@_0O@OJAOCNID@bracketscount?$AA@ 1000a360     lregex.obj
 0001:00009370       ??_C@_04BDLIKKMN@__gc?$AA@ 1000a370     lregex.obj
 0001:00009378       ??_C@_06DPFCLDIO@gmatch?$AA@ 1000a378     lregex.obj
 0001:00009380       ??_C@_07PPMFDHAH@gmatchW?$AA@ 1000a380     lregex.obj
 0001:00009388       ??_C@_09KIEPBIJC@far_regex?$AA@ 1000a388     lregex.obj
 0001:00009394       ??_C@_0BO@PBOFMCLL@attempt?5to?5access?5freed?5regex?$AA@ 1000a394     lregex.obj
 0001:000093b4       ??_C@_07IHINEPFG@?$CFs?5?$CI?$CFp?$CJ?$AA@ 1000a3b4     lregex.obj
 0001:000093bc       ??_C@_01KMDKNFGN@?1?$AA@   1000a3bc     lregex.obj
 0001:000093c0       ??_C@_0BE@BBBEAHLK@RECTL_CREATE?5failed?$AA@ 1000a3c0     lregex.obj
 0001:000093d4       ??_C@_0BL@HEFMPIBG@invalid?5regular?5expression?$AA@ 1000a3d4     lregex.obj
 0001:000093f0       ??_C@_0BK@JCLHPPNA@cannot?5add?5?$CFd?5stack?5slots?$AA@ 1000a3f0     lregex.obj
 0001:0000940c       ??_C@_0BM@MOHHGMBK@string?5or?5table?5or?5function?$AA@ 1000a40c     lregex.obj
 0001:00009428       ??_C@_0CG@IDFLGMFM@replace?5string?3?5invalid?5capture?5@ 1000a428     lregex.obj
 0001:00009450       ??_C@_0BJ@IMAIDFKH@invalid?5replacement?5type?$AA@ 1000a450     lregex.obj
 0001:0000946c       ??_C@_0BE@KPDOHKBE@invalid?5return?5type?$AA@ 1000a46c     lregex.obj
 0001:00009480       ??_C@_07NHABFFHN@__index?$AA@ 1000a480     lregex.obj
 0001:00009488       ??_C@_05FGAODPCE@regex?$AA@ 1000a488     lregex.obj
 0001:00009d38       ??_C@_0BC@PMGNICBE@MacroPluginReturn?$AA@ 1000ad38     luamacro.obj
 0001:00009d4c       ??_C@_02JIEIHMJD@wl?$AA@   1000ad4c     luamacro.obj
 0001:00009d50       ??_C@_15PMCGDJNJ@?$AAO?$AAK?$AA?$AA@ 1000ad50     luamacro.obj
 0001:00009d58       ??_C@_1BC@GBFPAMBP@?$AAL?$AAu?$AAa?$AAM?$AAa?$AAc?$AAr?$AAo?$AA?$AA@ 1000ad58     luamacro.obj
 0001:00009d70       ??_C@_1FA@DAFHIDEP@?$AAt?$AAo?$AAo?$AA?5?$AAm?$AAa?$AAn?$AAy?$AA?5?$AAv?$AAa?$AAl?$AAu?$AAe?$AAs?$AA?5?$AAt?$AAo?$AA?5?$AAp?$AAl?$AAa?$AAc?$AAe?$AA?5?$AAo?$AAn?$AAt?$AAo?$AA?5?$AAL?$AAu@ 1000ad70     luamacro.obj
 0001:00009dc0       ??_C@_0BN@ICDOMFBB@invalid?5argument?5?$CD?$CFd?5to?5?8?$CFs?8?$AA@ 1000adc0     luamacro.obj
 0001:00009de0       ??_C@_0BB@FCMFBGOM@invalid?5argument?$AA@ 1000ade0     luamacro.obj
 0001:0000a510       _usercontrol_methods       1000b510     lusercontrol.obj
 0001:0000a550       _usercontrol_functions     1000b550     lusercontrol.obj
 0001:0000a6c0       ??_C@_05MNDELLDN@__len?$AA@ 1000b6c0     lusercontrol.obj
 0001:0000a6c8       ??_C@_0L@GADKNKH@__newindex?$AA@ 1000b6c8     lusercontrol.obj
 0001:0000a6d4       ??_C@_0BC@KFJDHEIC@CreateUserControl?$AA@ 1000b6d4     lusercontrol.obj
 0001:0000a6e8       ??_C@_0BA@MDNLMOMP@far_usercontrol?$AA@ 1000b6e8     lusercontrol.obj
 0001:0000a6f8       ??_C@_0BH@DOPNHMGD@bounds?5checking?5failed?$AA@ 1000b6f8     lusercontrol.obj
 0001:0000a710       ??_C@_09LDLEBFOB@rawhandle?$AA@ 1000b710     lusercontrol.obj
 0001:0000a71c       ??_C@_04IMAAEPPE@Char?$AA@ 1000b71c     lusercontrol.obj
 0001:0000a724       ??_C@_0L@PLFFHFAH@Attributes?$AA@ 1000b724     lusercontrol.obj
 0001:0000a730       ??_C@_0BD@BPIMECDH@X?5must?5be?5positive?$AA@ 1000b730     lusercontrol.obj
 0001:0000a744       ??_C@_0BD@MIGOMCGP@Y?5must?5be?5positive?$AA@ 1000b744     lusercontrol.obj
 0001:0000a828       _timer_methods             1000b828     service.obj
 0001:0000a858       _filefilter_methods        1000b858     service.obj
 0001:0000a890       _dialog_methods            1000b890     service.obj
 0001:0000a8b8       _Settings_methods          1000b8b8     service.obj
 0001:0000a908       _editor_funcs              1000b908     service.obj
 0001:0000aa50       _viewer_funcs              1000ba50     service.obj
 0001:0000aab0       _panel_funcs               1000bab0     service.obj
 0001:0000ac20       _far_funcs                 1000bc20     service.obj
 0001:0000afa8       _far_Dialog                1000bfa8     service.obj
 0001:0000b240       _FarFileFilterType         1000c240     service.obj
 0001:0000b258       _FarTimerType              1000c258     service.obj
 0001:0000b264       _FarDialogType             1000c264     service.obj
 0001:0000b298       _SettingsType              1000c298     service.obj
 0001:0000b2a4       _SettingsHandles           1000c2a4     service.obj
 0001:0000b2c8       _PluginHandleType          1000c2c8     service.obj
 0001:0000b2e8       _AddMacroDataType          1000c2e8     service.obj
 0001:0000b318       _SavedScreenType           1000c318     service.obj
 0001:0000b328       _FAR_VIRTUALKEYS           1000c328     service.obj
 0001:0000b358       _FAR_FLAGSTABLE            1000c358     service.obj
 0001:0000b364       _FAR_DN_STORAGE            1000c364     service.obj
 0001:0000b558       _api_functions             1000c558     service.obj
 0001:0000b980       ??_C@_0P@LKPINHLK@FreeFileFilter?$AA@ 1000c980     service.obj
 0001:0000b990       ??_C@_0BA@JGEOEAE@OpenFiltersMenu?$AA@ 1000c990     service.obj
 0001:0000b9a0       ??_C@_0BB@OPPOFOAK@StartingToFilter?$AA@ 1000c9a0     service.obj
 0001:0000b9b4       ??_C@_0P@JDMCHDIM@IsFileInFilter?$AA@ 1000c9b4     service.obj
 0001:0000b9c4       ??_C@_04MIIPNNEF@send?$AA@ 1000c9c4     service.obj
 0001:0000b9cc       ??_C@_06JBKGCNBB@Delete?$AA@ 1000c9cc     service.obj
 0001:0000b9d4       ??_C@_04PAFOOALK@Enum?$AA@ 1000c9d4     service.obj
 0001:0000b9dc       ??_C@_04HJMOFLDF@Free?$AA@ 1000c9dc     service.obj
 0001:0000b9e4       ??_C@_03NNDHPFFO@Get?$AA@  1000c9e4     service.obj
 0001:0000b9e8       ??_C@_03CEMDFJG@Set?$AA@   1000c9e8     service.obj
 0001:0000b9ec       ??_C@_0N@OELJMCEC@CreateSubkey?$AA@ 1000c9ec     service.obj
 0001:0000b9fc       ??_C@_0L@CPCKAMD@OpenSubkey?$AA@ 1000c9fc     service.obj
 0001:0000ba08       ??_C@_08EGJLHNCO@AddColor?$AA@ 1000ca08     service.obj
 0001:0000ba14       ??_C@_0BD@DOFEEDDC@AddSessionBookmark?$AA@ 1000ca14     service.obj
 0001:0000ba28       ??_C@_0BG@IGFHDIIN@ClearSessionBookmarks?$AA@ 1000ca28     service.obj
 0001:0000ba40       ??_C@_08PDEJHGJI@DelColor?$AA@ 1000ca40     service.obj
 0001:0000ba4c       ??_C@_0M@LPIECDD@DeleteBlock?$AA@ 1000ca4c     service.obj
 0001:0000ba58       ??_C@_0L@BCLIBKOC@DeleteChar?$AA@ 1000ca58     service.obj
 0001:0000ba64       ??_C@_0BG@KOELEFCN@DeleteSessionBookmark?$AA@ 1000ca64     service.obj
 0001:0000ba7c       ??_C@_0N@EKENACAE@DeleteString?$AA@ 1000ca7c     service.obj
 0001:0000ba8c       ??_C@_06MJDIICIN@Editor?$AA@ 1000ca8c     service.obj
 0001:0000ba94       ??_C@_0L@HDLPOLMA@ExpandTabs?$AA@ 1000ca94     service.obj
 0001:0000baa0       ??_C@_0N@MGAOADJN@GetBookmarks?$AA@ 1000caa0     service.obj
 0001:0000bab0       ??_C@_08JOPFJIPE@GetColor?$AA@ 1000cab0     service.obj
 0001:0000babc       ??_C@_0M@FECPLAMN@GetFileName?$AA@ 1000cabc     service.obj
 0001:0000bac8       ??_C@_07NAJNLNAF@GetInfo?$AA@ 1000cac8     service.obj
 0001:0000bad0       ??_C@_0N@KIILHCLH@GetSelection?$AA@ 1000cad0     service.obj
 0001:0000bae0       ??_C@_0BE@LBJJGOGD@GetSessionBookmarks?$AA@ 1000cae0     service.obj
 0001:0000baf4       ??_C@_09HBLKHMEA@GetString?$AA@ 1000caf4     service.obj
 0001:0000bb00       ??_C@_0L@IDFHDAHP@GetStringW?$AA@ 1000cb00     service.obj
 0001:0000bb0c       ??_C@_0N@ICPGLOEG@InsertString?$AA@ 1000cb0c     service.obj
 0001:0000bb1c       ??_C@_0L@JMOIGJIA@InsertText?$AA@ 1000cb1c     service.obj
 0001:0000bb28       ??_C@_0M@BINOKANK@InsertTextW?$AA@ 1000cb28     service.obj
 0001:0000bb34       ??_C@_0BE@CNGODNDI@NextSessionBookmark?$AA@ 1000cb34     service.obj
 0001:0000bb48       ??_C@_0BE@IEBIGOAP@PrevSessionBookmark?$AA@ 1000cb48     service.obj
 0001:0000bb5c       ??_C@_0N@FNCEPAJJ@ProcessInput?$AA@ 1000cb5c     service.obj
 0001:0000bb6c       ??_C@_04GMBKPCGK@Quit?$AA@ 1000cb6c     service.obj
 0001:0000bb74       ??_C@_09KINLOJJJ@ReadInput?$AA@ 1000cb74     service.obj
 0001:0000bb80       ??_C@_09DBPLBJBJ@RealToTab?$AA@ 1000cb80     service.obj
 0001:0000bb8c       ??_C@_06KAPLBEK@Redraw?$AA@ 1000cb8c     service.obj
 0001:0000bb94       ??_C@_08FBDDPFPJ@SaveFile?$AA@ 1000cb94     service.obj
 0001:0000bba0       ??_C@_06HJGPBJLE@Select?$AA@ 1000cba0     service.obj
 0001:0000bba8       ??_C@_09PPEOOGEC@SetKeyBar?$AA@ 1000cba8     service.obj
 0001:0000bbb4       ??_C@_08CCKJEGOF@SetParam?$AA@ 1000cbb4     service.obj
 0001:0000bbc0       ??_C@_0M@GKIFPNAD@SetPosition?$AA@ 1000cbc0     service.obj
 0001:0000bbcc       ??_C@_09FPPPFNNC@SetString?$AA@ 1000cbcc     service.obj
 0001:0000bbd8       ??_C@_0L@JNHIIHDG@SetStringW?$AA@ 1000cbd8     service.obj
 0001:0000bbe4       ??_C@_08GMCCAJLF@SetTitle?$AA@ 1000cbe4     service.obj
 0001:0000bbf0       ??_C@_08JNAOBKMI@GetTitle?$AA@ 1000cbf0     service.obj
 0001:0000bbfc       ??_C@_0BF@LIMPGNED@SubscribeChangeEvent?$AA@ 1000cbfc     service.obj
 0001:0000bc14       ??_C@_09JFBCONJH@TabToReal?$AA@ 1000cc14     service.obj
 0001:0000bc20       ??_C@_08IBJJAHJG@UndoRedo?$AA@ 1000cc20     service.obj
 0001:0000bc2c       ??_C@_07JMDLHPJF@SetMode?$AA@ 1000cc2c     service.obj
 0001:0000bc34       ??_C@_06PJECNADJ@Viewer?$AA@ 1000cc34     service.obj
 0001:0000bc3c       ??_C@_0BB@PJGDGIKA@CheckPanelsExist?$AA@ 1000cc3c     service.obj
 0001:0000bc50       ??_C@_0P@DFBDDHFA@ClearSelection?$AA@ 1000cc50     service.obj
 0001:0000bc60       ??_C@_0L@KOHCMOPM@GetCmdLine?$AA@ 1000cc60     service.obj
 0001:0000bc6c       ??_C@_0O@NLDIMJEA@GetCmdLinePos?$AA@ 1000cc6c     service.obj
 0001:0000bc7c       ??_C@_0BE@CBPLLCEH@GetCmdLineSelection?$AA@ 1000cc7c     service.obj
 0001:0000bc90       ??_C@_0P@CMFANDFM@GetColumnTypes?$AA@ 1000cc90     service.obj
 0001:0000bca0       ??_C@_0BA@DJGLDCBG@GetColumnWidths?$AA@ 1000cca0     service.obj
 0001:0000bcb0       ??_C@_0BE@JPAIJBCI@GetCurrentPanelItem?$AA@ 1000ccb0     service.obj
 0001:0000bcc4       ??_C@_0BC@NGKPIKGL@GetPanelDirectory?$AA@ 1000ccc4     service.obj
 0001:0000bcd8       ??_C@_0P@GODLFFFJ@GetPanelFormat?$AA@ 1000ccd8     service.obj
 0001:0000bce8       ??_C@_0BB@LCMBHPNI@GetPanelHostFile?$AA@ 1000cce8     service.obj
 0001:0000bcfc       ??_C@_0N@HPIPGDFA@GetPanelInfo?$AA@ 1000ccfc     service.obj
 0001:0000bd0c       ??_C@_0N@HAFLAIHA@GetPanelItem?$AA@ 1000cd0c     service.obj
 0001:0000bd1c       ??_C@_0P@HCBKDPMP@GetPanelPrefix?$AA@ 1000cd1c     service.obj
 0001:0000bd2c       ??_C@_0BF@MEMFMMGB@GetSelectedPanelItem?$AA@ 1000cd2c     service.obj
 0001:0000bd44       ??_C@_0O@HEGDGAJG@GetUserScreen?$AA@ 1000cd44     service.obj
 0001:0000bd54       ??_C@_0O@EHOCCHAL@InsertCmdLine?$AA@ 1000cd54     service.obj
 0001:0000bd64       ??_C@_0O@OMMHIHHH@IsActivePanel?$AA@ 1000cd64     service.obj
 0001:0000bd74       ??_C@_0M@LCEPDNPK@RedrawPanel?$AA@ 1000cd74     service.obj
 0001:0000bd80       ??_C@_0P@OPKJJMLB@SetActivePanel?$AA@ 1000cd80     service.obj
 0001:0000bd90       ??_C@_0BF@LKMKIFPG@SetCaseSensitiveSort?$AA@ 1000cd90     service.obj
 0001:0000bda8       ??_C@_0L@LAFNHJLF@SetCmdLine?$AA@ 1000cda8     service.obj
 0001:0000bdb4       ??_C@_0O@KECGHKDH@SetCmdLinePos?$AA@ 1000cdb4     service.obj
 0001:0000bdc4       ??_C@_0BE@IPNAPCDL@SetCmdLineSelection?$AA@ 1000cdc4     service.obj
 0001:0000bdd8       ??_C@_0BE@PAPEKLCP@SetDirectoriesFirst?$AA@ 1000cdd8     service.obj
 0001:0000bdec       ??_C@_0P@NPNKOENM@SetNumericSort?$AA@ 1000cdec     service.obj
 0001:0000bdfc       ??_C@_0BC@PDKEABHF@SetPanelDirectory?$AA@ 1000cdfc     service.obj
 0001:0000be10       ??_C@_0N@NMDFLOPL@SetSelection?$AA@ 1000ce10     service.obj
 0001:0000be20       ??_C@_0M@CMMMGIDG@SetSortMode?$AA@ 1000ce20     service.obj
 0001:0000be2c       ??_C@_0N@HCHLALN@SetSortOrder?$AA@ 1000ce2c     service.obj
 0001:0000be3c       ??_C@_0O@LHNNDOB@SetUserScreen?$AA@ 1000ce3c     service.obj
 0001:0000be4c       ??_C@_0M@IENJPEBA@SetViewMode?$AA@ 1000ce4c     service.obj
 0001:0000be58       ??_C@_0M@EICBHAOA@UpdatePanel?$AA@ 1000ce58     service.obj
 0001:0000be64       ??_C@_0BC@BIIKJLKB@PluginStartupInfo?$AA@ 1000ce64     service.obj
 0001:0000be78       ??_C@_0L@PJAHNOGM@DialogInit?$AA@ 1000ce78     service.obj
 0001:0000be84       ??_C@_09DBEDLMHB@DialogRun?$AA@ 1000ce84     service.obj
 0001:0000be90       ??_C@_0L@DLFLHLOO@DialogFree?$AA@ 1000ce90     service.obj
 0001:0000be9c       ??_C@_0P@HLOFPDFP@SendDlgMessage?$AA@ 1000ce9c     service.obj
 0001:0000beac       ??_C@_0L@CKELNLCE@GetDlgItem?$AA@ 1000ceac     service.obj
 0001:0000beb8       ??_C@_0L@DEGEGMGN@SetDlgItem?$AA@ 1000ceb8     service.obj
 0001:0000bec4       ??_C@_0BK@EBIPEKDH@SubscribeDialogDrawEvents?$AA@ 1000cec4     service.obj
 0001:0000bee0       ??_C@_0L@MCFABBED@GetDirList?$AA@ 1000cee0     service.obj
 0001:0000beec       ??_C@_06KCCBBIBJ@GetMsg?$AA@ 1000ceec     service.obj
 0001:0000bef4       ??_C@_0BB@HIDBFOJJ@GetPluginDirList?$AA@ 1000cef4     service.obj
 0001:0000bf08       ??_C@_04IFEHPILC@Menu?$AA@ 1000cf08     service.obj
 0001:0000bf10       ??_C@_07BEIHKDLJ@Message?$AA@ 1000cf10     service.obj
 0001:0000bf18       ??_C@_0O@CGLFPNOD@RestoreScreen?$AA@ 1000cf18     service.obj
 0001:0000bf28       ??_C@_0L@PGGGPLFK@SaveScreen?$AA@ 1000cf28     service.obj
 0001:0000bf34       ??_C@_08DAHHHDJC@ShowHelp?$AA@ 1000cf34     service.obj
 0001:0000bf40       ??_C@_08IAADAJIH@InputBox?$AA@ 1000cf40     service.obj
 0001:0000bf4c       ??_C@_0L@HHLOIHOP@AdvControl?$AA@ 1000cf4c     service.obj
 0001:0000bf58       ??_C@_0N@GHGEMEN@MacroLoadAll?$AA@ 1000cf58     service.obj
 0001:0000bf68       ??_C@_0N@NAGBAPAE@MacroSaveAll?$AA@ 1000cf68     service.obj
 0001:0000bf78       ??_C@_0O@KGHDMPAJ@MacroGetState?$AA@ 1000cf78     service.obj
 0001:0000bf88       ??_C@_0N@PNLHCOIE@MacroGetArea?$AA@ 1000cf88     service.obj
 0001:0000bf98       ??_C@_09KGKKBHMO@MacroPost?$AA@ 1000cf98     service.obj
 0001:0000bfa4       ??_C@_0L@KBAKOGFP@MacroCheck?$AA@ 1000cfa4     service.obj
 0001:0000bfb0       ??_C@_08KAFLEHAN@MacroAdd?$AA@ 1000cfb0     service.obj
 0001:0000bfbc       ??_C@_0M@KFMHCNNB@MacroDelete?$AA@ 1000cfbc     service.obj
 0001:0000bfc8       ??_C@_0BC@MJDKBAPF@MacroGetLastError?$AA@ 1000cfc8     service.obj
 0001:0000bfdc       ??_C@_0N@COEPENFH@MacroExecute?$AA@ 1000cfdc     service.obj
 0001:0000bfec       ??_C@_0BB@BICELPOF@CreateFileFilter?$AA@ 1000cfec     service.obj
 0001:0000c000       ??_C@_0L@CHJBHF@LoadPlugin?$AA@ 1000d000     service.obj
 0001:0000c00c       ??_C@_0N@DHIONCLI@UnloadPlugin?$AA@ 1000d00c     service.obj
 0001:0000c01c       ??_C@_0BB@IJHIBGJA@ForcedLoadPlugin?$AA@ 1000d01c     service.obj
 0001:0000c030       ??_C@_0L@DACPHGGH@FindPlugin?$AA@ 1000d030     service.obj
 0001:0000c03c       ??_C@_0BF@KLOGLFMF@GetPluginInformation?$AA@ 1000d03c     service.obj
 0001:0000c054       ??_C@_0L@JIDCIJHM@GetPlugins?$AA@ 1000d054     service.obj
 0001:0000c060       ??_C@_0P@IKAEEPOB@IsPluginLoaded?$AA@ 1000d060     service.obj
 0001:0000c070       ??_C@_0P@HMKEDHIE@CreateSettings?$AA@ 1000d070     service.obj
 0001:0000c080       ??_C@_0N@GOMOBHDB@FreeSettings?$AA@ 1000d080     service.obj
 0001:0000c090       ??_C@_0M@IFKFGKML@ColorDialog?$AA@ 1000d090     service.obj
 0001:0000c09c       ??_C@_0BA@EOCNNPOG@CopyToClipboard?$AA@ 1000d09c     service.obj
 0001:0000c0ac       ??_C@_0BD@PLIHDKFC@PasteFromClipboard?$AA@ 1000d0ac     service.obj
 0001:0000c0c0       ??_C@_0BC@FJDIKOMH@InputRecordToName?$AA@ 1000d0c0     service.obj
 0001:0000c0d4       ??_C@_0BC@FFNOIDFI@NameToInputRecord?$AA@ 1000d0d4     service.obj
 0001:0000c0e8       ??_C@_08HGLFNLMB@LStricmp?$AA@ 1000d0e8     service.obj
 0001:0000c0f4       ??_C@_09GALOFBAC@LStrnicmp?$AA@ 1000d0f4     service.obj
 0001:0000c100       ??_C@_0M@KPPMMAOL@ProcessName?$AA@ 1000d100     service.obj
 0001:0000c10c       ??_C@_0M@KFCNKLDK@GetPathRoot?$AA@ 1000d10c     service.obj
 0001:0000c118       ??_C@_0BE@EPGHGPJC@GetReparsePointInfo?$AA@ 1000d118     service.obj
 0001:0000c12c       ??_C@_08DNJCLFF@LIsAlpha?$AA@ 1000d12c     service.obj
 0001:0000c138       ??_C@_0M@LKJIEECA@LIsAlphanum?$AA@ 1000d138     service.obj
 0001:0000c144       ??_C@_08MAHKICD@LIsLower?$AA@ 1000d144     service.obj
 0001:0000c150       ??_C@_08FHLJMDJK@LIsUpper?$AA@ 1000d150     service.obj
 0001:0000c15c       ??_C@_09LPKAHGM@LLowerBuf?$AA@ 1000d15c     service.obj
 0001:0000c168       ??_C@_09GLKFOOEP@LUpperBuf?$AA@ 1000d168     service.obj
 0001:0000c174       ??_C@_06ILCHIEBO@MkTemp?$AA@ 1000d174     service.obj
 0001:0000c17c       ??_C@_06DKBBJCCG@MkLink?$AA@ 1000d17c     service.obj
 0001:0000c184       ??_C@_0N@CCDDAJK@TruncPathStr?$AA@ 1000d184     service.obj
 0001:0000c194       ??_C@_08BNEIIKEJ@TruncStr?$AA@ 1000d194     service.obj
 0001:0000c1a0       ??_C@_0BA@CLEHBIPM@RecursiveSearch?$AA@ 1000d1a0     service.obj
 0001:0000c1b0       ??_C@_0M@HKHGOOHG@ConvertPath?$AA@ 1000d1b0     service.obj
 0001:0000c1bc       ??_C@_04OCDKHGII@XLat?$AA@ 1000d1bc     service.obj
 0001:0000c1c4       ??_C@_0P@BGLLKGOI@FormatFileSize?$AA@ 1000d1c4     service.obj
 0001:0000c1d4       ??_C@_08KJBLDCDF@FarClock?$AA@ 1000d1d4     service.obj
 0001:0000c1e0       ??_C@_0BD@ELMHPHAC@CPluginStartupInfo?$AA@ 1000d1e0     service.obj
 0001:0000c1f4       ??_C@_0BE@DJLJEKBK@GetCurrentDirectory?$AA@ 1000d1f4     service.obj
 0001:0000c208       ??_C@_0N@MOMBJEKA@GetFileOwner?$AA@ 1000d208     service.obj
 0001:0000c218       ??_C@_0BB@JBNBALEM@GetNumberOfLinks?$AA@ 1000d218     service.obj
 0001:0000c22c       ??_C@_0O@BJEAJNBH@MakeMenuItems?$AA@ 1000d22c     service.obj
 0001:0000c23c       ??_C@_04JLAJABDJ@Show?$AA@ 1000d23c     service.obj
 0001:0000c244       ??_C@_05NHFJDMOA@Timer?$AA@ 1000d244     service.obj
 0001:0000c24c       ??_C@_02KFNNKBCK@io?$AA@   1000d24c     service.obj
 0001:0000c250       ??_C@_02EHCHIAMF@os?$AA@   1000d250     service.obj
 0001:0000c254       ??_C@_04CFDJAKFL@math?$AA@ 1000d254     service.obj
 0001:0000c25c       ??_C@_07GAJMMAJO@unicode?$AA@ 1000d25c     service.obj
 0001:0000c264       ??_C@_03JECLAOEA@win?$AA@  1000d264     service.obj
 0001:0000c268       ??_C@_03EDMBFDDG@bit?$AA@  1000d268     service.obj
 0001:0000c26c       ??_C@_03DIJDOPEA@ffi?$AA@  1000d26c     service.obj
 0001:0000c270       ??_C@_03IGHFHLNJ@jit?$AA@  1000d270     service.obj
 0001:0000c274       ??_C@_07PHPIFDKI@LBUTTON?$AA@ 1000d274     service.obj
 0001:0000c27c       ??_C@_07JOMJHALB@RBUTTON?$AA@ 1000d27c     service.obj
 0001:0000c284       ??_C@_06JHILMIHF@CANCEL?$AA@ 1000d284     service.obj
 0001:0000c28c       ??_C@_07DLFCFDDG@MBUTTON?$AA@ 1000d28c     service.obj
 0001:0000c294       ??_C@_08OPILMHEG@XBUTTON1?$AA@ 1000d294     service.obj
 0001:0000c2a0       ??_C@_08MEKGJEIF@XBUTTON2?$AA@ 1000d2a0     service.obj
 0001:0000c2ac       ??_C@_04FJBHJJME@BACK?$AA@ 1000d2ac     service.obj
 0001:0000c2b4       ??_C@_03CJMDHCGG@TAB?$AA@  1000d2b4     service.obj
 0001:0000c2b8       ??_C@_05PONODPI@CLEAR?$AA@ 1000d2b8     service.obj
 0001:0000c2c0       ??_C@_06LJMOENAO@RETURN?$AA@ 1000d2c0     service.obj
 0001:0000c2c8       ??_C@_05OAHIEJBI@SHIFT?$AA@ 1000d2c8     service.obj
 0001:0000c2d0       ??_C@_07DBEDOPMC@CONTROL?$AA@ 1000d2d0     service.obj
 0001:0000c2d8       ??_C@_04IILMDFMO@MENU?$AA@ 1000d2d8     service.obj
 0001:0000c2e0       ??_C@_05DIAHPDGL@PAUSE?$AA@ 1000d2e0     service.obj
 0001:0000c2e8       ??_C@_07OPCFNGJB@CAPITAL?$AA@ 1000d2e8     service.obj
 0001:0000c2f0       ??_C@_04KGDAIAGM@KANA?$AA@ 1000d2f0     service.obj
 0001:0000c2f8       ??_C@_05PPKJGOLB@JUNJA?$AA@ 1000d2f8     service.obj
 0001:0000c300       ??_C@_05JEIAEFOF@FINAL?$AA@ 1000d300     service.obj
 0001:0000c308       ??_C@_05CHABPOPI@HANJA?$AA@ 1000d308     service.obj
 0001:0000c310       ??_C@_06CDPDIIDH@ESCAPE?$AA@ 1000d310     service.obj
 0001:0000c318       ??_C@_0L@ODNCKDCK@NONCONVERT?$AA@ 1000d318     service.obj
 0001:0000c324       ??_C@_06INBBKPI@ACCEPT?$AA@ 1000d324     service.obj
 0001:0000c32c       ??_C@_0L@HEHNEBED@MODECHANGE?$AA@ 1000d32c     service.obj
 0001:0000c338       ??_C@_05CAEOFMEP@SPACE?$AA@ 1000d338     service.obj
 0001:0000c340       ??_C@_05BFDHCIJM@PRIOR?$AA@ 1000d340     service.obj
 0001:0000c348       ??_C@_04MOKMKBJN@NEXT?$AA@ 1000d348     service.obj
 0001:0000c350       ??_C@_03JMGAKCCH@END?$AA@  1000d350     service.obj
 0001:0000c354       ??_C@_04GHGFPGNC@HOME?$AA@ 1000d354     service.obj
 0001:0000c35c       ??_C@_04KCNEHMIH@LEFT?$AA@ 1000d35c     service.obj
 0001:0000c364       ??_C@_02NAHCJHOC@UP?$AA@   1000d364     service.obj
 0001:0000c368       ??_C@_05PMAFOJDE@RIGHT?$AA@ 1000d368     service.obj
 0001:0000c370       ??_C@_04FANAOELO@DOWN?$AA@ 1000d370     service.obj
 0001:0000c378       ??_C@_06LCPJPOPK@SELECT?$AA@ 1000d378     service.obj
 0001:0000c380       ??_C@_05ECKPOFCN@PRINT?$AA@ 1000d380     service.obj
 0001:0000c388       ??_C@_07LBDEDADF@EXECUTE?$AA@ 1000d388     service.obj
 0001:0000c390       ??_C@_08EMOKHGD@SNAPSHOT?$AA@ 1000d390     service.obj
 0001:0000c39c       ??_C@_06OEMEAEKN@INSERT?$AA@ 1000d39c     service.obj
 0001:0000c3a4       ??_C@_06FKDAMKFP@DELETE?$AA@ 1000d3a4     service.obj
 0001:0000c3ac       ??_C@_04DOKPJKJF@HELP?$AA@ 1000d3ac     service.obj
 0001:0000c3b4       ??_C@_01GBGANLPD@0?$AA@    1000d3b4     service.obj
 0001:0000c3b8       ??_C@_01HIHLOKLC@1?$AA@    1000d3b8     service.obj
 0001:0000c3bc       ??_C@_01FDFGLJHB@2?$AA@    1000d3bc     service.obj
 0001:0000c3c0       ??_C@_01EKENIIDA@3?$AA@    1000d3c0     service.obj
 0001:0000c3c4       ??_C@_01FAMBOPH@4?$AA@     1000d3c4     service.obj
 0001:0000c3c8       ??_C@_01BMBHCPLG@5?$AA@    1000d3c8     service.obj
 0001:0000c3cc       ??_C@_01DHDKHMHF@6?$AA@    1000d3cc     service.obj
 0001:0000c3d0       ??_C@_01COCBENDE@7?$AA@    1000d3d0     service.obj
 0001:0000c3d4       ??_C@_01KJLJFBPL@8?$AA@    1000d3d4     service.obj
 0001:0000c3d8       ??_C@_01LAKCGALK@9?$AA@    1000d3d8     service.obj
 0001:0000c3dc       ??_C@_01FHEEJDEE@A?$AA@    1000d3dc     service.obj
 0001:0000c3e0       ??_C@_01HMGJMAIH@B?$AA@    1000d3e0     service.obj
 0001:0000c3e4       ??_C@_01GFHCPBMG@C?$AA@    1000d3e4     service.obj
 0001:0000c3e8       ??_C@_01CKDDGHAB@D?$AA@    1000d3e8     service.obj
 0001:0000c3ec       ??_C@_01DDCIFGEA@E?$AA@    1000d3ec     service.obj
 0001:0000c3f0       ??_C@_01BIAFAFID@F?$AA@    1000d3f0     service.obj
 0001:0000c3f4       ??_C@_01BBODEMC@G?$AA@     1000d3f4     service.obj
 0001:0000c3f8       ??_C@_01IGIGCIAN@H?$AA@    1000d3f8     service.obj
 0001:0000c3fc       ??_C@_01JPJNBJEM@I?$AA@    1000d3fc     service.obj
 0001:0000c400       ??_C@_01LELAEKIP@J?$AA@    1000d400     service.obj
 0001:0000c404       ??_C@_01KNKLHLMO@K?$AA@    1000d404     service.obj
 0001:0000c408       ??_C@_01OCOKONAJ@L?$AA@    1000d408     service.obj
 0001:0000c40c       ??_C@_01PLPBNMEI@M?$AA@    1000d40c     service.obj
 0001:0000c410       ??_C@_01NANMIPIL@N?$AA@    1000d410     service.obj
 0001:0000c414       ??_C@_01MJMHLOMK@O?$AA@    1000d414     service.obj
 0001:0000c418       ??_C@_01EJNLAFE@P?$AA@     1000d418     service.obj
 0001:0000c41c       ??_C@_01BNIGIBBF@Q?$AA@    1000d41c     service.obj
 0001:0000c420       ??_C@_01DGKLNCNG@R?$AA@    1000d420     service.obj
 0001:0000c424       ??_C@_01CPLAODJH@S?$AA@    1000d424     service.obj
 0001:0000c428       ??_C@_01GAPBHFFA@T?$AA@    1000d428     service.obj
 0001:0000c42c       ??_C@_01HJOKEEBB@U?$AA@    1000d42c     service.obj
 0001:0000c430       ??_C@_01FCMHBHNC@V?$AA@    1000d430     service.obj
 0001:0000c434       ??_C@_01ELNMCGJD@W?$AA@    1000d434     service.obj
 0001:0000c438       ??_C@_01MMEEDKFM@X?$AA@    1000d438     service.obj
 0001:0000c43c       ??_C@_01NFFPALBN@Y?$AA@    1000d43c     service.obj
 0001:0000c440       ??_C@_01POHCFINO@Z?$AA@    1000d440     service.obj
 0001:0000c444       ??_C@_04ODLFFOHF@LWIN?$AA@ 1000d444     service.obj
 0001:0000c44c       ??_C@_04DMGFHHJG@RWIN?$AA@ 1000d44c     service.obj
 0001:0000c454       ??_C@_04GKGJFGJO@APPS?$AA@ 1000d454     service.obj
 0001:0000c45c       ??_C@_05DJAECLDN@SLEEP?$AA@ 1000d45c     service.obj
 0001:0000c464       ??_C@_07NHIPMMJH@NUMPAD0?$AA@ 1000d464     service.obj
 0001:0000c46c       ??_C@_07MOJEPNNG@NUMPAD1?$AA@ 1000d46c     service.obj
 0001:0000c474       ??_C@_07OFLJKOBF@NUMPAD2?$AA@ 1000d474     service.obj
 0001:0000c47c       ??_C@_07PMKCJPFE@NUMPAD3?$AA@ 1000d47c     service.obj
 0001:0000c484       ??_C@_07LDODAJJD@NUMPAD4?$AA@ 1000d484     service.obj
 0001:0000c48c       ??_C@_07KKPIDINC@NUMPAD5?$AA@ 1000d48c     service.obj
 0001:0000c494       ??_C@_07IBNFGLBB@NUMPAD6?$AA@ 1000d494     service.obj
 0001:0000c49c       ??_C@_07JIMOFKFA@NUMPAD7?$AA@ 1000d49c     service.obj
 0001:0000c4a4       ??_C@_07BPFGEGJP@NUMPAD8?$AA@ 1000d4a4     service.obj
 0001:0000c4ac       ??_C@_07GENHHNO@NUMPAD9?$AA@ 1000d4ac     service.obj
 0001:0000c4b4       ??_C@_08LDEOAAGM@MULTIPLY?$AA@ 1000d4b4     service.obj
 0001:0000c4c0       ??_C@_03BOJFLAKG@ADD?$AA@  1000d4c0     service.obj
 0001:0000c4c4       ??_C@_09POPINEFK@SEPARATOR?$AA@ 1000d4c4     service.obj
 0001:0000c4d0       ??_C@_08MGBEENML@SUBTRACT?$AA@ 1000d4d0     service.obj
 0001:0000c4dc       ??_C@_07LJPMJDLL@DECIMAL?$AA@ 1000d4dc     service.obj
 0001:0000c4e4       ??_C@_06FBFCJJMP@DIVIDE?$AA@ 1000d4e4     service.obj
 0001:0000c4ec       ??_C@_02LCPENACN@F1?$AA@   1000d4ec     service.obj
 0001:0000c4f0       ??_C@_02JJNJIDOO@F2?$AA@   1000d4f0     service.obj
 0001:0000c4f4       ??_C@_02IAMCLCKP@F3?$AA@   1000d4f4     service.obj
 0001:0000c4f8       ??_C@_02MPIDCEGI@F4?$AA@   1000d4f8     service.obj
 0001:0000c4fc       ??_C@_02NGJIBFCJ@F5?$AA@   1000d4fc     service.obj
 0001:0000c500       ??_C@_02PNLFEGOK@F6?$AA@   1000d500     service.obj
 0001:0000c504       ??_C@_02OEKOHHKL@F7?$AA@   1000d504     service.obj
 0001:0000c508       ??_C@_02GDDGGLGE@F8?$AA@   1000d508     service.obj
 0001:0000c50c       ??_C@_02HKCNFKCF@F9?$AA@   1000d50c     service.obj
 0001:0000c510       ??_C@_03JKCLJOFG@F10?$AA@  1000d510     service.obj
 0001:0000c514       ??_C@_03IDDAKPBH@F11?$AA@  1000d514     service.obj
 0001:0000c518       ??_C@_03KIBNPMNE@F12?$AA@  1000d518     service.obj
 0001:0000c51c       ??_C@_03LBAGMNJF@F13?$AA@  1000d51c     service.obj
 0001:0000c520       ??_C@_03POEHFLFC@F14?$AA@  1000d520     service.obj
 0001:0000c524       ??_C@_03OHFMGKBD@F15?$AA@  1000d524     service.obj
 0001:0000c528       ??_C@_03MMHBDJNA@F16?$AA@  1000d528     service.obj
 0001:0000c52c       ??_C@_03NFGKAIJB@F17?$AA@  1000d52c     service.obj
 0001:0000c530       ??_C@_03FCPCBEFO@F18?$AA@  1000d530     service.obj
 0001:0000c534       ??_C@_03ELOJCFBP@F19?$AA@  1000d534     service.obj
 0001:0000c538       ??_C@_03JIGNCAAP@F20?$AA@  1000d538     service.obj
 0001:0000c53c       ??_C@_03IBHGBBEO@F21?$AA@  1000d53c     service.obj
 0001:0000c540       ??_C@_03KKFLECIN@F22?$AA@  1000d540     service.obj
 0001:0000c544       ??_C@_03LDEAHDMM@F23?$AA@  1000d544     service.obj
 0001:0000c548       ??_C@_03PMABOFAL@F24?$AA@  1000d548     service.obj
 0001:0000c54c       ??_C@_07FLMEHHJP@NUMLOCK?$AA@ 1000d54c     service.obj
 0001:0000c554       ??_C@_06FNIKALAE@SCROLL?$AA@ 1000d554     service.obj
 0001:0000c55c       ??_C@_0O@DBBJDALK@OEM_NEC_EQUAL?$AA@ 1000d55c     service.obj
 0001:0000c56c       ??_C@_0P@JKGCFGCD@OEM_FJ_MASSHOU?$AA@ 1000d56c     service.obj
 0001:0000c57c       ??_C@_0P@NIEOFNLG@OEM_FJ_TOUROKU?$AA@ 1000d57c     service.obj
 0001:0000c58c       ??_C@_0M@IBEHGLCM@OEM_FJ_LOYA?$AA@ 1000d58c     service.obj
 0001:0000c598       ??_C@_0M@FOJHECMP@OEM_FJ_ROYA?$AA@ 1000d598     service.obj
 0001:0000c5a4       ??_C@_06EPHNCIMI@LSHIFT?$AA@ 1000d5a4     service.obj
 0001:0000c5ac       ??_C@_06HIJMMPFL@RSHIFT?$AA@ 1000d5ac     service.obj
 0001:0000c5b4       ??_C@_08IKMONEBG@LCONTROL?$AA@ 1000d5b4     service.obj
 0001:0000c5c0       ??_C@_08OOMMENPF@RCONTROL?$AA@ 1000d5c0     service.obj
 0001:0000c5cc       ??_C@_05IHMGKJGH@LMENU?$AA@ 1000d5cc     service.obj
 0001:0000c5d4       ??_C@_05LOBKMKIM@RMENU?$AA@ 1000d5d4     service.obj
 0001:0000c5dc       ??_C@_0N@OAJIELLG@BROWSER_BACK?$AA@ 1000d5dc     service.obj
 0001:0000c5ec       ??_C@_0BA@ENOAJOGH@BROWSER_FORWARD?$AA@ 1000d5ec     service.obj
 0001:0000c5fc       ??_C@_0BA@GDNDIDGJ@BROWSER_REFRESH?$AA@ 1000d5fc     service.obj
 0001:0000c60c       ??_C@_0N@HKPDGANH@BROWSER_STOP?$AA@ 1000d60c     service.obj
 0001:0000c61c       ??_C@_0P@BEAEBJDD@BROWSER_SEARCH?$AA@ 1000d61c     service.obj
 0001:0000c62c       ??_C@_0BC@BOMJIH@BROWSER_FAVORITES?$AA@ 1000d62c     service.obj
 0001:0000c640       ??_C@_0N@NOOKCEKA@BROWSER_HOME?$AA@ 1000d640     service.obj
 0001:0000c650       ??_C@_0M@ENOHKBMG@VOLUME_MUTE?$AA@ 1000d650     service.obj
 0001:0000c65c       ??_C@_0M@JOOBBDNO@VOLUME_DOWN?$AA@ 1000d65c     service.obj
 0001:0000c668       ??_C@_09MGPMNMJC@VOLUME_UP?$AA@ 1000d668     service.obj
 0001:0000c674       ??_C@_0BB@KLAENPA@MEDIA_NEXT_TRACK?$AA@ 1000d674     service.obj
 0001:0000c688       ??_C@_0BB@CMOIJKPH@MEDIA_PREV_TRACK?$AA@ 1000d688     service.obj
 0001:0000c69c       ??_C@_0L@KBJOCDHK@MEDIA_STOP?$AA@ 1000d69c     service.obj
 0001:0000c6a8       ??_C@_0BB@HAEMIJHO@MEDIA_PLAY_PAUSE?$AA@ 1000d6a8     service.obj
 0001:0000c6bc       ??_C@_0M@GCIKMBID@LAUNCH_MAIL?$AA@ 1000d6bc     service.obj
 0001:0000c6c8       ??_C@_0BE@FADJJAPM@LAUNCH_MEDIA_SELECT?$AA@ 1000d6c8     service.obj
 0001:0000c6dc       ??_C@_0M@MGLJIDDM@LAUNCH_APP1?$AA@ 1000d6dc     service.obj
 0001:0000c6e8       ??_C@_0M@ONJENAPP@LAUNCH_APP2?$AA@ 1000d6e8     service.obj
 0001:0000c6f4       ??_C@_05OIODNPAD@OEM_1?$AA@ 1000d6f4     service.obj
 0001:0000c6fc       ??_C@_08LDJEIPBH@OEM_PLUS?$AA@ 1000d6fc     service.obj
 0001:0000c708       ??_C@_09CLPFJEOD@OEM_COMMA?$AA@ 1000d708     service.obj
 0001:0000c714       ??_C@_09OGMLCNMG@OEM_MINUS?$AA@ 1000d714     service.obj
 0001:0000c720       ??_C@_0L@DNNMNDGM@OEM_PERIOD?$AA@ 1000d720     service.obj
 0001:0000c72c       ??_C@_05MDMOIMMA@OEM_2?$AA@ 1000d72c     service.obj
 0001:0000c734       ??_C@_05NKNFLNIB@OEM_3?$AA@ 1000d734     service.obj
 0001:0000c73c       ??_C@_05JFJECLEG@OEM_4?$AA@ 1000d73c     service.obj
 0001:0000c744       ??_C@_05IMIPBKAH@OEM_5?$AA@ 1000d744     service.obj
 0001:0000c74c       ??_C@_05KHKCEJME@OEM_6?$AA@ 1000d74c     service.obj
 0001:0000c754       ??_C@_05LOLJHIIF@OEM_7?$AA@ 1000d754     service.obj
 0001:0000c75c       ??_C@_05DJCBGEEK@OEM_8?$AA@ 1000d75c     service.obj
 0001:0000c764       ??_C@_07PEFKMFIE@OEM_102?$AA@ 1000d764     service.obj
 0001:0000c76c       ??_C@_0L@EFLJCPAM@PROCESSKEY?$AA@ 1000d76c     service.obj
 0001:0000c778       ??_C@_06HOICDKCB@PACKET?$AA@ 1000d778     service.obj
 0001:0000c780       ??_C@_09CAKPMKHM@OEM_RESET?$AA@ 1000d780     service.obj
 0001:0000c78c       ??_C@_08INMNLJCK@OEM_JUMP?$AA@ 1000d78c     service.obj
 0001:0000c798       ??_C@_07JNOAEEG@OEM_PA1?$AA@ 1000d798     service.obj
 0001:0000c7a0       ??_C@_07CCPDFHIF@OEM_PA2?$AA@ 1000d7a0     service.obj
 0001:0000c7a8       ??_C@_07DLOIGGME@OEM_PA3?$AA@ 1000d7a8     service.obj
 0001:0000c7b0       ??_C@_0L@OCAIHDP@OEM_WSCTRL?$AA@ 1000d7b0     service.obj
 0001:0000c7bc       ??_C@_04BNGOAFAJ@ATTN?$AA@ 1000d7bc     service.obj
 0001:0000c7c4       ??_C@_05HGAHFFFL@CRSEL?$AA@ 1000d7c4     service.obj
 0001:0000c7cc       ??_C@_05OKOOKOOH@EXSEL?$AA@ 1000d7cc     service.obj
 0001:0000c7d4       ??_C@_05CCFENDFJ@EREOF?$AA@ 1000d7d4     service.obj
 0001:0000c7dc       ??_C@_04MKCNCBEG@PLAY?$AA@ 1000d7dc     service.obj
 0001:0000c7e4       ??_C@_04LGBIGMFG@ZOOM?$AA@ 1000d7e4     service.obj
 0001:0000c7ec       ??_C@_06LJIOOKLP@NONAME?$AA@ 1000d7ec     service.obj
 0001:0000c7f4       ??_C@_03KCLDMPAE@PA1?$AA@  1000d7f4     service.obj
 0001:0000c7f8       ??_C@_09MBBEHOCK@OEM_CLEAR?$AA@ 1000d7f8     service.obj
 0001:0000c804       ??_C@_05LCLENNFI@table?$AA@ 1000d804     service.obj
 0001:0000c80c       ??_C@_06ICGJLFIM@string?$AA@ 1000d80c     service.obj
 0001:0000c814       ??_C@_09GJGOMOL@lua51?4dll?$AA@ 1000d814     service.obj
 0001:0000c820       ??_C@_0M@PLOBHAKE@luaopen_bit?$AA@ 1000d820     service.obj
 0001:0000c82c       ??_C@_0M@IALDMMNC@luaopen_ffi?$AA@ 1000d82c     service.obj
 0001:0000c838       ??_C@_0M@DOFFFIEL@luaopen_jit?$AA@ 1000d838     service.obj
 0001:0000c844       ??_C@_0BE@OEPKKAAB@integer?5or?5userdata?$AA@ 1000d844     service.obj
 0001:0000c858       ??_C@_0BD@PNJHLBDA@invalid?5flag?3?5?$CC?$CFs?$CC?$AA@ 1000d858     service.obj
 0001:0000c86c       ??_C@_0N@JJLBBDOC@invalid?5flag?$AA@ 1000d86c     service.obj
 0001:0000c87c       ??_C@_0BJ@MIKGPOKL@invalid?5flag?5combination?$AA@ 1000d87c     service.obj
 0001:0000c898       ??_C@_0P@EANMLDOP@MousePositionX?$AA@ 1000d898     service.obj
 0001:0000c8a8       ??_C@_0P@FJMHICKO@MousePositionY?$AA@ 1000d8a8     service.obj
 0001:0000c8b8       ??_C@_0M@BJAICPIE@ButtonState?$AA@ 1000d8b8     service.obj
 0001:0000c8c4       ??_C@_0L@EMFBJIPA@EventFlags?$AA@ 1000d8c4     service.obj
 0001:0000c8d0       ??_C@_07EEJLMCNH@CurLine?$AA@ 1000d8d0     service.obj
 0001:0000c8d8       ??_C@_06EDBJMJDC@CurPos?$AA@ 1000d8d8     service.obj
 0001:0000c8e0       ??_C@_09EGONKHKB@CurTabPos?$AA@ 1000d8e0     service.obj
 0001:0000c8ec       ??_C@_0O@OKGGHEJK@TopScreenLine?$AA@ 1000d8ec     service.obj
 0001:0000c8fc       ??_C@_07GDAKJHLE@LeftPos?$AA@ 1000d8fc     service.obj
 0001:0000c904       ??_C@_08LLJICOLD@Overtype?$AA@ 1000d904     service.obj
 0001:0000c910       ??_C@_0L@GEIEADPN@ModuleName?$AA@ 1000d910     service.obj
 0001:0000c91c       ??_C@_09HOIHBHIM@ModuleDir?$AA@ 1000d91c     service.obj
 0001:0000c928       ??_C@_0L@JLHCLFBG@PluginGuid?$AA@ 1000d928     service.obj
 0001:0000c934       ??_C@_08GGMFPBHM@EditorID?$AA@ 1000d934     service.obj
 0001:0000c940       ??_C@_0M@CPDBGLHN@WindowSizeX?$AA@ 1000d940     service.obj
 0001:0000c94c       ??_C@_0M@DGCKFKDM@WindowSizeY?$AA@ 1000d94c     service.obj
 0001:0000c958       ??_C@_0L@PMKENHMA@TotalLines?$AA@ 1000d958     service.obj
 0001:0000c964       ??_C@_09HKBEFIPN@BlockType?$AA@ 1000d964     service.obj
 0001:0000c970       ??_C@_0P@GAEEHNHE@BlockStartLine?$AA@ 1000d970     service.obj
 0001:0000c980       ??_C@_07KHIHFBFN@Options?$AA@ 1000d980     service.obj
 0001:0000c988       ??_C@_07FLDNELFM@TabSize?$AA@ 1000d988     service.obj
 0001:0000c990       ??_C@_0O@EBLDFOPH@BookmarkCount?$AA@ 1000d990     service.obj
 0001:0000c9a0       ??_C@_0BF@ODFKBFAK@SessionBookmarkCount?$AA@ 1000d9a0     service.obj
 0001:0000c9b8       ??_C@_08CPAOHJDL@CurState?$AA@ 1000d9b8     service.obj
 0001:0000c9c4       ??_C@_0N@DAJMJAE@StringLength?$AA@ 1000d9c4     service.obj
 0001:0000c9d4       ??_C@_08JPMALCFA@SelStart?$AA@ 1000d9d4     service.obj
 0001:0000c9e0       ??_C@_06JLEHDHII@SelEnd?$AA@ 1000d9e0     service.obj
 0001:0000c9e8       ??_C@_0L@IFNFGDGN@StringText?$AA@ 1000d9e8     service.obj
 0001:0000c9f4       ??_C@_09IBGOAAEM@StringEOL?$AA@ 1000d9f4     service.obj
 0001:0000ca00       ??_C@_01LOCGONAA@?$AA?$AA@ 1000da00     service.obj
 0001:0000ca04       ??_C@_06MFLCIING@redraw?$AA@ 1000da04     service.obj
 0001:0000ca0c       ??_C@_07HICINA@restore?$AA@ 1000da0c     service.obj
 0001:0000ca14       ??_C@_0CG@LAKEGANL@must?5be?5?8redraw?8?0?5?8restore?8?0?5or?5@ 1000da14     service.obj
 0001:0000ca3c       ??_C@_04LIDDHMOL@Line?$AA@ 1000da3c     service.obj
 0001:0000ca44       ??_C@_06OIIFPIKD@Cursor?$AA@ 1000da44     service.obj
 0001:0000ca4c       ??_C@_0L@GDDEHGKI@ScreenLine?$AA@ 1000da4c     service.obj
 0001:0000ca58       ??_C@_0O@CIAFMMMB@BlockStartPos?$AA@ 1000da58     service.obj
 0001:0000ca68       ??_C@_0L@EKLJJHPF@BlockWidth?$AA@ 1000da68     service.obj
 0001:0000ca74       ??_C@_0M@NKKGBDGK@BlockHeight?$AA@ 1000da74     service.obj
 0001:0000ca80       ??_C@_09JFPCGCOC@StartLine?$AA@ 1000da80     service.obj
 0001:0000ca8c       ??_C@_08JBNOANJG@StartPos?$AA@ 1000da8c     service.obj
 0001:0000ca98       ??_C@_07DCKCOCOC@EndLine?$AA@ 1000da98     service.obj
 0001:0000caa0       ??_C@_06KGHIGMHC@EndPos?$AA@ 1000daa0     service.obj
 0001:0000caa8       ??_C@_0BA@HNIJJEO@ForegroundColor?$AA@ 1000daa8     service.obj
 0001:0000cab8       ??_C@_0BA@DPMBBMBG@BackgroundColor?$AA@ 1000dab8     service.obj
 0001:0000cac8       ??_C@_0O@NHKEGDJF@GUID?5required?$AA@ 1000dac8     service.obj
 0001:0000cad8       ??_C@_0BJ@BMOGHFAN@table?5or?5number?5expected?$AA@ 1000dad8     service.obj
 0001:0000caf4       ??_C@_08KGEIBGG@Priority?$AA@ 1000daf4     service.obj
 0001:0000cb00       ??_C@_05PDOBBJNA@Color?$AA@ 1000db00     service.obj
 0001:0000cb08       ??_C@_09KDLBEGCN@EventType?$AA@ 1000db08     service.obj
 0001:0000cb14       ??_C@_07HPHPOAEG@KeyDown?$AA@ 1000db14     service.obj
 0001:0000cb1c       ??_C@_0M@FGGHEADP@RepeatCount?$AA@ 1000db1c     service.obj
 0001:0000cb28       ??_C@_0BA@KCCLHPM@VirtualScanCode?$AA@ 1000db28     service.obj
 0001:0000cb38       ??_C@_0M@PBJKDIHH@UnicodeChar?$AA@ 1000db38     service.obj
 0001:0000cb44       ??_C@_05GIPJKPFG@SizeX?$AA@ 1000db44     service.obj
 0001:0000cb4c       ??_C@_05HBOCJOBH@SizeY?$AA@ 1000db4c     service.obj
 0001:0000cb54       ??_C@_09GEJJJAHL@CommandId?$AA@ 1000db54     service.obj
 0001:0000cb60       ??_C@_08GPNNBNIL@SetFocus?$AA@ 1000db60     service.obj
 0001:0000cb6c       ??_C@_0M@BEDENHPD@invalid?5key?$AA@ 1000db6c     service.obj
 0001:0000cb78       ??_C@_19IBCFILMC@?$AAM?$AAe?$AAn?$AAu?$AA?$AA@ 1000db78     service.obj
 0001:0000cb84       ??_C@_0BN@JBAMKCCJ@must?5be?5table?0?5string?5or?5nil?$AA@ 1000db84     service.obj
 0001:0000cba4       ??_C@_09FDAFFNEA@MaxHeight?$AA@ 1000dba4     service.obj
 0001:0000cbb0       ??_C@_06DDHCBBGN@Bottom?$AA@ 1000dbb0     service.obj
 0001:0000cbb8       ??_C@_09CFELDMD@HelpTopic?$AA@ 1000dbb8     service.obj
 0001:0000cbc4       ??_C@_0M@GGMLPAIK@SelectIndex?$AA@ 1000dbc4     service.obj
 0001:0000cbd0       ??_C@_02HOGEDOAB@Id?$AA@   1000dbd0     service.obj
 0001:0000cbd4       ??_C@_07FJOBMBFC@checked?$AA@ 1000dbd4     service.obj
 0001:0000cbdc       ??_C@_09MOAJOJKN@separator?$AA@ 1000dbdc     service.obj
 0001:0000cbe8       ??_C@_07DBNODEFN@disable?$AA@ 1000dbe8     service.obj
 0001:0000cbf0       ??_C@_06JHIAOIKD@grayed?$AA@ 1000dbf0     service.obj
 0001:0000cbf8       ??_C@_06JIKFICKK@hidden?$AA@ 1000dbf8     service.obj
 0001:0000cc00       ??_C@_08CJLOJPNI@selected?$AA@ 1000dc00     service.obj
 0001:0000cc0c       ??_C@_08MMCKBNNI@AccelKey?$AA@ 1000dc0c     service.obj
 0001:0000cc18       ??_C@_08PNHLLJE@BreakKey?$AA@ 1000dc18     service.obj
 0001:0000cc24       ??_C@_15FMBEJGOH@?$AAO?$AAk?$AA?$AA@ 1000dc24     service.obj
 0001:0000cc2c       ??_C@_1BC@IBCAPFAE@?$AAO?$AAk?$AAC?$AAa?$AAn?$AAc?$AAe?$AAl?$AA?$AA@ 1000dc2c     service.obj
 0001:0000cc40       ??_C@_1CC@HODOHOHB@?$AAA?$AAb?$AAo?$AAr?$AAt?$AAR?$AAe?$AAt?$AAr?$AAy?$AAI?$AAg?$AAn?$AAo?$AAr?$AAe?$AA?$AA@ 1000dc40     service.obj
 0001:0000cc64       ??_C@_1M@GGPOIMAD@?$AAY?$AAe?$AAs?$AAN?$AAo?$AA?$AA@ 1000dc64     service.obj
 0001:0000cc70       ??_C@_1BI@BNDFIGCI@?$AAY?$AAe?$AAs?$AAN?$AAo?$AAC?$AAa?$AAn?$AAc?$AAe?$AAl?$AA?$AA@ 1000dc70     service.obj
 0001:0000cc88       ??_C@_1BI@KMMIHPHF@?$AAR?$AAe?$AAt?$AAr?$AAy?$AAC?$AAa?$AAn?$AAc?$AAe?$AAl?$AA?$AA@ 1000dc88     service.obj
 0001:0000cca0       ??_C@_1DG@LMKDDADI@?$AA?$DM?$AAn?$AAo?$AAn?$AA?9?$AAs?$AAt?$AAr?$AAi?$AAn?$AAg?$AA?5?$AAe?$AAr?$AAr?$AAo?$AAr?$AA?5?$AAm?$AAe?$AAs?$AAs?$AAa?$AAg?$AAe?$AA?$DO?$AA?$AA@ 1000dca0     service.obj
 0001:0000ccd8       ??_C@_15IEGBJKPD@?$AA?3?$AA?6?$AA?$AA@ 1000dcd8     service.obj
 0001:0000cce0       ??_C@_19FFLPMPBO@?$AA?6?$AA?5?$AA?5?$AA?5?$AA?$AA@ 1000dce0     service.obj
 0001:0000ccec       ??_C@_15JCKODCLA@?$AA?6?$AA?7?$AA?$AA@ 1000dcec     service.obj
 0001:0000ccf4       ??_C@_1M@ILHOPKA@?$AAE?$AAr?$AAr?$AAo?$AAr?$AA?$AA@ 1000dcf4     service.obj
 0001:0000cd00       ??_C@_08FNIIFOJC@tostring?$AA@ 1000dd00     service.obj
 0001:0000cd0c       ??_C@_0BJ@JOELOGM@cannot?5convert?5to?5string?$AA@ 1000dd0c     service.obj
 0001:0000cd28       ??_C@_1BA@HHOMBECE@?$AAM?$AAe?$AAs?$AAs?$AAa?$AAg?$AAe?$AA?$AA@ 1000dd28     service.obj
 0001:0000cd38       ??_C@_17PAGBAIDI@?$AA?$DL?$AAO?$AAK?$AA?$AA@ 1000dd38     service.obj
 0001:0000cd40       ??_C@_09ENKGJCEC@OwnerGuid?$AA@ 1000dd40     service.obj
 0001:0000cd4c       ??_C@_0N@CCPLCIHE@PluginHandle?$AA@ 1000dd4c     service.obj
 0001:0000cd5c       ??_C@_09BKHPOLGD@PanelType?$AA@ 1000dd5c     service.obj
 0001:0000cd68       ??_C@_04GOOOJOPP@left?$AA@ 1000dd68     service.obj
 0001:0000cd70       ??_C@_03FGFCOCMD@top?$AA@  1000dd70     service.obj
 0001:0000cd74       ??_C@_05DHJDAOHK@right?$AA@ 1000dd74     service.obj
 0001:0000cd7c       ??_C@_06PMMPCIPB@bottom?$AA@ 1000dd7c     service.obj
 0001:0000cd84       ??_C@_09MCEJMINN@PanelRect?$AA@ 1000dd84     service.obj
 0001:0000cd90       ??_C@_0M@DDGFKGKJ@ItemsNumber?$AA@ 1000dd90     service.obj
 0001:0000cd9c       ??_C@_0BE@EOBAHHNK@SelectedItemsNumber?$AA@ 1000dd9c     service.obj
 0001:0000cdb0       ??_C@_0M@JMILNLLF@CurrentItem?$AA@ 1000ddb0     service.obj
 0001:0000cdbc       ??_C@_0N@CDHIFJIH@TopPanelItem?$AA@ 1000ddbc     service.obj
 0001:0000cdcc       ??_C@_08IMMBLBLF@ViewMode?$AA@ 1000ddcc     service.obj
 0001:0000cdd8       ??_C@_08CENECNJD@SortMode?$AA@ 1000ddd8     service.obj
 0001:0000cde4       ??_C@_04FABLJDN@Name?$AA@  1000dde4     service.obj
 0001:0000cdec       ??_C@_05LOJBNELM@Param?$AA@ 1000ddec     service.obj
 0001:0000cdf4       ??_C@_04PBAHLACE@File?$AA@ 1000ddf4     service.obj
 0001:0000cdfc       ??_C@_08HGEAFCFN@PluginId?$AA@ 1000ddfc     service.obj
 0001:0000ce08       ??_C@_0BA@MLHECKCE@table?5or?5string?$AA@ 1000de08     service.obj
 0001:0000ce18       ??_C@_0BD@CKJHMJBG@non?9positive?5index?$AA@ 1000de18     service.obj
 0001:0000ce2c       ??_C@_0BA@GNKNKKDM@number?5or?5table?$AA@ 1000de2c     service.obj
 0001:0000ce3c       ??_C@_0CI@DDAJHJKO@?$CFs?5?9?5unsupported?5type?5in?5dialog?5@ 1000de3c     service.obj
 0001:0000ce64       ??_C@_0CD@JIANOKII@unsupported?5flag?5in?5dialog?5item?5@ 1000de64     service.obj
 0001:0000ce88       ??_C@_0CB@EOGFCCCC@value?5at?5index?5?$CFd?5is?5not?5a?5table@ 1000de88     service.obj
 0001:0000ceac       ??_C@_0O@FEBHKEHB@closed?5dialog?$AA@ 1000deac     service.obj
 0001:0000cebc       ??_C@_0BK@NEMPGLFN@operation?5not?5implemented?$AA@ 1000debc     service.obj
 0001:0000ced8       ??_C@_04KPCPLBPL@Left?$AA@ 1000ded8     service.obj
 0001:0000cee0       ??_C@_03PGGAENPN@Top?$AA@  1000dee0     service.obj
 0001:0000cee4       ??_C@_05DADPALEM@Right?$AA@ 1000dee4     service.obj
 0001:0000ceec       ??_C@_0CK@JHNDGJBB@element?5?$CD?$CFd?5in?5argument?5?$CD4?5is?5no@ 1000deec     service.obj
 0001:0000cf18       ??_C@_0L@CECHCPAP@StartIndex?$AA@ 1000df18     service.obj
 0001:0000cf24       ??_C@_05IJGIMMHE@Count?$AA@ 1000df24     service.obj
 0001:0000cf2c       ??_C@_07NOCIGAPP@Pattern?$AA@ 1000df2c     service.obj
 0001:0000cf34       ??_C@_09IMOCKOO@SelectPos?$AA@ 1000df34     service.obj
 0001:0000cf40       ??_C@_06DJONBJOP@TopPos?$AA@ 1000df40     service.obj
 0001:0000cf48       ??_C@_09OGCBKCAK@MaxLength?$AA@ 1000df48     service.obj
 0001:0000cf54       ??_C@_05FNNGFGLF@Index?$AA@ 1000df54     service.obj
 0001:0000cf5c       ??_C@_07GHGHLGFI@GetType?$AA@ 1000df5c     service.obj
 0001:0000cf64       ??_C@_07MMLMCDAI@ValType?$AA@ 1000df64     service.obj
 0001:0000cf6c       ??_C@_05LPIJGKJ@Value?$AA@ 1000df6c     service.obj
 0001:0000cf74       ??_C@_0L@LPFMIAHH@helpstring?$AA@ 1000df74     service.obj
 0001:0000cf80       ??_C@_0P@NABDHFON@getvaluestring?$AA@ 1000df80     service.obj
 0001:0000cf90       ??_C@_0BJ@IINAPFDG@Items?$FL?$CFd?$FN?5is?5not?5a?5table?$AA@ 1000df90     service.obj
 0001:0000cfac       ??_C@_0CC@GBOJFNBI@error?5occured?5in?5dialog?5procedur@ 1000dfac     service.obj
 0001:0000cfd0       ??_C@_0M@EHMONPJO@?$CFs?5?$CIclosed?$CJ?$AA@ 1000dfd0     service.obj
 0001:0000cfdc       ??_C@_08GDAJJKGC@ViewerID?$AA@ 1000dfdc     service.obj
 0001:0000cfe8       ??_C@_07MJHBHMFM@FilePos?$AA@ 1000dfe8     service.obj
 0001:0000cff0       ??_C@_07FBAHDBGN@CurMode?$AA@ 1000dff0     service.obj
 0001:0000cff8       ??_C@_06IMBBKDFH@iParam?$AA@ 1000dff8     service.obj
 0001:0000d000       ??_C@_1BE@CGKCNEEP@?$AAI?$AAn?$AAp?$AAu?$AAt?$AA?5?$AAB?$AAo?$AAx?$AA?$AA@ 1000e000     service.obj
 0001:0000d014       ??_C@_1CA@PCDNIBFH@?$AAE?$AAn?$AAt?$AAe?$AAr?$AA?5?$AAt?$AAh?$AAe?$AA?5?$AAt?$AAe?$AAx?$AAt?$AA?3?$AA?$AA@ 1000e014     service.obj
 0001:0000d034       ??_C@_0BG@GAFLOAPP@command?5not?5supported?$AA@ 1000e034     service.obj
 0001:0000d04c       ??_C@_09MIJAKHKB@Completed?$AA@ 1000e04c     service.obj
 0001:0000d058       ??_C@_05KGEAEGFG@Total?$AA@ 1000e058     service.obj
 0001:0000d060       ??_C@_0P@DJOANNIK@?$CFd?4?$CFd?4?$CFd?4?$CFd?4?$CFd?$AA@ 1000e060     service.obj
 0001:0000d070       ??_C@_03FCCPIJGJ@Pos?$AA@  1000e070     service.obj
 0001:0000d074       ??_C@_08NNKIOIN@TypeName?$AA@ 1000e074     service.obj
 0001:0000d080       ??_C@_07ONPPLIAF@ErrCode?$AA@ 1000e080     service.obj
 0001:0000d088       ??_C@_07LJDOKIBM@ErrPosX?$AA@ 1000e088     service.obj
 0001:0000d090       ??_C@_07KACFJJFN@ErrPosY?$AA@ 1000e090     service.obj
 0001:0000d098       ??_C@_06HBEFEBCM@ErrSrc?$AA@ 1000e098     service.obj
 0001:0000d0a0       ??_C@_06LDIMCHFC@?$CF?$CKs?$CFs?5?$AA@ 1000e0a0     service.obj
 0001:0000d0a8       ??_C@_0CC@JIGPFMKG@global?5?$GAtostring?8?5is?5not?5functio@ 1000e0a8     service.obj
 0001:0000d0cc       ??_C@_0CH@OINAPBOJ@tostring?$CI?$CJ?5returned?5a?5non?9string@ 1000e0cc     service.obj
 0001:0000d0f4       ??_C@_06GBEMGMMA@?$CF?$CKd?$CFs?5?$AA@ 1000e0f4     service.obj
 0001:0000d0fc       ??_C@_04CIMGMMMG@text?$AA@ 1000e0fc     service.obj
 0001:0000d104       ??_C@_03CAOIPBNL@arg?$AA@  1000e104     service.obj
 0001:0000d108       ??_C@_0ME@JDKAEDFJ@local?5items?0n?$DN?4?4?4?6local?5bottom?$DNn@ 1000e108     service.obj
 0001:0000d1cc       ??_C@_0CG@FGNNCNLL@attempt?5to?5access?5invalid?5file?5f@ 1000e1cc     service.obj
 0001:0000d1f4       ??_C@_07BJOIOONN@Strings?$AA@ 1000e1f4     service.obj
 0001:0000d1fc       ??_C@_08FGAFMHLF@DiskMenu?$AA@ 1000e1fc     service.obj
 0001:0000d208       ??_C@_0L@NHENMPLN@PluginMenu?$AA@ 1000e208     service.obj
 0001:0000d214       ??_C@_0N@IEACHFBM@PluginConfig?$AA@ 1000e214     service.obj
 0001:0000d224       ??_C@_05GCJGCMFJ@PInfo?$AA@ 1000e224     service.obj
 0001:0000d22c       ??_C@_05HMEFBOHK@GInfo?$AA@ 1000e22c     service.obj
 0001:0000d234       ??_C@_0N@GAMEMCEE@invalid?5GUID?$AA@ 1000e234     service.obj
 0001:0000d244       ??_C@_0BP@NJEEOHDB@attempt?5to?5access?5closed?5timer?$AA@ 1000e244     service.obj
 0001:0000d264       ??_C@_05LGELBCGM@Close?$AA@ 1000e264     service.obj
 0001:0000d26c       ??_C@_07DOAOMMKG@Enabled?$AA@ 1000e26c     service.obj
 0001:0000d274       ??_C@_08KDKDEPAG@Interval?$AA@ 1000e274     service.obj
 0001:0000d280       ??_C@_07CIINKFND@OnTimer?$AA@ 1000e280     service.obj
 0001:0000d288       ??_C@_06EFCDMIMC@Closed?$AA@ 1000e288     service.obj
 0001:0000d290       ??_C@_0CE@LHJCBGGH@attempt?5to?5call?5non?9existent?5met@ 1000e290     service.obj
 0001:0000d2b4       ??_C@_0BO@PNFLEJKN@attempt?5to?5access?5a?5closed?5?$CFs?$AA@ 1000e2b4     service.obj
 0001:0000d2d4       ??_C@_04OKOFBOPB@Time?$AA@ 1000e2d4     service.obj
 0001:0000d2dc       ??_C@_04LADJNOK@Lock?$AA@  1000e2dc     service.obj
 0001:0000d2e4       ??_C@_0N@ECMJOJJG@MacroCallFar?$AA@ 1000e2e4     service.obj
 0001:0000d2f4       ??_C@_0BC@JJHHFNMP@FarMacroCallToLua?$AA@ 1000e2f4     service.obj
 0001:0000d308       ??_C@_06GIFLLBB@editor?$AA@ 1000e308     service.obj
 0001:0000d310       ??_C@_06DGPPOJKF@viewer?$AA@ 1000e310     service.obj
 0001:0000d318       ??_C@_01DICPFPGM@k?$AA@    1000e318     service.obj
 0001:0000d31c       ??_C@_06BPGFKLEK@__mode?$AA@ 1000e31c     service.obj
 0001:0000d324       ??_C@_1CC@OPOAGCKN@?$AA?2?$AAl?$AAu?$AAa?$AAf?$AAa?$AAr?$AA_?$AAi?$AAn?$AAi?$AAt?$AA?4?$AAl?$AAu?$AAa?$AA?$AA@ 1000e324     service.obj
 0001:0000d348       ??_C@_1BG@BDOBMIBP@?$AAF?$AAA?$AAR?$AAP?$AAR?$AAO?$AAF?$AAI?$AAL?$AAE?$AA?$AA@ 1000e348     service.obj
 0001:0000d360       ??_C@_04LHHHFLPP@utf8?$AA@ 1000e360     service.obj
 0001:0000d368       ??_C@_06ONNDGCDK@dofile?$AA@ 1000e368     service.obj
 0001:0000d370       ??_C@_08BNNFLGCJ@loadfile?$AA@ 1000e370     service.obj
 0001:0000d37c       ??_C@_03OFAPEBGM@?$CFs?6?$AA@ 1000e37c     service.obj
 0001:0000d380       __real@3ff0000000000000    1000e380     service.obj
 0001:0000d388       __real@4059000000000000    1000e388     service.obj
 0001:0000d390       __real@41e0000000000000    1000e390     service.obj
 0001:0000d398       __real@41f0000000000000    1000e398     service.obj
 0001:0000d428       ??_C@_04IHGKJMLH@byte?$AA@ 1000e428     slnunico.obj
 0001:0000d430       ??_C@_04ENMBGAPA@char?$AA@ 1000e430     slnunico.obj
 0001:0000d438       ??_C@_04GGLOKIEE@dump?$AA@ 1000e438     slnunico.obj
 0001:0000d440       ??_C@_06DLEPGFEF@format?$AA@ 1000e440     slnunico.obj
 0001:0000d448       ??_C@_05EIEIBDFD@gfind?$AA@ 1000e448     slnunico.obj
 0001:0000d450       ??_C@_03BKCJCHLK@len?$AA@  1000e450     slnunico.obj
 0001:0000d454       ??_C@_05IPJEPLHL@lower?$AA@ 1000e454     slnunico.obj
 0001:0000d45c       ??_C@_03HOKODIMJ@rep?$AA@  1000e45c     slnunico.obj
 0001:0000d460       ??_C@_07KOIEOCCE@reverse?$AA@ 1000e460     slnunico.obj
 0001:0000d468       ??_C@_05NECKJAMC@upper?$AA@ 1000e468     slnunico.obj
 0001:0000d470       ??_C@_09GCBMKPBD@utf8valid?$AA@ 1000e470     slnunico.obj
 0001:0000d47c       ??_C@_04GMGOKAFF@mode?$AA@ 1000e47c     slnunico.obj
 0001:0000d484       ??_C@_0BG@DFAIEAEC@string?5slice?5too?5long?$AA@ 1000e484     slnunico.obj
 0001:0000d49c       ??_C@_0O@EAJJMEEM@invalid?5value?$AA@ 1000e49c     slnunico.obj
 0001:0000d4ac       ??_C@_0BO@BNLBHKJN@unable?5to?5dump?5given?5function?$AA@ 1000e4ac     slnunico.obj
 0001:0000d4cc       ??_C@_0BG@LEHNKOGD@invalid?5capture?5index?$AA@ 1000e4cc     slnunico.obj
 0001:0000d4e4       ??_C@_0BI@ECNPHIBF@invalid?5pattern?5capture?$AA@ 1000e4e4     slnunico.obj
 0001:0000d4fc       ??_C@_0CD@PLJBIEHA@malformed?5pattern?5?$CIends?5with?5?8?$CF?$CF@ 1000e4fc     slnunico.obj
 0001:0000d520       ??_C@_0CA@CFGACOGB@malformed?5pattern?5?$CImissing?5?8?$FN?8?$CJ?$AA@ 1000e520     slnunico.obj
 0001:0000d540       ??_C@_0BD@NGJIMPLI@unbalanced?5pattern?$AA@ 1000e540     slnunico.obj
 0001:0000d554       ??_C@_0BC@IMEAEJPD@too?5many?5captures?$AA@ 1000e554     slnunico.obj
 0001:0000d568       ??_C@_0BD@BFKNEALP@unfinished?5capture?$AA@ 1000e568     slnunico.obj
 0001:0000d57c       ??_C@_0L@NLFJOONJ@?$FO$?$CK?$CL?$DP?4?$CI?$FL?$CF?9?$AA@ 1000e57c     slnunico.obj
 0001:0000d588       ??_C@_0CO@MAGJPEI@?8string?4gfind?8?5was?5renamed?5to?5?8s@ 1000e588     slnunico.obj
 0001:0000d5b8       ??_C@_0BP@PPPOBACA@string?1function?1table?5expected?$AA@ 1000e5b8     slnunico.obj
 0001:0000d5d8       ??_C@_0CB@LPDIHGGA@invalid?5replacement?5value?5?$CIa?5?$CFs?$CJ@ 1000e5d8     slnunico.obj
 0001:0000d5fc       ??_C@_02HIBBOKEN@?2r?$AA@  1000e5fc     slnunico.obj
 0001:0000d600       ??_C@_04MPDIABOK@?2000?$AA@ 1000e600     slnunico.obj
 0001:0000d608       ??_C@_05GGBDHNF@?9?$CL?5?$CD0?$AA@ 1000e608     slnunico.obj
 0001:0000d610       ??_C@_0CA@COOMGCAO@invalid?5format?5?$CIrepeated?5flags?$CJ?$AA@ 1000e610     slnunico.obj
 0001:0000d630       ??_C@_0CN@KALFEKPN@invalid?5format?5?$CIwidth?5or?5precisi@ 1000e630     slnunico.obj
 0001:0000d660       ??_C@_0CC@KIPBEOBI@invalid?5option?5?8?$CF?$CF?$CFc?8?5to?5?8format@ 1000e660     slnunico.obj
 0001:0000d684       ??_C@_0O@EJMKHGFJ@unicode?4ascii?$AA@ 1000e684     slnunico.obj
 0001:0000d694       ??_C@_0P@CMOFLLND@unicode?4latin1?$AA@ 1000e694     slnunico.obj
 0001:0000d6a4       ??_C@_0BB@EFCDCNG@unicode?4grapheme?$AA@ 1000e6a4     slnunico.obj
 0001:0000d6b8       ??_C@_0N@DKIDGKBP@unicode?4utf8?$AA@ 1000e6b8     slnunico.obj
 0001:0000d7b8       ??_C@_05DFJCHPDH@input?$AA@ 1000e7b8     uliolib51.obj
 0001:0000d7c0       ??_C@_06DKIGHACF@output?$AA@ 1000e7c0     uliolib51.obj
 0001:0000d7c8       ??_C@_03KCHOJKKI@set?$AA@  1000e7c8     uliolib51.obj
 0001:0000d7cc       ??_C@_03LIBLMJMB@cur?$AA@  1000e7cc     uliolib51.obj
 0001:0000d7d0       ??_C@_03JBJLGPFL@end?$AA@  1000e7d0     uliolib51.obj
 0001:0000d7d4       ??_C@_02KAJCLHKP@no?$AA@   1000e7d4     uliolib51.obj
 0001:0000d7d8       ??_C@_04PLMLMMEO@full?$AA@ 1000e7d8     uliolib51.obj
 0001:0000d7e0       ??_C@_04HJPCFDOP@line?$AA@ 1000e7e0     uliolib51.obj
 0001:0000d7e8       ??_C@_05LBOHBHFK@close?$AA@ 1000e7e8     uliolib51.obj
 0001:0000d7f0       ??_C@_05GLCAEPFP@flush?$AA@ 1000e7f0     uliolib51.obj
 0001:0000d7f8       ??_C@_05DENOCHIP@lines?$AA@ 1000e7f8     uliolib51.obj
 0001:0000d800       ??_C@_05IACAFMHP@popen?$AA@ 1000e800     uliolib51.obj
 0001:0000d808       ??_C@_07FKJPAINK@tmpfile?$AA@ 1000e808     uliolib51.obj
 0001:0000d810       ??_C@_05NGFEDHGN@write?$AA@ 1000e810     uliolib51.obj
 0001:0000d818       ??_C@_04EDECCOGL@seek?$AA@ 1000e818     uliolib51.obj
 0001:0000d820       ??_C@_07HHBPNGAN@setvbuf?$AA@ 1000e820     uliolib51.obj
 0001:0000d828       ??_C@_06DJHOIPC@?$CFs?3?5?$CFs?$AA@ 1000e828     uliolib51.obj
 0001:0000d830       ??_C@_02DKCKIIND@?$CFs?$AA@ 1000e830     uliolib51.obj
 0001:0000d834       ??_C@_05KCHOJJD@FILE?$CK?$AA@ 1000e834     uliolib51.obj
 0001:0000d83c       ??_C@_0M@IBKPHHKH@closed?5file?$AA@ 1000e83c     uliolib51.obj
 0001:0000d848       ??_C@_04DAMGJPCA@file?$AA@ 1000e848     uliolib51.obj
 0001:0000d850       ??_C@_0BN@LPOOHAOM@attempt?5to?5use?5a?5closed?5file?$AA@ 1000e850     uliolib51.obj
 0001:0000d870       ??_C@_0BL@PEFGCPAG@cannot?5close?5standard?5file?$AA@ 1000e870     uliolib51.obj
 0001:0000d88c       ??_C@_07DMJMBBKE@__close?$AA@ 1000e88c     uliolib51.obj
 0001:0000d894       ??_C@_0O@PLFAPHPG@file?5?$CIclosed?$CJ?$AA@ 1000e894     uliolib51.obj
 0001:0000d8a4       ??_C@_09BPMAMLLD@file?5?$CI?$CFp?$CJ?$AA@ 1000e8a4     uliolib51.obj
 0001:0000d8b0       ??_C@_17OBBFBLGE@?$AAr?$AAw?$AAa?$AA?$AA@ 1000e8b0     uliolib51.obj
 0001:0000d8b8       ??_C@_0CP@DHGANCPP@invalid?5mode?5?8?$CFs?8?5?$CIshould?5match?5@ 1000e8b8     uliolib51.obj
 0001:0000d8e8       ??_C@_0BL@JMNLNGCA@standard?5?$CFs?5file?5is?5closed?$AA@ 1000e8e8     uliolib51.obj
 0001:0000d904       ??_C@_13CIFDLIMG@?$AAw?$AA?$AA@ 1000e904     uliolib51.obj
 0001:0000d908       ??_C@_03DLDNIBIK@?$CFlf?$AA@ 1000e908     uliolib51.obj
 0001:0000d90c       ??_C@_0BD@IOJAAODF@too?5many?5arguments?$AA@ 1000e90c     uliolib51.obj
 0001:0000d920       ??_C@_0P@PJFAGLMH@invalid?5option?$AA@ 1000e920     uliolib51.obj
 0001:0000d930       ??_C@_0P@CENJCLHM@invalid?5format?$AA@ 1000e930     uliolib51.obj
 0001:0000d940       ??_C@_0BH@PBGIDLEF@file?5is?5already?5closed?$AA@ 1000e940     uliolib51.obj
 0001:0000d958       ??_C@_05CGOEHEFE@?$CF?414g?$AA@ 1000e958     uliolib51.obj
 0001:0000d960       ??_C@_05MHOFLBOO@stdin?$AA@ 1000e960     uliolib51.obj
 0001:0000d968       ??_C@_06DJDOIFHB@stdout?$AA@ 1000e968     uliolib51.obj
 0001:0000d970       ??_C@_06FJGNEBG@stderr?$AA@ 1000e970     uliolib51.obj
 0001:0000d9c0       ??_C@_07KOEABFCN@loadlib?$AA@ 1000e9c0     uloadlib51.obj
 0001:0000d9c8       ??_C@_06LNOHAKGK@seeall?$AA@ 1000e9c8     uloadlib51.obj
 0001:0000d9d0       ??_C@_06BIEEJMKO@module?$AA@ 1000e9d0     uloadlib51.obj
 0001:0000d9d8       ??_C@_07FFLLPPLH@require?$AA@ 1000e9d8     uloadlib51.obj
 0001:0000d9e0       ??_C@_0BN@GMPFCLAN@unable?5to?5get?5ModuleFileName?$AA@ 1000e9e0     uloadlib51.obj
 0001:0000da00       ??_C@_13MGDFOILI@?$AA?$CB?$AA?$AA@ 1000ea00     uloadlib51.obj
 0001:0000da04       ??_C@_09GMLHALBF@LOADLIB?3?5?$AA@ 1000ea04     uloadlib51.obj
 0001:0000da10       ??_C@_04HDOCAJNK@?$CFs?$CFs?$AA@ 1000ea10     uloadlib51.obj
 0001:0000da18       ??_C@_08HNNNOMMJ@_LOADLIB?$AA@ 1000ea18     uloadlib51.obj
 0001:0000da24       ??_C@_04HKFDNBLD@init?$AA@ 1000ea24     uloadlib51.obj
 0001:0000da2c       ??_C@_13FPGAJAPJ@?$AA?2?$AA?$AA@ 1000ea2c     uloadlib51.obj
 0001:0000da30       ??_C@_13JOFGPIOO@?$AA?4?$AA?$AA@ 1000ea30     uloadlib51.obj
 0001:0000da34       ??_C@_0BO@COFCKCAL@?8package?4?$CFs?8?5must?5be?5a?5string?$AA@ 1000ea34     uloadlib51.obj
 0001:0000da54       ??_C@_0CE@EPEHLLIH@?8package?4?$CFs?8?5contains?5invalid?5UT@ 1000ea54     uloadlib51.obj
 0001:0000da78       ??_C@_13HGPDMIBE@?$AA?$DP?$AA?$AA@ 1000ea78     uloadlib51.obj
 0001:0000da7c       ??_C@_0P@NEBKIMDC@?6?7no?5file?5?8?$CFs?8?$AA@ 1000ea7c     uloadlib51.obj
 0001:0000da8c       ??_C@_0CO@KHMIPLKM@error?5loading?5module?5?8?$CFs?8?5from?5f@ 1000ea8c     uloadlib51.obj
 0001:0000dabc       ??_C@_04LNEJFJGI@path?$AA@ 1000eabc     uloadlib51.obj
 0001:0000dac4       ??_C@_01IDAFKMJL@_?$AA@    1000eac4     uloadlib51.obj
 0001:0000dac8       ??_C@_01LFCBOECM@?4?$AA@   1000eac8     uloadlib51.obj
 0001:0000dacc       ??_C@_0L@KHKMBFOE@luaopen_?$CFs?$AA@ 1000eacc     uloadlib51.obj
 0001:0000dad8       ??_C@_05EEMJHCCC@cpath?$AA@ 1000ead8     uloadlib51.obj
 0001:0000dae0       ??_C@_0BO@KOILFIGK@?6?7no?5module?5?8?$CFs?8?5in?5file?5?8?$CFs?8?$AA@ 1000eae0     uloadlib51.obj
 0001:0000db00       ??_C@_0CC@CCJHFBLH@?8package?4preload?8?5must?5be?5a?5tabl@ 1000eb00     uloadlib51.obj
 0001:0000db24       ??_C@_0CB@NPNABMBF@?6?7no?5field?5package?4preload?$FL?8?$CFs?8?$FN@ 1000eb24     uloadlib51.obj
 0001:0000db48       ??_C@_07PINPBNPB@_LOADED?$AA@ 1000eb48     uloadlib51.obj
 0001:0000db50       ??_C@_0CL@DIEJCPFH@loop?5or?5previous?5error?5loading?5m@ 1000eb50     uloadlib51.obj
 0001:0000db7c       ??_C@_07JAOCDFCG@loaders?$AA@ 1000eb7c     uloadlib51.obj
 0001:0000db84       ??_C@_0CC@IGEJMOFI@?8package?4loaders?8?5must?5be?5a?5tabl@ 1000eb84     uloadlib51.obj
 0001:0000dba8       ??_C@_0BJ@HFHHABH@module?5?8?$CFs?8?5not?5found?3?$CFs?$AA@ 1000eba8     uloadlib51.obj
 0001:0000dbc4       ??_C@_01INIBCBCB@f?$AA@    1000ebc4     uloadlib51.obj
 0001:0000dbc8       ??_C@_0CI@GKOMOAFD@?8module?8?5not?5called?5from?5a?5Lua?5f@ 1000ebc8     uloadlib51.obj
 0001:0000dbf0       ??_C@_02CCIJHOCI@_M?$AA@   1000ebf0     uloadlib51.obj
 0001:0000dbf4       ??_C@_05ICMCJINN@_NAME?$AA@ 1000ebf4     uloadlib51.obj
 0001:0000dbfc       ??_C@_08HONLOGDK@_PACKAGE?$AA@ 1000ebfc     uloadlib51.obj
 0001:0000dc08       ??_C@_0BO@CBJIAGLF@name?5conflict?5for?5module?5?8?$CFs?8?$AA@ 1000ec08     uloadlib51.obj
 0001:0000dc28       ??_C@_17KOAMMDLI@?$AA?$DL?$AA?$AB?$AA?$DL?$AA?$AA@ 1000ec28     uloadlib51.obj
 0001:0000dc30       ??_C@_15HKKNGJC@?$AA?$DL?$AA?$DL?$AA?$AA@ 1000ec30     uloadlib51.obj
 0001:0000dc38       ??_C@_13GGAHEHIG@?$AA?$AB?$AA?$AA@ 1000ec38     uloadlib51.obj
 0001:0000dc40       ??_C@_1HE@JLDBNBHO@?$AA?4?$AA?2?$AA?$DP?$AA?4?$AAl?$AAu?$AAa?$AA?$DL?$AA?$CB?$AA?2?$AAl?$AAu?$AAa?$AA?2?$AA?$DP?$AA?4?$AAl?$AAu?$AAa?$AA?$DL?$AA?$CB?$AA?2?$AAl?$AAu?$AAa?$AA?2?$AA?$DP?$AA?2?$AAi?$AAn?$AAi?$AAt@ 1000ec40     uloadlib51.obj
 0001:0000dcb4       ??_C@_1BC@ILFFIBFI@?$AAL?$AAU?$AAA?$AA_?$AAP?$AAA?$AAT?$AAH?$AA?$AA@ 1000ecb4     uloadlib51.obj
 0001:0000dcc8       ??_C@_1DM@FGPGEDD@?$AA?4?$AA?2?$AA?$DP?$AA?4?$AAd?$AAl?$AAl?$AA?$DL?$AA?$CB?$AA?2?$AA?$DP?$AA?4?$AAd?$AAl?$AAl?$AA?$DL?$AA?$CB?$AA?2?$AAl?$AAo?$AAa?$AAd?$AAa?$AAl?$AAl?$AA?4?$AAd?$AAl?$AAl?$AA?$AA@ 1000ecc8     uloadlib51.obj
 0001:0000dd04       ??_C@_1BE@EFNILHBI@?$AAL?$AAU?$AAA?$AA_?$AAC?$AAP?$AAA?$AAT?$AAH?$AA?$AA@ 1000ed04     uloadlib51.obj
 0001:0000dd18       ??_C@_1BE@CKNDCMBB@?$AA?2?$AA?6?$AA?$DL?$AA?6?$AA?$DP?$AA?6?$AA?$CB?$AA?6?$AA?9?$AA?$AA@ 1000ed18     uloadlib51.obj
 0001:0000dd2c       ??_C@_06HEJKKHEK@config?$AA@ 1000ed2c     uloadlib51.obj
 0001:0000dd34       ??_C@_06IILMCCFO@loaded?$AA@ 1000ed34     uloadlib51.obj
 0001:0000dd40       _ustring_funcs             1000ed40     ustring.obj
 0001:0000de18       ??_C@_0BE@DEHGONAH@EnumSystemCodePages?$AA@ 1000ee18     ustring.obj
 0001:0000de2c       ??_C@_06FMJLOCAF@GetACP?$AA@ 1000ee2c     ustring.obj
 0001:0000de34       ??_C@_09HLFMNDA@GetCPInfo?$AA@ 1000ee34     ustring.obj
 0001:0000de40       ??_C@_0O@PIBBCLJF@GetCurrentDir?$AA@ 1000ee40     ustring.obj
 0001:0000de50       ??_C@_0N@IIBOJKJ@GetDriveType?$AA@ 1000ee50     ustring.obj
 0001:0000de60       ??_C@_0M@KHMMJMNI@GetFileAttr?$AA@ 1000ee60     ustring.obj
 0001:0000de6c       ??_C@_0M@ONGMCNNE@GetKeyState?$AA@ 1000ee6c     ustring.obj
 0001:0000de78       ??_C@_0BH@KKAFOIJJ@GetLogicalDriveStrings?$AA@ 1000ee78     ustring.obj
 0001:0000de90       ??_C@_08OMCNFONF@GetOEMCP?$AA@ 1000ee90     ustring.obj
 0001:0000de9c       ??_C@_0BD@IHIHPGDL@GlobalMemoryStatus?$AA@ 1000ee9c     ustring.obj
 0001:0000deb0       ??_C@_0BE@HCIKGJGE@MultiByteToWideChar?$AA@ 1000eeb0     ustring.obj
 0001:0000dec4       ??_C@_09EPINLGBH@OemToUtf8?$AA@ 1000eec4     ustring.obj
 0001:0000ded0       ??_C@_0BC@NFCPMJFM@OutputDebugString?$AA@ 1000eed0     ustring.obj
 0001:0000dee4       ??_C@_0BA@MNJFBAJH@SHGetFolderPath?$AA@ 1000eee4     ustring.obj
 0001:0000def4       ??_C@_0L@PMCLJMMJ@SearchPath?$AA@ 1000eef4     ustring.obj
 0001:0000df00       ??_C@_0O@IHAPJIOC@SetCurrentDir?$AA@ 1000ef00     ustring.obj
 0001:0000df10       ??_C@_0M@KINCEKFL@SetFileAttr?$AA@ 1000ef10     ustring.obj
 0001:0000df1c       ??_C@_05PFDOMJEF@Sleep?$AA@ 1000ef1c     ustring.obj
 0001:0000df24       ??_C@_0M@KJELMDJD@Utf16ToUtf8?$AA@ 1000ef24     ustring.obj
 0001:0000df30       ??_C@_09LCEKPEGC@Utf8ToOem?$AA@ 1000ef30     ustring.obj
 0001:0000df3c       ??_C@_0M@GJGCILHG@Utf8ToUtf16?$AA@ 1000ef3c     ustring.obj
 0001:0000df48       ??_C@_04NDFIEGPL@Uuid?$AA@ 1000ef48     ustring.obj
 0001:0000df50       ??_C@_0BE@LJADKLBD@WideCharToMultiByte?$AA@ 1000ef50     ustring.obj
 0001:0000df64       ??_C@_04GFOHBGIO@subW?$AA@ 1000ef64     ustring.obj
 0001:0000df6c       ??_C@_06FHFOAHML@system?$AA@ 1000ef6c     ustring.obj
 0001:0000df74       ??_C@_04NOFELICG@lenW?$AA@ 1000ef74     ustring.obj
 0001:0000df7c       ??_C@_0BB@BLJKPILH@system?5error?5?$CFd?6?$AA@ 1000ef7c     ustring.obj
 0001:0000df90       ??_C@_0BJ@MEAJDMDL@invalid?5multibyte?5string?$AA@ 1000ef90     ustring.obj
 0001:0000dfac       ??_C@_0BG@ELIKBHAO@invalid?5UTF?916?5string?$AA@ 1000efac     ustring.obj
 0001:0000dfc4       ??_C@_0M@KJGJBDLL@MaxCharSize?$AA@ 1000efc4     ustring.obj
 0001:0000dfd0       ??_C@_0M@IMOFNPBB@DefaultChar?$AA@ 1000efd0     ustring.obj
 0001:0000dfdc       ??_C@_08HIIJAENB@LeadByte?$AA@ 1000efdc     ustring.obj
 0001:0000dfe8       ??_C@_0BD@CBNPFFPH@UnicodeDefaultChar?$AA@ 1000efe8     ustring.obj
 0001:0000dffc       ??_C@_0N@DJCOCBOB@CodePageName?$AA@ 1000effc     ustring.obj
 0001:0000e00c       ??_C@_0N@IFJMFGJK@unknown?5type?$AA@ 1000f00c     ustring.obj
 0001:0000e01c       ??_C@_0BC@GPFCFLGN@no?5root?5directory?$AA@ 1000f01c     ustring.obj
 0001:0000e030       ??_C@_09HPGMKNKO@removable?$AA@ 1000f030     ustring.obj
 0001:0000e03c       ??_C@_05OFLEIIDM@fixed?$AA@ 1000f03c     ustring.obj
 0001:0000e044       ??_C@_06IMIHEKN@remote?$AA@ 1000f044     ustring.obj
 0001:0000e04c       ??_C@_05POABADMF@cdrom?$AA@ 1000f04c     ustring.obj
 0001:0000e054       ??_C@_07BHCBOAMP@ramdisk?$AA@ 1000f054     ustring.obj
 0001:0000e05c       ??_C@_0L@PLJFMBIJ@MemoryLoad?$AA@ 1000f05c     ustring.obj
 0001:0000e068       ??_C@_09MMAOIBBJ@TotalPhys?$AA@ 1000f068     ustring.obj
 0001:0000e074       ??_C@_09KFOEOLH@AvailPhys?$AA@ 1000f074     ustring.obj
 0001:0000e080       ??_C@_0O@PEEMGPEP@TotalPageFile?$AA@ 1000f080     ustring.obj
 0001:0000e090       ??_C@_0O@LLHOKNF@AvailPageFile?$AA@ 1000f090     ustring.obj
 0001:0000e0a0       ??_C@_0N@LCJEOHMM@TotalVirtual?$AA@ 1000f0a0     ustring.obj
 0001:0000e0b0       ??_C@_0N@EGHLANBF@AvailVirtual?$AA@ 1000f0b0     ustring.obj
 0001:0000e0c0       ??_C@_0BF@KKNLCGDE@AvailExtendedVirtual?$AA@ 1000f0c0     ustring.obj
 0001:0000e0d8       ??_C@_0P@KJDDGAFH@FileAttributes?$AA@ 1000f0d8     ustring.obj
 0001:0000e0e8       ??_C@_07JOJHCKGP@ustring?$AA@ 1000f0e8     ustring.obj
 0001:0000e980       ??_C@_0DJ@KKHMCMAP@bad?5field?5?$FL?$CFd?$FN?5in?5table?5stackpos@ 1000f980     util.obj
 0001:0000e9bc       ??_C@_0DJ@PFHHGAMM@bad?5field?5?8?$CFs?8?5in?5table?5stackpos@ 1000f9bc     util.obj
 0001:0000e9f8       ??_C@_06EBGNBFIA@number?$AA@ 1000f9f8     util.obj
 0001:0000ee80       _win_funcs                 1000fe80     win.obj
 0001:0000f360       ??_C@_0O@CFPMOCDP@CompareString?$AA@ 10010360     win.obj
 0001:0000f370       ??_C@_08PPLNFCGA@CopyFile?$AA@ 10010370     win.obj
 0001:0000f37c       ??_C@_09INHPLKKM@CreateDir?$AA@ 1001037c     win.obj
 0001:0000f388       ??_C@_0L@GPLPOFDC@DeleteFile?$AA@ 10010388     win.obj
 0001:0000f394       ??_C@_0N@FOJPHHPH@DeleteRegKey?$AA@ 10010394     win.obj
 0001:0000f3a4       ??_C@_0P@PCCDOIAL@DeleteRegValue?$AA@ 100103a4     win.obj
 0001:0000f3b4       ??_C@_0L@DGAGCFOP@EnumRegKey?$AA@ 100103b4     win.obj
 0001:0000f3c0       ??_C@_0N@PFFNCIBD@EnumRegValue?$AA@ 100103c0     win.obj
 0001:0000f3d0       ??_C@_0L@MGMEFCAE@ExtractKey?$AA@ 100103d0     win.obj
 0001:0000f3dc       ??_C@_0BI@EKFDIGHI@FileTimeToLocalFileTime?$AA@ 100103dc     win.obj
 0001:0000f3f4       ??_C@_0BF@KPJNHALE@FileTimeToSystemTime?$AA@ 100103f4     win.obj
 0001:0000f40c       ??_C@_0BL@NAIJNMLL@GetConsoleScreenBufferInfo?$AA@ 1001040c     win.obj
 0001:0000f428       ??_C@_06CALCCDMF@GetEnv?$AA@ 10010428     win.obj
 0001:0000f430       ??_C@_0M@EINGHLOA@GetFileInfo?$AA@ 10010430     win.obj
 0001:0000f43c       ??_C@_09GFGIAJLD@GetRegKey?$AA@ 1001043c     win.obj
 0001:0000f448       ??_C@_0BI@ENMDHCMK@GetSystemTimeAsFileTime?$AA@ 10010448     win.obj
 0001:0000f460       ??_C@_0P@GGGHOPAD@GetVirtualKeys?$AA@ 10010460     win.obj
 0001:0000f470       ??_C@_08CALLHOCI@MoveFile?$AA@ 10010470     win.obj
 0001:0000f47c       ??_C@_09EDKALOCB@RemoveDir?$AA@ 1001047c     win.obj
 0001:0000f488       ??_C@_0L@HBAGBENL@RenameFile?$AA@ 10010488     win.obj
 0001:0000f494       ??_C@_06LDCDJLBI@SetEnv?$AA@ 10010494     win.obj
 0001:0000f49c       ??_C@_09ELCNCICB@SetRegKey?$AA@ 1001049c     win.obj
 0001:0000f4a8       ??_C@_0N@BFFIJKHB@ShellExecute?$AA@ 100104a8     win.obj
 0001:0000f4b8       ??_C@_0BF@HBHGIPOG@SystemTimeToFileTime?$AA@ 100104b8     win.obj
 0001:0000f4d0       ??_C@_06DNONFAKH@wcscmp?$AA@ 100104d0     win.obj
 0001:0000f4d8       ??_C@_04CBBMIBLK@HKLM?$AA@ 100104d8     win.obj
 0001:0000f4e0       ??_C@_04LEMDOLAJ@HKCC?$AA@ 100104e0     win.obj
 0001:0000f4e8       ??_C@_04OHBKMIBJ@HKCR?$AA@ 100104e8     win.obj
 0001:0000f4f0       ??_C@_04KIFLFONO@HKCU?$AA@ 100104f0     win.obj
 0001:0000f4f8       ??_C@_03DLBIJLAB@HKU?$AA@  100104f8     win.obj
 0001:0000f4fc       ??_C@_0DA@DKALLFDI@must?5be?5?8HKLM?8?0?5?8HKCC?8?0?5?8HKCR?8?0?5@ 100104fc     win.obj
 0001:0000f52c       ??_C@_05KDALNKAH@dword?$AA@ 1001052c     win.obj
 0001:0000f534       ??_C@_06FNFBAEBE@binary?$AA@ 10010534     win.obj
 0001:0000f53c       ??_C@_0N@CBOMHLPN@expandstring?$AA@ 1001053c     win.obj
 0001:0000f54c       ??_C@_0M@PEGIPCHN@multistring?$AA@ 1001054c     win.obj
 0001:0000f558       ??_C@_0BH@NOJOGNJM@unsupported?5value?5type?$AA@ 10010558     win.obj
 0001:0000f570       ??_C@_0BD@MJODDCFG@OpenRegKey?5failed?4?$AA@ 10010570     win.obj
 0001:0000f584       ??_C@_0BI@COLHBIIE@RegQueryValueEx?5failed?4?$AA@ 10010584     win.obj
 0001:0000f59c       ??_C@_1BK@BIGILECK@?$AAA?$AAd?$AAv?$AAa?$AAp?$AAi?$AA3?$AA2?$AA?4?$AAd?$AAl?$AAl?$AA?$AA@ 1001059c     win.obj
 0001:0000f5b8       ??_C@_0BA@LILAPHGE@RegDeleteKeyExW?$AA@ 100105b8     win.obj
 0001:0000f5c8       ??_C@_0BG@HHFHBIKG@RegOpenKeyExW?5failed?4?$AA@ 100105c8     win.obj
 0001:0000f5e0       ??_C@_05DFPNHDMN@wYear?$AA@ 100105e0     win.obj
 0001:0000f5e8       ??_C@_06MGNNJGBJ@wMonth?$AA@ 100105e8     win.obj
 0001:0000f5f0       ??_C@_0L@OAHPHHP@wDayOfWeek?$AA@ 100105f0     win.obj
 0001:0000f5fc       ??_C@_04NBLBJIPP@wDay?$AA@ 100105fc     win.obj
 0001:0000f604       ??_C@_05BMOPCGDH@wHour?$AA@ 10010604     win.obj
 0001:0000f60c       ??_C@_07HPODENI@wMinute?$AA@ 1001060c     win.obj
 0001:0000f614       ??_C@_07IIEDHHJN@wSecond?$AA@ 10010614     win.obj
 0001:0000f61c       ??_C@_0O@HBAPEOKP@wMilliseconds?$AA@ 1001061c     win.obj
 0001:0000f62c       ??_C@_01LKDEMHDF@s?$AA@    1001062c     win.obj
 0001:0000f630       ??_C@_0BA@IAFODGNM@CursorPositionX?$AA@ 10010630     win.obj
 0001:0000f640       ??_C@_0BA@JJEFAHJN@CursorPositionY?$AA@ 10010640     win.obj
 0001:0000f650       ??_C@_0L@NFCEOFBF@WindowLeft?$AA@ 10010650     win.obj
 0001:0000f65c       ??_C@_09JHGOALHG@WindowTop?$AA@ 1001065c     win.obj
 0001:0000f668       ??_C@_0M@HHPHMPGH@WindowRight?$AA@ 10010668     win.obj
 0001:0000f674       ??_C@_0N@JPIJCAOJ@WindowBottom?$AA@ 10010674     win.obj
 0001:0000f684       ??_C@_0BD@DOLDEII@MaximumWindowSizeX?$AA@ 10010684     win.obj
 0001:0000f698       ??_C@_0BD@BKPAAFMJ@MaximumWindowSizeY?$AA@ 10010698     win.obj
 0001:0000f6ac       ??_C@_01PFHFFBPC@t?$AA@    100106ac     win.obj
 0001:0000f6b0       ??_C@_0BJ@LPJMBJJL@directory?5already?5exists?$AA@ 100106b0     win.obj
 0001:0000f6d0       __imp__EncodePointer@4     100106d0     vc_crt_fix.obj
 0001:0000f6d4       __imp__DecodePointer@4     100106d4     vc_crt_fix.obj
 0001:0000f6d8       __imp__GetModuleHandleExW@12 100106d8     vc_crt_fix.obj
 0001:0000f6dc       __imp__InitializeSListHead@4 100106dc     vc_crt_fix.obj
 0001:0000f6e0       __imp__InterlockedFlushSList@4 100106e0     vc_crt_fix.obj
 0001:0000f6e4       __imp__InterlockedPopEntrySList@4 100106e4     vc_crt_fix.obj
 0001:0000f6e8       __imp__InterlockedPushEntrySList@8 100106e8     vc_crt_fix.obj
 0001:0000f6ec       __imp__InterlockedPushListSListEx@16 100106ec     vc_crt_fix.obj
 0001:0000f6f0       __imp__RtlFirstEntrySList@4 100106f0     vc_crt_fix.obj
 0001:0000f6f4       __imp__QueryDepthSList@4   100106f4     vc_crt_fix.obj
 0001:0000f70c       ??_C@_0O@NLDKAIKN@EncodePointer?$AA@ 1001070c     vc_crt_fix_impl.obj
 0001:0000f71c       ??_C@_0O@KBPMFGHI@DecodePointer?$AA@ 1001071c     vc_crt_fix_impl.obj
 0001:0000f72c       ??_C@_0BD@GIGEJCNH@GetModuleHandleExW?$AA@ 1001072c     vc_crt_fix_impl.obj
 0001:0000f740       ??_C@_0BE@NBEJPEJA@InitializeSListHead?$AA@ 10010740     vc_crt_fix_impl.obj
 0001:0000f754       ??_C@_0BG@PLLPFLHB@InterlockedFlushSList?$AA@ 10010754     vc_crt_fix_impl.obj
 0001:0000f76c       ??_C@_0BJ@PNEEKDOK@InterlockedPopEntrySList?$AA@ 1001076c     vc_crt_fix_impl.obj
 0001:0000f788       ??_C@_0BK@JFGGAIOA@InterlockedPushEntrySList?$AA@ 10010788     vc_crt_fix_impl.obj
 0001:0000f7a4       ??_C@_0BL@FOECAEGO@InterlockedPushListSListEx?$AA@ 100107a4     vc_crt_fix_impl.obj
 0001:0000f7c0       ??_C@_0BD@FHMMIGCI@RtlFirstEntrySList?$AA@ 100107c0     vc_crt_fix_impl.obj
 0001:0000f7d4       ??_C@_0BA@FGPHPMJB@QueryDepthSList?$AA@ 100107d4     vc_crt_fix_impl.obj
 0001:0000f7e4       __pDefaultRawDllMain       100107e4     LIBCMT:dll_dllmain.obj
 0001:0000f7e4       __pRawDllMain              100107e4     LIBCMT:dll_dllmain.obj
 0001:0000f800       ??_C@_1BC@DNHGCMLG@?$AAa?$AAd?$AAv?$AAa?$AAp?$AAi?$AA3?$AA2?$AA?$AA@ 10010800     libvcruntime:winapi_downlevel.obj
 0001:0000f814       ??_C@_1DM@KHCHBNEB@?$AAa?$AAp?$AAi?$AA?9?$AAm?$AAs?$AA?9?$AAw?$AAi?$AAn?$AA?9?$AAc?$AAo?$AAr?$AAe?$AA?9?$AAf?$AAi?$AAb?$AAe?$AAr?$AAs?$AA?9?$AAl?$AA1?$AA?9?$AA1?$AA?9?$AA1?$AA?$AA@ 10010814     libvcruntime:winapi_downlevel.obj
 0001:0000f850       ??_C@_1DK@LPPGFMPP@?$AAa?$AAp?$AAi?$AA?9?$AAm?$AAs?$AA?9?$AAw?$AAi?$AAn?$AA?9?$AAc?$AAo?$AAr?$AAe?$AA?9?$AAs?$AAy?$AAn?$AAc?$AAh?$AA?9?$AAl?$AA1?$AA?9?$AA2?$AA?9?$AA0?$AA?$AA@ 10010850     libvcruntime:winapi_downlevel.obj
 0001:0000f88c       ??_C@_1BC@GDMECMAK@?$AAk?$AAe?$AAr?$AAn?$AAe?$AAl?$AA3?$AA2?$AA?$AA@ 1001088c     libvcruntime:winapi_downlevel.obj
 0001:0000f8a8       ??_C@_08KNHFBNJ@FlsAlloc?$AA@ 100108a8     libvcruntime:winapi_downlevel.obj
 0001:0000f8bc       ??_C@_07PEJMOBNF@FlsFree?$AA@ 100108bc     libvcruntime:winapi_downlevel.obj
 0001:0000f8cc       ??_C@_0M@GDNOONDI@FlsGetValue?$AA@ 100108cc     libvcruntime:winapi_downlevel.obj
 0001:0000f8e0       ??_C@_0M@JCPCPOEF@FlsSetValue?$AA@ 100108e0     libvcruntime:winapi_downlevel.obj
 0001:0000f8f4       ??_C@_0BM@HCFOFFN@InitializeCriticalSectionEx?$AA@ 100108f4     libvcruntime:winapi_downlevel.obj
 0001:0000faa0       ??_C@_08EHJDFFNH@__based?$CI?$AA@ 10010aa0     libvcruntime:undname.obj
 0001:0000faac       ??_C@_07KOLFKCDI@__cdecl?$AA@ 10010aac     libvcruntime:undname.obj
 0001:0000fab4       ??_C@_08GHMPAG@__pascal?$AA@ 10010ab4     libvcruntime:undname.obj
 0001:0000fac0       ??_C@_09IFJBGAPI@__stdcall?$AA@ 10010ac0     libvcruntime:undname.obj
 0001:0000facc       ??_C@_0L@NPHFGOKO@__thiscall?$AA@ 10010acc     libvcruntime:undname.obj
 0001:0000fad8       ??_C@_0L@JMKHOMEK@__fastcall?$AA@ 10010ad8     libvcruntime:undname.obj
 0001:0000fae4       ??_C@_0N@BCKKPABJ@__vectorcall?$AA@ 10010ae4     libvcruntime:undname.obj
 0001:0000faf4       ??_C@_09HIJEGCPM@__clrcall?$AA@ 10010af4     libvcruntime:undname.obj
 0001:0000fb00       ??_C@_06GHPCKEAG@__eabi?$AA@ 10010b00     libvcruntime:undname.obj
 0001:0000fb08       ??_C@_07JOMMBBKO@__ptr64?$AA@ 10010b08     libvcruntime:undname.obj
 0001:0000fb10       ??_C@_0L@PILCLIHE@__restrict?$AA@ 10010b10     libvcruntime:undname.obj
 0001:0000fb1c       ??_C@_0M@GFIIJFMG@__unaligned?$AA@ 10010b1c     libvcruntime:undname.obj
 0001:0000fb28       ??_C@_09DHDLOLLB@restrict?$CI?$AA@ 10010b28     libvcruntime:undname.obj
 0001:0000fb34       ??_C@_04NIHEBCM@?5new?$AA@ 10010b34     libvcruntime:undname.obj
 0001:0000fb3c       ??_C@_07FPCDHGMM@?5delete?$AA@ 10010b3c     libvcruntime:undname.obj
 0001:0000fb44       ??_C@_01NEMOKFLO@?$DN?$AA@ 10010b44     libvcruntime:undname.obj
 0001:0000fb48       ??_C@_02GPIOPFAK@?$DO?$DO?$AA@ 10010b48     libvcruntime:undname.obj
 0001:0000fb4c       ??_C@_02FODMEDOG@?$DM?$DM?$AA@ 10010b4c     libvcruntime:undname.obj
 0001:0000fb50       ??_C@_01DCLJPIOD@?$CB?$AA@ 10010b50     libvcruntime:undname.obj
 0001:0000fb54       ??_C@_02EGOFBIJA@?$DN?$DN?$AA@ 10010b54     libvcruntime:undname.obj
 0001:0000fb58       ??_C@_02FDNJECIE@?$CB?$DN?$AA@ 10010b58     libvcruntime:undname.obj
 0001:0000fb5c       ??_C@_02GPECMEKF@?$FL?$FN?$AA@ 10010b5c     libvcruntime:undname.obj
 0001:0000fb60       ??_C@_08LHJFAFGD@operator?$AA@ 10010b60     libvcruntime:undname.obj
 0001:0000fb6c       ??_C@_02HBOOOICD@?9?$DO?$AA@ 10010b6c     libvcruntime:undname.obj
 0001:0000fb70       ??_C@_01NBENCBCI@?$CK?$AA@ 10010b70     libvcruntime:undname.obj
 0001:0000fb74       ??_C@_02ECNGHCIF@?$CL?$CL?$AA@ 10010b74     libvcruntime:undname.obj
 0001:0000fb78       ??_C@_02BAABKJLB@?9?9?$AA@ 10010b78     libvcruntime:undname.obj
 0001:0000fb7c       ??_C@_01JOAMLHOP@?9?$AA@   10010b7c     libvcruntime:undname.obj
 0001:0000fb80       ??_C@_01MIFGBAGJ@?$CL?$AA@ 10010b80     libvcruntime:undname.obj
 0001:0000fb84       ??_C@_01HNPIGOCE@?$CG?$AA@ 10010b84     libvcruntime:undname.obj
 0001:0000fb88       ??_C@_03MNHNFDLC@?9?$DO?$CK?$AA@ 10010b88     libvcruntime:undname.obj
 0001:0000fb8c       ??_C@_01FGNFDNOH@?$CF?$AA@ 10010b8c     libvcruntime:undname.obj
 0001:0000fb90       ??_C@_01MNNFJEPP@?$DM?$AA@ 10010b90     libvcruntime:undname.obj
 0001:0000fb94       ??_C@_02EHCHHCKH@?$DM?$DN?$AA@ 10010b94     libvcruntime:undname.obj
 0001:0000fb98       ??_C@_01PPODPGHN@?$DO?$AA@ 10010b98     libvcruntime:undname.obj
 0001:0000fb9c       ??_C@_02EEKDKGMJ@?$DO?$DN?$AA@ 10010b9c     libvcruntime:undname.obj
 0001:0000fba0       ??_C@_01IHBHIGKO@?0?$AA@   10010ba0     libvcruntime:undname.obj
 0001:0000fba4       ??_C@_02HCKGKOFO@?$CI?$CJ?$AA@ 10010ba4     libvcruntime:undname.obj
 0001:0000fba8       ??_C@_01PJKLJHI@?$HO?$AA@  10010ba8     libvcruntime:undname.obj
 0001:0000fbac       ??_C@_01JKBOJNNK@?$FO?$AA@ 10010bac     libvcruntime:undname.obj
 0001:0000fbb0       ??_C@_01DNKMNLPK@?$HM?$AA@ 10010bb0     libvcruntime:undname.obj
 0001:0000fbb4       ??_C@_02PPKAJPJL@?$CG?$CG?$AA@ 10010bb4     libvcruntime:undname.obj
 0001:0000fbb8       ??_C@_02NONPIBCD@?$HM?$HM?$AA@ 10010bb8     libvcruntime:undname.obj
 0001:0000fbbc       ??_C@_02FPIMKNGF@?$CK?$DN?$AA@ 10010bbc     libvcruntime:undname.obj
 0001:0000fbc0       ??_C@_02FOEOMHFC@?$CL?$DN?$AA@ 10010bc0     libvcruntime:undname.obj
 0001:0000fbc4       ??_C@_02FKMDLLOA@?9?$DN?$AA@ 10010bc4     libvcruntime:undname.obj
 0001:0000fbc8       ??_C@_02FJEHGPIO@?1?$DN?$AA@ 10010bc8     libvcruntime:undname.obj
 0001:0000fbcc       ??_C@_02FENAOKFI@?$CF?$DN?$AA@ 10010bcc     libvcruntime:undname.obj
 0001:0000fbd0       ??_C@_03IKFCCPFF@?$DO?$DO?$DN?$AA@ 10010bd0     libvcruntime:undname.obj
 0001:0000fbd4       ??_C@_03CDNPDDLA@?$DM?$DM?$DN?$AA@ 10010bd4     libvcruntime:undname.obj
 0001:0000fbd8       ??_C@_02FGJGFEAB@?$CG?$DN?$AA@ 10010bd8     libvcruntime:undname.obj
 0001:0000fbdc       ??_C@_02DHLNPPGH@?$HM?$DN?$AA@ 10010bdc     libvcruntime:undname.obj
 0001:0000fbe0       ??_C@_02MHEGNOJ@?$FO?$DN?$AA@ 10010be0     libvcruntime:undname.obj
 0001:0000fbe4       ??_C@_09IFPLHPGF@?$GAvftable?8?$AA@ 10010be4     libvcruntime:undname.obj
 0001:0000fbf0       ??_C@_09BLBHBJP@?$GAvbtable?8?$AA@ 10010bf0     libvcruntime:undname.obj
 0001:0000fbfc       ??_C@_07FEEIOKP@?$GAvcall?8?$AA@ 10010bfc     libvcruntime:undname.obj
 0001:0000fc04       ??_C@_08LLFFHHDJ@?$GAtypeof?8?$AA@ 10010c04     libvcruntime:undname.obj
 0001:0000fc10       ??_C@_0BF@KDPPACIK@?$GAlocal?5static?5guard?8?$AA@ 10010c10     libvcruntime:undname.obj
 0001:0000fc28       ??_C@_08OBABFOLI@?$GAstring?8?$AA@ 10010c28     libvcruntime:undname.obj
 0001:0000fc34       ??_C@_0BD@JDLKDPAB@?$GAvbase?5destructor?8?$AA@ 10010c34     libvcruntime:undname.obj
 0001:0000fc48       ??_C@_0BN@DEGPLNFK@?$GAvector?5deleting?5destructor?8?$AA@ 10010c48     libvcruntime:undname.obj
 0001:0000fc68       ??_C@_0BO@OBMKPJIG@?$GAdefault?5constructor?5closure?8?$AA@ 10010c68     libvcruntime:undname.obj
 0001:0000fc88       ??_C@_0BN@IMDCHIKM@?$GAscalar?5deleting?5destructor?8?$AA@ 10010c88     libvcruntime:undname.obj
 0001:0000fca8       ??_C@_0BO@PFGOCPJJ@?$GAvector?5constructor?5iterator?8?$AA@ 10010ca8     libvcruntime:undname.obj
 0001:0000fcc8       ??_C@_0BN@LFPFMEDL@?$GAvector?5destructor?5iterator?8?$AA@ 10010cc8     libvcruntime:undname.obj
 0001:0000fce8       ??_C@_0CE@IKBNEHA@?$GAvector?5vbase?5constructor?5iterat@ 10010ce8     libvcruntime:undname.obj
 0001:0000fd0c       ??_C@_0BL@NILFHHPC@?$GAvirtual?5displacement?5map?8?$AA@ 10010d0c     libvcruntime:undname.obj
 0001:0000fd28       ??_C@_0CB@JONCMFFK@?$GAeh?5vector?5constructor?5iterator?8@ 10010d28     libvcruntime:undname.obj
 0001:0000fd4c       ??_C@_0CA@GCEOPDGL@?$GAeh?5vector?5destructor?5iterator?8?$AA@ 10010d4c     libvcruntime:undname.obj
 0001:0000fd6c       ??_C@_0CH@OOJPLCPH@?$GAeh?5vector?5vbase?5constructor?5ite@ 10010d6c     libvcruntime:undname.obj
 0001:0000fd94       ??_C@_0BL@LLKPOHJI@?$GAcopy?5constructor?5closure?8?$AA@ 10010d94     libvcruntime:undname.obj
 0001:0000fdb0       ??_C@_0BA@KBCDOMBN@?$GAudt?5returning?8?$AA@ 10010db0     libvcruntime:undname.obj
 0001:0000fdc0       ??_C@_03KLGMFNMG@?$GAEH?$AA@ 10010dc0     libvcruntime:undname.obj
 0001:0000fdc4       ??_C@_05KHLCHHI@?$GARTTI?$AA@ 10010dc4     libvcruntime:undname.obj
 0001:0000fdcc       ??_C@_0BA@KKLDJDLB@?$GAlocal?5vftable?8?$AA@ 10010dcc     libvcruntime:undname.obj
 0001:0000fddc       ??_C@_0CE@IIHCMGGL@?$GAlocal?5vftable?5constructor?5closu@ 10010ddc     libvcruntime:undname.obj
 0001:0000fe00       ??_C@_06FHBGPFGH@?5new?$FL?$FN?$AA@ 10010e00     libvcruntime:undname.obj
 0001:0000fe08       ??_C@_09LBNFPBCA@?5delete?$FL?$FN?$AA@ 10010e08     libvcruntime:undname.obj
 0001:0000fe14       ??_C@_0P@HJKNJFNN@?$GAomni?5callsig?8?$AA@ 10010e14     libvcruntime:undname.obj
 0001:0000fe24       ??_C@_0BL@CNOONJFP@?$GAplacement?5delete?5closure?8?$AA@ 10010e24     libvcruntime:undname.obj
 0001:0000fe40       ??_C@_0BN@CKNJLHMB@?$GAplacement?5delete?$FL?$FN?5closure?8?$AA@ 10010e40     libvcruntime:undname.obj
 0001:0000fe60       ??_C@_0CG@CFDHKGGD@?$GAmanaged?5vector?5constructor?5iter@ 10010e60     libvcruntime:undname.obj
 0001:0000fe88       ??_C@_0CF@IMGKMJNO@?$GAmanaged?5vector?5destructor?5itera@ 10010e88     libvcruntime:undname.obj
 0001:0000feb0       ??_C@_0CG@HLDDJMAG@?$GAeh?5vector?5copy?5constructor?5iter@ 10010eb0     libvcruntime:undname.obj
 0001:0000fed8       ??_C@_0CM@FCBBDIGB@?$GAeh?5vector?5vbase?5copy?5constructo@ 10010ed8     libvcruntime:undname.obj
 0001:0000ff04       ??_C@_0BL@CLIPGLGB@?$GAdynamic?5initializer?5for?5?8?$AA@ 10010f04     libvcruntime:undname.obj
 0001:0000ff20       ??_C@_0CB@PDBIFEP@?$GAdynamic?5atexit?5destructor?5for?5?8@ 10010f20     libvcruntime:undname.obj
 0001:0000ff44       ??_C@_0CD@CGAJBKEJ@?$GAvector?5copy?5constructor?5iterato@ 10010f44     libvcruntime:undname.obj
 0001:0000ff68       ??_C@_0CJ@GJELGAMM@?$GAvector?5vbase?5copy?5constructor?5i@ 10010f68     libvcruntime:undname.obj
 0001:0000ff94       ??_C@_0CL@FGIJHLCE@?$GAmanaged?5vector?5copy?5constructor@ 10010f94     libvcruntime:undname.obj
 0001:0000ffc0       ??_C@_0BM@PMGGMLDN@?$GAlocal?5static?5thread?5guard?8?$AA@ 10010fc0     libvcruntime:undname.obj
 0001:0000ffdc       ??_C@_0N@BDNMDMOL@operator?5?$CC?$CC?5?$AA@ 10010fdc     libvcruntime:undname.obj
 0001:0000ffec       ??_C@_0BC@DAFEJGAK@?5Type?5Descriptor?8?$AA@ 10010fec     libvcruntime:undname.obj
 0001:00010000       ??_C@_0BM@LDKODKLH@?5Base?5Class?5Descriptor?5at?5?$CI?$AA@ 10011000     libvcruntime:undname.obj
 0001:0001001c       ??_C@_0BD@LGICGFMM@?5Base?5Class?5Array?8?$AA@ 1001101c     libvcruntime:undname.obj
 0001:00010030       ??_C@_0BN@MECKDCOJ@?5Class?5Hierarchy?5Descriptor?8?$AA@ 10011030     libvcruntime:undname.obj
 0001:00010050       ??_C@_0BK@CFCOFLF@?5Complete?5Object?5Locator?8?$AA@ 10011050     libvcruntime:undname.obj
 0001:00010070       _standard_lookup_table     10011070     libucrt:output.obj
 0001:000100cc       ??_C@_06OJHGLDPL@?$CInull?$CJ?$AA@ 100110cc     libucrt:output.obj
 0001:000100d4       ??_C@_1O@CEDCILHN@?$AA?$CI?$AAn?$AAu?$AAl?$AAl?$AA?$CJ?$AA?$AA@ 100110d4     libucrt:output.obj
 0001:00010250       ??_C@_0EA@FCLIIPNN@Visual?5C?$CL?$CL?5CRT?3?5Not?5enough?5memor@ 10011250     libucrt:strerror.obj
 0001:000102d0       ?large_power_data@?1??multiply_by_power_of_ten@__crt_strtox@@YA_NAAUbig_integer@2@I@Z@4QBIB 100112d0     libucrt:input.obj
 0001:00010bd8       ?large_power_indices@?1??multiply_by_power_of_ten@__crt_strtox@@YA_NAAUbig_integer@2@I@Z@4QBUunpack_index@?1??12@YA_N0I@Z@B 10011bd8     libucrt:input.obj
 0001:00010c70       ?small_powers_of_ten@?6??multiply_by_power_of_ten@__crt_strtox@@YA_NAAUbig_integer@2@I@Z@4QBIB 10011c70     libucrt:input.obj
 0001:00010c98       ??_C@_1GE@DPGDJKLM@?$AAm?$AAi?$AAn?$AAk?$AAe?$AAr?$AAn?$AAe?$AAl?$AA?2?$AAc?$AAr?$AAt?$AAs?$AA?2?$AAu?$AAc?$AAr?$AAt?$AA?2?$AAi?$AAn?$AAc?$AA?2?$AAc?$AAo?$AAr?$AAe?$AAc?$AAr?$AAt?$AA_@ 10011c98     libucrt:input.obj
 0001:00010d00       ??_C@_1FM@FELNCOBF@?$AA_?$AA_?$AAc?$AAr?$AAt?$AA_?$AAs?$AAt?$AAr?$AAt?$AAo?$AAx?$AA?3?$AA?3?$AAf?$AAl?$AAo?$AAa?$AAt?$AAi?$AAn?$AAg?$AA_?$AAp?$AAo?$AAi?$AAn?$AAt?$AA_?$AAv?$AAa?$AAl@ 10011d00     libucrt:input.obj
 0001:00010d5c       ??_C@_1BG@GEMHBGAF@?$AA_?$AAi?$AAs?$AA_?$AAd?$AAo?$AAu?$AAb?$AAl?$AAe?$AA?$AA@ 10011d5c     libucrt:input.obj
 0001:00010d78       ??_C@_1FK@JOJELFFO@?$AA_?$AA_?$AAc?$AAr?$AAt?$AA_?$AAs?$AAt?$AAr?$AAt?$AAo?$AAx?$AA?3?$AA?3?$AAf?$AAl?$AAo?$AAa?$AAt?$AAi?$AAn?$AAg?$AA_?$AAp?$AAo?$AAi?$AAn?$AAt?$AA_?$AAv?$AAa?$AAl@ 10011d78     libucrt:input.obj
 0001:00010dd4       ??_C@_1BI@BANMPGJI@?$AA?$CB?$AA_?$AAi?$AAs?$AA_?$AAd?$AAo?$AAu?$AAb?$AAl?$AAe?$AA?$AA@ 10011dd4     libucrt:input.obj
 0001:00010df0       ?constraints@?1??is_length_valid@__crt_stdio_input@@YA_NW4conversion_mode@2@W4length_modifier@2@@Z@4QAY0M@$$CBEA 10011df0     libucrt:input.obj
 0001:00010e68       ?inf_uppercase@?2???$parse_floating_point_possible_infinity@DV?$input_adapter_character_source@V?$stream_input_adapter@D@__crt_stdio_input@@@__crt_strtox@@_K@__crt_strtox@@YA?AW4floating_point_parse_result@1@AADAAV?$input_adapter_character_source@V?$stream_input_adapter@D@__crt_stdio_input@@@1@_K@Z@4QBDB 10011e68     libucrt:input.obj
 0001:00010e6c       ?inf_lowercase@?2???$parse_floating_point_possible_infinity@DV?$input_adapter_character_source@V?$stream_input_adapter@D@__crt_stdio_input@@@__crt_strtox@@_K@__crt_strtox@@YA?AW4floating_point_parse_result@1@AADAAV?$input_adapter_character_source@V?$stream_input_adapter@D@__crt_stdio_input@@@1@_K@Z@4QBDB 10011e6c     libucrt:input.obj
 0001:00010e70       ?inity_uppercase@?5???$parse_floating_point_possible_infinity@DV?$input_adapter_character_source@V?$stream_input_adapter@D@__crt_stdio_input@@@__crt_strtox@@_K@__crt_strtox@@YA?AW4floating_point_parse_result@1@AADAAV?$input_adapter_character_source@V?$stream_input_adapter@D@__crt_stdio_input@@@1@_K@Z@4QBDB 10011e70     libucrt:input.obj
 0001:00010e78       ?inity_lowercase@?5???$parse_floating_point_possible_infinity@DV?$input_adapter_character_source@V?$stream_input_adapter@D@__crt_stdio_input@@@__crt_strtox@@_K@__crt_strtox@@YA?AW4floating_point_parse_result@1@AADAAV?$input_adapter_character_source@V?$stream_input_adapter@D@__crt_stdio_input@@@1@_K@Z@4QBDB 10011e78     libucrt:input.obj
 0001:00010e80       ?uppercase@?2???$parse_floating_point_possible_nan@DV?$input_adapter_character_source@V?$stream_input_adapter@D@__crt_stdio_input@@@__crt_strtox@@_K@__crt_strtox@@YA?AW4floating_point_parse_result@1@AADAAV?$input_adapter_character_source@V?$stream_input_adapter@D@__crt_stdio_input@@@1@_K@Z@4QBDB 10011e80     libucrt:input.obj
 0001:00010e84       ?lowercase@?2???$parse_floating_point_possible_nan@DV?$input_adapter_character_source@V?$stream_input_adapter@D@__crt_stdio_input@@@__crt_strtox@@_K@__crt_strtox@@YA?AW4floating_point_parse_result@1@AADAAV?$input_adapter_character_source@V?$stream_input_adapter@D@__crt_stdio_input@@@1@_K@Z@4QBDB 10011e84     libucrt:input.obj
 0001:00010e88       ?uppercase@?1???$parse_floating_point_possible_nan_is_snan@DV?$input_adapter_character_source@V?$stream_input_adapter@D@__crt_stdio_input@@@__crt_strtox@@@__crt_strtox@@YA_NAADAAV?$input_adapter_character_source@V?$stream_input_adapter@D@__crt_stdio_input@@@1@@Z@4QBDB 10011e88     libucrt:input.obj
 0001:00010e90       ?lowercase@?1???$parse_floating_point_possible_nan_is_snan@DV?$input_adapter_character_source@V?$stream_input_adapter@D@__crt_stdio_input@@@__crt_strtox@@@__crt_strtox@@YA_NAADAAV?$input_adapter_character_source@V?$stream_input_adapter@D@__crt_stdio_input@@@1@@Z@4QBDB 10011e90     libucrt:input.obj
 0001:00010e98       ?uppercase@?1???$parse_floating_point_possible_nan_is_ind@DV?$input_adapter_character_source@V?$stream_input_adapter@D@__crt_stdio_input@@@__crt_strtox@@@__crt_strtox@@YA_NAADAAV?$input_adapter_character_source@V?$stream_input_adapter@D@__crt_stdio_input@@@1@@Z@4QBDB 10011e98     libucrt:input.obj
 0001:00010e9c       ?lowercase@?1???$parse_floating_point_possible_nan_is_ind@DV?$input_adapter_character_source@V?$stream_input_adapter@D@__crt_stdio_input@@@__crt_strtox@@@__crt_strtox@@YA_NAADAAV?$input_adapter_character_source@V?$stream_input_adapter@D@__crt_stdio_input@@@1@@Z@4QBDB 10011e9c     libucrt:input.obj
 0001:00010ec8       ___acrt_exception_action_table 10011ec8     libucrt:exception_filter.obj
 0001:00010f58       ___acrt_signal_action_table_count 10011f58     libucrt:exception_filter.obj
 0001:00010f5c       ___acrt_signal_action_first_fpe_index 10011f5c     libucrt:exception_filter.obj
 0001:00010f60       ___acrt_signal_action_fpe_count 10011f60     libucrt:exception_filter.obj
 0001:00010f64       ??_C@_1BI@BGOHAHKC@?$AAm?$AAs?$AAc?$AAo?$AAr?$AAe?$AAe?$AA?4?$AAd?$AAl?$AAl?$AA?$AA@ 10011f64     libucrt:exit.obj
 0001:00010f7c       ??_C@_0P@MIGLKIOC@CorExitProcess?$AA@ 10011f7c     libucrt:exit.obj
 0001:00011008       ??_C@_03OEIAHPBN@INF?$AA@  10012008     libucrt:cvt.obj
 0001:0001100c       ??_C@_03OJHLLCGB@inf?$AA@  1001200c     libucrt:cvt.obj
 0001:00011010       ??_C@_03LKNCIKJB@NAN?$AA@  10012010     libucrt:cvt.obj
 0001:00011014       ??_C@_03LHCJEHON@nan?$AA@  10012014     libucrt:cvt.obj
 0001:00011018       ??_C@_09OFJJIMPC@NAN?$CISNAN?$CJ?$AA@ 10012018     libucrt:cvt.obj
 0001:00011024       ??_C@_09IPFBKMDL@nan?$CIsnan?$CJ?$AA@ 10012024     libucrt:cvt.obj
 0001:00011030       ??_C@_08IKHNHAJ@NAN?$CIIND?$CJ?$AA@ 10012030     libucrt:cvt.obj
 0001:0001103c       ??_C@_08OFCDMILK@nan?$CIind?$CJ?$AA@ 1001203c     libucrt:cvt.obj
 0001:00011048       ??_C@_05KLBDPFGC@e?$CL000?$AA@ 10012048     libucrt:cvt.obj
 0001:00011050       ??_C@_03KOEHGMDN@Sun?$AA@  10012050     libucrt:nlsdata.obj
 0001:00011054       ??_C@_03PDAGKDH@Mon?$AA@   10012054     libucrt:nlsdata.obj
 0001:00011058       ??_C@_03NAGEINEP@Tue?$AA@  10012058     libucrt:nlsdata.obj
 0001:0001105c       ??_C@_03MHOMLAJA@Wed?$AA@  1001205c     libucrt:nlsdata.obj
 0001:00011060       ??_C@_03IOFIKPDN@Thu?$AA@  10012060     libucrt:nlsdata.obj
 0001:00011064       ??_C@_03IDIOELNC@Fri?$AA@  10012064     libucrt:nlsdata.obj
 0001:00011068       ??_C@_03FEFJNEK@Sat?$AA@   10012068     libucrt:nlsdata.obj
 0001:0001106c       ??_C@_06OOPIFAJ@Sunday?$AA@ 1001206c     libucrt:nlsdata.obj
 0001:00011074       ??_C@_06JLEDEDGH@Monday?$AA@ 10012074     libucrt:nlsdata.obj
 0001:0001107c       ??_C@_07BAAGCFCM@Tuesday?$AA@ 1001207c     libucrt:nlsdata.obj
 0001:00011084       ??_C@_09DLIGFAKA@Wednesday?$AA@ 10012084     libucrt:nlsdata.obj
 0001:00011090       ??_C@_08HACCIKIA@Thursday?$AA@ 10012090     libucrt:nlsdata.obj
 0001:0001109c       ??_C@_06JECMNKMI@Friday?$AA@ 1001209c     libucrt:nlsdata.obj
 0001:000110a4       ??_C@_08INBOOONO@Saturday?$AA@ 100120a4     libucrt:nlsdata.obj
 0001:000110b0       ??_C@_03JIHJHPIE@Jan?$AA@  100120b0     libucrt:nlsdata.obj
 0001:000110b4       ??_C@_03HJBDCHOM@Feb?$AA@  100120b4     libucrt:nlsdata.obj
 0001:000110b8       ??_C@_03ODNJBKGA@Mar?$AA@  100120b8     libucrt:nlsdata.obj
 0001:000110bc       ??_C@_03LEOLGMJP@Apr?$AA@  100120bc     libucrt:nlsdata.obj
 0001:000110c0       ??_C@_03CNMDKL@May?$AA@    100120c0     libucrt:nlsdata.obj
 0001:000110c4       ??_C@_03IDFGHECI@Jun?$AA@  100120c4     libucrt:nlsdata.obj
 0001:000110c8       ??_C@_03LBGABGKK@Jul?$AA@  100120c8     libucrt:nlsdata.obj
 0001:000110cc       ??_C@_03IFJFEIGA@Aug?$AA@  100120cc     libucrt:nlsdata.obj
 0001:000110d0       ??_C@_03GGCAPAJC@Sep?$AA@  100120d0     libucrt:nlsdata.obj
 0001:000110d4       ??_C@_03BMAOKBAD@Oct?$AA@  100120d4     libucrt:nlsdata.obj
 0001:000110d8       ??_C@_03JPJOFNIA@Nov?$AA@  100120d8     libucrt:nlsdata.obj
 0001:000110dc       ??_C@_03MKABNOCG@Dec?$AA@  100120dc     libucrt:nlsdata.obj
 0001:000110e0       ??_C@_07CGJPFGJA@January?$AA@ 100120e0     libucrt:nlsdata.obj
 0001:000110e8       ??_C@_08GNJGEPFN@February?$AA@ 100120e8     libucrt:nlsdata.obj
 0001:000110f4       ??_C@_05HPCKOFNC@March?$AA@ 100120f4     libucrt:nlsdata.obj
 0001:000110fc       ??_C@_05DMJDNLEJ@April?$AA@ 100120fc     libucrt:nlsdata.obj
 0001:00011104       ??_C@_04CNLMGBGM@June?$AA@ 10012104     libucrt:nlsdata.obj
 0001:0001110c       ??_C@_04MIEPOIFP@July?$AA@ 1001210c     libucrt:nlsdata.obj
 0001:00011114       ??_C@_06LBBHFDDG@August?$AA@ 10012114     libucrt:nlsdata.obj
 0001:0001111c       ??_C@_09BHHEALKD@September?$AA@ 1001211c     libucrt:nlsdata.obj
 0001:00011128       ??_C@_07JJNFCEND@October?$AA@ 10012128     libucrt:nlsdata.obj
 0001:00011130       ??_C@_08HCHEGEOA@November?$AA@ 10012130     libucrt:nlsdata.obj
 0001:0001113c       ??_C@_08EDHMEBNP@December?$AA@ 1001213c     libucrt:nlsdata.obj
 0001:00011148       ??_C@_02DEDBPAFC@AM?$AA@   10012148     libucrt:nlsdata.obj
 0001:0001114c       ??_C@_02CJNFDJBF@PM?$AA@   1001214c     libucrt:nlsdata.obj
 0001:00011150       ??_C@_08BPBNCDIB@MM?1dd?1yy?$AA@ 10012150     libucrt:nlsdata.obj
 0001:0001115c       ??_C@_0BE@CKGJFCPC@dddd?0?5MMMM?5dd?0?5yyyy?$AA@ 1001215c     libucrt:nlsdata.obj
 0001:00011170       ??_C@_08JCCMCCIL@HH?3mm?3ss?$AA@ 10012170     libucrt:nlsdata.obj
 0001:0001117c       ??_C@_17MBGCMIPB@?$AAS?$AAu?$AAn?$AA?$AA@ 1001217c     libucrt:nlsdata.obj
 0001:00011184       ??_C@_17KBOMKBF@?$AAM?$AAo?$AAn?$AA?$AA@ 10012184     libucrt:nlsdata.obj
 0001:0001118c       ??_C@_17BMKGEGOJ@?$AAT?$AAu?$AAe?$AA?$AA@ 1001218c     libucrt:nlsdata.obj
 0001:00011194       ??_C@_17CJEDCEPE@?$AAW?$AAe?$AAd?$AA?$AA@ 10012194     libucrt:nlsdata.obj
 0001:0001119c       ??_C@_17PDPHAADD@?$AAT?$AAh?$AAu?$AA?$AA@ 1001219c     libucrt:nlsdata.obj
 0001:000111a4       ??_C@_17HFOLPPLP@?$AAF?$AAr?$AAi?$AA?$AA@ 100121a4     libucrt:nlsdata.obj
 0001:000111ac       ??_C@_17GGIBDPIH@?$AAS?$AAa?$AAt?$AA?$AA@ 100121ac     libucrt:nlsdata.obj
 0001:000111b4       ??_C@_1O@IHNHDHPB@?$AAS?$AAu?$AAn?$AAd?$AAa?$AAy?$AA?$AA@ 100121b4     libucrt:nlsdata.obj
 0001:000111c4       ??_C@_1O@MMNBFLIA@?$AAM?$AAo?$AAn?$AAd?$AAa?$AAy?$AA?$AA@ 100121c4     libucrt:nlsdata.obj
 0001:000111d4       ??_C@_1BA@ENFBFFEK@?$AAT?$AAu?$AAe?$AAs?$AAd?$AAa?$AAy?$AA?$AA@ 100121d4     libucrt:nlsdata.obj
 0001:000111e4       ??_C@_1BE@EBOGMDOH@?$AAW?$AAe?$AAd?$AAn?$AAe?$AAs?$AAd?$AAa?$AAy?$AA?$AA@ 100121e4     libucrt:nlsdata.obj
 0001:000111f8       ??_C@_1BC@HHMNLIHE@?$AAT?$AAh?$AAu?$AAr?$AAs?$AAd?$AAa?$AAy?$AA?$AA@ 100121f8     libucrt:nlsdata.obj
 0001:0001120c       ??_C@_1O@PDICJHAG@?$AAF?$AAr?$AAi?$AAd?$AAa?$AAy?$AA?$AA@ 1001220c     libucrt:nlsdata.obj
 0001:0001121c       ??_C@_1BC@ENMNNPAJ@?$AAS?$AAa?$AAt?$AAu?$AAr?$AAd?$AAa?$AAy?$AA?$AA@ 1001221c     libucrt:nlsdata.obj
 0001:00011230       ??_C@_17DKNBKCHM@?$AAJ?$AAa?$AAn?$AA?$AA@ 10012230     libucrt:nlsdata.obj
 0001:00011238       ??_C@_17LMDJEKJN@?$AAF?$AAe?$AAb?$AA?$AA@ 10012238     libucrt:nlsdata.obj
 0001:00011240       ??_C@_17CKNLEDEC@?$AAM?$AAa?$AAr?$AA?$AA@ 10012240     libucrt:nlsdata.obj
 0001:00011248       ??_C@_17LFPOIHDD@?$AAA?$AAp?$AAr?$AA?$AA@ 10012248     libucrt:nlsdata.obj
 0001:00011250       ??_C@_17PNNKMEED@?$AAM?$AAa?$AAy?$AA?$AA@ 10012250     libucrt:nlsdata.obj
 0001:00011258       ??_C@_17KCJGOCPB@?$AAJ?$AAu?$AAn?$AA?$AA@ 10012258     libucrt:nlsdata.obj
 0001:00011260       ??_C@_17IJPCKHK@?$AAJ?$AAu?$AAl?$AA?$AA@ 10012260     libucrt:nlsdata.obj
 0001:00011268       ??_C@_17ICPELBCN@?$AAA?$AAu?$AAg?$AA?$AA@ 10012268     libucrt:nlsdata.obj
 0001:00011270       ??_C@_17HCHCOKMG@?$AAS?$AAe?$AAp?$AA?$AA@ 10012270     libucrt:nlsdata.obj
 0001:00011278       ??_C@_17FNLKOI@?$AAO?$AAc?$AAt?$AA?$AA@ 10012278     libucrt:nlsdata.obj
 0001:00011280       ??_C@_17BBDMLCIG@?$AAN?$AAo?$AAv?$AA?$AA@ 10012280     libucrt:nlsdata.obj
 0001:00011288       ??_C@_17EGKACKIF@?$AAD?$AAe?$AAc?$AA?$AA@ 10012288     libucrt:nlsdata.obj
 0001:00011290       ??_C@_1BA@EFMEIEBA@?$AAJ?$AAa?$AAn?$AAu?$AAa?$AAr?$AAy?$AA?$AA@ 10012290     libucrt:nlsdata.obj
 0001:000112a0       ??_C@_1BC@JGDDFFAM@?$AAF?$AAe?$AAb?$AAr?$AAu?$AAa?$AAr?$AAy?$AA?$AA@ 100122a0     libucrt:nlsdata.obj
 0001:000112b4       ??_C@_1M@IKEENEDF@?$AAM?$AAa?$AAr?$AAc?$AAh?$AA?$AA@ 100122b4     libucrt:nlsdata.obj
 0001:000112c0       ??_C@_1M@GJNLMHFD@?$AAA?$AAp?$AAr?$AAi?$AAl?$AA?$AA@ 100122c0     libucrt:nlsdata.obj
 0001:000112cc       ??_C@_19EPFLPGAP@?$AAJ?$AAu?$AAn?$AAe?$AA?$AA@ 100122cc     libucrt:nlsdata.obj
 0001:000112d8       ??_C@_19BIFMLPCD@?$AAJ?$AAu?$AAl?$AAy?$AA?$AA@ 100122d8     libucrt:nlsdata.obj
 0001:000112e4       ??_C@_1O@PAHLKOAC@?$AAA?$AAu?$AAg?$AAu?$AAs?$AAt?$AA?$AA@ 100122e4     libucrt:nlsdata.obj
 0001:000112f4       ??_C@_1BE@DKAAMBJL@?$AAS?$AAe?$AAp?$AAt?$AAe?$AAm?$AAb?$AAe?$AAr?$AA?$AA@ 100122f4     libucrt:nlsdata.obj
 0001:00011308       ??_C@_1BA@EPANDLNG@?$AAO?$AAc?$AAt?$AAo?$AAb?$AAe?$AAr?$AA?$AA@ 10012308     libucrt:nlsdata.obj
 0001:00011318       ??_C@_1BC@BGLIFPF@?$AAN?$AAo?$AAv?$AAe?$AAm?$AAb?$AAe?$AAr?$AA?$AA@ 10012318     libucrt:nlsdata.obj
 0001:0001132c       ??_C@_1BC@FEMKIFH@?$AAD?$AAe?$AAc?$AAe?$AAm?$AAb?$AAe?$AAr?$AA?$AA@ 1001232c     libucrt:nlsdata.obj
 0001:00011340       ??_C@_15ODEHAHHF@?$AAA?$AAM?$AA?$AA@ 10012340     libucrt:nlsdata.obj
 0001:00011348       ??_C@_15CLMNNGEL@?$AAP?$AAM?$AA?$AA@ 10012348     libucrt:nlsdata.obj
 0001:00011350       ??_C@_1BC@IEBCMHCM@?$AAM?$AAM?$AA?1?$AAd?$AAd?$AA?1?$AAy?$AAy?$AA?$AA@ 10012350     libucrt:nlsdata.obj
 0001:00011364       ??_C@_1CI@KNAKOEBC@?$AAd?$AAd?$AAd?$AAd?$AA?0?$AA?5?$AAM?$AAM?$AAM?$AAM?$AA?5?$AAd?$AAd?$AA?0?$AA?5?$AAy?$AAy?$AAy?$AAy?$AA?$AA@ 10012364     libucrt:nlsdata.obj
 0001:0001138c       ??_C@_1BC@GDGBMEMK@?$AAH?$AAH?$AA?3?$AAm?$AAm?$AA?3?$AAs?$AAs?$AA?$AA@ 1001238c     libucrt:nlsdata.obj
 0001:000113a0       ??_C@_1M@BMHNFIME@?$AAe?$AAn?$AA?9?$AAU?$AAS?$AA?$AA@ 100123a0     libucrt:nlsdata.obj
 0001:000113b0       ___lc_time_c               100123b0     libucrt:nlsdata.obj
 0001:00011514       ?ccs@?BL@???$__acrt_stdio_parse_mode@_W@@YA?AU__acrt_stdio_stream_mode@@QB_W@Z@4QB_WB 10012514     libucrt:openfile.obj
 0001:0001151c       ?utf8_encoding@?BL@???$__acrt_stdio_parse_mode@_W@@YA?AU__acrt_stdio_stream_mode@@QB_W@Z@4QB_WB 1001251c     libucrt:openfile.obj
 0001:00011528       ?utf16_encoding@?BL@???$__acrt_stdio_parse_mode@_W@@YA?AU__acrt_stdio_stream_mode@@QB_W@Z@4QB_WB 10012528     libucrt:openfile.obj
 0001:00011538       ?unicode_encoding@?BL@???$__acrt_stdio_parse_mode@_W@@YA?AU__acrt_stdio_stream_mode@@QB_W@Z@4QB_WB 10012538     libucrt:openfile.obj
 0001:00011560       __sys_errlist              10012560     libucrt:syserr.obj
 0001:00011610       ??_C@_08INEPGKHH@No?5error?$AA@ 10012610     libucrt:syserr.obj
 0001:0001161c       ??_C@_0BI@BJFCGOHL@Operation?5not?5permitted?$AA@ 1001261c     libucrt:syserr.obj
 0001:00011634       ??_C@_0BK@FMDHKPNF@No?5such?5file?5or?5directory?$AA@ 10012634     libucrt:syserr.obj
 0001:00011650       ??_C@_0BA@FKIAIBGA@No?5such?5process?$AA@ 10012650     libucrt:syserr.obj
 0001:00011660       ??_C@_0BK@FJBOAFDK@Interrupted?5function?5call?$AA@ 10012660     libucrt:syserr.obj
 0001:0001167c       ??_C@_0BD@KKNFOBBD@Input?1output?5error?$AA@ 1001267c     libucrt:syserr.obj
 0001:00011690       ??_C@_0BK@DPKMCKJ@No?5such?5device?5or?5address?$AA@ 10012690     libucrt:syserr.obj
 0001:000116ac       ??_C@_0BC@MFFGCDFL@Arg?5list?5too?5long?$AA@ 100126ac     libucrt:syserr.obj
 0001:000116c0       ??_C@_0BC@HKPNECK@Exec?5format?5error?$AA@ 100126c0     libucrt:syserr.obj
 0001:000116d4       ??_C@_0BE@NFGDDCEF@Bad?5file?5descriptor?$AA@ 100126d4     libucrt:syserr.obj
 0001:000116e8       ??_C@_0BD@LOHELEP@No?5child?5processes?$AA@ 100126e8     libucrt:syserr.obj
 0001:000116fc       ??_C@_0CB@EPFKGNAK@Resource?5temporarily?5unavailable@ 100126fc     libucrt:syserr.obj
 0001:00011720       ??_C@_0BB@IMDKMPFB@Not?5enough?5space?$AA@ 10012720     libucrt:syserr.obj
 0001:00011734       ??_C@_0BC@HFNFNKAI@Permission?5denied?$AA@ 10012734     libucrt:syserr.obj
 0001:00011748       ??_C@_0M@LOEHLCJD@Bad?5address?$AA@ 10012748     libucrt:syserr.obj
 0001:00011754       ??_C@_0O@NIPGCINC@Unknown?5error?$AA@ 10012754     libucrt:syserr.obj
 0001:00011764       ??_C@_0BA@BIBLIOEK@Resource?5device?$AA@ 10012764     libucrt:syserr.obj
 0001:00011774       ??_C@_0M@NAAJNNGH@File?5exists?$AA@ 10012774     libucrt:syserr.obj
 0001:00011780       ??_C@_0O@OAMDNOCP@Improper?5link?$AA@ 10012780     libucrt:syserr.obj
 0001:00011790       ??_C@_0P@NLEIANHE@No?5such?5device?$AA@ 10012790     libucrt:syserr.obj
 0001:000117a0       ??_C@_0BA@CJBACOOL@Not?5a?5directory?$AA@ 100127a0     libucrt:syserr.obj
 0001:000117b0       ??_C@_0P@NDHGCGKE@Is?5a?5directory?$AA@ 100127b0     libucrt:syserr.obj
 0001:000117c0       ??_C@_0BB@HMGGCEBG@Invalid?5argument?$AA@ 100127c0     libucrt:syserr.obj
 0001:000117d4       ??_C@_0BO@IIFBODJE@Too?5many?5open?5files?5in?5system?$AA@ 100127d4     libucrt:syserr.obj
 0001:000117f4       ??_C@_0BE@INBJMKGG@Too?5many?5open?5files?$AA@ 100127f4     libucrt:syserr.obj
 0001:00011808       ??_C@_0CE@ONOKNLPF@Inappropriate?5I?1O?5control?5operat@ 10012808     libucrt:syserr.obj
 0001:0001182c       ??_C@_0P@LFMMIPAE@File?5too?5large?$AA@ 1001282c     libucrt:syserr.obj
 0001:0001183c       ??_C@_0BI@FEALHKLD@No?5space?5left?5on?5device?$AA@ 1001283c     libucrt:syserr.obj
 0001:00011854       ??_C@_0N@FEHLOILP@Invalid?5seek?$AA@ 10012854     libucrt:syserr.obj
 0001:00011864       ??_C@_0BG@DDBFNKBH@Read?9only?5file?5system?$AA@ 10012864     libucrt:syserr.obj
 0001:0001187c       ??_C@_0P@PKCJJLLM@Too?5many?5links?$AA@ 1001287c     libucrt:syserr.obj
 0001:0001188c       ??_C@_0M@LHEPIIOM@Broken?5pipe?$AA@ 1001288c     libucrt:syserr.obj
 0001:00011898       ??_C@_0N@MMJPGLJK@Domain?5error?$AA@ 10012898     libucrt:syserr.obj
 0001:000118a8       ??_C@_0BB@FCBJFCAJ@Result?5too?5large?$AA@ 100128a8     libucrt:syserr.obj
 0001:000118bc       ??_C@_0BK@JAEBMJJM@Resource?5deadlock?5avoided?$AA@ 100128bc     libucrt:syserr.obj
 0001:000118d8       ??_C@_0BC@BEDIHIDK@Filename?5too?5long?$AA@ 100128d8     libucrt:syserr.obj
 0001:000118ec       ??_C@_0BD@CLHBCGPB@No?5locks?5available?$AA@ 100128ec     libucrt:syserr.obj
 0001:00011900       ??_C@_0BJ@IHEHINLI@Function?5not?5implemented?$AA@ 10012900     libucrt:syserr.obj
 0001:0001191c       ??_C@_0BE@ICMCHPHH@Directory?5not?5empty?$AA@ 1001291c     libucrt:syserr.obj
 0001:00011930       ??_C@_0BG@KLEAJEFJ@Illegal?5byte?5sequence?$AA@ 10012930     libucrt:syserr.obj
 0001:00011948       __sys_nerr                 10012948     libucrt:syserr.obj
 0001:000119a0       ??_C@_1EG@CNNIPFIM@?$AAa?$AAp?$AAi?$AA?9?$AAm?$AAs?$AA?9?$AAw?$AAi?$AAn?$AA?9?$AAa?$AAp?$AAp?$AAm?$AAo?$AAd?$AAe?$AAl?$AA?9?$AAr?$AAu?$AAn?$AAt?$AAi?$AAm?$AAe?$AA?9?$AAl?$AA1?$AA?9?$AA1@ 100129a0     libucrt:winapi_thunks.obj
 0001:000119e8       ??_C@_1EA@JGEFHKEI@?$AAa?$AAp?$AAi?$AA?9?$AAm?$AAs?$AA?9?$AAw?$AAi?$AAn?$AA?9?$AAc?$AAo?$AAr?$AAe?$AA?9?$AAd?$AAa?$AAt?$AAe?$AAt?$AAi?$AAm?$AAe?$AA?9?$AAl?$AA1?$AA?9?$AA1?$AA?9?$AA1?$AA?$AA@ 100129e8     libucrt:winapi_thunks.obj
 0001:00011a28       ??_C@_1DI@GCIAAENM@?$AAa?$AAp?$AAi?$AA?9?$AAm?$AAs?$AA?9?$AAw?$AAi?$AAn?$AA?9?$AAc?$AAo?$AAr?$AAe?$AA?9?$AAf?$AAi?$AAl?$AAe?$AA?9?$AAl?$AA2?$AA?9?$AA1?$AA?9?$AA1?$AA?$AA@ 10012a28     libucrt:winapi_thunks.obj
 0001:00011a60       ??_C@_1EI@MPIAOHOC@?$AAa?$AAp?$AAi?$AA?9?$AAm?$AAs?$AA?9?$AAw?$AAi?$AAn?$AA?9?$AAc?$AAo?$AAr?$AAe?$AA?9?$AAl?$AAo?$AAc?$AAa?$AAl?$AAi?$AAz?$AAa?$AAt?$AAi?$AAo?$AAn?$AA?9?$AAl?$AA1?$AA?9@ 10012a60     libucrt:winapi_thunks.obj
 0001:00011aa8       ??_C@_1FK@FPHCKFIE@?$AAa?$AAp?$AAi?$AA?9?$AAm?$AAs?$AA?9?$AAw?$AAi?$AAn?$AA?9?$AAc?$AAo?$AAr?$AAe?$AA?9?$AAl?$AAo?$AAc?$AAa?$AAl?$AAi?$AAz?$AAa?$AAt?$AAi?$AAo?$AAn?$AA?9?$AAo?$AAb?$AAs@ 10012aa8     libucrt:winapi_thunks.obj
 0001:00011b08       ??_C@_1EM@DILCGIIO@?$AAa?$AAp?$AAi?$AA?9?$AAm?$AAs?$AA?9?$AAw?$AAi?$AAn?$AA?9?$AAc?$AAo?$AAr?$AAe?$AA?9?$AAp?$AAr?$AAo?$AAc?$AAe?$AAs?$AAs?$AAt?$AAh?$AAr?$AAe?$AAa?$AAd?$AAs?$AA?9?$AAl@ 10012b08     libucrt:winapi_thunks.obj
 0001:00011b54       ??_C@_1DM@LNCGDDPN@?$AAa?$AAp?$AAi?$AA?9?$AAm?$AAs?$AA?9?$AAw?$AAi?$AAn?$AA?9?$AAc?$AAo?$AAr?$AAe?$AA?9?$AAs?$AAt?$AAr?$AAi?$AAn?$AAg?$AA?9?$AAl?$AA1?$AA?9?$AA1?$AA?9?$AA0?$AA?$AA@ 10012b54     libucrt:winapi_thunks.obj
 0001:00011b90       ??_C@_1DO@FPAPJEMD@?$AAa?$AAp?$AAi?$AA?9?$AAm?$AAs?$AA?9?$AAw?$AAi?$AAn?$AA?9?$AAc?$AAo?$AAr?$AAe?$AA?9?$AAs?$AAy?$AAs?$AAi?$AAn?$AAf?$AAo?$AA?9?$AAl?$AA1?$AA?9?$AA2?$AA?9?$AA1?$AA?$AA@ 10012b90     libucrt:winapi_thunks.obj
 0001:00011bd0       ??_C@_1DK@NDHNAHIO@?$AAa?$AAp?$AAi?$AA?9?$AAm?$AAs?$AA?9?$AAw?$AAi?$AAn?$AA?9?$AAc?$AAo?$AAr?$AAe?$AA?9?$AAw?$AAi?$AAn?$AAr?$AAt?$AA?9?$AAl?$AA1?$AA?9?$AA1?$AA?9?$AA0?$AA?$AA@ 10012bd0     libucrt:winapi_thunks.obj
 0001:00011c0c       ??_C@_1DM@KGHDGBCM@?$AAa?$AAp?$AAi?$AA?9?$AAm?$AAs?$AA?9?$AAw?$AAi?$AAn?$AA?9?$AAc?$AAo?$AAr?$AAe?$AA?9?$AAx?$AAs?$AAt?$AAa?$AAt?$AAe?$AA?9?$AAl?$AA2?$AA?9?$AA1?$AA?9?$AA0?$AA?$AA@ 10012c0c     libucrt:winapi_thunks.obj
 0001:00011c48       ??_C@_1EO@IJIOEFOH@?$AAa?$AAp?$AAi?$AA?9?$AAm?$AAs?$AA?9?$AAw?$AAi?$AAn?$AA?9?$AAr?$AAt?$AAc?$AAo?$AAr?$AAe?$AA?9?$AAn?$AAt?$AAu?$AAs?$AAe?$AAr?$AA?9?$AAw?$AAi?$AAn?$AAd?$AAo?$AAw?$AA?9@ 10012c48     libucrt:winapi_thunks.obj
 0001:00011c98       ??_C@_1FG@HHGEKANL@?$AAa?$AAp?$AAi?$AA?9?$AAm?$AAs?$AA?9?$AAw?$AAi?$AAn?$AA?9?$AAs?$AAe?$AAc?$AAu?$AAr?$AAi?$AAt?$AAy?$AA?9?$AAs?$AAy?$AAs?$AAt?$AAe?$AAm?$AAf?$AAu?$AAn?$AAc?$AAt?$AAi@ 10012c98     libucrt:winapi_thunks.obj
 0001:00011cf0       ??_C@_1FG@NCKKOLKO@?$AAe?$AAx?$AAt?$AA?9?$AAm?$AAs?$AA?9?$AAw?$AAi?$AAn?$AA?9?$AAk?$AAe?$AAr?$AAn?$AAe?$AAl?$AA3?$AA2?$AA?9?$AAp?$AAa?$AAc?$AAk?$AAa?$AAg?$AAe?$AA?9?$AAc?$AAu?$AAr?$AAr@ 10012cf0     libucrt:winapi_thunks.obj
 0001:00011d48       ??_C@_1EG@DBIOJECG@?$AAe?$AAx?$AAt?$AA?9?$AAm?$AAs?$AA?9?$AAw?$AAi?$AAn?$AA?9?$AAn?$AAt?$AAu?$AAs?$AAe?$AAr?$AA?9?$AAd?$AAi?$AAa?$AAl?$AAo?$AAg?$AAb?$AAo?$AAx?$AA?9?$AAl?$AA1?$AA?9?$AA1@ 10012d48     libucrt:winapi_thunks.obj
 0001:00011d90       ??_C@_1EO@FIHMJCLF@?$AAe?$AAx?$AAt?$AA?9?$AAm?$AAs?$AA?9?$AAw?$AAi?$AAn?$AA?9?$AAn?$AAt?$AAu?$AAs?$AAe?$AAr?$AA?9?$AAw?$AAi?$AAn?$AAd?$AAo?$AAw?$AAs?$AAt?$AAa?$AAt?$AAi?$AAo?$AAn?$AA?9@ 10012d90     libucrt:winapi_thunks.obj
 0001:00011de0       ??_C@_1O@BCCLBEOE@?$AAu?$AAs?$AAe?$AAr?$AA3?$AA2?$AA?$AA@ 10012de0     libucrt:winapi_thunks.obj
 0001:00011df4       ??_C@_0BA@FHFNEAED@AreFileApisANSI?$AA@ 10012df4     libucrt:winapi_thunks.obj
 0001:00011e0c       ??_C@_0BA@IHGNDAEB@CompareStringEx?$AA@ 10012e0c     libucrt:winapi_thunks.obj
 0001:00011e44       ??_C@_0BE@JOGNEJCI@GetCurrentPackageId?$AA@ 10012e44     libucrt:winapi_thunks.obj
 0001:00011e68       ??_C@_0O@KKBNKAPF@LCMapStringEx?$AA@ 10012e68     libucrt:winapi_thunks.obj
 0001:00011e80       ??_C@_0BB@HBDEELFH@LocaleNameToLCID?$AA@ 10012e80     libucrt:winapi_thunks.obj
 0001:00011e98       __wctype                   10012e98     libucrt:ctype.obj
 0001:000120a0       ___newctype                100130a0     libucrt:ctype.obj
 0001:000123a0       ___newclmap                100133a0     libucrt:ctype.obj
 0001:00012520       ___newcumap                10013520     libucrt:ctype.obj
 0001:000126e0       ??_C@_1M@HPNHIDJI@?$AAj?$AAa?$AA?9?$AAJ?$AAP?$AA?$AA@ 100136e0     libucrt:mbctype.obj
 0001:000126ec       ??_C@_1M@BIBDDEMK@?$AAz?$AAh?$AA?9?$AAC?$AAN?$AA?$AA@ 100136ec     libucrt:mbctype.obj
 0001:000126f8       ??_C@_1M@JLOOOEGK@?$AAk?$AAo?$AA?9?$AAK?$AAR?$AA?$AA@ 100136f8     libucrt:mbctype.obj
 0001:00012704       ??_C@_1M@CLNBBOPM@?$AAz?$AAh?$AA?9?$AAT?$AAW?$AA?$AA@ 10013704     libucrt:mbctype.obj
 0001:00012710       ??_C@_05DNEBIAHO@1?$CDINF?$AA@ 10013710     libucrt:cfout.obj
 0001:00012718       ??_C@_06IMKFLFPG@1?$CDQNAN?$AA@ 10013718     libucrt:cfout.obj
 0001:00012720       ??_C@_06PGGFOGJG@1?$CDSNAN?$AA@ 10013720     libucrt:cfout.obj
 0001:00012728       ??_C@_05PHHOCPM@1?$CDIND?$AA@ 10013728     libucrt:cfout.obj
 0001:00012730       ??_C@_15PJPFLCCM@?$AAu?$AAk?$AA?$AA@ 10013730     libucrt:get_qualified_locale.obj
 0001:00012e58       ??_C@_15EMKDOKLE@?$AAa?$AAr?$AA?$AA@ 10013e58     libucrt:lcidtoname_downlevel.obj
 0001:00012e60       ??_C@_15KNPADPLH@?$AAb?$AAg?$AA?$AA@ 10013e60     libucrt:lcidtoname_downlevel.obj
 0001:00012e68       ??_C@_15EDMHLDMO@?$AAc?$AAa?$AA?$AA@ 10013e68     libucrt:lcidtoname_downlevel.obj
 0001:00012e70       ??_C@_1O@BPEAJADD@?$AAz?$AAh?$AA?9?$AAC?$AAH?$AAS?$AA?$AA@ 10013e70     libucrt:lcidtoname_downlevel.obj
 0001:00012e80       ??_C@_15LJNHCMNK@?$AAc?$AAs?$AA?$AA@ 10013e80     libucrt:lcidtoname_downlevel.obj
 0001:00012e88       ??_C@_15FOMCIDHG@?$AAd?$AAa?$AA?$AA@ 10013e88     libucrt:lcidtoname_downlevel.obj
 0001:00012e90       ??_C@_15NBKABECB@?$AAd?$AAe?$AA?$AA@ 10013e90     libucrt:lcidtoname_downlevel.obj
 0001:00012e98       ??_C@_15GHPEIIAO@?$AAe?$AAl?$AA?$AA@ 10013e98     libucrt:lcidtoname_downlevel.obj
 0001:00012ea0       ??_C@_15MNPNEAIF@?$AAe?$AAn?$AA?$AA@ 10013ea0     libucrt:lcidtoname_downlevel.obj
 0001:00012ea8       ??_C@_15GPIOMPMH@?$AAe?$AAs?$AA?$AA@ 10013ea8     libucrt:lcidtoname_downlevel.obj
 0001:00012eb0       ??_C@_15NGLOAKJC@?$AAf?$AAi?$AA?$AA@ 10013eb0     libucrt:lcidtoname_downlevel.obj
 0001:00012eb8       ??_C@_15FBKGNKAM@?$AAf?$AAr?$AA?$AA@ 10013eb8     libucrt:lcidtoname_downlevel.obj
 0001:00012ec0       ??_C@_15KGGCNEFK@?$AAh?$AAe?$AA?$AA@ 10013ec0     libucrt:lcidtoname_downlevel.obj
 0001:00012ec8       ??_C@_15PGHLIDMF@?$AAh?$AAu?$AA?$AA@ 10013ec8     libucrt:lcidtoname_downlevel.obj
 0001:00012ed0       ??_C@_15BIEMAPLM@?$AAi?$AAs?$AA?$AA@ 10013ed0     libucrt:lcidtoname_downlevel.obj
 0001:00012ed8       ??_C@_15IFJLDHAF@?$AAi?$AAt?$AA?$AA@ 10013ed8     libucrt:lcidtoname_downlevel.obj
 0001:00012ee0       ??_C@_15GEMIOCAG@?$AAj?$AAa?$AA?$AA@ 10013ee0     libucrt:lcidtoname_downlevel.obj
 0001:00012ee8       ??_C@_15EPELEGJA@?$AAk?$AAo?$AA?$AA@ 10013ee8     libucrt:lcidtoname_downlevel.obj
 0001:00012ef0       ??_C@_15NDDHIMN@?$AAn?$AAl?$AA?$AA@ 10013ef0     libucrt:lcidtoname_downlevel.obj
 0001:00012ef8       ??_C@_15BPIGNHCD@?$AAn?$AAo?$AA?$AA@ 10013ef8     libucrt:lcidtoname_downlevel.obj
 0001:00012f00       ??_C@_15DEOPBLCG@?$AAp?$AAl?$AA?$AA@ 10013f00     libucrt:lcidtoname_downlevel.obj
 0001:00012f08       ??_C@_15KBECGEFG@?$AAp?$AAt?$AA?$AA@ 10013f08     libucrt:lcidtoname_downlevel.obj
 0001:00012f10       ??_C@_15GLJCBFMD@?$AAr?$AAo?$AA?$AA@ 10013f10     libucrt:lcidtoname_downlevel.obj
 0001:00012f18       ??_C@_15FEDGKCDI@?$AAr?$AAu?$AA?$AA@ 10013f18     libucrt:lcidtoname_downlevel.obj
 0001:00012f20       ??_C@_15GLKMLLHM@?$AAh?$AAr?$AA?$AA@ 10013f20     libucrt:lcidtoname_downlevel.obj
 0001:00012f28       ??_C@_15CPKMFBDB@?$AAs?$AAk?$AA?$AA@ 10013f28     libucrt:lcidtoname_downlevel.obj
 0001:00012f30       ??_C@_15BAAIOGMK@?$AAs?$AAq?$AA?$AA@ 10013f30     libucrt:lcidtoname_downlevel.obj
 0001:00012f38       ??_C@_15INNPNOHD@?$AAs?$AAv?$AA?$AA@ 10013f38     libucrt:lcidtoname_downlevel.obj
 0001:00012f40       ??_C@_15CABMMOGH@?$AAt?$AAh?$AA?$AA@ 10013f40     libucrt:lcidtoname_downlevel.obj
 0001:00012f48       ??_C@_15BPLIHJJM@?$AAt?$AAr?$AA?$AA@ 10013f48     libucrt:lcidtoname_downlevel.obj
 0001:00012f50       ??_C@_15NEOEKKDJ@?$AAu?$AAr?$AA?$AA@ 10013f50     libucrt:lcidtoname_downlevel.obj
 0001:00012f58       ??_C@_15NFICGAJK@?$AAi?$AAd?$AA?$AA@ 10013f58     libucrt:lcidtoname_downlevel.obj
 0001:00012f60       ??_C@_15HPJPHDM@?$AAb?$AAe?$AA?$AA@ 10013f60     libucrt:lcidtoname_downlevel.obj
 0001:00012f68       ??_C@_15LCHLGJII@?$AAs?$AAl?$AA?$AA@ 10013f68     libucrt:lcidtoname_downlevel.obj
 0001:00012f70       ??_C@_15PCFJPHHO@?$AAe?$AAt?$AA?$AA@ 10013f70     libucrt:lcidtoname_downlevel.obj
 0001:00012f78       ??_C@_15HPFPGODN@?$AAl?$AAv?$AA?$AA@ 10013f78     libucrt:lcidtoname_downlevel.obj
 0001:00012f80       ??_C@_15NFFGKGLG@?$AAl?$AAt?$AA?$AA@ 10013f80     libucrt:lcidtoname_downlevel.obj
 0001:00012f88       ??_C@_15BDAKCCHN@?$AAf?$AAa?$AA?$AA@ 10013f88     libucrt:lcidtoname_downlevel.obj
 0001:00012f90       ??_C@_15NFGIAIAJ@?$AAv?$AAi?$AA?$AA@ 10013f90     libucrt:lcidtoname_downlevel.obj
 0001:00012f98       ??_C@_15LMKNDMHN@?$AAh?$AAy?$AA?$AA@ 10013f98     libucrt:lcidtoname_downlevel.obj
 0001:00012fa0       ??_C@_15IJBHMCFL@?$AAa?$AAz?$AA?$AA@ 10013fa0     libucrt:lcidtoname_downlevel.obj
 0001:00012fa8       ??_C@_15EKOFJABL@?$AAe?$AAu?$AA?$AA@ 10013fa8     libucrt:lcidtoname_downlevel.obj
 0001:00012fb0       ??_C@_15BGHADCNK@?$AAm?$AAk?$AA?$AA@ 10013fb0     libucrt:lcidtoname_downlevel.obj
 0001:00012fb8       ??_C@_15JDNICKHM@?$AAa?$AAf?$AA?$AA@ 10013fb8     libucrt:lcidtoname_downlevel.obj
 0001:00012fc0       ??_C@_15KPJEDBKD@?$AAk?$AAa?$AA?$AA@ 10013fc0     libucrt:lcidtoname_downlevel.obj
 0001:00012fc8       ??_C@_15PDNFFFEO@?$AAf?$AAo?$AA?$AA@ 10013fc8     libucrt:lcidtoname_downlevel.obj
 0001:00012fd0       ??_C@_15OMLEGLOC@?$AAh?$AAi?$AA?$AA@ 10013fd0     libucrt:lcidtoname_downlevel.obj
 0001:00012fd8       ??_C@_15IDNNENKK@?$AAm?$AAs?$AA?$AA@ 10013fd8     libucrt:lcidtoname_downlevel.obj
 0001:00012fe0       ??_C@_15MACJNBMH@?$AAk?$AAk?$AA?$AA@ 10013fe0     libucrt:lcidtoname_downlevel.obj
 0001:00012fe8       ??_C@_15DKDJEOND@?$AAk?$AAy?$AA?$AA@ 10013fe8     libucrt:lcidtoname_downlevel.obj
 0001:00012ff0       ??_C@_15DFGDLJBG@?$AAs?$AAw?$AA?$AA@ 10013ff0     libucrt:lcidtoname_downlevel.obj
 0001:00012ff8       ??_C@_15BBFAICNG@?$AAu?$AAz?$AA?$AA@ 10013ff8     libucrt:lcidtoname_downlevel.obj
 0001:00013000       ??_C@_15DKNDCGEA@?$AAt?$AAt?$AA?$AA@ 10014000     libucrt:lcidtoname_downlevel.obj
 0001:00013008       ??_C@_15MGIFMDPL@?$AAp?$AAa?$AA?$AA@ 10014008     libucrt:lcidtoname_downlevel.obj
 0001:00013010       ??_C@_15HCNDBBA@?$AAg?$AAu?$AA?$AA@ 10014010     libucrt:lcidtoname_downlevel.obj
 0001:00013018       ??_C@_15FNBEIBON@?$AAt?$AAa?$AA?$AA@ 10014018     libucrt:lcidtoname_downlevel.obj
 0001:00013020       ??_C@_15NCHGBGLK@?$AAt?$AAe?$AA?$AA@ 10014020     libucrt:lcidtoname_downlevel.obj
 0001:00013028       ??_C@_15PHPHCBPF@?$AAk?$AAn?$AA?$AA@ 10014028     libucrt:lcidtoname_downlevel.obj
 0001:00013030       ??_C@_15DLGBCKMP@?$AAm?$AAr?$AA?$AA@ 10014030     libucrt:lcidtoname_downlevel.obj
 0001:00013038       ??_C@_15EABBLBFF@?$AAs?$AAa?$AA?$AA@ 10014038     libucrt:lcidtoname_downlevel.obj
 0001:00013040       ??_C@_15CBKOMCOI@?$AAm?$AAn?$AA?$AA@ 10014040     libucrt:lcidtoname_downlevel.obj
 0001:00013048       ??_C@_15CKDMCJAF@?$AAg?$AAl?$AA?$AA@ 10014048     libucrt:lcidtoname_downlevel.obj
 0001:00013050       ??_C@_17CNJFBPG@?$AAk?$AAo?$AAk?$AA?$AA@ 10014050     libucrt:lcidtoname_downlevel.obj
 0001:00013058       ??_C@_17FFBJICPL@?$AAs?$AAy?$AAr?$AA?$AA@ 10014058     libucrt:lcidtoname_downlevel.obj
 0001:00013060       ??_C@_17KPNDCPAF@?$AAd?$AAi?$AAv?$AA?$AA@ 10014060     libucrt:lcidtoname_downlevel.obj
 0001:00013068       ??_C@_1M@OKAHONE@?$AAa?$AAr?$AA?9?$AAS?$AAA?$AA?$AA@ 10014068     libucrt:lcidtoname_downlevel.obj
 0001:00013074       ??_C@_1M@FFFIGIGK@?$AAb?$AAg?$AA?9?$AAB?$AAG?$AA?$AA@ 10014074     libucrt:lcidtoname_downlevel.obj
 0001:00013080       ??_C@_1M@BJNKEDC@?$AAc?$AAa?$AA?9?$AAE?$AAS?$AA?$AA@ 10014080     libucrt:lcidtoname_downlevel.obj
 0001:0001308c       ??_C@_1M@IJJHFJHA@?$AAc?$AAs?$AA?9?$AAC?$AAZ?$AA?$AA@ 1001408c     libucrt:lcidtoname_downlevel.obj
 0001:00013098       ??_C@_1M@CLPEOBGI@?$AAd?$AAa?$AA?9?$AAD?$AAK?$AA?$AA@ 10014098     libucrt:lcidtoname_downlevel.obj
 0001:000130a4       ??_C@_1M@MCMADGCB@?$AAd?$AAe?$AA?9?$AAD?$AAE?$AA?$AA@ 100140a4     libucrt:lcidtoname_downlevel.obj
 0001:000130b0       ??_C@_1M@OOCKEMAM@?$AAe?$AAl?$AA?9?$AAG?$AAR?$AA?$AA@ 100140b0     libucrt:lcidtoname_downlevel.obj
 0001:000130bc       ??_C@_1M@DDNJFGID@?$AAf?$AAi?$AA?9?$AAF?$AAI?$AA?$AA@ 100140bc     libucrt:lcidtoname_downlevel.obj
 0001:000130c8       ??_C@_1M@GLIPPMAC@?$AAf?$AAr?$AA?9?$AAF?$AAR?$AA?$AA@ 100140c8     libucrt:lcidtoname_downlevel.obj
 0001:000130d4       ??_C@_1M@GFMCHPE@?$AAh?$AAe?$AA?9?$AAI?$AAL?$AA?$AA@ 100140d4     libucrt:lcidtoname_downlevel.obj
 0001:000130e0       ??_C@_1M@MHLPGNKM@?$AAh?$AAu?$AA?9?$AAH?$AAU?$AA?$AA@ 100140e0     libucrt:lcidtoname_downlevel.obj
 0001:000130ec       ??_C@_1M@LPDDNNPN@?$AAi?$AAs?$AA?9?$AAI?$AAS?$AA?$AA@ 100140ec     libucrt:lcidtoname_downlevel.obj
 0001:000130f8       ??_C@_1M@MADIPODN@?$AAi?$AAt?$AA?9?$AAI?$AAT?$AA?$AA@ 100140f8     libucrt:lcidtoname_downlevel.obj
 0001:00013104       ??_C@_1M@IHBJJGG@?$AAn?$AAl?$AA?9?$AAN?$AAL?$AA?$AA@ 10014104     libucrt:lcidtoname_downlevel.obj
 0001:00013110       ??_C@_1M@EANAGDL@?$AAn?$AAb?$AA?9?$AAN?$AAO?$AA?$AA@ 10014110     libucrt:lcidtoname_downlevel.obj
 0001:0001311c       ??_C@_1M@NEIEMEGP@?$AAp?$AAl?$AA?9?$AAP?$AAL?$AA?$AA@ 1001411c     libucrt:lcidtoname_downlevel.obj
 0001:00013128       ??_C@_1M@BOCFIGEP@?$AAp?$AAt?$AA?9?$AAB?$AAR?$AA?$AA@ 10014128     libucrt:lcidtoname_downlevel.obj
 0001:00013134       ??_C@_1M@IMPFOPBG@?$AAr?$AAo?$AA?9?$AAR?$AAO?$AA?$AA@ 10014134     libucrt:lcidtoname_downlevel.obj
 0001:00013140       ??_C@_1M@IDNNEJMM@?$AAr?$AAu?$AA?9?$AAR?$AAU?$AA?$AA@ 10014140     libucrt:lcidtoname_downlevel.obj
 0001:0001314c       ??_C@_1M@LILEEOGM@?$AAh?$AAr?$AA?9?$AAH?$AAR?$AA?$AA@ 1001414c     libucrt:lcidtoname_downlevel.obj
 0001:00013158       ??_C@_1M@FKIFEHPB@?$AAs?$AAk?$AA?9?$AAS?$AAK?$AA?$AA@ 10014158     libucrt:lcidtoname_downlevel.obj
 0001:00013164       ??_C@_1M@LJMAMNPJ@?$AAs?$AAq?$AA?9?$AAA?$AAL?$AA?$AA@ 10014164     libucrt:lcidtoname_downlevel.obj
 0001:00013170       ??_C@_1M@GIAKDKJK@?$AAs?$AAv?$AA?9?$AAS?$AAE?$AA?$AA@ 10014170     libucrt:lcidtoname_downlevel.obj
 0001:0001317c       ??_C@_1M@MKJKIKCL@?$AAt?$AAh?$AA?9?$AAT?$AAH?$AA?$AA@ 1001417c     libucrt:lcidtoname_downlevel.obj
 0001:00013188       ??_C@_1M@MFLCCMPB@?$AAt?$AAr?$AA?9?$AAT?$AAR?$AA?$AA@ 10014188     libucrt:lcidtoname_downlevel.obj
 0001:00013194       ??_C@_1M@OIJHDKJN@?$AAu?$AAr?$AA?9?$AAP?$AAK?$AA?$AA@ 10014194     libucrt:lcidtoname_downlevel.obj
 0001:000131a0       ??_C@_1M@LHIPCIEK@?$AAi?$AAd?$AA?9?$AAI?$AAD?$AA?$AA@ 100141a0     libucrt:lcidtoname_downlevel.obj
 0001:000131ac       ??_C@_1M@MFMOBGI@?$AAu?$AAk?$AA?9?$AAU?$AAA?$AA?$AA@ 100141ac     libucrt:lcidtoname_downlevel.obj
 0001:000131b8       ??_C@_1M@OBGLJIPL@?$AAb?$AAe?$AA?9?$AAB?$AAY?$AA?$AA@ 100141b8     libucrt:lcidtoname_downlevel.obj
 0001:000131c4       ??_C@_1M@BCFAJEAD@?$AAs?$AAl?$AA?9?$AAS?$AAI?$AA?$AA@ 100141c4     libucrt:lcidtoname_downlevel.obj
 0001:000131d0       ??_C@_1M@FKFFEDDN@?$AAe?$AAt?$AA?9?$AAE?$AAE?$AA?$AA@ 100141d0     libucrt:lcidtoname_downlevel.obj
 0001:000131dc       ??_C@_1M@KGKKAACI@?$AAl?$AAv?$AA?9?$AAL?$AAV?$AA?$AA@ 100141dc     libucrt:lcidtoname_downlevel.obj
 0001:000131e8       ??_C@_1M@IFGBIJO@?$AAl?$AAt?$AA?9?$AAL?$AAT?$AA?$AA@ 100141e8     libucrt:lcidtoname_downlevel.obj
 0001:000131f4       ??_C@_1M@FGEAHEDM@?$AAf?$AAa?$AA?9?$AAI?$AAR?$AA?$AA@ 100141f4     libucrt:lcidtoname_downlevel.obj
 0001:00013200       ??_C@_1M@KBMAIBFN@?$AAv?$AAi?$AA?9?$AAV?$AAN?$AA?$AA@ 10014200     libucrt:lcidtoname_downlevel.obj
 0001:0001320c       ??_C@_1M@GPCBKDJK@?$AAh?$AAy?$AA?9?$AAA?$AAM?$AA?$AA@ 1001420c     libucrt:lcidtoname_downlevel.obj
 0001:00013218       ??_C@_1BG@BECMDDJB@?$AAa?$AAz?$AA?9?$AAA?$AAZ?$AA?9?$AAL?$AAa?$AAt?$AAn?$AA?$AA@ 10014218     libucrt:lcidtoname_downlevel.obj
 0001:00013230       ??_C@_1M@MAOFCAEA@?$AAe?$AAu?$AA?9?$AAE?$AAS?$AA?$AA@ 10014230     libucrt:lcidtoname_downlevel.obj
 0001:0001323c       ??_C@_1M@IGHABKPI@?$AAm?$AAk?$AA?9?$AAM?$AAK?$AA?$AA@ 1001423c     libucrt:lcidtoname_downlevel.obj
 0001:00013248       ??_C@_1M@IAIGNEJG@?$AAt?$AAn?$AA?9?$AAZ?$AAA?$AA?$AA@ 10014248     libucrt:lcidtoname_downlevel.obj
 0001:00013254       ??_C@_1M@IIJCOJFA@?$AAx?$AAh?$AA?9?$AAZ?$AAA?$AA?$AA@ 10014254     libucrt:lcidtoname_downlevel.obj
 0001:00013260       ??_C@_1M@LGPJHNJH@?$AAz?$AAu?$AA?9?$AAZ?$AAA?$AA?$AA@ 10014260     libucrt:lcidtoname_downlevel.obj
 0001:0001326c       ??_C@_1M@HOKAOIO@?$AAa?$AAf?$AA?9?$AAZ?$AAA?$AA?$AA@ 1001426c     libucrt:lcidtoname_downlevel.obj
 0001:00013278       ??_C@_1M@DPCLHLIE@?$AAk?$AAa?$AA?9?$AAG?$AAE?$AA?$AA@ 10014278     libucrt:lcidtoname_downlevel.obj
 0001:00013284       ??_C@_1M@BLKMHJBI@?$AAf?$AAo?$AA?9?$AAF?$AAO?$AA?$AA@ 10014284     libucrt:lcidtoname_downlevel.obj
 0001:00013290       ??_C@_1M@LGGJAPPB@?$AAh?$AAi?$AA?9?$AAI?$AAN?$AA?$AA@ 10014290     libucrt:lcidtoname_downlevel.obj
 0001:0001329c       ??_C@_1M@FIKPIHFE@?$AAm?$AAt?$AA?9?$AAM?$AAT?$AA?$AA@ 1001429c     libucrt:lcidtoname_downlevel.obj
 0001:000132a8       ??_C@_1M@HEGGPBFA@?$AAs?$AAe?$AA?9?$AAN?$AAO?$AA?$AA@ 100142a8     libucrt:lcidtoname_downlevel.obj
 0001:000132b4       ??_C@_1M@EIBJEEPA@?$AAm?$AAs?$AA?9?$AAM?$AAY?$AA?$AA@ 100142b4     libucrt:lcidtoname_downlevel.obj
 0001:000132c0       ??_C@_1M@FHLBGMPP@?$AAk?$AAk?$AA?9?$AAK?$AAZ?$AA?$AA@ 100142c0     libucrt:lcidtoname_downlevel.obj
 0001:000132cc       ??_C@_1M@NGJJLCGI@?$AAk?$AAy?$AA?9?$AAK?$AAG?$AA?$AA@ 100142cc     libucrt:lcidtoname_downlevel.obj
 0001:000132d8       ??_C@_1M@GIENNBFC@?$AAs?$AAw?$AA?9?$AAK?$AAE?$AA?$AA@ 100142d8     libucrt:lcidtoname_downlevel.obj
 0001:000132e4       ??_C@_1BG@NDGMJIMJ@?$AAu?$AAz?$AA?9?$AAU?$AAZ?$AA?9?$AAL?$AAa?$AAt?$AAn?$AA?$AA@ 100142e4     libucrt:lcidtoname_downlevel.obj
 0001:000132fc       ??_C@_1M@IDCCIHBC@?$AAt?$AAt?$AA?9?$AAR?$AAU?$AA?$AA@ 100142fc     libucrt:lcidtoname_downlevel.obj
 0001:00013308       ??_C@_1M@LOICPMOJ@?$AAb?$AAn?$AA?9?$AAI?$AAN?$AA?$AA@ 10014308     libucrt:lcidtoname_downlevel.obj
 0001:00013314       ??_C@_1M@KPKKNEAH@?$AAp?$AAa?$AA?9?$AAI?$AAN?$AA?$AA@ 10014314     libucrt:lcidtoname_downlevel.obj
 0001:00013320       ??_C@_1M@PJGPPBOG@?$AAg?$AAu?$AA?9?$AAI?$AAN?$AA?$AA@ 10014320     libucrt:lcidtoname_downlevel.obj
 0001:0001332c       ??_C@_1M@KMKMOPHI@?$AAt?$AAa?$AA?9?$AAI?$AAN?$AA?$AA@ 1001432c     libucrt:lcidtoname_downlevel.obj
 0001:00013338       ??_C@_1M@KFEHEPAC@?$AAt?$AAe?$AA?9?$AAI?$AAN?$AA?$AA@ 10014338     libucrt:lcidtoname_downlevel.obj
 0001:00013344       ??_C@_1M@CDCLMGHI@?$AAk?$AAn?$AA?9?$AAI?$AAN?$AA?$AA@ 10014344     libucrt:lcidtoname_downlevel.obj
 0001:00013350       ??_C@_1M@MIODLDKF@?$AAm?$AAl?$AA?9?$AAI?$AAN?$AA?$AA@ 10014350     libucrt:lcidtoname_downlevel.obj
 0001:0001335c       ??_C@_1M@PBIEACPO@?$AAm?$AAr?$AA?9?$AAI?$AAN?$AA?$AA@ 1001435c     libucrt:lcidtoname_downlevel.obj
 0001:00013368       ??_C@_1M@NIDEAGPH@?$AAs?$AAa?$AA?9?$AAI?$AAN?$AA?$AA@ 10014368     libucrt:lcidtoname_downlevel.obj
 0001:00013374       ??_C@_1M@FHIHCBIO@?$AAm?$AAn?$AA?9?$AAM?$AAN?$AA?$AA@ 10014374     libucrt:lcidtoname_downlevel.obj
 0001:00013380       ??_C@_1M@JAIJPENP@?$AAc?$AAy?$AA?9?$AAG?$AAB?$AA?$AA@ 10014380     libucrt:lcidtoname_downlevel.obj
 0001:0001338c       ??_C@_1M@PHGFBEPN@?$AAg?$AAl?$AA?9?$AAE?$AAS?$AA?$AA@ 1001438c     libucrt:lcidtoname_downlevel.obj
 0001:00013398       ??_C@_1O@KPIPDNCP@?$AAk?$AAo?$AAk?$AA?9?$AAI?$AAN?$AA?$AA@ 10014398     libucrt:lcidtoname_downlevel.obj
 0001:000133a8       ??_C@_1O@KNHJLDJA@?$AAs?$AAy?$AAr?$AA?9?$AAS?$AAY?$AA?$AA@ 100143a8     libucrt:lcidtoname_downlevel.obj
 0001:000133b8       ??_C@_1O@MKEKBLAH@?$AAd?$AAi?$AAv?$AA?9?$AAM?$AAV?$AA?$AA@ 100143b8     libucrt:lcidtoname_downlevel.obj
 0001:000133c8       ??_C@_1O@OHDCKDDF@?$AAq?$AAu?$AAz?$AA?9?$AAB?$AAO?$AA?$AA@ 100143c8     libucrt:lcidtoname_downlevel.obj
 0001:000133d8       ??_C@_1M@LEPJNLFD@?$AAn?$AAs?$AA?9?$AAZ?$AAA?$AA?$AA@ 100143d8     libucrt:lcidtoname_downlevel.obj
 0001:000133e4       ??_C@_1M@OMLEIIJB@?$AAm?$AAi?$AA?9?$AAN?$AAZ?$AA?$AA@ 100143e4     libucrt:lcidtoname_downlevel.obj
 0001:000133f0       ??_C@_1M@PMPEAILG@?$AAa?$AAr?$AA?9?$AAI?$AAQ?$AA?$AA@ 100143f0     libucrt:lcidtoname_downlevel.obj
 0001:000133fc       ??_C@_1M@CNKPNOEE@?$AAd?$AAe?$AA?9?$AAC?$AAH?$AA?$AA@ 100143fc     libucrt:lcidtoname_downlevel.obj
 0001:00013408       ??_C@_1M@LKMGMLKO@?$AAe?$AAn?$AA?9?$AAG?$AAB?$AA?$AA@ 10014408     libucrt:lcidtoname_downlevel.obj
 0001:00013414       ??_C@_1M@PGKJFFGL@?$AAe?$AAs?$AA?9?$AAM?$AAX?$AA?$AA@ 10014414     libucrt:lcidtoname_downlevel.obj
 0001:00013420       ??_C@_1M@DNNANBDC@?$AAf?$AAr?$AA?9?$AAB?$AAE?$AA?$AA@ 10014420     libucrt:lcidtoname_downlevel.obj
 0001:0001342c       ??_C@_1M@HLGMDFHM@?$AAi?$AAt?$AA?9?$AAC?$AAH?$AA?$AA@ 1001442c     libucrt:lcidtoname_downlevel.obj
 0001:00013438       ??_C@_1M@CLLBGJH@?$AAn?$AAl?$AA?9?$AAB?$AAE?$AA?$AA@ 10014438     libucrt:lcidtoname_downlevel.obj
 0001:00013444       ??_C@_1M@BODBOGLF@?$AAn?$AAn?$AA?9?$AAN?$AAO?$AA?$AA@ 10014444     libucrt:lcidtoname_downlevel.obj
 0001:00013450       ??_C@_1M@HFFAHKAD@?$AAp?$AAt?$AA?9?$AAP?$AAT?$AA?$AA@ 10014450     libucrt:lcidtoname_downlevel.obj
 0001:0001345c       ??_C@_1BG@LNOAKHIE@?$AAs?$AAr?$AA?9?$AAS?$AAP?$AA?9?$AAL?$AAa?$AAt?$AAn?$AA?$AA@ 1001445c     libucrt:lcidtoname_downlevel.obj
 0001:00013474       ??_C@_1M@HBMHBGAK@?$AAs?$AAv?$AA?9?$AAF?$AAI?$AA?$AA@ 10014474     libucrt:lcidtoname_downlevel.obj
 0001:00013480       ??_C@_1BG@DGCJGJBE@?$AAa?$AAz?$AA?9?$AAA?$AAZ?$AA?9?$AAC?$AAy?$AAr?$AAl?$AA?$AA@ 10014480     libucrt:lcidtoname_downlevel.obj
 0001:00013498       ??_C@_1M@KEJDAAHB@?$AAs?$AAe?$AA?9?$AAS?$AAE?$AA?$AA@ 10014498     libucrt:lcidtoname_downlevel.obj
 0001:000134a4       ??_C@_1M@HEIBJJAD@?$AAm?$AAs?$AA?9?$AAB?$AAN?$AA?$AA@ 100144a4     libucrt:lcidtoname_downlevel.obj
 0001:000134b0       ??_C@_1BG@PBGJMCEM@?$AAu?$AAz?$AA?9?$AAU?$AAZ?$AA?9?$AAC?$AAy?$AAr?$AAl?$AA?$AA@ 100144b0     libucrt:lcidtoname_downlevel.obj
 0001:000134c8       ??_C@_1O@LAOBCMDF@?$AAq?$AAu?$AAz?$AA?9?$AAE?$AAC?$AA?$AA@ 100144c8     libucrt:lcidtoname_downlevel.obj
 0001:000134d8       ??_C@_1M@POEEMAIO@?$AAa?$AAr?$AA?9?$AAE?$AAG?$AA?$AA@ 100144d8     libucrt:lcidtoname_downlevel.obj
 0001:000134e4       ??_C@_1M@EFAKDEDL@?$AAz?$AAh?$AA?9?$AAH?$AAK?$AA?$AA@ 100144e4     libucrt:lcidtoname_downlevel.obj
 0001:000134f0       ??_C@_1M@HKKIJHGI@?$AAd?$AAe?$AA?9?$AAA?$AAT?$AA?$AA@ 100144f0     libucrt:lcidtoname_downlevel.obj
 0001:000134fc       ??_C@_1M@KBFBEHJF@?$AAe?$AAn?$AA?9?$AAA?$AAU?$AA?$AA@ 100144fc     libucrt:lcidtoname_downlevel.obj
 0001:00013508       ??_C@_1M@MNPLFAAH@?$AAe?$AAs?$AA?9?$AAE?$AAS?$AA?$AA@ 10014508     libucrt:lcidtoname_downlevel.obj
 0001:00013514       ??_C@_1M@HJOOJFMA@?$AAf?$AAr?$AA?9?$AAC?$AAA?$AA?$AA@ 10014514     libucrt:lcidtoname_downlevel.obj
 0001:00013520       ??_C@_1BG@JPOFPNAB@?$AAs?$AAr?$AA?9?$AAS?$AAP?$AA?9?$AAC?$AAy?$AAr?$AAl?$AA?$AA@ 10014520     libucrt:lcidtoname_downlevel.obj
 0001:00013538       ??_C@_1M@LNFOCMOB@?$AAs?$AAe?$AA?9?$AAF?$AAI?$AA?$AA@ 10014538     libucrt:lcidtoname_downlevel.obj
 0001:00013544       ??_C@_1O@MGJBOAMB@?$AAq?$AAu?$AAz?$AA?9?$AAP?$AAE?$AA?$AA@ 10014544     libucrt:lcidtoname_downlevel.obj
 0001:00013554       ??_C@_1M@GJINLBOK@?$AAa?$AAr?$AA?9?$AAL?$AAY?$AA?$AA@ 10014554     libucrt:lcidtoname_downlevel.obj
 0001:00013560       ??_C@_1M@GGMNHJNL@?$AAz?$AAh?$AA?9?$AAS?$AAG?$AA?$AA@ 10014560     libucrt:lcidtoname_downlevel.obj
 0001:0001356c       ??_C@_1M@HOIKODND@?$AAd?$AAe?$AA?9?$AAL?$AAU?$AA?$AA@ 1001456c     libucrt:lcidtoname_downlevel.obj
 0001:00013578       ??_C@_1M@DDOCCGFG@?$AAe?$AAn?$AA?9?$AAC?$AAA?$AA?$AA@ 10014578     libucrt:lcidtoname_downlevel.obj
 0001:00013584       ??_C@_1M@BNOEMJLF@?$AAe?$AAs?$AA?9?$AAG?$AAT?$AA?$AA@ 10014584     libucrt:lcidtoname_downlevel.obj
 0001:00013590       ??_C@_1M@EOGNKEK@?$AAf?$AAr?$AA?9?$AAC?$AAH?$AA?$AA@ 10014590     libucrt:lcidtoname_downlevel.obj
 0001:0001359c       ??_C@_1M@FLIDJFHL@?$AAh?$AAr?$AA?9?$AAB?$AAA?$AA?$AA@ 1001459c     libucrt:lcidtoname_downlevel.obj
 0001:000135a8       ??_C@_1O@FMCELNAJ@?$AAs?$AAm?$AAj?$AA?9?$AAN?$AAO?$AA?$AA@ 100145a8     libucrt:lcidtoname_downlevel.obj
 0001:000135b8       ??_C@_1M@JHGLJMGJ@?$AAa?$AAr?$AA?9?$AAD?$AAZ?$AA?$AA@ 100145b8     libucrt:lcidtoname_downlevel.obj
 0001:000135c4       ??_C@_1M@JKKFDCNP@?$AAz?$AAh?$AA?9?$AAM?$AAO?$AA?$AA@ 100145c4     libucrt:lcidtoname_downlevel.obj
 0001:000135d0       ??_C@_1M@GEEFALPE@?$AAd?$AAe?$AA?9?$AAL?$AAI?$AA?$AA@ 100145d0     libucrt:lcidtoname_downlevel.obj
 0001:000135dc       ??_C@_1M@IGEOFBG@?$AAe?$AAn?$AA?9?$AAN?$AAZ?$AA?$AA@ 100145dc     libucrt:lcidtoname_downlevel.obj
 0001:000135e8       ??_C@_1M@KDBONEHP@?$AAe?$AAs?$AA?9?$AAC?$AAR?$AA?$AA@ 100145e8     libucrt:lcidtoname_downlevel.obj
 0001:000135f4       ??_C@_1M@FHMDOHNN@?$AAf?$AAr?$AA?9?$AAL?$AAU?$AA?$AA@ 100145f4     libucrt:lcidtoname_downlevel.obj
 0001:00013600       ??_C@_1BG@NFKKMAFG@?$AAb?$AAs?$AA?9?$AAB?$AAA?$AA?9?$AAL?$AAa?$AAt?$AAn?$AA?$AA@ 10014600     libucrt:lcidtoname_downlevel.obj
 0001:00013618       ??_C@_1O@IMNBEMCI@?$AAs?$AAm?$AAj?$AA?9?$AAS?$AAE?$AA?$AA@ 10014618     libucrt:lcidtoname_downlevel.obj
 0001:00013628       ??_C@_1M@DHHMBNDP@?$AAa?$AAr?$AA?9?$AAM?$AAA?$AA?$AA@ 10014628     libucrt:lcidtoname_downlevel.obj
 0001:00013634       ??_C@_1M@BNBLJCGH@?$AAe?$AAn?$AA?9?$AAI?$AAE?$AA?$AA@ 10014634     libucrt:lcidtoname_downlevel.obj
 0001:00013640       ??_C@_1M@GEPAFMDL@?$AAe?$AAs?$AA?9?$AAP?$AAA?$AA?$AA@ 10014640     libucrt:lcidtoname_downlevel.obj
 0001:0001364c       ??_C@_1M@OJONDMDL@?$AAf?$AAr?$AA?9?$AAM?$AAC?$AA?$AA@ 1001464c     libucrt:lcidtoname_downlevel.obj
 0001:00013658       ??_C@_1BG@OBCNFJB@?$AAs?$AAr?$AA?9?$AAB?$AAA?$AA?9?$AAL?$AAa?$AAt?$AAn?$AA?$AA@ 10014658     libucrt:lcidtoname_downlevel.obj
 0001:00013670       ??_C@_1O@KEMEEGPO@?$AAs?$AAm?$AAa?$AA?9?$AAN?$AAO?$AA?$AA@ 10014670     libucrt:lcidtoname_downlevel.obj
 0001:00013680       ??_C@_1M@ELMGFODK@?$AAa?$AAr?$AA?9?$AAT?$AAN?$AA?$AA@ 10014680     libucrt:lcidtoname_downlevel.obj
 0001:0001368c       ??_C@_1M@BHDLHFAF@?$AAe?$AAn?$AA?9?$AAZ?$AAA?$AA?$AA@ 1001468c     libucrt:lcidtoname_downlevel.obj
 0001:00013698       ??_C@_1M@BMGIGLIF@?$AAe?$AAs?$AA?9?$AAD?$AAO?$AA?$AA@ 10014698     libucrt:lcidtoname_downlevel.obj
 0001:000136a4       ??_C@_1BG@CMBHIPBE@?$AAs?$AAr?$AA?9?$AAB?$AAA?$AA?9?$AAC?$AAy?$AAr?$AAl?$AA?$AA@ 100146a4     libucrt:lcidtoname_downlevel.obj
 0001:000136bc       ??_C@_1O@HEDBLHNP@?$AAs?$AAm?$AAa?$AA?9?$AAS?$AAE?$AA?$AA@ 100146bc     libucrt:lcidtoname_downlevel.obj
 0001:000136cc       ??_C@_1M@DAGCADIM@?$AAa?$AAr?$AA?9?$AAO?$AAM?$AA?$AA@ 100146cc     libucrt:lcidtoname_downlevel.obj
 0001:000136d8       ??_C@_1M@FODLMICG@?$AAe?$AAn?$AA?9?$AAJ?$AAM?$AA?$AA@ 100146d8     libucrt:lcidtoname_downlevel.obj
 0001:000136e4       ??_C@_1M@DNMLCIHB@?$AAe?$AAs?$AA?9?$AAV?$AAE?$AA?$AA@ 100146e4     libucrt:lcidtoname_downlevel.obj
 0001:000136f0       ??_C@_1O@EOKHMKJK@?$AAs?$AAm?$AAs?$AA?9?$AAF?$AAI?$AA?$AA@ 100146f0     libucrt:lcidtoname_downlevel.obj
 0001:00013700       ??_C@_1M@CAFJMKOF@?$AAa?$AAr?$AA?9?$AAY?$AAE?$AA?$AA@ 10014700     libucrt:lcidtoname_downlevel.obj
 0001:0001370c       ??_C@_1M@CBFHIJLI@?$AAe?$AAn?$AA?9?$AAC?$AAB?$AA?$AA@ 1001470c     libucrt:lcidtoname_downlevel.obj
 0001:00013718       ??_C@_1M@BGNFLDN@?$AAe?$AAs?$AA?9?$AAC?$AAO?$AA?$AA@ 10014718     libucrt:lcidtoname_downlevel.obj
 0001:00013724       ??_C@_1O@JMPHMAMC@?$AAs?$AAm?$AAn?$AA?9?$AAF?$AAI?$AA?$AA@ 10014724     libucrt:lcidtoname_downlevel.obj
 0001:00013734       ??_C@_1M@JLANABKE@?$AAa?$AAr?$AA?9?$AAS?$AAY?$AA?$AA@ 10014734     libucrt:lcidtoname_downlevel.obj
 0001:00013740       ??_C@_1M@HPKGCFGN@?$AAe?$AAn?$AA?9?$AAB?$AAZ?$AA?$AA@ 10014740     libucrt:lcidtoname_downlevel.obj
 0001:0001374c       ??_C@_1M@OLJCMLGM@?$AAe?$AAs?$AA?9?$AAP?$AAE?$AA?$AA@ 1001474c     libucrt:lcidtoname_downlevel.obj
 0001:00013758       ??_C@_1M@MKKGFKLE@?$AAa?$AAr?$AA?9?$AAJ?$AAO?$AA?$AA@ 10014758     libucrt:lcidtoname_downlevel.obj
 0001:00013764       ??_C@_1M@EKPGLDNI@?$AAe?$AAn?$AA?9?$AAT?$AAT?$AA?$AA@ 10014764     libucrt:lcidtoname_downlevel.obj
 0001:00013770       ??_C@_1M@OONGHFHE@?$AAe?$AAs?$AA?9?$AAA?$AAR?$AA?$AA@ 10014770     libucrt:lcidtoname_downlevel.obj
 0001:0001377c       ??_C@_1M@OOJFGBHE@?$AAa?$AAr?$AA?9?$AAL?$AAB?$AA?$AA@ 1001477c     libucrt:lcidtoname_downlevel.obj
 0001:00013788       ??_C@_1M@GCEJHNEG@?$AAe?$AAn?$AA?9?$AAZ?$AAW?$AA?$AA@ 10014788     libucrt:lcidtoname_downlevel.obj
 0001:00013794       ??_C@_1M@JNOCAHJI@?$AAe?$AAs?$AA?9?$AAE?$AAC?$AA?$AA@ 10014794     libucrt:lcidtoname_downlevel.obj
 0001:000137a0       ??_C@_1M@JEFHPGGB@?$AAa?$AAr?$AA?9?$AAK?$AAW?$AA?$AA@ 100147a0     libucrt:lcidtoname_downlevel.obj
 0001:000137ac       ??_C@_1M@MLKIBJOJ@?$AAe?$AAn?$AA?9?$AAP?$AAH?$AA?$AA@ 100147ac     libucrt:lcidtoname_downlevel.obj
 0001:000137b8       ??_C@_1M@BDNIPEND@?$AAe?$AAs?$AA?9?$AAC?$AAL?$AA?$AA@ 100147b8     libucrt:lcidtoname_downlevel.obj
 0001:000137c4       ??_C@_1M@MPNMEKBD@?$AAa?$AAr?$AA?9?$AAA?$AAE?$AA?$AA@ 100147c4     libucrt:lcidtoname_downlevel.obj
 0001:000137d0       ??_C@_1M@KBJALCPI@?$AAe?$AAs?$AA?9?$AAU?$AAY?$AA?$AA@ 100147d0     libucrt:lcidtoname_downlevel.obj
 0001:000137dc       ??_C@_1M@LLCCOAGA@?$AAa?$AAr?$AA?9?$AAB?$AAH?$AA?$AA@ 100147dc     libucrt:lcidtoname_downlevel.obj
 0001:000137e8       ??_C@_1M@PBFNCDEL@?$AAe?$AAs?$AA?9?$AAP?$AAY?$AA?$AA@ 100147e8     libucrt:lcidtoname_downlevel.obj
 0001:000137f4       ??_C@_1M@EDGINPNP@?$AAa?$AAr?$AA?9?$AAQ?$AAA?$AA?$AA@ 100147f4     libucrt:lcidtoname_downlevel.obj
 0001:00013800       ??_C@_1M@MKDBIIJI@?$AAe?$AAs?$AA?9?$AAB?$AAO?$AA?$AA@ 10014800     libucrt:lcidtoname_downlevel.obj
 0001:0001380c       ??_C@_1M@CPKKEBLD@?$AAe?$AAs?$AA?9?$AAS?$AAV?$AA?$AA@ 1001480c     libucrt:lcidtoname_downlevel.obj
 0001:00013818       ??_C@_1M@NDBGMMJL@?$AAe?$AAs?$AA?9?$AAH?$AAN?$AA?$AA@ 10014818     libucrt:lcidtoname_downlevel.obj
 0001:00013824       ??_C@_1M@JIJIBHDP@?$AAe?$AAs?$AA?9?$AAN?$AAI?$AA?$AA@ 10014824     libucrt:lcidtoname_downlevel.obj
 0001:00013830       ??_C@_1M@CGFMKEEK@?$AAe?$AAs?$AA?9?$AAP?$AAR?$AA?$AA@ 10014830     libucrt:lcidtoname_downlevel.obj
 0001:0001383c       ??_C@_1O@ICJHKIIK@?$AAz?$AAh?$AA?9?$AAC?$AAH?$AAT?$AA?$AA@ 1001483c     libucrt:lcidtoname_downlevel.obj
 0001:0001384c       ??_C@_15CLNEJCE@?$AAs?$AAr?$AA?$AA@ 1001484c     libucrt:lcidtoname_downlevel.obj
 0001:00013f78       ??_C@_1M@KAHEKEIG@?$AAa?$AAf?$AA?9?$AAz?$AAa?$AA?$AA@ 10014f78     libucrt:lcidtoname_downlevel.obj
 0001:00013f84       ??_C@_1M@GIECOABL@?$AAa?$AAr?$AA?9?$AAa?$AAe?$AA?$AA@ 10014f84     libucrt:lcidtoname_downlevel.obj
 0001:00013f90       ??_C@_1M@BMLMEKGI@?$AAa?$AAr?$AA?9?$AAb?$AAh?$AA?$AA@ 10014f90     libucrt:lcidtoname_downlevel.obj
 0001:00013f9c       ??_C@_1M@DAPFDGGB@?$AAa?$AAr?$AA?9?$AAd?$AAz?$AA?$AA@ 10014f9c     libucrt:lcidtoname_downlevel.obj
 0001:00013fa8       ??_C@_1M@FJNKGKIG@?$AAa?$AAr?$AA?9?$AAe?$AAg?$AA?$AA@ 10014fa8     libucrt:lcidtoname_downlevel.obj
 0001:00013fb4       ??_C@_1M@FLGKKCLO@?$AAa?$AAr?$AA?9?$AAi?$AAq?$AA?$AA@ 10014fb4     libucrt:lcidtoname_downlevel.obj
 0001:00013fc0       ??_C@_1M@GNDIPALM@?$AAa?$AAr?$AA?9?$AAj?$AAo?$AA?$AA@ 10014fc0     libucrt:lcidtoname_downlevel.obj
 0001:00013fcc       ??_C@_1M@DDMJFMGJ@?$AAa?$AAr?$AA?9?$AAk?$AAw?$AA?$AA@ 10014fcc     libucrt:lcidtoname_downlevel.obj
 0001:00013fd8       ??_C@_1M@EJALMLHM@?$AAa?$AAr?$AA?9?$AAl?$AAb?$AA?$AA@ 10014fd8     libucrt:lcidtoname_downlevel.obj
 0001:00013fe4       ??_C@_1M@MOBDBLOC@?$AAa?$AAr?$AA?9?$AAl?$AAy?$AA?$AA@ 10014fe4     libucrt:lcidtoname_downlevel.obj
 0001:00013ff0       ??_C@_1M@JAOCLHDH@?$AAa?$AAr?$AA?9?$AAm?$AAa?$AA?$AA@ 10014ff0     libucrt:lcidtoname_downlevel.obj
 0001:00013ffc       ??_C@_1M@JHPMKJIE@?$AAa?$AAr?$AA?9?$AAo?$AAm?$AA?$AA@ 10014ffc     libucrt:lcidtoname_downlevel.obj
 0001:00014008       ??_C@_1M@OEPGHFNH@?$AAa?$AAr?$AA?9?$AAq?$AAa?$AA?$AA@ 10015008     libucrt:lcidtoname_downlevel.obj
 0001:00014014       ??_C@_1M@KJDONENM@?$AAa?$AAr?$AA?9?$AAs?$AAa?$AA?$AA@ 10015014     libucrt:lcidtoname_downlevel.obj
 0001:00014020       ??_C@_1M@DMJDKLKM@?$AAa?$AAr?$AA?9?$AAs?$AAy?$AA?$AA@ 10015020     libucrt:lcidtoname_downlevel.obj
 0001:0001402c       ??_C@_1M@OMFIPEDC@?$AAa?$AAr?$AA?9?$AAt?$AAn?$AA?$AA@ 1001502c     libucrt:lcidtoname_downlevel.obj
 0001:00014038       ??_C@_1M@IHMHGAON@?$AAa?$AAr?$AA?9?$AAy?$AAe?$AA?$AA@ 10015038     libucrt:lcidtoname_downlevel.obj
 0001:00014044       ??_C@_1BG@KDCPGJGB@?$AAa?$AAz?$AA?9?$AAa?$AAz?$AA?9?$AAc?$AAy?$AAr?$AAl?$AA?$AA@ 10015044     libucrt:lcidtoname_downlevel.obj
 0001:0001405c       ??_C@_1BG@IBCKDDOE@?$AAa?$AAz?$AA?9?$AAa?$AAz?$AA?9?$AAl?$AAa?$AAt?$AAn?$AA?$AA@ 1001505c     libucrt:lcidtoname_downlevel.obj
 0001:00014074       ??_C@_1M@EGPFDCPD@?$AAb?$AAe?$AA?9?$AAb?$AAy?$AA?$AA@ 10015074     libucrt:lcidtoname_downlevel.obj
 0001:00014080       ??_C@_1M@PCMGMCGC@?$AAb?$AAg?$AA?9?$AAb?$AAg?$AA?$AA@ 10015080     libucrt:lcidtoname_downlevel.obj
 0001:0001408c       ??_C@_1M@BJBMFGOB@?$AAb?$AAn?$AA?9?$AAi?$AAn?$AA?$AA@ 1001508c     libucrt:lcidtoname_downlevel.obj
 0001:00014098       ??_C@_1BG@EAKMMACD@?$AAb?$AAs?$AA?9?$AAb?$AAa?$AA?9?$AAl?$AAa?$AAt?$AAn?$AA?$AA@ 10015098     libucrt:lcidtoname_downlevel.obj
 0001:000140b0       ??_C@_1M@KGADAODK@?$AAc?$AAa?$AA?9?$AAe?$AAs?$AA?$AA@ 100150b0     libucrt:lcidtoname_downlevel.obj
 0001:000140bc       ??_C@_1M@COAJPDHI@?$AAc?$AAs?$AA?9?$AAc?$AAz?$AA?$AA@ 100150bc     libucrt:lcidtoname_downlevel.obj
 0001:000140c8       ??_C@_1M@DHBHFONH@?$AAc?$AAy?$AA?9?$AAg?$AAb?$AA?$AA@ 100150c8     libucrt:lcidtoname_downlevel.obj
 0001:000140d4       ??_C@_1M@IMGKELGA@?$AAd?$AAa?$AA?9?$AAd?$AAk?$AA?$AA@ 100150d4     libucrt:lcidtoname_downlevel.obj
 0001:000140e0       ??_C@_1M@NNDGDNGA@?$AAd?$AAe?$AA?9?$AAa?$AAt?$AA?$AA@ 100150e0     libucrt:lcidtoname_downlevel.obj
 0001:000140ec       ??_C@_1M@IKDBHEEM@?$AAd?$AAe?$AA?9?$AAc?$AAh?$AA?$AA@ 100150ec     libucrt:lcidtoname_downlevel.obj
 0001:000140f8       ??_C@_1M@GFFOJMCJ@?$AAd?$AAe?$AA?9?$AAd?$AAe?$AA?$AA@ 100150f8     libucrt:lcidtoname_downlevel.obj
 0001:00014104       ??_C@_1M@MDNLKBPM@?$AAd?$AAe?$AA?9?$AAl?$AAi?$AA?$AA@ 10015104     libucrt:lcidtoname_downlevel.obj
 0001:00014110       ??_C@_1M@NJBEEJNL@?$AAd?$AAe?$AA?9?$AAl?$AAu?$AA?$AA@ 10015110     libucrt:lcidtoname_downlevel.obj
 0001:0001411c       ??_C@_1O@GNNELBAP@?$AAd?$AAi?$AAv?$AA?9?$AAm?$AAv?$AA?$AA@ 1001511c     libucrt:lcidtoname_downlevel.obj
 0001:0001412c       ??_C@_1M@EJLEOGAE@?$AAe?$AAl?$AA?9?$AAg?$AAr?$AA?$AA@ 1001512c     libucrt:lcidtoname_downlevel.obj
 0001:00014138       ??_C@_1M@GMPONJN@?$AAe?$AAn?$AA?9?$AAa?$AAu?$AA?$AA@ 10015138     libucrt:lcidtoname_downlevel.obj
 0001:00014144       ??_C@_1M@NIDIIPGF@?$AAe?$AAn?$AA?9?$AAb?$AAz?$AA?$AA@ 10015144     libucrt:lcidtoname_downlevel.obj
 0001:00014150       ??_C@_1M@JEHMIMFO@?$AAe?$AAn?$AA?9?$AAc?$AAa?$AA?$AA@ 10015150     libucrt:lcidtoname_downlevel.obj
 0001:0001415c       ??_C@_1M@IGMJCDLA@?$AAe?$AAn?$AA?9?$AAc?$AAb?$AA?$AA@ 1001515c     libucrt:lcidtoname_downlevel.obj
 0001:00014168       ??_C@_1M@BNFIGBKG@?$AAe?$AAn?$AA?9?$AAg?$AAb?$AA?$AA@ 10015168     libucrt:lcidtoname_downlevel.obj
 0001:00014174       ??_C@_1M@LKIFDIGP@?$AAe?$AAn?$AA?9?$AAi?$AAe?$AA?$AA@ 10015174     libucrt:lcidtoname_downlevel.obj
 0001:00014180       ??_C@_1M@PJKFGCCO@?$AAe?$AAn?$AA?9?$AAj?$AAm?$AA?$AA@ 10015180     libucrt:lcidtoname_downlevel.obj
 0001:0001418c       ??_C@_1M@KPPKEPBO@?$AAe?$AAn?$AA?9?$AAn?$AAz?$AA?$AA@ 1001518c     libucrt:lcidtoname_downlevel.obj
 0001:00014198       ??_C@_1M@GMDGLDOB@?$AAe?$AAn?$AA?9?$AAp?$AAh?$AA?$AA@ 10015198     libucrt:lcidtoname_downlevel.obj
 0001:000141a4       ??_C@_1M@ONGIBJNA@?$AAe?$AAn?$AA?9?$AAt?$AAt?$AA?$AA@ 100151a4     libucrt:lcidtoname_downlevel.obj
 0001:000141b0       ??_C@_1M@LLODPCMM@?$AAe?$AAn?$AA?9?$AAu?$AAs?$AA?$AA@ 100151b0     libucrt:lcidtoname_downlevel.obj
 0001:000141bc       ??_C@_1M@LAKFNPAN@?$AAe?$AAn?$AA?9?$AAz?$AAa?$AA?$AA@ 100151bc     libucrt:lcidtoname_downlevel.obj
 0001:000141c8       ??_C@_1M@MFNHNHEO@?$AAe?$AAn?$AA?9?$AAz?$AAw?$AA?$AA@ 100151c8     libucrt:lcidtoname_downlevel.obj
 0001:000141d4       ??_C@_1M@EJEINPHM@?$AAe?$AAs?$AA?9?$AAa?$AAr?$AA?$AA@ 100151d4     libucrt:lcidtoname_downlevel.obj
 0001:000141e0       ??_C@_1M@GNKPCCJA@?$AAe?$AAs?$AA?9?$AAb?$AAo?$AA?$AA@ 100151e0     libucrt:lcidtoname_downlevel.obj
 0001:000141ec       ??_C@_1M@LEEGFONL@?$AAe?$AAs?$AA?9?$AAc?$AAl?$AA?$AA@ 100151ec     libucrt:lcidtoname_downlevel.obj
 0001:000141f8       ??_C@_1M@KGPDPBDF@?$AAe?$AAs?$AA?9?$AAc?$AAo?$AA?$AA@ 100151f8     libucrt:lcidtoname_downlevel.obj
 0001:00014204       ??_C@_1M@EIAHOHH@?$AAe?$AAs?$AA?9?$AAc?$AAr?$AA?$AA@ 10015204     libucrt:lcidtoname_downlevel.obj
 0001:00014210       ??_C@_1M@LLPGMBIN@?$AAe?$AAs?$AA?9?$AAd?$AAo?$AA?$AA@ 10015210     libucrt:lcidtoname_downlevel.obj
 0001:0001421c       ??_C@_1M@DKHMKNJA@?$AAe?$AAs?$AA?9?$AAe?$AAc?$AA?$AA@ 1001521c     libucrt:lcidtoname_downlevel.obj
 0001:00014228       ??_C@_1M@GKGFPKAP@?$AAe?$AAs?$AA?9?$AAe?$AAs?$AA?$AA@ 10015228     libucrt:lcidtoname_downlevel.obj
 0001:00014234       ??_C@_1M@LKHKGDLN@?$AAe?$AAs?$AA?9?$AAg?$AAt?$AA?$AA@ 10015234     libucrt:lcidtoname_downlevel.obj
 0001:00014240       ??_C@_1M@HEIIGGJD@?$AAe?$AAs?$AA?9?$AAh?$AAn?$AA?$AA@ 10015240     libucrt:lcidtoname_downlevel.obj
 0001:0001424c       ??_C@_1M@FBDHPPGD@?$AAe?$AAs?$AA?9?$AAm?$AAx?$AA?$AA@ 1001524c     libucrt:lcidtoname_downlevel.obj
 0001:00014258       ??_C@_1M@DPAGLNDH@?$AAe?$AAs?$AA?9?$AAn?$AAi?$AA?$AA@ 10015258     libucrt:lcidtoname_downlevel.obj
 0001:00014264       ??_C@_1M@MDGOPGDD@?$AAe?$AAs?$AA?9?$AAp?$AAa?$AA?$AA@ 10015264     libucrt:lcidtoname_downlevel.obj
 0001:00014270       ??_C@_1M@EMAMGBGE@?$AAe?$AAs?$AA?9?$AAp?$AAe?$AA?$AA@ 10015270     libucrt:lcidtoname_downlevel.obj
 0001:0001427c       ??_C@_1M@IBMCAOEC@?$AAe?$AAs?$AA?9?$AAp?$AAr?$AA?$AA@ 1001527c     libucrt:lcidtoname_downlevel.obj
 0001:00014288       ??_C@_1M@FGMDIJED@?$AAe?$AAs?$AA?9?$AAp?$AAy?$AA?$AA@ 10015288     libucrt:lcidtoname_downlevel.obj
 0001:00014294       ??_C@_1M@IIDEOLLL@?$AAe?$AAs?$AA?9?$AAs?$AAv?$AA?$AA@ 10015294     libucrt:lcidtoname_downlevel.obj
 0001:000142a0       ??_C@_1M@GAOBIPA@?$AAe?$AAs?$AA?9?$AAu?$AAy?$AA?$AA@ 100152a0     libucrt:lcidtoname_downlevel.obj
 0001:000142ac       ??_C@_1M@JKFFICHJ@?$AAe?$AAs?$AA?9?$AAv?$AAe?$AA?$AA@ 100152ac     libucrt:lcidtoname_downlevel.obj
 0001:000142b8       ??_C@_1M@PNMLOJDF@?$AAe?$AAt?$AA?9?$AAe?$AAe?$AA?$AA@ 100152b8     libucrt:lcidtoname_downlevel.obj
 0001:000142c4       ??_C@_1M@GHHLIKEI@?$AAe?$AAu?$AA?9?$AAe?$AAs?$AA?$AA@ 100152c4     libucrt:lcidtoname_downlevel.obj
 0001:000142d0       ??_C@_1M@PBNONODE@?$AAf?$AAa?$AA?9?$AAi?$AAr?$AA?$AA@ 100152d0     libucrt:lcidtoname_downlevel.obj
 0001:000142dc       ??_C@_1M@JEEHPMIL@?$AAf?$AAi?$AA?9?$AAf?$AAi?$AA?$AA@ 100152dc     libucrt:lcidtoname_downlevel.obj
 0001:000142e8       ??_C@_1M@LMDCNDBA@?$AAf?$AAo?$AA?9?$AAf?$AAo?$AA?$AA@ 100152e8     libucrt:lcidtoname_downlevel.obj
 0001:000142f4       ??_C@_1M@JKEOHLDK@?$AAf?$AAr?$AA?9?$AAb?$AAe?$AA?$AA@ 100152f4     libucrt:lcidtoname_downlevel.obj
 0001:00014300       ??_C@_1M@NOHADPMI@?$AAf?$AAr?$AA?9?$AAc?$AAa?$AA?$AA@ 10015300     libucrt:lcidtoname_downlevel.obj
 0001:0001430c       ??_C@_1M@KDHIHAEC@?$AAf?$AAr?$AA?9?$AAc?$AAh?$AA?$AA@ 1001530c     libucrt:lcidtoname_downlevel.obj
 0001:00014318       ??_C@_1M@MMBBFGAK@?$AAf?$AAr?$AA?9?$AAf?$AAr?$AA?$AA@ 10015318     libucrt:lcidtoname_downlevel.obj
 0001:00014324       ??_C@_1M@PAFNENNF@?$AAf?$AAr?$AA?9?$AAl?$AAu?$AA?$AA@ 10015324     libucrt:lcidtoname_downlevel.obj
 0001:00014330       ??_C@_1M@EOHDJGDD@?$AAf?$AAr?$AA?9?$AAm?$AAc?$AA?$AA@ 10015330     libucrt:lcidtoname_downlevel.obj
 0001:0001433c       ??_C@_1M@FAPLLOPF@?$AAg?$AAl?$AA?9?$AAe?$AAs?$AA?$AA@ 1001533c     libucrt:lcidtoname_downlevel.obj
 0001:00014348       ??_C@_1M@FOPBFLOO@?$AAg?$AAu?$AA?9?$AAi?$AAn?$AA?$AA@ 10015348     libucrt:lcidtoname_downlevel.obj
 0001:00014354       ??_C@_1M@KBMCINPM@?$AAh?$AAe?$AA?9?$AAi?$AAl?$AA?$AA@ 10015354     libucrt:lcidtoname_downlevel.obj
 0001:00014360       ??_C@_1M@BBPHKFPJ@?$AAh?$AAi?$AA?9?$AAi?$AAn?$AA?$AA@ 10015360     libucrt:lcidtoname_downlevel.obj
 0001:0001436c       ??_C@_1M@PMBNDPHD@?$AAh?$AAr?$AA?9?$AAb?$AAa?$AA?$AA@ 1001536c     libucrt:lcidtoname_downlevel.obj
 0001:00014378       ??_C@_1M@BPCKOEGE@?$AAh?$AAr?$AA?9?$AAh?$AAr?$AA?$AA@ 10015378     libucrt:lcidtoname_downlevel.obj
 0001:00014384       ??_C@_1M@GACBMHKE@?$AAh?$AAu?$AA?9?$AAh?$AAu?$AA?$AA@ 10015384     libucrt:lcidtoname_downlevel.obj
 0001:00014390       ??_C@_1M@MILPAJJC@?$AAh?$AAy?$AA?9?$AAa?$AAm?$AA?$AA@ 10015390     libucrt:lcidtoname_downlevel.obj
 0001:0001439c       ??_C@_1M@BABBICEC@?$AAi?$AAd?$AA?9?$AAi?$AAd?$AA?$AA@ 1001539c     libucrt:lcidtoname_downlevel.obj
 0001:000143a8       ??_C@_1M@BIKNHHPF@?$AAi?$AAs?$AA?9?$AAi?$AAs?$AA?$AA@ 100153a8     libucrt:lcidtoname_downlevel.obj
 0001:000143b4       ??_C@_1M@NMPCJPHE@?$AAi?$AAt?$AA?9?$AAc?$AAh?$AA?$AA@ 100153b4     libucrt:lcidtoname_downlevel.obj
 0001:000143c0       ??_C@_1M@GHKGFEDF@?$AAi?$AAt?$AA?9?$AAi?$AAt?$AA?$AA@ 100153c0     libucrt:lcidtoname_downlevel.obj
 0001:000143cc       ??_C@_1M@NIEJCJJA@?$AAj?$AAa?$AA?9?$AAj?$AAp?$AA?$AA@ 100153cc     libucrt:lcidtoname_downlevel.obj
 0001:000143d8       ??_C@_1M@JILFNBIM@?$AAk?$AAa?$AA?9?$AAg?$AAe?$AA?$AA@ 100153d8     libucrt:lcidtoname_downlevel.obj
 0001:000143e4       ??_C@_1M@PACPMGPH@?$AAk?$AAk?$AA?9?$AAk?$AAz?$AA?$AA@ 100153e4     libucrt:lcidtoname_downlevel.obj
 0001:000143f0       ??_C@_1M@IELFGMHA@?$AAk?$AAn?$AA?9?$AAi?$AAn?$AA?$AA@ 100153f0     libucrt:lcidtoname_downlevel.obj
 0001:000143fc       ??_C@_1O@IBBJHCH@?$AAk?$AAo?$AAk?$AA?9?$AAi?$AAn?$AA?$AA@ 100153fc     libucrt:lcidtoname_downlevel.obj
 0001:0001440c       ??_C@_1M@DMHAEOGC@?$AAk?$AAo?$AA?9?$AAk?$AAr?$AA?$AA@ 1001540c     libucrt:lcidtoname_downlevel.obj
 0001:00014418       ??_C@_1M@HBAHBIGA@?$AAk?$AAy?$AA?9?$AAk?$AAg?$AA?$AA@ 10015418     libucrt:lcidtoname_downlevel.obj
 0001:00014424       ??_C@_1M@KPMILCJG@?$AAl?$AAt?$AA?9?$AAl?$AAt?$AA?$AA@ 10015424     libucrt:lcidtoname_downlevel.obj
 0001:00014430       ??_C@_1M@BDEKKCA@?$AAl?$AAv?$AA?9?$AAl?$AAv?$AA?$AA@ 10015430     libucrt:lcidtoname_downlevel.obj
 0001:0001443c       ??_C@_1M@ELCKCCJJ@?$AAm?$AAi?$AA?9?$AAn?$AAz?$AA?$AA@ 1001543c     libucrt:lcidtoname_downlevel.obj
 0001:00014448       ??_C@_1M@CBOOLAPA@?$AAm?$AAk?$AA?9?$AAm?$AAk?$AA?$AA@ 10015448     libucrt:lcidtoname_downlevel.obj
 0001:00014454       ??_C@_1M@GPHNBJKN@?$AAm?$AAl?$AA?9?$AAi?$AAn?$AA?$AA@ 10015454     libucrt:lcidtoname_downlevel.obj
 0001:00014460       ??_C@_1M@PABJILIG@?$AAm?$AAn?$AA?9?$AAm?$AAn?$AA?$AA@ 10015460     libucrt:lcidtoname_downlevel.obj
 0001:0001446c       ??_C@_1M@FGBKKIPG@?$AAm?$AAr?$AA?9?$AAi?$AAn?$AA?$AA@ 1001546c     libucrt:lcidtoname_downlevel.obj
 0001:00014478       ??_C@_1M@NDBPDDAL@?$AAm?$AAs?$AA?9?$AAb?$AAn?$AA?$AA@ 10015478     libucrt:lcidtoname_downlevel.obj
 0001:00014484       ??_C@_1M@OPIHOOPI@?$AAm?$AAs?$AA?9?$AAm?$AAy?$AA?$AA@ 10015484     libucrt:lcidtoname_downlevel.obj
 0001:00014490       ??_C@_1M@PPDBCNFM@?$AAm?$AAt?$AA?9?$AAm?$AAt?$AA?$AA@ 10015490     libucrt:lcidtoname_downlevel.obj
 0001:0001449c       ??_C@_1M@KDJDKMDD@?$AAn?$AAb?$AA?9?$AAn?$AAo?$AA?$AA@ 1001549c     libucrt:lcidtoname_downlevel.obj
 0001:000144a8       ??_C@_1M@KFCFLMJP@?$AAn?$AAl?$AA?9?$AAb?$AAe?$AA?$AA@ 100154a8     libucrt:lcidtoname_downlevel.obj
 0001:000144b4       ??_C@_1M@KPOPDDGO@?$AAn?$AAl?$AA?9?$AAn?$AAl?$AA?$AA@ 100154b4     libucrt:lcidtoname_downlevel.obj
 0001:000144c0       ??_C@_1M@LJKPEMLN@?$AAn?$AAn?$AA?9?$AAn?$AAo?$AA?$AA@ 100154c0     libucrt:lcidtoname_downlevel.obj
 0001:000144cc       ??_C@_1M@BDGHHBFL@?$AAn?$AAs?$AA?9?$AAz?$AAa?$AA?$AA@ 100154cc     libucrt:lcidtoname_downlevel.obj
 0001:000144d8       ??_C@_1M@IDEHOAP@?$AAp?$AAa?$AA?9?$AAi?$AAn?$AA?$AA@ 100154d8     libucrt:lcidtoname_downlevel.obj
 0001:000144e4       ??_C@_1M@HDBKGOGH@?$AAp?$AAl?$AA?9?$AAp?$AAl?$AA?$AA@ 100154e4     libucrt:lcidtoname_downlevel.obj
 0001:000144f0       ??_C@_1M@LJLLCMEH@?$AAp?$AAt?$AA?9?$AAb?$AAr?$AA?$AA@ 100154f0     libucrt:lcidtoname_downlevel.obj
 0001:000144fc       ??_C@_1M@NCMONAAL@?$AAp?$AAt?$AA?9?$AAp?$AAt?$AA?$AA@ 100154fc     libucrt:lcidtoname_downlevel.obj
 0001:00014508       ??_C@_1O@EAKMAJDN@?$AAq?$AAu?$AAz?$AA?9?$AAb?$AAo?$AA?$AA@ 10015508     libucrt:lcidtoname_downlevel.obj
 0001:00014518       ??_C@_1O@BHHPIGDN@?$AAq?$AAu?$AAz?$AA?9?$AAe?$AAc?$AA?$AA@ 10015518     libucrt:lcidtoname_downlevel.obj
 0001:00014528       ??_C@_1O@GBAPEKMJ@?$AAq?$AAu?$AAz?$AA?9?$AAp?$AAe?$AA?$AA@ 10015528     libucrt:lcidtoname_downlevel.obj
 0001:00014538       ??_C@_1M@CLGLEFBO@?$AAr?$AAo?$AA?9?$AAr?$AAo?$AA?$AA@ 10015538     libucrt:lcidtoname_downlevel.obj
 0001:00014544       ??_C@_1M@CEEDODME@?$AAr?$AAu?$AA?9?$AAr?$AAu?$AA?$AA@ 10015544     libucrt:lcidtoname_downlevel.obj
 0001:00014550       ??_C@_1M@HPKKKMPP@?$AAs?$AAa?$AA?9?$AAi?$AAn?$AA?$AA@ 10015550     libucrt:lcidtoname_downlevel.obj
 0001:0001455c       ??_C@_1M@BKMAIGOJ@?$AAs?$AAe?$AA?9?$AAf?$AAi?$AA?$AA@ 1001555c     libucrt:lcidtoname_downlevel.obj
 0001:00014568       ??_C@_1M@NDPIFLFI@?$AAs?$AAe?$AA?9?$AAn?$AAo?$AA?$AA@ 10015568     libucrt:lcidtoname_downlevel.obj
 0001:00014574       ??_C@_1M@DANKKHJ@?$AAs?$AAe?$AA?9?$AAs?$AAe?$AA?$AA@ 10015574     libucrt:lcidtoname_downlevel.obj
 0001:00014580       ??_C@_1M@PNBLONPJ@?$AAs?$AAk?$AA?9?$AAs?$AAk?$AA?$AA@ 10015580     libucrt:lcidtoname_downlevel.obj
 0001:0001458c       ??_C@_1M@LFMODOAL@?$AAs?$AAl?$AA?9?$AAs?$AAi?$AA?$AA@ 1001558c     libucrt:lcidtoname_downlevel.obj
 0001:00014598       ??_C@_1O@DFKOMPG@?$AAs?$AAm?$AAa?$AA?9?$AAn?$AAo?$AA?$AA@ 10015598     libucrt:lcidtoname_downlevel.obj
 0001:000145a8       ??_C@_1O@NDKPBNNH@?$AAs?$AAm?$AAa?$AA?9?$AAs?$AAe?$AA?$AA@ 100155a8     libucrt:lcidtoname_downlevel.obj
 0001:000145b8       ??_C@_1O@PLLKBHAB@?$AAs?$AAm?$AAj?$AA?9?$AAn?$AAo?$AA?$AA@ 100155b8     libucrt:lcidtoname_downlevel.obj
 0001:000145c8       ??_C@_1O@CLEPOGCA@?$AAs?$AAm?$AAj?$AA?9?$AAs?$AAe?$AA?$AA@ 100155c8     libucrt:lcidtoname_downlevel.obj
 0001:000145d8       ??_C@_1O@DLGJGKMK@?$AAs?$AAm?$AAn?$AA?9?$AAf?$AAi?$AA?$AA@ 100155d8     libucrt:lcidtoname_downlevel.obj
 0001:000145e8       ??_C@_1O@OJDJGAJC@?$AAs?$AAm?$AAs?$AA?9?$AAf?$AAi?$AA?$AA@ 100155e8     libucrt:lcidtoname_downlevel.obj
 0001:000145f8       ??_C@_1M@BOFOGHPB@?$AAs?$AAq?$AA?9?$AAa?$AAl?$AA?$AA@ 100155f8     libucrt:lcidtoname_downlevel.obj
 0001:00014604       ??_C@_1BG@LJBBIPGB@?$AAs?$AAr?$AA?9?$AAb?$AAa?$AA?9?$AAc?$AAy?$AAr?$AAl?$AA?$AA@ 10015604     libucrt:lcidtoname_downlevel.obj
 0001:0001461c       ??_C@_1BG@JLBENFOE@?$AAs?$AAr?$AA?9?$AAb?$AAa?$AA?9?$AAl?$AAa?$AAt?$AAn?$AA?$AA@ 1001561c     libucrt:lcidtoname_downlevel.obj
 0001:00014634       ??_C@_1BG@KODPNHE@?$AAs?$AAr?$AA?9?$AAs?$AAp?$AA?9?$AAc?$AAy?$AAr?$AAl?$AA?$AA@ 10015634     libucrt:lcidtoname_downlevel.obj
 0001:0001464c       ??_C@_1BG@CIOGKHPB@?$AAs?$AAr?$AA?9?$AAs?$AAp?$AA?9?$AAl?$AAa?$AAt?$AAn?$AA?$AA@ 1001564c     libucrt:lcidtoname_downlevel.obj
 0001:00014664       ??_C@_1M@NGFJLMAC@?$AAs?$AAv?$AA?9?$AAf?$AAi?$AA?$AA@ 10015664     libucrt:lcidtoname_downlevel.obj
 0001:00014670       ??_C@_1M@MPJEJAJC@?$AAs?$AAv?$AA?9?$AAs?$AAe?$AA?$AA@ 10015670     libucrt:lcidtoname_downlevel.obj
 0001:0001467c       ??_C@_1M@MPNDHLFK@?$AAs?$AAw?$AA?9?$AAk?$AAe?$AA?$AA@ 1001567c     libucrt:lcidtoname_downlevel.obj
 0001:00014688       ??_C@_1O@KOHBJJI@?$AAs?$AAy?$AAr?$AA?9?$AAs?$AAy?$AA?$AA@ 10015688     libucrt:lcidtoname_downlevel.obj
 0001:00014698       ??_C@_1M@LDCEFHA@?$AAt?$AAa?$AA?9?$AAi?$AAn?$AA?$AA@ 10015698     libucrt:lcidtoname_downlevel.obj
 0001:000146a4       ??_C@_1M@CNJOFAK@?$AAt?$AAe?$AA?9?$AAi?$AAn?$AA?$AA@ 100156a4     libucrt:lcidtoname_downlevel.obj
 0001:000146b0       ??_C@_1M@GNAECACD@?$AAt?$AAh?$AA?9?$AAt?$AAh?$AA?$AA@ 100156b0     libucrt:lcidtoname_downlevel.obj
 0001:000146bc       ??_C@_1M@CHBIHOJO@?$AAt?$AAn?$AA?9?$AAz?$AAa?$AA?$AA@ 100156bc     libucrt:lcidtoname_downlevel.obj
 0001:000146c8       ??_C@_1M@GCCMIGPJ@?$AAt?$AAr?$AA?9?$AAt?$AAr?$AA?$AA@ 100156c8     libucrt:lcidtoname_downlevel.obj
 0001:000146d4       ??_C@_1M@CELMCNBK@?$AAt?$AAt?$AA?9?$AAr?$AAu?$AA?$AA@ 100156d4     libucrt:lcidtoname_downlevel.obj
 0001:000146e0       ??_C@_1M@KLMCELGA@?$AAu?$AAk?$AA?9?$AAu?$AAa?$AA?$AA@ 100156e0     libucrt:lcidtoname_downlevel.obj
 0001:000146ec       ??_C@_1M@EPAJJAJF@?$AAu?$AAr?$AA?9?$AAp?$AAk?$AA?$AA@ 100156ec     libucrt:lcidtoname_downlevel.obj
 0001:000146f8       ??_C@_1BG@GEGPMCDJ@?$AAu?$AAz?$AA?9?$AAu?$AAz?$AA?9?$AAc?$AAy?$AAr?$AAl?$AA?$AA@ 100156f8     libucrt:lcidtoname_downlevel.obj
 0001:00014710       ??_C@_1BG@EGGKJILM@?$AAu?$AAz?$AA?9?$AAu?$AAz?$AA?9?$AAl?$AAa?$AAt?$AAn?$AA?$AA@ 10015710     libucrt:lcidtoname_downlevel.obj
 0001:00014728       ??_C@_1M@GFOCLFF@?$AAv?$AAi?$AA?9?$AAv?$AAn?$AA?$AA@ 10015728     libucrt:lcidtoname_downlevel.obj
 0001:00014734       ??_C@_1M@CPAMEDFI@?$AAx?$AAh?$AA?9?$AAz?$AAa?$AA?$AA@ 10015734     libucrt:lcidtoname_downlevel.obj
 0001:00014740       ??_C@_1O@EBKIFIGN@?$AAz?$AAh?$AA?9?$AAc?$AAh?$AAs?$AA?$AA@ 10015740     libucrt:lcidtoname_downlevel.obj
 0001:00014750       ??_C@_1O@NMHPGANE@?$AAz?$AAh?$AA?9?$AAc?$AAh?$AAt?$AA?$AA@ 10015750     libucrt:lcidtoname_downlevel.obj
 0001:00014760       ??_C@_1M@LPINJOMC@?$AAz?$AAh?$AA?9?$AAc?$AAn?$AA?$AA@ 10015760     libucrt:lcidtoname_downlevel.obj
 0001:0001476c       ??_C@_1M@OCJEJODD@?$AAz?$AAh?$AA?9?$AAh?$AAk?$AA?$AA@ 1001576c     libucrt:lcidtoname_downlevel.obj
 0001:00014778       ??_C@_1M@DNDLJINH@?$AAz?$AAh?$AA?9?$AAm?$AAo?$AA?$AA@ 10015778     libucrt:lcidtoname_downlevel.obj
 0001:00014784       ??_C@_1M@MBFDNDND@?$AAz?$AAh?$AA?9?$AAs?$AAg?$AA?$AA@ 10015784     libucrt:lcidtoname_downlevel.obj
 0001:00014790       ??_C@_1M@IMEPLEPE@?$AAz?$AAh?$AA?9?$AAt?$AAw?$AA?$AA@ 10015790     libucrt:lcidtoname_downlevel.obj
 0001:0001479c       ??_C@_1M@BBGHNHJP@?$AAz?$AAu?$AA?9?$AAz?$AAa?$AA?$AA@ 1001579c     libucrt:lcidtoname_downlevel.obj
 0001:00014808       ??_C@_1BA@BALFACEM@?$AAC?$AAO?$AAN?$AAO?$AAU?$AAT?$AA$?$AA?$AA@ 10015808     libucrt:initcon.obj
 0001:00014920       __infinity                 10015920     libucrt:87tran.obj
 0001:0001492a       __minfinity                1001592a     libucrt:87tran.obj
 0001:00014934       __logemax                  10015934     libucrt:87tran.obj
 0001:0001495a       __OP_EXPjmptab             1001595a     libucrt:87tran.obj
 0001:00014980       __indefinite               10015980     libucrt:87disp.obj
 0001:0001498a       __piby2                    1001598a     libucrt:87disp.obj
 0001:00014994       __piby4                    10015994     libucrt:87disp.obj
 0001:000149c8       __DEFAULT_CW_in_mem        100159c8     libucrt:common.obj
 0001:000149ca       __pi_by_2_to_61            100159ca     libucrt:common.obj
 0001:00014a04       ??_C@_03MGHMBJCF@log?$AA@  10015a04     libucrt:libm_error.obj
 0001:00014a08       ??_C@_05HGHHAHAP@log10?$AA@ 10015a08     libucrt:libm_error.obj
 0001:00014a10       ??_C@_03KHJOGHMM@exp?$AA@  10015a10     libucrt:libm_error.obj
 0001:00014a14       ??_C@_03JGHBODFD@pow?$AA@  10015a14     libucrt:libm_error.obj
 0001:00014a18       ??_C@_04FIHNOPOL@asin?$AA@ 10015a18     libucrt:libm_error.obj
 0001:00014a20       ??_C@_04PDIFKINK@acos?$AA@ 10015a20     libucrt:libm_error.obj
 0001:00014a28       ??_C@_04EIAKFFMI@sqrt?$AA@ 10015a28     libucrt:libm_error.obj
 0001:00014a30       ___acrt_log10_table_t      10015a30     libucrt:log10_tables.obj
 0001:00014e40       ___acrt_log10_table_cb     10015e40     libucrt:log10_tables.obj
 0001:00015250       __real@3fe0000000000000    10016250     libucrt:powhlp.obj
 0001:00015258       ??_C@_04FJHINJAO@tanh?$AA@ 10016258     libucrt:fpexcept.obj
 0001:00015260       ??_C@_04MLLJIGOK@atan?$AA@ 10016260     libucrt:fpexcept.obj
 0001:00015268       ??_C@_05KNGEOGJB@atan2?$AA@ 10016268     libucrt:fpexcept.obj
 0001:00015270       ??_C@_03BLEJJJBH@sin?$AA@  10016270     libucrt:fpexcept.obj
 0001:00015274       ??_C@_03LALBNOCG@cos?$AA@  10016274     libucrt:fpexcept.obj
 0001:00015278       ??_C@_03IIINPABG@tan?$AA@  10016278     libucrt:fpexcept.obj
 0001:0001527c       ??_C@_04GFPJNGEK@ceil?$AA@ 1001627c     libucrt:fpexcept.obj
 0001:00015284       ??_C@_05PBJFFIGL@floor?$AA@ 10016284     libucrt:fpexcept.obj
 0001:0001528c       ??_C@_04ODHECPBC@fabs?$AA@ 1001628c     libucrt:fpexcept.obj
 0001:00015294       ??_C@_04EHEDPDJG@modf?$AA@ 10016294     libucrt:fpexcept.obj
 0001:0001529c       ??_C@_05CEJMAHNP@ldexp?$AA@ 1001629c     libucrt:fpexcept.obj
 0001:000152a4       ??_C@_05KBKMEMPO@_cabs?$AA@ 100162a4     libucrt:fpexcept.obj
 0001:000152ac       ??_C@_06MEIMCGCF@_hypot?$AA@ 100162ac     libucrt:fpexcept.obj
 0001:000152b4       ??_C@_04KEPJIHGP@fmod?$AA@ 100162b4     libucrt:fpexcept.obj
 0001:000152bc       ??_C@_05GKKHEGJL@frexp?$AA@ 100162bc     libucrt:fpexcept.obj
 0001:000152c4       ??_C@_03MJLDFKDL@_y0?$AA@  100162c4     libucrt:fpexcept.obj
 0001:000152c8       ??_C@_03NAKIGLHK@_y1?$AA@  100162c8     libucrt:fpexcept.obj
 0001:000152cc       ??_C@_03ONILCKOB@_yn?$AA@  100162cc     libucrt:fpexcept.obj
 0001:000152d0       ??_C@_05JGDBENOH@_logb?$AA@ 100162d0     libucrt:fpexcept.obj
 0001:000152d8       ??_C@_0L@KDOEJCKC@_nextafter?$AA@ 100162d8     libucrt:fpexcept.obj
 0001:000153d0       ??_C@_04COOMCNPB@sinh?$AA@ 100163d0     libucrt:fpexcept.obj
 0001:000153d8       ??_C@_04HPJJNFIM@cosh?$AA@ 100163d8     libucrt:fpexcept.obj
 0001:000153e0       __d_inf                    100163e0     libucrt:util.obj
 0001:000153e8       __d_max                    100163e8     libucrt:util.obj
 0001:000153f0       __d_mzero                  100163f0     libucrt:util.obj
 0001:00015420       __load_config_used         10016420     LIBCMT:loadcfg.obj
 0001:00015480       ___safe_se_handler_table   10016480     <linker-defined>
 0001:00015718       ___rtc_iaa                 10016718     LIBCMT:_initsect_.obj
 0001:0001571c       ___rtc_izz                 1001671c     LIBCMT:_initsect_.obj
 0001:00015720       ___rtc_taa                 10016720     LIBCMT:_initsect_.obj
 0001:00015724       ___rtc_tzz                 10016724     LIBCMT:_initsect_.obj
 0001:00015730       __alloca_probe             10016730 f   chkstk.obj
 0001:00015730       __chkstk                   10016730 f   chkstk.obj
 0001:00016460       ___local_stdio_printf_options 10017460 f i bit64.obj
 0001:00016470       _bit64_getvalue            10017470 f   bit64.obj
 0001:000164f0       _bit64_push                100174f0 f   bit64.obj
 0001:00016580       _bit64_pushuserdata        10017580 f   bit64.obj
 0001:000166a0       _luaopen_bit64             100176a0 f   bit64.obj
 0001:000166e0       _sprintf                   100176e0 f i bit64.obj
 0001:00016710       _AddBufToCollector         10017710 f   exported.obj
 0001:00016760       _AddStringToCollectorField 10017760 f   exported.obj
 0001:00016840       _CreateStringsArray        10017840 f   exported.obj
 0001:00016980       _DestroyCollector          10017980 f   exported.obj
 0001:000169c0       _FarPanelItemFreeCallback@8 100179c0 f   exported.obj
 0001:00016c30       _FillFindData              10017c30 f   exported.obj
 0001:00016f60       _FillPluginPanelItem       10017f60 f   exported.obj
 0001:00017150       _GetExportFunction         10018150 f   exported.obj
 0001:000171d0       _LF_Analyse                100181d0 f   exported.obj
 0001:00017270       _LF_CloseAnalyse           10018270 f   exported.obj
 0001:00017290       _LF_ClosePanel             10018290 f   exported.obj
 0001:00017330       _LF_Compare                10018330 f   exported.obj
 0001:000173e0       _LF_Configure              100183e0 f   exported.obj
 0001:00017440       _LF_DeleteFiles            10018440 f   exported.obj
 0001:000174f0       _LF_ExitFAR                100184f0 f   exported.obj
 0001:00017550       _LF_FreeContentData        10018550 f   exported.obj
 0001:00017580       _LF_FreeFindData           10018580 f   exported.obj
 0001:000175d0       _LF_GetContentData         100185d0 f   exported.obj
 0001:000176e0       _LF_GetContentFields       100186e0 f   exported.obj
 0001:00017770       _LF_GetFiles               10018770 f   exported.obj
 0001:000178a0       _LF_GetFindData            100188a0 f   exported.obj
 0001:00017970       _LF_GetGlobalInfo          10018970 f   exported.obj
 0001:00017d00       _LF_GetOpenPanelInfo       10018d00 f   exported.obj
 0001:00018350       _LF_GetPluginInfo          10019350 f   exported.obj
 0001:00018450       _LF_MakeDirectory          10019450 f   exported.obj
 0001:00018550       _LF_Open                   10019550 f   exported.obj
 0001:000188b0       _LF_ProcessConsoleInput    100198b0 f   exported.obj
 0001:00018990       _LF_ProcessDialogEvent     10019990 f   exported.obj
 0001:00018b50       _LF_ProcessEditorEvent     10019b50 f   exported.obj
 0001:00018c80       _LF_ProcessEditorInput     10019c80 f   exported.obj
 0001:00018ce0       _LF_ProcessHostFile        10019ce0 f   exported.obj
 0001:00018db0       _LF_ProcessPanelEvent      10019db0 f   exported.obj
 0001:00018e70       _LF_ProcessPanelInput      10019e70 f   exported.obj
 0001:00018f00       _LF_ProcessSynchroEvent    10019f00 f   exported.obj
 0001:000190b0       _LF_ProcessViewerEvent     1001a0b0 f   exported.obj
 0001:00019130       _LF_PutFiles               1001a130 f   exported.obj
 0001:00019210       _LF_RunDefaultScript       1001a210 f   exported.obj
 0001:00019220       _LF_SetDirectory           1001a220 f   exported.obj
 0001:000192c0       _LF_SetFindList            1001a2c0 f   exported.obj
 0001:00019350       _PackMacroValues           1001a350 f   exported.obj
 0001:000194f0       _PushFarMacroValue         1001a4f0 f   exported.obj
 0001:00019640       _ReplacePluginInfoCollector 1001a640 f   exported.obj
 0001:00019860       _UpdateFileSelection       1001a860 f   exported.obj
 0001:00019920       _getPluginMenuItems        1001a920 f   exported.obj
 0001:000199b0       _pcall_msg                 1001a9b0 f   exported.obj
 0001:00019a60       _traceback                 1001aa60 f   exported.obj
 0001:00019af0       _push_flags_table          1001aaf0 f   flags.obj
 0001:00019b40       _SetFarColors              1001ab40 f   keysandcolors.obj
 0001:00019b90       _LF_Gsub                   1001ab90 f   lflua.obj
 0001:00019ca0       _LF_LoadFile               1001aca0 f   lflua.obj
 0001:00019f40       _luaB_dofileW              1001af40 f   lflua.obj
 0001:00019f90       _luaB_loadfileW            1001af90 f   lflua.obj
 0001:0001a030       _method_gc                 1001b030 f   lregex.obj
 0001:0001a090       _method_tostring           1001b090 f   lregex.obj
 0001:0001a0e0       _func_Gmatch               1001b0e0 f   lregex.obj
 0001:0001a0f0       _func_GmatchW              1001b0f0 f   lregex.obj
 0001:0001a100       _method_bracketscount      1001b100 f   lregex.obj
 0001:0001a160       _func_New                  1001b160 f   lregex.obj
 0001:0001a190       _method_find               1001b190 f   lregex.obj
 0001:0001a1b0       _func_find                 1001b1b0 f   lregex.obj
 0001:0001a1d0       _method_findW              1001b1d0 f   lregex.obj
 0001:0001a1f0       _func_findW                1001b1f0 f   lregex.obj
 0001:0001a210       _method_match              1001b210 f   lregex.obj
 0001:0001a230       _func_match                1001b230 f   lregex.obj
 0001:0001a250       _method_matchW             1001b250 f   lregex.obj
 0001:0001a270       _func_matchW               1001b270 f   lregex.obj
 0001:0001a290       _method_gsub               1001b290 f   lregex.obj
 0001:0001a2b0       _func_gsub                 1001b2b0 f   lregex.obj
 0001:0001a2d0       _method_gsubW              1001b2d0 f   lregex.obj
 0001:0001a2f0       _func_gsubW                1001b2f0 f   lregex.obj
 0001:0001a310       __Gmatch                   1001b310 f   lregex.obj
 0001:0001a3f0       __regex_gmatch_closure     1001b3f0 f   lregex.obj
 0001:0001a4d0       _check_regex_pattern       1001b4d0 f   lregex.obj
 0001:0001a570       _luaopen_regex             1001b570 f   lregex.obj
 0001:0001a5e0       _push_far_regex            1001b5e0 f   lregex.obj
 0001:0001a650       _regex_gmatch_closure      1001b650 f   lregex.obj
 0001:0001a660       _regex_gmatch_closureW     1001b660 f   lregex.obj
 0001:0001a670       _rx_find_match             1001b670 f   lregex.obj
 0001:0001a8a0       _rx_gsub                   1001b8a0 f   lregex.obj
 0001:0001b0d0       _Open_Luamacro             1001c0d0 f   luamacro.obj
 0001:0001b460       _far_FarMacroCallToLua     1001c460 f   luamacro.obj
 0001:0001b4d0       _far_MacroCallFar          1001c4d0 f   luamacro.obj
 0001:0001b6b0       _uc_len                    1001c6b0 f   lusercontrol.obj
 0001:0001b920       _CheckFarUserControl       1001c920 f   lusercontrol.obj
 0001:0001b940       _luaopen_usercontrol       1001c940 f   lusercontrol.obj
 0001:0001b980       _CreateRegKey              1001c980 f   reg.obj
 0001:0001b9c0       _OpenRegKey                1001c9c0 f   reg.obj
 0001:0001b9f0       _SetRegKeyArr              1001c9f0 f   reg.obj
 0001:0001ba50       _SetRegKeyDword            1001ca50 f   reg.obj
 0001:0001bab0       _SetRegKeyStr              1001cab0 f   reg.obj
 0001:00024bd0       _ConvertLuaValue           10025bd0 f   service.obj
 0001:00024d20       _CreateList                10025d20 f   service.obj
 0001:00024ee0       _DialogHandleEqual         10025ee0 f   service.obj
 0001:00024f20       _DllMain@12                10025f20 f   service.obj
 0001:00025140       _FillInputRecord           10026140 f   service.obj
 0001:000255d0       _GetFarColor               100265d0 f   service.obj
 0001:00025740       _GetFlagCombination        10026740 f   service.obj
 0001:00025980       _GetFlagsFromTable         10026980 f   service.obj
 0001:00025ad0       _GetPluginData             10026ad0 f   service.obj
 0001:00025af0       _IsLuaJIT                  10026af0 f   service.obj
 0001:00025b00       _LF_DlgProc                10026b00 f   service.obj
 0001:00025c50       _LF_DoFile                 10026c50 f   service.obj
 0001:00025ce0       _LF_Error                  10026ce0 f   service.obj
 0001:00025da0       _LF_GetLuafarAPI           10026da0 f   service.obj
 0001:00025dd0       _LF_InitLuaState1          10026dd0 f   service.obj
 0001:00025f20       _LF_InitLuaState2          10026f20 f   service.obj
 0001:00025fc0       _LF_MacroCallback          10026fc0 f   service.obj
 0001:00025fd0       _LF_Message                10026fd0 f   service.obj
 0001:00026460       ___except_validate_context_record 10027460 f   libvcruntime:jbcxrval.obj
 0001:00026460       ___except_validate_jump_buffer 10027460 f   libvcruntime:jbcxrval.obj
 0001:00026460       _LF_ProcessEnvVars         10027460 f   service.obj
 0001:00026460       @_guard_check_icall_nop@4  10027460 f   LIBCMT:guard_support.obj
 0001:00026470       _LF_RunLuafarInit          10027470 f   service.obj
 0001:00026530       _MacroAddCallback@12       10027530 f   service.obj
 0001:000266a0       _NewDialogData             100276a0 f   service.obj
 0001:00026710       _NewVirtualKeyTable        10027710 f   service.obj
 0001:00026790       _OptFlags                  10027790 f   service.obj
 0001:000267f0       _OptHandle                 100277f0 f   service.obj
 0001:00026910       _ProcessDNResult           10027910 f   service.obj
 0001:00026cf0       _PushDMParams              10027cf0 f   service.obj
 0001:00026dd0       _PushDNParams              10027dd0 f   service.obj
 0001:00027280       _PushFarColor              10028280 f   service.obj
 0001:00027310       _PushInputRecord           10028310 f   service.obj
 0001:000275a0       _PushPanelItem             100285a0 f   service.obj
 0001:000277f0       _PushPanelItems            100287f0 f   service.obj
 0001:00027ad0       _PutFlagsToTable           10028ad0 f   service.obj
 0001:00027b00       _PutMouseEvent             10028b00 f   service.obj
 0001:00028270       _TimerCallback@8           10029270 f   service.obj
 0001:00028800       _dir_exist                 10029800 f   service.obj
 0001:00028820       _fprintf                   10029820 f i service.obj
 0001:00028ec0       _pushFileTime              10029ec0 f   service.obj
 0001:00029f90       __snwprintf                1002af90 f i slnunico.obj
 0001:0002a660       _luaopen_unicode           1002b660 f   slnunico.obj
 0001:0002c4b0       ___local_stdio_scanf_options 1002d4b0 f i uliolib51.obj
 0001:0002c540       _fscanf                    1002d540 f i uliolib51.obj
 0001:0002cad0       _luaopen_uio               1002dad0 f   uliolib51.obj
 0001:0002d7d0       _luaopen_upackage          1002e7d0 f   uloadlib51.obj
 0001:0002dc20       _ustring_GetDriveType      1002ec20 f   ustring.obj
 0001:0002dd10       _ustring_Uuid              1002ed10 f   ustring.obj
 0001:0002ddf0       _ustring_SearchPath        1002edf0 f   ustring.obj
 0001:0002dff0       _ustring_GlobalMemoryStatus 1002eff0 f   ustring.obj
 0001:0002e2f0       _ustring_Sleep             1002f2f0 f   ustring.obj
 0001:0002e330       _ustring_SetFileAttr       1002f330 f   ustring.obj
 0001:0002e420       _ustring_GetFileAttr       1002f420 f   ustring.obj
 0001:0002e500       _ustring_SHGetFolderPath   1002f500 f   ustring.obj
 0001:0002e600       _ustring_sub               1002f600 f   ustring.obj
 0001:0002e690       _ustring_len               1002f690 f   ustring.obj
 0001:0002e8b0       _ustring_GetCurrentDir     1002f8b0 f   ustring.obj
 0001:0002ea50       _ustring_SetCurrentDir     1002fa50 f   ustring.obj
 0001:0002eb30       _ustring_GetKeyState       1002fb30 f   ustring.obj
 0001:0002eb70       _ustring_WideCharToMultiByte 1002fb70 f   ustring.obj
 0001:0002eca0       _ustring_MultiByteToWideChar 1002fca0 f   ustring.obj
 0001:0002ede0       _ustring_OemToUtf8         1002fde0 f   ustring.obj
 0001:0002eea0       _ustring_Utf8ToOem         1002fea0 f   ustring.obj
 0001:0002ef50       _ustring_Utf16ToUtf8       1002ff50 f   ustring.obj
 0001:0002ef90       _ustring_Utf8ToUtf16       1002ff90 f   ustring.obj
 0001:0002f040       _ustring_GetACP            10030040 f   ustring.obj
 0001:0002f060       _ustring_GetOEMCP          10030060 f   ustring.obj
 0001:0002f080       _ustring_EnumSystemCodePages 10030080 f   ustring.obj
 0001:0002f0f0       _ustring_GetCPInfo         100300f0 f   ustring.obj
 0001:0002f2f0       _ustring_GetLogicalDriveStrings 100302f0 f   ustring.obj
 0001:0002f430       _DecodeAttributes          10030430 f   ustring.obj
 0001:0002f500       _EnumCodePagesProc@4       10030500 f   ustring.obj
 0001:0002f5c0       _GetBoolFromTable          100305c0 f   ustring.obj
 0001:0002f5f0       _GetOptBoolFromTable       100305f0 f   ustring.obj
 0001:0002f650       _GetOptIntFromArray        10030650 f   ustring.obj
 0001:0002f6a0       _GetOptIntFromTable        100306a0 f   ustring.obj
 0001:0002f6f0       _GetOptNumFromTable        100306f0 f   ustring.obj
 0001:0002f740       _PushAttrString            10030740 f   ustring.obj
 0001:0002f7d0       _PutAttrToTable            100307d0 f   ustring.obj
 0001:0002f800       _PutBoolToTable            10030800 f   ustring.obj
 0001:0002f820       _PutIntToArray             10030820 f   ustring.obj
 0001:0002f860       _PutIntToTable             10030860 f   ustring.obj
 0001:0002f8a0       _PutLStrToTable            100308a0 f   ustring.obj
 0001:0002f8d0       _PutNumToTable             100308d0 f   ustring.obj
 0001:0002f900       _PutStrToArray             10030900 f   ustring.obj
 0001:0002f930       _PutStrToTable             10030930 f   ustring.obj
 0001:0002f950       _PutWStrToArray            10030950 f   ustring.obj
 0001:0002f990       _PutWStrToTable            10030990 f   ustring.obj
 0001:0002f9c0       _SysErrorReturn            100309c0 f   ustring.obj
 0001:0002f9f0       _check_utf16_string        100309f0 f   ustring.obj
 0001:0002fa20       _check_utf8_string         10030a20 f   ustring.obj
 0001:0002fa40       _convert_multibyte_string  10030a40 f   ustring.obj
 0001:0002fb40       _luaopen_ustring           10030b40 f   ustring.obj
 0001:0002fb90       _opt_utf16_string          10030b90 f   ustring.obj
 0001:0002fbb0       _opt_utf8_string           10030bb0 f   ustring.obj
 0001:0002fc90       _push_multibyte_string     10030c90 f   ustring.obj
 0001:0002fd40       _push_utf16_string         10030d40 f   ustring.obj
 0001:0002fd80       _push_utf8_string          10030d80 f   ustring.obj
 0001:0002fda0       _pusherror                 10030da0 f   ustring.obj
 0001:0002fdc0       _pusherrorcode             10030dc0 f   ustring.obj
 0001:0002fe30       _utf8_to_utf16             10030e30 f   ustring.obj
 0001:0002fe50       _GetAttrFromTable          10030e50 f   util.obj
 0001:0002fea0       _GetFileSizeFromTable      10030ea0 f   util.obj
 0001:0002ff40       _GetFileTimeFromTable      10030f40 f   util.obj
 0001:0002ffc0       _GetIntFromArray           10030fc0 f   util.obj
 0001:00030040       _PutFileTimeToTable        10031040 f   util.obj
 0001:00030090       _luaLF_FieldError          10031090 f   util.obj
 0001:000300d0       _luaLF_SlotError           100310d0 f   util.obj
 0001:000314c0       _luaopen_win               100324c0 f   win.obj
 0001:000317f0       _DecodePointerWrapper@4    100327f0 f   vc_crt_fix_impl.obj
 0001:00031830       _EncodePointerWrapper@4    10032830 f   vc_crt_fix_impl.obj
 0001:00031870       _GetModuleHandleExWWrapper@12 10032870 f   vc_crt_fix_impl.obj
 0001:000318b0       _InitializeSListHeadWrapper@4 100328b0 f   vc_crt_fix_impl.obj
 0001:00031900       _InterlockedFlushSListWrapper@4 10032900 f   vc_crt_fix_impl.obj
 0001:00031940       _InterlockedPopEntrySListWrapper@4 10032940 f   vc_crt_fix_impl.obj
 0001:00031980       _InterlockedPushEntrySListWrapper@8 10032980 f   vc_crt_fix_impl.obj
 0001:000319c0       _InterlockedPushListSListExWrapper@16 100329c0 f   vc_crt_fix_impl.obj
 0001:00031a00       _QueryDepthSListWrapper@4  10032a00 f   vc_crt_fix_impl.obj
 0001:00031a40       _RtlFirstEntrySListWrapper@4 10032a40 f   vc_crt_fix_impl.obj
 0001:00031a80       _lua_gettop                10032a80 f   lua51:lua51.dll
 0001:00031a86       _lua_settop                10032a86 f   lua51:lua51.dll
 0001:00031a8c       _lua_type                  10032a8c f   lua51:lua51.dll
 0001:00031a92       _lua_rawequal              10032a92 f   lua51:lua51.dll
 0001:00031a98       _lua_tonumber              10032a98 f   lua51:lua51.dll
 0001:00031a9e       _lua_tolstring             10032a9e f   lua51:lua51.dll
 0001:00031aa4       _lua_touserdata            10032aa4 f   lua51:lua51.dll
 0001:00031aaa       _lua_pushnil               10032aaa f   lua51:lua51.dll
 0001:00031ab0       _lua_pushnumber            10032ab0 f   lua51:lua51.dll
 0001:00031ab6       _lua_pushstring            10032ab6 f   lua51:lua51.dll
 0001:00031abc       _lua_pushboolean           10032abc f   lua51:lua51.dll
 0001:00031ac2       _lua_getfield              10032ac2 f   lua51:lua51.dll
 0001:00031ac8       _lua_newuserdata           10032ac8 f   lua51:lua51.dll
 0001:00031ace       _lua_getmetatable          10032ace f   lua51:lua51.dll
 0001:00031ad4       _lua_setmetatable          10032ad4 f   lua51:lua51.dll
 0001:00031ada       _luaL_register             10032ada f   lua51:lua51.dll
 0001:00031ae0       _luaL_argerror             10032ae0 f   lua51:lua51.dll
 0001:00031ae6       _luaL_checkinteger         10032ae6 f   lua51:lua51.dll
 0001:00031aec       _luaL_newmetatable         10032aec f   lua51:lua51.dll
 0001:00031af2       _lua_pushvalue             10032af2 f   lua51:lua51.dll
 0001:00031af8       _lua_remove                10032af8 f   lua51:lua51.dll
 0001:00031afe       _lua_insert                10032afe f   lua51:lua51.dll
 0001:00031b04       _lua_isnumber              10032b04 f   lua51:lua51.dll
 0001:00031b0a       _lua_isstring              10032b0a f   lua51:lua51.dll
 0001:00031b10       _lua_tointeger             10032b10 f   lua51:lua51.dll
 0001:00031b16       _lua_toboolean             10032b16 f   lua51:lua51.dll
 0001:00031b1c       _lua_objlen                10032b1c f   lua51:lua51.dll
 0001:00031b22       _lua_pushinteger           10032b22 f   lua51:lua51.dll
 0001:00031b28       _lua_pushlstring           10032b28 f   lua51:lua51.dll
 0001:00031b2e       _lua_pushcclosure          10032b2e f   lua51:lua51.dll
 0001:00031b34       _lua_pushlightuserdata     10032b34 f   lua51:lua51.dll
 0001:00031b3a       _lua_gettable              10032b3a f   lua51:lua51.dll
 0001:00031b40       _lua_rawgeti               10032b40 f   lua51:lua51.dll
 0001:00031b46       _lua_createtable           10032b46 f   lua51:lua51.dll
 0001:00031b4c       _lua_setfield              10032b4c f   lua51:lua51.dll
 0001:00031b52       _lua_rawseti               10032b52 f   lua51:lua51.dll
 0001:00031b58       _lua_call                  10032b58 f   lua51:lua51.dll
 0001:00031b5e       _lua_pcall                 10032b5e f   lua51:lua51.dll
 0001:00031b64       _lua_gc                    10032b64 f   lua51:lua51.dll
 0001:00031b6a       _luaL_ref                  10032b6a f   lua51:lua51.dll
 0001:00031b70       _luaL_unref                10032b70 f   lua51:lua51.dll
 0001:00031b76       _luaL_loadstring           10032b76 f   lua51:lua51.dll
 0001:00031b7c       _lua_pushfstring           10032b7c f   lua51:lua51.dll
 0001:00031b82       _lua_load                  10032b82 f   lua51:lua51.dll
 0001:00031b88       _lua_error                 10032b88 f   lua51:lua51.dll
 0001:00031b8e       _lua_concat                10032b8e f   lua51:lua51.dll
 0001:00031b94       _luaL_buffinit             10032b94 f   lua51:lua51.dll
 0001:00031b9a       _luaL_addlstring           10032b9a f   lua51:lua51.dll
 0001:00031ba0       _luaL_pushresult           10032ba0 f   lua51:lua51.dll
 0001:00031ba6       _lua_replace               10032ba6 f   lua51:lua51.dll
 0001:00031bac       _lua_checkstack            10032bac f   lua51:lua51.dll
 0001:00031bb2       _luaL_checklstring         10032bb2 f   lua51:lua51.dll
 0001:00031bb8       _luaL_optlstring           10032bb8 f   lua51:lua51.dll
 0001:00031bbe       _luaL_optinteger           10032bbe f   lua51:lua51.dll
 0001:00031bc4       _luaL_checkudata           10032bc4 f   lua51:lua51.dll
 0001:00031bca       _luaL_error                10032bca f   lua51:lua51.dll
 0001:00031bd0       _luaL_addvalue             10032bd0 f   lua51:lua51.dll
 0001:00031bd6       _lua_getstack              10032bd6 f   lua51:lua51.dll
 0001:00031bdc       _lua_getinfo               10032bdc f   lua51:lua51.dll
 0001:00031be2       _luaL_checktype            10032be2 f   lua51:lua51.dll
 0001:00031be8       _luaopen_base              10032be8 f   lua51:lua51.dll
 0001:00031bee       _luaopen_table             10032bee f   lua51:lua51.dll
 0001:00031bf4       _luaopen_os                10032bf4 f   lua51:lua51.dll
 0001:00031bfa       _luaopen_string            10032bfa f   lua51:lua51.dll
 0001:00031c00       _luaopen_math              10032c00 f   lua51:lua51.dll
 0001:00031c06       _luaopen_debug             10032c06 f   lua51:lua51.dll
 0001:00031c0c       _lua_rawget                10032c0c f   lua51:lua51.dll
 0001:00031c12       _lua_getfenv               10032c12 f   lua51:lua51.dll
 0001:00031c18       _lua_settable              10032c18 f   lua51:lua51.dll
 0001:00031c1e       _lua_rawset                10032c1e f   lua51:lua51.dll
 0001:00031c24       _lua_setfenv               10032c24 f   lua51:lua51.dll
 0001:00031c2a       _lua_next                  10032c2a f   lua51:lua51.dll
 0001:00031c30       _lua_getallocf             10032c30 f   lua51:lua51.dll
 0001:00031c36       _lua_setallocf             10032c36 f   lua51:lua51.dll
 0001:00031c3c       _luaL_typerror             10032c3c f   lua51:lua51.dll
 0001:00031c42       _luaL_checknumber          10032c42 f   lua51:lua51.dll
 0001:00031c48       _luaL_optnumber            10032c48 f   lua51:lua51.dll
 0001:00031c4e       _luaL_checkany             10032c4e f   lua51:lua51.dll
 0001:00031c54       _lua_typename              10032c54 f   lua51:lua51.dll
 0001:00031c5a       _lua_dump                  10032c5a f   lua51:lua51.dll
 0001:00031c60       _luaL_checkstack           10032c60 f   lua51:lua51.dll
 0001:00031c66       _luaL_prepbuffer           10032c66 f   lua51:lua51.dll
 0001:00031c6c       _lua_tocfunction           10032c6c f   lua51:lua51.dll
 0001:00031c72       _luaL_checkoption          10032c72 f   lua51:lua51.dll
 0001:00031c78       _lua_iscfunction           10032c78 f   lua51:lua51.dll
 0001:00031c7e       _luaL_gsub                 10032c7e f   lua51:lua51.dll
 0001:00031c84       _luaL_findtable            10032c84 f   lua51:lua51.dll
 0001:00031c8a       _lua_isuserdata            10032c8a f   lua51:lua51.dll
 0001:00031c90       __alldiv                   10032c90 f   LIBCMT:lldiv.obj
 0001:00031d40       __allmul                   10032d40 f   LIBCMT:llmul.obj
 0001:00031d80       __allrem                   10032d80 f   LIBCMT:llrem.obj
 0001:00031e40       __allshl                   10032e40 f   LIBCMT:llshl.obj
 0001:00031e60       __allshr                   10032e60 f   LIBCMT:llshr.obj
 0001:00031e90       __aullshr                  10032e90 f   LIBCMT:ullshr.obj
 0001:00031eb0       __ftol2_sse                10032eb0 f   LIBCMT:_ftol2_.obj
 0001:00031eb9       __ftol2_pentium4           10032eb9 f   LIBCMT:_ftol2_.obj
 0001:00031ecc       __ftol2_sse_excpt          10032ecc f   LIBCMT:_ftol2_.obj
 0001:00031ef0       __ftol2                    10032ef0 f   LIBCMT:_ftol2_.obj
 0001:00031f70       __alldvrm                  10032f70 f   LIBCMT:lldvrm.obj
 0001:00032357       __DllMainCRTStartup@12     10033357 f   LIBCMT:dll_dllmain.obj
 0001:0003237a       ___isa_available_init      1003337a f   LIBCMT:_cpu_disp_.obj
 0001:00032558       ___scrt_acquire_startup_lock 10033558 f   LIBCMT:utility.obj
 0001:0003258d       ___scrt_dllmain_after_initialize_c 1003358d f   LIBCMT:utility.obj
 0001:000325b8       ___scrt_dllmain_before_initialize_c 100335b8 f   LIBCMT:utility.obj
 0001:000325c6       ___scrt_dllmain_crt_thread_attach 100335c6 f   LIBCMT:utility.obj
 0001:000325e5       ___scrt_dllmain_crt_thread_detach 100335e5 f   LIBCMT:utility.obj
 0001:000325f2       ___scrt_dllmain_exception_filter 100335f2 f   LIBCMT:utility.obj
 0001:00032625       ___scrt_dllmain_uninitialize_c 10033625 f   LIBCMT:utility.obj
 0001:00032648       ___scrt_dllmain_uninitialize_critical 10033648 f   LIBCMT:utility.obj
 0001:00032655       ___scrt_initialize_crt     10033655 f   LIBCMT:utility.obj
 0001:0003268e       ___scrt_initialize_onexit_tables 1003368e f   LIBCMT:utility.obj
 0001:00032725       ___scrt_is_nonwritable_in_current_image 10033725 f   LIBCMT:utility.obj
 0001:000327af       ___scrt_release_startup_lock 100337af f   LIBCMT:utility.obj
 0001:000327cc       ___scrt_uninitialize_crt   100337cc f   LIBCMT:utility.obj
 0001:000327f4       __onexit                   100337f4 f   LIBCMT:utility.obj
 0001:0003282f       _atexit                    1003382f f   LIBCMT:utility.obj
 0001:00032844       ___security_init_cookie    10033844 f   LIBCMT:gs_support.obj
 0001:000328e0       ?__scrt_initialize_type_info@@YAXXZ 100338e0 f   LIBCMT:tncleanup.obj
 0001:000328ec       ?__scrt_uninitialize_type_info@@YAXXZ 100338ec f   LIBCMT:tncleanup.obj
 0001:000328f8       ___scrt_initialize_default_local_stdio_options 100338f8 f   LIBCMT:default_local_stdio_options.obj
 0001:00032915       ___scrt_get_dyn_tls_init_callback 10033915 f   LIBCMT:dyn_tls_init.obj
 0001:0003291b       ___scrt_fastfail           1003391b f   LIBCMT:utility_desktop.obj
 0001:00032a36       __crt_debugger_hook        10033a36 f   LIBCMT:utility_desktop.obj
 0001:00032a3e       __RTC_Initialize           10033a3e f   LIBCMT:_initsect_.obj
 0001:00032a69       __RTC_Terminate            10033a69 f   LIBCMT:_initsect_.obj
 0001:00032a94       @_guard_check_icall@4      10033a94 f i LIBCMT:checkcfg.obj
 0001:00032aa0       __SEH_prolog4              10033aa0 f   LIBCMT:_sehprolg4_.obj
 0001:00032ae6       __SEH_epilog4              10033ae6 f   LIBCMT:_sehprolg4_.obj
 0001:00032afb       __get_startup_argv_mode    10033afb f   LIBCMT:argv_mode.obj
 0001:00032aff       ___scrt_is_ucrt_dll_in_use 10033aff f   LIBCMT:ucrt_detection.obj
 0001:00032b0b       @__security_check_cookie@4 10033b0b f   LIBCMT:_secchk_.obj
 0001:00032b1c       ___raise_securityfailure   10033b1c f   LIBCMT:gs_report.obj
 0001:00032b44       ___report_gsfailure        10033b44 f   LIBCMT:gs_report.obj
 0001:00032c3f       _wcsrchr                   10033c3f f   libvcruntime:wcsrchr.obj
 0001:00032ce0       _memcpy                    10033ce0 f   libvcruntime:memcpy.obj
 0001:00033260       _memset                    10034260 f   libvcruntime:memset.obj
 0001:000333ba       _wcsstr                    100343ba f   libvcruntime:wcsstr.obj
 0001:00033640       _strchr                    10034640 f   libvcruntime:strchr.obj
 0001:000336ae       ___from_strstr_to_strchr   100346ae     libvcruntime:strchr.obj
 0001:0003376b       _wcschr                    1003476b f   libvcruntime:wcschr.obj
 0001:00033820       _memchr                    10034820 f   libvcruntime:memchr.obj
 0001:000338d0       _strrchr                   100348d0 f   libvcruntime:strrchr.obj
 0001:00033a50       __except_handler4          10034a50 f   libvcruntime:_chandler4_.obj
 0001:00033bb6       ___vcrt_initialize         10034bb6 f   libvcruntime:initialization.obj
 0001:00033bdf       ___vcrt_thread_attach      10034bdf f   libvcruntime:initialization.obj
 0001:00033bea       ___vcrt_thread_detach      10034bea f   libvcruntime:initialization.obj
 0001:00033bf5       ___vcrt_uninitialize       10034bf5 f   libvcruntime:initialization.obj
 0001:00033c14       ___vcrt_uninitialize_critical 10034c14 f   libvcruntime:initialization.obj
 0001:00033c1c       ___std_type_info_destroy_list 10034c1c f   libvcruntime:std_type_info.obj
 0001:00033c40       __local_unwind4            10034c40 f   libvcruntime:_exsup4_.obj
 0001:00033d16       __seh_longjmp_unwind4@4    10034d16 f   libvcruntime:_exsup4_.obj
 0001:00033d3e       @_EH4_CallFilterFunc@8     10034d3e f   libvcruntime:_exsup4_.obj
 0001:00033d55       @_EH4_TransferToHandler@8  10034d55 f   libvcruntime:_exsup4_.obj
 0001:00033d6e       @_EH4_GlobalUnwind2@8      10034d6e f   libvcruntime:_exsup4_.obj
 0001:00033d87       @_EH4_LocalUnwind@16       10034d87 f   libvcruntime:_exsup4_.obj
 0001:00033d9e       ___vcrt_freefls@4          10034d9e f   libvcruntime:per_thread_data.obj
 0001:00033dba       ___vcrt_freeptd            10034dba f   libvcruntime:per_thread_data.obj
 0001:00033df0       ___vcrt_getptd_noexit      10034df0 f   libvcruntime:per_thread_data.obj
 0001:00033e82       ___vcrt_initialize_ptd     10034e82 f   libvcruntime:per_thread_data.obj
 0001:00033eb5       ___vcrt_uninitialize_ptd   10034eb5 f   libvcruntime:per_thread_data.obj
 0001:00033ed0       ___vcrt_initialize_locks   10034ed0 f   libvcruntime:locks.obj
 0001:00033f0c       ___vcrt_uninitialize_locks 10034f0c f   libvcruntime:locks.obj
 0001:00033f3b       ??$__crt_fast_encode_pointer@PAP6AXXZ@@YAPAP6AXXZQAP6AXXZ@Z 10034f3b f i LIBCMT:utility.obj
 0001:00033f3b       ??$__crt_fast_encode_pointer@PAX@@YAPAXQAX@Z 10034f3b f i libvcruntime:winapi_downlevel.obj
 0001:00034079       ___vcrt_FlsAlloc           10035079 f   libvcruntime:winapi_downlevel.obj
 0001:000340b3       ___vcrt_FlsFree            100350b3 f   libvcruntime:winapi_downlevel.obj
 0001:000340ed       ___vcrt_FlsGetValue        100350ed f   libvcruntime:winapi_downlevel.obj
 0001:00034127       ___vcrt_FlsSetValue        10035127 f   libvcruntime:winapi_downlevel.obj
 0001:00034164       ___vcrt_InitializeCriticalSectionEx 10035164 f   libvcruntime:winapi_downlevel.obj
 0001:000341aa       ___vcrt_initialize_winapi_thunks 100351aa f   libvcruntime:winapi_downlevel.obj
 0001:000341e4       ___vcrt_uninitialize_winapi_thunks 100351e4 f   libvcruntime:winapi_downlevel.obj
 0001:00034216       ___vcrt_initialize_pure_virtual_call_handler 10035216 f   libvcruntime:purevirt_data.obj
 0001:00034240       __global_unwind2           10035240 f   libvcruntime:_exsup_.obj
 0001:000342a5       __local_unwind2            100352a5 f   libvcruntime:_exsup_.obj
 0001:00034329       __abnormal_termination     10035329 f   libvcruntime:_exsup_.obj
 0001:0003434c       __NLG_Notify1              1003534c f   libvcruntime:_exsup_.obj
 0001:00034355       __NLG_Notify               10035355 f   libvcruntime:_exsup_.obj
 0001:0003436c       __NLG_Dispatch             1003536c     libvcruntime:_exsup_.obj
 0001:0003436c       __NLG_Dispatch2            1003536c     libvcruntime:_exsup_.obj
 0001:00034374       __NLG_Call                 10035374 f   libvcruntime:_exsup_.obj
 0001:00034376       __NLG_Return2              10035376     libvcruntime:_exsup_.obj
 0001:00034377       ??$?RV<lambda_db08b09ef7aa9d4f8620ce68402612bc>@@AAV<lambda_4f2c1eaeead2a5fc776db5b62ea0fb9b>@@V<lambda_3ae262bc35d4ba6a3825c4f6bcaaf95c>@@@?$__crt_seh_guarded_call@H@@QAEH$$QAV<lambda_db08b09ef7aa9d4f8620ce68402612bc>@@AAV<lambda_4f2c1eaeead2a5fc776db5b62ea0fb9b>@@$$QAV<lambda_3ae262bc35d4ba6a3825c4f6bcaaf95c>@@@Z 10035377 f i libucrt:output.obj
 0001:000343c8       ??$__acrt_lock_stream_and_call@V<lambda_4f2c1eaeead2a5fc776db5b62ea0fb9b>@@@@YAHQAU_iobuf@@$$QAV<lambda_4f2c1eaeead2a5fc776db5b62ea0fb9b>@@@Z 100353c8 f i libucrt:output.obj
 0001:000346f1       ??$count@D@formatting_buffer@__crt_stdio_output@@QBEIXZ 100356f1 f i libucrt:output.obj
 0001:00034709       ??$ensure_buffer_is_big_enough@D@formatting_buffer@__crt_stdio_output@@QAE_NI@Z 10035709 f i libucrt:output.obj
 0001:0003478f       ??$is_wide_character_specifier@D@__crt_stdio_output@@YA_N_KDW4length_modifier@0@@Z 1003578f f i libucrt:output.obj
 0001:000347cf       ??$is_wide_character_specifier@_W@__crt_stdio_output@@YA_N_K_WW4length_modifier@0@@Z 100357cf f i libucrt:output.obj
 0001:0003481e       ??$scratch_data@D@formatting_buffer@__crt_stdio_output@@QAEPADXZ 1003581e f i libucrt:output.obj
 0001:0003483c       ??$type_case_integer_parse_into_buffer@I@?$output_processor@DV?$stream_output_adapter@D@__crt_stdio_output@@V?$standard_base@DV?$stream_output_adapter@D@__crt_stdio_output@@@2@@__crt_stdio_output@@AAEXII_N@Z 1003583c f i libucrt:output.obj
 0001:0003483c       ??$type_case_integer_parse_into_buffer@I@?$output_processor@_WV?$string_output_adapter@_W@__crt_stdio_output@@V?$standard_base@_WV?$string_output_adapter@_W@__crt_stdio_output@@@2@@__crt_stdio_output@@AAEXII_N@Z 1003583c f i libucrt:output.obj
 0001:0003483c       ??$type_case_integer_parse_into_buffer@I@?$output_processor@DV?$string_output_adapter@D@__crt_stdio_output@@V?$standard_base@DV?$string_output_adapter@D@__crt_stdio_output@@@2@@__crt_stdio_output@@AAEXII_N@Z 1003583c f i libucrt:output.obj
 0001:000348b1       ??$type_case_integer_parse_into_buffer@_K@?$output_processor@DV?$stream_output_adapter@D@__crt_stdio_output@@V?$standard_base@DV?$stream_output_adapter@D@__crt_stdio_output@@@2@@__crt_stdio_output@@AAEX_KI_N@Z 100358b1 f i libucrt:output.obj
 0001:000348b1       ??$type_case_integer_parse_into_buffer@_K@?$output_processor@_WV?$string_output_adapter@_W@__crt_stdio_output@@V?$standard_base@_WV?$string_output_adapter@_W@__crt_stdio_output@@@2@@__crt_stdio_output@@AAEX_KI_N@Z 100358b1 f i libucrt:output.obj
 0001:000348b1       ??$type_case_integer_parse_into_buffer@_K@?$output_processor@DV?$string_output_adapter@D@__crt_stdio_output@@V?$standard_base@DV?$string_output_adapter@D@__crt_stdio_output@@@2@@__crt_stdio_output@@AAEX_KI_N@Z 100358b1 f i libucrt:output.obj
 0001:00034939       ??$write_multiple_characters@V?$stream_output_adapter@D@__crt_stdio_output@@D@__crt_stdio_output@@YAXABV?$stream_output_adapter@D@0@DHQAH@Z 10035939 f i libucrt:output.obj
 0001:00034965       ??$write_multiple_characters@V?$string_output_adapter@D@__crt_stdio_output@@D@__crt_stdio_output@@YAXABV?$string_output_adapter@D@0@DHQAH@Z 10035965 f i libucrt:output.obj
 0001:00034991       ??$write_multiple_characters@V?$string_output_adapter@_W@__crt_stdio_output@@D@__crt_stdio_output@@YAXABV?$string_output_adapter@_W@0@DHQAH@Z 10035991 f i libucrt:output.obj
 0001:000349c2       ??0?$common_data@D@__crt_stdio_output@@IAE@XZ 100359c2 f i libucrt:output.obj
 0001:00034a09       ??0?$common_data@_W@__crt_stdio_output@@IAE@XZ 10035a09 f i libucrt:output.obj
 0001:00034a55       ??0?$output_adapter_data@DV?$string_output_adapter@D@__crt_stdio_output@@@__crt_stdio_output@@IAE@ABV?$string_output_adapter@D@1@_KQBDQAU__crt_locale_pointers@@QAD@Z 10035a55 f i libucrt:output.obj
 0001:00034a55       ??0?$output_adapter_data@DV?$stream_output_adapter@D@__crt_stdio_output@@@__crt_stdio_output@@IAE@ABV?$stream_output_adapter@D@1@_KQBDQAU__crt_locale_pointers@@QAD@Z 10035a55 f i libucrt:output.obj
 0001:00034a91       ??0?$output_adapter_data@_WV?$string_output_adapter@_W@__crt_stdio_output@@@__crt_stdio_output@@IAE@ABV?$string_output_adapter@_W@1@_KQB_WQAU__crt_locale_pointers@@QAD@Z 10035a91 f i libucrt:output.obj
 0001:00034acd       ??0?$output_processor@DV?$stream_output_adapter@D@__crt_stdio_output@@V?$standard_base@DV?$stream_output_adapter@D@__crt_stdio_output@@@2@@__crt_stdio_output@@QAE@ABV?$stream_output_adapter@D@1@_KQBDQAU__crt_locale_pointers@@QAD@Z 10035acd f i libucrt:output.obj
 0001:00034acd       ??0?$output_processor@DV?$string_output_adapter@D@__crt_stdio_output@@V?$standard_base@DV?$string_output_adapter@D@__crt_stdio_output@@@2@@__crt_stdio_output@@QAE@ABV?$string_output_adapter@D@1@_KQBDQAU__crt_locale_pointers@@QAD@Z 10035acd f i libucrt:output.obj
 0001:00034b02       ??0?$output_processor@_WV?$string_output_adapter@_W@__crt_stdio_output@@V?$standard_base@_WV?$string_output_adapter@_W@__crt_stdio_output@@@2@@__crt_stdio_output@@QAE@ABV?$string_output_adapter@_W@1@_KQB_WQAU__crt_locale_pointers@@QAD@Z 10035b02 f i libucrt:output.obj
 0001:00034b37       ??0_LocaleUpdate@@QAE@QAU__crt_locale_pointers@@@Z 10035b37 f i libucrt:output.obj
 0001:00034bba       ??1formatting_buffer@__crt_stdio_output@@QAE@XZ 10035bba f i libucrt:output.obj
 0001:00034bd4       ??4?$__crt_unique_heap_ptr@DU__crt_internal_free_policy@@@@QAEAAV0@$$QAV0@@Z 10035bd4 f i libucrt:output.obj
 0001:00034cb5       ?crop_zeroes@__crt_stdio_output@@YAXPADQAU__crt_locale_pointers@@@Z 10035cb5 f i libucrt:output.obj
 0001:00034d0c       ?find_next_state@?$output_processor@DV?$string_output_adapter@D@__crt_stdio_output@@V?$standard_base@DV?$string_output_adapter@D@__crt_stdio_output@@@2@@__crt_stdio_output@@ABE?AW4state@2@DW432@@Z 10035d0c f i libucrt:output.obj
 0001:00034d0c       ?find_next_state@?$output_processor@DV?$stream_output_adapter@D@__crt_stdio_output@@V?$standard_base@DV?$stream_output_adapter@D@__crt_stdio_output@@@2@@__crt_stdio_output@@ABE?AW4state@2@DW432@@Z 10035d0c f i libucrt:output.obj
 0001:00034d3e       ?find_next_state@?$output_processor@_WV?$string_output_adapter@_W@__crt_stdio_output@@V?$standard_base@_WV?$string_output_adapter@_W@__crt_stdio_output@@@2@@__crt_stdio_output@@ABE?AW4state@2@_WW432@@Z 10035d3e f i libucrt:output.obj
 0001:00034d72       ?force_decimal_point@__crt_stdio_output@@YAXPADQAU__crt_locale_pointers@@@Z 10035d72 f i libucrt:output.obj
 0001:00034dce       ?parse_int_from_format_string@?$output_processor@DV?$string_output_adapter@D@__crt_stdio_output@@V?$standard_base@DV?$string_output_adapter@D@__crt_stdio_output@@@2@@__crt_stdio_output@@AAE_NQAH@Z 10035dce f i libucrt:output.obj
 0001:00034dce       ?parse_int_from_format_string@?$output_processor@DV?$stream_output_adapter@D@__crt_stdio_output@@V?$standard_base@DV?$stream_output_adapter@D@__crt_stdio_output@@@2@@__crt_stdio_output@@AAE_NQAH@Z 10035dce f i libucrt:output.obj
 0001:00034e2a       ?parse_int_from_format_string@?$output_processor@_WV?$string_output_adapter@_W@__crt_stdio_output@@V?$standard_base@_WV?$string_output_adapter@_W@__crt_stdio_output@@@2@@__crt_stdio_output@@AAE_NQAH@Z 10035e2a f i libucrt:output.obj
 0001:00034e88       ?process@?$output_processor@DV?$stream_output_adapter@D@__crt_stdio_output@@V?$standard_base@DV?$stream_output_adapter@D@__crt_stdio_output@@@2@@__crt_stdio_output@@QAEHXZ 10035e88 f i libucrt:output.obj
 0001:00034fa4       ?process@?$output_processor@DV?$string_output_adapter@D@__crt_stdio_output@@V?$standard_base@DV?$string_output_adapter@D@__crt_stdio_output@@@2@@__crt_stdio_output@@QAEHXZ 10035fa4 f i libucrt:output.obj
 0001:000350c0       ?process@?$output_processor@_WV?$string_output_adapter@_W@__crt_stdio_output@@V?$standard_base@_WV?$string_output_adapter@_W@__crt_stdio_output@@@2@@__crt_stdio_output@@QAEHXZ 100360c0 f i libucrt:output.obj
 0001:000351e0       ?state_case_flag@?$output_processor@DV?$stream_output_adapter@D@__crt_stdio_output@@V?$standard_base@DV?$stream_output_adapter@D@__crt_stdio_output@@@2@@__crt_stdio_output@@AAE_NXZ 100361e0 f i libucrt:output.obj
 0001:000351e0       ?state_case_flag@?$output_processor@DV?$string_output_adapter@D@__crt_stdio_output@@V?$standard_base@DV?$string_output_adapter@D@__crt_stdio_output@@@2@@__crt_stdio_output@@AAE_NXZ 100361e0 f i libucrt:output.obj
 0001:0003521d       ?state_case_flag@?$output_processor@_WV?$string_output_adapter@_W@__crt_stdio_output@@V?$standard_base@_WV?$string_output_adapter@_W@__crt_stdio_output@@@2@@__crt_stdio_output@@AAE_NXZ 1003621d f i libucrt:output.obj
 0001:0003525a       ?state_case_normal@?$output_processor@DV?$stream_output_adapter@D@__crt_stdio_output@@V?$standard_base@DV?$stream_output_adapter@D@__crt_stdio_output@@@2@@__crt_stdio_output@@AAE_NXZ 1003625a f i libucrt:output.obj
 0001:00035279       ?state_case_normal@?$output_processor@DV?$string_output_adapter@D@__crt_stdio_output@@V?$standard_base@DV?$string_output_adapter@D@__crt_stdio_output@@@2@@__crt_stdio_output@@AAE_NXZ 10036279 f i libucrt:output.obj
 0001:00035298       ?state_case_normal@?$output_processor@_WV?$string_output_adapter@_W@__crt_stdio_output@@V?$standard_base@_WV?$string_output_adapter@_W@__crt_stdio_output@@@2@@__crt_stdio_output@@AAE_NXZ 10036298 f i libucrt:output.obj
 0001:000352b7       ?state_case_normal_common@?$output_processor@DV?$stream_output_adapter@D@__crt_stdio_output@@V?$standard_base@DV?$stream_output_adapter@D@__crt_stdio_output@@@2@@__crt_stdio_output@@AAE_NXZ 100362b7 f i libucrt:output.obj
 0001:000352e1       ?state_case_normal_common@?$output_processor@DV?$string_output_adapter@D@__crt_stdio_output@@V?$standard_base@DV?$string_output_adapter@D@__crt_stdio_output@@@2@@__crt_stdio_output@@AAE_NXZ 100362e1 f i libucrt:output.obj
 0001:0003530b       ?state_case_normal_common@?$output_processor@_WV?$string_output_adapter@_W@__crt_stdio_output@@V?$standard_base@_WV?$string_output_adapter@_W@__crt_stdio_output@@@2@@__crt_stdio_output@@AAE_NXZ 1003630b f i libucrt:output.obj
 0001:00035326       ?state_case_normal_tchar@?$output_processor@DV?$stream_output_adapter@D@__crt_stdio_output@@V?$standard_base@DV?$stream_output_adapter@D@__crt_stdio_output@@@2@@__crt_stdio_output@@AAE_ND@Z 10036326 f i libucrt:output.obj
 0001:00035387       ?state_case_normal_tchar@?$output_processor@DV?$string_output_adapter@D@__crt_stdio_output@@V?$standard_base@DV?$string_output_adapter@D@__crt_stdio_output@@@2@@__crt_stdio_output@@AAE_ND@Z 10036387 f i libucrt:output.obj
 0001:000353e8       ?state_case_precision@?$output_processor@DV?$string_output_adapter@D@__crt_stdio_output@@V?$standard_base@DV?$string_output_adapter@D@__crt_stdio_output@@@2@@__crt_stdio_output@@AAE_NXZ 100363e8 f i libucrt:output.obj
 0001:000353e8       ?state_case_precision@?$output_processor@DV?$stream_output_adapter@D@__crt_stdio_output@@V?$standard_base@DV?$stream_output_adapter@D@__crt_stdio_output@@@2@@__crt_stdio_output@@AAE_NXZ 100363e8 f i libucrt:output.obj
 0001:00035410       ?state_case_precision@?$output_processor@_WV?$string_output_adapter@_W@__crt_stdio_output@@V?$standard_base@_WV?$string_output_adapter@_W@__crt_stdio_output@@@2@@__crt_stdio_output@@AAE_NXZ 10036410 f i libucrt:output.obj
 0001:00035439       ?state_case_size@?$output_processor@DV?$stream_output_adapter@D@__crt_stdio_output@@V?$standard_base@DV?$stream_output_adapter@D@__crt_stdio_output@@@2@@__crt_stdio_output@@AAE_NXZ 10036439 f i libucrt:output.obj
 0001:000355a2       ?state_case_size@?$output_processor@DV?$string_output_adapter@D@__crt_stdio_output@@V?$standard_base@DV?$string_output_adapter@D@__crt_stdio_output@@@2@@__crt_stdio_output@@AAE_NXZ 100365a2 f i libucrt:output.obj
 0001:0003570b       ?state_case_size@?$output_processor@_WV?$string_output_adapter@_W@__crt_stdio_output@@V?$standard_base@_WV?$string_output_adapter@_W@__crt_stdio_output@@@2@@__crt_stdio_output@@AAE_NXZ 1003670b f i libucrt:output.obj
 0001:00035887       ?state_case_type@?$output_processor@DV?$stream_output_adapter@D@__crt_stdio_output@@V?$standard_base@DV?$stream_output_adapter@D@__crt_stdio_output@@@2@@__crt_stdio_output@@AAE_NXZ 10036887 f i libucrt:output.obj
 0001:00035ab6       ?state_case_type@?$output_processor@DV?$string_output_adapter@D@__crt_stdio_output@@V?$standard_base@DV?$string_output_adapter@D@__crt_stdio_output@@@2@@__crt_stdio_output@@AAE_NXZ 10036ab6 f i libucrt:output.obj
 0001:00035ce5       ?state_case_type@?$output_processor@_WV?$string_output_adapter@_W@__crt_stdio_output@@V?$standard_base@_WV?$string_output_adapter@_W@__crt_stdio_output@@@2@@__crt_stdio_output@@AAE_NXZ 10036ce5 f i libucrt:output.obj
 0001:00035f42       ?state_case_width@?$output_processor@DV?$string_output_adapter@D@__crt_stdio_output@@V?$standard_base@DV?$string_output_adapter@D@__crt_stdio_output@@@2@@__crt_stdio_output@@AAE_NXZ 10036f42 f i libucrt:output.obj
 0001:00035f42       ?state_case_width@?$output_processor@DV?$stream_output_adapter@D@__crt_stdio_output@@V?$standard_base@DV?$stream_output_adapter@D@__crt_stdio_output@@@2@@__crt_stdio_output@@AAE_NXZ 10036f42 f i libucrt:output.obj
 0001:00035f6d       ?state_case_width@?$output_processor@_WV?$string_output_adapter@_W@__crt_stdio_output@@V?$standard_base@_WV?$string_output_adapter@_W@__crt_stdio_output@@@2@@__crt_stdio_output@@AAE_NXZ 10036f6d f i libucrt:output.obj
 0001:00035f99       ?to_integer_size@__crt_stdio_output@@YAIW4length_modifier@1@@Z 10036f99 f i libucrt:output.obj
 0001:00035ff5       ?type_case_Z@?$output_processor@DV?$string_output_adapter@D@__crt_stdio_output@@V?$standard_base@DV?$string_output_adapter@D@__crt_stdio_output@@@2@@__crt_stdio_output@@AAE_NXZ 10036ff5 f i libucrt:output.obj
 0001:00035ff5       ?type_case_Z@?$output_processor@DV?$stream_output_adapter@D@__crt_stdio_output@@V?$standard_base@DV?$stream_output_adapter@D@__crt_stdio_output@@@2@@__crt_stdio_output@@AAE_NXZ 10036ff5 f i libucrt:output.obj
 0001:00036058       ?type_case_Z@?$output_processor@_WV?$string_output_adapter@_W@__crt_stdio_output@@V?$standard_base@_WV?$string_output_adapter@_W@__crt_stdio_output@@@2@@__crt_stdio_output@@AAE_NXZ 10037058 f i libucrt:output.obj
 0001:000360bb       ?type_case_a@?$output_processor@DV?$string_output_adapter@D@__crt_stdio_output@@V?$standard_base@DV?$string_output_adapter@D@__crt_stdio_output@@@2@@__crt_stdio_output@@AAE_NXZ 100370bb f i libucrt:output.obj
 0001:000360bb       ?type_case_a@?$output_processor@DV?$stream_output_adapter@D@__crt_stdio_output@@V?$standard_base@DV?$stream_output_adapter@D@__crt_stdio_output@@@2@@__crt_stdio_output@@AAE_NXZ 100370bb f i libucrt:output.obj
 0001:00036215       ?type_case_a@?$output_processor@_WV?$string_output_adapter@_W@__crt_stdio_output@@V?$standard_base@_WV?$string_output_adapter@_W@__crt_stdio_output@@@2@@__crt_stdio_output@@AAE_NXZ 10037215 f i libucrt:output.obj
 0001:00036387       ?type_case_c_tchar@?$output_processor@DV?$stream_output_adapter@D@__crt_stdio_output@@V?$standard_base@DV?$stream_output_adapter@D@__crt_stdio_output@@@2@@__crt_stdio_output@@AAE_ND@Z 10037387 f i libucrt:output.obj
 0001:00036387       ?type_case_c_tchar@?$output_processor@DV?$string_output_adapter@D@__crt_stdio_output@@V?$standard_base@DV?$string_output_adapter@D@__crt_stdio_output@@@2@@__crt_stdio_output@@AAE_ND@Z 10037387 f i libucrt:output.obj
 0001:00036417       ?type_case_c_tchar@?$output_processor@_WV?$string_output_adapter@_W@__crt_stdio_output@@V?$standard_base@_WV?$string_output_adapter@_W@__crt_stdio_output@@@2@@__crt_stdio_output@@AAE_N_W@Z 10037417 f i libucrt:output.obj
 0001:000364af       ?type_case_integer@?$output_processor@DV?$stream_output_adapter@D@__crt_stdio_output@@V?$standard_base@DV?$stream_output_adapter@D@__crt_stdio_output@@@2@@__crt_stdio_output@@AAE_NI_N@Z 100374af f i libucrt:output.obj
 0001:000364af       ?type_case_integer@?$output_processor@DV?$string_output_adapter@D@__crt_stdio_output@@V?$standard_base@DV?$string_output_adapter@D@__crt_stdio_output@@@2@@__crt_stdio_output@@AAE_NI_N@Z 100374af f i libucrt:output.obj
 0001:000364af       ?type_case_integer@?$output_processor@_WV?$string_output_adapter@_W@__crt_stdio_output@@V?$standard_base@_WV?$string_output_adapter@_W@__crt_stdio_output@@@2@@__crt_stdio_output@@AAE_NI_N@Z 100374af f i libucrt:output.obj
 0001:000365f9       ?type_case_n@?$output_processor@DV?$stream_output_adapter@D@__crt_stdio_output@@V?$standard_base@DV?$stream_output_adapter@D@__crt_stdio_output@@@2@@__crt_stdio_output@@AAE_NXZ 100375f9 f i libucrt:output.obj
 0001:000365f9       ?type_case_n@?$output_processor@_WV?$string_output_adapter@_W@__crt_stdio_output@@V?$standard_base@_WV?$string_output_adapter@_W@__crt_stdio_output@@@2@@__crt_stdio_output@@AAE_NXZ 100375f9 f i libucrt:output.obj
 0001:000365f9       ?type_case_n@?$output_processor@DV?$string_output_adapter@D@__crt_stdio_output@@V?$standard_base@DV?$string_output_adapter@D@__crt_stdio_output@@@2@@__crt_stdio_output@@AAE_NXZ 100375f9 f i libucrt:output.obj
 0001:0003666d       ?type_case_o@?$output_processor@DV?$string_output_adapter@D@__crt_stdio_output@@V?$standard_base@DV?$string_output_adapter@D@__crt_stdio_output@@@2@@__crt_stdio_output@@AAE_NXZ 1003766d f i libucrt:output.obj
 0001:0003666d       ?type_case_o@?$output_processor@_WV?$string_output_adapter@_W@__crt_stdio_output@@V?$standard_base@_WV?$string_output_adapter@_W@__crt_stdio_output@@@2@@__crt_stdio_output@@AAE_NXZ 1003766d f i libucrt:output.obj
 0001:0003666d       ?type_case_o@?$output_processor@DV?$stream_output_adapter@D@__crt_stdio_output@@V?$standard_base@DV?$stream_output_adapter@D@__crt_stdio_output@@@2@@__crt_stdio_output@@AAE_NXZ 1003766d f i libucrt:output.obj
 0001:0003668c       ?type_case_p@?$output_processor@DV?$stream_output_adapter@D@__crt_stdio_output@@V?$standard_base@DV?$stream_output_adapter@D@__crt_stdio_output@@@2@@__crt_stdio_output@@AAE_NXZ 1003768c f i libucrt:output.obj
 0001:0003668c       ?type_case_p@?$output_processor@DV?$string_output_adapter@D@__crt_stdio_output@@V?$standard_base@DV?$string_output_adapter@D@__crt_stdio_output@@@2@@__crt_stdio_output@@AAE_NXZ 1003768c f i libucrt:output.obj
 0001:0003668c       ?type_case_p@?$output_processor@_WV?$string_output_adapter@_W@__crt_stdio_output@@V?$standard_base@_WV?$string_output_adapter@_W@__crt_stdio_output@@@2@@__crt_stdio_output@@AAE_NXZ 1003768c f i libucrt:output.obj
 0001:000366a4       ?type_case_s@?$output_processor@DV?$string_output_adapter@D@__crt_stdio_output@@V?$standard_base@DV?$string_output_adapter@D@__crt_stdio_output@@@2@@__crt_stdio_output@@AAE_NXZ 100376a4 f i libucrt:output.obj
 0001:000366a4       ?type_case_s@?$output_processor@DV?$stream_output_adapter@D@__crt_stdio_output@@V?$standard_base@DV?$stream_output_adapter@D@__crt_stdio_output@@@2@@__crt_stdio_output@@AAE_NXZ 100376a4 f i libucrt:output.obj
 0001:00036717       ?type_case_s@?$output_processor@_WV?$string_output_adapter@_W@__crt_stdio_output@@V?$standard_base@_WV?$string_output_adapter@_W@__crt_stdio_output@@@2@@__crt_stdio_output@@AAE_NXZ 10037717 f i libucrt:output.obj
 0001:0003678b       ?type_case_s_compute_narrow_string_length@?$output_processor@_WV?$string_output_adapter@_W@__crt_stdio_output@@V?$standard_base@_WV?$string_output_adapter@_W@__crt_stdio_output@@@2@@__crt_stdio_output@@ABEHH_W@Z 1003778b f i libucrt:output.obj
 0001:000367cb       ?validate_stream_is_ansi_if_required@?$__acrt_stdio_char_traits@D@@SA_NQAU_iobuf@@@Z 100377cb f i libucrt:output.obj
 0001:0003684d       ?write_character@?$stream_output_adapter@D@__crt_stdio_output@@QBEXDQAH@Z 1003784d f i libucrt:output.obj
 0001:0003688a       ?write_character@?$string_output_adapter@D@__crt_stdio_output@@QBE_NDQAH@Z 1003788a f i libucrt:output.obj
 0001:000368cc       ?write_character@?$string_output_adapter@_W@__crt_stdio_output@@QBE_N_WQAH@Z 100378cc f i libucrt:output.obj
 0001:00036911       ?write_stored_string_tchar@?$output_processor@DV?$stream_output_adapter@D@__crt_stdio_output@@V?$standard_base@DV?$stream_output_adapter@D@__crt_stdio_output@@@2@@__crt_stdio_output@@AAE_ND@Z 10037911 f i libucrt:output.obj
 0001:000369b8       ?write_stored_string_tchar@?$output_processor@DV?$string_output_adapter@D@__crt_stdio_output@@V?$standard_base@DV?$string_output_adapter@D@__crt_stdio_output@@@2@@__crt_stdio_output@@AAE_ND@Z 100379b8 f i libucrt:output.obj
 0001:00036a5f       ?write_stored_string_tchar@?$output_processor@_WV?$string_output_adapter@_W@__crt_stdio_output@@V?$standard_base@_WV?$string_output_adapter@_W@__crt_stdio_output@@@2@@__crt_stdio_output@@AAE_N_W@Z 10037a5f f i libucrt:output.obj
 0001:00036aea       ?write_string@?$stream_output_adapter@D@__crt_stdio_output@@QBEXQBDHQAH1@Z 10037aea f i libucrt:output.obj
 0001:00036b74       ?write_string@?$string_output_adapter@D@__crt_stdio_output@@QBEXQBDHQAH1@Z 10037b74 f i libucrt:output.obj
 0001:00036c07       ?write_string@?$string_output_adapter@_W@__crt_stdio_output@@QBEXQB_WHQAH1@Z 10037c07 f i libucrt:output.obj
 0001:00036ca1       ___stdio_common_vfprintf   10037ca1 f   libucrt:output.obj
 0001:00036d18       ___stdio_common_vsprintf   10037d18 f   libucrt:output.obj
 0001:00036d3c       ___stdio_common_vswprintf  10037d3c f   libucrt:output.obj
 0001:00036d60       _wcsdup                    10037d60 f   libucrt:wcsdup.obj
 0001:00036d60       __wcsdup                   10037d60 f   libucrt:wcsdup.obj
 0001:00036dc1       _free                      10037dc1 f   libucrt:free.obj
 0001:00036dc6       _malloc                    10037dc6 f   libucrt:malloc.obj
 0001:00036e92       __wfopen                   10037e92 f   libucrt:fopen.obj
 0001:00036ea9       __fclose_nolock            10037ea9 f   libucrt:fclose.obj
 0001:00036f1f       _fclose                    10037f1f f   libucrt:fclose.obj
 0001:0003704a       __clearfp                  1003804a f   libucrt:ieee87.obj
 0001:00037128       __control87                10038128 f   libucrt:ieee87.obj
 0001:000374c3       ___acrt_errno_from_os_error 100384c3 f   libucrt:errno.obj
 0001:00037506       ___acrt_errno_map_os_error 10038506 f   libucrt:errno.obj
 0001:00037529       ___doserrno                10038529 f   libucrt:errno.obj
 0001:0003753c       __errno                    1003853c f   libucrt:errno.obj
 0001:000375cb       __get_sys_err_msg          100385cb f i libucrt:strerror.obj
 0001:000375ef       _strerror                  100385ef f   libucrt:strerror.obj
 0001:000375fa       ___acrt_initialize_stdio   100385fa f   libucrt:_file.obj
 0001:000376c2       ___acrt_iob_func           100386c2 f   libucrt:_file.obj
 0001:000376d2       ___acrt_uninitialize_stdio 100386d2 f   libucrt:_file.obj
 0001:0003771e       __lock_file                1003871e f   libucrt:_file.obj
 0001:00037732       __unlock_file              10038732 f   libucrt:_file.obj
 0001:00037859       __wfreopen                 10038859 f   libucrt:freopen.obj
 0001:00037881       _feof                      10038881 f   libucrt:feoferr.obj
 0001:000378ac       _ferror                    100388ac f   libucrt:feoferr.obj
 0001:000378d7       __fread_nolock_s           100388d7 f   libucrt:fread.obj
 0001:00037aa3       _fread                     10038aa3 f   libucrt:fread.obj
 0001:00037ac0       _fread_s                   10038ac0 f   libucrt:fread.obj
 0001:00037bd4       __fgetc_nolock             10038bd4 f   libucrt:fgetc.obj
 0001:00037c10       __getc_nolock              10038c10 f   libucrt:fgetc.obj
 0001:00037c1b       _fgetc                     10038c1b f   libucrt:fgetc.obj
 0001:00037d1d       _getc                      10038d1d f   libucrt:fgetc.obj
 0001:00037d28       _rewind                    10038d28 f   libucrt:rewind.obj
 0001:00037df6       __ungetc_nolock            10038df6 f   libucrt:ungetc.obj
 0001:00037ee5       _ungetc                    10038ee5 f   libucrt:ungetc.obj
 0001:00037f55       _iswctype                  10038f55 f   libucrt:iswctype.obj
 0001:00037fb4       __chvalidchk_l             10038fb4 f i libucrt:_ctype.obj
 0001:00037fde       __ischartype_l             10038fde f i libucrt:_ctype.obj
 0001:00038011       __isdigit_l                10039011 f i libucrt:_ctype.obj
 0001:00038049       __isspace_l                10039049 f i libucrt:_ctype.obj
 0001:00038081       _isdigit                   10039081 f i libucrt:_ctype.obj
 0001:000380ae       _isspace                   100390ae f i libucrt:_ctype.obj
 0001:000380db       _wcsncpy                   100390db f   libucrt:wcsncpy.obj
 0001:0003811e       __wcsicmp                  1003911e f   libucrt:wcsicmp.obj
 0001:000381b3       __wcsicmp_l                100391b3 f   libucrt:wcsicmp.obj
 0001:000382a0       _strncmp                   100392a0 f   libucrt:strncmp.obj
 0001:00038320       _strncpy                   10039320 f   libucrt:strncpy.obj
 0001:00038450       _strpbrk                   10039450 f   libucrt:strpbrk.obj
 0001:00038a0c       ?__crt_stdio_path_requires_backslash@@YA_NQB_W@Z 10039a0c f i libucrt:popen.obj
 0001:00038ab9       __pclose                   10039ab9 f   libucrt:popen.obj
 0001:00038b8d       __wpopen                   10039b8d f   libucrt:popen.obj
 0001:00038b98       _clearerr                  10039b98 f   libucrt:clearerr.obj
 0001:00038b9d       _clearerr_s                10039b9d f   libucrt:clearerr.obj
 0001:00038c48       ___acrt_stdio_flush_nolock 10039c48 f   libucrt:fflush.obj
 0001:00038cae       __fflush_nolock            10039cae f   libucrt:fflush.obj
 0001:00038cf5       __flushall                 10039cf5 f   libucrt:fflush.obj
 0001:00038dd6       _fflush                    10039dd6 f   libucrt:fflush.obj
 0001:00038ef4       _fgets                     10039ef4 f   libucrt:fgets.obj
 0001:00038eff       ?LongLongSub@@YAJ_J0PA_J@Z 10039eff f i libucrt:fseek.obj
 0001:000391b9       _fseek                     1003a1b9 f   libucrt:fseek.obj
 0001:00039720       __ftelli64_nolock          1003a720 f   libucrt:ftell.obj
 0001:0003972b       _ftell                     1003a72b f   libucrt:ftell.obj
 0001:00039736       ??$?RV<lambda_11b4f7b0d3157825a5656a18eba1ae27>@@AAV<lambda_b51c0495177f500e782686251704ae76>@@V<lambda_cf89b47920b5017557bfe891e78aca36>@@@?$__crt_seh_guarded_call@I@@QAEI$$QAV<lambda_11b4f7b0d3157825a5656a18eba1ae27>@@AAV<lambda_b51c0495177f500e782686251704ae76>@@$$QAV<lambda_cf89b47920b5017557bfe891e78aca36>@@@Z 1003a736 f i libucrt:fwrite.obj
 0001:00039787       ??$__acrt_lock_stream_and_call@V<lambda_b51c0495177f500e782686251704ae76>@@@@YAIQAU_iobuf@@$$QAV<lambda_b51c0495177f500e782686251704ae76>@@@Z 1003a787 f i libucrt:fwrite.obj
 0001:000397f5       __fwrite_nolock            1003a7f5 f   libucrt:fwrite.obj
 0001:0003996e       _fwrite                    1003a96e f   libucrt:fwrite.obj
 0001:000399c6       ??$?RV<lambda_d92cfe8357b99225085016881b624cb0>@@AAV<lambda_b721fa326cdb32351d23dfa67958c160>@@V<lambda_42d75b0848218ec137fa420c8ba9fdf9>@@@?$__crt_seh_guarded_call@H@@QAEH$$QAV<lambda_d92cfe8357b99225085016881b624cb0>@@AAV<lambda_b721fa326cdb32351d23dfa67958c160>@@$$QAV<lambda_42d75b0848218ec137fa420c8ba9fdf9>@@@Z 1003a9c6 f i libucrt:setvbuf.obj
 0001:00039a17       ??$__acrt_lock_stream_and_call@V<lambda_b721fa326cdb32351d23dfa67958c160>@@@@YAHQAU_iobuf@@$$QAV<lambda_b721fa326cdb32351d23dfa67958c160>@@@Z 1003aa17 f i libucrt:setvbuf.obj
 0001:00039b0c       _setvbuf                   1003ab0c f   libucrt:setvbuf.obj
 0001:00039e9a       ___acrt_stdio_free_tmpfile_name_buffers_nolock 1003ae9a f   libucrt:tmpfile.obj
 0001:00039ed8       _tmpfile                   1003aed8 f   libucrt:tmpfile.obj
 0001:00039ef6       ??$?RV<lambda_948e0c831b1eafdf53315a00da3ad7eb>@@AAV<lambda_d82aded7e80d0a2836af81596bef263e>@@V<lambda_9cb36f98846f17dfe48cc7d4c6a6fede>@@@?$__crt_seh_guarded_call@H@@QAEH$$QAV<lambda_948e0c831b1eafdf53315a00da3ad7eb>@@AAV<lambda_d82aded7e80d0a2836af81596bef263e>@@$$QAV<lambda_9cb36f98846f17dfe48cc7d4c6a6fede>@@@Z 1003aef6 f i libucrt:input.obj
 0001:00039f47       ??$__acrt_lock_stream_and_call@V<lambda_d82aded7e80d0a2836af81596bef263e>@@@@YAHQAU_iobuf@@$$QAV<lambda_d82aded7e80d0a2836af81596bef263e>@@@Z 1003af47 f i libucrt:input.obj
 0001:00039f6f       ??$assemble_floating_point_ind@N@__crt_strtox@@YAXAAN@Z 1003af6f f i libucrt:input.obj
 0001:00039f9e       ??$assemble_floating_point_infinity@N@__crt_strtox@@YAX_NAAN@Z 1003af9e f i libucrt:input.obj
 0001:00039fdd       ??$assemble_floating_point_qnan@N@__crt_strtox@@YAX_NAAN@Z 1003afdd f i libucrt:input.obj
 0001:0003a01c       ??$assemble_floating_point_snan@N@__crt_strtox@@YAX_NAAN@Z 1003b01c f i libucrt:input.obj
 0001:0003a060       ??$assemble_floating_point_value_t@M@__crt_strtox@@YA?AW4SLD_STATUS@@_NH_KAAM@Z 1003b060 f i libucrt:input.obj
 0001:0003a090       ??$assemble_floating_point_value_t@N@__crt_strtox@@YA?AW4SLD_STATUS@@_NH_KAAN@Z 1003b090 f i libucrt:input.obj
 0001:0003a0ef       ??$assemble_floating_point_zero@N@__crt_strtox@@YAX_NAAN@Z 1003b0ef f i libucrt:input.obj
 0001:0003a12e       ??$convert_decimal_string_to_floating_type@M@__crt_strtox@@YA?AW4SLD_STATUS@@ABUfloating_point_string@0@AAM@Z 1003b12e f i libucrt:input.obj
 0001:0003a151       ??$convert_decimal_string_to_floating_type@N@__crt_strtox@@YA?AW4SLD_STATUS@@ABUfloating_point_string@0@AAN@Z 1003b151 f i libucrt:input.obj
 0001:0003a174       ??$convert_hexadecimal_string_to_floating_type@M@__crt_strtox@@YA?AW4SLD_STATUS@@ABUfloating_point_string@0@AAM@Z 1003b174 f i libucrt:input.obj
 0001:0003a197       ??$convert_hexadecimal_string_to_floating_type@N@__crt_strtox@@YA?AW4SLD_STATUS@@ABUfloating_point_string@0@AAN@Z 1003b197 f i libucrt:input.obj
 0001:0003a1ba       ??$is_overflow_condition@_K@__crt_strtox@@YA_NI_K@Z 1003b1ba f i libucrt:input.obj
 0001:0003a1fd       ??$make_input_adapter_character_source@V?$stream_input_adapter@D@__crt_stdio_input@@@__crt_strtox@@YA?AV?$input_adapter_character_source@V?$stream_input_adapter@D@__crt_stdio_input@@@0@QAV?$stream_input_adapter@D@__crt_stdio_input@@_KQA_N@Z 1003b1fd f i libucrt:input.obj
 0001:0003a21b       ??$parse_floating_point@V?$input_adapter_character_source@V?$stream_input_adapter@D@__crt_stdio_input@@@__crt_strtox@@M@__crt_strtox@@YA?AW4SLD_STATUS@@QAU__crt_locale_pointers@@V?$input_adapter_character_source@V?$stream_input_adapter@D@__crt_stdio_input@@@0@QAM@Z 1003b21b f i libucrt:input.obj
 0001:0003a296       ??$parse_floating_point@V?$input_adapter_character_source@V?$stream_input_adapter@D@__crt_stdio_input@@@__crt_strtox@@N@__crt_strtox@@YA?AW4SLD_STATUS@@QAU__crt_locale_pointers@@V?$input_adapter_character_source@V?$stream_input_adapter@D@__crt_stdio_input@@@0@QAN@Z 1003b296 f i libucrt:input.obj
 0001:0003a311       ??$parse_floating_point_from_source@V?$input_adapter_character_source@V?$stream_input_adapter@D@__crt_stdio_input@@@__crt_strtox@@@__crt_strtox@@YA?AW4floating_point_parse_result@0@QAU__crt_locale_pointers@@AAV?$input_adapter_character_source@V?$stream_input_adapter@D@__crt_stdio_input@@@0@AAUfloating_point_string@0@@Z 1003b311 f i libucrt:input.obj
 0001:0003a778       ??$parse_floating_point_possible_infinity@DV?$input_adapter_character_source@V?$stream_input_adapter@D@__crt_stdio_input@@@__crt_strtox@@_K@__crt_strtox@@YA?AW4floating_point_parse_result@0@AADAAV?$input_adapter_character_source@V?$stream_input_adapter@D@__crt_stdio_input@@@0@_K@Z 1003b778 f i libucrt:input.obj
 0001:0003a839       ??$parse_floating_point_possible_nan@DV?$input_adapter_character_source@V?$stream_input_adapter@D@__crt_stdio_input@@@__crt_strtox@@_K@__crt_strtox@@YA?AW4floating_point_parse_result@0@AADAAV?$input_adapter_character_source@V?$stream_input_adapter@D@__crt_stdio_input@@@0@_K@Z 1003b839 f i libucrt:input.obj
 0001:0003a94b       ??$parse_floating_point_possible_nan_is_ind@DV?$input_adapter_character_source@V?$stream_input_adapter@D@__crt_stdio_input@@@__crt_strtox@@@__crt_strtox@@YA_NAADAAV?$input_adapter_character_source@V?$stream_input_adapter@D@__crt_stdio_input@@@0@@Z 1003b94b f i libucrt:input.obj
 0001:0003a985       ??$parse_floating_point_possible_nan_is_snan@DV?$input_adapter_character_source@V?$stream_input_adapter@D@__crt_stdio_input@@@__crt_strtox@@@__crt_strtox@@YA_NAADAAV?$input_adapter_character_source@V?$stream_input_adapter@D@__crt_stdio_input@@@0@@Z 1003b985 f i libucrt:input.obj
 0001:0003a9bf       ??$parse_floating_point_write_result@M@__crt_strtox@@YA?AW4SLD_STATUS@@W4floating_point_parse_result@0@ABUfloating_point_string@0@QAM@Z 1003b9bf f i libucrt:input.obj
 0001:0003aacf       ??$parse_floating_point_write_result@N@__crt_strtox@@YA?AW4SLD_STATUS@@W4floating_point_parse_result@0@ABUfloating_point_string@0@QAN@Z 1003bacf f i libucrt:input.obj
 0001:0003abd3       ??$parse_integer@_KV?$input_adapter_character_source@V?$stream_input_adapter@D@__crt_stdio_input@@@__crt_strtox@@@__crt_strtox@@YA_KQAU__crt_locale_pointers@@V?$input_adapter_character_source@V?$stream_input_adapter@D@__crt_stdio_input@@@0@H_N@Z 1003bbd3 f i libucrt:input.obj
 0001:0003ae84       ??$process_floating_point_specifier_t@M@?$input_processor@DV?$stream_input_adapter@D@__crt_stdio_input@@@__crt_stdio_input@@AAE_NXZ 1003be84 f i libucrt:input.obj
 0001:0003aeec       ??$process_floating_point_specifier_t@N@?$input_processor@DV?$stream_input_adapter@D@__crt_stdio_input@@@__crt_stdio_input@@AAE_NXZ 1003beec f i libucrt:input.obj
 0001:0003af54       ??$process_string_specifier_tchar@D@?$input_processor@DV?$stream_input_adapter@D@__crt_stdio_input@@@__crt_stdio_input@@AAE_NW4conversion_mode@1@D@Z 1003bf54 f i libucrt:input.obj
 0001:0003b0c8       ??$process_string_specifier_tchar@_W@?$input_processor@DV?$stream_input_adapter@D@__crt_stdio_input@@@__crt_stdio_input@@AAE_NW4conversion_mode@1@_W@Z 1003c0c8 f i libucrt:input.obj
 0001:0003b246       ??$skip_whitespace@Vstream_input_adapter@__crt_stdio_input@@D@__crt_stdio_input@@YAHAAV?$stream_input_adapter@D@0@QAU__crt_locale_pointers@@@Z 1003c246 f i libucrt:input.obj
 0001:0003b27d       ??$write_floating_point@M@?$input_processor@DV?$stream_input_adapter@D@__crt_stdio_input@@@__crt_stdio_input@@AAE_NABM@Z 1003c27d f i libucrt:input.obj
 0001:0003b2b4       ??$write_floating_point@N@?$input_processor@DV?$stream_input_adapter@D@__crt_stdio_input@@@__crt_stdio_input@@AAE_NABN@Z 1003c2b4 f i libucrt:input.obj
 0001:0003b2f1       ??0?$format_string_parser@D@__crt_stdio_input@@QAE@_KQBE@Z 1003c2f1 f i libucrt:input.obj
 0001:0003b33b       ??0?$input_adapter_character_source@V?$stream_input_adapter@D@__crt_stdio_input@@@__crt_strtox@@QAE@QAV?$stream_input_adapter@D@__crt_stdio_input@@_KQA_N@Z 1003c33b f i libucrt:input.obj
 0001:0003b36c       ??0?$input_processor@DV?$stream_input_adapter@D@__crt_stdio_input@@@__crt_stdio_input@@QAE@ABV?$stream_input_adapter@D@1@_KQBDQAU__crt_locale_pointers@@QAD@Z 1003c36c f i libucrt:input.obj
 0001:0003b465       ?advance@?$format_string_parser@D@__crt_stdio_input@@QAE_NXZ 1003c465 f i libucrt:input.obj
 0001:0003b585       ?as_double@floating_point_value@__crt_strtox@@QBEAANXZ 1003c585 f i libucrt:input.obj
 0001:0003b5aa       ?as_float@floating_point_value@__crt_strtox@@QBEAAMXZ 1003c5aa f i libucrt:input.obj
 0001:0003b5cf       ?assemble_floating_point_infinity@__crt_strtox@@YAX_NABVfloating_point_value@1@@Z 1003c5cf f i libucrt:input.obj
 0001:0003b609       ?assemble_floating_point_value@__crt_strtox@@YA?AW4SLD_STATUS@@_KH_N1ABVfloating_point_value@1@@Z 1003c609 f i libucrt:input.obj
 0001:0003b955       ?assemble_floating_point_value_from_big_integer@__crt_strtox@@YA?AW4SLD_STATUS@@ABUbig_integer@1@I_N1ABVfloating_point_value@1@@Z 1003c955 f i libucrt:input.obj
 0001:0003bae3       ?assemble_floating_point_zero@__crt_strtox@@YAX_NABVfloating_point_value@1@@Z 1003cae3 f i libucrt:input.obj
 0001:0003bb17       ?convert_decimal_string_to_floating_type_common@__crt_strtox@@YA?AW4SLD_STATUS@@ABUfloating_point_string@1@ABVfloating_point_value@1@@Z 1003cb17 f i libucrt:input.obj
 0001:0003d8da       ?convert_hexadecimal_string_to_floating_type_common@__crt_strtox@@YA?AW4SLD_STATUS@@ABUfloating_point_string@1@ABVfloating_point_value@1@@Z 1003e8da f i libucrt:input.obj
 0001:0003d986       ?denormal_mantissa_mask@floating_point_value@__crt_strtox@@QBE_KXZ 1003e986 f i libucrt:input.obj
 0001:0003d9a0       ?divide@__crt_strtox@@YA_KAAUbig_integer@1@ABU21@@Z 1003e9a0 f i libucrt:input.obj
 0001:0003de4e       ?get@?$input_adapter_character_source@V?$stream_input_adapter@D@__crt_stdio_input@@@__crt_strtox@@QAEDXZ 1003ee4e f i libucrt:input.obj
 0001:0003de87       ?invert@?$scanset_buffer@E@__crt_stdio_input@@QAEXXZ 1003ee87 f i libucrt:input.obj
 0001:0003dea5       ?is_character_allowed_in_string@?$input_processor@DV?$stream_input_adapter@D@__crt_stdio_input@@@__crt_stdio_input@@ABE_NW4conversion_mode@2@H@Z 1003eea5 f i libucrt:input.obj
 0001:0003deeb       ?length@?$format_string_parser@D@__crt_stdio_input@@QBEIXZ 1003eeeb f i libucrt:input.obj
 0001:0003df2c       ?normal_mantissa_mask@floating_point_value@__crt_strtox@@QBE_KXZ 1003ef2c f i libucrt:input.obj
 0001:0003df43       ?process@?$input_processor@DV?$stream_input_adapter@D@__crt_stdio_input@@@__crt_stdio_input@@QAEHXZ 1003ef43 f i libucrt:input.obj
 0001:0003dfcf       ?process_character_count_specifier@?$input_processor@DV?$stream_input_adapter@D@__crt_stdio_input@@@__crt_stdio_input@@AAE_NXZ 1003efcf f i libucrt:input.obj
 0001:0003dfe5       ?process_conversion_specifier@?$input_processor@DV?$stream_input_adapter@D@__crt_stdio_input@@@__crt_stdio_input@@AAE_NXZ 1003efe5 f i libucrt:input.obj
 0001:0003e059       ?process_floating_point_specifier@?$input_processor@DV?$stream_input_adapter@D@__crt_stdio_input@@@__crt_stdio_input@@AAE_NXZ 1003f059 f i libucrt:input.obj
 0001:0003e089       ?process_integer_specifier@?$input_processor@DV?$stream_input_adapter@D@__crt_stdio_input@@@__crt_stdio_input@@AAE_NI_N@Z 1003f089 f i libucrt:input.obj
 0001:0003e0ef       ?process_literal_character@?$input_processor@DV?$stream_input_adapter@D@__crt_stdio_input@@@__crt_stdio_input@@AAE_NXZ 1003f0ef f i libucrt:input.obj
 0001:0003e125       ?process_literal_character_tchar@?$input_processor@DV?$stream_input_adapter@D@__crt_stdio_input@@@__crt_stdio_input@@AAE_ND@Z 1003f125 f i libucrt:input.obj
 0001:0003e184       ?process_state@?$input_processor@DV?$stream_input_adapter@D@__crt_stdio_input@@@__crt_stdio_input@@AAE_NXZ 1003f184 f i libucrt:input.obj
 0001:0003e1ba       ?process_string_specifier@?$input_processor@DV?$stream_input_adapter@D@__crt_stdio_input@@@__crt_stdio_input@@AAE_NW4conversion_mode@2@@Z 1003f1ba f i libucrt:input.obj
 0001:0003e202       ?process_whitespace@?$input_processor@DV?$stream_input_adapter@D@__crt_stdio_input@@@__crt_stdio_input@@AAE_NXZ 1003f202 f i libucrt:input.obj
 0001:0003e21f       ?restore_state@?$input_adapter_character_source@V?$stream_input_adapter@D@__crt_stdio_input@@@__crt_strtox@@QAE_N_K@Z 1003f21f f i libucrt:input.obj
 0001:0003e244       ?scan_conversion_specifier@?$format_string_parser@D@__crt_stdio_input@@AAE_NXZ 1003f244 f i libucrt:input.obj
 0001:0003e3af       ?scan_optional_field_width@?$format_string_parser@D@__crt_stdio_input@@AAE_NXZ 1003f3af f i libucrt:input.obj
 0001:0003e44e       ?scan_optional_length_modifier@?$format_string_parser@D@__crt_stdio_input@@AAEXXZ 1003f44e f i libucrt:input.obj
 0001:0003e56e       ?scan_optional_literal_character_trail_bytes_tchar@?$format_string_parser@D@__crt_stdio_input@@AAE_ND@Z 1003f56e f i libucrt:input.obj
 0001:0003e5c3       ?scan_optional_wide_modifier@?$format_string_parser@D@__crt_stdio_input@@AAEXXZ 1003f5c3 f i libucrt:input.obj
 0001:0003e5e1       ?scan_scanset_range@?$format_string_parser@D@__crt_stdio_input@@AAE_NXZ 1003f5e1 f i libucrt:input.obj
 0001:0003e6e8       ?set@?$scanset_buffer@E@__crt_stdio_input@@QAEXE@Z 1003f6e8 f i libucrt:input.obj
 0001:0003e713       ?set_wide_for_c_s_or_scanset@?$format_string_parser@D@__crt_stdio_input@@AAEXXZ 1003f713 f i libucrt:input.obj
 0001:0003e733       ?test@?$scanset_buffer@E@__crt_stdio_input@@QBE_NE@Z 1003f733 f i libucrt:input.obj
 0001:0003e764       ?to_floating_point_length@__crt_stdio_input@@YAIW4length_modifier@1@@Z 1003f764 f i libucrt:input.obj
 0001:0003e787       ?to_integer_length@__crt_stdio_input@@YAIW4length_modifier@1@@Z 1003f787 f i libucrt:input.obj
 0001:0003e7df       ?unget@?$input_adapter_character_source@V?$stream_input_adapter@D@__crt_stdio_input@@@__crt_strtox@@QAEXD@Z 1003f7df f i libucrt:input.obj
 0001:0003e820       ?unget@?$stream_input_adapter@D@__crt_stdio_input@@QAEXH@Z 1003f820 f i libucrt:input.obj
 0001:0003e83e       ?validate@?$format_string_parser@D@__crt_stdio_input@@QBE_NXZ 1003f83e f i libucrt:input.obj
 0001:0003e85a       ?validate@?$input_adapter_character_source@V?$stream_input_adapter@D@__crt_stdio_input@@@__crt_strtox@@QBE_NXZ 1003f85a f i libucrt:input.obj
 0001:0003e87b       ?validate@?$stream_input_adapter@D@__crt_stdio_input@@QBE_NXZ 1003f87b f i libucrt:input.obj
 0001:0003e87b       ?validate@?$stream_output_adapter@D@__crt_stdio_output@@QBE_NXZ 1003f87b f i libucrt:output.obj
 0001:0003e89c       ?write_character@?$input_processor@DV?$stream_input_adapter@D@__crt_stdio_input@@@__crt_stdio_input@@AAE_NQA_WIAAPA_WAAID@Z 1003f89c f i libucrt:input.obj
 0001:0003e916       ?write_integer@?$input_processor@DV?$stream_input_adapter@D@__crt_stdio_input@@@__crt_stdio_input@@AAE_N_K_N@Z 1003f916 f i libucrt:input.obj
 0001:0003e98d       ___stdio_common_vfscanf    1003f98d f   libucrt:input.obj
 0001:0003ec17       __wdupenv_s                1003fc17 f   libucrt:getenv.obj
 0001:0003ec35       __wgetenv                  1003fc35 f   libucrt:getenv.obj
 0001:0003ed40       __wsystem                  1003fd40 f   libucrt:system.obj
 0001:0003ed4b       _wcscmp                    1003fd4b f   libucrt:wcscmp.obj
 0001:0003ed8b       __initterm                 1003fd8b f   libucrt:initterm.obj
 0001:0003ede7       __initterm_e               1003fde7 f   libucrt:initterm.obj
 0001:0003ee2c       __seh_filter_dll           1003fe2c f   libucrt:exception_filter.obj
 0001:0003ee4c       __seh_filter_exe           1003fe4c f   libucrt:exception_filter.obj
 0001:0003f1da       ___acrt_initialize_thread_local_exit_callback 100401da f   libucrt:exit.obj
 0001:0003f1e9       __cexit                    100401e9 f   libucrt:exit.obj
 0001:0003f1f8       __exit                     100401f8 f   libucrt:exit.obj
 0001:0003f20e       __is_c_termination_complete 1004020e f   libucrt:exit.obj
 0001:0003f4ad       ___acrt_allocate_buffer_for_argv 100404ad f   libucrt:argv_parsing.obj
 0001:0003f502       __configure_narrow_argv    10040502 f   libucrt:argv_parsing.obj
 0001:0003f85c       ??$uninitialize@A6AXAAPAPAD@Z@?$dual_state_global@PAPAD@__crt_state_management@@QAEXA6AXAAPAPAD@Z@Z 1004085c f i libucrt:environment_initialization.obj
 0001:0003f85c       ??$uninitialize@A6AXAAPAPA_W@Z@?$dual_state_global@PAPA_W@__crt_state_management@@QAEXA6AXAAPAPA_W@Z@Z 1004085c f i libucrt:environment_initialization.obj
 0001:0003f8d2       ___dcrt_get_or_create_wide_environment_nolock 100408d2 f   libucrt:environment_initialization.obj
 0001:0003f8d7       ___dcrt_uninitialize_environments_nolock 100408d7 f   libucrt:environment_initialization.obj
 0001:0003f90e       __initialize_narrow_environment 1004090e f   libucrt:environment_initialization.obj
 0001:0003f913       ??$?RV<lambda_800076c951b434888f4765a74a194fcc>@@AAV<lambda_4e60a939b0d047cfe11ddc22648dfba9>@@V<lambda_6dbb1268764f43b569ce7b67e331d33a>@@@?$__crt_seh_guarded_call@H@@QAEH$$QAV<lambda_800076c951b434888f4765a74a194fcc>@@AAV<lambda_4e60a939b0d047cfe11ddc22648dfba9>@@$$QAV<lambda_6dbb1268764f43b569ce7b67e331d33a>@@@Z 10040913 f i libucrt:onexit.obj
 0001:0003f964       ??$?RV<lambda_995298e7d72eb4c2aab26c0585b3abe5>@@AAV<lambda_275893d493268fdec8709772e3fcec0e>@@V<lambda_293819299cbf9a7022e18b56a874bb5c>@@@?$__crt_seh_guarded_call@H@@QAEH$$QAV<lambda_995298e7d72eb4c2aab26c0585b3abe5>@@AAV<lambda_275893d493268fdec8709772e3fcec0e>@@$$QAV<lambda_293819299cbf9a7022e18b56a874bb5c>@@@Z 10040964 f i libucrt:onexit.obj
 0001:0003f9b5       ??$__acrt_lock_and_call@V<lambda_275893d493268fdec8709772e3fcec0e>@@@@YAHW4__acrt_lock_id@@$$QAV<lambda_275893d493268fdec8709772e3fcec0e>@@@Z 100409b5 f i libucrt:onexit.obj
 0001:0003f9dd       ??$__acrt_lock_and_call@V<lambda_4e60a939b0d047cfe11ddc22648dfba9>@@@@YAHW4__acrt_lock_id@@$$QAV<lambda_4e60a939b0d047cfe11ddc22648dfba9>@@@Z 100409dd f i libucrt:onexit.obj
 0001:0003fa05       ??$__crt_fast_encode_pointer@P6AHXZ@@YAP6AHXZQ6AHXZ@Z 10040a05 f i libucrt:onexit.obj
 0001:0003fc85       __crt_atexit               10040c85 f   libucrt:onexit.obj
 0001:0003fc9b       __execute_onexit_table     10040c9b f   libucrt:onexit.obj
 0001:0003fcb8       __initialize_onexit_table  10040cb8 f   libucrt:onexit.obj
 0001:0003fcf5       __register_onexit_function 10040cf5 f   libucrt:onexit.obj
 0001:0003fd45       ___acrt_uninitialize_command_line 10040d45 f   libucrt:argv_data.obj
 0001:0003fe0d       ___acrt_initialize         10040e0d f   libucrt:initialization.obj
 0001:0003fe1f       ___acrt_thread_attach      10040e1f f   libucrt:initialization.obj
 0001:0003fe2a       ___acrt_thread_detach      10040e2a f   libucrt:initialization.obj
 0001:0003fe32       ___acrt_uninitialize       10040e32 f   libucrt:initialization.obj
 0001:0003fe44       ___acrt_uninitialize_critical 10040e44 f   libucrt:initialization.obj
 0001:0003fe56       _terminate                 10040e56 f   libucrt:terminate.obj
 0001:0004000e       __freea_crt                1004100e f i libucrt:strupr.obj
 0001:0004002e       __strupr                   1004102e f   libucrt:strupr.obj
 0001:0004002e       _strupr                    1004102e f   libucrt:strupr.obj
 0001:0004008b       __strupr_s_l               1004108b f   libucrt:strupr.obj
 0001:000400c4       __free_base                100410c4 f   libucrt:free_base.obj
 0001:000400fe       __malloc_base              100410fe f   libucrt:malloc_base.obj
 0001:0004014c       _strcpy_s                  1004114c f   libucrt:strcpy_s.obj
 0001:000401a6       _abort                     100411a6 f   libucrt:abort.obj
 0001:000401e9       __calloc_base              100411e9 f   libucrt:calloc_base.obj
 0001:00040246       ??$is_overflow_condition@K@__crt_strtox@@YA_NIK@Z 10041246 f i libucrt:atox.obj
 0001:00040279       ??$parse_integer@KV?$c_string_character_source@D@__crt_strtox@@@__crt_strtox@@YAKQAU__crt_locale_pointers@@V?$c_string_character_source@D@0@H_N@Z 10041279 f i libucrt:atox.obj
 0001:000404a1       ??$parse_integer@KV?$c_string_character_source@_W@__crt_strtox@@@__crt_strtox@@YAKQAU__crt_locale_pointers@@V?$c_string_character_source@_W@0@H_N@Z 100414a1 f i libucrt:atox.obj
 0001:00040b86       ??$parse_integer@_KV?$c_string_character_source@D@__crt_strtox@@@__crt_strtox@@YA_KQAU__crt_locale_pointers@@V?$c_string_character_source@D@0@H_N@Z 10041b86 f i libucrt:atox.obj
 0001:00040e2c       ?unget@?$c_string_character_source@D@__crt_strtox@@QAEXD@Z 10041e2c f i libucrt:atox.obj
 0001:00040e54       ?unget@?$c_string_character_source@_W@__crt_strtox@@QAEX_W@Z 10041e54 f i libucrt:atox.obj
 0001:00040e80       ?validate@?$string_output_adapter@_W@__crt_stdio_output@@QBE_NXZ 10041e80 f i libucrt:output.obj
 0001:00040e80       ?validate@?$c_string_character_source@_W@__crt_strtox@@QBE_NXZ 10041e80 f i libucrt:atox.obj
 0001:00040e80       ?validate@?$c_string_character_source@D@__crt_strtox@@QBE_NXZ 10041e80 f i libucrt:atox.obj
 0001:00040e80       ?validate@?$string_output_adapter@D@__crt_stdio_output@@QBE_NXZ 10041e80 f i libucrt:output.obj
 0001:00040e9b       ___acrt_call_reportfault   10041e9b f   libucrt:invalid_parameter.obj
 0001:00040fd6       ___acrt_initialize_invalid_parameter_handler 10041fd6 f   libucrt:invalid_parameter.obj
 0001:00040fea       __invalid_parameter        10041fea f   libucrt:invalid_parameter.obj
 0001:00041065       __invalid_parameter_noinfo 10042065 f   libucrt:invalid_parameter.obj
 0001:00041075       __invoke_watson            10042075 f   libucrt:invalid_parameter.obj
 0001:0004120f       __tolower_l                1004220f f   libucrt:tolower_toupper.obj
 0001:00041229       _tolower                   10042229 f   libucrt:tolower_toupper.obj
 0001:00041259       ??$make_c_string_character_source@DPAPAD@__crt_strtox@@YA?AV?$c_string_character_source@D@0@QBDQAPAD@Z 10042259 f i libucrt:strtox.obj
 0001:00041259       ??$make_c_string_character_source@_WPAPA_W@__crt_strtox@@YA?AV?$c_string_character_source@_W@0@QB_WQAPA_W@Z 10042259 f i libucrt:strtox.obj
 0001:00041274       _strtol                    10042274 f   libucrt:strtox.obj
 0001:000412a0       _strtoull                  100422a0 f   libucrt:strtox.obj
 0001:000412cc       _wcstol                    100422cc f   libucrt:strtox.obj
 0001:000412f8       __mbtowc_l                 100422f8 f   libucrt:mbtowc.obj
 0001:000413f2       _mbtowc                    100423f2 f   libucrt:mbtowc.obj
 0001:0004140c       __wctomb_s_l               1004240c f   libucrt:wctomb.obj
 0001:0004152d       _wctomb_s                  1004252d f   libucrt:wctomb.obj
 0001:0004154a       _strnlen                   1004254a f   libucrt:strnlen.obj
 0001:00041671       _wcsnlen                   10042671 f   libucrt:strnlen.obj
 0001:00041828       ??$?RV<lambda_3518db117f0e7cdb002338c5d3c47b6c>@@AAV<lambda_b2ea41f6bbb362cd97d94c6828d90b61>@@V<lambda_abdedf541bb04549bc734292b4a045d4>@@@?$__crt_seh_guarded_call@X@@QAEX$$QAV<lambda_3518db117f0e7cdb002338c5d3c47b6c>@@AAV<lambda_b2ea41f6bbb362cd97d94c6828d90b61>@@$$QAV<lambda_abdedf541bb04549bc734292b4a045d4>@@@Z 10042828 f i libucrt:per_thread_data.obj
 0001:00041878       ??$?RV<lambda_51b6e8b1eb166f2a3faf91f424b38130>@@AAV<lambda_6250bd4b2a391816dd638c3bf72b0bcb>@@V<lambda_0b5a4a3e68152e1d9b943535f5f47bed>@@@?$__crt_seh_guarded_call@X@@QAEX$$QAV<lambda_51b6e8b1eb166f2a3faf91f424b38130>@@AAV<lambda_6250bd4b2a391816dd638c3bf72b0bcb>@@$$QAV<lambda_0b5a4a3e68152e1d9b943535f5f47bed>@@@Z 10042878 f i libucrt:per_thread_data.obj
 0001:000418d9       ??$?RV<lambda_5b71d36f03204c0beab531769a5b5694>@@AAV<lambda_be2b3da3f62db62e9dad5dc70221a656>@@V<lambda_8f9ce462984622f9bf76b59e2aaaf805>@@@?$__crt_seh_guarded_call@X@@QAEX$$QAV<lambda_5b71d36f03204c0beab531769a5b5694>@@AAV<lambda_be2b3da3f62db62e9dad5dc70221a656>@@$$QAV<lambda_8f9ce462984622f9bf76b59e2aaaf805>@@@Z 100428d9 f i libucrt:per_thread_data.obj
 0001:00041924       ??$?RV<lambda_9df27f884b057bc3edfc946cb5b7cf47>@@AAV<lambda_e69574bed617af4e071282c136b37893>@@V<lambda_cc0d902bcbbeb830f749456577db4721>@@@?$__crt_seh_guarded_call@X@@QAEX$$QAV<lambda_9df27f884b057bc3edfc946cb5b7cf47>@@AAV<lambda_e69574bed617af4e071282c136b37893>@@$$QAV<lambda_cc0d902bcbbeb830f749456577db4721>@@@Z 10042924 f i libucrt:per_thread_data.obj
 0001:0004196c       ??$__acrt_lock_and_call@V<lambda_6250bd4b2a391816dd638c3bf72b0bcb>@@@@YAXW4__acrt_lock_id@@$$QAV<lambda_6250bd4b2a391816dd638c3bf72b0bcb>@@@Z 1004296c f i libucrt:per_thread_data.obj
 0001:00041994       ??$__acrt_lock_and_call@V<lambda_b2ea41f6bbb362cd97d94c6828d90b61>@@@@YAXW4__acrt_lock_id@@$$QAV<lambda_b2ea41f6bbb362cd97d94c6828d90b61>@@@Z 10042994 f i libucrt:per_thread_data.obj
 0001:000419bc       ??$__acrt_lock_and_call@V<lambda_be2b3da3f62db62e9dad5dc70221a656>@@@@YAXW4__acrt_lock_id@@$$QAV<lambda_be2b3da3f62db62e9dad5dc70221a656>@@@Z 100429bc f i libucrt:per_thread_data.obj
 0001:000419e4       ??$__acrt_lock_and_call@V<lambda_e69574bed617af4e071282c136b37893>@@@@YAXW4__acrt_lock_id@@$$QAV<lambda_e69574bed617af4e071282c136b37893>@@@Z 100429e4 f i libucrt:per_thread_data.obj
 0001:00041b9a       ___acrt_freeptd            10042b9a f   libucrt:per_thread_data.obj
 0001:00041bc6       ___acrt_getptd             10042bc6 f   libucrt:per_thread_data.obj
 0001:00041c4a       ___acrt_getptd_noexit      10042c4a f   libucrt:per_thread_data.obj
 0001:00041ccf       ___acrt_initialize_ptd     10042ccf f   libucrt:per_thread_data.obj
 0001:00041cfb       ___acrt_uninitialize_ptd   10042cfb f   libucrt:per_thread_data.obj
 0001:00041d15       ___acrt_update_locale_info 10042d15 f   libucrt:locale_update.obj
 0001:00041d42       ___acrt_update_multibyte_info 10042d42 f   libucrt:locale_update.obj
 0001:00041d6f       ?__acrt_fp_classify@@YA?AW4__acrt_fp_class@@ABN@Z 10042d6f f i libucrt:cvt.obj
 0001:00041ddb       ?__acrt_fp_is_negative@@YA_NABN@Z 10042ddb f i libucrt:cvt.obj
 0001:0004263a       ___acrt_fp_format          1004363a f   libucrt:cvt.obj
 0001:00042784       __fileno                   10043784 f   libucrt:fileno.obj
 0001:000427aa       __fputc_nolock             100437aa f   libucrt:fputc.obj
 0001:000427d3       __get_printf_count_output  100437d3 f   libucrt:printf_count_output.obj
 0001:000427e8       ___acrt_stdio_begin_temporary_buffering_nolock 100437e8 f   libucrt:_sftbuf.obj
 0001:0004289d       ___acrt_stdio_end_temporary_buffering_nolock 1004389d f   libucrt:_sftbuf.obj
 0001:000428d6       ___acrt_set_locale_changed 100438d6 f   libucrt:wsetlocale.obj
 0001:000428e1       ___acrt_uninitialize_locale 100438e1 f   libucrt:wsetlocale.obj
 0001:00042a9f       ___acrt_initialize_lowio   10043a9f f   libucrt:ioinit.obj
 0001:00042af5       ___acrt_uninitialize_lowio 10043af5 f   libucrt:ioinit.obj
 0001:00042b21       _wcscpy_s                  10043b21 f   libucrt:wcscpy_s.obj
 0001:00042b85       ?__acrt_stdio_allocate_stream@@YA?AV__crt_stdio_stream@@XZ 10043b85 f   libucrt:stream.obj
 0001:00042be4       ?__acrt_stdio_free_stream@@YAXV__crt_stdio_stream@@@Z 10043be4 f   libucrt:stream.obj
 0001:00042ce2       ??$__acrt_stdio_parse_mode@_W@@YA?AU__acrt_stdio_stream_mode@@QB_W@Z 10043ce2 f i libucrt:openfile.obj
 0001:00042fab       ?__acrt_stdio_parse_mode_D@@YA_NAAU__acrt_stdio_stream_mode@@@Z 10043fab f i libucrt:openfile.obj
 0001:00042fc6       ?__acrt_stdio_parse_mode_T@@YA_NAAU__acrt_stdio_stream_mode@@@Z 10043fc6 f i libucrt:openfile.obj
 0001:00042fe5       ?__acrt_stdio_parse_mode_b@@YA_NAAU__acrt_stdio_stream_mode@@@Z 10043fe5 f i libucrt:openfile.obj
 0001:00043005       ?__acrt_stdio_parse_mode_c@@YA_NAAU__acrt_stdio_stream_mode@@AA_N@Z 10044005 f i libucrt:openfile.obj
 0001:00043027       ?__acrt_stdio_parse_mode_n@@YA_NAAU__acrt_stdio_stream_mode@@AA_N@Z 10044027 f i libucrt:openfile.obj
 0001:00043049       ?__acrt_stdio_parse_mode_plus@@YA_NAAU__acrt_stdio_stream_mode@@AA_N@Z 10044049 f i libucrt:openfile.obj
 0001:0004307e       ?__acrt_stdio_parse_mode_t@@YA_NAAU__acrt_stdio_stream_mode@@@Z 1004407e f i libucrt:openfile.obj
 0001:0004309e       __wopenfile                1004409e f   libucrt:openfile.obj
 0001:000430a9       ??$?RV<lambda_123407a5e2ac06da108355a851863b7a>@@AAV<lambda_2fe9b910cf3cbf4a0ab98a02ba45b3ec>@@V<lambda_ae55bdf541ad94d75914d381c370e64d>@@@?$__crt_seh_guarded_call@H@@QAEH$$QAV<lambda_123407a5e2ac06da108355a851863b7a>@@AAV<lambda_2fe9b910cf3cbf4a0ab98a02ba45b3ec>@@$$QAV<lambda_ae55bdf541ad94d75914d381c370e64d>@@@Z 100440a9 f i libucrt:close.obj
 0001:0004312b       ??$__acrt_lowio_lock_fh_and_call@V<lambda_2fe9b910cf3cbf4a0ab98a02ba45b3ec>@@@@YAHH$$QAV<lambda_2fe9b910cf3cbf4a0ab98a02ba45b3ec>@@@Z 1004412b f i libucrt:close.obj
 0001:00043153       __close                    10044153 f   libucrt:close.obj
 0001:000431d2       __close_nolock             100441d2 f   libucrt:close.obj
 0001:0004326e       ___acrt_stdio_free_buffer_nolock 1004426e f   libucrt:_freebuf.obj
 0001:000432ac       ??$?RV<lambda_a048d3beccc847880fc8490e18b82769>@@AAV<lambda_ec61778202f4f5fc7e7711acc23c3bca>@@V<lambda_f7496a158712204296dd6628a163878e>@@@?$__crt_seh_guarded_call@P6AXH@Z@@QAEP6AXH@Z$$QAV<lambda_a048d3beccc847880fc8490e18b82769>@@AAV<lambda_ec61778202f4f5fc7e7711acc23c3bca>@@$$QAV<lambda_f7496a158712204296dd6628a163878e>@@@Z 100442ac f i libucrt:signal.obj
 0001:00043306       ??$__acrt_lock_and_call@V<lambda_ec61778202f4f5fc7e7711acc23c3bca>@@@@YAP6AXH@ZW4__acrt_lock_id@@$$QAV<lambda_ec61778202f4f5fc7e7711acc23c3bca>@@@Z 10044306 f i libucrt:signal.obj
 0001:00043398       ___acrt_get_sigabrt_handler 10044398 f   libucrt:signal.obj
 0001:000433af       ___acrt_initialize_signal_handlers 100443af f   libucrt:signal.obj
 0001:000433ea       ___fpecode                 100443ea f   libucrt:signal.obj
 0001:000433f3       _raise                     100443f3 f   libucrt:signal.obj
 0001:000435fb       ___set_fpsr_sse2           100445fb f   libucrt:fpctrl.obj
 0001:00043671       __clrfp                    10044671 f   libucrt:fpctrl.obj
 0001:00043684       __ctrlfp                   10044684 f   libucrt:fpctrl.obj
 0001:000436b0       __set_statfp               100446b0 f   libucrt:fpctrl.obj
 0001:0004370b       __statfp                   1004470b f   libucrt:fpctrl.obj
 0001:0004371d       ___sys_errlist             1004471d f   libucrt:syserr.obj
 0001:00043723       ___sys_nerr                10044723 f   libucrt:syserr.obj
 0001:000437da       _strncpy_s                 100447da f   libucrt:strncpy_s.obj
 0001:00043916       ___acrt_AreFileApisANSI@0  10044916 f   libucrt:winapi_thunks.obj
 0001:00043964       ___acrt_CompareStringEx@36 10044964 f   libucrt:winapi_thunks.obj
 0001:000439d8       ___acrt_FlsAlloc@4         100449d8 f   libucrt:winapi_thunks.obj
 0001:00043a2e       ___acrt_FlsFree@4          10044a2e f   libucrt:winapi_thunks.obj
 0001:00043a84       ___acrt_FlsGetValue@4      10044a84 f   libucrt:winapi_thunks.obj
 0001:00043ada       ___acrt_FlsSetValue@8      10044ada f   libucrt:winapi_thunks.obj
 0001:00043b33       ___acrt_InitializeCriticalSectionEx@12 10044b33 f   libucrt:winapi_thunks.obj
 0001:00043b95       ___acrt_LCMapStringEx@36   10044b95 f   libucrt:winapi_thunks.obj
 0001:00043c1d       ___acrt_LocaleNameToLCID@8 10044c1d f   libucrt:winapi_thunks.obj
 0001:00043c79       ___acrt_initialize_winapi_thunks 10044c79 f   libucrt:winapi_thunks.obj
 0001:00043c9f       ___acrt_is_packaged_app    10044c9f f   libucrt:winapi_thunks.obj
 0001:00043d26       ___acrt_uninitialize_winapi_thunks 10044d26 f   libucrt:winapi_thunks.obj
 0001:00043d5c       __fcloseall                10044d5c f   libucrt:closeall.obj
 0001:000442e4       __read                     100452e4 f   libucrt:read.obj
 0001:000443f7       __read_nolock              100453f7 f   libucrt:read.obj
 0001:0004492d       ___acrt_stdio_refill_and_read_narrow_nolock 1004592d f   libucrt:_filbuf.obj
 0001:00044c81       __lseek                    10045c81 f   libucrt:lseek.obj
 0001:00044c8c       __lseeki64                 10045c8c f   libucrt:lseek.obj
 0001:00044ca7       __lseeki64_nolock          10045ca7 f   libucrt:lseek.obj
 0001:00044cc2       ___acrt_stdio_allocate_buffer_nolock 10045cc2 f   libucrt:_getbuf.obj
 0001:00044d1f       ___pctype_func             10045d1f f   libucrt:ctype.obj
 0001:00044d45       __isctype_l                10045d45 f   libucrt:isctype.obj
 0001:00044e17       __towlower_l               10045e17 f   libucrt:towlower.obj
 0001:00044ee0       __recalloc                 10045ee0 f   libucrt:recalloc.obj
 0001:00044eeb       __recalloc_base            10045eeb f   libucrt:recalloc.obj
 0001:00044f58       _wcscat_s                  10045f58 f   libucrt:wcscat_s.obj
 0001:00044fcd       __cwait                    10045fcd f   libucrt:wait.obj
 0001:0004514b       ___acrt_wgetpath           1004614b f   libucrt:getpath.obj
 0001:00045156       ___acrt_initialize_locks   10046156 f   libucrt:locks.obj
 0001:00045197       ___acrt_lock               10046197 f   libucrt:locks.obj
 0001:000451ae       ___acrt_uninitialize_locks 100461ae f   libucrt:locks.obj
 0001:000451df       ___acrt_unlock             100461df f   libucrt:locks.obj
 0001:000451f6       __waccess_s                100461f6 f   libucrt:waccess.obj
 0001:000452b6       __pipe                     100462b6 f   libucrt:pipe.obj
 0001:0004563d       __wfdopen                  1004663d f   libucrt:fdopen.obj
 0001:00045648       ??$?RV<lambda_61cee617f5178ae960314fd4d05640a0>@@AAV<lambda_6978c1fb23f02e42e1d9e99668cc68aa>@@V<lambda_9cd88cf8ad10232537feb2133f08c833>@@@?$__crt_seh_guarded_call@H@@QAEH$$QAV<lambda_61cee617f5178ae960314fd4d05640a0>@@AAV<lambda_6978c1fb23f02e42e1d9e99668cc68aa>@@$$QAV<lambda_9cd88cf8ad10232537feb2133f08c833>@@@Z 10046648 f i libucrt:commit.obj
 0001:000456e0       ??$__acrt_lowio_lock_fh_and_call@V<lambda_6978c1fb23f02e42e1d9e99668cc68aa>@@@@YAHH$$QAV<lambda_6978c1fb23f02e42e1d9e99668cc68aa>@@@Z 100466e0 f i libucrt:commit.obj
 0001:00045708       __commit                   10046708 f   libucrt:commit.obj
 0001:00045d07       __write                    10046d07 f   libucrt:write.obj
 0001:00045df2       __write_nolock             10046df2 f   libucrt:write.obj
 0001:000461db       ___acrt_stdio_flush_and_write_narrow_nolock 100471db f   libucrt:_flsbuf.obj
 0001:000462ea       __ui64toa_s                100472ea f   libucrt:xtoa.obj
 0001:0004630a       __strdup                   1004730a f   libucrt:strdup.obj
 0001:00046360       ___acrt_GetTempPathA       10047360 f   libucrt:gettemppath.obj
 0001:00046a87       __sopen_nolock             10047a87 f   libucrt:open.obj
 0001:00046ad8       __sopen_s                  10047ad8 f   libucrt:open.obj
 0001:00046af8       __wsopen_nolock            10047af8 f   libucrt:open.obj
 0001:00046e21       __wsopen_s                 10047e21 f   libucrt:open.obj
 0001:00046e41       ___acrt_uninitialize_tmpfile 10047e41 f   libucrt:rmtmp.obj
 0001:00046e4b       __rmtmp                    10047e4b f   libucrt:rmtmp.obj
 0001:00046ee2       _fegetround                10047ee2 f   libucrt:fegetround.obj
 0001:00046eed       _calloc                    10047eed f   libucrt:calloc.obj
 0001:00046ef8       __wcsnicoll                10047ef8 f   libucrt:wcsnicol.obj
 0001:00046fc8       __wcsnicoll_l              10047fc8 f   libucrt:wcsnicol.obj
 0001:000470f5       ??$?RV<lambda_eee62cb4a147bfbb98180ad682ce6e17>@@AAV<lambda_5056f36f92c185fae794536d1ce2027b>@@V<lambda_57c77e0e75d6a1e6f8ecaa6bd26c2518>@@@?$__crt_seh_guarded_call@_N@@QAE_N$$QAV<lambda_eee62cb4a147bfbb98180ad682ce6e17>@@AAV<lambda_5056f36f92c185fae794536d1ce2027b>@@$$QAV<lambda_57c77e0e75d6a1e6f8ecaa6bd26c2518>@@@Z 100480f5 f i libucrt:spawnv.obj
 0001:00047146       ??$__acrt_lock_and_call@V<lambda_5056f36f92c185fae794536d1ce2027b>@@@@YA_NW4__acrt_lock_id@@$$QAV<lambda_5056f36f92c185fae794536d1ce2027b>@@@Z 10048146 f i libucrt:spawnv.obj
 0001:000476e4       __wspawnve                 100486e4 f   libucrt:spawnv.obj
 0001:000479d8       __wspawnvpe                100489d8 f   libucrt:spawnvp.obj
 0001:00047da5       ??1?$argument_list@D@?A0xb0e4b824@@QAE@XZ 10048da5 f i libucrt:argv_wildcards.obj
 0001:00047dca       ?append@?$argument_list@D@?A0xb0e4b824@@QAEHQAD@Z 10048dca f i libucrt:argv_wildcards.obj
 0001:00047dff       ?expand_if_necessary@?$argument_list@D@?A0xb0e4b824@@AAEHXZ 10048dff f i libucrt:argv_wildcards.obj
 0001:00047e86       ___acrt_expand_narrow_argv_wildcards 10048e86 f   libucrt:argv_wildcards.obj
 0001:00047e91       ??$?RV<lambda_978dc153c237d78434369da87b74ff60>@@AAV<lambda_ad1ced32f4ac17aa236e5ef05d6b3b7c>@@V<lambda_4a8533e2866a575feecb8298ce776b0d>@@@?$__crt_seh_guarded_call@X@@QAEX$$QAV<lambda_978dc153c237d78434369da87b74ff60>@@AAV<lambda_ad1ced32f4ac17aa236e5ef05d6b3b7c>@@$$QAV<lambda_4a8533e2866a575feecb8298ce776b0d>@@@Z 10048e91 f i libucrt:mbctype.obj
 0001:00047ed4       ??$__acrt_lock_and_call@V<lambda_ad1ced32f4ac17aa236e5ef05d6b3b7c>@@@@YAXW4__acrt_lock_id@@$$QAV<lambda_ad1ced32f4ac17aa236e5ef05d6b3b7c>@@@Z 10048ed4 f i libucrt:mbctype.obj
 0001:0004836b       ___acrt_initialize_multibyte 1004936b f   libucrt:mbctype.obj
 0001:00048389       ___acrt_update_thread_multibyte_data 10049389 f   libucrt:mbctype.obj
 0001:0004842b       __setmbcp_nolock           1004942b f   libucrt:mbctype.obj
 0001:00048675       __ismbblead                10049675 f   libucrt:ismbbyte.obj
 0001:0004868d       ___acrt_initialize_command_line 1004968d f   libucrt:argv_data.obj
 0001:000486dd       ___dcrt_get_narrow_environment_from_os 100496dd f   libucrt:get_environment_from_os.obj
 0001:00048760       ___dcrt_get_wide_environment_from_os 10049760 f   libucrt:get_environment_from_os.obj
 0001:00048b02       ___dcrt_set_variable_in_wide_environment_nolock 10049b02 f   libucrt:setenv.obj
 0001:00048b0d       ___acrt_initialize_heap    10049b0d f   libucrt:heap_handle.obj
 0001:00048b1e       ___acrt_uninitialize_heap  10049b1e f   libucrt:heap_handle.obj
 0001:00048b28       ___acrt_execute_initializers 10049b28 f   libucrt:shared_initialization.obj
 0001:00048bab       ___acrt_execute_uninitializers 10049bab f   libucrt:shared_initialization.obj
 0001:00048bf8       ?initialize@?$dual_state_global@PAU__crt_locale_data@@@__crt_state_management@@QAEXQAU__crt_locale_data@@@Z 10049bf8 f i libucrt:initialization.obj
 0001:00048bf8       ?initialize@?$dual_state_global@PAPA_W@__crt_state_management@@QAEXQAPA_W@Z 10049bf8 f i libucrt:environment_initialization.obj
 0001:00048bf8       ?initialize@?$dual_state_global@P6AXH@Z@__crt_state_management@@QAEXQ6AXH@Z@Z 10049bf8 f i libucrt:signal.obj
 0001:00048bf8       ?initialize@?$dual_state_global@PAPAD@__crt_state_management@@QAEXQAPAD@Z 10049bf8 f i libucrt:environment_initialization.obj
 0001:00048bf8       ?initialize@?$dual_state_global@P6AXPB_W00II@Z@__crt_state_management@@QAEXQ6AXPB_W00II@Z@Z 10049bf8 f i libucrt:invalid_parameter.obj
 0001:00048bf8       ?initialize@?$dual_state_global@P6AHI@Z@__crt_state_management@@QAEXQ6AHI@Z@Z 10049bf8 f i libucrt:new_handler.obj
 0001:00048bf8       ?initialize@?$dual_state_global@P6AHPAU_exception@@@Z@__crt_state_management@@QAEXQ6AHPAU_exception@@@Z@Z 10049bf8 f i libucrt:matherr.obj
 0001:00048c29       ___acrt_initialize_new_handler 10049c29 f   libucrt:new_handler.obj
 0001:00048c3d       __callnewh                 10049c3d f   libucrt:new_handler.obj
 0001:00048c81       __query_new_handler        10049c81 f   libucrt:new_handler.obj
 0001:00048cd3       ___acrt_has_user_matherr   10049cd3 f   libucrt:matherr.obj
 0001:00048cec       ___acrt_initialize_user_matherr 10049cec f   libucrt:matherr.obj
 0001:00048d00       ___acrt_invoke_user_matherr 10049d00 f   libucrt:matherr.obj
 0001:00048f66       ___acrt_LCMapStringA       10049f66 f   libucrt:lcmapstringa.obj
 0001:00048fb1       __query_new_mode           10049fb1 f   libucrt:new_mode.obj
 0001:00048fb7       __isleadbyte_l             10049fb7 f i libucrt:_wctype.obj
 0001:00048ff0       ___acrt_add_locale_ref     10049ff0 f   libucrt:locale_refcounting.obj
 0001:0004906d       ___acrt_free_locale        1004a06d f   libucrt:locale_refcounting.obj
 0001:000491b7       ___acrt_locale_add_lc_time_reference 1004a1b7 f   libucrt:locale_refcounting.obj
 0001:000491e0       ___acrt_locale_free_lc_time_if_unreferenced 1004a1e0 f   libucrt:locale_refcounting.obj
 0001:00049210       ___acrt_locale_release_lc_time_reference 1004a210 f   libucrt:locale_refcounting.obj
 0001:00049239       ___acrt_release_locale_ref 1004a239 f   libucrt:locale_refcounting.obj
 0001:000492ba       ___acrt_update_thread_locale_data 1004a2ba f   libucrt:locale_refcounting.obj
 0001:00049331       __updatetlocinfoEx_nolock  1004a331 f   libucrt:locale_refcounting.obj
 0001:00049381       ___acrt_fp_strflt_to_string 1004a381 f   libucrt:_fptostr.obj
 0001:0004943d       ??0scoped_fp_state_reset@?A0x48fbfdd4@@QAE@XZ 1004a43d f i libucrt:cfout.obj
 0001:00049467       ___acrt_fltout             1004a467 f   libucrt:cfout.obj
 0001:0004a803       __isatty                   1004b803 f   libucrt:isatty.obj
 0001:0004a859       ___acrt_locale_free_monetary 1004b859 f   libucrt:initmon.obj
 0001:0004a957       ___acrt_locale_free_numeric 1004b957 f   libucrt:initnum.obj
 0001:0004a9fc       ___acrt_locale_free_time   1004b9fc f   libucrt:inittime.obj
 0001:0004aae0       _wcsncmp                   1004bae0 f   libucrt:wcsncmp.obj
 0001:0004ab1a       ___acrt_GetStringTypeA     1004bb1a f   libucrt:getstringtypea.obj
 0001:0004ac37       ___acrt_lowio_create_handle_array 1004bc37 f   libucrt:osfinfo.obj
 0001:0004acb1       ___acrt_lowio_destroy_handle_array 1004bcb1 f   libucrt:osfinfo.obj
 0001:0004ace6       ___acrt_lowio_ensure_fh_exists 1004bce6 f   libucrt:osfinfo.obj
 0001:0004ad7e       ___acrt_lowio_lock_fh      1004bd7e f   libucrt:osfinfo.obj
 0001:0004ada1       ___acrt_lowio_set_os_handle 1004bda1 f   libucrt:osfinfo.obj
 0001:0004ae35       ___acrt_lowio_unlock_fh    1004be35 f   libucrt:osfinfo.obj
 0001:0004ae58       __alloc_osfhnd             1004be58 f   libucrt:osfinfo.obj
 0001:0004af6a       __free_osfhnd              1004bf6a f   libucrt:osfinfo.obj
 0001:0004affb       __get_osfhandle            1004bffb f   libucrt:osfinfo.obj
 0001:0004b065       __wcsnicmp                 1004c065 f   libucrt:wcsnicmp.obj
 0001:0004b11d       __wcsnicmp_l               1004c11d f   libucrt:wcsnicmp.obj
 0001:0004b2da       ___acrt_DownlevelLocaleNameToLCID 1004c2da f   libucrt:lcidtoname_downlevel.obj
 0001:0004b306       ___acrt_LCMapStringW       1004c306 f   libucrt:lcmapstringw.obj
 0001:0004b344       __msize                    1004c344 f   libucrt:msize.obj
 0001:0004b377       __realloc_base             1004c377 f   libucrt:realloc_base.obj
 0001:0004b3e0       ___acrt_copy_path_to_wide_string 1004c3e0 f   libucrt:string_utilities.obj
 0001:0004b4a7       __get_fmode                1004c4a7 f   libucrt:setmode.obj
 0001:0004b4d3       __setmode_nolock           1004c4d3 f   libucrt:setmode.obj
 0001:0004b5a4       __putwch_nolock            1004c5a4 f   libucrt:putwch.obj
 0001:0004b5e9       __chsize_nolock            1004c5e9 f   libucrt:chsize.obj
 0001:0004ba1d       __getfpcontrolword         1004ca1d f   libucrt:_fenvutils.obj
 0001:0004ba60       __getfpstatusword          1004ca60 f   libucrt:_fenvutils.obj
 0001:0004bb08       __setfpcontrolword         1004cb08 f   libucrt:_fenvutils.obj
 0001:0004bb88       __setfpstatusword          1004cb88 f   libucrt:_fenvutils.obj
 0001:0004bc08       ___acrt_CompareStringW     1004cc08 f   libucrt:comparestringw.obj
 0001:0004c0a8       ___acrt_pack_wide_command_line_and_environment 1004d0a8 f   libucrt:cenvarg.obj
 0001:0004c210       _qsort                     1004d210 f   libucrt:qsort.obj
 0001:0004c5aa       __mbsdec                   1004d5aa f   libucrt:mbsdec.obj
 0001:0004c5c1       __mbsdec_l                 1004d5c1 f   libucrt:mbsdec.obj
 0001:0004c65d       ___strncnt                 1004d65d f   libucrt:strncnt.obj
 0001:0004c679       _fegetenv                  1004d679 f   libucrt:fegetenv.obj
 0001:0004c696       _fesetenv                  1004d696 f   libucrt:fesetenv.obj
 0001:0004c6df       _feholdexcept              1004d6df f   libucrt:feholdexcept.obj
 0001:0004c730       _log10                     1004d730 f   libucrt:log10.obj
 0001:0004c770       __CIlog10                  1004d770 f   libucrt:log10.obj
 0001:0004c7ab       __CIlog10_default          1004d7ab f   libucrt:log10.obj
 0001:0004c7bf       __log10_default            1004d7bf     libucrt:log10.obj
 0001:0004c880       _ceil                      1004d880 f   libucrt:ceil_pentium4.obj
 0001:0004c8c0       __ceil_pentium4            1004d8c0 f   libucrt:ceil_pentium4.obj
 0001:0004c99d       __query_app_type           1004d99d f   libucrt:report_runtime_error.obj
 0001:0004c9b0       ___ascii_strnicmp          1004d9b0 f   libucrt:_strnicm.obj
 0001:0004ca11       ___dcrt_lowio_initialize_console_output 1004da11 f   libucrt:initcon.obj
 0001:0004ca30       ___dcrt_terminate_console_output 1004da30 f   libucrt:initcon.obj
 0001:0004ca47       ___acrt_initialize_sse2    1004da47 f   libucrt:mathfcns.obj
 0001:0004ca60       __CIlog10_pentium4         1004da60 f   libucrt:log10_pentium4.obj
 0001:0004ca78       __log10_pentium4           1004da78     libucrt:log10_pentium4.obj
 0001:0004cd01       __fFEXP                    1004dd01     libucrt:87tran.obj
 0001:0004cd58       __rtinfpopse               1004dd58     libucrt:87tran.obj
 0001:0004cd5a       __rtinfnpopse              1004dd5a     libucrt:87tran.obj
 0001:0004cd6a       __fFLN                     1004dd6a     libucrt:87tran.obj
 0001:0004ce1f       __rtinfpop                 1004de1f     libucrt:87tran.obj
 0001:0004ce21       __rtinfnpop                1004de21     libucrt:87tran.obj
 0001:0004ce3e       __ffexpm1                  1004de3e     libucrt:87tran.obj
 0001:0004cef0       __trandisp1                1004def0 f   libucrt:87disp.obj
 0001:0004cf57       __trandisp2                1004df57 f   libucrt:87disp.obj
 0001:0004cfe3       __rttospopde               1004dfe3     libucrt:87disp.obj
 0001:0004cfe8       __rttospop                 1004dfe8     libucrt:87disp.obj
 0001:0004cfea       __rtnospop                 1004dfea     libucrt:87disp.obj
 0001:0004cfec       __rttosnpop                1004dfec     libucrt:87disp.obj
 0001:0004cfed       __rtnospopde               1004dfed     libucrt:87disp.obj
 0001:0004cff4       __rtzeropop                1004dff4     libucrt:87disp.obj
 0001:0004cff6       __rtzeronpop               1004dff6     libucrt:87disp.obj
 0001:0004cffb       __rtzerospop               1004dffb     libucrt:87disp.obj
 0001:0004d008       __rtonepop                 1004e008     libucrt:87disp.obj
 0001:0004d00a       __rtonenpop                1004e00a     libucrt:87disp.obj
 0001:0004d00f       __tosnan1                  1004e00f     libucrt:87disp.obj
 0001:0004d03a       __nosnan2                  1004e03a     libucrt:87disp.obj
 0001:0004d03c       __tosnan2                  1004e03c     libucrt:87disp.obj
 0001:0004d064       __nan2                     1004e064     libucrt:87disp.obj
 0001:0004d0a3       __rtindfpop                1004e0a3     libucrt:87disp.obj
 0001:0004d0a5       __rtindfnpop               1004e0a5     libucrt:87disp.obj
 0001:0004d0b6       __rttosnpopde              1004e0b6     libucrt:87disp.obj
 0001:0004d0c0       __rtatan2inf               1004e0c0     libucrt:87disp.obj
 0001:0004d0dd       __rtchsifneg               1004e0dd     libucrt:87disp.obj
 0001:0004d0f0       __twoToTOS                 1004e0f0 f   libucrt:common.obj
 0001:0004d105       __load_CW                  1004e105 f   libucrt:common.obj
 0001:0004d11c       __convertTOStoQNaN         1004e11c f   libucrt:common.obj
 0001:0004d135       __fload_withFB             1004e135 f   libucrt:common.obj
 0001:0004d178       __checkTOS_withFB          1004e178 f   libucrt:common.obj
 0001:0004d18e       __fast_exit                1004e18e f   libucrt:common.obj
 0001:0004d19b       __math_exit                1004e19b f   libucrt:common.obj
 0001:0004d1c5       __check_overflow_exit      1004e1c5 f   libucrt:common.obj
 0001:0004d1d9       __check_range_exit         1004e1d9 f   libucrt:common.obj
 0001:0004d280       __startTwoArgErrorHandling 1004e280 f   libucrt:genexcep.obj
 0001:0004d297       __startOneArgErrorHandling 1004e297 f   libucrt:genexcep.obj
 0001:0004d2d3       ___libm_error_support      1004e2d3 f   libucrt:libm_error.obj
 0001:0004d4eb       __ceil_default             1004e4eb f   libucrt:ceil.obj
 0001:0004d5a4       __d_inttype                1004e5a4 f   libucrt:powhlp.obj
 0001:0004d60e       __powhlp                   1004e60e f   libucrt:powhlp.obj
 0001:0004d739       __87except                 1004e739 f   libucrt:87except.obj
 0001:0004d844       __frnd                     1004e844 f   libucrt:frnd.obj
 0001:0004d85a       __errcode                  1004e85a f   libucrt:fpexcept.obj
 0001:0004d88e       __except1                  1004e88e f   libucrt:fpexcept.obj
 0001:0004d95c       __handle_exc               1004e95c f   libucrt:fpexcept.obj
 0001:0004db3c       __raise_exc                1004eb3c f   libucrt:fpexcept.obj
 0001:0004db5f       __raise_exc_ex             1004eb5f f   libucrt:fpexcept.obj
 0001:0004de50       __set_errno_from_matherr   1004ee50 f   libucrt:fpexcept.obj
 0001:0004de7f       __umatherr                 1004ee7f f   libucrt:fpexcept.obj
 0001:0004df21       __decomp                   1004ef21 f   libucrt:util.obj
 0001:0004dff5       __set_exp                  1004eff5 f   libucrt:util.obj
 0001:0004e024       __sptype                   1004f024 f   libucrt:util.obj
 0001:0004e082       __fpclass                  1004f082 f   libucrt:ieeemisc.obj
 0001:0004e126       _IsProcessorFeaturePresent@4 1004f126 f   kernel32:KERNEL32.dll
 0001:0004e12c       _RtlUnwind@16              1004f12c f   kernel32:KERNEL32.dll
 0001:0004e140       __FindPESection            1004f140 f   LIBCMT:pesect.obj
 0001:0004e190       __IsNonwritableInCurrentImage 1004f190 f   LIBCMT:pesect.obj
 0001:0004e250       __ValidateImageBase        1004f250 f   LIBCMT:pesect.obj
 0001:0004e290       __aulldvrm                 1004f290 f   LIBCMT:ulldvrm.obj
 0001:0004e330       __SEH_prolog4_GS           1004f330 f   LIBCMT:_sehprolg4gs_.obj
 0001:0004e379       __SEH_epilog4_GS           1004f379 f   LIBCMT:_sehprolg4gs_.obj
 0001:0004e390       __alloca_probe_16          1004f390 f   LIBCMT:alloca16.obj
 0001:0004e3a6       __alloca_probe_8           1004f3a6     LIBCMT:alloca16.obj
 0001:0004e3c0       _memmove                   1004f3c0 f   libvcruntime:memmove.obj
 0002:00000000       _Keys                      10051000     flags.obj
 0002:00000b20       _VirtualKeyStrings         10051b20     service.obj
 0002:00007c90       __fltused                  10058c90     LIBCMT:fltused.obj
 0002:00007ca0       ___isa_enabled             10058ca0     LIBCMT:_cpu_disp_.obj
 0002:00007ca4       ___scrt_native_dllmain_reason 10058ca4     LIBCMT:utility.obj
 0002:00007cb0       ___security_cookie_complement 10058cb0     LIBCMT:gs_cookie.obj
 0002:00007cb4       ___security_cookie         10058cb4     LIBCMT:gs_cookie.obj
 0002:00007cd0       __NLG_Destination          10058cd0     libvcruntime:_exsup_.obj
 0002:00007ce8       __iob                      10058ce8     libucrt:_file.obj
 0002:00007d90       ___abort_behavior          10058d90     libucrt:abort.obj
 0002:00007d98       ___acrt_initial_locale_data 10058d98     libucrt:nlsdata.obj
 0002:00007e50       ___acrt_initial_locale_pointers 10058e50     libucrt:nlsdata.obj
 0002:00007e58       ___acrt_wide_c_locale_string 10058e58     libucrt:nlsdata.obj
 0002:00007e60       ___badioinfo               10058e60     libucrt:ioinit.obj
 0002:00007e98       __lookuptrailbytes         10058e98     libucrt:read.obj
 0002:00007f98       __pwctype                  10058f98     libucrt:ctype.obj
 0002:00008090       __mbctype                  10059090     libucrt:mbctype.obj
 0002:00008198       __mbcasemap                10059198     libucrt:mbctype.obj
 0002:00008298       ___acrt_initial_multibyte_data 10059298     libucrt:mbctype.obj
 0002:000084b8       ___acrt_current_multibyte_data 100594b8     libucrt:mbctype.obj
 0002:000084bc       ___globallocalestatus      100594bc     libucrt:glstatus.obj
 0002:000084c0       ___acrt_lconv_static_decimal 100594c0     libucrt:localeconv.obj
 0002:000084c4       ___acrt_lconv_static_W_decimal 100594c4     libucrt:localeconv.obj
 0002:000084c8       ___acrt_lconv_c            100594c8     libucrt:localeconv.obj
 0002:00008520       ___dcrt_lowio_console_output_handle 10059520     libucrt:initcon.obj
 0002:00008590       ___isa_available           10059590     LIBCMT:_cpu_disp_.obj
 0002:00008594       ___favor                   10059594     LIBCMT:_cpu_disp_.obj
 0002:00008598       ___scrt_current_native_startup_state 10059598     LIBCMT:utility.obj
 0002:0000859c       ___scrt_native_startup_lock 1005959c     LIBCMT:utility.obj
 0002:000085c0       ?__type_info_root_node@@3U__type_info_node@@A 100595c0     LIBCMT:tncleanup.obj
 0002:000085c8       ___scrt_debugger_hook_flag 100595c8     LIBCMT:utility_desktop.obj
 0002:00008964       ___pPurecall               10059964     libvcruntime:purevirt_data.obj
 0002:00008968       ?pArgList@UnDecorator@@0PAVReplicator@@A 10059968     libvcruntime:undname.obj
 0002:0000896c       ?pZNameList@UnDecorator@@0PAVReplicator@@A 1005996c     libvcruntime:undname.obj
 0002:00008970       ?pTemplateArgList@UnDecorator@@0PAVReplicator@@A 10059970     libvcruntime:undname.obj
 0002:00008974       ?gName@UnDecorator@@0PBDB  10059974     libvcruntime:undname.obj
 0002:00008978       ?name@UnDecorator@@0PBDB   10059978     libvcruntime:undname.obj
 0002:0000897c       ?outputString@UnDecorator@@0PADA 1005997c     libvcruntime:undname.obj
 0002:00008980       ?maxStringLength@UnDecorator@@0HA 10059980     libvcruntime:undname.obj
 0002:00008984       ?disableFlags@UnDecorator@@0KA 10059984     libvcruntime:undname.obj
 0002:00008988       ?fExplicitTemplateParams@UnDecorator@@0_NA 10059988     libvcruntime:undname.obj
 0002:00008989       ?fGetTemplateArgumentList@UnDecorator@@0_NA 10059989     libvcruntime:undname.obj
 0002:0000898c       ?m_pGetParameter@UnDecorator@@0P6APADJ@ZA 1005998c     libvcruntime:undname.obj
 0002:000089a4       __nstream                  100599a4     libucrt:_file.obj
 0002:000089a8       ___piob                    100599a8     libucrt:_file.obj
 0002:000089ac       __cflush                   100599ac     libucrt:_file.obj
 0002:00008ae8       __environ_table            10059ae8     libucrt:environment_initialization.obj
 0002:00008aec       __wenviron_table           10059aec     libucrt:environment_initialization.obj
 0002:00008af0       ___dcrt_initial_wide_environment 10059af0     libucrt:environment_initialization.obj
 0002:00008af4       ___dcrt_initial_narrow_environment 10059af4     libucrt:environment_initialization.obj
 0002:00008af8       ___acrt_atexit_table       10059af8     libucrt:onexit.obj
 0002:00008b04       ___acrt_at_quick_exit_table 10059b04     libucrt:onexit.obj
 0002:00008b18       ___acrt_stdout_buffer      10059b18     libucrt:_sftbuf.obj
 0002:00008b1c       ___acrt_stderr_buffer      10059b1c     libucrt:_sftbuf.obj
 0002:00008b20       ___acrt_locale_changed_data 10059b20     libucrt:wsetlocale.obj
 0002:00008b24       ___acrt_current_locale_data 10059b24     libucrt:nlsdata.obj
 0002:00008b28       ___pioinfo                 10059b28     libucrt:ioinit.obj
 0002:00008d28       __nhandle                  10059d28     libucrt:ioinit.obj
 0002:00008f54       __commode                  10059f54     libucrt:ncommode.obj
 0002:00008f58       ___mblocalename            10059f58     libucrt:mbctype.obj
 0002:00008f5c       ___mbcodepage              10059f5c     libucrt:mbctype.obj
 0002:00008f60       ___ismbcodepage            10059f60     libucrt:mbctype.obj
 0002:00008f64       ___mbulinfo                10059f64     libucrt:mbctype.obj
 0002:00008f78       ___argc                    10059f78     libucrt:argv_data.obj
 0002:00008f7c       ___argv                    10059f7c     libucrt:argv_data.obj
 0002:00008f80       ___wargv                   10059f80     libucrt:argv_data.obj
 0002:00008f84       __acmdln                   10059f84     libucrt:argv_data.obj
 0002:00008f88       __wcmdln                   10059f88     libucrt:argv_data.obj
 0002:00008f8c       __pgmptr                   10059f8c     libucrt:argv_data.obj
 0002:00008f90       ___acrt_heap               10059f90     libucrt:heap_handle.obj
 0002:00008fa0       ___acrt_lconv_static_null  10059fa0     libucrt:localeconv.obj
 0002:00008fa4       ___acrt_lconv_static_W_null 10059fa4     libucrt:localeconv.obj
 0002:00008fa8       __umaskval                 10059fa8     libucrt:umask.obj
 0002:00008fb0       __fmode                    10059fb0     libucrt:txtmode.obj
 0002:00008fb4       ___fastflag                10059fb4     libucrt:fp_flags.obj
 0002:00008fc0       _EnumCP                    10059fc0     <common>
 0002:00008fc8       ?_OptionsStorage@?1??__local_stdio_scanf_options@@9@9 10059fc8     <common>
 0002:00008fd0       ?_OptionsStorage@?1??__local_stdio_printf_options@@9@9 10059fd0     <common>
 0002:00008fd8       ___scrt_ucrt_dll_is_in_use 10059fd8     <common>
 0002:00008fdc       ___dyn_tls_init_callback   10059fdc     <common>
 0002:00008fe0       __pDestructExceptionObject 10059fe0     <common>
 0002:00008fe4       __pmatherr                 10059fe4     <common>
 0002:00008fe8       ___use_sse2_mathfcns       10059fe8     <common>
 0003:00000000       __imp__RegEnumKeyExW@32    1005a000     advapi32:ADVAPI32.dll
 0003:00000004       __imp__RegDeleteValueW@8   1005a004     advapi32:ADVAPI32.dll
 0003:00000008       __imp__RegDeleteKeyW@8     1005a008     advapi32:ADVAPI32.dll
 0003:0000000c       __imp__RegSetValueExW@24   1005a00c     advapi32:ADVAPI32.dll
 0003:00000010       __imp__RegQueryValueExW@24 1005a010     advapi32:ADVAPI32.dll
 0003:00000014       __imp__RegOpenKeyExW@20    1005a014     advapi32:ADVAPI32.dll
 0003:00000018       __imp__RegCreateKeyExW@36  1005a018     advapi32:ADVAPI32.dll
 0003:0000001c       __imp__RegCloseKey@4       1005a01c     advapi32:ADVAPI32.dll
 0003:00000020       __imp__RegEnumValueW@32    1005a020     advapi32:ADVAPI32.dll
 0003:00000024       \177ADVAPI32_NULL_THUNK_DATA 1005a024     advapi32:ADVAPI32.dll
 0003:00000028       __imp__GetConsoleScreenBufferInfo@8 1005a028     kernel32:KERNEL32.dll
 0003:0000002c       __imp__FreeLibrary@4       1005a02c     kernel32:KERNEL32.dll
 0003:00000030       __imp__GetModuleFileNameW@12 1005a030     kernel32:KERNEL32.dll
 0003:00000034       __imp__LoadLibraryW@4      1005a034     kernel32:KERNEL32.dll
 0003:00000038       __imp__SetCurrentDirectoryW@4 1005a038     kernel32:KERNEL32.dll
 0003:0000003c       __imp__GetCurrentDirectoryW@8 1005a03c     kernel32:KERNEL32.dll
 0003:00000040       __imp__SearchPathW@24      1005a040     kernel32:KERNEL32.dll
 0003:00000044       __imp__GetDriveTypeW@4     1005a044     kernel32:KERNEL32.dll
 0003:00000048       __imp__GetLogicalDriveStringsW@8 1005a048     kernel32:KERNEL32.dll
 0003:0000004c       __imp__SetFileAttributesW@8 1005a04c     kernel32:KERNEL32.dll
 0003:00000050       __imp__OutputDebugStringW@4 1005a050     kernel32:KERNEL32.dll
 0003:00000054       __imp__GetLastError@0      1005a054     kernel32:KERNEL32.dll
 0003:00000058       __imp__Sleep@4             1005a058     kernel32:KERNEL32.dll
 0003:0000005c       __imp__GlobalMemoryStatusEx@4 1005a05c     kernel32:KERNEL32.dll
 0003:00000060       __imp__FormatMessageW@28   1005a060     kernel32:KERNEL32.dll
 0003:00000064       __imp__MultiByteToWideChar@24 1005a064     kernel32:KERNEL32.dll
 0003:00000068       __imp__WideCharToMultiByte@32 1005a068     kernel32:KERNEL32.dll
 0003:0000006c       __imp__GetACP@0            1005a06c     kernel32:KERNEL32.dll
 0003:00000070       __imp__GetOEMCP@0          1005a070     kernel32:KERNEL32.dll
 0003:00000074       __imp__GetCPInfoExW@12     1005a074     kernel32:KERNEL32.dll
 0003:00000078       __imp__GetProcAddress@8    1005a078     kernel32:KERNEL32.dll
 0003:0000007c       __imp__SetEnvironmentVariableW@8 1005a07c     kernel32:KERNEL32.dll
 0003:00000080       __imp__CreateDirectoryW@8  1005a080     kernel32:KERNEL32.dll
 0003:00000084       __imp__DeleteFileW@4       1005a084     kernel32:KERNEL32.dll
 0003:00000088       __imp__FileTimeToLocalFileTime@8 1005a088     kernel32:KERNEL32.dll
 0003:0000008c       __imp__FindClose@4         1005a08c     kernel32:KERNEL32.dll
 0003:00000090       __imp__FindFirstFileW@8    1005a090     kernel32:KERNEL32.dll
 0003:00000094       __imp__RemoveDirectoryW@4  1005a094     kernel32:KERNEL32.dll
 0003:00000098       __imp__GetSystemTimeAsFileTime@4 1005a098     kernel32:KERNEL32.dll
 0003:0000009c       __imp__GetModuleHandleW@4  1005a09c     kernel32:KERNEL32.dll
 0003:000000a0       __imp__CopyFileW@12        1005a0a0     kernel32:KERNEL32.dll
 0003:000000a4       __imp__MoveFileExW@12      1005a0a4     kernel32:KERNEL32.dll
 0003:000000a8       __imp__FileTimeToSystemTime@8 1005a0a8     kernel32:KERNEL32.dll
 0003:000000ac       __imp__SystemTimeToFileTime@8 1005a0ac     kernel32:KERNEL32.dll
 0003:000000b0       __imp__CompareStringW@24   1005a0b0     kernel32:KERNEL32.dll
 0003:000000b4       __imp__PeekConsoleInputW@16 1005a0b4     kernel32:KERNEL32.dll
 0003:000000b8       __imp__ReadConsoleInputW@16 1005a0b8     kernel32:KERNEL32.dll
 0003:000000bc       __imp__SetLastError@4      1005a0bc     kernel32:KERNEL32.dll
 0003:000000c0       __imp__GetModuleHandleA@4  1005a0c0     kernel32:KERNEL32.dll
 0003:000000c4       __imp__DeleteTimerQueueTimer@12 1005a0c4     kernel32:KERNEL32.dll
 0003:000000c8       __imp__ChangeTimerQueueTimer@16 1005a0c8     kernel32:KERNEL32.dll
 0003:000000cc       __imp__CreateTimerQueueTimer@28 1005a0cc     kernel32:KERNEL32.dll
 0003:000000d0       __imp__CreateTimerQueue@0  1005a0d0     kernel32:KERNEL32.dll
 0003:000000d4       __imp__GetFileAttributesW@4 1005a0d4     kernel32:KERNEL32.dll
 0003:000000d8       __imp__GetEnvironmentVariableW@12 1005a0d8     kernel32:KERNEL32.dll
 0003:000000dc       __imp__GetStdHandle@4      1005a0dc     kernel32:KERNEL32.dll
 0003:000000e0       __imp__EnumSystemCodePagesW@8 1005a0e0     kernel32:KERNEL32.dll
 0003:000000e4       __imp__DeleteTimerQueueEx@8 1005a0e4     kernel32:KERNEL32.dll
 0003:000000e8       __imp__SetEndOfFile@4      1005a0e8     kernel32:KERNEL32.dll
 0003:000000ec       __imp__WriteConsoleW@20    1005a0ec     kernel32:KERNEL32.dll
 0003:000000f0       __imp__HeapReAlloc@16      1005a0f0     kernel32:KERNEL32.dll
 0003:000000f4       __imp__HeapSize@12         1005a0f4     kernel32:KERNEL32.dll
 0003:000000f8       __imp__SetStdHandle@8      1005a0f8     kernel32:KERNEL32.dll
 0003:000000fc       __imp__GetProcessHeap@0    1005a0fc     kernel32:KERNEL32.dll
 0003:00000100       __imp__FreeEnvironmentStringsW@4 1005a100     kernel32:KERNEL32.dll
 0003:00000104       __imp__GetEnvironmentStringsW@0 1005a104     kernel32:KERNEL32.dll
 0003:00000108       __imp__GetCommandLineW@0   1005a108     kernel32:KERNEL32.dll
 0003:0000010c       __imp__GetCommandLineA@0   1005a10c     kernel32:KERNEL32.dll
 0003:00000110       __imp__GetCPInfo@8         1005a110     kernel32:KERNEL32.dll
 0003:00000114       __imp__IsValidCodePage@4   1005a114     kernel32:KERNEL32.dll
 0003:00000118       __imp__FindNextFileA@8     1005a118     kernel32:KERNEL32.dll
 0003:0000011c       __imp__FindFirstFileExA@24 1005a11c     kernel32:KERNEL32.dll
 0003:00000120       __imp__CreateFileW@28      1005a120     kernel32:KERNEL32.dll
 0003:00000124       __imp__GetConsoleCP@0      1005a124     kernel32:KERNEL32.dll
 0003:00000128       __imp__WriteFile@20        1005a128     kernel32:KERNEL32.dll
 0003:0000012c       __imp__FlushFileBuffers@4  1005a12c     kernel32:KERNEL32.dll
 0003:00000130       __imp__CreatePipe@16       1005a130     kernel32:KERNEL32.dll
 0003:00000134       __imp__GetFileAttributesExW@12 1005a134     kernel32:KERNEL32.dll
 0003:00000138       __imp__GetExitCodeProcess@8 1005a138     kernel32:KERNEL32.dll
 0003:0000013c       __imp__WaitForSingleObject@8 1005a13c     kernel32:KERNEL32.dll
 0003:00000140       __imp__SetFilePointerEx@20 1005a140     kernel32:KERNEL32.dll
 0003:00000144       __imp__ReadConsoleW@20     1005a144     kernel32:KERNEL32.dll
 0003:00000148       __imp__GetConsoleMode@8    1005a148     kernel32:KERNEL32.dll
 0003:0000014c       __imp__LCMapStringW@24     1005a14c     kernel32:KERNEL32.dll
 0003:00000150       __imp__GetFileType@4       1005a150     kernel32:KERNEL32.dll
 0003:00000154       __imp__HeapAlloc@12        1005a154     kernel32:KERNEL32.dll
 0003:00000158       __imp__HeapFree@12         1005a158     kernel32:KERNEL32.dll
 0003:0000015c       __imp__GetModuleFileNameA@12 1005a15c     kernel32:KERNEL32.dll
 0003:00000160       __imp__ExitProcess@4       1005a160     kernel32:KERNEL32.dll
 0003:00000164       __imp__GetTempPathW@8      1005a164     kernel32:KERNEL32.dll
 0003:00000168       __imp__ReadFile@20         1005a168     kernel32:KERNEL32.dll
 0003:0000016c       __imp__CreateProcessW@40   1005a16c     kernel32:KERNEL32.dll
 0003:00000170       __imp__DuplicateHandle@28  1005a170     kernel32:KERNEL32.dll
 0003:00000174       __imp__CloseHandle@4       1005a174     kernel32:KERNEL32.dll
 0003:00000178       __imp__GetStringTypeW@16   1005a178     kernel32:KERNEL32.dll
 0003:0000017c       __imp__LoadLibraryExW@12   1005a17c     kernel32:KERNEL32.dll
 0003:00000180       __imp__TlsFree@4           1005a180     kernel32:KERNEL32.dll
 0003:00000184       __imp__TlsSetValue@8       1005a184     kernel32:KERNEL32.dll
 0003:00000188       __imp__TlsGetValue@4       1005a188     kernel32:KERNEL32.dll
 0003:0000018c       __imp__RaiseException@16   1005a18c     kernel32:KERNEL32.dll
 0003:00000190       __imp__TlsAlloc@0          1005a190     kernel32:KERNEL32.dll
 0003:00000194       __imp__InitializeCriticalSectionAndSpinCount@8 1005a194     kernel32:KERNEL32.dll
 0003:00000198       __imp__DeleteCriticalSection@4 1005a198     kernel32:KERNEL32.dll
 0003:0000019c       __imp__LeaveCriticalSection@4 1005a19c     kernel32:KERNEL32.dll
 0003:000001a0       __imp__EnterCriticalSection@4 1005a1a0     kernel32:KERNEL32.dll
 0003:000001a4       __imp__RtlUnwind@16        1005a1a4     kernel32:KERNEL32.dll
 0003:000001a8       __imp__TerminateProcess@8  1005a1a8     kernel32:KERNEL32.dll
 0003:000001ac       __imp__GetCurrentProcess@0 1005a1ac     kernel32:KERNEL32.dll
 0003:000001b0       __imp__GetStartupInfoW@4   1005a1b0     kernel32:KERNEL32.dll
 0003:000001b4       __imp__SetUnhandledExceptionFilter@4 1005a1b4     kernel32:KERNEL32.dll
 0003:000001b8       __imp__UnhandledExceptionFilter@4 1005a1b8     kernel32:KERNEL32.dll
 0003:000001bc       __imp__IsDebuggerPresent@0 1005a1bc     kernel32:KERNEL32.dll
 0003:000001c0       __imp__GetCurrentThreadId@0 1005a1c0     kernel32:KERNEL32.dll
 0003:000001c4       __imp__GetCurrentProcessId@0 1005a1c4     kernel32:KERNEL32.dll
 0003:000001c8       __imp__QueryPerformanceCounter@4 1005a1c8     kernel32:KERNEL32.dll
 0003:000001cc       __imp__IsProcessorFeaturePresent@4 1005a1cc     kernel32:KERNEL32.dll
 0003:000001d0       \177KERNEL32_NULL_THUNK_DATA 1005a1d0     kernel32:KERNEL32.dll
 0003:000001d4       __imp__RpcStringFreeA@4    1005a1d4     rpcrt4:RPCRT4.dll
 0003:000001d8       __imp__UuidCreate@4        1005a1d8     rpcrt4:RPCRT4.dll
 0003:000001dc       __imp__UuidToStringA@8     1005a1dc     rpcrt4:RPCRT4.dll
 0003:000001e0       __imp__UuidFromStringA@8   1005a1e0     rpcrt4:RPCRT4.dll
 0003:000001e4       \177RPCRT4_NULL_THUNK_DATA 1005a1e4     rpcrt4:RPCRT4.dll
 0003:000001e8       __imp__ShellExecuteW@24    1005a1e8     shell32:SHELL32.dll
 0003:000001ec       __imp__SHGetFolderPathW@20 1005a1ec     shell32:SHELL32.dll
 0003:000001f0       \177SHELL32_NULL_THUNK_DATA 1005a1f0     shell32:SHELL32.dll
 0003:000001f4       __imp__GetKeyState@4       1005a1f4     user32:USER32.dll
 0003:000001f8       \177USER32_NULL_THUNK_DATA 1005a1f8     user32:USER32.dll
 0003:000001fc       __imp__lua_typename        1005a1fc     lua51:lua51.dll
 0003:00000200       __imp__lua_dump            1005a200     lua51:lua51.dll
 0003:00000204       __imp__luaL_checkstack     1005a204     lua51:lua51.dll
 0003:00000208       __imp__luaL_prepbuffer     1005a208     lua51:lua51.dll
 0003:0000020c       __imp__lua_tocfunction     1005a20c     lua51:lua51.dll
 0003:00000210       __imp__luaL_checkoption    1005a210     lua51:lua51.dll
 0003:00000214       __imp__lua_iscfunction     1005a214     lua51:lua51.dll
 0003:00000218       __imp__luaL_gsub           1005a218     lua51:lua51.dll
 0003:0000021c       __imp__luaL_findtable      1005a21c     lua51:lua51.dll
 0003:00000220       __imp__lua_isuserdata      1005a220     lua51:lua51.dll
 0003:00000224       __imp__luaL_checkany       1005a224     lua51:lua51.dll
 0003:00000228       __imp__luaL_optnumber      1005a228     lua51:lua51.dll
 0003:0000022c       __imp__luaL_checknumber    1005a22c     lua51:lua51.dll
 0003:00000230       __imp__luaL_typerror       1005a230     lua51:lua51.dll
 0003:00000234       __imp__lua_setallocf       1005a234     lua51:lua51.dll
 0003:00000238       __imp__lua_getfenv         1005a238     lua51:lua51.dll
 0003:0000023c       __imp__lua_rawget          1005a23c     lua51:lua51.dll
 0003:00000240       __imp__luaopen_debug       1005a240     lua51:lua51.dll
 0003:00000244       __imp__luaopen_math        1005a244     lua51:lua51.dll
 0003:00000248       __imp__luaopen_string      1005a248     lua51:lua51.dll
 0003:0000024c       __imp__luaopen_os          1005a24c     lua51:lua51.dll
 0003:00000250       __imp__luaopen_table       1005a250     lua51:lua51.dll
 0003:00000254       __imp__luaopen_base        1005a254     lua51:lua51.dll
 0003:00000258       __imp__luaL_checktype      1005a258     lua51:lua51.dll
 0003:0000025c       __imp__lua_getinfo         1005a25c     lua51:lua51.dll
 0003:00000260       __imp__lua_getstack        1005a260     lua51:lua51.dll
 0003:00000264       __imp__luaL_addvalue       1005a264     lua51:lua51.dll
 0003:00000268       __imp__luaL_error          1005a268     lua51:lua51.dll
 0003:0000026c       __imp__luaL_checkudata     1005a26c     lua51:lua51.dll
 0003:00000270       __imp__luaL_optinteger     1005a270     lua51:lua51.dll
 0003:00000274       __imp__luaL_optlstring     1005a274     lua51:lua51.dll
 0003:00000278       __imp__lua_checkstack      1005a278     lua51:lua51.dll
 0003:0000027c       __imp__lua_replace         1005a27c     lua51:lua51.dll
 0003:00000280       __imp__luaL_pushresult     1005a280     lua51:lua51.dll
 0003:00000284       __imp__luaL_addlstring     1005a284     lua51:lua51.dll
 0003:00000288       __imp__luaL_buffinit       1005a288     lua51:lua51.dll
 0003:0000028c       __imp__lua_concat          1005a28c     lua51:lua51.dll
 0003:00000290       __imp__lua_getallocf       1005a290     lua51:lua51.dll
 0003:00000294       __imp__lua_load            1005a294     lua51:lua51.dll
 0003:00000298       __imp__lua_pushfstring     1005a298     lua51:lua51.dll
 0003:0000029c       __imp__luaL_loadstring     1005a29c     lua51:lua51.dll
 0003:000002a0       __imp__luaL_unref          1005a2a0     lua51:lua51.dll
 0003:000002a4       __imp__luaL_ref            1005a2a4     lua51:lua51.dll
 0003:000002a8       __imp__lua_gc              1005a2a8     lua51:lua51.dll
 0003:000002ac       __imp__lua_pcall           1005a2ac     lua51:lua51.dll
 0003:000002b0       __imp__lua_call            1005a2b0     lua51:lua51.dll
 0003:000002b4       __imp__lua_rawseti         1005a2b4     lua51:lua51.dll
 0003:000002b8       __imp__lua_setfield        1005a2b8     lua51:lua51.dll
 0003:000002bc       __imp__lua_createtable     1005a2bc     lua51:lua51.dll
 0003:000002c0       __imp__lua_rawgeti         1005a2c0     lua51:lua51.dll
 0003:000002c4       __imp__lua_gettable        1005a2c4     lua51:lua51.dll
 0003:000002c8       __imp__lua_pushlightuserdata 1005a2c8     lua51:lua51.dll
 0003:000002cc       __imp__lua_pushcclosure    1005a2cc     lua51:lua51.dll
 0003:000002d0       __imp__lua_pushlstring     1005a2d0     lua51:lua51.dll
 0003:000002d4       __imp__lua_pushinteger     1005a2d4     lua51:lua51.dll
 0003:000002d8       __imp__lua_objlen          1005a2d8     lua51:lua51.dll
 0003:000002dc       __imp__lua_toboolean       1005a2dc     lua51:lua51.dll
 0003:000002e0       __imp__lua_tointeger       1005a2e0     lua51:lua51.dll
 0003:000002e4       __imp__lua_isstring        1005a2e4     lua51:lua51.dll
 0003:000002e8       __imp__lua_isnumber        1005a2e8     lua51:lua51.dll
 0003:000002ec       __imp__lua_insert          1005a2ec     lua51:lua51.dll
 0003:000002f0       __imp__lua_remove          1005a2f0     lua51:lua51.dll
 0003:000002f4       __imp__lua_pushvalue       1005a2f4     lua51:lua51.dll
 0003:000002f8       __imp__luaL_newmetatable   1005a2f8     lua51:lua51.dll
 0003:000002fc       __imp__luaL_checkinteger   1005a2fc     lua51:lua51.dll
 0003:00000300       __imp__luaL_argerror       1005a300     lua51:lua51.dll
 0003:00000304       __imp__luaL_register       1005a304     lua51:lua51.dll
 0003:00000308       __imp__lua_setmetatable    1005a308     lua51:lua51.dll
 0003:0000030c       __imp__lua_getmetatable    1005a30c     lua51:lua51.dll
 0003:00000310       __imp__lua_newuserdata     1005a310     lua51:lua51.dll
 0003:00000314       __imp__lua_getfield        1005a314     lua51:lua51.dll
 0003:00000318       __imp__lua_pushboolean     1005a318     lua51:lua51.dll
 0003:0000031c       __imp__lua_pushstring      1005a31c     lua51:lua51.dll
 0003:00000320       __imp__lua_pushnumber      1005a320     lua51:lua51.dll
 0003:00000324       __imp__lua_pushnil         1005a324     lua51:lua51.dll
 0003:00000328       __imp__lua_touserdata      1005a328     lua51:lua51.dll
 0003:0000032c       __imp__lua_tolstring       1005a32c     lua51:lua51.dll
 0003:00000330       __imp__lua_tonumber        1005a330     lua51:lua51.dll
 0003:00000334       __imp__lua_rawequal        1005a334     lua51:lua51.dll
 0003:00000338       __imp__lua_type            1005a338     lua51:lua51.dll
 0003:0000033c       __imp__lua_settop          1005a33c     lua51:lua51.dll
 0003:00000340       __imp__lua_gettop          1005a340     lua51:lua51.dll
 0003:00000344       __imp__lua_next            1005a344     lua51:lua51.dll
 0003:00000348       __imp__lua_setfenv         1005a348     lua51:lua51.dll
 0003:0000034c       __imp__lua_rawset          1005a34c     lua51:lua51.dll
 0003:00000350       __imp__lua_error           1005a350     lua51:lua51.dll
 0003:00000354       __imp__lua_settable        1005a354     lua51:lua51.dll
 0003:00000358       __imp__luaL_checklstring   1005a358     lua51:lua51.dll
 0003:0000035c       \177lua51_NULL_THUNK_DATA  1005a35c     lua51:lua51.dll
 0003:00000360       ___guard_check_icall_fptr  1005a360     LIBCMT:guard_support.obj
 0003:00000364       __IMPORT_DESCRIPTOR_KERNEL32 1005a364     kernel32:KERNEL32.dll
 0003:00000378       __IMPORT_DESCRIPTOR_USER32 1005a378     user32:USER32.dll
 0003:0000038c       __IMPORT_DESCRIPTOR_ADVAPI32 1005a38c     advapi32:ADVAPI32.dll
 0003:000003a0       __IMPORT_DESCRIPTOR_SHELL32 1005a3a0     shell32:SHELL32.dll
 0003:000003b4       __IMPORT_DESCRIPTOR_lua51  1005a3b4     lua51:lua51.dll
 0003:000003c8       __IMPORT_DESCRIPTOR_RPCRT4 1005a3c8     rpcrt4:RPCRT4.dll
 0003:000003dc       __NULL_IMPORT_DESCRIPTOR   1005a3dc     kernel32:KERNEL32.dll

 entry point at        0001:00032357

 Static symbols

 0001:00000050       _funcs                     10001050     bit64.obj
 0001:000000e0       _metamethods               100010e0     bit64.obj
 0001:00000210       _FHELP_NOSHOWERROR         10001210     exported.obj
 0001:00000218       _FHELP_SELFHELP            10001218     exported.obj
 0001:00000220       _FHELP_FARHELP             10001220     exported.obj
 0001:00000228       _FHELP_CUSTOMFILE          10001228     exported.obj
 0001:00000230       _FHELP_CUSTOMPATH          10001230     exported.obj
 0001:00000238       _FHELP_GUID                10001238     exported.obj
 0001:00000240       _FHELP_USECONTENTS         10001240     exported.obj
 0001:00000248       _FHELP_NONE                10001248     exported.obj
 0001:00000250       _FFFS_COMMAS               10001250     exported.obj
 0001:00000258       _FFFS_FLOATSIZE            10001258     exported.obj
 0001:00000260       _FFFS_SHOWBYTESINDEX       10001260     exported.obj
 0001:00000268       _FFFS_ECONOMIC             10001268     exported.obj
 0001:00000270       _FFFS_THOUSAND             10001270     exported.obj
 0001:00000278       _FFFS_MINSIZEINDEX         10001278     exported.obj
 0001:00000280       _FFFS_MINSIZEINDEX_MASK    10001280     exported.obj
 0001:00000288       _FFFS_NONE                 10001288     exported.obj
 0001:00000290       _KMFLAGS_SILENTCHECK       10001290     exported.obj
 0001:00000298       _KMFLAGS_NOSENDKEYSTOPLUGINS 10001298     exported.obj
 0001:000002a0       _KMFLAGS_ENABLEOUTPUT      100012a0     exported.obj
 0001:000002a8       _KMFLAGS_LANGMASK          100012a8     exported.obj
 0001:000002b0       _KMFLAGS_LUA               100012b0     exported.obj
 0001:000002b8       _KMFLAGS_MOONSCRIPT        100012b8     exported.obj
 0001:000002c0       _KMFLAGS_NONE              100012c0     exported.obj
 0001:000002c8       _AKMFLAGS_NONE             100012c8     exported.obj
 0001:000002d0       _FSETCLR_REDRAW            100012d0     exported.obj
 0001:000002d8       _FSETCLR_NONE              100012d8     exported.obj
 0001:000002e0       _WIF_MODIFIED              100012e0     exported.obj
 0001:000002e8       _WIF_CURRENT               100012e8     exported.obj
 0001:000002f0       _WIF_MODAL                 100012f0     exported.obj
 0001:000002f8       _WIF_NONE                  100012f8     exported.obj
 0001:00000300       _PF_PRELOAD                10001300     exported.obj
 0001:00000308       _PF_DISABLEPANELS          10001308     exported.obj
 0001:00000310       _PF_EDITOR                 10001310     exported.obj
 0001:00000318       _PF_VIEWER                 10001318     exported.obj
 0001:00000320       _PF_FULLCMDLINE            10001320     exported.obj
 0001:00000328       _PF_DIALOG                 10001328     exported.obj
 0001:00000330       _PF_NONE                   10001330     exported.obj
 0001:00000338       _VOPT_SAVEFILEPOSITION     10001338     exported.obj
 0001:00000340       _VOPT_AUTODETECTCODEPAGE   10001340     exported.obj
 0001:00000348       _VOPT_SHOWTITLEBAR         10001348     exported.obj
 0001:00000350       _VOPT_SHOWKEYBAR           10001350     exported.obj
 0001:00000358       _VOPT_SHOWSCROLLBAR        10001358     exported.obj
 0001:00000360       _VOPT_QUICKVIEW            10001360     exported.obj
 0001:00000368       _VOPT_NONE                 10001368     exported.obj
 0001:00000370       _VSMFL_REDRAW              10001370     exported.obj
 0001:00000378       _VSMFL_NONE                10001378     exported.obj
 0001:00000380       _VSP_NOREDRAW              10001380     exported.obj
 0001:00000388       _VSP_PERCENT               10001388     exported.obj
 0001:00000390       _VSP_RELATIVE              10001390     exported.obj
 0001:00000398       _VSP_NORETNEWPOS           10001398     exported.obj
 0001:000003a0       _VSP_NONE                  100013a0     exported.obj
 0001:000003a8       _IPLFLAGS_SEPARATOR        100013a8     exported.obj
 0001:000003b0       _IPLFLAGS_NONE             100013b0     exported.obj
 0001:000003b8       _VMF_WRAP                  100013b8     exported.obj
 0001:000003c0       _PMFLAGS_FULLSCREEN        100013c0     exported.obj
 0001:000003c8       _VMF_WORDWRAP              100013c8     exported.obj
 0001:000003d0       _VMF_NONE                  100013d0     exported.obj
 0001:000003d8       _PMFLAGS_DETAILEDSTATUS    100013d8     exported.obj
 0001:000003e0       _PMFLAGS_ALIGNEXTENSIONS   100013e0     exported.obj
 0001:000003e8       _PMFLAGS_CASECONVERSION    100013e8     exported.obj
 0001:000003f0       _PMFLAGS_NONE              100013f0     exported.obj
 0001:000003f8       _FCF_FG_4BIT               100013f8     exported.obj
 0001:00000400       _FCF_BG_4BIT               10001400     exported.obj
 0001:00000408       _FCF_4BITMASK              10001408     exported.obj
 0001:00000410       _FCF_RAWATTR_MASK          10001410     exported.obj
 0001:00000418       _FCF_EXTENDEDFLAGS         10001418     exported.obj
 0001:00000420       _FCF_FG_BOLD               10001420     exported.obj
 0001:00000428       _FCF_FG_ITALIC             10001428     exported.obj
 0001:00000430       _FCF_FG_UNDERLINE          10001430     exported.obj
 0001:00000438       _FCF_STYLEMASK             10001438     exported.obj
 0001:00000440       _OPIF_DISABLEFILTER        10001440     exported.obj
 0001:00000448       _FCF_NONE                  10001448     exported.obj
 0001:00000450       _OPIF_DISABLESORTGROUPS    10001450     exported.obj
 0001:00000458       _OPIF_DISABLEHIGHLIGHTING  10001458     exported.obj
 0001:00000460       _OPIF_ADDDOTS              10001460     exported.obj
 0001:00000468       _OPIF_RAWSELECTION         10001468     exported.obj
 0001:00000470       _OPIF_REALNAMES            10001470     exported.obj
 0001:00000478       _OPIF_SHOWNAMESONLY        10001478     exported.obj
 0001:00000480       _OPIF_SHOWRIGHTALIGNNAMES  10001480     exported.obj
 0001:00000488       _OPIF_SHOWPRESERVECASE     10001488     exported.obj
 0001:00000490       _OPIF_COMPAREFATTIME       10001490     exported.obj
 0001:00000498       _OPIF_EXTERNALGET          10001498     exported.obj
 0001:000004a0       _OPIF_EXTERNALPUT          100014a0     exported.obj
 0001:000004a8       _OPIF_EXTERNALDELETE       100014a8     exported.obj
 0001:000004b0       _OPIF_EXTERNALMKDIR        100014b0     exported.obj
 0001:000004b8       _OPIF_USEATTRHIGHLIGHTING  100014b8     exported.obj
 0001:000004c0       _OPIF_USECRC32             100014c0     exported.obj
 0001:000004c8       _OPIF_USEFREESIZE          100014c8     exported.obj
 0001:000004d0       _OPIF_SHORTCUT             100014d0     exported.obj
 0001:000004d8       _OPIF_NONE                 100014d8     exported.obj
 0001:000004e0       _CDF_NONE                  100014e0     exported.obj
 0001:000004e8       _FMSG_WARNING              100014e8     exported.obj
 0001:000004f0       _FMSG_ERRORTYPE            100014f0     exported.obj
 0001:00000524       _PDF_DIALOGEVENTDRAWENABLE 10001524     exported.obj
 0001:00000528       _FMSG_KEEPBACKGROUND       10001528     exported.obj
 0001:00000530       _OPM_SILENT                10001530     exported.obj
 0001:00000550       _OPM_FIND                  10001550     exported.obj
 0001:00000558       _FMSG_LEFTALIGN            10001558     exported.obj
 0001:00000560       _FMSG_ALLINONE             10001560     exported.obj
 0001:00000570       _OPM_VIEW                  10001570     exported.obj
 0001:00000578       _OPM_EDIT                  10001578     exported.obj
 0001:00000580       _FMSG_MB_OK                10001580     exported.obj
 0001:00000588       _FMSG_MB_OKCANCEL          10001588     exported.obj
 0001:00000590       _OPM_TOPLEVEL              10001590     exported.obj
 0001:00000598       _OPM_DESCR                 10001598     exported.obj
 0001:000005a0       _FMSG_MB_ABORTRETRYIGNORE  100015a0     exported.obj
 0001:000005a8       _OPM_QUICKVIEW             100015a8     exported.obj
 0001:000005b0       _FMSG_MB_YESNO             100015b0     exported.obj
 0001:000005b8       _OPM_PGDN                  100015b8     exported.obj
 0001:000005c0       _FMSG_MB_YESNOCANCEL       100015c0     exported.obj
 0001:000005c8       _FMSG_MB_RETRYCANCEL       100015c8     exported.obj
 0001:000005d0       _OPM_COMMANDS              100015d0     exported.obj
 0001:000005d8       _OPM_NONE                  100015d8     exported.obj
 0001:000005e0       _FMSG_NONE                 100015e0     exported.obj
 0001:000005e8       _FOSF_ACTIVE               100015e8     exported.obj
 0001:000005f0       _DIF_BOXCOLOR              100015f0     exported.obj
 0001:000005f8       _FOSF_NONE                 100015f8     exported.obj
 0001:00000600       _DIF_GROUP                 10001600     exported.obj
 0001:00000608       _DIF_LEFTTEXT              10001608     exported.obj
 0001:00000610       _DIF_MOVESELECT            10001610     exported.obj
 0001:00000618       _DIF_SHOWAMPERSAND         10001618     exported.obj
 0001:00000620       _DIF_CENTERGROUP           10001620     exported.obj
 0001:00000628       _DIF_NOBRACKETS            10001628     exported.obj
 0001:00000630       _DIF_MANUALADDHISTORY      10001630     exported.obj
 0001:00000638       _DIF_SEPARATOR             10001638     exported.obj
 0001:00000640       _DIF_SEPARATOR2            10001640     exported.obj
 0001:00000648       _DIF_EDITOR                10001648     exported.obj
 0001:00000650       _DIF_LISTNOAMPERSAND       10001650     exported.obj
 0001:00000658       _DIF_LISTNOBOX             10001658     exported.obj
 0001:00000660       _DIF_HISTORY               10001660     exported.obj
 0001:00000668       _DIF_BTNNOCLOSE            10001668     exported.obj
 0001:00000670       _DIF_CENTERTEXT            10001670     exported.obj
 0001:00000678       _PDF_PROCESSINGERROR       10001678     exported.obj
 0001:00000680       _DIF_SEPARATORUSER         10001680     exported.obj
 0001:00000688       _DIF_SETSHIELD             10001688     exported.obj
 0001:00000690       _DIF_EDITEXPAND            10001690     exported.obj
 0001:00000698       _DIF_DROPDOWNLIST          10001698     exported.obj
 0001:000006a0       _DIF_USELASTHISTORY        100016a0     exported.obj
 0001:000006a8       _DIF_MASKEDIT              100016a8     exported.obj
 0001:000006b0       _DIF_LISTTRACKMOUSE        100016b0     exported.obj
 0001:000006b8       _DIF_LISTTRACKMOUSEINFOCUS 100016b8     exported.obj
 0001:000006c0       _DIF_SELECTONENTRY         100016c0     exported.obj
 0001:000006c8       _DIF_3STATE                100016c8     exported.obj
 0001:000006d0       _DIF_EDITPATH              100016d0     exported.obj
 0001:000006d8       _DIF_LISTWRAPMODE          100016d8     exported.obj
 0001:000006e0       _DIF_NOAUTOCOMPLETE        100016e0     exported.obj
 0001:000006e8       _DIF_LISTAUTOHIGHLIGHT     100016e8     exported.obj
 0001:000006f0       _DIF_LISTNOCLOSE           100016f0     exported.obj
 0001:000006f8       _DIF_EDITPATHEXEC          100016f8     exported.obj
 0001:00000700       _DIF_HIDDEN                10001700     exported.obj
 0001:00000708       _DIF_READONLY              10001708     exported.obj
 0001:00000710       _DIF_NOFOCUS               10001710     exported.obj
 0001:00000718       _DIF_DISABLE               10001718     exported.obj
 0001:00000720       _DIF_DEFAULTBUTTON         10001720     exported.obj
 0001:00000728       _DIF_FOCUS                 10001728     exported.obj
 0001:00000730       _DIF_RIGHTTEXT             10001730     exported.obj
 0001:00000738       _DIF_WORDWRAP              10001738     exported.obj
 0001:00000740       _DIF_NONE                  10001740     exported.obj
 0001:00000748       _ECF_TABMARKFIRST          10001748     exported.obj
 0001:00000750       _ECF_TABMARKCURRENT        10001750     exported.obj
 0001:00000758       _ECF_AUTODELETE            10001758     exported.obj
 0001:00000760       _ECF_NONE                  10001760     exported.obj
 0001:00000768       _FIB_ENABLEEMPTY           10001768     exported.obj
 0001:00000770       _LIF_SELECTED              10001770     exported.obj
 0001:00000778       _FIB_PASSWORD              10001778     exported.obj
 0001:00000780       _FIB_EXPANDENV             10001780     exported.obj
 0001:00000788       _LIF_CHECKED               10001788     exported.obj
 0001:00000790       _LIF_SEPARATOR             10001790     exported.obj
 0001:00000798       _FIB_NOUSELASTHISTORY      10001798     exported.obj
 0001:000007a0       _FIB_BUTTONS               100017a0     exported.obj
 0001:000007a8       _LIF_DISABLE               100017a8     exported.obj
 0001:000007b0       _LIF_GRAYED                100017b0     exported.obj
 0001:000007b8       _FIB_NOAMPERSAND           100017b8     exported.obj
 0001:000007c0       _FIB_EDITPATH              100017c0     exported.obj
 0001:000007c8       _LIF_HIDDEN                100017c8     exported.obj
 0001:000007d0       _LIF_DELETEUSERDATA        100017d0     exported.obj
 0001:000007d8       _FIB_EDITPATHEXEC          100017d8     exported.obj
 0001:000007e0       _LIF_NONE                  100017e0     exported.obj
 0001:000007e8       _FIB_NONE                  100017e8     exported.obj
 0001:000007f0       _PCIF_FROMMAIN             100017f0     exported.obj
 0001:000007f8       _PCIF_NONE                 100017f8     exported.obj
 0001:00000800       _LIFIND_EXACTMATCH         10001800     exported.obj
 0001:00000808       _LIFIND_NONE               10001808     exported.obj
 0001:00000810       _LINFO_SHOWNOBOX           10001810     exported.obj
 0001:00000818       _FPF_LOADED                10001818     exported.obj
 0001:00000820       _LINFO_AUTOHIGHLIGHT       10001820     exported.obj
 0001:00000828       _LINFO_REVERSEHIGHLIGHT    10001828     exported.obj
 0001:00000830       _FPF_ANSI                  10001830     exported.obj
 0001:00000838       _LINFO_WRAPMODE            10001838     exported.obj
 0001:00000840       _FPF_NONE                  10001840     exported.obj
 0001:00000848       _LINFO_SHOWAMPERSAND       10001848     exported.obj
 0001:00000850       _LINFO_NONE                10001850     exported.obj
 0001:00000858       _FarGuid                   10001858     exported.obj
 0001:00000868       _FDLG_WARNING              10001868     exported.obj
 0001:00000870       _FDLG_SMALLDIALOG          10001870     exported.obj
 0001:00000878       _FDLG_NODRAWSHADOW         10001878     exported.obj
 0001:00000880       _FDLG_NODRAWPANEL          10001880     exported.obj
 0001:00000888       _FDLG_KEEPCONSOLETITLE     10001888     exported.obj
 0001:00000890       _FDLG_NONE                 10001890     exported.obj
 0001:00000898       _MIF_SELECTED              10001898     exported.obj
 0001:000008a0       _MIF_CHECKED               100018a0     exported.obj
 0001:000008a8       _MIF_SEPARATOR             100018a8     exported.obj
 0001:000008b0       _MIF_DISABLE               100018b0     exported.obj
 0001:000008b8       _MIF_GRAYED                100018b8     exported.obj
 0001:000008c0       _MIF_HIDDEN                100018c0     exported.obj
 0001:000008c8       _MIF_NONE                  100018c8     exported.obj
 0001:000008d0       _FMENU_SHOWAMPERSAND       100018d0     exported.obj
 0001:000008d8       _FMENU_WRAPMODE            100018d8     exported.obj
 0001:000008e0       _FMENU_AUTOHIGHLIGHT       100018e0     exported.obj
 0001:000008e8       _FMENU_REVERSEAUTOHIGHLIGHT 100018e8     exported.obj
 0001:000008f0       _FMENU_CHANGECONSOLETITLE  100018f0     exported.obj
 0001:000008f8       _FMENU_NONE                100018f8     exported.obj
 0001:00000900       _PPIF_SELECTED             10001900     exported.obj
 0001:00000908       _PPIF_PROCESSDESCR         10001908     exported.obj
 0001:00000910       _PPIF_NONE                 10001910     exported.obj
 0001:00000918       _PFLAGS_SHOWHIDDEN         10001918     exported.obj
 0001:00000920       _PFLAGS_HIGHLIGHT          10001920     exported.obj
 0001:00000928       _PFLAGS_REVERSESORTORDER   10001928     exported.obj
 0001:00000930       _PFLAGS_USESORTGROUPS      10001930     exported.obj
 0001:00000938       _PFLAGS_SELECTEDFIRST      10001938     exported.obj
 0001:00000940       _PFLAGS_REALNAMES          10001940     exported.obj
 0001:00000948       _PFLAGS_NUMERICSORT        10001948     exported.obj
 0001:00000950       _PFLAGS_PANELLEFT          10001950     exported.obj
 0001:00000958       _PFLAGS_DIRECTORIESFIRST   10001958     exported.obj
 0001:00000960       _PFLAGS_USECRC32           10001960     exported.obj
 0001:00000968       _PFLAGS_CASESENSITIVESORT  10001968     exported.obj
 0001:00000970       _PFLAGS_PLUGIN             10001970     exported.obj
 0001:00000978       _PFLAGS_VISIBLE            10001978     exported.obj
 0001:00000980       _PFLAGS_FOCUS              10001980     exported.obj
 0001:00000988       _PFLAGS_ALTERNATIVENAMES   10001988     exported.obj
 0001:00000990       _PFLAGS_SHORTCUT           10001990     exported.obj
 0001:00000998       _PFLAGS_NONE               10001998     exported.obj
 0001:000009a0       _PN_CMPNAME                100019a0     exported.obj
 0001:000009a8       _PN_CMPNAMELIST            100019a8     exported.obj
 0001:000009b0       _PN_GENERATENAME           100019b0     exported.obj
 0001:000009b8       _PN_CHECKMASK              100019b8     exported.obj
 0001:000009c0       _PN_SKIPPATH               100019c0     exported.obj
 0001:000009c8       _PN_SHOWERRORMESSAGE       100019c8     exported.obj
 0001:000009d0       _PN_NONE                   100019d0     exported.obj
 0001:000009d8       _XLAT_SWITCHKEYBLAYOUT     100019d8     exported.obj
 0001:000009e0       _XLAT_SWITCHKEYBBEEP       100019e0     exported.obj
 0001:000009e8       _XLAT_USEKEYBLAYOUTNAME    100019e8     exported.obj
 0001:000009f0       _XLAT_CONVERTALLCMDLINE    100019f0     exported.obj
 0001:000009f8       _XLAT_NONE                 100019f8     exported.obj
 0001:00000a00       _VF_NONMODAL               10001a00     exported.obj
 0001:00000a08       _VF_DELETEONCLOSE          10001a08     exported.obj
 0001:00000a10       _VF_ENABLE_F6              10001a10     exported.obj
 0001:00000a18       _VF_DISABLEHISTORY         10001a18     exported.obj
 0001:00000a20       _VF_IMMEDIATERETURN        10001a20     exported.obj
 0001:00000a28       _VF_DELETEONLYFILEONCLOSE  10001a28     exported.obj
 0001:00000a30       _VF_NONE                   10001a30     exported.obj
 0001:00000a38       _FRS_RETUPDIR              10001a38     exported.obj
 0001:00000a40       _FRS_RECUR                 10001a40     exported.obj
 0001:00000a48       _FRS_SCANSYMLINK           10001a48     exported.obj
 0001:00000a50       _FRS_NONE                  10001a50     exported.obj
 0001:00000a58       _EF_NONMODAL               10001a58     exported.obj
 0001:00000a60       _EF_CREATENEW              10001a60     exported.obj
 0001:00000a68       _EF_ENABLE_F6              10001a68     exported.obj
 0001:00000a70       _EF_DISABLEHISTORY         10001a70     exported.obj
 0001:00000a78       _EF_DELETEONCLOSE          10001a78     exported.obj
 0001:00000a80       _EF_IMMEDIATERETURN        10001a80     exported.obj
 0001:00000a88       _EF_DELETEONLYFILEONCLOSE  10001a88     exported.obj
 0001:00000a90       _EF_LOCKED                 10001a90     exported.obj
 0001:00000a98       _EF_DISABLESAVEPOS         10001a98     exported.obj
 0001:00000aa0       _EF_OPENMODE_MASK          10001aa0     exported.obj
 0001:00000aa8       _EF_OPENMODE_QUERY         10001aa8     exported.obj
 0001:00000ab0       _EF_OPENMODE_NEWIFOPEN     10001ab0     exported.obj
 0001:00000ab8       _EF_OPENMODE_USEEXISTING   10001ab8     exported.obj
 0001:00000ac0       _EF_OPENMODE_BREAKIFOPEN   10001ac0     exported.obj
 0001:00000ac8       _EF_OPENMODE_RELOADIFOPEN  10001ac8     exported.obj
 0001:00000ad0       _EN_NONE                   10001ad0     exported.obj
 0001:00000ad8       _MLF_SHOWERRMSG            10001ad8     exported.obj
 0001:00000ae0       _MLF_DONOTUPDATEPANEL      10001ae0     exported.obj
 0001:00000ae8       _MLF_HOLDTARGET            10001ae8     exported.obj
 0001:00000af0       _MLF_NONE                  10001af0     exported.obj
 0001:00001160       _FPF_LOADED                10002160     flags.obj
 0001:00001168       _LINFO_AUTOHIGHLIGHT       10002168     flags.obj
 0001:00001170       _LINFO_REVERSEHIGHLIGHT    10002170     flags.obj
 0001:00001178       _FPF_ANSI                  10002178     flags.obj
 0001:00001180       _LINFO_WRAPMODE            10002180     flags.obj
 0001:00001188       _FPF_NONE                  10002188     flags.obj
 0001:00001190       _LINFO_SHOWAMPERSAND       10002190     flags.obj
 0001:00001198       _LINFO_NONE                10002198     flags.obj
 0001:000011a0       _FarGuid                   100021a0     flags.obj
 0001:000011b0       _FDLG_WARNING              100021b0     flags.obj
 0001:000011b8       _FDLG_SMALLDIALOG          100021b8     flags.obj
 0001:000011c0       _FDLG_NODRAWSHADOW         100021c0     flags.obj
 0001:000011c8       _FDLG_NODRAWPANEL          100021c8     flags.obj
 0001:000011d0       _FDLG_KEEPCONSOLETITLE     100021d0     flags.obj
 0001:000011d8       _FDLG_NONE                 100021d8     flags.obj
 0001:000011e0       _MIF_SELECTED              100021e0     flags.obj
 0001:000011e8       _MIF_CHECKED               100021e8     flags.obj
 0001:000011f0       _MIF_SEPARATOR             100021f0     flags.obj
 0001:000011f8       _MIF_DISABLE               100021f8     flags.obj
 0001:00001200       _MIF_GRAYED                10002200     flags.obj
 0001:00001208       _MIF_HIDDEN                10002208     flags.obj
 0001:00001210       _MIF_NONE                  10002210     flags.obj
 0001:00001218       _FMENU_SHOWAMPERSAND       10002218     flags.obj
 0001:00001220       _FMENU_WRAPMODE            10002220     flags.obj
 0001:00001228       _FMENU_AUTOHIGHLIGHT       10002228     flags.obj
 0001:00001230       _FMENU_REVERSEAUTOHIGHLIGHT 10002230     flags.obj
 0001:00001238       _FMENU_CHANGECONSOLETITLE  10002238     flags.obj
 0001:00001240       _FMENU_NONE                10002240     flags.obj
 0001:00001248       _PPIF_SELECTED             10002248     flags.obj
 0001:00001250       _PPIF_PROCESSDESCR         10002250     flags.obj
 0001:00001258       _PPIF_NONE                 10002258     flags.obj
 0001:00001260       _PFLAGS_SHOWHIDDEN         10002260     flags.obj
 0001:00001268       _PFLAGS_HIGHLIGHT          10002268     flags.obj
 0001:00001270       _PFLAGS_REVERSESORTORDER   10002270     flags.obj
 0001:00001278       _PFLAGS_USESORTGROUPS      10002278     flags.obj
 0001:00001280       _PFLAGS_SELECTEDFIRST      10002280     flags.obj
 0001:00001288       _PFLAGS_REALNAMES          10002288     flags.obj
 0001:00001290       _PFLAGS_NUMERICSORT        10002290     flags.obj
 0001:00001298       _PFLAGS_PANELLEFT          10002298     flags.obj
 0001:000012a0       _PFLAGS_DIRECTORIESFIRST   100022a0     flags.obj
 0001:000012a8       _PFLAGS_USECRC32           100022a8     flags.obj
 0001:000012b0       _PFLAGS_CASESENSITIVESORT  100022b0     flags.obj
 0001:000012b8       _PFLAGS_PLUGIN             100022b8     flags.obj
 0001:000012c0       _PFLAGS_VISIBLE            100022c0     flags.obj
 0001:000012c8       _PFLAGS_FOCUS              100022c8     flags.obj
 0001:000012d0       _PFLAGS_ALTERNATIVENAMES   100022d0     flags.obj
 0001:000012d8       _PFLAGS_SHORTCUT           100022d8     flags.obj
 0001:000012e0       _PFLAGS_NONE               100022e0     flags.obj
 0001:000012e8       _PN_CMPNAME                100022e8     flags.obj
 0001:000012f0       _PN_CMPNAMELIST            100022f0     flags.obj
 0001:000012f8       _PN_GENERATENAME           100022f8     flags.obj
 0001:00001300       _PN_CHECKMASK              10002300     flags.obj
 0001:00001308       _PN_SKIPPATH               10002308     flags.obj
 0001:00001310       _PN_SHOWERRORMESSAGE       10002310     flags.obj
 0001:00001318       _PN_NONE                   10002318     flags.obj
 0001:00001320       _XLAT_SWITCHKEYBLAYOUT     10002320     flags.obj
 0001:00001328       _XLAT_SWITCHKEYBBEEP       10002328     flags.obj
 0001:00001330       _XLAT_USEKEYBLAYOUTNAME    10002330     flags.obj
 0001:00001338       _XLAT_CONVERTALLCMDLINE    10002338     flags.obj
 0001:00001340       _XLAT_NONE                 10002340     flags.obj
 0001:00001348       _VF_NONMODAL               10002348     flags.obj
 0001:00001350       _VF_DELETEONCLOSE          10002350     flags.obj
 0001:00001358       _VF_ENABLE_F6              10002358     flags.obj
 0001:00001360       _VF_DISABLEHISTORY         10002360     flags.obj
 0001:00001368       _VF_IMMEDIATERETURN        10002368     flags.obj
 0001:00001370       _VF_DELETEONLYFILEONCLOSE  10002370     flags.obj
 0001:00001378       _VF_NONE                   10002378     flags.obj
 0001:00001380       _FRS_RETUPDIR              10002380     flags.obj
 0001:00001388       _FRS_RECUR                 10002388     flags.obj
 0001:00001390       _FRS_SCANSYMLINK           10002390     flags.obj
 0001:00001398       _FRS_NONE                  10002398     flags.obj
 0001:000013a0       _EF_NONMODAL               100023a0     flags.obj
 0001:000013a8       _EF_CREATENEW              100023a8     flags.obj
 0001:000013b0       _EF_ENABLE_F6              100023b0     flags.obj
 0001:000013b8       _EF_DISABLEHISTORY         100023b8     flags.obj
 0001:000013c0       _EF_DELETEONCLOSE          100023c0     flags.obj
 0001:000013c8       _EF_IMMEDIATERETURN        100023c8     flags.obj
 0001:000013d0       _EF_DELETEONLYFILEONCLOSE  100023d0     flags.obj
 0001:000013d8       _EF_LOCKED                 100023d8     flags.obj
 0001:000013e0       _EF_DISABLESAVEPOS         100023e0     flags.obj
 0001:000013e8       _EF_OPENMODE_MASK          100023e8     flags.obj
 0001:000013f0       _EF_OPENMODE_QUERY         100023f0     flags.obj
 0001:000013f8       _EF_OPENMODE_NEWIFOPEN     100023f8     flags.obj
 0001:00001400       _EF_OPENMODE_USEEXISTING   10002400     flags.obj
 0001:00001408       _EF_OPENMODE_BREAKIFOPEN   10002408     flags.obj
 0001:00001410       _EF_OPENMODE_RELOADIFOPEN  10002410     flags.obj
 0001:00001418       _EN_NONE                   10002418     flags.obj
 0001:00001420       _MLF_SHOWERRMSG            10002420     flags.obj
 0001:00001428       _MLF_DONOTUPDATEPANEL      10002428     flags.obj
 0001:00001430       _MLF_HOLDTARGET            10002430     flags.obj
 0001:00001438       _MLF_NONE                  10002438     flags.obj
 0001:00001440       _FHELP_NOSHOWERROR         10002440     flags.obj
 0001:00001448       _FHELP_SELFHELP            10002448     flags.obj
 0001:00001450       _FHELP_FARHELP             10002450     flags.obj
 0001:00001458       _FHELP_CUSTOMFILE          10002458     flags.obj
 0001:00001460       _FHELP_CUSTOMPATH          10002460     flags.obj
 0001:00001468       _FHELP_GUID                10002468     flags.obj
 0001:00001470       _FHELP_USECONTENTS         10002470     flags.obj
 0001:00001478       _FHELP_NONE                10002478     flags.obj
 0001:00001480       _FFFS_COMMAS               10002480     flags.obj
 0001:00001488       _FFFS_FLOATSIZE            10002488     flags.obj
 0001:00001490       _FFFS_SHOWBYTESINDEX       10002490     flags.obj
 0001:00001498       _FFFS_ECONOMIC             10002498     flags.obj
 0001:000014a0       _FFFS_THOUSAND             100024a0     flags.obj
 0001:000014a8       _FFFS_MINSIZEINDEX         100024a8     flags.obj
 0001:000014b0       _FFFS_MINSIZEINDEX_MASK    100024b0     flags.obj
 0001:000014b8       _FFFS_NONE                 100024b8     flags.obj
 0001:000014c0       _KMFLAGS_SILENTCHECK       100024c0     flags.obj
 0001:000014c8       _KMFLAGS_NOSENDKEYSTOPLUGINS 100024c8     flags.obj
 0001:000014d0       _KMFLAGS_ENABLEOUTPUT      100024d0     flags.obj
 0001:000014d8       _KMFLAGS_LANGMASK          100024d8     flags.obj
 0001:000014e0       _KMFLAGS_LUA               100024e0     flags.obj
 0001:000014e8       _KMFLAGS_MOONSCRIPT        100024e8     flags.obj
 0001:000014f0       _KMFLAGS_NONE              100024f0     flags.obj
 0001:000014f8       _AKMFLAGS_NONE             100024f8     flags.obj
 0001:00001500       _FSETCLR_REDRAW            10002500     flags.obj
 0001:00001508       _FSETCLR_NONE              10002508     flags.obj
 0001:00001510       _WIF_MODIFIED              10002510     flags.obj
 0001:00001518       _WIF_CURRENT               10002518     flags.obj
 0001:00001520       _WIF_MODAL                 10002520     flags.obj
 0001:00001528       _WIF_NONE                  10002528     flags.obj
 0001:00001530       _PF_PRELOAD                10002530     flags.obj
 0001:00001538       _PF_DISABLEPANELS          10002538     flags.obj
 0001:00001540       _PF_EDITOR                 10002540     flags.obj
 0001:00001548       _PF_VIEWER                 10002548     flags.obj
 0001:00001550       _PF_FULLCMDLINE            10002550     flags.obj
 0001:00001558       _PF_DIALOG                 10002558     flags.obj
 0001:00001560       _PF_NONE                   10002560     flags.obj
 0001:00001568       _VOPT_SAVEFILEPOSITION     10002568     flags.obj
 0001:00001570       _VOPT_AUTODETECTCODEPAGE   10002570     flags.obj
 0001:00001578       _VOPT_SHOWTITLEBAR         10002578     flags.obj
 0001:00001580       _VOPT_SHOWKEYBAR           10002580     flags.obj
 0001:00001588       _VOPT_SHOWSCROLLBAR        10002588     flags.obj
 0001:00001590       _VOPT_QUICKVIEW            10002590     flags.obj
 0001:00001598       _VOPT_NONE                 10002598     flags.obj
 0001:000015a0       _VSMFL_REDRAW              100025a0     flags.obj
 0001:000015a8       _VSMFL_NONE                100025a8     flags.obj
 0001:000015b0       _VSP_NOREDRAW              100025b0     flags.obj
 0001:000015b8       _VSP_PERCENT               100025b8     flags.obj
 0001:000015c0       _VSP_RELATIVE              100025c0     flags.obj
 0001:000015c8       _VSP_NORETNEWPOS           100025c8     flags.obj
 0001:000015d0       _VSP_NONE                  100025d0     flags.obj
 0001:000015d8       _IPLFLAGS_SEPARATOR        100025d8     flags.obj
 0001:000015e0       _IPLFLAGS_NONE             100025e0     flags.obj
 0001:000015e8       _VMF_WRAP                  100025e8     flags.obj
 0001:000015f0       _PMFLAGS_FULLSCREEN        100025f0     flags.obj
 0001:000015f8       _VMF_WORDWRAP              100025f8     flags.obj
 0001:00001600       _VMF_NONE                  10002600     flags.obj
 0001:00001608       _PMFLAGS_DETAILEDSTATUS    10002608     flags.obj
 0001:00001610       _PMFLAGS_ALIGNEXTENSIONS   10002610     flags.obj
 0001:00001618       _PMFLAGS_CASECONVERSION    10002618     flags.obj
 0001:00001620       _PMFLAGS_NONE              10002620     flags.obj
 0001:00001628       _FCF_FG_4BIT               10002628     flags.obj
 0001:00001630       _FCF_BG_4BIT               10002630     flags.obj
 0001:00001638       _FCF_4BITMASK              10002638     flags.obj
 0001:00001640       _FCF_RAWATTR_MASK          10002640     flags.obj
 0001:00001648       _FCF_EXTENDEDFLAGS         10002648     flags.obj
 0001:00001650       _FCF_FG_BOLD               10002650     flags.obj
 0001:00001658       _FCF_FG_ITALIC             10002658     flags.obj
 0001:00001660       _FCF_FG_UNDERLINE          10002660     flags.obj
 0001:00001668       _FCF_STYLEMASK             10002668     flags.obj
 0001:00001670       _OPIF_DISABLEFILTER        10002670     flags.obj
 0001:00001678       _FCF_NONE                  10002678     flags.obj
 0001:00001680       _OPIF_DISABLESORTGROUPS    10002680     flags.obj
 0001:00001688       _OPIF_DISABLEHIGHLIGHTING  10002688     flags.obj
 0001:00001690       _OPIF_ADDDOTS              10002690     flags.obj
 0001:00001698       _OPIF_RAWSELECTION         10002698     flags.obj
 0001:000016a0       _OPIF_REALNAMES            100026a0     flags.obj
 0001:000016a8       _OPIF_SHOWNAMESONLY        100026a8     flags.obj
 0001:000016b0       _OPIF_SHOWRIGHTALIGNNAMES  100026b0     flags.obj
 0001:000016b8       _OPIF_SHOWPRESERVECASE     100026b8     flags.obj
 0001:000016c0       _OPIF_COMPAREFATTIME       100026c0     flags.obj
 0001:000016c8       _OPIF_EXTERNALGET          100026c8     flags.obj
 0001:000016d0       _OPIF_EXTERNALPUT          100026d0     flags.obj
 0001:000016d8       _OPIF_EXTERNALDELETE       100026d8     flags.obj
 0001:000016e0       _OPIF_EXTERNALMKDIR        100026e0     flags.obj
 0001:000016e8       _OPIF_USEATTRHIGHLIGHTING  100026e8     flags.obj
 0001:000016f0       _OPIF_USECRC32             100026f0     flags.obj
 0001:000016f8       _OPIF_USEFREESIZE          100026f8     flags.obj
 0001:00001700       _OPIF_SHORTCUT             10002700     flags.obj
 0001:00001708       _OPIF_NONE                 10002708     flags.obj
 0001:00001710       _CDF_NONE                  10002710     flags.obj
 0001:00001718       _FMSG_WARNING              10002718     flags.obj
 0001:00001720       _FMSG_ERRORTYPE            10002720     flags.obj
 0001:00001728       _FMSG_KEEPBACKGROUND       10002728     flags.obj
 0001:00001730       _OPM_SILENT                10002730     flags.obj
 0001:00001738       _OPM_FIND                  10002738     flags.obj
 0001:00001740       _FMSG_LEFTALIGN            10002740     flags.obj
 0001:00001748       _FMSG_ALLINONE             10002748     flags.obj
 0001:00001750       _OPM_VIEW                  10002750     flags.obj
 0001:00001758       _OPM_EDIT                  10002758     flags.obj
 0001:00001760       _FMSG_MB_OK                10002760     flags.obj
 0001:00001768       _FMSG_MB_OKCANCEL          10002768     flags.obj
 0001:00001770       _OPM_TOPLEVEL              10002770     flags.obj
 0001:00001778       _OPM_DESCR                 10002778     flags.obj
 0001:00001780       _FMSG_MB_ABORTRETRYIGNORE  10002780     flags.obj
 0001:00001788       _OPM_QUICKVIEW             10002788     flags.obj
 0001:00001790       _FMSG_MB_YESNO             10002790     flags.obj
 0001:00001798       _OPM_PGDN                  10002798     flags.obj
 0001:000017a0       _FMSG_MB_YESNOCANCEL       100027a0     flags.obj
 0001:000017a8       _FMSG_MB_RETRYCANCEL       100027a8     flags.obj
 0001:000017b0       _OPM_COMMANDS              100027b0     flags.obj
 0001:000017b8       _OPM_NONE                  100027b8     flags.obj
 0001:000017c0       _FMSG_NONE                 100027c0     flags.obj
 0001:000017c8       _FOSF_ACTIVE               100027c8     flags.obj
 0001:000017d0       _DIF_BOXCOLOR              100027d0     flags.obj
 0001:000017d8       _FOSF_NONE                 100027d8     flags.obj
 0001:000017e0       _DIF_GROUP                 100027e0     flags.obj
 0001:000017e8       _DIF_LEFTTEXT              100027e8     flags.obj
 0001:00002e28       _DIF_MOVESELECT            10003e28     flags.obj
 0001:00002e30       _DIF_SHOWAMPERSAND         10003e30     flags.obj
 0001:00002e38       _DIF_CENTERGROUP           10003e38     flags.obj
 0001:00002e40       _DIF_NOBRACKETS            10003e40     flags.obj
 0001:00002e48       _DIF_MANUALADDHISTORY      10003e48     flags.obj
 0001:00002e50       _DIF_SEPARATOR             10003e50     flags.obj
 0001:00002e58       _DIF_SEPARATOR2            10003e58     flags.obj
 0001:00002e60       _DIF_EDITOR                10003e60     flags.obj
 0001:00002e68       _DIF_LISTNOAMPERSAND       10003e68     flags.obj
 0001:00002e70       _DIF_LISTNOBOX             10003e70     flags.obj
 0001:00002e78       _DIF_HISTORY               10003e78     flags.obj
 0001:00002e80       _DIF_BTNNOCLOSE            10003e80     flags.obj
 0001:00002e88       _DIF_CENTERTEXT            10003e88     flags.obj
 0001:00002e90       _DIF_SEPARATORUSER         10003e90     flags.obj
 0001:00002e98       _DIF_SETSHIELD             10003e98     flags.obj
 0001:00002ea0       _DIF_EDITEXPAND            10003ea0     flags.obj
 0001:00002ea8       _DIF_DROPDOWNLIST          10003ea8     flags.obj
 0001:00002eb0       _DIF_USELASTHISTORY        10003eb0     flags.obj
 0001:00002eb8       _DIF_MASKEDIT              10003eb8     flags.obj
 0001:00002ec0       _DIF_LISTTRACKMOUSE        10003ec0     flags.obj
 0001:00002ec8       _DIF_LISTTRACKMOUSEINFOCUS 10003ec8     flags.obj
 0001:00002ed0       _DIF_SELECTONENTRY         10003ed0     flags.obj
 0001:00002ed8       _DIF_3STATE                10003ed8     flags.obj
 0001:00002ee0       _DIF_EDITPATH              10003ee0     flags.obj
 0001:00002ee8       _DIF_LISTWRAPMODE          10003ee8     flags.obj
 0001:00002ef0       _DIF_NOAUTOCOMPLETE        10003ef0     flags.obj
 0001:00002ef8       _DIF_LISTAUTOHIGHLIGHT     10003ef8     flags.obj
 0001:00002f00       _DIF_LISTNOCLOSE           10003f00     flags.obj
 0001:00002f08       _DIF_EDITPATHEXEC          10003f08     flags.obj
 0001:00002f10       _DIF_HIDDEN                10003f10     flags.obj
 0001:00002f18       _DIF_READONLY              10003f18     flags.obj
 0001:00002f20       _DIF_NOFOCUS               10003f20     flags.obj
 0001:00002f28       _DIF_DISABLE               10003f28     flags.obj
 0001:00002f30       _DIF_DEFAULTBUTTON         10003f30     flags.obj
 0001:00002f38       _DIF_FOCUS                 10003f38     flags.obj
 0001:00002f40       _DIF_RIGHTTEXT             10003f40     flags.obj
 0001:00002f48       _DIF_WORDWRAP              10003f48     flags.obj
 0001:00002f50       _DIF_NONE                  10003f50     flags.obj
 0001:00002f58       _ECF_TABMARKFIRST          10003f58     flags.obj
 0001:00002f60       _ECF_TABMARKCURRENT        10003f60     flags.obj
 0001:00002f68       _ECF_AUTODELETE            10003f68     flags.obj
 0001:00002f70       _ECF_NONE                  10003f70     flags.obj
 0001:00002f78       _FIB_ENABLEEMPTY           10003f78     flags.obj
 0001:00002f80       _LIF_SELECTED              10003f80     flags.obj
 0001:00002f88       _FIB_PASSWORD              10003f88     flags.obj
 0001:00002f90       _FIB_EXPANDENV             10003f90     flags.obj
 0001:00002f98       _LIF_CHECKED               10003f98     flags.obj
 0001:00002fa0       _LIF_SEPARATOR             10003fa0     flags.obj
 0001:00002fa8       _FIB_NOUSELASTHISTORY      10003fa8     flags.obj
 0001:00002fb0       _FIB_BUTTONS               10003fb0     flags.obj
 0001:00002fb8       _LIF_DISABLE               10003fb8     flags.obj
 0001:00002fc0       _LIF_GRAYED                10003fc0     flags.obj
 0001:00002fc8       _FIB_NOAMPERSAND           10003fc8     flags.obj
 0001:00002fd0       _FIB_EDITPATH              10003fd0     flags.obj
 0001:00002fd8       _LIF_HIDDEN                10003fd8     flags.obj
 0001:00002fe0       _LIF_DELETEUSERDATA        10003fe0     flags.obj
 0001:00002fe8       _FIB_EDITPATHEXEC          10003fe8     flags.obj
 0001:00002ff0       _LIF_NONE                  10003ff0     flags.obj
 0001:00002ff8       _FIB_NONE                  10003ff8     flags.obj
 0001:00003000       _PCIF_FROMMAIN             10004000     flags.obj
 0001:00003008       _PCIF_NONE                 10004008     flags.obj
 0001:00003010       _LIFIND_EXACTMATCH         10004010     flags.obj
 0001:00003018       _LIFIND_NONE               10004018     flags.obj
 0001:00003020       _LINFO_SHOWNOBOX           10004020     flags.obj
 0001:00005ee0       _colors                    10006ee0     keysandcolors.obj
 0001:00006e40       _guids                     10007e40     keysandcolors.obj
 0001:00008110       _FSETCLR_REDRAW            10009110     lflua.obj
 0001:00008118       _FSETCLR_NONE              10009118     lflua.obj
 0001:00008120       _WIF_MODIFIED              10009120     lflua.obj
 0001:00008128       _WIF_CURRENT               10009128     lflua.obj
 0001:00008130       _WIF_MODAL                 10009130     lflua.obj
 0001:00008138       _WIF_NONE                  10009138     lflua.obj
 0001:00008140       _PF_PRELOAD                10009140     lflua.obj
 0001:00008148       _PF_DISABLEPANELS          10009148     lflua.obj
 0001:00008150       _PF_EDITOR                 10009150     lflua.obj
 0001:00008158       _PF_VIEWER                 10009158     lflua.obj
 0001:00008160       _PF_FULLCMDLINE            10009160     lflua.obj
 0001:00008168       _PF_DIALOG                 10009168     lflua.obj
 0001:00008170       _PF_NONE                   10009170     lflua.obj
 0001:00008178       _VOPT_SAVEFILEPOSITION     10009178     lflua.obj
 0001:00008180       _VOPT_AUTODETECTCODEPAGE   10009180     lflua.obj
 0001:00008188       _VOPT_SHOWTITLEBAR         10009188     lflua.obj
 0001:00008190       _VOPT_SHOWKEYBAR           10009190     lflua.obj
 0001:00008198       _VOPT_SHOWSCROLLBAR        10009198     lflua.obj
 0001:000081a0       _VOPT_QUICKVIEW            100091a0     lflua.obj
 0001:000081a8       _VOPT_NONE                 100091a8     lflua.obj
 0001:000081b0       _VSMFL_REDRAW              100091b0     lflua.obj
 0001:000081b8       _VSMFL_NONE                100091b8     lflua.obj
 0001:000081c0       _VSP_NOREDRAW              100091c0     lflua.obj
 0001:000081c8       _VSP_PERCENT               100091c8     lflua.obj
 0001:000081d0       _VSP_RELATIVE              100091d0     lflua.obj
 0001:000081d8       _VSP_NORETNEWPOS           100091d8     lflua.obj
 0001:000081e0       _VSP_NONE                  100091e0     lflua.obj
 0001:000081e8       _IPLFLAGS_SEPARATOR        100091e8     lflua.obj
 0001:000081f0       _IPLFLAGS_NONE             100091f0     lflua.obj
 0001:000081f8       _VMF_WRAP                  100091f8     lflua.obj
 0001:00008200       _PMFLAGS_FULLSCREEN        10009200     lflua.obj
 0001:00008208       _VMF_WORDWRAP              10009208     lflua.obj
 0001:00008210       _VMF_NONE                  10009210     lflua.obj
 0001:00008218       _PMFLAGS_DETAILEDSTATUS    10009218     lflua.obj
 0001:00008220       _PMFLAGS_ALIGNEXTENSIONS   10009220     lflua.obj
 0001:00008228       _PMFLAGS_CASECONVERSION    10009228     lflua.obj
 0001:00008230       _PMFLAGS_NONE              10009230     lflua.obj
 0001:00008238       _FCF_FG_4BIT               10009238     lflua.obj
 0001:00008240       _FCF_BG_4BIT               10009240     lflua.obj
 0001:00008248       _FCF_4BITMASK              10009248     lflua.obj
 0001:00008250       _FCF_RAWATTR_MASK          10009250     lflua.obj
 0001:00008258       _FCF_EXTENDEDFLAGS         10009258     lflua.obj
 0001:00008260       _FCF_FG_BOLD               10009260     lflua.obj
 0001:00008268       _FCF_FG_ITALIC             10009268     lflua.obj
 0001:00008270       _FCF_FG_UNDERLINE          10009270     lflua.obj
 0001:00008278       _FCF_STYLEMASK             10009278     lflua.obj
 0001:00008280       _OPIF_DISABLEFILTER        10009280     lflua.obj
 0001:00008288       _FCF_NONE                  10009288     lflua.obj
 0001:00008290       _OPIF_DISABLESORTGROUPS    10009290     lflua.obj
 0001:00008298       _OPIF_DISABLEHIGHLIGHTING  10009298     lflua.obj
 0001:000082a0       _OPIF_ADDDOTS              100092a0     lflua.obj
 0001:000082a8       _OPIF_RAWSELECTION         100092a8     lflua.obj
 0001:000082b0       _OPIF_REALNAMES            100092b0     lflua.obj
 0001:000082b8       _OPIF_SHOWNAMESONLY        100092b8     lflua.obj
 0001:000082c0       _OPIF_SHOWRIGHTALIGNNAMES  100092c0     lflua.obj
 0001:000082c8       _OPIF_SHOWPRESERVECASE     100092c8     lflua.obj
 0001:000082d0       _OPIF_COMPAREFATTIME       100092d0     lflua.obj
 0001:000082d8       _OPIF_EXTERNALGET          100092d8     lflua.obj
 0001:000082e0       _OPIF_EXTERNALPUT          100092e0     lflua.obj
 0001:000082e8       _OPIF_EXTERNALDELETE       100092e8     lflua.obj
 0001:000082f0       _OPIF_EXTERNALMKDIR        100092f0     lflua.obj
 0001:000082f8       _OPIF_USEATTRHIGHLIGHTING  100092f8     lflua.obj
 0001:00008300       _OPIF_USECRC32             10009300     lflua.obj
 0001:00008308       _OPIF_USEFREESIZE          10009308     lflua.obj
 0001:00008310       _OPIF_SHORTCUT             10009310     lflua.obj
 0001:00008318       _OPIF_NONE                 10009318     lflua.obj
 0001:00008320       _CDF_NONE                  10009320     lflua.obj
 0001:00008328       _FMSG_WARNING              10009328     lflua.obj
 0001:00008330       _FMSG_ERRORTYPE            10009330     lflua.obj
 0001:00008338       _FMSG_KEEPBACKGROUND       10009338     lflua.obj
 0001:00008340       _OPM_SILENT                10009340     lflua.obj
 0001:00008348       _OPM_FIND                  10009348     lflua.obj
 0001:00008350       _FMSG_LEFTALIGN            10009350     lflua.obj
 0001:00008358       _FMSG_ALLINONE             10009358     lflua.obj
 0001:00008360       _OPM_VIEW                  10009360     lflua.obj
 0001:00008368       _OPM_EDIT                  10009368     lflua.obj
 0001:00008370       _FMSG_MB_OK                10009370     lflua.obj
 0001:00008378       _FMSG_MB_OKCANCEL          10009378     lflua.obj
 0001:00008380       _OPM_TOPLEVEL              10009380     lflua.obj
 0001:00008388       _OPM_DESCR                 10009388     lflua.obj
 0001:00008390       _FMSG_MB_ABORTRETRYIGNORE  10009390     lflua.obj
 0001:00008398       _OPM_QUICKVIEW             10009398     lflua.obj
 0001:000083a0       _FMSG_MB_YESNO             100093a0     lflua.obj
 0001:000083a8       _OPM_PGDN                  100093a8     lflua.obj
 0001:000083b0       _FMSG_MB_YESNOCANCEL       100093b0     lflua.obj
 0001:000083b8       _FMSG_MB_RETRYCANCEL       100093b8     lflua.obj
 0001:000083c0       _OPM_COMMANDS              100093c0     lflua.obj
 0001:000083c8       _OPM_NONE                  100093c8     lflua.obj
 0001:000083d0       _FMSG_NONE                 100093d0     lflua.obj
 0001:000083d8       _FOSF_ACTIVE               100093d8     lflua.obj
 0001:000083e0       _DIF_BOXCOLOR              100093e0     lflua.obj
 0001:000083e8       _FOSF_NONE                 100093e8     lflua.obj
 0001:000083f0       _DIF_GROUP                 100093f0     lflua.obj
 0001:000083f8       _DIF_LEFTTEXT              100093f8     lflua.obj
 0001:00008400       _DIF_MOVESELECT            10009400     lflua.obj
 0001:00008408       _DIF_SHOWAMPERSAND         10009408     lflua.obj
 0001:00008410       _DIF_CENTERGROUP           10009410     lflua.obj
 0001:00008418       _DIF_NOBRACKETS            10009418     lflua.obj
 0001:00008420       _DIF_MANUALADDHISTORY      10009420     lflua.obj
 0001:00008428       _DIF_SEPARATOR             10009428     lflua.obj
 0001:00008430       _DIF_SEPARATOR2            10009430     lflua.obj
 0001:00008438       _DIF_EDITOR                10009438     lflua.obj
 0001:00008440       _DIF_LISTNOAMPERSAND       10009440     lflua.obj
 0001:00008448       _DIF_LISTNOBOX             10009448     lflua.obj
 0001:00008450       _DIF_HISTORY               10009450     lflua.obj
 0001:00008458       _DIF_BTNNOCLOSE            10009458     lflua.obj
 0001:00008460       _DIF_CENTERTEXT            10009460     lflua.obj
 0001:00008468       _DIF_SEPARATORUSER         10009468     lflua.obj
 0001:00008470       _DIF_SETSHIELD             10009470     lflua.obj
 0001:00008478       _DIF_EDITEXPAND            10009478     lflua.obj
 0001:00008480       _DIF_DROPDOWNLIST          10009480     lflua.obj
 0001:00008488       _DIF_USELASTHISTORY        10009488     lflua.obj
 0001:00008490       _DIF_MASKEDIT              10009490     lflua.obj
 0001:00008498       _DIF_LISTTRACKMOUSE        10009498     lflua.obj
 0001:000084a0       _DIF_LISTTRACKMOUSEINFOCUS 100094a0     lflua.obj
 0001:000084a8       _DIF_SELECTONENTRY         100094a8     lflua.obj
 0001:000084b0       _DIF_3STATE                100094b0     lflua.obj
 0001:000084b8       _DIF_EDITPATH              100094b8     lflua.obj
 0001:000084c0       _DIF_LISTWRAPMODE          100094c0     lflua.obj
 0001:000084c8       _DIF_NOAUTOCOMPLETE        100094c8     lflua.obj
 0001:000084d0       _DIF_LISTAUTOHIGHLIGHT     100094d0     lflua.obj
 0001:000084d8       _DIF_LISTNOCLOSE           100094d8     lflua.obj
 0001:000084e0       _DIF_EDITPATHEXEC          100094e0     lflua.obj
 0001:000084e8       _DIF_HIDDEN                100094e8     lflua.obj
 0001:000084f0       _DIF_READONLY              100094f0     lflua.obj
 0001:000084f8       _DIF_NOFOCUS               100094f8     lflua.obj
 0001:00008500       _DIF_DISABLE               10009500     lflua.obj
 0001:00008508       _DIF_DEFAULTBUTTON         10009508     lflua.obj
 0001:00008510       _DIF_FOCUS                 10009510     lflua.obj
 0001:00008518       _DIF_RIGHTTEXT             10009518     lflua.obj
 0001:00008520       _DIF_WORDWRAP              10009520     lflua.obj
 0001:00008528       _DIF_NONE                  10009528     lflua.obj
 0001:00008530       _ECF_TABMARKFIRST          10009530     lflua.obj
 0001:00008538       _ECF_TABMARKCURRENT        10009538     lflua.obj
 0001:00008540       _ECF_AUTODELETE            10009540     lflua.obj
 0001:00008548       _ECF_NONE                  10009548     lflua.obj
 0001:00008550       _FIB_ENABLEEMPTY           10009550     lflua.obj
 0001:00008558       _LIF_SELECTED              10009558     lflua.obj
 0001:00008560       _FIB_PASSWORD              10009560     lflua.obj
 0001:00008568       _FIB_EXPANDENV             10009568     lflua.obj
 0001:00008570       _LIF_CHECKED               10009570     lflua.obj
 0001:00008578       _LIF_SEPARATOR             10009578     lflua.obj
 0001:00008580       _FIB_NOUSELASTHISTORY      10009580     lflua.obj
 0001:00008588       _FIB_BUTTONS               10009588     lflua.obj
 0001:00008590       _LIF_DISABLE               10009590     lflua.obj
 0001:00008598       _LIF_GRAYED                10009598     lflua.obj
 0001:000085a0       _FIB_NOAMPERSAND           100095a0     lflua.obj
 0001:000085a8       _FIB_EDITPATH              100095a8     lflua.obj
 0001:000085b0       _LIF_HIDDEN                100095b0     lflua.obj
 0001:000085b8       _LIF_DELETEUSERDATA        100095b8     lflua.obj
 0001:000085c0       _FIB_EDITPATHEXEC          100095c0     lflua.obj
 0001:000085c8       _LIF_NONE                  100095c8     lflua.obj
 0001:000085d0       _FIB_NONE                  100095d0     lflua.obj
 0001:000085d8       _PCIF_FROMMAIN             100095d8     lflua.obj
 0001:000085e0       _PCIF_NONE                 100095e0     lflua.obj
 0001:000085e8       _LIFIND_EXACTMATCH         100095e8     lflua.obj
 0001:000085f0       _LIFIND_NONE               100095f0     lflua.obj
 0001:000085f8       _LINFO_SHOWNOBOX           100095f8     lflua.obj
 0001:00008600       _FPF_LOADED                10009600     lflua.obj
 0001:00008608       _LINFO_AUTOHIGHLIGHT       10009608     lflua.obj
 0001:00008610       _LINFO_REVERSEHIGHLIGHT    10009610     lflua.obj
 0001:00008618       _FPF_ANSI                  10009618     lflua.obj
 0001:00008620       _LINFO_WRAPMODE            10009620     lflua.obj
 0001:00008628       _FPF_NONE                  10009628     lflua.obj
 0001:00008630       _LINFO_SHOWAMPERSAND       10009630     lflua.obj
 0001:00008638       _LINFO_NONE                10009638     lflua.obj
 0001:00008640       _FarGuid                   10009640     lflua.obj
 0001:00008650       _FDLG_WARNING              10009650     lflua.obj
 0001:00008658       _FDLG_SMALLDIALOG          10009658     lflua.obj
 0001:00008660       _FDLG_NODRAWSHADOW         10009660     lflua.obj
 0001:00008668       _FDLG_NODRAWPANEL          10009668     lflua.obj
 0001:00008670       _FDLG_KEEPCONSOLETITLE     10009670     lflua.obj
 0001:00008678       _FDLG_NONE                 10009678     lflua.obj
 0001:00008680       _PDF_DIALOGEVENTDRAWENABLE 10009680     lflua.obj
 0001:00008684       _PDF_PROCESSINGERROR       10009684     lflua.obj
 0001:00008688       _MIF_SELECTED              10009688     lflua.obj
 0001:00008690       _MIF_CHECKED               10009690     lflua.obj
 0001:00008698       _MIF_SEPARATOR             10009698     lflua.obj
 0001:000086a0       _MIF_DISABLE               100096a0     lflua.obj
 0001:000086a8       _MIF_GRAYED                100096a8     lflua.obj
 0001:000086b0       _MIF_HIDDEN                100096b0     lflua.obj
 0001:000086b8       _MIF_NONE                  100096b8     lflua.obj
 0001:000086c0       _FMENU_SHOWAMPERSAND       100096c0     lflua.obj
 0001:000086c8       _FMENU_WRAPMODE            100096c8     lflua.obj
 0001:000086d0       _FMENU_AUTOHIGHLIGHT       100096d0     lflua.obj
 0001:000086d8       _FMENU_REVERSEAUTOHIGHLIGHT 100096d8     lflua.obj
 0001:000086e0       _FMENU_CHANGECONSOLETITLE  100096e0     lflua.obj
 0001:000086e8       _FMENU_NONE                100096e8     lflua.obj
 0001:000086f0       _PPIF_SELECTED             100096f0     lflua.obj
 0001:000086f8       _PPIF_PROCESSDESCR         100096f8     lflua.obj
 0001:00008700       _PPIF_NONE                 10009700     lflua.obj
 0001:00008708       _PFLAGS_SHOWHIDDEN         10009708     lflua.obj
 0001:00008710       _PFLAGS_HIGHLIGHT          10009710     lflua.obj
 0001:00008718       _PFLAGS_REVERSESORTORDER   10009718     lflua.obj
 0001:00008720       _PFLAGS_USESORTGROUPS      10009720     lflua.obj
 0001:00008728       _PFLAGS_SELECTEDFIRST      10009728     lflua.obj
 0001:00008730       _PFLAGS_REALNAMES          10009730     lflua.obj
 0001:00008738       _PFLAGS_NUMERICSORT        10009738     lflua.obj
 0001:00008740       _PFLAGS_PANELLEFT          10009740     lflua.obj
 0001:00008748       _PFLAGS_DIRECTORIESFIRST   10009748     lflua.obj
 0001:00008750       _PFLAGS_USECRC32           10009750     lflua.obj
 0001:00008758       _PFLAGS_CASESENSITIVESORT  10009758     lflua.obj
 0001:00008760       _PFLAGS_PLUGIN             10009760     lflua.obj
 0001:00008768       _PFLAGS_VISIBLE            10009768     lflua.obj
 0001:00008770       _PFLAGS_FOCUS              10009770     lflua.obj
 0001:00008778       _PFLAGS_ALTERNATIVENAMES   10009778     lflua.obj
 0001:00008780       _PFLAGS_SHORTCUT           10009780     lflua.obj
 0001:00008788       _PFLAGS_NONE               10009788     lflua.obj
 0001:00008790       _PN_CMPNAME                10009790     lflua.obj
 0001:00008798       _PN_CMPNAMELIST            10009798     lflua.obj
 0001:000087a0       _PN_GENERATENAME           100097a0     lflua.obj
 0001:000087a8       _PN_CHECKMASK              100097a8     lflua.obj
 0001:000087b0       _PN_SKIPPATH               100097b0     lflua.obj
 0001:000087b8       _PN_SHOWERRORMESSAGE       100097b8     lflua.obj
 0001:000087c0       _PN_NONE                   100097c0     lflua.obj
 0001:000087c8       _XLAT_SWITCHKEYBLAYOUT     100097c8     lflua.obj
 0001:000087d0       _XLAT_SWITCHKEYBBEEP       100097d0     lflua.obj
 0001:000087d8       _XLAT_USEKEYBLAYOUTNAME    100097d8     lflua.obj
 0001:000087e0       _XLAT_CONVERTALLCMDLINE    100097e0     lflua.obj
 0001:000087e8       _XLAT_NONE                 100097e8     lflua.obj
 0001:000087f0       _VF_NONMODAL               100097f0     lflua.obj
 0001:000087f8       _VF_DELETEONCLOSE          100097f8     lflua.obj
 0001:00008800       _VF_ENABLE_F6              10009800     lflua.obj
 0001:00008808       _VF_DISABLEHISTORY         10009808     lflua.obj
 0001:00008810       _VF_IMMEDIATERETURN        10009810     lflua.obj
 0001:00008818       _VF_DELETEONLYFILEONCLOSE  10009818     lflua.obj
 0001:00008820       _VF_NONE                   10009820     lflua.obj
 0001:00008828       _FRS_RETUPDIR              10009828     lflua.obj
 0001:00008830       _FRS_RECUR                 10009830     lflua.obj
 0001:00008838       _FRS_SCANSYMLINK           10009838     lflua.obj
 0001:00008840       _FRS_NONE                  10009840     lflua.obj
 0001:00008848       _EF_NONMODAL               10009848     lflua.obj
 0001:00008850       _EF_CREATENEW              10009850     lflua.obj
 0001:00008858       _EF_ENABLE_F6              10009858     lflua.obj
 0001:00008860       _EF_DISABLEHISTORY         10009860     lflua.obj
 0001:00008868       _EF_DELETEONCLOSE          10009868     lflua.obj
 0001:00008870       _EF_IMMEDIATERETURN        10009870     lflua.obj
 0001:00008878       _EF_DELETEONLYFILEONCLOSE  10009878     lflua.obj
 0001:00008880       _EF_LOCKED                 10009880     lflua.obj
 0001:00008888       _EF_DISABLESAVEPOS         10009888     lflua.obj
 0001:00008890       _EF_OPENMODE_MASK          10009890     lflua.obj
 0001:00008898       _EF_OPENMODE_QUERY         10009898     lflua.obj
 0001:000088a0       _EF_OPENMODE_NEWIFOPEN     100098a0     lflua.obj
 0001:000088a8       _EF_OPENMODE_USEEXISTING   100098a8     lflua.obj
 0001:000088b0       _EF_OPENMODE_BREAKIFOPEN   100098b0     lflua.obj
 0001:000088b8       _EF_OPENMODE_RELOADIFOPEN  100098b8     lflua.obj
 0001:000088c0       _EN_NONE                   100098c0     lflua.obj
 0001:000088c8       _MLF_SHOWERRMSG            100098c8     lflua.obj
 0001:000088d0       _MLF_DONOTUPDATEPANEL      100098d0     lflua.obj
 0001:000088d8       _MLF_HOLDTARGET            100098d8     lflua.obj
 0001:000088e0       _MLF_NONE                  100098e0     lflua.obj
 0001:000088e8       _FHELP_NOSHOWERROR         100098e8     lflua.obj
 0001:000088f0       _FHELP_SELFHELP            100098f0     lflua.obj
 0001:000088f8       _FHELP_FARHELP             100098f8     lflua.obj
 0001:00008900       _FHELP_CUSTOMFILE          10009900     lflua.obj
 0001:00008908       _FHELP_CUSTOMPATH          10009908     lflua.obj
 0001:00008910       _FHELP_GUID                10009910     lflua.obj
 0001:00008918       _FHELP_USECONTENTS         10009918     lflua.obj
 0001:00008920       _FHELP_NONE                10009920     lflua.obj
 0001:00008928       _FFFS_COMMAS               10009928     lflua.obj
 0001:00008930       _FFFS_FLOATSIZE            10009930     lflua.obj
 0001:00008938       _FFFS_SHOWBYTESINDEX       10009938     lflua.obj
 0001:00008940       _FFFS_ECONOMIC             10009940     lflua.obj
 0001:00008948       _FFFS_THOUSAND             10009948     lflua.obj
 0001:00008950       _FFFS_MINSIZEINDEX         10009950     lflua.obj
 0001:00008958       _FFFS_MINSIZEINDEX_MASK    10009958     lflua.obj
 0001:00008960       _FFFS_NONE                 10009960     lflua.obj
 0001:00008968       _KMFLAGS_SILENTCHECK       10009968     lflua.obj
 0001:00008970       _KMFLAGS_NOSENDKEYSTOPLUGINS 10009970     lflua.obj
 0001:00008978       _KMFLAGS_ENABLEOUTPUT      10009978     lflua.obj
 0001:00008980       _KMFLAGS_LANGMASK          10009980     lflua.obj
 0001:00008988       _KMFLAGS_LUA               10009988     lflua.obj
 0001:00008990       _KMFLAGS_MOONSCRIPT        10009990     lflua.obj
 0001:00008998       _KMFLAGS_NONE              10009998     lflua.obj
 0001:000089a0       _AKMFLAGS_NONE             100099a0     lflua.obj
 0001:000089f8       _FHELP_USECONTENTS         100099f8     lregex.obj
 0001:00008a00       _FHELP_NONE                10009a00     lregex.obj
 0001:00008a08       _FFFS_COMMAS               10009a08     lregex.obj
 0001:00008a10       _FFFS_FLOATSIZE            10009a10     lregex.obj
 0001:00008a18       _FFFS_SHOWBYTESINDEX       10009a18     lregex.obj
 0001:00008a20       _FFFS_ECONOMIC             10009a20     lregex.obj
 0001:00008a28       _FFFS_THOUSAND             10009a28     lregex.obj
 0001:00008a30       _FFFS_MINSIZEINDEX         10009a30     lregex.obj
 0001:00008a38       _FFFS_MINSIZEINDEX_MASK    10009a38     lregex.obj
 0001:00008a40       _FFFS_NONE                 10009a40     lregex.obj
 0001:00008a48       _KMFLAGS_SILENTCHECK       10009a48     lregex.obj
 0001:00008a50       _KMFLAGS_NOSENDKEYSTOPLUGINS 10009a50     lregex.obj
 0001:00008a58       _KMFLAGS_ENABLEOUTPUT      10009a58     lregex.obj
 0001:00008a60       _KMFLAGS_LANGMASK          10009a60     lregex.obj
 0001:00008a68       _KMFLAGS_LUA               10009a68     lregex.obj
 0001:00008a70       _KMFLAGS_MOONSCRIPT        10009a70     lregex.obj
 0001:00008a78       _KMFLAGS_NONE              10009a78     lregex.obj
 0001:00008a80       _AKMFLAGS_NONE             10009a80     lregex.obj
 0001:00008a88       _FSETCLR_REDRAW            10009a88     lregex.obj
 0001:00008a90       _FSETCLR_NONE              10009a90     lregex.obj
 0001:00008a98       _WIF_MODIFIED              10009a98     lregex.obj
 0001:00008aa0       _WIF_CURRENT               10009aa0     lregex.obj
 0001:00008aa8       _WIF_MODAL                 10009aa8     lregex.obj
 0001:00008ab0       _WIF_NONE                  10009ab0     lregex.obj
 0001:00008ab8       _PF_PRELOAD                10009ab8     lregex.obj
 0001:00008ac0       _PF_DISABLEPANELS          10009ac0     lregex.obj
 0001:00008ac8       _PF_EDITOR                 10009ac8     lregex.obj
 0001:00008ad0       _PF_VIEWER                 10009ad0     lregex.obj
 0001:00008ad8       _PF_FULLCMDLINE            10009ad8     lregex.obj
 0001:00008ae0       _PF_DIALOG                 10009ae0     lregex.obj
 0001:00008ae8       _PF_NONE                   10009ae8     lregex.obj
 0001:00008af0       _VOPT_SAVEFILEPOSITION     10009af0     lregex.obj
 0001:00008af8       _VOPT_AUTODETECTCODEPAGE   10009af8     lregex.obj
 0001:00008b00       _VOPT_SHOWTITLEBAR         10009b00     lregex.obj
 0001:00008b08       _VOPT_SHOWKEYBAR           10009b08     lregex.obj
 0001:00008b10       _VOPT_SHOWSCROLLBAR        10009b10     lregex.obj
 0001:00008b18       _VOPT_QUICKVIEW            10009b18     lregex.obj
 0001:00008b20       _VOPT_NONE                 10009b20     lregex.obj
 0001:00008b28       _VSMFL_REDRAW              10009b28     lregex.obj
 0001:00008b30       _VSMFL_NONE                10009b30     lregex.obj
 0001:00008b38       _VSP_NOREDRAW              10009b38     lregex.obj
 0001:00008b40       _VSP_PERCENT               10009b40     lregex.obj
 0001:00008b48       _VSP_RELATIVE              10009b48     lregex.obj
 0001:00008b50       _VSP_NORETNEWPOS           10009b50     lregex.obj
 0001:00008b58       _VSP_NONE                  10009b58     lregex.obj
 0001:00008b60       _IPLFLAGS_SEPARATOR        10009b60     lregex.obj
 0001:00008b68       _IPLFLAGS_NONE             10009b68     lregex.obj
 0001:00008b70       _VMF_WRAP                  10009b70     lregex.obj
 0001:00008b78       _PMFLAGS_FULLSCREEN        10009b78     lregex.obj
 0001:00008b80       _VMF_WORDWRAP              10009b80     lregex.obj
 0001:00008b88       _VMF_NONE                  10009b88     lregex.obj
 0001:00008b90       _PMFLAGS_DETAILEDSTATUS    10009b90     lregex.obj
 0001:00008b98       _PMFLAGS_ALIGNEXTENSIONS   10009b98     lregex.obj
 0001:00008ba0       _PMFLAGS_CASECONVERSION    10009ba0     lregex.obj
 0001:00008ba8       _PMFLAGS_NONE              10009ba8     lregex.obj
 0001:00008bb0       _FCF_FG_4BIT               10009bb0     lregex.obj
 0001:00008bb8       _FCF_BG_4BIT               10009bb8     lregex.obj
 0001:00008bc0       _FCF_4BITMASK              10009bc0     lregex.obj
 0001:00008bc8       _FCF_RAWATTR_MASK          10009bc8     lregex.obj
 0001:00008bd0       _FCF_EXTENDEDFLAGS         10009bd0     lregex.obj
 0001:00008bd8       _FCF_FG_BOLD               10009bd8     lregex.obj
 0001:00008be0       _FCF_FG_ITALIC             10009be0     lregex.obj
 0001:00008be8       _FCF_FG_UNDERLINE          10009be8     lregex.obj
 0001:00008bf0       _FCF_STYLEMASK             10009bf0     lregex.obj
 0001:00008bf8       _OPIF_DISABLEFILTER        10009bf8     lregex.obj
 0001:00008c00       _FCF_NONE                  10009c00     lregex.obj
 0001:00008c08       _OPIF_DISABLESORTGROUPS    10009c08     lregex.obj
 0001:00008c10       _OPIF_DISABLEHIGHLIGHTING  10009c10     lregex.obj
 0001:00008c18       _OPIF_ADDDOTS              10009c18     lregex.obj
 0001:00008c20       _OPIF_RAWSELECTION         10009c20     lregex.obj
 0001:00008c28       _OPIF_REALNAMES            10009c28     lregex.obj
 0001:00008c30       _OPIF_SHOWNAMESONLY        10009c30     lregex.obj
 0001:00008c38       _OPIF_SHOWRIGHTALIGNNAMES  10009c38     lregex.obj
 0001:00008c40       _OPIF_SHOWPRESERVECASE     10009c40     lregex.obj
 0001:00008c48       _OPIF_COMPAREFATTIME       10009c48     lregex.obj
 0001:00008c50       _OPIF_EXTERNALGET          10009c50     lregex.obj
 0001:00008c58       _OPIF_EXTERNALPUT          10009c58     lregex.obj
 0001:00008c60       _OPIF_EXTERNALDELETE       10009c60     lregex.obj
 0001:00008c68       _OPIF_EXTERNALMKDIR        10009c68     lregex.obj
 0001:00008c70       _OPIF_USEATTRHIGHLIGHTING  10009c70     lregex.obj
 0001:00008c78       _OPIF_USECRC32             10009c78     lregex.obj
 0001:00008c80       _OPIF_USEFREESIZE          10009c80     lregex.obj
 0001:00008c88       _OPIF_SHORTCUT             10009c88     lregex.obj
 0001:00008c90       _OPIF_NONE                 10009c90     lregex.obj
 0001:00008c98       _CDF_NONE                  10009c98     lregex.obj
 0001:00008ca0       _FMSG_WARNING              10009ca0     lregex.obj
 0001:00008ca8       _FMSG_ERRORTYPE            10009ca8     lregex.obj
 0001:00008cb0       _FMSG_KEEPBACKGROUND       10009cb0     lregex.obj
 0001:00008cb8       _OPM_SILENT                10009cb8     lregex.obj
 0001:00008cc0       _OPM_FIND                  10009cc0     lregex.obj
 0001:00008cc8       _FMSG_LEFTALIGN            10009cc8     lregex.obj
 0001:00008cd0       _FMSG_ALLINONE             10009cd0     lregex.obj
 0001:00008cd8       _OPM_VIEW                  10009cd8     lregex.obj
 0001:00008ce0       _OPM_EDIT                  10009ce0     lregex.obj
 0001:00008ce8       _FMSG_MB_OK                10009ce8     lregex.obj
 0001:00008cf0       _FMSG_MB_OKCANCEL          10009cf0     lregex.obj
 0001:00008cf8       _OPM_TOPLEVEL              10009cf8     lregex.obj
 0001:00008d00       _OPM_DESCR                 10009d00     lregex.obj
 0001:00008d08       _FMSG_MB_ABORTRETRYIGNORE  10009d08     lregex.obj
 0001:00008d10       _OPM_QUICKVIEW             10009d10     lregex.obj
 0001:00008d18       _FMSG_MB_YESNO             10009d18     lregex.obj
 0001:00008d20       _OPM_PGDN                  10009d20     lregex.obj
 0001:00008d28       _FMSG_MB_YESNOCANCEL       10009d28     lregex.obj
 0001:00008d30       _FMSG_MB_RETRYCANCEL       10009d30     lregex.obj
 0001:00008d38       _OPM_COMMANDS              10009d38     lregex.obj
 0001:00008d40       _OPM_NONE                  10009d40     lregex.obj
 0001:00008d48       _FMSG_NONE                 10009d48     lregex.obj
 0001:00008d50       _FOSF_ACTIVE               10009d50     lregex.obj
 0001:00008d58       _DIF_BOXCOLOR              10009d58     lregex.obj
 0001:00008d60       _FOSF_NONE                 10009d60     lregex.obj
 0001:00008d68       _DIF_GROUP                 10009d68     lregex.obj
 0001:00008d70       _DIF_LEFTTEXT              10009d70     lregex.obj
 0001:00008d78       _DIF_MOVESELECT            10009d78     lregex.obj
 0001:00008d80       _DIF_SHOWAMPERSAND         10009d80     lregex.obj
 0001:00008d88       _DIF_CENTERGROUP           10009d88     lregex.obj
 0001:00008d90       _DIF_NOBRACKETS            10009d90     lregex.obj
 0001:00008d98       _DIF_MANUALADDHISTORY      10009d98     lregex.obj
 0001:00008da0       _DIF_SEPARATOR             10009da0     lregex.obj
 0001:00008da8       _DIF_SEPARATOR2            10009da8     lregex.obj
 0001:00008db0       _DIF_EDITOR                10009db0     lregex.obj
 0001:00008db8       _DIF_LISTNOAMPERSAND       10009db8     lregex.obj
 0001:00008dc0       _DIF_LISTNOBOX             10009dc0     lregex.obj
 0001:00008dc8       _DIF_HISTORY               10009dc8     lregex.obj
 0001:00008e20       _DIF_BTNNOCLOSE            10009e20     lregex.obj
 0001:00008e28       _PDF_DIALOGEVENTDRAWENABLE 10009e28     lregex.obj
 0001:00008e2c       _PDF_PROCESSINGERROR       10009e2c     lregex.obj
 0001:00008e30       _DIF_CENTERTEXT            10009e30     lregex.obj
 0001:00008e38       _DIF_SEPARATORUSER         10009e38     lregex.obj
 0001:00008e40       _DIF_SETSHIELD             10009e40     lregex.obj
 0001:00008e48       _DIF_EDITEXPAND            10009e48     lregex.obj
 0001:00008e50       _DIF_DROPDOWNLIST          10009e50     lregex.obj
 0001:00008e58       _DIF_USELASTHISTORY        10009e58     lregex.obj
 0001:00008e60       _DIF_MASKEDIT              10009e60     lregex.obj
 0001:00008e68       _DIF_LISTTRACKMOUSE        10009e68     lregex.obj
 0001:00008e70       _DIF_LISTTRACKMOUSEINFOCUS 10009e70     lregex.obj
 0001:00008e78       _DIF_SELECTONENTRY         10009e78     lregex.obj
 0001:00008ed0       _DIF_3STATE                10009ed0     lregex.obj
 0001:00008ed8       _DIF_EDITPATH              10009ed8     lregex.obj
 0001:00008ee0       _DIF_LISTWRAPMODE          10009ee0     lregex.obj
 0001:00008ee8       _DIF_NOAUTOCOMPLETE        10009ee8     lregex.obj
 0001:00008ef0       _DIF_LISTAUTOHIGHLIGHT     10009ef0     lregex.obj
 0001:00008ef8       _DIF_LISTNOCLOSE           10009ef8     lregex.obj
 0001:00008f00       _DIF_EDITPATHEXEC          10009f00     lregex.obj
 0001:00008f08       _DIF_HIDDEN                10009f08     lregex.obj
 0001:00008f10       _DIF_READONLY              10009f10     lregex.obj
 0001:00008f18       _DIF_NOFOCUS               10009f18     lregex.obj
 0001:00008f20       _DIF_DISABLE               10009f20     lregex.obj
 0001:00008f28       _DIF_DEFAULTBUTTON         10009f28     lregex.obj
 0001:00008f30       _DIF_FOCUS                 10009f30     lregex.obj
 0001:00008f38       _DIF_RIGHTTEXT             10009f38     lregex.obj
 0001:00008f40       _DIF_WORDWRAP              10009f40     lregex.obj
 0001:00008f48       _DIF_NONE                  10009f48     lregex.obj
 0001:00008f50       _ECF_TABMARKFIRST          10009f50     lregex.obj
 0001:00008f58       _ECF_TABMARKCURRENT        10009f58     lregex.obj
 0001:00008f60       _ECF_AUTODELETE            10009f60     lregex.obj
 0001:00008f68       _ECF_NONE                  10009f68     lregex.obj
 0001:00008f70       _FIB_ENABLEEMPTY           10009f70     lregex.obj
 0001:00008f78       _LIF_SELECTED              10009f78     lregex.obj
 0001:00008f80       _FIB_PASSWORD              10009f80     lregex.obj
 0001:00008f88       _FIB_EXPANDENV             10009f88     lregex.obj
 0001:00008f90       _LIF_CHECKED               10009f90     lregex.obj
 0001:00008f98       _LIF_SEPARATOR             10009f98     lregex.obj
 0001:00008fa0       _FIB_NOUSELASTHISTORY      10009fa0     lregex.obj
 0001:00008fa8       _FIB_BUTTONS               10009fa8     lregex.obj
 0001:00008fb0       _LIF_DISABLE               10009fb0     lregex.obj
 0001:00008fb8       _LIF_GRAYED                10009fb8     lregex.obj
 0001:00008fc0       _FIB_NOAMPERSAND           10009fc0     lregex.obj
 0001:00008fc8       _FIB_EDITPATH              10009fc8     lregex.obj
 0001:00008fd0       _LIF_HIDDEN                10009fd0     lregex.obj
 0001:00008fd8       _LIF_DELETEUSERDATA        10009fd8     lregex.obj
 0001:00008fe0       _FIB_EDITPATHEXEC          10009fe0     lregex.obj
 0001:00008fe8       _LIF_NONE                  10009fe8     lregex.obj
 0001:00008ff0       _FIB_NONE                  10009ff0     lregex.obj
 0001:00008ff8       _PCIF_FROMMAIN             10009ff8     lregex.obj
 0001:00009000       _PCIF_NONE                 1000a000     lregex.obj
 0001:00009008       _LIFIND_EXACTMATCH         1000a008     lregex.obj
 0001:00009010       _LIFIND_NONE               1000a010     lregex.obj
 0001:00009018       _LINFO_SHOWNOBOX           1000a018     lregex.obj
 0001:00009020       _FPF_LOADED                1000a020     lregex.obj
 0001:00009028       _LINFO_AUTOHIGHLIGHT       1000a028     lregex.obj
 0001:00009030       _LINFO_REVERSEHIGHLIGHT    1000a030     lregex.obj
 0001:00009038       _FPF_ANSI                  1000a038     lregex.obj
 0001:00009040       _LINFO_WRAPMODE            1000a040     lregex.obj
 0001:00009048       _FPF_NONE                  1000a048     lregex.obj
 0001:00009050       _LINFO_SHOWAMPERSAND       1000a050     lregex.obj
 0001:00009058       _LINFO_NONE                1000a058     lregex.obj
 0001:00009060       _FarGuid                   1000a060     lregex.obj
 0001:00009070       _FDLG_WARNING              1000a070     lregex.obj
 0001:00009078       _FDLG_SMALLDIALOG          1000a078     lregex.obj
 0001:00009080       _FDLG_NODRAWSHADOW         1000a080     lregex.obj
 0001:00009088       _FDLG_NODRAWPANEL          1000a088     lregex.obj
 0001:00009090       _FDLG_KEEPCONSOLETITLE     1000a090     lregex.obj
 0001:00009098       _FDLG_NONE                 1000a098     lregex.obj
 0001:000090a0       _MIF_SELECTED              1000a0a0     lregex.obj
 0001:000090a8       _MIF_CHECKED               1000a0a8     lregex.obj
 0001:000090b0       _MIF_SEPARATOR             1000a0b0     lregex.obj
 0001:000090b8       _MIF_DISABLE               1000a0b8     lregex.obj
 0001:000090c0       _MIF_GRAYED                1000a0c0     lregex.obj
 0001:000090c8       _MIF_HIDDEN                1000a0c8     lregex.obj
 0001:000090d0       _MIF_NONE                  1000a0d0     lregex.obj
 0001:000090d8       _FMENU_SHOWAMPERSAND       1000a0d8     lregex.obj
 0001:000090e0       _FMENU_WRAPMODE            1000a0e0     lregex.obj
 0001:000090e8       _FMENU_AUTOHIGHLIGHT       1000a0e8     lregex.obj
 0001:000090f0       _FMENU_REVERSEAUTOHIGHLIGHT 1000a0f0     lregex.obj
 0001:000090f8       _FMENU_CHANGECONSOLETITLE  1000a0f8     lregex.obj
 0001:00009100       _FMENU_NONE                1000a100     lregex.obj
 0001:00009108       _PPIF_SELECTED             1000a108     lregex.obj
 0001:00009110       _PPIF_PROCESSDESCR         1000a110     lregex.obj
 0001:00009118       _PPIF_NONE                 1000a118     lregex.obj
 0001:00009120       _PFLAGS_SHOWHIDDEN         1000a120     lregex.obj
 0001:00009128       _PFLAGS_HIGHLIGHT          1000a128     lregex.obj
 0001:00009130       _PFLAGS_REVERSESORTORDER   1000a130     lregex.obj
 0001:00009138       _PFLAGS_USESORTGROUPS      1000a138     lregex.obj
 0001:00009140       _PFLAGS_SELECTEDFIRST      1000a140     lregex.obj
 0001:00009148       _PFLAGS_REALNAMES          1000a148     lregex.obj
 0001:00009150       _PFLAGS_NUMERICSORT        1000a150     lregex.obj
 0001:00009158       _PFLAGS_PANELLEFT          1000a158     lregex.obj
 0001:00009160       _PFLAGS_DIRECTORIESFIRST   1000a160     lregex.obj
 0001:00009168       _PFLAGS_USECRC32           1000a168     lregex.obj
 0001:00009170       _PFLAGS_CASESENSITIVESORT  1000a170     lregex.obj
 0001:00009178       _PFLAGS_PLUGIN             1000a178     lregex.obj
 0001:00009180       _PFLAGS_VISIBLE            1000a180     lregex.obj
 0001:00009188       _PFLAGS_FOCUS              1000a188     lregex.obj
 0001:00009190       _PFLAGS_ALTERNATIVENAMES   1000a190     lregex.obj
 0001:00009198       _PFLAGS_SHORTCUT           1000a198     lregex.obj
 0001:000091a0       _PFLAGS_NONE               1000a1a0     lregex.obj
 0001:000091a8       _PN_CMPNAME                1000a1a8     lregex.obj
 0001:000091b0       _PN_CMPNAMELIST            1000a1b0     lregex.obj
 0001:000091b8       _PN_GENERATENAME           1000a1b8     lregex.obj
 0001:000091c0       _PN_CHECKMASK              1000a1c0     lregex.obj
 0001:000091c8       _PN_SKIPPATH               1000a1c8     lregex.obj
 0001:000091d0       _PN_SHOWERRORMESSAGE       1000a1d0     lregex.obj
 0001:000091d8       _PN_NONE                   1000a1d8     lregex.obj
 0001:000091e0       _XLAT_SWITCHKEYBLAYOUT     1000a1e0     lregex.obj
 0001:000091e8       _XLAT_SWITCHKEYBBEEP       1000a1e8     lregex.obj
 0001:000091f0       _XLAT_USEKEYBLAYOUTNAME    1000a1f0     lregex.obj
 0001:000091f8       _XLAT_CONVERTALLCMDLINE    1000a1f8     lregex.obj
 0001:00009200       _XLAT_NONE                 1000a200     lregex.obj
 0001:00009208       _VF_NONMODAL               1000a208     lregex.obj
 0001:00009210       _VF_DELETEONCLOSE          1000a210     lregex.obj
 0001:00009218       _VF_ENABLE_F6              1000a218     lregex.obj
 0001:00009220       _VF_DISABLEHISTORY         1000a220     lregex.obj
 0001:00009228       _VF_IMMEDIATERETURN        1000a228     lregex.obj
 0001:00009230       _VF_DELETEONLYFILEONCLOSE  1000a230     lregex.obj
 0001:00009238       _VF_NONE                   1000a238     lregex.obj
 0001:00009240       _FRS_RETUPDIR              1000a240     lregex.obj
 0001:00009248       _FRS_RECUR                 1000a248     lregex.obj
 0001:00009250       _FRS_SCANSYMLINK           1000a250     lregex.obj
 0001:00009258       _FRS_NONE                  1000a258     lregex.obj
 0001:00009260       _EF_NONMODAL               1000a260     lregex.obj
 0001:00009268       _EF_CREATENEW              1000a268     lregex.obj
 0001:00009270       _EF_ENABLE_F6              1000a270     lregex.obj
 0001:00009278       _EF_DISABLEHISTORY         1000a278     lregex.obj
 0001:00009280       _EF_DELETEONCLOSE          1000a280     lregex.obj
 0001:00009288       _EF_IMMEDIATERETURN        1000a288     lregex.obj
 0001:00009290       _EF_DELETEONLYFILEONCLOSE  1000a290     lregex.obj
 0001:00009298       _EF_LOCKED                 1000a298     lregex.obj
 0001:000092a0       _EF_DISABLESAVEPOS         1000a2a0     lregex.obj
 0001:000092a8       _EF_OPENMODE_MASK          1000a2a8     lregex.obj
 0001:000092b0       _EF_OPENMODE_QUERY         1000a2b0     lregex.obj
 0001:000092b8       _EF_OPENMODE_NEWIFOPEN     1000a2b8     lregex.obj
 0001:000092c0       _EF_OPENMODE_USEEXISTING   1000a2c0     lregex.obj
 0001:000092c8       _EF_OPENMODE_BREAKIFOPEN   1000a2c8     lregex.obj
 0001:000092d0       _EF_OPENMODE_RELOADIFOPEN  1000a2d0     lregex.obj
 0001:000092d8       _EN_NONE                   1000a2d8     lregex.obj
 0001:000092e0       _MLF_SHOWERRMSG            1000a2e0     lregex.obj
 0001:000092e8       _MLF_DONOTUPDATEPANEL      1000a2e8     lregex.obj
 0001:000092f0       _MLF_HOLDTARGET            1000a2f0     lregex.obj
 0001:000092f8       _MLF_NONE                  1000a2f8     lregex.obj
 0001:00009300       _FHELP_NOSHOWERROR         1000a300     lregex.obj
 0001:00009308       _FHELP_SELFHELP            1000a308     lregex.obj
 0001:00009310       _FHELP_FARHELP             1000a310     lregex.obj
 0001:00009318       _FHELP_CUSTOMFILE          1000a318     lregex.obj
 0001:00009320       _FHELP_CUSTOMPATH          1000a320     lregex.obj
 0001:00009328       _FHELP_GUID                1000a328     lregex.obj
 0001:00009490       _FHELP_USECONTENTS         1000a490     luamacro.obj
 0001:00009498       _FHELP_NONE                1000a498     luamacro.obj
 0001:000094a0       _FFFS_COMMAS               1000a4a0     luamacro.obj
 0001:000094a8       _LuamacroGuid              1000a4a8     luamacro.obj
 0001:000094b8       _FFFS_FLOATSIZE            1000a4b8     luamacro.obj
 0001:000094c0       _FFFS_SHOWBYTESINDEX       1000a4c0     luamacro.obj
 0001:000094c8       _FFFS_ECONOMIC             1000a4c8     luamacro.obj
 0001:000094d0       _FFFS_THOUSAND             1000a4d0     luamacro.obj
 0001:000094d8       _FFFS_MINSIZEINDEX         1000a4d8     luamacro.obj
 0001:000094e0       _FFFS_MINSIZEINDEX_MASK    1000a4e0     luamacro.obj
 0001:000094e8       _FFFS_NONE                 1000a4e8     luamacro.obj
 0001:000094f0       _KMFLAGS_SILENTCHECK       1000a4f0     luamacro.obj
 0001:000094f8       _KMFLAGS_NOSENDKEYSTOPLUGINS 1000a4f8     luamacro.obj
 0001:00009500       _KMFLAGS_ENABLEOUTPUT      1000a500     luamacro.obj
 0001:00009508       _KMFLAGS_LANGMASK          1000a508     luamacro.obj
 0001:00009510       _KMFLAGS_LUA               1000a510     luamacro.obj
 0001:00009518       _KMFLAGS_MOONSCRIPT        1000a518     luamacro.obj
 0001:00009520       _KMFLAGS_NONE              1000a520     luamacro.obj
 0001:00009528       _AKMFLAGS_NONE             1000a528     luamacro.obj
 0001:00009530       _FSETCLR_REDRAW            1000a530     luamacro.obj
 0001:00009538       _FSETCLR_NONE              1000a538     luamacro.obj
 0001:00009540       _WIF_MODIFIED              1000a540     luamacro.obj
 0001:00009548       _WIF_CURRENT               1000a548     luamacro.obj
 0001:00009550       _WIF_MODAL                 1000a550     luamacro.obj
 0001:00009558       _WIF_NONE                  1000a558     luamacro.obj
 0001:00009560       _PF_PRELOAD                1000a560     luamacro.obj
 0001:00009568       _PF_DISABLEPANELS          1000a568     luamacro.obj
 0001:00009570       _PF_EDITOR                 1000a570     luamacro.obj
 0001:00009578       _PF_VIEWER                 1000a578     luamacro.obj
 0001:00009580       _PF_FULLCMDLINE            1000a580     luamacro.obj
 0001:00009588       _PF_DIALOG                 1000a588     luamacro.obj
 0001:00009590       _PF_NONE                   1000a590     luamacro.obj
 0001:00009598       _VOPT_SAVEFILEPOSITION     1000a598     luamacro.obj
 0001:000095a0       _VOPT_AUTODETECTCODEPAGE   1000a5a0     luamacro.obj
 0001:000095a8       _VOPT_SHOWTITLEBAR         1000a5a8     luamacro.obj
 0001:000095b0       _VOPT_SHOWKEYBAR           1000a5b0     luamacro.obj
 0001:000095b8       _VOPT_SHOWSCROLLBAR        1000a5b8     luamacro.obj
 0001:000095c0       _VOPT_QUICKVIEW            1000a5c0     luamacro.obj
 0001:000095c8       _VOPT_NONE                 1000a5c8     luamacro.obj
 0001:000095d0       _VSMFL_REDRAW              1000a5d0     luamacro.obj
 0001:000095d8       _VSMFL_NONE                1000a5d8     luamacro.obj
 0001:000095e0       _VSP_NOREDRAW              1000a5e0     luamacro.obj
 0001:000095e8       _VSP_PERCENT               1000a5e8     luamacro.obj
 0001:000095f0       _VSP_RELATIVE              1000a5f0     luamacro.obj
 0001:000095f8       _VSP_NORETNEWPOS           1000a5f8     luamacro.obj
 0001:00009600       _VSP_NONE                  1000a600     luamacro.obj
 0001:00009608       _IPLFLAGS_SEPARATOR        1000a608     luamacro.obj
 0001:00009610       _IPLFLAGS_NONE             1000a610     luamacro.obj
 0001:00009618       _VMF_WRAP                  1000a618     luamacro.obj
 0001:00009620       _PMFLAGS_FULLSCREEN        1000a620     luamacro.obj
 0001:00009628       _VMF_WORDWRAP              1000a628     luamacro.obj
 0001:00009630       _VMF_NONE                  1000a630     luamacro.obj
 0001:00009638       _PMFLAGS_DETAILEDSTATUS    1000a638     luamacro.obj
 0001:00009640       _PMFLAGS_ALIGNEXTENSIONS   1000a640     luamacro.obj
 0001:00009648       _PMFLAGS_CASECONVERSION    1000a648     luamacro.obj
 0001:00009650       _PMFLAGS_NONE              1000a650     luamacro.obj
 0001:00009658       _FCF_FG_4BIT               1000a658     luamacro.obj
 0001:00009660       _FCF_BG_4BIT               1000a660     luamacro.obj
 0001:00009668       _FCF_4BITMASK              1000a668     luamacro.obj
 0001:00009670       _FCF_RAWATTR_MASK          1000a670     luamacro.obj
 0001:00009678       _FCF_EXTENDEDFLAGS         1000a678     luamacro.obj
 0001:00009680       _FCF_FG_BOLD               1000a680     luamacro.obj
 0001:00009688       _FCF_FG_ITALIC             1000a688     luamacro.obj
 0001:00009690       _FCF_FG_UNDERLINE          1000a690     luamacro.obj
 0001:00009698       _FCF_STYLEMASK             1000a698     luamacro.obj
 0001:000096a0       _OPIF_DISABLEFILTER        1000a6a0     luamacro.obj
 0001:000096a8       _FCF_NONE                  1000a6a8     luamacro.obj
 0001:000096b0       _OPIF_DISABLESORTGROUPS    1000a6b0     luamacro.obj
 0001:000096b8       _OPIF_DISABLEHIGHLIGHTING  1000a6b8     luamacro.obj
 0001:000096c0       _OPIF_ADDDOTS              1000a6c0     luamacro.obj
 0001:000096c8       _OPIF_RAWSELECTION         1000a6c8     luamacro.obj
 0001:000096d0       _OPIF_REALNAMES            1000a6d0     luamacro.obj
 0001:000096d8       _OPIF_SHOWNAMESONLY        1000a6d8     luamacro.obj
 0001:000096e0       _OPIF_SHOWRIGHTALIGNNAMES  1000a6e0     luamacro.obj
 0001:000096e8       _OPIF_SHOWPRESERVECASE     1000a6e8     luamacro.obj
 0001:000096f0       _OPIF_COMPAREFATTIME       1000a6f0     luamacro.obj
 0001:000096f8       _OPIF_EXTERNALGET          1000a6f8     luamacro.obj
 0001:00009700       _OPIF_EXTERNALPUT          1000a700     luamacro.obj
 0001:00009708       _OPIF_EXTERNALDELETE       1000a708     luamacro.obj
 0001:00009710       _OPIF_EXTERNALMKDIR        1000a710     luamacro.obj
 0001:00009718       _OPIF_USEATTRHIGHLIGHTING  1000a718     luamacro.obj
 0001:00009720       _OPIF_USECRC32             1000a720     luamacro.obj
 0001:00009728       _OPIF_USEFREESIZE          1000a728     luamacro.obj
 0001:00009730       _OPIF_SHORTCUT             1000a730     luamacro.obj
 0001:00009738       _OPIF_NONE                 1000a738     luamacro.obj
 0001:00009740       _CDF_NONE                  1000a740     luamacro.obj
 0001:00009748       _FMSG_WARNING              1000a748     luamacro.obj
 0001:00009750       _FMSG_ERRORTYPE            1000a750     luamacro.obj
 0001:00009758       _FMSG_KEEPBACKGROUND       1000a758     luamacro.obj
 0001:00009760       _OPM_SILENT                1000a760     luamacro.obj
 0001:00009768       _OPM_FIND                  1000a768     luamacro.obj
 0001:00009770       _FMSG_LEFTALIGN            1000a770     luamacro.obj
 0001:00009778       _FMSG_ALLINONE             1000a778     luamacro.obj
 0001:00009780       _OPM_VIEW                  1000a780     luamacro.obj
 0001:00009788       _OPM_EDIT                  1000a788     luamacro.obj
 0001:00009790       _FMSG_MB_OK                1000a790     luamacro.obj
 0001:00009798       _FMSG_MB_OKCANCEL          1000a798     luamacro.obj
 0001:000097a0       _OPM_TOPLEVEL              1000a7a0     luamacro.obj
 0001:000097a8       _OPM_DESCR                 1000a7a8     luamacro.obj
 0001:000097b0       _FMSG_MB_ABORTRETRYIGNORE  1000a7b0     luamacro.obj
 0001:000097b8       _OPM_QUICKVIEW             1000a7b8     luamacro.obj
 0001:000097c0       _FMSG_MB_YESNO             1000a7c0     luamacro.obj
 0001:000097c8       _OPM_PGDN                  1000a7c8     luamacro.obj
 0001:000097d0       _FMSG_MB_YESNOCANCEL       1000a7d0     luamacro.obj
 0001:000097d8       _FMSG_MB_RETRYCANCEL       1000a7d8     luamacro.obj
 0001:000097e0       _OPM_COMMANDS              1000a7e0     luamacro.obj
 0001:000097e8       _OPM_NONE                  1000a7e8     luamacro.obj
 0001:000097f0       _FMSG_NONE                 1000a7f0     luamacro.obj
 0001:000097f8       _FOSF_ACTIVE               1000a7f8     luamacro.obj
 0001:00009800       _DIF_BOXCOLOR              1000a800     luamacro.obj
 0001:00009808       _FOSF_NONE                 1000a808     luamacro.obj
 0001:00009810       _DIF_GROUP                 1000a810     luamacro.obj
 0001:00009818       _DIF_LEFTTEXT              1000a818     luamacro.obj
 0001:00009820       _DIF_MOVESELECT            1000a820     luamacro.obj
 0001:00009828       _DIF_SHOWAMPERSAND         1000a828     luamacro.obj
 0001:00009830       _DIF_CENTERGROUP           1000a830     luamacro.obj
 0001:00009838       _DIF_NOBRACKETS            1000a838     luamacro.obj
 0001:00009840       _DIF_MANUALADDHISTORY      1000a840     luamacro.obj
 0001:00009848       _DIF_SEPARATOR             1000a848     luamacro.obj
 0001:00009850       _DIF_SEPARATOR2            1000a850     luamacro.obj
 0001:00009858       _DIF_EDITOR                1000a858     luamacro.obj
 0001:00009860       _DIF_LISTNOAMPERSAND       1000a860     luamacro.obj
 0001:00009868       _DIF_LISTNOBOX             1000a868     luamacro.obj
 0001:00009870       _DIF_HISTORY               1000a870     luamacro.obj
 0001:00009878       _DIF_BTNNOCLOSE            1000a878     luamacro.obj
 0001:00009880       _PDF_DIALOGEVENTDRAWENABLE 1000a880     luamacro.obj
 0001:00009884       _PDF_PROCESSINGERROR       1000a884     luamacro.obj
 0001:00009888       _DIF_CENTERTEXT            1000a888     luamacro.obj
 0001:00009890       _DIF_SEPARATORUSER         1000a890     luamacro.obj
 0001:00009898       _DIF_SETSHIELD             1000a898     luamacro.obj
 0001:000098a0       _DIF_EDITEXPAND            1000a8a0     luamacro.obj
 0001:000098a8       _DIF_DROPDOWNLIST          1000a8a8     luamacro.obj
 0001:000098b0       _DIF_USELASTHISTORY        1000a8b0     luamacro.obj
 0001:000098b8       _DIF_MASKEDIT              1000a8b8     luamacro.obj
 0001:000098c0       _DIF_LISTTRACKMOUSE        1000a8c0     luamacro.obj
 0001:000098c8       _DIF_LISTTRACKMOUSEINFOCUS 1000a8c8     luamacro.obj
 0001:000098d0       _DIF_SELECTONENTRY         1000a8d0     luamacro.obj
 0001:000098d8       _DIF_3STATE                1000a8d8     luamacro.obj
 0001:000098e0       _DIF_EDITPATH              1000a8e0     luamacro.obj
 0001:000098e8       _DIF_LISTWRAPMODE          1000a8e8     luamacro.obj
 0001:000098f0       _DIF_NOAUTOCOMPLETE        1000a8f0     luamacro.obj
 0001:000098f8       _DIF_LISTAUTOHIGHLIGHT     1000a8f8     luamacro.obj
 0001:00009900       _DIF_LISTNOCLOSE           1000a900     luamacro.obj
 0001:00009908       _DIF_EDITPATHEXEC          1000a908     luamacro.obj
 0001:00009910       _DIF_HIDDEN                1000a910     luamacro.obj
 0001:00009918       _DIF_READONLY              1000a918     luamacro.obj
 0001:00009920       _DIF_NOFOCUS               1000a920     luamacro.obj
 0001:00009928       _DIF_DISABLE               1000a928     luamacro.obj
 0001:00009930       _DIF_DEFAULTBUTTON         1000a930     luamacro.obj
 0001:00009938       _DIF_FOCUS                 1000a938     luamacro.obj
 0001:00009940       _DIF_RIGHTTEXT             1000a940     luamacro.obj
 0001:00009948       _DIF_WORDWRAP              1000a948     luamacro.obj
 0001:00009950       _DIF_NONE                  1000a950     luamacro.obj
 0001:00009958       _ECF_TABMARKFIRST          1000a958     luamacro.obj
 0001:00009960       _ECF_TABMARKCURRENT        1000a960     luamacro.obj
 0001:00009968       _ECF_AUTODELETE            1000a968     luamacro.obj
 0001:00009970       _ECF_NONE                  1000a970     luamacro.obj
 0001:00009978       _FIB_ENABLEEMPTY           1000a978     luamacro.obj
 0001:00009980       _LIF_SELECTED              1000a980     luamacro.obj
 0001:00009988       _FIB_PASSWORD              1000a988     luamacro.obj
 0001:00009990       _FIB_EXPANDENV             1000a990     luamacro.obj
 0001:00009998       _LIF_CHECKED               1000a998     luamacro.obj
 0001:000099a0       _LIF_SEPARATOR             1000a9a0     luamacro.obj
 0001:000099a8       _FIB_NOUSELASTHISTORY      1000a9a8     luamacro.obj
 0001:000099b0       _FIB_BUTTONS               1000a9b0     luamacro.obj
 0001:000099b8       _LIF_DISABLE               1000a9b8     luamacro.obj
 0001:000099c0       _LIF_GRAYED                1000a9c0     luamacro.obj
 0001:000099c8       _FIB_NOAMPERSAND           1000a9c8     luamacro.obj
 0001:000099d0       _FIB_EDITPATH              1000a9d0     luamacro.obj
 0001:000099d8       _LIF_HIDDEN                1000a9d8     luamacro.obj
 0001:000099e0       _LIF_DELETEUSERDATA        1000a9e0     luamacro.obj
 0001:000099e8       _FIB_EDITPATHEXEC          1000a9e8     luamacro.obj
 0001:000099f0       _LIF_NONE                  1000a9f0     luamacro.obj
 0001:000099f8       _FIB_NONE                  1000a9f8     luamacro.obj
 0001:00009a00       _PCIF_FROMMAIN             1000aa00     luamacro.obj
 0001:00009a08       _PCIF_NONE                 1000aa08     luamacro.obj
 0001:00009a10       _LIFIND_EXACTMATCH         1000aa10     luamacro.obj
 0001:00009a18       _LIFIND_NONE               1000aa18     luamacro.obj
 0001:00009a20       _LINFO_SHOWNOBOX           1000aa20     luamacro.obj
 0001:00009a28       _FPF_LOADED                1000aa28     luamacro.obj
 0001:00009a30       _LINFO_AUTOHIGHLIGHT       1000aa30     luamacro.obj
 0001:00009a38       _LINFO_REVERSEHIGHLIGHT    1000aa38     luamacro.obj
 0001:00009a40       _FPF_ANSI                  1000aa40     luamacro.obj
 0001:00009a48       _LINFO_WRAPMODE            1000aa48     luamacro.obj
 0001:00009a50       _FPF_NONE                  1000aa50     luamacro.obj
 0001:00009a58       _LINFO_SHOWAMPERSAND       1000aa58     luamacro.obj
 0001:00009a60       _LINFO_NONE                1000aa60     luamacro.obj
 0001:00009a68       _FarGuid                   1000aa68     luamacro.obj
 0001:00009a78       _FDLG_WARNING              1000aa78     luamacro.obj
 0001:00009a80       _FDLG_SMALLDIALOG          1000aa80     luamacro.obj
 0001:00009a88       _FDLG_NODRAWSHADOW         1000aa88     luamacro.obj
 0001:00009a90       _FDLG_NODRAWPANEL          1000aa90     luamacro.obj
 0001:00009a98       _FDLG_KEEPCONSOLETITLE     1000aa98     luamacro.obj
 0001:00009aa0       _FDLG_NONE                 1000aaa0     luamacro.obj
 0001:00009aa8       _MIF_SELECTED              1000aaa8     luamacro.obj
 0001:00009ab0       _MIF_CHECKED               1000aab0     luamacro.obj
 0001:00009ab8       _MIF_SEPARATOR             1000aab8     luamacro.obj
 0001:00009ac0       _MIF_DISABLE               1000aac0     luamacro.obj
 0001:00009ac8       _MIF_GRAYED                1000aac8     luamacro.obj
 0001:00009ad0       _MIF_HIDDEN                1000aad0     luamacro.obj
 0001:00009ad8       _MIF_NONE                  1000aad8     luamacro.obj
 0001:00009ae0       _FMENU_SHOWAMPERSAND       1000aae0     luamacro.obj
 0001:00009ae8       _FMENU_WRAPMODE            1000aae8     luamacro.obj
 0001:00009af0       _FMENU_AUTOHIGHLIGHT       1000aaf0     luamacro.obj
 0001:00009af8       _FMENU_REVERSEAUTOHIGHLIGHT 1000aaf8     luamacro.obj
 0001:00009b00       _FMENU_CHANGECONSOLETITLE  1000ab00     luamacro.obj
 0001:00009b08       _FMENU_NONE                1000ab08     luamacro.obj
 0001:00009b10       _PPIF_SELECTED             1000ab10     luamacro.obj
 0001:00009b18       _PPIF_PROCESSDESCR         1000ab18     luamacro.obj
 0001:00009b20       _PPIF_NONE                 1000ab20     luamacro.obj
 0001:00009b28       _PFLAGS_SHOWHIDDEN         1000ab28     luamacro.obj
 0001:00009b30       _PFLAGS_HIGHLIGHT          1000ab30     luamacro.obj
 0001:00009b38       _PFLAGS_REVERSESORTORDER   1000ab38     luamacro.obj
 0001:00009b40       _PFLAGS_USESORTGROUPS      1000ab40     luamacro.obj
 0001:00009b48       _PFLAGS_SELECTEDFIRST      1000ab48     luamacro.obj
 0001:00009b50       _PFLAGS_REALNAMES          1000ab50     luamacro.obj
 0001:00009b58       _PFLAGS_NUMERICSORT        1000ab58     luamacro.obj
 0001:00009b60       _PFLAGS_PANELLEFT          1000ab60     luamacro.obj
 0001:00009b68       _PFLAGS_DIRECTORIESFIRST   1000ab68     luamacro.obj
 0001:00009b70       _PFLAGS_USECRC32           1000ab70     luamacro.obj
 0001:00009b78       _PFLAGS_CASESENSITIVESORT  1000ab78     luamacro.obj
 0001:00009b80       _PFLAGS_PLUGIN             1000ab80     luamacro.obj
 0001:00009b88       _PFLAGS_VISIBLE            1000ab88     luamacro.obj
 0001:00009b90       _PFLAGS_FOCUS              1000ab90     luamacro.obj
 0001:00009b98       _PFLAGS_ALTERNATIVENAMES   1000ab98     luamacro.obj
 0001:00009ba0       _PFLAGS_SHORTCUT           1000aba0     luamacro.obj
 0001:00009ba8       _PFLAGS_NONE               1000aba8     luamacro.obj
 0001:00009bb0       _PN_CMPNAME                1000abb0     luamacro.obj
 0001:00009bb8       _PN_CMPNAMELIST            1000abb8     luamacro.obj
 0001:00009bc0       _PN_GENERATENAME           1000abc0     luamacro.obj
 0001:00009bc8       _PN_CHECKMASK              1000abc8     luamacro.obj
 0001:00009bd0       _PN_SKIPPATH               1000abd0     luamacro.obj
 0001:00009bd8       _PN_SHOWERRORMESSAGE       1000abd8     luamacro.obj
 0001:00009be0       _PN_NONE                   1000abe0     luamacro.obj
 0001:00009be8       _XLAT_SWITCHKEYBLAYOUT     1000abe8     luamacro.obj
 0001:00009bf0       _XLAT_SWITCHKEYBBEEP       1000abf0     luamacro.obj
 0001:00009bf8       _XLAT_USEKEYBLAYOUTNAME    1000abf8     luamacro.obj
 0001:00009c00       _XLAT_CONVERTALLCMDLINE    1000ac00     luamacro.obj
 0001:00009c08       _XLAT_NONE                 1000ac08     luamacro.obj
 0001:00009c10       _VF_NONMODAL               1000ac10     luamacro.obj
 0001:00009c18       _VF_DELETEONCLOSE          1000ac18     luamacro.obj
 0001:00009c20       _VF_ENABLE_F6              1000ac20     luamacro.obj
 0001:00009c28       _VF_DISABLEHISTORY         1000ac28     luamacro.obj
 0001:00009c30       _VF_IMMEDIATERETURN        1000ac30     luamacro.obj
 0001:00009c38       _VF_DELETEONLYFILEONCLOSE  1000ac38     luamacro.obj
 0001:00009c40       _VF_NONE                   1000ac40     luamacro.obj
 0001:00009c48       _FRS_RETUPDIR              1000ac48     luamacro.obj
 0001:00009c50       _FRS_RECUR                 1000ac50     luamacro.obj
 0001:00009c58       _FRS_SCANSYMLINK           1000ac58     luamacro.obj
 0001:00009c60       _FRS_NONE                  1000ac60     luamacro.obj
 0001:00009c68       _EF_NONMODAL               1000ac68     luamacro.obj
 0001:00009c70       _EF_CREATENEW              1000ac70     luamacro.obj
 0001:00009c78       _EF_ENABLE_F6              1000ac78     luamacro.obj
 0001:00009c80       _EF_DISABLEHISTORY         1000ac80     luamacro.obj
 0001:00009c88       _EF_DELETEONCLOSE          1000ac88     luamacro.obj
 0001:00009c90       _EF_IMMEDIATERETURN        1000ac90     luamacro.obj
 0001:00009c98       _EF_DELETEONLYFILEONCLOSE  1000ac98     luamacro.obj
 0001:00009ca0       _EF_LOCKED                 1000aca0     luamacro.obj
 0001:00009ca8       _EF_DISABLESAVEPOS         1000aca8     luamacro.obj
 0001:00009cb0       _EF_OPENMODE_MASK          1000acb0     luamacro.obj
 0001:00009cb8       _EF_OPENMODE_QUERY         1000acb8     luamacro.obj
 0001:00009cc0       _EF_OPENMODE_NEWIFOPEN     1000acc0     luamacro.obj
 0001:00009cc8       _EF_OPENMODE_USEEXISTING   1000acc8     luamacro.obj
 0001:00009cd0       _EF_OPENMODE_BREAKIFOPEN   1000acd0     luamacro.obj
 0001:00009cd8       _EF_OPENMODE_RELOADIFOPEN  1000acd8     luamacro.obj
 0001:00009ce0       _EN_NONE                   1000ace0     luamacro.obj
 0001:00009ce8       _MLF_SHOWERRMSG            1000ace8     luamacro.obj
 0001:00009cf0       _MLF_DONOTUPDATEPANEL      1000acf0     luamacro.obj
 0001:00009cf8       _MLF_HOLDTARGET            1000acf8     luamacro.obj
 0001:00009d00       _MLF_NONE                  1000ad00     luamacro.obj
 0001:00009d08       _FHELP_NOSHOWERROR         1000ad08     luamacro.obj
 0001:00009d10       _FHELP_SELFHELP            1000ad10     luamacro.obj
 0001:00009d18       _FHELP_FARHELP             1000ad18     luamacro.obj
 0001:00009d20       _FHELP_CUSTOMFILE          1000ad20     luamacro.obj
 0001:00009d28       _FHELP_CUSTOMPATH          1000ad28     luamacro.obj
 0001:00009d30       _FHELP_GUID                1000ad30     luamacro.obj
 0001:00009df8       _FSETCLR_REDRAW            1000adf8     lusercontrol.obj
 0001:00009e00       _FSETCLR_NONE              1000ae00     lusercontrol.obj
 0001:00009e08       _WIF_MODIFIED              1000ae08     lusercontrol.obj
 0001:00009e10       _WIF_CURRENT               1000ae10     lusercontrol.obj
 0001:00009e18       _WIF_MODAL                 1000ae18     lusercontrol.obj
 0001:00009e20       _WIF_NONE                  1000ae20     lusercontrol.obj
 0001:00009e28       _PF_PRELOAD                1000ae28     lusercontrol.obj
 0001:00009e30       _PF_DISABLEPANELS          1000ae30     lusercontrol.obj
 0001:00009e38       _PF_EDITOR                 1000ae38     lusercontrol.obj
 0001:00009e40       _PF_VIEWER                 1000ae40     lusercontrol.obj
 0001:00009e48       _PF_FULLCMDLINE            1000ae48     lusercontrol.obj
 0001:00009e50       _PF_DIALOG                 1000ae50     lusercontrol.obj
 0001:00009e58       _PF_NONE                   1000ae58     lusercontrol.obj
 0001:00009e60       _VOPT_SAVEFILEPOSITION     1000ae60     lusercontrol.obj
 0001:00009e68       _VOPT_AUTODETECTCODEPAGE   1000ae68     lusercontrol.obj
 0001:00009e70       _VOPT_SHOWTITLEBAR         1000ae70     lusercontrol.obj
 0001:00009e78       _VOPT_SHOWKEYBAR           1000ae78     lusercontrol.obj
 0001:00009e80       _VOPT_SHOWSCROLLBAR        1000ae80     lusercontrol.obj
 0001:00009e88       _VOPT_QUICKVIEW            1000ae88     lusercontrol.obj
 0001:00009e90       _VOPT_NONE                 1000ae90     lusercontrol.obj
 0001:00009e98       _VSMFL_REDRAW              1000ae98     lusercontrol.obj
 0001:00009ea0       _VSMFL_NONE                1000aea0     lusercontrol.obj
 0001:00009ea8       _VSP_NOREDRAW              1000aea8     lusercontrol.obj
 0001:00009eb0       _VSP_PERCENT               1000aeb0     lusercontrol.obj
 0001:00009eb8       _VSP_RELATIVE              1000aeb8     lusercontrol.obj
 0001:00009ec0       _VSP_NORETNEWPOS           1000aec0     lusercontrol.obj
 0001:00009ec8       _VSP_NONE                  1000aec8     lusercontrol.obj
 0001:00009ed0       _IPLFLAGS_SEPARATOR        1000aed0     lusercontrol.obj
 0001:00009ed8       _IPLFLAGS_NONE             1000aed8     lusercontrol.obj
 0001:00009ee0       _VMF_WRAP                  1000aee0     lusercontrol.obj
 0001:00009ee8       _PMFLAGS_FULLSCREEN        1000aee8     lusercontrol.obj
 0001:00009ef0       _VMF_WORDWRAP              1000aef0     lusercontrol.obj
 0001:00009ef8       _VMF_NONE                  1000aef8     lusercontrol.obj
 0001:00009f00       _PMFLAGS_DETAILEDSTATUS    1000af00     lusercontrol.obj
 0001:00009f08       _PMFLAGS_ALIGNEXTENSIONS   1000af08     lusercontrol.obj
 0001:00009f10       _PMFLAGS_CASECONVERSION    1000af10     lusercontrol.obj
 0001:00009f18       _PMFLAGS_NONE              1000af18     lusercontrol.obj
 0001:00009f20       _FCF_FG_4BIT               1000af20     lusercontrol.obj
 0001:00009f28       _FCF_BG_4BIT               1000af28     lusercontrol.obj
 0001:00009f30       _FCF_4BITMASK              1000af30     lusercontrol.obj
 0001:00009f38       _FCF_RAWATTR_MASK          1000af38     lusercontrol.obj
 0001:00009f40       _FCF_EXTENDEDFLAGS         1000af40     lusercontrol.obj
 0001:00009f48       _FCF_FG_BOLD               1000af48     lusercontrol.obj
 0001:00009f50       _FCF_FG_ITALIC             1000af50     lusercontrol.obj
 0001:00009f58       _FCF_FG_UNDERLINE          1000af58     lusercontrol.obj
 0001:00009f60       _FCF_STYLEMASK             1000af60     lusercontrol.obj
 0001:00009f68       _OPIF_DISABLEFILTER        1000af68     lusercontrol.obj
 0001:00009f70       _FCF_NONE                  1000af70     lusercontrol.obj
 0001:00009f78       _OPIF_DISABLESORTGROUPS    1000af78     lusercontrol.obj
 0001:00009f80       _OPIF_DISABLEHIGHLIGHTING  1000af80     lusercontrol.obj
 0001:00009f88       _OPIF_ADDDOTS              1000af88     lusercontrol.obj
 0001:00009f90       _OPIF_RAWSELECTION         1000af90     lusercontrol.obj
 0001:00009f98       _OPIF_REALNAMES            1000af98     lusercontrol.obj
 0001:00009fa0       _OPIF_SHOWNAMESONLY        1000afa0     lusercontrol.obj
 0001:00009fa8       _OPIF_SHOWRIGHTALIGNNAMES  1000afa8     lusercontrol.obj
 0001:00009fb0       _OPIF_SHOWPRESERVECASE     1000afb0     lusercontrol.obj
 0001:00009fb8       _OPIF_COMPAREFATTIME       1000afb8     lusercontrol.obj
 0001:00009fc0       _OPIF_EXTERNALGET          1000afc0     lusercontrol.obj
 0001:00009fc8       _OPIF_EXTERNALPUT          1000afc8     lusercontrol.obj
 0001:00009fd0       _OPIF_EXTERNALDELETE       1000afd0     lusercontrol.obj
 0001:00009fd8       _OPIF_EXTERNALMKDIR        1000afd8     lusercontrol.obj
 0001:00009fe0       _OPIF_USEATTRHIGHLIGHTING  1000afe0     lusercontrol.obj
 0001:00009fe8       _OPIF_USECRC32             1000afe8     lusercontrol.obj
 0001:00009ff0       _OPIF_USEFREESIZE          1000aff0     lusercontrol.obj
 0001:00009ff8       _OPIF_SHORTCUT             1000aff8     lusercontrol.obj
 0001:0000a000       _OPIF_NONE                 1000b000     lusercontrol.obj
 0001:0000a008       _CDF_NONE                  1000b008     lusercontrol.obj
 0001:0000a010       _FMSG_WARNING              1000b010     lusercontrol.obj
 0001:0000a018       _FMSG_ERRORTYPE            1000b018     lusercontrol.obj
 0001:0000a020       _FMSG_KEEPBACKGROUND       1000b020     lusercontrol.obj
 0001:0000a028       _OPM_SILENT                1000b028     lusercontrol.obj
 0001:0000a030       _OPM_FIND                  1000b030     lusercontrol.obj
 0001:0000a038       _FMSG_LEFTALIGN            1000b038     lusercontrol.obj
 0001:0000a040       _FMSG_ALLINONE             1000b040     lusercontrol.obj
 0001:0000a048       _OPM_VIEW                  1000b048     lusercontrol.obj
 0001:0000a050       _OPM_EDIT                  1000b050     lusercontrol.obj
 0001:0000a058       _FMSG_MB_OK                1000b058     lusercontrol.obj
 0001:0000a060       _FMSG_MB_OKCANCEL          1000b060     lusercontrol.obj
 0001:0000a068       _OPM_TOPLEVEL              1000b068     lusercontrol.obj
 0001:0000a070       _OPM_DESCR                 1000b070     lusercontrol.obj
 0001:0000a078       _FMSG_MB_ABORTRETRYIGNORE  1000b078     lusercontrol.obj
 0001:0000a080       _OPM_QUICKVIEW             1000b080     lusercontrol.obj
 0001:0000a088       _FMSG_MB_YESNO             1000b088     lusercontrol.obj
 0001:0000a090       _OPM_PGDN                  1000b090     lusercontrol.obj
 0001:0000a098       _FMSG_MB_YESNOCANCEL       1000b098     lusercontrol.obj
 0001:0000a0a0       _FMSG_MB_RETRYCANCEL       1000b0a0     lusercontrol.obj
 0001:0000a0a8       _OPM_COMMANDS              1000b0a8     lusercontrol.obj
 0001:0000a0b0       _OPM_NONE                  1000b0b0     lusercontrol.obj
 0001:0000a0b8       _FMSG_NONE                 1000b0b8     lusercontrol.obj
 0001:0000a0c0       _FOSF_ACTIVE               1000b0c0     lusercontrol.obj
 0001:0000a0c8       _DIF_BOXCOLOR              1000b0c8     lusercontrol.obj
 0001:0000a0d0       _FOSF_NONE                 1000b0d0     lusercontrol.obj
 0001:0000a0d8       _DIF_GROUP                 1000b0d8     lusercontrol.obj
 0001:0000a0e0       _DIF_LEFTTEXT              1000b0e0     lusercontrol.obj
 0001:0000a0e8       _DIF_MOVESELECT            1000b0e8     lusercontrol.obj
 0001:0000a0f0       _DIF_SHOWAMPERSAND         1000b0f0     lusercontrol.obj
 0001:0000a0f8       _DIF_CENTERGROUP           1000b0f8     lusercontrol.obj
 0001:0000a100       _DIF_NOBRACKETS            1000b100     lusercontrol.obj
 0001:0000a108       _DIF_MANUALADDHISTORY      1000b108     lusercontrol.obj
 0001:0000a110       _DIF_SEPARATOR             1000b110     lusercontrol.obj
 0001:0000a118       _DIF_SEPARATOR2            1000b118     lusercontrol.obj
 0001:0000a120       _DIF_EDITOR                1000b120     lusercontrol.obj
 0001:0000a128       _DIF_LISTNOAMPERSAND       1000b128     lusercontrol.obj
 0001:0000a130       _DIF_LISTNOBOX             1000b130     lusercontrol.obj
 0001:0000a138       _DIF_HISTORY               1000b138     lusercontrol.obj
 0001:0000a140       _DIF_BTNNOCLOSE            1000b140     lusercontrol.obj
 0001:0000a148       _DIF_CENTERTEXT            1000b148     lusercontrol.obj
 0001:0000a150       _DIF_SEPARATORUSER         1000b150     lusercontrol.obj
 0001:0000a158       _DIF_SETSHIELD             1000b158     lusercontrol.obj
 0001:0000a160       _DIF_EDITEXPAND            1000b160     lusercontrol.obj
 0001:0000a168       _DIF_DROPDOWNLIST          1000b168     lusercontrol.obj
 0001:0000a170       _DIF_USELASTHISTORY        1000b170     lusercontrol.obj
 0001:0000a178       _DIF_MASKEDIT              1000b178     lusercontrol.obj
 0001:0000a180       _DIF_LISTTRACKMOUSE        1000b180     lusercontrol.obj
 0001:0000a188       _DIF_LISTTRACKMOUSEINFOCUS 1000b188     lusercontrol.obj
 0001:0000a190       _DIF_SELECTONENTRY         1000b190     lusercontrol.obj
 0001:0000a198       _DIF_3STATE                1000b198     lusercontrol.obj
 0001:0000a1a0       _DIF_EDITPATH              1000b1a0     lusercontrol.obj
 0001:0000a1a8       _DIF_LISTWRAPMODE          1000b1a8     lusercontrol.obj
 0001:0000a1b0       _DIF_NOAUTOCOMPLETE        1000b1b0     lusercontrol.obj
 0001:0000a1b8       _DIF_LISTAUTOHIGHLIGHT     1000b1b8     lusercontrol.obj
 0001:0000a1c0       _DIF_LISTNOCLOSE           1000b1c0     lusercontrol.obj
 0001:0000a1c8       _DIF_EDITPATHEXEC          1000b1c8     lusercontrol.obj
 0001:0000a1d0       _DIF_HIDDEN                1000b1d0     lusercontrol.obj
 0001:0000a1d8       _DIF_READONLY              1000b1d8     lusercontrol.obj
 0001:0000a1e0       _DIF_NOFOCUS               1000b1e0     lusercontrol.obj
 0001:0000a1e8       _DIF_DISABLE               1000b1e8     lusercontrol.obj
 0001:0000a1f0       _DIF_DEFAULTBUTTON         1000b1f0     lusercontrol.obj
 0001:0000a1f8       _DIF_FOCUS                 1000b1f8     lusercontrol.obj
 0001:0000a200       _DIF_RIGHTTEXT             1000b200     lusercontrol.obj
 0001:0000a208       _DIF_WORDWRAP              1000b208     lusercontrol.obj
 0001:0000a210       _DIF_NONE                  1000b210     lusercontrol.obj
 0001:0000a218       _ECF_TABMARKFIRST          1000b218     lusercontrol.obj
 0001:0000a220       _ECF_TABMARKCURRENT        1000b220     lusercontrol.obj
 0001:0000a228       _ECF_AUTODELETE            1000b228     lusercontrol.obj
 0001:0000a230       _ECF_NONE                  1000b230     lusercontrol.obj
 0001:0000a238       _FIB_ENABLEEMPTY           1000b238     lusercontrol.obj
 0001:0000a240       _LIF_SELECTED              1000b240     lusercontrol.obj
 0001:0000a248       _FIB_PASSWORD              1000b248     lusercontrol.obj
 0001:0000a250       _FIB_EXPANDENV             1000b250     lusercontrol.obj
 0001:0000a258       _LIF_CHECKED               1000b258     lusercontrol.obj
 0001:0000a260       _LIF_SEPARATOR             1000b260     lusercontrol.obj
 0001:0000a268       _FIB_NOUSELASTHISTORY      1000b268     lusercontrol.obj
 0001:0000a270       _FIB_BUTTONS               1000b270     lusercontrol.obj
 0001:0000a278       _LIF_DISABLE               1000b278     lusercontrol.obj
 0001:0000a280       _LIF_GRAYED                1000b280     lusercontrol.obj
 0001:0000a288       _FIB_NOAMPERSAND           1000b288     lusercontrol.obj
 0001:0000a290       _FIB_EDITPATH              1000b290     lusercontrol.obj
 0001:0000a298       _LIF_HIDDEN                1000b298     lusercontrol.obj
 0001:0000a2a0       _LIF_DELETEUSERDATA        1000b2a0     lusercontrol.obj
 0001:0000a2a8       _FIB_EDITPATHEXEC          1000b2a8     lusercontrol.obj
 0001:0000a2b0       _LIF_NONE                  1000b2b0     lusercontrol.obj
 0001:0000a2b8       _FIB_NONE                  1000b2b8     lusercontrol.obj
 0001:0000a2c0       _PCIF_FROMMAIN             1000b2c0     lusercontrol.obj
 0001:0000a2c8       _PCIF_NONE                 1000b2c8     lusercontrol.obj
 0001:0000a2d0       _LIFIND_EXACTMATCH         1000b2d0     lusercontrol.obj
 0001:0000a2d8       _LIFIND_NONE               1000b2d8     lusercontrol.obj
 0001:0000a2e0       _LINFO_SHOWNOBOX           1000b2e0     lusercontrol.obj
 0001:0000a2e8       _FPF_LOADED                1000b2e8     lusercontrol.obj
 0001:0000a2f0       _LINFO_AUTOHIGHLIGHT       1000b2f0     lusercontrol.obj
 0001:0000a2f8       _LINFO_REVERSEHIGHLIGHT    1000b2f8     lusercontrol.obj
 0001:0000a300       _FPF_ANSI                  1000b300     lusercontrol.obj
 0001:0000a308       _LINFO_WRAPMODE            1000b308     lusercontrol.obj
 0001:0000a310       _FPF_NONE                  1000b310     lusercontrol.obj
 0001:0000a318       _LINFO_SHOWAMPERSAND       1000b318     lusercontrol.obj
 0001:0000a320       _LINFO_NONE                1000b320     lusercontrol.obj
 0001:0000a328       _FarGuid                   1000b328     lusercontrol.obj
 0001:0000a338       _FDLG_WARNING              1000b338     lusercontrol.obj
 0001:0000a340       _FDLG_SMALLDIALOG          1000b340     lusercontrol.obj
 0001:0000a348       _FDLG_NODRAWSHADOW         1000b348     lusercontrol.obj
 0001:0000a350       _FDLG_NODRAWPANEL          1000b350     lusercontrol.obj
 0001:0000a358       _FDLG_KEEPCONSOLETITLE     1000b358     lusercontrol.obj
 0001:0000a360       _FDLG_NONE                 1000b360     lusercontrol.obj
 0001:0000a368       _MIF_SELECTED              1000b368     lusercontrol.obj
 0001:0000a370       _MIF_CHECKED               1000b370     lusercontrol.obj
 0001:0000a378       _MIF_SEPARATOR             1000b378     lusercontrol.obj
 0001:0000a380       _MIF_DISABLE               1000b380     lusercontrol.obj
 0001:0000a388       _MIF_GRAYED                1000b388     lusercontrol.obj
 0001:0000a390       _MIF_HIDDEN                1000b390     lusercontrol.obj
 0001:0000a398       _MIF_NONE                  1000b398     lusercontrol.obj
 0001:0000a3a0       _FMENU_SHOWAMPERSAND       1000b3a0     lusercontrol.obj
 0001:0000a3a8       _FMENU_WRAPMODE            1000b3a8     lusercontrol.obj
 0001:0000a3b0       _FMENU_AUTOHIGHLIGHT       1000b3b0     lusercontrol.obj
 0001:0000a3b8       _FMENU_REVERSEAUTOHIGHLIGHT 1000b3b8     lusercontrol.obj
 0001:0000a3c0       _FMENU_CHANGECONSOLETITLE  1000b3c0     lusercontrol.obj
 0001:0000a3c8       _FMENU_NONE                1000b3c8     lusercontrol.obj
 0001:0000a3d0       _PPIF_SELECTED             1000b3d0     lusercontrol.obj
 0001:0000a3d8       _PPIF_PROCESSDESCR         1000b3d8     lusercontrol.obj
 0001:0000a3e0       _PPIF_NONE                 1000b3e0     lusercontrol.obj
 0001:0000a3e8       _PFLAGS_SHOWHIDDEN         1000b3e8     lusercontrol.obj
 0001:0000a3f0       _PFLAGS_HIGHLIGHT          1000b3f0     lusercontrol.obj
 0001:0000a3f8       _PFLAGS_REVERSESORTORDER   1000b3f8     lusercontrol.obj
 0001:0000a400       _PFLAGS_USESORTGROUPS      1000b400     lusercontrol.obj
 0001:0000a408       _PFLAGS_SELECTEDFIRST      1000b408     lusercontrol.obj
 0001:0000a410       _PFLAGS_REALNAMES          1000b410     lusercontrol.obj
 0001:0000a418       _PFLAGS_NUMERICSORT        1000b418     lusercontrol.obj
 0001:0000a420       _PFLAGS_PANELLEFT          1000b420     lusercontrol.obj
 0001:0000a428       _PFLAGS_DIRECTORIESFIRST   1000b428     lusercontrol.obj
 0001:0000a430       _PFLAGS_USECRC32           1000b430     lusercontrol.obj
 0001:0000a438       _PFLAGS_CASESENSITIVESORT  1000b438     lusercontrol.obj
 0001:0000a440       _PFLAGS_PLUGIN             1000b440     lusercontrol.obj
 0001:0000a448       _PFLAGS_VISIBLE            1000b448     lusercontrol.obj
 0001:0000a450       _PFLAGS_FOCUS              1000b450     lusercontrol.obj
 0001:0000a458       _PFLAGS_ALTERNATIVENAMES   1000b458     lusercontrol.obj
 0001:0000a460       _PFLAGS_SHORTCUT           1000b460     lusercontrol.obj
 0001:0000a468       _PFLAGS_NONE               1000b468     lusercontrol.obj
 0001:0000a470       _PN_CMPNAME                1000b470     lusercontrol.obj
 0001:0000a478       _PN_CMPNAMELIST            1000b478     lusercontrol.obj
 0001:0000a480       _PN_GENERATENAME           1000b480     lusercontrol.obj
 0001:0000a488       _PN_CHECKMASK              1000b488     lusercontrol.obj
 0001:0000a490       _PN_SKIPPATH               1000b490     lusercontrol.obj
 0001:0000a498       _PN_SHOWERRORMESSAGE       1000b498     lusercontrol.obj
 0001:0000a4a0       _PN_NONE                   1000b4a0     lusercontrol.obj
 0001:0000a4a8       _XLAT_SWITCHKEYBLAYOUT     1000b4a8     lusercontrol.obj
 0001:0000a4b0       _XLAT_SWITCHKEYBBEEP       1000b4b0     lusercontrol.obj
 0001:0000a4b8       _XLAT_USEKEYBLAYOUTNAME    1000b4b8     lusercontrol.obj
 0001:0000a4c0       _XLAT_CONVERTALLCMDLINE    1000b4c0     lusercontrol.obj
 0001:0000a4c8       _XLAT_NONE                 1000b4c8     lusercontrol.obj
 0001:0000a4d0       _VF_NONMODAL               1000b4d0     lusercontrol.obj
 0001:0000a4d8       _VF_DELETEONCLOSE          1000b4d8     lusercontrol.obj
 0001:0000a4e0       _VF_ENABLE_F6              1000b4e0     lusercontrol.obj
 0001:0000a4e8       _VF_DISABLEHISTORY         1000b4e8     lusercontrol.obj
 0001:0000a4f0       _VF_IMMEDIATERETURN        1000b4f0     lusercontrol.obj
 0001:0000a4f8       _VF_DELETEONLYFILEONCLOSE  1000b4f8     lusercontrol.obj
 0001:0000a500       _VF_NONE                   1000b500     lusercontrol.obj
 0001:0000a508       _FRS_RETUPDIR              1000b508     lusercontrol.obj
 0001:0000a538       _FRS_RECUR                 1000b538     lusercontrol.obj
 0001:0000a540       _FRS_SCANSYMLINK           1000b540     lusercontrol.obj
 0001:0000a548       _FRS_NONE                  1000b548     lusercontrol.obj
 0001:0000a560       _EF_NONMODAL               1000b560     lusercontrol.obj
 0001:0000a568       _EF_CREATENEW              1000b568     lusercontrol.obj
 0001:0000a570       _EF_ENABLE_F6              1000b570     lusercontrol.obj
 0001:0000a578       _EF_DISABLEHISTORY         1000b578     lusercontrol.obj
 0001:0000a580       _EF_DELETEONCLOSE          1000b580     lusercontrol.obj
 0001:0000a588       _EF_IMMEDIATERETURN        1000b588     lusercontrol.obj
 0001:0000a590       _EF_DELETEONLYFILEONCLOSE  1000b590     lusercontrol.obj
 0001:0000a598       _EF_LOCKED                 1000b598     lusercontrol.obj
 0001:0000a5a0       _EF_DISABLESAVEPOS         1000b5a0     lusercontrol.obj
 0001:0000a5a8       _EF_OPENMODE_MASK          1000b5a8     lusercontrol.obj
 0001:0000a5b0       _EF_OPENMODE_QUERY         1000b5b0     lusercontrol.obj
 0001:0000a5b8       _EF_OPENMODE_NEWIFOPEN     1000b5b8     lusercontrol.obj
 0001:0000a5c0       _EF_OPENMODE_USEEXISTING   1000b5c0     lusercontrol.obj
 0001:0000a5c8       _EF_OPENMODE_BREAKIFOPEN   1000b5c8     lusercontrol.obj
 0001:0000a5d0       _EF_OPENMODE_RELOADIFOPEN  1000b5d0     lusercontrol.obj
 0001:0000a5d8       _EN_NONE                   1000b5d8     lusercontrol.obj
 0001:0000a5e0       _MLF_SHOWERRMSG            1000b5e0     lusercontrol.obj
 0001:0000a5e8       _MLF_DONOTUPDATEPANEL      1000b5e8     lusercontrol.obj
 0001:0000a5f0       _MLF_HOLDTARGET            1000b5f0     lusercontrol.obj
 0001:0000a5f8       _MLF_NONE                  1000b5f8     lusercontrol.obj
 0001:0000a600       _FHELP_NOSHOWERROR         1000b600     lusercontrol.obj
 0001:0000a608       _FHELP_SELFHELP            1000b608     lusercontrol.obj
 0001:0000a610       _FHELP_FARHELP             1000b610     lusercontrol.obj
 0001:0000a618       _FHELP_CUSTOMFILE          1000b618     lusercontrol.obj
 0001:0000a620       _FHELP_CUSTOMPATH          1000b620     lusercontrol.obj
 0001:0000a628       _FHELP_GUID                1000b628     lusercontrol.obj
 0001:0000a630       _FHELP_USECONTENTS         1000b630     lusercontrol.obj
 0001:0000a638       _FHELP_NONE                1000b638     lusercontrol.obj
 0001:0000a640       _FFFS_COMMAS               1000b640     lusercontrol.obj
 0001:0000a648       _FFFS_FLOATSIZE            1000b648     lusercontrol.obj
 0001:0000a650       _FFFS_SHOWBYTESINDEX       1000b650     lusercontrol.obj
 0001:0000a658       _FFFS_ECONOMIC             1000b658     lusercontrol.obj
 0001:0000a660       _FFFS_THOUSAND             1000b660     lusercontrol.obj
 0001:0000a668       _FFFS_MINSIZEINDEX         1000b668     lusercontrol.obj
 0001:0000a670       _FFFS_MINSIZEINDEX_MASK    1000b670     lusercontrol.obj
 0001:0000a678       _FFFS_NONE                 1000b678     lusercontrol.obj
 0001:0000a680       _KMFLAGS_SILENTCHECK       1000b680     lusercontrol.obj
 0001:0000a688       _KMFLAGS_NOSENDKEYSTOPLUGINS 1000b688     lusercontrol.obj
 0001:0000a690       _KMFLAGS_ENABLEOUTPUT      1000b690     lusercontrol.obj
 0001:0000a698       _KMFLAGS_LANGMASK          1000b698     lusercontrol.obj
 0001:0000a6a0       _KMFLAGS_LUA               1000b6a0     lusercontrol.obj
 0001:0000a6a8       _KMFLAGS_MOONSCRIPT        1000b6a8     lusercontrol.obj
 0001:0000a6b0       _KMFLAGS_NONE              1000b6b0     lusercontrol.obj
 0001:0000a6b8       _AKMFLAGS_NONE             1000b6b8     lusercontrol.obj
 0001:0000a758       _FHELP_NOSHOWERROR         1000b758     service.obj
 0001:0000a760       _FHELP_SELFHELP            1000b760     service.obj
 0001:0000a768       _FHELP_FARHELP             1000b768     service.obj
 0001:0000a770       _FHELP_CUSTOMFILE          1000b770     service.obj
 0001:0000a778       _FHELP_CUSTOMPATH          1000b778     service.obj
 0001:0000a780       _FHELP_GUID                1000b780     service.obj
 0001:0000a788       _FHELP_USECONTENTS         1000b788     service.obj
 0001:0000a790       _FHELP_NONE                1000b790     service.obj
 0001:0000a798       _FFFS_COMMAS               1000b798     service.obj
 0001:0000a7a0       _FFFS_FLOATSIZE            1000b7a0     service.obj
 0001:0000a7a8       _FFFS_SHOWBYTESINDEX       1000b7a8     service.obj
 0001:0000a7b0       _FFFS_ECONOMIC             1000b7b0     service.obj
 0001:0000a7b8       _FFFS_THOUSAND             1000b7b8     service.obj
 0001:0000a7c0       _FFFS_MINSIZEINDEX         1000b7c0     service.obj
 0001:0000a7c8       _FFFS_MINSIZEINDEX_MASK    1000b7c8     service.obj
 0001:0000a7d0       _FFFS_NONE                 1000b7d0     service.obj
 0001:0000a7d8       ?C@?3??far_InputRecordToName@@9@9 1000b7d8     service.obj
 0001:0000a7e0       ?A@?3??far_InputRecordToName@@9@9 1000b7e0     service.obj
 0001:0000a7e8       ?S@?3??far_InputRecordToName@@9@9 1000b7e8     service.obj
 0001:0000a7f0       _KMFLAGS_SILENTCHECK       1000b7f0     service.obj
 0001:0000a7f8       _KMFLAGS_NOSENDKEYSTOPLUGINS 1000b7f8     service.obj
 0001:0000a800       _KMFLAGS_ENABLEOUTPUT      1000b800     service.obj
 0001:0000a808       _KMFLAGS_LANGMASK          1000b808     service.obj
 0001:0000a810       _KMFLAGS_LUA               1000b810     service.obj
 0001:0000a818       _KMFLAGS_MOONSCRIPT        1000b818     service.obj
 0001:0000a820       _KMFLAGS_NONE              1000b820     service.obj
 0001:0000a850       _AKMFLAGS_NONE             1000b850     service.obj
 0001:0000aaa0       _FSETCLR_REDRAW            1000baa0     service.obj
 0001:0000aaa8       _FSETCLR_NONE              1000baa8     service.obj
 0001:0000abc8       _WIF_MODIFIED              1000bbc8     service.obj
 0001:0000abd0       _WIF_CURRENT               1000bbd0     service.obj
 0001:0000abd8       _WIF_MODAL                 1000bbd8     service.obj
 0001:0000abe0       _WIF_NONE                  1000bbe0     service.obj
 0001:0000abe8       _PF_PRELOAD                1000bbe8     service.obj
 0001:0000abf0       _PF_DISABLEPANELS          1000bbf0     service.obj
 0001:0000abf8       _PF_EDITOR                 1000bbf8     service.obj
 0001:0000ac00       _PF_VIEWER                 1000bc00     service.obj
 0001:0000ac08       _PF_FULLCMDLINE            1000bc08     service.obj
 0001:0000ac10       _PF_DIALOG                 1000bc10     service.obj
 0001:0000ac18       _PF_NONE                   1000bc18     service.obj
 0001:0000ae60       _VOPT_SAVEFILEPOSITION     1000be60     service.obj
 0001:0000ae68       _VOPT_AUTODETECTCODEPAGE   1000be68     service.obj
 0001:0000ae70       _VOPT_SHOWTITLEBAR         1000be70     service.obj
 0001:0000ae78       _VOPT_SHOWKEYBAR           1000be78     service.obj
 0001:0000ae80       _VOPT_SHOWSCROLLBAR        1000be80     service.obj
 0001:0000ae88       _VOPT_QUICKVIEW            1000be88     service.obj
 0001:0000ae90       _VOPT_NONE                 1000be90     service.obj
 0001:0000ae98       _VSMFL_REDRAW              1000be98     service.obj
 0001:0000aea0       _VSMFL_NONE                1000bea0     service.obj
 0001:0000aea8       _VSP_NOREDRAW              1000bea8     service.obj
 0001:0000aeb0       _VSP_PERCENT               1000beb0     service.obj
 0001:0000aeb8       _VSP_RELATIVE              1000beb8     service.obj
 0001:0000aec0       _VSP_NORETNEWPOS           1000bec0     service.obj
 0001:0000aec8       _VSP_NONE                  1000bec8     service.obj
 0001:0000aed0       _IPLFLAGS_SEPARATOR        1000bed0     service.obj
 0001:0000aed8       _IPLFLAGS_NONE             1000bed8     service.obj
 0001:0000aee0       _VMF_WRAP                  1000bee0     service.obj
 0001:0000aee8       _PMFLAGS_FULLSCREEN        1000bee8     service.obj
 0001:0000aef0       _VMF_WORDWRAP              1000bef0     service.obj
 0001:0000aef8       _VMF_NONE                  1000bef8     service.obj
 0001:0000af00       _PMFLAGS_DETAILEDSTATUS    1000bf00     service.obj
 0001:0000af08       _PMFLAGS_ALIGNEXTENSIONS   1000bf08     service.obj
 0001:0000af10       _PMFLAGS_CASECONVERSION    1000bf10     service.obj
 0001:0000af18       _PMFLAGS_NONE              1000bf18     service.obj
 0001:0000af20       _FCF_FG_4BIT               1000bf20     service.obj
 0001:0000af28       _FCF_BG_4BIT               1000bf28     service.obj
 0001:0000af30       _FCF_4BITMASK              1000bf30     service.obj
 0001:0000af38       _FCF_RAWATTR_MASK          1000bf38     service.obj
 0001:0000af40       _FCF_EXTENDEDFLAGS         1000bf40     service.obj
 0001:0000af48       _FCF_FG_BOLD               1000bf48     service.obj
 0001:0000af50       _FCF_FG_ITALIC             1000bf50     service.obj
 0001:0000af58       _FCF_FG_UNDERLINE          1000bf58     service.obj
 0001:0000af60       _FCF_STYLEMASK             1000bf60     service.obj
 0001:0000af68       _OPIF_DISABLEFILTER        1000bf68     service.obj
 0001:0000af70       _FCF_NONE                  1000bf70     service.obj
 0001:0000af78       _OPIF_DISABLESORTGROUPS    1000bf78     service.obj
 0001:0000af80       _OPIF_DISABLEHIGHLIGHTING  1000bf80     service.obj
 0001:0000af88       _OPIF_ADDDOTS              1000bf88     service.obj
 0001:0000af90       _OPIF_RAWSELECTION         1000bf90     service.obj
 0001:0000af98       _OPIF_REALNAMES            1000bf98     service.obj
 0001:0000afa0       _OPIF_SHOWNAMESONLY        1000bfa0     service.obj
 0001:0000b1d8       _OPIF_SHOWRIGHTALIGNNAMES  1000c1d8     service.obj
 0001:0000b1e0       _OPIF_SHOWPRESERVECASE     1000c1e0     service.obj
 0001:0000b1e8       _OPIF_COMPAREFATTIME       1000c1e8     service.obj
 0001:0000b1f0       _OPIF_EXTERNALGET          1000c1f0     service.obj
 0001:0000b1f8       _OPIF_EXTERNALPUT          1000c1f8     service.obj
 0001:0000b200       _OPIF_EXTERNALDELETE       1000c200     service.obj
 0001:0000b208       _OPIF_EXTERNALMKDIR        1000c208     service.obj
 0001:0000b210       _OPIF_USEATTRHIGHLIGHTING  1000c210     service.obj
 0001:0000b218       _OPIF_USECRC32             1000c218     service.obj
 0001:0000b220       _OPIF_USEFREESIZE          1000c220     service.obj
 0001:0000b228       _OPIF_SHORTCUT             1000c228     service.obj
 0001:0000b230       _OPIF_NONE                 1000c230     service.obj
 0001:0000b238       _CDF_NONE                  1000c238     service.obj
 0001:0000b250       _FMSG_WARNING              1000c250     service.obj
 0001:0000b270       _FMSG_ERRORTYPE            1000c270     service.obj
 0001:0000b278       _FMSG_KEEPBACKGROUND       1000c278     service.obj
 0001:0000b280       _OPM_SILENT                1000c280     service.obj
 0001:0000b288       _OPM_FIND                  1000c288     service.obj
 0001:0000b290       _FMSG_LEFTALIGN            1000c290     service.obj
 0001:0000b2b8       _FMSG_ALLINONE             1000c2b8     service.obj
 0001:0000b2c0       _OPM_VIEW                  1000c2c0     service.obj
 0001:0000b2d8       _OPM_EDIT                  1000c2d8     service.obj
 0001:0000b2e0       _FMSG_MB_OK                1000c2e0     service.obj
 0001:0000b2f8       _FMSG_MB_OKCANCEL          1000c2f8     service.obj
 0001:0000b300       _OPM_TOPLEVEL              1000c300     service.obj
 0001:0000b308       _OPM_DESCR                 1000c308     service.obj
 0001:0000b310       _FMSG_MB_ABORTRETRYIGNORE  1000c310     service.obj
 0001:0000b338       _OPM_QUICKVIEW             1000c338     service.obj
 0001:0000b340       _FMSG_MB_YESNO             1000c340     service.obj
 0001:0000b348       _OPM_PGDN                  1000c348     service.obj
 0001:0000b350       _FMSG_MB_YESNOCANCEL       1000c350     service.obj
 0001:0000b374       _PDF_DIALOGEVENTDRAWENABLE 1000c374     service.obj
 0001:0000b378       _FMSG_MB_RETRYCANCEL       1000c378     service.obj
 0001:0000b380       _OPM_COMMANDS              1000c380     service.obj
 0001:0000b388       _OPM_NONE                  1000c388     service.obj
 0001:0000b390       _FMSG_NONE                 1000c390     service.obj
 0001:0000b398       _lualibs                   1000c398     service.obj
 0001:0000b3f8       _FOSF_ACTIVE               1000c3f8     service.obj
 0001:0000b400       _DIF_BOXCOLOR              1000c400     service.obj
 0001:0000b408       _FOSF_NONE                 1000c408     service.obj
 0001:0000b410       _DIF_GROUP                 1000c410     service.obj
 0001:0000b418       _DIF_LEFTTEXT              1000c418     service.obj
 0001:0000b420       _DIF_MOVESELECT            1000c420     service.obj
 0001:0000b428       _DIF_SHOWAMPERSAND         1000c428     service.obj
 0001:0000b430       _DIF_CENTERGROUP           1000c430     service.obj
 0001:0000b438       _DIF_NOBRACKETS            1000c438     service.obj
 0001:0000b440       _DIF_MANUALADDHISTORY      1000c440     service.obj
 0001:0000b448       _DIF_SEPARATOR             1000c448     service.obj
 0001:0000b450       _DIF_SEPARATOR2            1000c450     service.obj
 0001:0000b458       _DIF_EDITOR                1000c458     service.obj
 0001:0000b460       _DIF_LISTNOAMPERSAND       1000c460     service.obj
 0001:0000b468       _DIF_LISTNOBOX             1000c468     service.obj
 0001:0000b470       _DIF_HISTORY               1000c470     service.obj
 0001:0000b478       _DIF_BTNNOCLOSE            1000c478     service.obj
 0001:0000b480       _DIF_CENTERTEXT            1000c480     service.obj
 0001:0000b488       _DIF_SEPARATORUSER         1000c488     service.obj
 0001:0000b490       _DIF_SETSHIELD             1000c490     service.obj
 0001:0000b498       _PDF_PROCESSINGERROR       1000c498     service.obj
 0001:0000b4a0       _DIF_EDITEXPAND            1000c4a0     service.obj
 0001:0000b4a8       _DIF_DROPDOWNLIST          1000c4a8     service.obj
 0001:0000b4b0       _DIF_USELASTHISTORY        1000c4b0     service.obj
 0001:0000b4b8       _DIF_MASKEDIT              1000c4b8     service.obj
 0001:0000b4c0       _DIF_LISTTRACKMOUSE        1000c4c0     service.obj
 0001:0000b4c8       _DIF_LISTTRACKMOUSEINFOCUS 1000c4c8     service.obj
 0001:0000b4d0       _DIF_SELECTONENTRY         1000c4d0     service.obj
 0001:0000b4d8       _DIF_3STATE                1000c4d8     service.obj
 0001:0000b4e0       _DIF_EDITPATH              1000c4e0     service.obj
 0001:0000b4e8       _DIF_LISTWRAPMODE          1000c4e8     service.obj
 0001:0000b4f0       _DIF_NOAUTOCOMPLETE        1000c4f0     service.obj
 0001:0000b4f8       _DIF_LISTAUTOHIGHLIGHT     1000c4f8     service.obj
 0001:0000b500       _DIF_LISTNOCLOSE           1000c500     service.obj
 0001:0000b508       _DIF_EDITPATHEXEC          1000c508     service.obj
 0001:0000b510       _DIF_HIDDEN                1000c510     service.obj
 0001:0000b518       _DIF_READONLY              1000c518     service.obj
 0001:0000b520       _DIF_NOFOCUS               1000c520     service.obj
 0001:0000b528       _DIF_DISABLE               1000c528     service.obj
 0001:0000b530       _DIF_DEFAULTBUTTON         1000c530     service.obj
 0001:0000b538       _DIF_FOCUS                 1000c538     service.obj
 0001:0000b540       _DIF_RIGHTTEXT             1000c540     service.obj
 0001:0000b548       _DIF_WORDWRAP              1000c548     service.obj
 0001:0000b550       _DIF_NONE                  1000c550     service.obj
 0001:0000b5b8       _ECF_TABMARKFIRST          1000c5b8     service.obj
 0001:0000b5c0       _ECF_TABMARKCURRENT        1000c5c0     service.obj
 0001:0000b5c8       _ECF_AUTODELETE            1000c5c8     service.obj
 0001:0000b5d0       _ECF_NONE                  1000c5d0     service.obj
 0001:0000b5d8       _FIB_ENABLEEMPTY           1000c5d8     service.obj
 0001:0000b5e0       _LIF_SELECTED              1000c5e0     service.obj
 0001:0000b5e8       _FIB_PASSWORD              1000c5e8     service.obj
 0001:0000b5f0       _FIB_EXPANDENV             1000c5f0     service.obj
 0001:0000b5f8       _LIF_CHECKED               1000c5f8     service.obj
 0001:0000b600       _LIF_SEPARATOR             1000c600     service.obj
 0001:0000b608       _FIB_NOUSELASTHISTORY      1000c608     service.obj
 0001:0000b610       _FIB_BUTTONS               1000c610     service.obj
 0001:0000b618       _LIF_DISABLE               1000c618     service.obj
 0001:0000b620       _LIF_GRAYED                1000c620     service.obj
 0001:0000b628       _FIB_NOAMPERSAND           1000c628     service.obj
 0001:0000b630       _FIB_EDITPATH              1000c630     service.obj
 0001:0000b638       _LIF_HIDDEN                1000c638     service.obj
 0001:0000b640       _LIF_DELETEUSERDATA        1000c640     service.obj
 0001:0000b648       _FIB_EDITPATHEXEC          1000c648     service.obj
 0001:0000b650       _LIF_NONE                  1000c650     service.obj
 0001:0000b658       _FIB_NONE                  1000c658     service.obj
 0001:0000b660       _PCIF_FROMMAIN             1000c660     service.obj
 0001:0000b668       _PCIF_NONE                 1000c668     service.obj
 0001:0000b670       _LIFIND_EXACTMATCH         1000c670     service.obj
 0001:0000b678       _LIFIND_NONE               1000c678     service.obj
 0001:0000b680       _LINFO_SHOWNOBOX           1000c680     service.obj
 0001:0000b688       _FPF_LOADED                1000c688     service.obj
 0001:0000b690       _LINFO_AUTOHIGHLIGHT       1000c690     service.obj
 0001:0000b698       _LINFO_REVERSEHIGHLIGHT    1000c698     service.obj
 0001:0000b6a0       _FPF_ANSI                  1000c6a0     service.obj
 0001:0000b6a8       _LINFO_WRAPMODE            1000c6a8     service.obj
 0001:0000b6b0       _FPF_NONE                  1000c6b0     service.obj
 0001:0000b6b8       _LINFO_SHOWAMPERSAND       1000c6b8     service.obj
 0001:0000b6c0       _LINFO_NONE                1000c6c0     service.obj
 0001:0000b6c8       _FarGuid                   1000c6c8     service.obj
 0001:0000b6d8       ?key@?3??far_Menu@@9@9     1000c6d8     service.obj
 0001:0000b6e0       _FDLG_WARNING              1000c6e0     service.obj
 0001:0000b6e8       _FDLG_SMALLDIALOG          1000c6e8     service.obj
 0001:0000b6f0       _FDLG_NODRAWSHADOW         1000c6f0     service.obj
 0001:0000b6f8       _FDLG_NODRAWPANEL          1000c6f8     service.obj
 0001:0000b700       _FDLG_KEEPCONSOLETITLE     1000c700     service.obj
 0001:0000b708       _FDLG_NONE                 1000c708     service.obj
 0001:0000b710       _MIF_SELECTED              1000c710     service.obj
 0001:0000b718       _MIF_CHECKED               1000c718     service.obj
 0001:0000b720       _MIF_SEPARATOR             1000c720     service.obj
 0001:0000b728       _MIF_DISABLE               1000c728     service.obj
 0001:0000b730       _MIF_GRAYED                1000c730     service.obj
 0001:0000b738       _MIF_HIDDEN                1000c738     service.obj
 0001:0000b740       _MIF_NONE                  1000c740     service.obj
 0001:0000b748       _FMENU_SHOWAMPERSAND       1000c748     service.obj
 0001:0000b750       _FMENU_WRAPMODE            1000c750     service.obj
 0001:0000b758       _FMENU_AUTOHIGHLIGHT       1000c758     service.obj
 0001:0000b760       _FMENU_REVERSEAUTOHIGHLIGHT 1000c760     service.obj
 0001:0000b768       _FMENU_CHANGECONSOLETITLE  1000c768     service.obj
 0001:0000b770       _FMENU_NONE                1000c770     service.obj
 0001:0000b778       _PPIF_SELECTED             1000c778     service.obj
 0001:0000b780       _PPIF_PROCESSDESCR         1000c780     service.obj
 0001:0000b788       _PPIF_NONE                 1000c788     service.obj
 0001:0000b790       _PFLAGS_SHOWHIDDEN         1000c790     service.obj
 0001:0000b798       _PFLAGS_HIGHLIGHT          1000c798     service.obj
 0001:0000b7a0       _PFLAGS_REVERSESORTORDER   1000c7a0     service.obj
 0001:0000b7a8       _PFLAGS_USESORTGROUPS      1000c7a8     service.obj
 0001:0000b7b0       _PFLAGS_SELECTEDFIRST      1000c7b0     service.obj
 0001:0000b7b8       _PFLAGS_REALNAMES          1000c7b8     service.obj
 0001:0000b7c0       _PFLAGS_NUMERICSORT        1000c7c0     service.obj
 0001:0000b7c8       _PFLAGS_PANELLEFT          1000c7c8     service.obj
 0001:0000b7d0       _PFLAGS_DIRECTORIESFIRST   1000c7d0     service.obj
 0001:0000b7d8       _PFLAGS_USECRC32           1000c7d8     service.obj
 0001:0000b7e0       _PFLAGS_CASESENSITIVESORT  1000c7e0     service.obj
 0001:0000b7e8       _PFLAGS_PLUGIN             1000c7e8     service.obj
 0001:0000b7f0       _PFLAGS_VISIBLE            1000c7f0     service.obj
 0001:0000b7f8       _PFLAGS_FOCUS              1000c7f8     service.obj
 0001:0000b800       _PFLAGS_ALTERNATIVENAMES   1000c800     service.obj
 0001:0000b808       _PFLAGS_SHORTCUT           1000c808     service.obj
 0001:0000b810       _PFLAGS_NONE               1000c810     service.obj
 0001:0000b818       _PN_CMPNAME                1000c818     service.obj
 0001:0000b820       _PN_CMPNAMELIST            1000c820     service.obj
 0001:0000b828       _PN_GENERATENAME           1000c828     service.obj
 0001:0000b830       _PN_CHECKMASK              1000c830     service.obj
 0001:0000b838       _PN_SKIPPATH               1000c838     service.obj
 0001:0000b840       _PN_SHOWERRORMESSAGE       1000c840     service.obj
 0001:0000b848       _PN_NONE                   1000c848     service.obj
 0001:0000b850       _XLAT_SWITCHKEYBLAYOUT     1000c850     service.obj
 0001:0000b858       _XLAT_SWITCHKEYBBEEP       1000c858     service.obj
 0001:0000b860       _XLAT_USEKEYBLAYOUTNAME    1000c860     service.obj
 0001:0000b868       _XLAT_CONVERTALLCMDLINE    1000c868     service.obj
 0001:0000b870       _XLAT_NONE                 1000c870     service.obj
 0001:0000b878       ?FarGuid@?1??far_CreateSettings@@9@9 1000c878     service.obj
 0001:0000b888       _VF_NONMODAL               1000c888     service.obj
 0001:0000b890       _VF_DELETEONCLOSE          1000c890     service.obj
 0001:0000b898       _VF_ENABLE_F6              1000c898     service.obj
 0001:0000b8a0       _VF_DISABLEHISTORY         1000c8a0     service.obj
 0001:0000b8a8       _VF_IMMEDIATERETURN        1000c8a8     service.obj
 0001:0000b8b0       _VF_DELETEONLYFILEONCLOSE  1000c8b0     service.obj
 0001:0000b8b8       _VF_NONE                   1000c8b8     service.obj
 0001:0000b8c0       _FRS_RETUPDIR              1000c8c0     service.obj
 0001:0000b8c8       _FRS_RECUR                 1000c8c8     service.obj
 0001:0000b8d0       _FRS_SCANSYMLINK           1000c8d0     service.obj
 0001:0000b8d8       _FRS_NONE                  1000c8d8     service.obj
 0001:0000b8e0       _EF_NONMODAL               1000c8e0     service.obj
 0001:0000b8e8       _EF_CREATENEW              1000c8e8     service.obj
 0001:0000b8f0       _EF_ENABLE_F6              1000c8f0     service.obj
 0001:0000b8f8       _EF_DISABLEHISTORY         1000c8f8     service.obj
 0001:0000b900       _EF_DELETEONCLOSE          1000c900     service.obj
 0001:0000b908       _EF_IMMEDIATERETURN        1000c908     service.obj
 0001:0000b910       _EF_DELETEONLYFILEONCLOSE  1000c910     service.obj
 0001:0000b918       _EF_LOCKED                 1000c918     service.obj
 0001:0000b920       _EF_DISABLESAVEPOS         1000c920     service.obj
 0001:0000b928       _EF_OPENMODE_MASK          1000c928     service.obj
 0001:0000b930       _EF_OPENMODE_QUERY         1000c930     service.obj
 0001:0000b938       _EF_OPENMODE_NEWIFOPEN     1000c938     service.obj
 0001:0000b940       _EF_OPENMODE_USEEXISTING   1000c940     service.obj
 0001:0000b948       _EF_OPENMODE_BREAKIFOPEN   1000c948     service.obj
 0001:0000b950       _EF_OPENMODE_RELOADIFOPEN  1000c950     service.obj
 0001:0000b958       _EN_NONE                   1000c958     service.obj
 0001:0000b960       _MLF_SHOWERRMSG            1000c960     service.obj
 0001:0000b968       _MLF_DONOTUPDATEPANEL      1000c968     service.obj
 0001:0000b970       _MLF_HOLDTARGET            1000c970     service.obj
 0001:0000b978       _MLF_NONE                  1000c978     service.obj
 0001:0000d3a0       _uniclib                   1000e3a0     slnunico.obj
 0001:0000d6c8       _fnames                    1000e6c8     uliolib51.obj
 0001:0000d6d0       ?mode@?1??f_seek@@9@9      1000e6d0     uliolib51.obj
 0001:0000d6dc       ?modenames@?1??f_seek@@9@9 1000e6dc     uliolib51.obj
 0001:0000d6ec       ?mode@?1??f_setvbuf@@9@9   1000e6ec     uliolib51.obj
 0001:0000d6f8       ?modenames@?1??f_setvbuf@@9@9 1000e6f8     uliolib51.obj
 0001:0000d708       _iolib                     1000e708     uliolib51.obj
 0001:0000d768       _flib                      1000e768     uliolib51.obj
 0001:0000d978       _sentinel_                 1000e978     uloadlib51.obj
 0001:0000d97c       _pk_funcs                  1000e97c     uloadlib51.obj
 0001:0000d994       _ll_funcs                  1000e994     uloadlib51.obj
 0001:0000d9ac       _loaders                   1000e9ac     uloadlib51.obj
 0001:0000e0f0       _FSETCLR_REDRAW            1000f0f0     util.obj
 0001:0000e0f8       _FSETCLR_NONE              1000f0f8     util.obj
 0001:0000e100       _WIF_MODIFIED              1000f100     util.obj
 0001:0000e108       _WIF_CURRENT               1000f108     util.obj
 0001:0000e110       _WIF_MODAL                 1000f110     util.obj
 0001:0000e118       _WIF_NONE                  1000f118     util.obj
 0001:0000e120       _PF_PRELOAD                1000f120     util.obj
 0001:0000e128       _PF_DISABLEPANELS          1000f128     util.obj
 0001:0000e130       _PF_EDITOR                 1000f130     util.obj
 0001:0000e138       _PF_VIEWER                 1000f138     util.obj
 0001:0000e140       _PF_FULLCMDLINE            1000f140     util.obj
 0001:0000e148       _PF_DIALOG                 1000f148     util.obj
 0001:0000e150       _PF_NONE                   1000f150     util.obj
 0001:0000e158       _VOPT_SAVEFILEPOSITION     1000f158     util.obj
 0001:0000e160       _VOPT_AUTODETECTCODEPAGE   1000f160     util.obj
 0001:0000e168       _VOPT_SHOWTITLEBAR         1000f168     util.obj
 0001:0000e170       _VOPT_SHOWKEYBAR           1000f170     util.obj
 0001:0000e178       _VOPT_SHOWSCROLLBAR        1000f178     util.obj
 0001:0000e180       _VOPT_QUICKVIEW            1000f180     util.obj
 0001:0000e188       _VOPT_NONE                 1000f188     util.obj
 0001:0000e190       _VSMFL_REDRAW              1000f190     util.obj
 0001:0000e198       _VSMFL_NONE                1000f198     util.obj
 0001:0000e1a0       _VSP_NOREDRAW              1000f1a0     util.obj
 0001:0000e1a8       _VSP_PERCENT               1000f1a8     util.obj
 0001:0000e1b0       _VSP_RELATIVE              1000f1b0     util.obj
 0001:0000e1b8       _VSP_NORETNEWPOS           1000f1b8     util.obj
 0001:0000e1c0       _VSP_NONE                  1000f1c0     util.obj
 0001:0000e1c8       _IPLFLAGS_SEPARATOR        1000f1c8     util.obj
 0001:0000e1d0       _IPLFLAGS_NONE             1000f1d0     util.obj
 0001:0000e1d8       _VMF_WRAP                  1000f1d8     util.obj
 0001:0000e1e0       _PMFLAGS_FULLSCREEN        1000f1e0     util.obj
 0001:0000e1e8       _VMF_WORDWRAP              1000f1e8     util.obj
 0001:0000e1f0       _VMF_NONE                  1000f1f0     util.obj
 0001:0000e1f8       _PMFLAGS_DETAILEDSTATUS    1000f1f8     util.obj
 0001:0000e200       _PMFLAGS_ALIGNEXTENSIONS   1000f200     util.obj
 0001:0000e208       _PMFLAGS_CASECONVERSION    1000f208     util.obj
 0001:0000e210       _PMFLAGS_NONE              1000f210     util.obj
 0001:0000e218       _FCF_FG_4BIT               1000f218     util.obj
 0001:0000e220       _FCF_BG_4BIT               1000f220     util.obj
 0001:0000e228       _FCF_4BITMASK              1000f228     util.obj
 0001:0000e230       _FCF_RAWATTR_MASK          1000f230     util.obj
 0001:0000e238       _FCF_EXTENDEDFLAGS         1000f238     util.obj
 0001:0000e240       _FCF_FG_BOLD               1000f240     util.obj
 0001:0000e248       _FCF_FG_ITALIC             1000f248     util.obj
 0001:0000e250       _FCF_FG_UNDERLINE          1000f250     util.obj
 0001:0000e258       _FCF_STYLEMASK             1000f258     util.obj
 0001:0000e260       _OPIF_DISABLEFILTER        1000f260     util.obj
 0001:0000e268       _FCF_NONE                  1000f268     util.obj
 0001:0000e270       _OPIF_DISABLESORTGROUPS    1000f270     util.obj
 0001:0000e278       _OPIF_DISABLEHIGHLIGHTING  1000f278     util.obj
 0001:0000e280       _OPIF_ADDDOTS              1000f280     util.obj
 0001:0000e288       _OPIF_RAWSELECTION         1000f288     util.obj
 0001:0000e290       _OPIF_REALNAMES            1000f290     util.obj
 0001:0000e298       _OPIF_SHOWNAMESONLY        1000f298     util.obj
 0001:0000e2a0       _OPIF_SHOWRIGHTALIGNNAMES  1000f2a0     util.obj
 0001:0000e2a8       _OPIF_SHOWPRESERVECASE     1000f2a8     util.obj
 0001:0000e2b0       _OPIF_COMPAREFATTIME       1000f2b0     util.obj
 0001:0000e2b8       _OPIF_EXTERNALGET          1000f2b8     util.obj
 0001:0000e2c0       _OPIF_EXTERNALPUT          1000f2c0     util.obj
 0001:0000e2c8       _OPIF_EXTERNALDELETE       1000f2c8     util.obj
 0001:0000e2d0       _OPIF_EXTERNALMKDIR        1000f2d0     util.obj
 0001:0000e2d8       _OPIF_USEATTRHIGHLIGHTING  1000f2d8     util.obj
 0001:0000e2e0       _OPIF_USECRC32             1000f2e0     util.obj
 0001:0000e2e8       _OPIF_USEFREESIZE          1000f2e8     util.obj
 0001:0000e2f0       _OPIF_SHORTCUT             1000f2f0     util.obj
 0001:0000e2f8       _OPIF_NONE                 1000f2f8     util.obj
 0001:0000e300       _CDF_NONE                  1000f300     util.obj
 0001:0000e308       _FMSG_WARNING              1000f308     util.obj
 0001:0000e310       _FMSG_ERRORTYPE            1000f310     util.obj
 0001:0000e318       _FMSG_KEEPBACKGROUND       1000f318     util.obj
 0001:0000e320       _OPM_SILENT                1000f320     util.obj
 0001:0000e328       _OPM_FIND                  1000f328     util.obj
 0001:0000e330       _FMSG_LEFTALIGN            1000f330     util.obj
 0001:0000e338       _FMSG_ALLINONE             1000f338     util.obj
 0001:0000e340       _OPM_VIEW                  1000f340     util.obj
 0001:0000e348       _OPM_EDIT                  1000f348     util.obj
 0001:0000e350       _FMSG_MB_OK                1000f350     util.obj
 0001:0000e358       _FMSG_MB_OKCANCEL          1000f358     util.obj
 0001:0000e360       _OPM_TOPLEVEL              1000f360     util.obj
 0001:0000e368       _OPM_DESCR                 1000f368     util.obj
 0001:0000e370       _FMSG_MB_ABORTRETRYIGNORE  1000f370     util.obj
 0001:0000e378       _OPM_QUICKVIEW             1000f378     util.obj
 0001:0000e380       _FMSG_MB_YESNO             1000f380     util.obj
 0001:0000e388       _OPM_PGDN                  1000f388     util.obj
 0001:0000e390       _FMSG_MB_YESNOCANCEL       1000f390     util.obj
 0001:0000e398       _FMSG_MB_RETRYCANCEL       1000f398     util.obj
 0001:0000e3a0       _OPM_COMMANDS              1000f3a0     util.obj
 0001:0000e3a8       _OPM_NONE                  1000f3a8     util.obj
 0001:0000e3b0       _FMSG_NONE                 1000f3b0     util.obj
 0001:0000e3b8       _FOSF_ACTIVE               1000f3b8     util.obj
 0001:0000e3c0       _DIF_BOXCOLOR              1000f3c0     util.obj
 0001:0000e3c8       _FOSF_NONE                 1000f3c8     util.obj
 0001:0000e3d0       _DIF_GROUP                 1000f3d0     util.obj
 0001:0000e3d8       _DIF_LEFTTEXT              1000f3d8     util.obj
 0001:0000e3e0       _DIF_MOVESELECT            1000f3e0     util.obj
 0001:0000e3e8       _DIF_SHOWAMPERSAND         1000f3e8     util.obj
 0001:0000e3f0       _DIF_CENTERGROUP           1000f3f0     util.obj
 0001:0000e3f8       _DIF_NOBRACKETS            1000f3f8     util.obj
 0001:0000e400       _DIF_MANUALADDHISTORY      1000f400     util.obj
 0001:0000e408       _DIF_SEPARATOR             1000f408     util.obj
 0001:0000e410       _DIF_SEPARATOR2            1000f410     util.obj
 0001:0000e418       _DIF_EDITOR                1000f418     util.obj
 0001:0000e420       _DIF_LISTNOAMPERSAND       1000f420     util.obj
 0001:0000e428       _DIF_LISTNOBOX             1000f428     util.obj
 0001:0000e430       _DIF_HISTORY               1000f430     util.obj
 0001:0000e438       _DIF_BTNNOCLOSE            1000f438     util.obj
 0001:0000e440       _DIF_CENTERTEXT            1000f440     util.obj
 0001:0000e448       _DIF_SEPARATORUSER         1000f448     util.obj
 0001:0000e450       _DIF_SETSHIELD             1000f450     util.obj
 0001:0000e458       _DIF_EDITEXPAND            1000f458     util.obj
 0001:0000e460       _DIF_DROPDOWNLIST          1000f460     util.obj
 0001:0000e468       _DIF_USELASTHISTORY        1000f468     util.obj
 0001:0000e470       _DIF_MASKEDIT              1000f470     util.obj
 0001:0000e478       _DIF_LISTTRACKMOUSE        1000f478     util.obj
 0001:0000e480       _DIF_LISTTRACKMOUSEINFOCUS 1000f480     util.obj
 0001:0000e488       _DIF_SELECTONENTRY         1000f488     util.obj
 0001:0000e490       _DIF_3STATE                1000f490     util.obj
 0001:0000e498       _DIF_EDITPATH              1000f498     util.obj
 0001:0000e4a0       _DIF_LISTWRAPMODE          1000f4a0     util.obj
 0001:0000e4a8       _DIF_NOAUTOCOMPLETE        1000f4a8     util.obj
 0001:0000e4b0       _DIF_LISTAUTOHIGHLIGHT     1000f4b0     util.obj
 0001:0000e4b8       _DIF_LISTNOCLOSE           1000f4b8     util.obj
 0001:0000e4c0       _DIF_EDITPATHEXEC          1000f4c0     util.obj
 0001:0000e4c8       _DIF_HIDDEN                1000f4c8     util.obj
 0001:0000e4d0       _DIF_READONLY              1000f4d0     util.obj
 0001:0000e4d8       _DIF_NOFOCUS               1000f4d8     util.obj
 0001:0000e4e0       _DIF_DISABLE               1000f4e0     util.obj
 0001:0000e4e8       _DIF_DEFAULTBUTTON         1000f4e8     util.obj
 0001:0000e4f0       _DIF_FOCUS                 1000f4f0     util.obj
 0001:0000e4f8       _DIF_RIGHTTEXT             1000f4f8     util.obj
 0001:0000e500       _DIF_WORDWRAP              1000f500     util.obj
 0001:0000e508       _DIF_NONE                  1000f508     util.obj
 0001:0000e510       _ECF_TABMARKFIRST          1000f510     util.obj
 0001:0000e518       _ECF_TABMARKCURRENT        1000f518     util.obj
 0001:0000e520       _ECF_AUTODELETE            1000f520     util.obj
 0001:0000e528       _ECF_NONE                  1000f528     util.obj
 0001:0000e530       _FIB_ENABLEEMPTY           1000f530     util.obj
 0001:0000e538       _LIF_SELECTED              1000f538     util.obj
 0001:0000e540       _FIB_PASSWORD              1000f540     util.obj
 0001:0000e548       _FIB_EXPANDENV             1000f548     util.obj
 0001:0000e550       _LIF_CHECKED               1000f550     util.obj
 0001:0000e558       _LIF_SEPARATOR             1000f558     util.obj
 0001:0000e560       _FIB_NOUSELASTHISTORY      1000f560     util.obj
 0001:0000e568       _FIB_BUTTONS               1000f568     util.obj
 0001:0000e570       _LIF_DISABLE               1000f570     util.obj
 0001:0000e578       _LIF_GRAYED                1000f578     util.obj
 0001:0000e580       _FIB_NOAMPERSAND           1000f580     util.obj
 0001:0000e588       _FIB_EDITPATH              1000f588     util.obj
 0001:0000e590       _LIF_HIDDEN                1000f590     util.obj
 0001:0000e598       _LIF_DELETEUSERDATA        1000f598     util.obj
 0001:0000e5a0       _FIB_EDITPATHEXEC          1000f5a0     util.obj
 0001:0000e5a8       _LIF_NONE                  1000f5a8     util.obj
 0001:0000e5b0       _FIB_NONE                  1000f5b0     util.obj
 0001:0000e5b8       _PCIF_FROMMAIN             1000f5b8     util.obj
 0001:0000e5c0       _PCIF_NONE                 1000f5c0     util.obj
 0001:0000e5c8       _LIFIND_EXACTMATCH         1000f5c8     util.obj
 0001:0000e5d0       _LIFIND_NONE               1000f5d0     util.obj
 0001:0000e5d8       _LINFO_SHOWNOBOX           1000f5d8     util.obj
 0001:0000e5e0       _FPF_LOADED                1000f5e0     util.obj
 0001:0000e5e8       _LINFO_AUTOHIGHLIGHT       1000f5e8     util.obj
 0001:0000e5f0       _LINFO_REVERSEHIGHLIGHT    1000f5f0     util.obj
 0001:0000e5f8       _FPF_ANSI                  1000f5f8     util.obj
 0001:0000e600       _LINFO_WRAPMODE            1000f600     util.obj
 0001:0000e608       _FPF_NONE                  1000f608     util.obj
 0001:0000e610       _LINFO_SHOWAMPERSAND       1000f610     util.obj
 0001:0000e618       _LINFO_NONE                1000f618     util.obj
 0001:0000e620       _FarGuid                   1000f620     util.obj
 0001:0000e630       _FDLG_WARNING              1000f630     util.obj
 0001:0000e638       _FDLG_SMALLDIALOG          1000f638     util.obj
 0001:0000e640       _FDLG_NODRAWSHADOW         1000f640     util.obj
 0001:0000e648       _FDLG_NODRAWPANEL          1000f648     util.obj
 0001:0000e650       _FDLG_KEEPCONSOLETITLE     1000f650     util.obj
 0001:0000e658       _FDLG_NONE                 1000f658     util.obj
 0001:0000e660       _MIF_SELECTED              1000f660     util.obj
 0001:0000e668       _MIF_CHECKED               1000f668     util.obj
 0001:0000e670       _MIF_SEPARATOR             1000f670     util.obj
 0001:0000e678       _MIF_DISABLE               1000f678     util.obj
 0001:0000e680       _MIF_GRAYED                1000f680     util.obj
 0001:0000e688       _MIF_HIDDEN                1000f688     util.obj
 0001:0000e690       _MIF_NONE                  1000f690     util.obj
 0001:0000e698       _FMENU_SHOWAMPERSAND       1000f698     util.obj
 0001:0000e6a0       _FMENU_WRAPMODE            1000f6a0     util.obj
 0001:0000e6a8       _FMENU_AUTOHIGHLIGHT       1000f6a8     util.obj
 0001:0000e6b0       _FMENU_REVERSEAUTOHIGHLIGHT 1000f6b0     util.obj
 0001:0000e6b8       _FMENU_CHANGECONSOLETITLE  1000f6b8     util.obj
 0001:0000e6c0       _FMENU_NONE                1000f6c0     util.obj
 0001:0000e6c8       _PPIF_SELECTED             1000f6c8     util.obj
 0001:0000e6d0       _PPIF_PROCESSDESCR         1000f6d0     util.obj
 0001:0000e6d8       _PPIF_NONE                 1000f6d8     util.obj
 0001:0000e6e0       _PFLAGS_SHOWHIDDEN         1000f6e0     util.obj
 0001:0000e6e8       _PFLAGS_HIGHLIGHT          1000f6e8     util.obj
 0001:0000e6f0       _PFLAGS_REVERSESORTORDER   1000f6f0     util.obj
 0001:0000e6f8       _PFLAGS_USESORTGROUPS      1000f6f8     util.obj
 0001:0000e700       _PFLAGS_SELECTEDFIRST      1000f700     util.obj
 0001:0000e708       _PFLAGS_REALNAMES          1000f708     util.obj
 0001:0000e710       _PFLAGS_NUMERICSORT        1000f710     util.obj
 0001:0000e718       _PFLAGS_PANELLEFT          1000f718     util.obj
 0001:0000e720       _PFLAGS_DIRECTORIESFIRST   1000f720     util.obj
 0001:0000e728       _PFLAGS_USECRC32           1000f728     util.obj
 0001:0000e730       _PFLAGS_CASESENSITIVESORT  1000f730     util.obj
 0001:0000e738       _PFLAGS_PLUGIN             1000f738     util.obj
 0001:0000e740       _PFLAGS_VISIBLE            1000f740     util.obj
 0001:0000e748       _PFLAGS_FOCUS              1000f748     util.obj
 0001:0000e750       _PFLAGS_ALTERNATIVENAMES   1000f750     util.obj
 0001:0000e758       _PFLAGS_SHORTCUT           1000f758     util.obj
 0001:0000e760       _PFLAGS_NONE               1000f760     util.obj
 0001:0000e768       _PN_CMPNAME                1000f768     util.obj
 0001:0000e770       _PN_CMPNAMELIST            1000f770     util.obj
 0001:0000e778       _PN_GENERATENAME           1000f778     util.obj
 0001:0000e780       _PN_CHECKMASK              1000f780     util.obj
 0001:0000e788       _PN_SKIPPATH               1000f788     util.obj
 0001:0000e790       _PN_SHOWERRORMESSAGE       1000f790     util.obj
 0001:0000e798       _PN_NONE                   1000f798     util.obj
 0001:0000e7a0       _XLAT_SWITCHKEYBLAYOUT     1000f7a0     util.obj
 0001:0000e7a8       _XLAT_SWITCHKEYBBEEP       1000f7a8     util.obj
 0001:0000e7b0       _XLAT_USEKEYBLAYOUTNAME    1000f7b0     util.obj
 0001:0000e7b8       _XLAT_CONVERTALLCMDLINE    1000f7b8     util.obj
 0001:0000e7c0       _XLAT_NONE                 1000f7c0     util.obj
 0001:0000e7c8       _VF_NONMODAL               1000f7c8     util.obj
 0001:0000e7d0       _VF_DELETEONCLOSE          1000f7d0     util.obj
 0001:0000e7d8       _VF_ENABLE_F6              1000f7d8     util.obj
 0001:0000e7e0       _VF_DISABLEHISTORY         1000f7e0     util.obj
 0001:0000e7e8       _VF_IMMEDIATERETURN        1000f7e8     util.obj
 0001:0000e7f0       _VF_DELETEONLYFILEONCLOSE  1000f7f0     util.obj
 0001:0000e7f8       _VF_NONE                   1000f7f8     util.obj
 0001:0000e800       _FRS_RETUPDIR              1000f800     util.obj
 0001:0000e808       _FRS_RECUR                 1000f808     util.obj
 0001:0000e810       _FRS_SCANSYMLINK           1000f810     util.obj
 0001:0000e818       _FRS_NONE                  1000f818     util.obj
 0001:0000e820       _EF_NONMODAL               1000f820     util.obj
 0001:0000e828       _EF_CREATENEW              1000f828     util.obj
 0001:0000e830       _EF_ENABLE_F6              1000f830     util.obj
 0001:0000e838       _EF_DISABLEHISTORY         1000f838     util.obj
 0001:0000e840       _EF_DELETEONCLOSE          1000f840     util.obj
 0001:0000e848       _EF_IMMEDIATERETURN        1000f848     util.obj
 0001:0000e850       _EF_DELETEONLYFILEONCLOSE  1000f850     util.obj
 0001:0000e858       _EF_LOCKED                 1000f858     util.obj
 0001:0000e860       _EF_DISABLESAVEPOS         1000f860     util.obj
 0001:0000e868       _EF_OPENMODE_MASK          1000f868     util.obj
 0001:0000e870       _EF_OPENMODE_QUERY         1000f870     util.obj
 0001:0000e878       _EF_OPENMODE_NEWIFOPEN     1000f878     util.obj
 0001:0000e880       _EF_OPENMODE_USEEXISTING   1000f880     util.obj
 0001:0000e888       _EF_OPENMODE_BREAKIFOPEN   1000f888     util.obj
 0001:0000e890       _EF_OPENMODE_RELOADIFOPEN  1000f890     util.obj
 0001:0000e898       _EN_NONE                   1000f898     util.obj
 0001:0000e8a0       _MLF_SHOWERRMSG            1000f8a0     util.obj
 0001:0000e8a8       _MLF_DONOTUPDATEPANEL      1000f8a8     util.obj
 0001:0000e8b0       _MLF_HOLDTARGET            1000f8b0     util.obj
 0001:0000e8b8       _MLF_NONE                  1000f8b8     util.obj
 0001:0000e8c0       _FHELP_NOSHOWERROR         1000f8c0     util.obj
 0001:0000e8c8       _FHELP_SELFHELP            1000f8c8     util.obj
 0001:0000e8d0       _FHELP_FARHELP             1000f8d0     util.obj
 0001:0000e8d8       _FHELP_CUSTOMFILE          1000f8d8     util.obj
 0001:0000e8e0       _FHELP_CUSTOMPATH          1000f8e0     util.obj
 0001:0000e8e8       _FHELP_GUID                1000f8e8     util.obj
 0001:0000e8f0       _FHELP_USECONTENTS         1000f8f0     util.obj
 0001:0000e8f8       _FHELP_NONE                1000f8f8     util.obj
 0001:0000e900       _FFFS_COMMAS               1000f900     util.obj
 0001:0000e908       _FFFS_FLOATSIZE            1000f908     util.obj
 0001:0000e910       _FFFS_SHOWBYTESINDEX       1000f910     util.obj
 0001:0000e918       _FFFS_ECONOMIC             1000f918     util.obj
 0001:0000e920       _FFFS_THOUSAND             1000f920     util.obj
 0001:0000e928       _FFFS_MINSIZEINDEX         1000f928     util.obj
 0001:0000e930       _FFFS_MINSIZEINDEX_MASK    1000f930     util.obj
 0001:0000e938       _FFFS_NONE                 1000f938     util.obj
 0001:0000e940       _KMFLAGS_SILENTCHECK       1000f940     util.obj
 0001:0000e948       _KMFLAGS_NOSENDKEYSTOPLUGINS 1000f948     util.obj
 0001:0000e950       _KMFLAGS_ENABLEOUTPUT      1000f950     util.obj
 0001:0000e958       _KMFLAGS_LANGMASK          1000f958     util.obj
 0001:0000e960       _KMFLAGS_LUA               1000f960     util.obj
 0001:0000e968       _KMFLAGS_MOONSCRIPT        1000f968     util.obj
 0001:0000e970       _KMFLAGS_NONE              1000f970     util.obj
 0001:0000e978       _AKMFLAGS_NONE             1000f978     util.obj
 0001:0000ea00       _VF_NONMODAL               1000fa00     win.obj
 0001:0000ea08       _VF_DELETEONCLOSE          1000fa08     win.obj
 0001:0000ea10       _VF_ENABLE_F6              1000fa10     win.obj
 0001:0000ea18       _VF_DISABLEHISTORY         1000fa18     win.obj
 0001:0000ea20       _VF_IMMEDIATERETURN        1000fa20     win.obj
 0001:0000ea28       _VF_DELETEONLYFILEONCLOSE  1000fa28     win.obj
 0001:0000ea30       _VF_NONE                   1000fa30     win.obj
 0001:0000ea38       _FRS_RETUPDIR              1000fa38     win.obj
 0001:0000ea40       _FRS_RECUR                 1000fa40     win.obj
 0001:0000ea48       _FRS_SCANSYMLINK           1000fa48     win.obj
 0001:0000ea50       _FRS_NONE                  1000fa50     win.obj
 0001:0000ea58       _EF_NONMODAL               1000fa58     win.obj
 0001:0000ea60       _EF_CREATENEW              1000fa60     win.obj
 0001:0000ea68       _EF_ENABLE_F6              1000fa68     win.obj
 0001:0000ea70       _EF_DISABLEHISTORY         1000fa70     win.obj
 0001:0000ea78       _EF_DELETEONCLOSE          1000fa78     win.obj
 0001:0000ea80       _EF_IMMEDIATERETURN        1000fa80     win.obj
 0001:0000ea88       _EF_DELETEONLYFILEONCLOSE  1000fa88     win.obj
 0001:0000ea90       _EF_LOCKED                 1000fa90     win.obj
 0001:0000ea98       _EF_DISABLESAVEPOS         1000fa98     win.obj
 0001:0000eaa0       _EF_OPENMODE_MASK          1000faa0     win.obj
 0001:0000eaa8       _EF_OPENMODE_QUERY         1000faa8     win.obj
 0001:0000eab0       _EF_OPENMODE_NEWIFOPEN     1000fab0     win.obj
 0001:0000eab8       _EF_OPENMODE_USEEXISTING   1000fab8     win.obj
 0001:0000eac0       _EF_OPENMODE_BREAKIFOPEN   1000fac0     win.obj
 0001:0000eac8       _EF_OPENMODE_RELOADIFOPEN  1000fac8     win.obj
 0001:0000ead0       _EN_NONE                   1000fad0     win.obj
 0001:0000ead8       _MLF_SHOWERRMSG            1000fad8     win.obj
 0001:0000eae0       _MLF_DONOTUPDATEPANEL      1000fae0     win.obj
 0001:0000eae8       _MLF_HOLDTARGET            1000fae8     win.obj
 0001:0000eaf0       _MLF_NONE                  1000faf0     win.obj
 0001:0000eaf8       _FHELP_NOSHOWERROR         1000faf8     win.obj
 0001:0000eb00       _FHELP_SELFHELP            1000fb00     win.obj
 0001:0000eb08       _FHELP_FARHELP             1000fb08     win.obj
 0001:0000eb10       _FHELP_CUSTOMFILE          1000fb10     win.obj
 0001:0000eb18       _FHELP_CUSTOMPATH          1000fb18     win.obj
 0001:0000eb20       _FHELP_GUID                1000fb20     win.obj
 0001:0000eb28       _FHELP_USECONTENTS         1000fb28     win.obj
 0001:0000eb30       _FHELP_NONE                1000fb30     win.obj
 0001:0000eb38       _FFFS_COMMAS               1000fb38     win.obj
 0001:0000eb40       _FFFS_FLOATSIZE            1000fb40     win.obj
 0001:0000eb48       _FFFS_SHOWBYTESINDEX       1000fb48     win.obj
 0001:0000eb50       _FFFS_ECONOMIC             1000fb50     win.obj
 0001:0000eb58       _FFFS_THOUSAND             1000fb58     win.obj
 0001:0000eb60       _FFFS_MINSIZEINDEX         1000fb60     win.obj
 0001:0000eb68       _FFFS_MINSIZEINDEX_MASK    1000fb68     win.obj
 0001:0000eb70       _FFFS_NONE                 1000fb70     win.obj
 0001:0000eb78       _KMFLAGS_SILENTCHECK       1000fb78     win.obj
 0001:0000eb80       _KMFLAGS_NOSENDKEYSTOPLUGINS 1000fb80     win.obj
 0001:0000eb88       _KMFLAGS_ENABLEOUTPUT      1000fb88     win.obj
 0001:0000eb90       _KMFLAGS_LANGMASK          1000fb90     win.obj
 0001:0000eb98       _KMFLAGS_LUA               1000fb98     win.obj
 0001:0000eba0       _KMFLAGS_MOONSCRIPT        1000fba0     win.obj
 0001:0000eba8       _KMFLAGS_NONE              1000fba8     win.obj
 0001:0000ebb0       _AKMFLAGS_NONE             1000fbb0     win.obj
 0001:0000ebb8       _FSETCLR_REDRAW            1000fbb8     win.obj
 0001:0000ebc0       _FSETCLR_NONE              1000fbc0     win.obj
 0001:0000ebc8       _WIF_MODIFIED              1000fbc8     win.obj
 0001:0000ebd0       _WIF_CURRENT               1000fbd0     win.obj
 0001:0000ebd8       _WIF_MODAL                 1000fbd8     win.obj
 0001:0000ebe0       _WIF_NONE                  1000fbe0     win.obj
 0001:0000ebe8       _PF_PRELOAD                1000fbe8     win.obj
 0001:0000ebf0       _PF_DISABLEPANELS          1000fbf0     win.obj
 0001:0000ebf8       _PF_EDITOR                 1000fbf8     win.obj
 0001:0000ec00       _PF_VIEWER                 1000fc00     win.obj
 0001:0000ec08       _PF_FULLCMDLINE            1000fc08     win.obj
 0001:0000ec10       _PF_DIALOG                 1000fc10     win.obj
 0001:0000ec18       _PF_NONE                   1000fc18     win.obj
 0001:0000ec20       _VOPT_SAVEFILEPOSITION     1000fc20     win.obj
 0001:0000ec28       _VOPT_AUTODETECTCODEPAGE   1000fc28     win.obj
 0001:0000ec30       _VOPT_SHOWTITLEBAR         1000fc30     win.obj
 0001:0000ec38       _VOPT_SHOWKEYBAR           1000fc38     win.obj
 0001:0000ec40       _VOPT_SHOWSCROLLBAR        1000fc40     win.obj
 0001:0000ec48       _VOPT_QUICKVIEW            1000fc48     win.obj
 0001:0000ec50       _VOPT_NONE                 1000fc50     win.obj
 0001:0000ec58       _VSMFL_REDRAW              1000fc58     win.obj
 0001:0000ec60       _VSMFL_NONE                1000fc60     win.obj
 0001:0000ec68       _VSP_NOREDRAW              1000fc68     win.obj
 0001:0000ec70       _VSP_PERCENT               1000fc70     win.obj
 0001:0000ec78       _VSP_RELATIVE              1000fc78     win.obj
 0001:0000ec80       _VSP_NORETNEWPOS           1000fc80     win.obj
 0001:0000ec88       _VSP_NONE                  1000fc88     win.obj
 0001:0000ec90       _IPLFLAGS_SEPARATOR        1000fc90     win.obj
 0001:0000ec98       _IPLFLAGS_NONE             1000fc98     win.obj
 0001:0000eca0       _VMF_WRAP                  1000fca0     win.obj
 0001:0000eca8       _PMFLAGS_FULLSCREEN        1000fca8     win.obj
 0001:0000ecb0       _VMF_WORDWRAP              1000fcb0     win.obj
 0001:0000ecb8       _VMF_NONE                  1000fcb8     win.obj
 0001:0000ecc0       _PMFLAGS_DETAILEDSTATUS    1000fcc0     win.obj
 0001:0000ecc8       _PMFLAGS_ALIGNEXTENSIONS   1000fcc8     win.obj
 0001:0000ecd0       _PMFLAGS_CASECONVERSION    1000fcd0     win.obj
 0001:0000ecd8       _PMFLAGS_NONE              1000fcd8     win.obj
 0001:0000ece0       _FCF_FG_4BIT               1000fce0     win.obj
 0001:0000ece8       _FCF_BG_4BIT               1000fce8     win.obj
 0001:0000ecf0       _FCF_4BITMASK              1000fcf0     win.obj
 0001:0000ecf8       _FCF_RAWATTR_MASK          1000fcf8     win.obj
 0001:0000ed00       _FCF_EXTENDEDFLAGS         1000fd00     win.obj
 0001:0000ed08       _FCF_FG_BOLD               1000fd08     win.obj
 0001:0000ed10       _FCF_FG_ITALIC             1000fd10     win.obj
 0001:0000ed18       _FCF_FG_UNDERLINE          1000fd18     win.obj
 0001:0000ed20       _FCF_STYLEMASK             1000fd20     win.obj
 0001:0000ed28       _OPIF_DISABLEFILTER        1000fd28     win.obj
 0001:0000ed30       _FCF_NONE                  1000fd30     win.obj
 0001:0000ed38       _OPIF_DISABLESORTGROUPS    1000fd38     win.obj
 0001:0000ed40       _OPIF_DISABLEHIGHLIGHTING  1000fd40     win.obj
 0001:0000ed48       _OPIF_ADDDOTS              1000fd48     win.obj
 0001:0000ed50       _OPIF_RAWSELECTION         1000fd50     win.obj
 0001:0000ed58       _OPIF_REALNAMES            1000fd58     win.obj
 0001:0000ed60       _OPIF_SHOWNAMESONLY        1000fd60     win.obj
 0001:0000ed68       _OPIF_SHOWRIGHTALIGNNAMES  1000fd68     win.obj
 0001:0000ed70       _OPIF_SHOWPRESERVECASE     1000fd70     win.obj
 0001:0000ed78       _OPIF_COMPAREFATTIME       1000fd78     win.obj
 0001:0000ed80       _OPIF_EXTERNALGET          1000fd80     win.obj
 0001:0000ed88       _OPIF_EXTERNALPUT          1000fd88     win.obj
 0001:0000ed90       _OPIF_EXTERNALDELETE       1000fd90     win.obj
 0001:0000ed98       _OPIF_EXTERNALMKDIR        1000fd98     win.obj
 0001:0000eda0       _OPIF_USEATTRHIGHLIGHTING  1000fda0     win.obj
 0001:0000eda8       _OPIF_USECRC32             1000fda8     win.obj
 0001:0000edb0       _OPIF_USEFREESIZE          1000fdb0     win.obj
 0001:0000edb8       _OPIF_SHORTCUT             1000fdb8     win.obj
 0001:0000edc0       _OPIF_NONE                 1000fdc0     win.obj
 0001:0000edc8       _CDF_NONE                  1000fdc8     win.obj
 0001:0000edd0       _FMSG_WARNING              1000fdd0     win.obj
 0001:0000edd8       _FMSG_ERRORTYPE            1000fdd8     win.obj
 0001:0000ede0       _FMSG_KEEPBACKGROUND       1000fde0     win.obj
 0001:0000ede8       _OPM_SILENT                1000fde8     win.obj
 0001:0000edf0       _OPM_FIND                  1000fdf0     win.obj
 0001:0000edf8       _FMSG_LEFTALIGN            1000fdf8     win.obj
 0001:0000ee00       _FMSG_ALLINONE             1000fe00     win.obj
 0001:0000ee08       _OPM_VIEW                  1000fe08     win.obj
 0001:0000ee10       _OPM_EDIT                  1000fe10     win.obj
 0001:0000ee18       _FMSG_MB_OK                1000fe18     win.obj
 0001:0000ee20       _FMSG_MB_OKCANCEL          1000fe20     win.obj
 0001:0000ee28       _OPM_TOPLEVEL              1000fe28     win.obj
 0001:0000ee30       _OPM_DESCR                 1000fe30     win.obj
 0001:0000ee38       _FMSG_MB_ABORTRETRYIGNORE  1000fe38     win.obj
 0001:0000ee40       _OPM_QUICKVIEW             1000fe40     win.obj
 0001:0000ee48       _FMSG_MB_YESNO             1000fe48     win.obj
 0001:0000ee50       _OPM_PGDN                  1000fe50     win.obj
 0001:0000ee58       _FMSG_MB_YESNOCANCEL       1000fe58     win.obj
 0001:0000ee60       _FMSG_MB_RETRYCANCEL       1000fe60     win.obj
 0001:0000ee68       _OPM_COMMANDS              1000fe68     win.obj
 0001:0000ee70       _OPM_NONE                  1000fe70     win.obj
 0001:0000ee78       _FMSG_NONE                 1000fe78     win.obj
 0001:0000ef50       _FOSF_ACTIVE               1000ff50     win.obj
 0001:0000ef58       _DIF_BOXCOLOR              1000ff58     win.obj
 0001:0000ef60       _FOSF_NONE                 1000ff60     win.obj
 0001:0000ef68       _DIF_GROUP                 1000ff68     win.obj
 0001:0000ef70       _DIF_LEFTTEXT              1000ff70     win.obj
 0001:0000ef78       _DIF_MOVESELECT            1000ff78     win.obj
 0001:0000ef80       _DIF_SHOWAMPERSAND         1000ff80     win.obj
 0001:0000ef88       _DIF_CENTERGROUP           1000ff88     win.obj
 0001:0000ef90       _DIF_NOBRACKETS            1000ff90     win.obj
 0001:0000ef98       _DIF_MANUALADDHISTORY      1000ff98     win.obj
 0001:0000efa0       _DIF_SEPARATOR             1000ffa0     win.obj
 0001:0000efa8       _DIF_SEPARATOR2            1000ffa8     win.obj
 0001:0000efb0       _DIF_EDITOR                1000ffb0     win.obj
 0001:0000efb8       _DIF_LISTNOAMPERSAND       1000ffb8     win.obj
 0001:0000efc0       _DIF_LISTNOBOX             1000ffc0     win.obj
 0001:0000efc8       _DIF_HISTORY               1000ffc8     win.obj
 0001:0000efd0       _DIF_BTNNOCLOSE            1000ffd0     win.obj
 0001:0000efd8       _DIF_CENTERTEXT            1000ffd8     win.obj
 0001:0000efe0       _DIF_SEPARATORUSER         1000ffe0     win.obj
 0001:0000efe8       _DIF_SETSHIELD             1000ffe8     win.obj
 0001:0000eff0       _DIF_EDITEXPAND            1000fff0     win.obj
 0001:0000eff8       _DIF_DROPDOWNLIST          1000fff8     win.obj
 0001:0000f000       _DIF_USELASTHISTORY        10010000     win.obj
 0001:0000f008       _DIF_MASKEDIT              10010008     win.obj
 0001:0000f010       _DIF_LISTTRACKMOUSE        10010010     win.obj
 0001:0000f018       _DIF_LISTTRACKMOUSEINFOCUS 10010018     win.obj
 0001:0000f020       _DIF_SELECTONENTRY         10010020     win.obj
 0001:0000f028       _DIF_3STATE                10010028     win.obj
 0001:0000f030       _DIF_EDITPATH              10010030     win.obj
 0001:0000f038       _DIF_LISTWRAPMODE          10010038     win.obj
 0001:0000f040       _DIF_NOAUTOCOMPLETE        10010040     win.obj
 0001:0000f048       _DIF_LISTAUTOHIGHLIGHT     10010048     win.obj
 0001:0000f050       _DIF_LISTNOCLOSE           10010050     win.obj
 0001:0000f058       _DIF_EDITPATHEXEC          10010058     win.obj
 0001:0000f060       _DIF_HIDDEN                10010060     win.obj
 0001:0000f068       _DIF_READONLY              10010068     win.obj
 0001:0000f070       _DIF_NOFOCUS               10010070     win.obj
 0001:0000f078       _DIF_DISABLE               10010078     win.obj
 0001:0000f080       _DIF_DEFAULTBUTTON         10010080     win.obj
 0001:0000f088       _DIF_FOCUS                 10010088     win.obj
 0001:0000f090       _DIF_RIGHTTEXT             10010090     win.obj
 0001:0000f098       _DIF_WORDWRAP              10010098     win.obj
 0001:0000f0a0       _DIF_NONE                  100100a0     win.obj
 0001:0000f0a8       _ECF_TABMARKFIRST          100100a8     win.obj
 0001:0000f0b0       _ECF_TABMARKCURRENT        100100b0     win.obj
 0001:0000f0b8       _ECF_AUTODELETE            100100b8     win.obj
 0001:0000f0c0       _ECF_NONE                  100100c0     win.obj
 0001:0000f0c8       _FIB_ENABLEEMPTY           100100c8     win.obj
 0001:0000f0d0       _LIF_SELECTED              100100d0     win.obj
 0001:0000f0d8       _FIB_PASSWORD              100100d8     win.obj
 0001:0000f0e0       _FIB_EXPANDENV             100100e0     win.obj
 0001:0000f0e8       _LIF_CHECKED               100100e8     win.obj
 0001:0000f0f0       _LIF_SEPARATOR             100100f0     win.obj
 0001:0000f0f8       _FIB_NOUSELASTHISTORY      100100f8     win.obj
 0001:0000f100       _FIB_BUTTONS               10010100     win.obj
 0001:0000f108       _LIF_DISABLE               10010108     win.obj
 0001:0000f110       _LIF_GRAYED                10010110     win.obj
 0001:0000f118       _FIB_NOAMPERSAND           10010118     win.obj
 0001:0000f120       _FIB_EDITPATH              10010120     win.obj
 0001:0000f128       _LIF_HIDDEN                10010128     win.obj
 0001:0000f130       _LIF_DELETEUSERDATA        10010130     win.obj
 0001:0000f138       _FIB_EDITPATHEXEC          10010138     win.obj
 0001:0000f140       _LIF_NONE                  10010140     win.obj
 0001:0000f148       _FIB_NONE                  10010148     win.obj
 0001:0000f150       _PCIF_FROMMAIN             10010150     win.obj
 0001:0000f158       _PCIF_NONE                 10010158     win.obj
 0001:0000f160       _LIFIND_EXACTMATCH         10010160     win.obj
 0001:0000f168       _LIFIND_NONE               10010168     win.obj
 0001:0000f170       _LINFO_SHOWNOBOX           10010170     win.obj
 0001:0000f178       _FPF_LOADED                10010178     win.obj
 0001:0000f180       _LINFO_AUTOHIGHLIGHT       10010180     win.obj
 0001:0000f188       _LINFO_REVERSEHIGHLIGHT    10010188     win.obj
 0001:0000f190       _FPF_ANSI                  10010190     win.obj
 0001:0000f198       _LINFO_WRAPMODE            10010198     win.obj
 0001:0000f1a0       _FPF_NONE                  100101a0     win.obj
 0001:0000f1a8       _LINFO_SHOWAMPERSAND       100101a8     win.obj
 0001:0000f1b0       _LINFO_NONE                100101b0     win.obj
 0001:0000f1b8       _FarGuid                   100101b8     win.obj
 0001:0000f1c8       _FDLG_WARNING              100101c8     win.obj
 0001:0000f1d0       _FDLG_SMALLDIALOG          100101d0     win.obj
 0001:0000f1d8       _FDLG_NODRAWSHADOW         100101d8     win.obj
 0001:0000f1e0       _FDLG_NODRAWPANEL          100101e0     win.obj
 0001:0000f1e8       _FDLG_KEEPCONSOLETITLE     100101e8     win.obj
 0001:0000f1f0       _FDLG_NONE                 100101f0     win.obj
 0001:0000f1f8       _MIF_SELECTED              100101f8     win.obj
 0001:0000f200       _MIF_CHECKED               10010200     win.obj
 0001:0000f208       _MIF_SEPARATOR             10010208     win.obj
 0001:0000f210       _MIF_DISABLE               10010210     win.obj
 0001:0000f218       _MIF_GRAYED                10010218     win.obj
 0001:0000f220       _MIF_HIDDEN                10010220     win.obj
 0001:0000f228       _MIF_NONE                  10010228     win.obj
 0001:0000f230       _FMENU_SHOWAMPERSAND       10010230     win.obj
 0001:0000f238       _FMENU_WRAPMODE            10010238     win.obj
 0001:0000f240       _FMENU_AUTOHIGHLIGHT       10010240     win.obj
 0001:0000f248       _FMENU_REVERSEAUTOHIGHLIGHT 10010248     win.obj
 0001:0000f250       _FMENU_CHANGECONSOLETITLE  10010250     win.obj
 0001:0000f258       _FMENU_NONE                10010258     win.obj
 0001:0000f260       _PPIF_SELECTED             10010260     win.obj
 0001:0000f268       _PPIF_PROCESSDESCR         10010268     win.obj
 0001:0000f270       _PPIF_NONE                 10010270     win.obj
 0001:0000f278       _PFLAGS_SHOWHIDDEN         10010278     win.obj
 0001:0000f280       _PFLAGS_HIGHLIGHT          10010280     win.obj
 0001:0000f288       _PFLAGS_REVERSESORTORDER   10010288     win.obj
 0001:0000f290       _PFLAGS_USESORTGROUPS      10010290     win.obj
 0001:0000f298       _PFLAGS_SELECTEDFIRST      10010298     win.obj
 0001:0000f2a0       _PFLAGS_REALNAMES          100102a0     win.obj
 0001:0000f2a8       _PFLAGS_NUMERICSORT        100102a8     win.obj
 0001:0000f2b0       _PFLAGS_PANELLEFT          100102b0     win.obj
 0001:0000f2b8       _PFLAGS_DIRECTORIESFIRST   100102b8     win.obj
 0001:0000f2c0       _PFLAGS_USECRC32           100102c0     win.obj
 0001:0000f2c8       _PFLAGS_CASESENSITIVESORT  100102c8     win.obj
 0001:0000f2d0       _PFLAGS_PLUGIN             100102d0     win.obj
 0001:0000f2d8       _PFLAGS_VISIBLE            100102d8     win.obj
 0001:0000f2e0       _PFLAGS_FOCUS              100102e0     win.obj
 0001:0000f2e8       _PFLAGS_ALTERNATIVENAMES   100102e8     win.obj
 0001:0000f2f0       _PFLAGS_SHORTCUT           100102f0     win.obj
 0001:0000f2f8       _PFLAGS_NONE               100102f8     win.obj
 0001:0000f300       _PN_CMPNAME                10010300     win.obj
 0001:0000f308       _PN_CMPNAMELIST            10010308     win.obj
 0001:0000f310       _PN_GENERATENAME           10010310     win.obj
 0001:0000f318       _PN_CHECKMASK              10010318     win.obj
 0001:0000f320       _PN_SKIPPATH               10010320     win.obj
 0001:0000f328       _PN_SHOWERRORMESSAGE       10010328     win.obj
 0001:0000f330       _PN_NONE                   10010330     win.obj
 0001:0000f338       _XLAT_SWITCHKEYBLAYOUT     10010338     win.obj
 0001:0000f340       _XLAT_SWITCHKEYBBEEP       10010340     win.obj
 0001:0000f348       _XLAT_USEKEYBLAYOUTNAME    10010348     win.obj
 0001:0000f350       _XLAT_CONVERTALLCMDLINE    10010350     win.obj
 0001:0000f358       _XLAT_NONE                 10010358     win.obj
 0001:0000f6f8       ?kernel32@@3QB_WB          100106f8     vc_crt_fix_impl.obj
 0001:0000f7e8       _GS_ExceptionPointers      100107e8     LIBCMT:gs_report.obj
 0001:0000f7f0       ?module_names@?A0x89697e75@@3QBQB_WB 100107f0     libvcruntime:winapi_downlevel.obj
 0001:0000f8a0       ?candidate_modules@?1??try_get_FlsAlloc@@YAP6GKP6GXPAX@Z@ZXZ@4QBW4module_id@?A0x89697e75@@B 100108a0     libvcruntime:winapi_downlevel.obj
 0001:0000f8b4       ?candidate_modules@?1??try_get_FlsFree@@YAP6GHK@ZXZ@4QBW4module_id@?A0x89697e75@@B 100108b4     libvcruntime:winapi_downlevel.obj
 0001:0000f8c4       ?candidate_modules@?1??try_get_FlsGetValue@@YAP6GPAXK@ZXZ@4QBW4module_id@?A0x89697e75@@B 100108c4     libvcruntime:winapi_downlevel.obj
 0001:0000f8d8       ?candidate_modules@?1??try_get_FlsSetValue@@YAP6GHKPAX@ZXZ@4QBW4module_id@?A0x89697e75@@B 100108d8     libvcruntime:winapi_downlevel.obj
 0001:0000f8ec       ?candidate_modules@?1??try_get_InitializeCriticalSectionEx@@YAP6GHPAU_RTL_CRITICAL_SECTION@@KK@ZXZ@4QBW4module_id@?A0x89697e75@@B 100108ec     libvcruntime:winapi_downlevel.obj
 0001:0000f910       ?tokenTable@@3QBQBDB       10010910     libvcruntime:undname.obj
 0001:0000f948       ?nameTable@@3QBQBDB        10010948     libvcruntime:undname.obj
 0001:0000fa8c       ?rttiTable@@3QBQBDB        10010a8c     libvcruntime:undname.obj
 0001:000100e8       _errtable                  100110e8     libucrt:errno.obj
 0001:00010290       ?default_cmd_exe@?8???$common_popen_nolock@_W@@YAPAU_iobuf@@QB_W0HAAY01H@Z@4QB_WB 10011290     libucrt:popen.obj
 0001:000102a0       ?slash_c@?8???$common_popen_nolock@_W@@YAPAU_iobuf@@QB_W0HAAY01H@Z@4QB_WB 100112a0     libucrt:popen.obj
 0001:000102ac       ?comspec_name@?1???$get_comspec@_W@@YAPB_WXZ@4QB_WB 100112ac     libucrt:popen.obj
 0001:000102bc       ?backslash@?L@???$get_executable_path@_W@@YAPB_WQB_W@Z@4QB_WB 100112bc     libucrt:popen.obj
 0001:000102c0       ?path_name@?1???$get_path@_W@@YAPB_WXZ@4QB_WB 100112c0     libucrt:popen.obj
 0001:00010ea0       ?comspec_name@?1???$common_system@_W@@YAHQB_W@Z@4QB_WB 10011ea0     libucrt:system.obj
 0001:00010eb0       ?cmd_exe@?1???$common_system@_W@@YAHQB_W@Z@4QB_WB 10011eb0     libucrt:system.obj
 0001:00010ec0       ?slash_c@?1???$common_system@_W@@YAHQB_W@Z@4QB_WB 10011ec0     libucrt:system.obj
 0001:00010f90       ___acrt_initializers       10011f90     libucrt:initialization.obj
 0001:00011548       _over                      10012548     libucrt:fpctrl.obj
 0001:00011554       _under                     10012554     libucrt:fpctrl.obj
 0001:00011950       _module_names              10012950     libucrt:winapi_thunks.obj
 0001:00011df0       ?candidate_modules@?1??try_get_AreFileApisANSI@@YAP6GHXZXZ@4QBW4module_id@?A0x352e5c4b@@B 10012df0     libucrt:winapi_thunks.obj
 0001:00011e04       ?candidate_modules@?1??try_get_CompareStringEx@@YAP6GHPB_WK0H0HPAU_nlsversioninfo@@PAXJ@ZXZ@4QBW4module_id@?A0x352e5c4b@@B 10012e04     libucrt:winapi_thunks.obj
 0001:00011e1c       ?candidate_modules@?1??try_get_FlsAlloc@@YAP6GKP6GXPAX@Z@ZXZ@4QBW4module_id@?A0x352e5c4b@@B 10012e1c     libucrt:winapi_thunks.obj
 0001:00011e24       ?candidate_modules@?1??try_get_FlsFree@@YAP6GHK@ZXZ@4QBW4module_id@?A0x352e5c4b@@B 10012e24     libucrt:winapi_thunks.obj
 0001:00011e2c       ?candidate_modules@?1??try_get_FlsGetValue@@YAP6GPAXK@ZXZ@4QBW4module_id@?A0x352e5c4b@@B 10012e2c     libucrt:winapi_thunks.obj
 0001:00011e34       ?candidate_modules@?1??try_get_FlsSetValue@@YAP6GHKPAX@ZXZ@4QBW4module_id@?A0x352e5c4b@@B 10012e34     libucrt:winapi_thunks.obj
 0001:00011e3c       ?candidate_modules@?1??try_get_GetCurrentPackageId@@YAP6GJPAIPAE@ZXZ@4QBW4module_id@?A0x352e5c4b@@B 10012e3c     libucrt:winapi_thunks.obj
 0001:00011e58       ?candidate_modules@?1??try_get_InitializeCriticalSectionEx@@YAP6GHPAU_RTL_CRITICAL_SECTION@@KK@ZXZ@4QBW4module_id@?A0x352e5c4b@@B 10012e58     libucrt:winapi_thunks.obj
 0001:00011e60       ?candidate_modules@?1??try_get_LCMapStringEx@@YAP6GHPB_WK0HPA_WHPAU_nlsversioninfo@@PAXJ@ZXZ@4QBW4module_id@?A0x352e5c4b@@B 10012e60     libucrt:winapi_thunks.obj
 0001:00011e78       ?candidate_modules@?1??try_get_LocaleNameToLCID@@YAP6GKPB_WK@ZXZ@4QBW4module_id@?A0x352e5c4b@@B 10012e78     libucrt:winapi_thunks.obj
 0001:000126a0       ?dot_slash@?CD@???$common_spawnv@_W@@YAHHQB_WQBQB_W1@Z@4QB_WB 100136a0     libucrt:spawnv.obj
 0001:000126a8       ?extensions@?DB@???$common_spawnv@_W@@YAHHQB_WQBQB_W1@Z@4QAY04$$CB_WA 100136a8     libucrt:spawnv.obj
 0001:000126d0       __mb_locale_names          100136d0     libucrt:mbctype.obj
 0001:00012738       _LcidToLocaleNameTable     10013738     libucrt:lcidtoname_downlevel.obj
 0001:00013858       _LocaleNameToIndexTable    10014858     libucrt:lcidtoname_downlevel.obj
 0001:000147a8       ?equal_sign@?BP@???$construct_environment_block@_W@@YAHQBQB_WQAPA_W@Z@4QB_WB 100157a8     libucrt:cenvarg.obj
 0001:000147b0       LOG_name                   100157b0     libucrt:log10.obj
 0001:000147c0       _One                       100157c0     libucrt:ceil_pentium4.obj
 0001:000147d0       _Bns                       100157d0     libucrt:ceil_pentium4.obj
 0001:000147e0       _Zero                      100157e0     libucrt:ceil_pentium4.obj
 0001:000147f0       _S                         100157f0     libucrt:ceil_pentium4.obj
 0001:00014800       _NegZero                   10015800     libucrt:ceil_pentium4.obj
 0001:00014820       emask                      10015820     libucrt:log10_pentium4.obj
 0001:00014830       CC                         10015830     libucrt:log10_pentium4.obj
 0001:00014840       Magic                      10015840     libucrt:log10_pentium4.obj
 0001:00014850       hi_mask                    10015850     libucrt:log10_pentium4.obj
 0001:00014860       LOG10_2                    10015860     libucrt:log10_pentium4.obj
 0001:00014870       place_L                    10015870     libucrt:log10_pentium4.obj
 0001:00014890       One                        10015890     libucrt:log10_pentium4.obj
 0001:000148a0       Zero                       100158a0     libucrt:log10_pentium4.obj
 0001:000148b0       Two52                      100158b0     libucrt:log10_pentium4.obj
 0001:000148c0       Infs                       100158c0     libucrt:log10_pentium4.obj
 0001:000148d0       NaN                        100158d0     libucrt:log10_pentium4.obj
 0001:000148e0       coeff                      100158e0     libucrt:log10_pentium4.obj
 0001:0001493e       _log2max                   1001593e     libucrt:87tran.obj
 0001:00014948       _smallarg                  10015948     libucrt:87tran.obj
 0001:00014952       _half                      10015952     libucrt:87tran.obj
 0001:0001499e       One                        1001599e     libucrt:87disp.obj
 0001:000149a6       Three                      100159a6     libucrt:87disp.obj
 0001:000149ae       XAMtoTagTab                100159ae     libucrt:87disp.obj
 0001:000149c0       One                        100159c0     libucrt:common.obj
 0001:000149d4       DblMax                     100159d4     libucrt:common.obj
 0001:000149dc       DblMin                     100159dc     libucrt:common.obj
 0001:000149e4       IeeeAdjO                   100159e4     libucrt:common.obj
 0001:000149ec       IeeeAdjU                   100159ec     libucrt:common.obj
 0001:000149f4       _infinity                  100159f4     libucrt:common.obj
 0001:000149fc       _zero                      100159fc     libucrt:common.obj
 0001:000152e8       ?_names@?1??_get_fname@@9@9 100162e8     libucrt:fpexcept.obj
 0001:00015730       $$000000                   10016730     chkstk.obj
 0001:00015760       _band                      10016760 f   bit64.obj
 0001:00015890       _bor                       10016890 f   bit64.obj
 0001:000159c0       _bxor                      100169c0 f   bit64.obj
 0001:00015af0       _bnot                      10016af0 f   bit64.obj
 0001:00015b10       _lshift                    10016b10 f   bit64.obj
 0001:00015b70       _rshift                    10016b70 f   bit64.obj
 0001:00015bd0       _arshift                   10016bd0 f   bit64.obj
 0001:00015c30       _f_new                     10016c30 f   bit64.obj
 0001:00015e70       _f_tostring                10016e70 f   bit64.obj
 0001:00015eb0       _f_type                    10016eb0 f   bit64.obj
 0001:00015f20       _f_add                     10016f20 f   bit64.obj
 0001:00016050       _f_sub                     10017050 f   bit64.obj
 0001:00016090       _f_mul                     10017090 f   bit64.obj
 0001:000161d0       _f_div                     100171d0 f   bit64.obj
 0001:000162c0       _f_mod                     100172c0 f   bit64.obj
 0001:00016310       _f_unm                     10017310 f   bit64.obj
 0001:00016340       _f_eq                      10017340 f   bit64.obj
 0001:000163a0       _f_lt                      100173a0 f   bit64.obj
 0001:00016400       _f_le                      10017400 f   bit64.obj
 0001:000165c0       _check64                   100175c0 f   bit64.obj
 0001:000167c0       _CheckReloadDefaultScript  100177c0 f   exported.obj
 0001:000169f0       _FillFarMacroCall          100179f0 f   exported.obj
 0001:00016be0       _FillFarMacroCall_Callback@12 10017be0 f   exported.obj
 0001:00019490       _PushAnalyseInfo           1001a490 f   exported.obj
 0001:000195f0       _RegisterObject            1001a5f0 f   exported.obj
 0001:00019670       _RunDefaultScript          1001a670 f   exported.obj
 0001:00019e90       _errfile                   1001ae90 f   lflua.obj
 0001:00019ee0       _getF                      1001aee0 f   lflua.obj
 0001:00019fd0       _skipBOM                   1001afd0 f   lflua.obj
 0001:0001aff0       _FL_PushParams             1001bff0 f   luamacro.obj
 0001:0001b060       _InitMPR                   1001c060 f   luamacro.obj
 0001:0001b0b0       _MacroCallFarCallback@12   1001c0b0 f   luamacro.obj
 0001:0001b680       _uc_tostring               1001c680 f   lusercontrol.obj
 0001:0001b6e0       _uc_index                  1001c6e0 f   lusercontrol.obj
 0001:0001b7c0       _uc_newindex               1001c7c0 f   lusercontrol.obj
 0001:0001b890       _uc_New                    1001c890 f   lusercontrol.obj
 0001:0001bb30       _panel_SetDirectoriesFirst 1001cb30 f   service.obj
 0001:0001bb40       _panel_UpdatePanel         1001cb40 f   service.obj
 0001:0001bb50       _Settings_delete           1001cb50 f   service.obj
 0001:0001bbf0       _far_CopyToClipboard       1001cbf0 f   service.obj
 0001:0001bc90       _panel_SetSortMode         1001cc90 f   service.obj
 0001:0001bca0       _panel_SetViewMode         1001cca0 f   service.obj
 0001:0001bcb0       _Settings_createsubkey     1001ccb0 f   service.obj
 0001:0001bdb0       _panel_GetPanelDirectory   1001cdb0 f   service.obj
 0001:0001bec0       _far_PasteFromClipboard    1001cec0 f   service.obj
 0001:0001bf90       _Settings_opensubkey       1001cf90 f   service.obj
 0001:0001c040       _panel_SetPanelDirectory   1001d040 f   service.obj
 0001:0001c200       _far_InputRecordToName     1001d200 f   service.obj
 0001:0001c3d0       _editor_GetString          1001d3d0 f   service.obj
 0001:0001c3e0       _Settings_enum             1001d3e0 f   service.obj
 0001:0001c690       _editor_GetStringW         1001d690 f   service.obj
 0001:0001c6a0       _panel_GetCmdLine          1001d6a0 f   service.obj
 0001:0001c710       _far_NameToInputRecord     1001d710 f   service.obj
 0001:0001c780       _editor_SetString          1001d780 f   service.obj
 0001:0001c790       _panel_SetCmdLine          1001d790 f   service.obj
 0001:0001c7f0       _editor_SetStringW         1001d7f0 f   service.obj
 0001:0001c800       _far_LStricmp              1001d800 f   service.obj
 0001:0001c850       _editor_InsertString       1001d850 f   service.obj
 0001:0001c8c0       _Settings_free             1001d8c0 f   service.obj
 0001:0001c940       _panel_GetCmdLinePos       1001d940 f   service.obj
 0001:0001c9b0       _far_LStrnicmp             1001d9b0 f   service.obj
 0001:0001ca20       _editor_DeleteString       1001da20 f   service.obj
 0001:0001ca70       _panel_SetCmdLinePos       1001da70 f   service.obj
 0001:0001cad0       _far_FreeSettings          1001dad0 f   service.obj
 0001:0001cb50       _panel_InsertCmdLine       1001db50 f   service.obj
 0001:0001cbb0       _far_ProcessName           1001dbb0 f   service.obj
 0001:0001cdc0       _Settings_tostring         1001ddc0 f   service.obj
 0001:0001ce20       _panel_GetCmdLineSelection 1001de20 f   service.obj
 0001:0001cec0       _far_ColorDialog           1001dec0 f   service.obj
 0001:0001cfd0       _panel_SetCmdLineSelection 1001dfd0 f   service.obj
 0001:0001d060       _editor_InsertText         1001e060 f   service.obj
 0001:0001d0c0       _far_GetReparsePointInfo   1001e0c0 f   service.obj
 0001:0001d150       _editor_InsertTextW        1001e150 f   service.obj
 0001:0001d160       _editor_DeleteChar         1001e160 f   service.obj
 0001:0001d1b0       _editor_DeleteBlock        1001e1b0 f   service.obj
 0001:0001d200       _far_LIsAlpha              1001e200 f   service.obj
 0001:0001d250       _editor_UndoRedo           1001e250 f   service.obj
 0001:0001d2c0       _far_LIsAlphanum           1001e2c0 f   service.obj
 0001:0001d310       _far_LIsLower              1001e310 f   service.obj
 0001:0001d360       _far_LIsUpper              1001e360 f   service.obj
 0001:0001d3b0       _panel_SetSelection        1001e3b0 f   service.obj
 0001:0001d3c0       _panel_ClearSelection      1001e3c0 f   service.obj
 0001:0001d3d0       _panel_SetUserScreen       1001e3d0 f   service.obj
 0001:0001d420       _panel_GetUserScreen       1001e420 f   service.obj
 0001:0001d470       _far_LLowerBuf             1001e470 f   service.obj
 0001:0001d4d0       _far_LUpperBuf             1001e4d0 f   service.obj
 0001:0001d530       _panel_IsActivePanel       1001e530 f   service.obj
 0001:0001d580       _far_MkTemp                1001e580 f   service.obj
 0001:0001d600       _panel_SetActivePanel      1001e600 f   service.obj
 0001:0001d680       _far_GetDirList            1001e680 f   service.obj
 0001:0001d9b0       _far_MkLink                1001e9b0 f   service.obj
 0001:0001da80       _editor_SetKeyBar          1001ea80 f   service.obj
 0001:0001da90       _far_GetPathRoot           1001ea90 f   service.obj
 0001:0001db00       _viewer_SetKeyBar          1001eb00 f   service.obj
 0001:0001db10       _far_GetPluginDirList      1001eb10 f   service.obj
 0001:0001dba0       _editor_SetParam           1001eba0 f   service.obj
 0001:0001dcd0       _far_RestoreScreen         1001ecd0 f   service.obj
 0001:0001dd50       _far_SaveScreen            1001ed50 f   service.obj
 0001:0001ddf0       _editor_SetPosition        1001edf0 f   service.obj
 0001:0001ded0       _far_TruncPathStr          1001eed0 f   service.obj
 0001:0001dee0       _far_TruncStr              1001eee0 f   service.obj
 0001:0001def0       _editor_Redraw             1001eef0 f   service.obj
 0001:0001df40       _editor_ExpandTabs         1001ef40 f   service.obj
 0001:0001dfa0       _far_RecursiveSearch       1001efa0 f   service.obj
 0001:0001e0c0       _far_ConvertPath           1001f0c0 f   service.obj
 0001:0001e160       _editor_GetBookmarks       1001f160 f   service.obj
 0001:0001e170       _editor_GetSessionBookmarks 1001f170 f   service.obj
 0001:0001e180       _editor_AddSessionBookmark 1001f180 f   service.obj
 0001:0001e1d0       _far_AdvControl            1001f1d0 f   service.obj
 0001:0001e8a4       $LN73                      1001f8a4     service.obj
 0001:0001e8e8       $LN54                      1001f8e8     service.obj
 0001:0001e910       _editor_ClearSessionBookmarks 1001f910 f   service.obj
 0001:0001e960       _editor_DeleteSessionBookmark 1001f960 f   service.obj
 0001:0001e9c0       _editor_NextSessionBookmark 1001f9c0 f   service.obj
 0001:0001ea10       _editor_PrevSessionBookmark 1001fa10 f   service.obj
 0001:0001ea60       _editor_SetTitle           1001fa60 f   service.obj
 0001:0001eac0       _editor_GetTitle           1001fac0 f   service.obj
 0001:0001eb60       _editor_Quit               1001fb60 f   service.obj
 0001:0001ebb0       _editor_Select             1001fbb0 f   service.obj
 0001:0001ec80       _editor_GetSelection       1001fc80 f   service.obj
 0001:0001ef40       _far_MacroLoadAll          1001ff40 f   service.obj
 0001:0001f000       _far_MacroSaveAll          10020000 f   service.obj
 0001:0001f040       _far_MacroGetState         10020040 f   service.obj
 0001:0001f080       _far_MacroGetArea          10020080 f   service.obj
 0001:0001f0c0       _editor_TabToReal          100200c0 f   service.obj
 0001:0001f0d0       _far_MacroPost             100200d0 f   service.obj
 0001:0001f0e0       _editor_RealToTab          100200e0 f   service.obj
 0001:0001f0f0       _far_MacroCheck            100200f0 f   service.obj
 0001:0001f100       _far_MacroGetLastError     10020100 f   service.obj
 0001:0001f1c0       _far_SendDlgMessage        100201c0 f   service.obj
 0001:00020264       $LN163                     10021264     service.obj
 0001:00020270       $LN151                     10021270     service.obj
 0001:000202b4       $LN164                     100212b4     service.obj
 0001:0002033c       $LN152                     1002133c     service.obj
 0001:00020380       _far_MacroAdd              10021380 f   service.obj
 0001:00020570       _editor_AddColor           10021570 f   service.obj
 0001:000206c0       _far_MacroDelete           100216c0 f   service.obj
 0001:00020750       _editor_DelColor           10021750 f   service.obj
 0001:000207e0       _editor_GetColor           100217e0 f   service.obj
 0001:00020940       _far_MacroExecute          10021940 f   service.obj
 0001:00020a80       _editor_SaveFile           10021a80 f   service.obj
 0001:00020b10       _far_CPluginStartupInfo    10021b10 f   service.obj
 0001:00020b40       _far_MakeMenuItems         10021b40 f   service.obj
 0001:00020df0       _editor_ReadInput          10021df0 f   service.obj
 0001:00020e60       _far_Show                  10021e60 f   service.obj
 0001:00020ee0       _editor_ProcessInput       10021ee0 f   service.obj
 0001:00020f50       _editor_SubscribeChangeEvent 10021f50 f   service.obj
 0001:00020fe0       _far_Menu                  10021fe0 f   service.obj
 0001:000218e0       _far_CreateFileFilter      100228e0 f   service.obj
 0001:00021980       _filefilter_Free           10022980 f   service.obj
 0001:00021a00       _filefilter_gc             10022a00 f   service.obj
 0001:00021a10       _filefilter_tostring       10022a10 f   service.obj
 0001:00021a60       _filefilter_OpenMenu       10022a60 f   service.obj
 0001:00021ad0       _filefilter_Starting       10022ad0 f   service.obj
 0001:00021b40       _filefilter_IsFileInFilter 10022b40 f   service.obj
 0001:00021be0       _far_LoadPlugin            10022be0 f   service.obj
 0001:00021bf0       _far_ForcedLoadPlugin      10022bf0 f   service.obj
 0001:00021c00       _far_UnloadPlugin          10022c00 f   service.obj
 0001:00021c50       _far_FindPlugin            10022c50 f   service.obj
 0001:00021cf0       _far_GetPluginInformation  10022cf0 f   service.obj
 0001:00021f00       _far_DialogInit            10022f00 f   service.obj
 0001:000221c0       _far_GetPlugins            100231c0 f   service.obj
 0001:00022290       _far_IsPluginLoaded        10023290 f   service.obj
 0001:00022390       _far_DialogRun             10023390 f   service.obj
 0001:00022440       _far_XLat                  10023440 f   service.obj
 0001:00022530       _far_DialogFree            10023530 f   service.obj
 0001:00022590       _far_GetFileOwner          10023590 f   service.obj
 0001:00022620       _dialog_tostring           10023620 f   service.obj
 0001:00022680       _far_GetNumberOfLinks      10023680 f   service.obj
 0001:000226d0       _far_FormatFileSize        100236d0 f   service.obj
 0001:000227e0       _dialog_rawhandle          100237e0 f   service.obj
 0001:00022820       _far_FarClock              10023820 f   service.obj
 0001:00022890       _far_GetDlgItem            10023890 f   service.obj
 0001:00022900       _far_SetDlgItem            10023900 f   service.obj
 0001:00022960       _far_Message               10023960 f   service.obj
 0001:00022aa0       _far_SubscribeDialogDrawEvents 10023aa0 f   service.obj
 0001:00022ac0       _far_Timer                 10023ac0 f   service.obj
 0001:00022c40       _editor_Editor             10023c40 f   service.obj
 0001:00022d50       _viewer_Viewer             10023d50 f   service.obj
 0001:00022e40       _panel_CheckPanelsExist    10023e40 f   service.obj
 0001:00022e80       _panel_ClosePanel          10023e80 f   service.obj
 0001:00022ed0       _timer_Close               10023ed0 f   service.obj
 0001:00022ef0       _viewer_GetFileName        10023ef0 f   service.obj
 0001:00022fa0       _timer_tostring            10023fa0 f   service.obj
 0001:00022ff0       _panel_GetPanelInfo        10023ff0 f   service.obj
 0001:000231d0       _viewer_GetInfo            100241d0 f   service.obj
 0001:00023470       _timer_index               10024470 f   service.obj
 0001:00023620       _viewer_Quit               10024620 f   service.obj
 0001:00023660       _timer_newindex            10024660 f   service.obj
 0001:000237c0       _viewer_Redraw             100247c0 f   service.obj
 0001:00023800       _far_PluginStartupInfo     10024800 f   service.obj
 0001:000238a0       _viewer_Select             100248a0 f   service.obj
 0001:00023930       _panel_GetPanelItem        10024930 f   service.obj
 0001:00023940       _panel_GetSelectedPanelItem 10024940 f   service.obj
 0001:00023950       _viewer_SetPosition        10024950 f   service.obj
 0001:00023b20       _panel_GetCurrentPanelItem 10024b20 f   service.obj
 0001:00023b30       _far_GetCurrentDirectory   10024b30 f   service.obj
 0001:00023b90       _far_CreateSettings        10024b90 f   service.obj
 0001:00023d40       _viewer_SetMode            10024d40 f   service.obj
 0001:00023e60       _panel_GetPanelFormat      10024e60 f   service.obj
 0001:00023e70       _panel_GetPanelHostFile    10024e70 f   service.obj
 0001:00023e80       _editor_GetFileName        10024e80 f   service.obj
 0001:00023f30       _panel_GetColumnTypes      10024f30 f   service.obj
 0001:00023f40       _far_ShowHelp              10024f40 f   service.obj
 0001:00023fd0       _panel_GetColumnWidths     10024fd0 f   service.obj
 0001:00023fe0       _editor_GetInfo            10024fe0 f   service.obj
 0001:00024350       _panel_GetPanelPrefix      10025350 f   service.obj
 0001:00024360       _far_InputBox              10025360 f   service.obj
 0001:000244f0       _panel_RedrawPanel         100254f0 f   service.obj
 0001:000245d0       _Settings_set              100255d0 f   service.obj
 0001:000246e0       _far_GetMsg                100256e0 f   service.obj
 0001:00024740       _panel_SetCaseSensitiveSort 10025740 f   service.obj
 0001:00024750       _Settings_get              10025750 f   service.obj
 0001:00024860       _panel_SetNumericSort      10025860 f   service.obj
 0001:00024870       _panel_SetSortOrder        10025870 f   service.obj
 0001:00024880       _far_Text                  10025880 f   service.obj
 0001:00024910       _AddMacroData_gc           10025910 f   service.obj
 0001:00024920       _ChangePanelSelection      10025920 f   service.obj
 0001:00024b20       _CheckFlags                10025b20 f   service.obj
 0001:00024b70       _CheckFlagsFromTable       10025b70 f   service.obj
 0001:00024ea0       _CreateSynchroData         10025ea0 f   service.obj
 0001:00024ec0       _CustomAllocator           10025ec0 f   service.obj
 0001:00024f90       _FastGetString             10025f90 f   service.obj
 0001:00025010       _FillEditorSelect          10026010 f   service.obj
 0001:000250c0       _FillEditorSetPosition     100260c0 f   service.obj
 0001:000252e8       $LN16                      100262e8     service.obj
 0001:00025300       $LN13                      10026300     service.obj
 0001:00025310       _FillKeyBarTitles          10026310 f   service.obj
 0001:000254a0       _FrsUserFunc@12            100264a0 f   service.obj
 0001:00025560       _GetDialogItemType         10026560 f   service.obj
 0001:0002595c       $LN36                      1002695c     service.obj
 0001:000259c0       _GetMouseEvent             100269c0 f   service.obj
 0001:00025a30       _GetOptGuid                10026a30 f   service.obj
 0001:000265c0       _MacroSendString           100275c0 f   service.obj
 0001:00026850       $LN11                      10027850     service.obj
 0001:00026880       _OptInputRecord            10027880 f   service.obj
 0001:00026b60       _PushBookmarks             10027b60 f   service.obj
 0001:00026d80       $LN17                      10027d80     service.obj
 0001:00026d8c       $LN13                      10027d8c     service.obj
 0001:00026fc0       $LN36                      10027fc0     service.obj
 0001:00026fcc       $LN30                      10027fcc     service.obj
 0001:00026fe4       $LN37                      10027fe4     service.obj
 0001:00027008       $LN31                      10028008     service.obj
 0001:00027020       _PushDlgItem               10028020 f   service.obj
 0001:00027140       _PushDlgItemNum            10028140 f   service.obj
 0001:00027200       _PushEditorSetPosition     10028200 f   service.obj
 0001:000274cc       $LN16                      100284cc     service.obj
 0001:000274e4       $LN11                      100284e4     service.obj
 0001:00027500       _PushList                  10028500 f   service.obj
 0001:00027a80       _PushPluginHandle          10028a80 f   service.obj
 0001:00027c00       _PutPluginMenuItemToTable  10028c00 f   service.obj
 0001:00027cd0       _PutVersionInfoToTable     10028cd0 f   service.obj
 0001:00027d30       _SetDlgItem                10028d30 f   service.obj
 0001:00027da0       _SetFarDialogItem          10028da0 f   service.obj
 0001:00028010       _SetKeyBar                 10029010 f   service.obj
 0001:00028150       _SetPanelBooleanProperty   10029150 f   service.obj
 0001:000281e0       _SetPanelIntegerProperty   100291e0 f   service.obj
 0001:000282d0       __EditorGetString          100292d0 f   service.obj
 0001:00028500       __EditorInsertText         10029500 f   service.obj
 0001:000285e0       __EditorSetString          100295e0 f   service.obj
 0001:000286d0       __EditorTabConvert         100296d0 f   service.obj
 0001:00028770       _check_env_flag            10029770 f   service.obj
 0001:00028850       _get_env_flag              10029850 f   service.obj
 0001:00028978       $LN17                      10029978     service.obj
 0001:00028990       _get_panel_item            10029990 f   service.obj
 0001:00028a90       _get_string_info           10029a90 f   service.obj
 0001:00028b60       _luaopen_far               10029b60 f   service.obj
 0001:00028e30       _plugin_load               10029e30 f   service.obj
 0001:00028f10       _truncstring               10029f10 f   service.obj
 0001:00028fc0       _unic_gsub                 10029fc0 f   slnunico.obj
 0001:00029160       _str_format                1002a160 f   slnunico.obj
 0001:0002944c       $LN39                      1002a44c     slnunico.obj
 0001:00029468       $LN33                      1002a468     slnunico.obj
 0001:000294a0       _utf8_valid                1002a4a0 f   slnunico.obj
 0001:00029570       _unic_len                  1002a570 f   slnunico.obj
 0001:000295f0       _unic_sub                  1002a5f0 f   slnunico.obj
 0001:00029740       _str_reverse               1002a740 f   slnunico.obj
 0001:000298a0       _unic_lower                1002a8a0 f   slnunico.obj
 0001:000299f0       _unic_upper                1002a9f0 f   slnunico.obj
 0001:00029b40       _str_rep                   1002ab40 f   slnunico.obj
 0001:00029bc0       _unic_byte                 1002abc0 f   slnunico.obj
 0001:00029d60       _unic_char                 1002ad60 f   slnunico.obj
 0001:00029e50       _str_dump                  1002ae50 f   slnunico.obj
 0001:00029ec0       _unic_find                 1002aec0 f   slnunico.obj
 0001:00029ed0       _unic_match                1002aed0 f   slnunico.obj
 0001:00029ee0       _gmatch                    1002aee0 f   slnunico.obj
 0001:00029f70       _gfind_nodef               1002af70 f   slnunico.obj
 0001:00029fd0       _add_s                     1002afd0 f   slnunico.obj
 0001:0002a0c0       _add_value                 1002b0c0 f   slnunico.obj
 0001:0002a1d0       $LN13                      1002b1d0     slnunico.obj
 0001:0002a1e0       _addquoted                 1002b1e0 f   slnunico.obj
 0001:0002a2b0       $LN25                      1002b2b0     slnunico.obj
 0001:0002a2c0       $LN21                      1002b2c0     slnunico.obj
 0001:0002a320       _classend                  1002b320 f   slnunico.obj
 0001:0002a3d0       _end_capture               1002b3d0 f   slnunico.obj
 0001:0002a430       _gmatch_aux                1002b430 f   slnunico.obj
 0001:0002a510       _grab_one_utf8             1002b510 f   slnunico.obj
 0001:0002a5a0       _lmemfind                  1002b5a0 f   slnunico.obj
 0001:0002a790       _match                     1002b790 f   slnunico.obj
 0001:0002a914       $LN50                      1002b914     slnunico.obj
 0001:0002a92c       $LN46                      1002b92c     slnunico.obj
 0001:0002a958       $LN51                      1002b958     slnunico.obj
 0001:0002a96c       $LN47                      1002b96c     slnunico.obj
 0001:0002a990       _match_capture             1002b990 f   slnunico.obj
 0001:0002aa30       _match_class               1002ba30 f   slnunico.obj
 0001:0002ab48       $LN28                      1002bb48     slnunico.obj
 0001:0002ab78       $LN26                      1002bb78     slnunico.obj
 0001:0002aba0       _matchbalance              1002bba0 f   slnunico.obj
 0001:0002ac00       _max_expand                1002bc00 f   slnunico.obj
 0001:0002acf0       _min_expand                1002bcf0 f   slnunico.obj
 0001:0002b000       _push_captures             1002c000 f   slnunico.obj
 0001:0002b0c0       _push_onecapture           1002c0c0 f   slnunico.obj
 0001:0002b150       _scanformat                1002c150 f   slnunico.obj
 0001:0002b250       _singlematch               1002c250 f   slnunico.obj
 0001:0002b540       _start_capture             1002c540 f   slnunico.obj
 0001:0002b590       _unic_find_aux             1002c590 f   slnunico.obj
 0001:0002b7a0       _utf8_count                1002c7a0 f   slnunico.obj
 0001:0002b840       _utf8_deco                 1002c840 f   slnunico.obj
 0001:0002b910       _utf8_enco                 1002c910 f   slnunico.obj
 0001:0002ba00       _utf8_graphext             1002ca00 f   slnunico.obj
 0001:0002bb20       _utf8_oced                 1002cb20 f   slnunico.obj
 0001:0002bc00       _writer                    1002cc00 f   slnunico.obj
 0001:0002bc20       _io_type                   1002cc20 f   uliolib51.obj
 0001:0002bcc0       _io_close                  1002ccc0 f   uliolib51.obj
 0001:0002bd40       _io_gc                     1002cd40 f   uliolib51.obj
 0001:0002bd90       _io_tostring               1002cd90 f   uliolib51.obj
 0001:0002bde0       _io_open                   1002cde0 f   uliolib51.obj
 0001:0002bec0       _io_popen                  1002cec0 f   uliolib51.obj
 0001:0002bf40       _io_tmpfile                1002cf40 f   uliolib51.obj
 0001:0002bfc0       _io_input                  1002cfc0 f   uliolib51.obj
 0001:0002bfe0       _io_output                 1002cfe0 f   uliolib51.obj
 0001:0002c000       _f_lines                   1002d000 f   uliolib51.obj
 0001:0002c050       _io_lines                  1002d050 f   uliolib51.obj
 0001:0002c100       _io_read                   1002d100 f   uliolib51.obj
 0001:0002c150       _f_read                    1002d150 f   uliolib51.obj
 0001:0002c190       _io_write                  1002d190 f   uliolib51.obj
 0001:0002c1e0       _f_write                   1002d1e0 f   uliolib51.obj
 0001:0002c220       _f_seek                    1002d220 f   uliolib51.obj
 0001:0002c2d0       _f_setvbuf                 1002d2d0 f   uliolib51.obj
 0001:0002c380       _io_flush                  1002d380 f   uliolib51.obj
 0001:0002c420       _f_flush                   1002d420 f   uliolib51.obj
 0001:0002c4c0       _aux_close                 1002d4c0 f   uliolib51.obj
 0001:0002c4f0       _fileerror                 1002d4f0 f   uliolib51.obj
 0001:0002c570       _g_iofile                  1002d570 f   uliolib51.obj
 0001:0002c660       _g_read                    1002d660 f   uliolib51.obj
 0001:0002c810       _g_write                   1002d810 f   uliolib51.obj
 0001:0002c900       _io_fclose                 1002d900 f   uliolib51.obj
 0001:0002c980       _io_noclose                1002d980 f   uliolib51.obj
 0001:0002c9b0       _io_pclose                 1002d9b0 f   uliolib51.obj
 0001:0002ca30       _io_readline               1002da30 f   uliolib51.obj
 0001:0002ccf0       _pushresult                1002dcf0 f   uliolib51.obj
 0001:0002cd90       _read_chars                1002dd90 f   uliolib51.obj
 0001:0002ce30       _read_line                 1002de30 f   uliolib51.obj
 0001:0002cf00       _read_number               1002df00 f   uliolib51.obj
 0001:0002cf50       _ll_loadlib                1002df50 f   uloadlib51.obj
 0001:0002cfc0       _loader_Lua                1002dfc0 f   uloadlib51.obj
 0001:0002d010       _loader_C                  1002e010 f   uloadlib51.obj
 0001:0002d0a0       _loader_Croot              1002e0a0 f   uloadlib51.obj
 0001:0002d140       _loader_preload            1002e140 f   uloadlib51.obj
 0001:0002d1b0       _ll_require                1002e1b0 f   uloadlib51.obj
 0001:0002d360       _ll_module                 1002e360 f   uloadlib51.obj
 0001:0002d440       _ll_seeall                 1002e440 f   uloadlib51.obj
 0001:0002d4a0       _dooptions                 1002e4a0 f   uloadlib51.obj
 0001:0002d4e0       _findfile                  1002e4e0 f   uloadlib51.obj
 0001:0002d620       _gctm                      1002e620 f   uloadlib51.obj
 0001:0002d650       _ll_loadfunc               1002e650 f   uloadlib51.obj
 0001:0002d6d0       _ll_register               1002e6d0 f   uloadlib51.obj
 0001:0002d780       _loaderror                 1002e780 f   uloadlib51.obj
 0001:0002d920       _mkfuncname                1002e920 f   uloadlib51.obj
 0001:0002d970       _modinit                   1002e970 f   uloadlib51.obj
 0001:0002d9e0       _pushnexttemplate          1002e9e0 f   uloadlib51.obj
 0001:0002da70       _setfenv                   1002ea70 f   uloadlib51.obj
 0001:0002dae0       _setpath                   1002eae0 f   uloadlib51.obj
 0001:0002db90       _setprogdir                1002eb90 f   uloadlib51.obj
 0001:0002dcf0       $LN13                      1002ecf0     ustring.obj
 0001:0002e6c0       _ustring_OutputDebugString 1002f6c0 f   ustring.obj
 0001:0002e880       _ustring_system            1002f880 f   ustring.obj
 0001:00030110       _win_DeleteRegKey          10031110 f   win.obj
 0001:00030190       _win_DeleteRegValue        10031190 f   win.obj
 0001:00030220       _win_EnumRegKey            10031220 f   win.obj
 0001:00030310       _win_EnumRegValue          10031310 f   win.obj
 0001:00030400       _win_ExtractKey            10031400 f   win.obj
 0001:00030450       _win_GetFileInfo           10031450 f   win.obj
 0001:000304c0       _win_GetSystemTimeAsFileTime 100314c0 f   win.obj
 0001:000304f0       _win_FileTimeToSystemTime  100314f0 f   win.obj
 0001:00030560       _win_SystemTimeToFileTime  10031560 f   win.obj
 0001:00030660       _win_FileTimeToLocalFileTime 10031660 f   win.obj
 0001:000306d0       _win_CompareString         100316d0 f   win.obj
 0001:00030860       _win_wcscmp                10031860 f   win.obj
 0001:000308b0       _win_GetVirtualKeys        100318b0 f   win.obj
 0001:000308d0       _win_GetConsoleScreenBufferInfo 100318d0 f   win.obj
 0001:000309e0       _win_CopyFile              100319e0 f   win.obj
 0001:00030a50       _win_MoveFile              10031a50 f   win.obj
 0001:00030b20       _win_DeleteFile            10031b20 f   win.obj
 0001:00030b60       _win_CreateDir             10031b60 f   win.obj
 0001:00030c40       _win_RemoveDir             10031c40 f   win.obj
 0001:00030c80       _win_ShellExecute          10031c80 f   win.obj
 0001:00030d20       _win_GetEnv                10031d20 f   win.obj
 0001:00030dc0       _win_SetEnv                10031dc0 f   win.obj
 0001:00030e00       _win_SetRegKey             10031e00 f   win.obj
 0001:00031070       _win_GetRegKey             10032070 f   win.obj
 0001:000311f8       $LN17                      100321f8     win.obj
 0001:00031220       _CheckHKey                 10032220 f   win.obj
 0001:00031370       _ExtractKey                10032370 f   win.obj
 0001:000313f0       _PushWinFindData           100323f0 f   win.obj
 0001:00031530       _mkdir                     10032530 f   win.obj
 0001:000316d0       _pushSystemTime            100326d0 f   win.obj
 0001:00031770       ?EncodePointer@implementation@?1??EncodePointerWrapper@@YGPAXPAX@Z@SGPAX0@Z 10032770 f   vc_crt_fix_impl.obj
 0001:00031770       ?DecodePointer@implementation@?1??DecodePointerWrapper@@YGPAXPAX@Z@SGPAX0@Z 10032770 f   vc_crt_fix_impl.obj
 0001:00031780       ?GetModuleHandleExW@implementation@?1??GetModuleHandleExWWrapper@@YGHKPB_WPAPAUHINSTANCE__@@@Z@SGHK01@Z 10032780 f   vc_crt_fix_impl.obj
 0001:000317b0       ?InitializeSListHead@implementation@?1??InitializeSListHeadWrapper@@YGXPAT_SLIST_HEADER@@@Z@SGX0@Z 100327b0 f   vc_crt_fix_impl.obj
 0001:000317c0       ?InterlockedPopEntrySList@implementation@?1??InterlockedPopEntrySListWrapper@@YGPAU_SINGLE_LIST_ENTRY@@PAT_SLIST_HEADER@@@Z@SGPAU3@0@Z 100327c0 f   vc_crt_fix_impl.obj
 0001:000317c0       ?InterlockedFlushSList@implementation@?1??InterlockedFlushSListWrapper@@YGPAU_SINGLE_LIST_ENTRY@@PAT_SLIST_HEADER@@@Z@SGPAU3@0@Z 100327c0 f   vc_crt_fix_impl.obj
 0001:000317c0       ?RtlFirstEntrySList@implementation@?1??RtlFirstEntrySListWrapper@@YGPAU_SINGLE_LIST_ENTRY@@PAT_SLIST_HEADER@@@Z@SGPAU3@0@Z 100327c0 f   vc_crt_fix_impl.obj
 0001:000317c0       ?QueryDepthSList@implementation@?1??QueryDepthSListWrapper@@YGGPAT_SLIST_HEADER@@@Z@SGG0@Z 100327c0 f   vc_crt_fix_impl.obj
 0001:000317d0       ?InterlockedPushEntrySList@implementation@?1??InterlockedPushEntrySListWrapper@@YGPAU_SINGLE_LIST_ENTRY@@PAT_SLIST_HEADER@@PAU3@@Z@SGPAU3@01@Z 100327d0 f   vc_crt_fix_impl.obj
 0001:000317e0       ?InterlockedPushListSListEx@implementation@?1??InterlockedPushListSListExWrapper@@YGPAU_SINGLE_LIST_ENTRY@@PAT_SLIST_HEADER@@PAU3@1K@Z@SGPAU3@011K@Z 100327e0 f   vc_crt_fix_impl.obj
 0001:00031c90       $$000000                   10032c90     LIBCMT:lldiv.obj
 0001:00031d40       $$000000                   10032d40     LIBCMT:llmul.obj
 0001:00031d80       $$000000                   10032d80     LIBCMT:llrem.obj
 0001:00031e40       $$000000                   10032e40     LIBCMT:llshl.obj
 0001:00031e60       $$000000                   10032e60     LIBCMT:llshr.obj
 0001:00031e90       $$000000                   10032e90     LIBCMT:ullshr.obj
 0001:00031eb0       $$000000                   10032eb0     LIBCMT:_ftol2_.obj
 0001:00031f70       $$000000                   10032f70     LIBCMT:lldvrm.obj
 0001:0003204f       ?dllmain_crt_dispatch@@YGHQAUHINSTANCE__@@KQAX@Z 1003304f f   LIBCMT:dll_dllmain.obj
 0001:000320a2       ?dllmain_crt_process_attach@@YAHQAUHINSTANCE__@@QAX@Z 100330a2 f   LIBCMT:dll_dllmain.obj
 0001:000321b4       ?dllmain_crt_process_detach@@YAH_N@Z 100331b4 f   LIBCMT:dll_dllmain.obj
 0001:00032231       ?dllmain_dispatch@@YAHQAUHINSTANCE__@@KQAX@Z 10033231 f   LIBCMT:dll_dllmain.obj
 0001:0003232d       ?dllmain_raw@@YGHQAUHINSTANCE__@@KQAX@Z 1003332d f   LIBCMT:dll_dllmain.obj
 0001:00032514       ?find_pe_section@@YAPAU_IMAGE_SECTION_HEADER@@QAEI@Z 10033514 f   LIBCMT:utility.obj
 0001:00032aa0       $$000000                   10033aa0     LIBCMT:_sehprolg4_.obj
 0001:00032ce0       $$000000                   10033ce0     libvcruntime:memcpy.obj
 0001:00032f44       TrailingUpVec              10033f44     libvcruntime:memcpy.obj
 0001:00032ff0       TrailingDownVec            10033ff0     libvcruntime:memcpy.obj
 0001:00033260       $$000000                   10034260     libvcruntime:memset.obj
 0001:00033640       $$000000                   10034640     libvcruntime:strchr.obj
 0001:00033820       $$000000                   10034820     libvcruntime:memchr.obj
 0001:000338d0       $$000000                   100348d0     libvcruntime:strrchr.obj
 0001:00033a10       _ValidateLocalCookies      10034a10 f   libvcruntime:_chandler4_.obj
 0001:00033c40       $$000000                   10034c40     libvcruntime:_exsup4_.obj
 0001:00033cd0       __unwind_handler4          10034cd0 f   libvcruntime:_exsup4_.obj
 0001:00033f58       ?try_get_function@@YAPAXW4function_id@?A0x89697e75@@QBDQBW4module_id@2@2@Z 10034f58 f   libvcruntime:winapi_downlevel.obj
 0001:00033ff8       ?try_get_module@@YAPAUHINSTANCE__@@W4module_id@?A0x89697e75@@@Z 10034ff8 f   libvcruntime:winapi_downlevel.obj
 0001:00034240       $$000000                   10035240     libvcruntime:_exsup_.obj
 0001:00034260       __unwind_handler           10035260 f   libvcruntime:_exsup_.obj
 0001:000343f0       ??$common_vsprintf@Vstandard_base@__crt_stdio_output@@D@@YAH_KQADIQBDQAU__crt_locale_pointers@@1@Z 100353f0 f   libucrt:output.obj
 0001:0003456c       ??$common_vsprintf@Vstandard_base@__crt_stdio_output@@_W@@YAH_KQA_WIQB_WQAU__crt_locale_pointers@@QAD@Z 1003556c f   libucrt:output.obj
 0001:00034bf8       ??R<lambda_4f2c1eaeead2a5fc776db5b62ea0fb9b>@@QBEHXZ 10035bf8 f   libucrt:output.obj
 0001:00034f84       $LN54                      10035f84     libucrt:output.obj
 0001:000350a0       $LN54                      100360a0     libucrt:output.obj
 0001:000351c0       $LN54                      100361c0     libucrt:output.obj
 0001:00035fc5       $LN19                      10036fc5     libucrt:output.obj
 0001:00036dd1       ??$common_fsopen@_W@@YAPAU_iobuf@@QB_W0H@Z 10037dd1 f   libucrt:fopen.obj
 0001:00036f9f       ___hw_cw_sse2              10037f9f f   libucrt:ieee87.obj
 0001:0003742a       __hw_cw                    1003842a f   libucrt:ieee87.obj
 0001:0003754f       ??$common_strerror@D@@YAPADH@Z 1003854f f   libucrt:strerror.obj
 0001:00037746       ??$common_freopen@_W@@YAHQAPAU_iobuf@@QB_W1V__crt_stdio_stream@@H@Z 10038746 f   libucrt:freopen.obj
 0001:00037b53       _memcpy_s                  10038b53 f   libucrt:fread.obj
 0001:00037b53       _memcpy_s                  10038b53 f   libucrt:cfout.obj
 0001:00037b53       _memcpy_s                  10038b53 f   libucrt:mbctype.obj
 0001:00037b53       _memcpy_s                  10038b53 f   libucrt:input.obj
 0001:000382a0       $$000000                   100392a0     libucrt:strncmp.obj
 0001:00038320       $$000000                   10039320     libucrt:strncpy.obj
 0001:00038450       $$000000                   10039450     libucrt:strpbrk.obj
 0001:00038490       ??$common_popen@_W@@YAPAU_iobuf@@QB_W0@Z 10039490 f   libucrt:popen.obj
 0001:000385bc       ??$common_popen_nolock@_W@@YAPAU_iobuf@@QB_W0HAAY01H@Z 100395bc f   libucrt:popen.obj
 0001:00038819       ??$convert_popen_type_to_fdopen_mode@_W@@YA?AU?$fdopen_mode@_W@?A0x256a5dd0@@QB_W@Z 10039819 f   libucrt:popen.obj
 0001:0003887f       ??$get_comspec@_W@@YAPB_WXZ 1003987f f   libucrt:popen.obj
 0001:000388bd       ??$get_executable_path@_W@@YAPB_WQB_W@Z 100398bd f   libucrt:popen.obj
 0001:000389ce       ??$get_path@_W@@YAPB_WXZ   100399ce f   libucrt:popen.obj
 0001:00038a46       ?idtab@@YAPAUprocess_handle_pair@?A0x256a5dd0@@QAU_iobuf@@@Z 10039a46 f   libucrt:popen.obj
 0001:00038cfe       _common_flush_all          10039cfe f   libucrt:fflush.obj
 0001:00038e2f       ??$common_fgets@D@@YAPADQADHV__crt_stdio_stream@@@Z 10039e2f f   libucrt:fgets.obj
 0001:00038f80       ?common_fseek@@YAHV__crt_stdio_stream@@_JH@Z 10039f80 f   libucrt:fseek.obj
 0001:00039007       ?common_fseek_binary_mode_read_only_fast_track_nolock@@YA_NV__crt_stdio_stream@@_JH@Z 1003a007 f   libucrt:fseek.obj
 0001:000390e0       ?common_fseek_nolock@@YAHV__crt_stdio_stream@@_JH@Z 1003a0e0 f   libucrt:fseek.obj
 0001:000391d4       ??$common_ftell@J@@YAJV__crt_stdio_stream@@@Z 1003a1d4 f   libucrt:ftell.obj
 0001:00039241       ??$common_ftell_nolock@J@@YAJV__crt_stdio_stream@@@Z 1003a241 f   libucrt:ftell.obj
 0001:0003926c       ??$common_ftell_nolock@_J@@YA_JV__crt_stdio_stream@@@Z 1003a26c f   libucrt:ftell.obj
 0001:00039401       ?common_ftell_read_mode_nolock@@YA_JV__crt_stdio_stream@@_J1@Z 1003a401 f   libucrt:ftell.obj
 0001:00039585       ?common_ftell_translated_utf8_nolock@@YA_JV__crt_stdio_stream@@_J@Z 1003a585 f   libucrt:ftell.obj
 0001:000397af       ??R<lambda_b51c0495177f500e782686251704ae76>@@QBEIXZ 1003a7af f   libucrt:fwrite.obj
 0001:00039a3f       ??R<lambda_b721fa326cdb32351d23dfa67958c160>@@QBEHXZ 1003aa3f f   libucrt:setvbuf.obj
 0001:00039ad9       ?set_buffer@@YAHV__crt_stdio_stream@@QADIH@Z 1003aad9 f   libucrt:setvbuf.obj
 0001:00039b82       ??$generate_tmpfile_file_name@D@@YA_NQADI@Z 1003ab82 f   libucrt:tmpfile.obj
 0001:00039bfa       ??$get_tmpfile_buffer_nolock@D@@YAPADW4buffer_id@?A0xaff43c62@@@Z 1003abfa f   libucrt:tmpfile.obj
 0001:00039c34       ??$initialize_tmpfile_buffer_nolock@D@@YA_NW4buffer_id@?A0xaff43c62@@@Z 1003ac34 f   libucrt:tmpfile.obj
 0001:00039cd7       ?common_tmpfile@@YAHQAPAU_iobuf@@H@Z 1003acd7 f   libucrt:tmpfile.obj
 0001:00039d50       ?common_tmpfile_nolock@@YAHQAPAU_iobuf@@H@Z 1003ad50 f   libucrt:tmpfile.obj
 0001:0003aaa7       $LN38                      1003baa7     libucrt:input.obj
 0001:0003abab       $LN21                      1003bbab     libucrt:input.obj
 0001:0003b3b9       ??R<lambda_46b61f845ab707e407a45eac8005babe>@@QBE_NXZ 1003c3b9 f   libucrt:input.obj
 0001:0003b3b9       ??R<lambda_8c3c021eaae193171a8be69849aba706>@@QBE_NXZ 1003c3b9 f   libucrt:input.obj
 0001:0003b3b9       ??R<lambda_661b0265ab3c2216dbae5485f8b1b26f>@@QBE_NXZ 1003c3b9 f   libucrt:input.obj
 0001:0003b3e3       ??R<lambda_d82aded7e80d0a2836af81596bef263e>@@QBEHXZ 1003c3e3 f   libucrt:input.obj
 0001:0003e031       $LN22                      1003f031     libucrt:input.obj
 0001:0003e7b3       $LN18                      1003f7b3     libucrt:input.obj
 0001:0003ea04       ??$common_dupenv_s@_W@@YAHQAPA_WQAIQB_WHQBDH@Z 1003fa04 f   libucrt:getenv.obj
 0001:0003ea5f       ??$common_dupenv_s_nolock@_W@@YAHQAPA_WQAIQB_WHQBDH@Z 1003fa5f f   libucrt:getenv.obj
 0001:0003eb0d       ??$common_getenv@_W@@YAPA_WQB_W@Z 1003fb0d f   libucrt:getenv.obj
 0001:0003eb8d       ??$common_getenv_nolock@_W@@YAPA_WQB_W@Z 1003fb8d f   libucrt:getenv.obj
 0001:0003ec40       ??$common_system@_W@@YAHQB_W@Z 1003fc40 f   libucrt:system.obj
 0001:0003efbf       ?atexit_exception_filter@@YAHK@Z 1003ffbf f   libucrt:exit.obj
 0001:0003efd2       ?common_exit@@YAXHW4_crt_exit_cleanup_mode@@W4_crt_exit_return_mode@@@Z 1003ffd2 f   libucrt:exit.obj
 0001:0003f0eb       ?exit_or_terminate_process@@YAXI@Z 100400eb f   libucrt:exit.obj
 0001:0003f12c       ?is_managed_app@@YA_NXZ    1004012c f   libucrt:exit.obj
 0001:0003f170       ?try_cor_exit_process@@YAXI@Z 10040170 f   libucrt:exit.obj
 0001:0003f214       ??$common_configure_argv@D@@YAHW4_crt_argv_mode@@@Z 10040214 f   libucrt:argv_parsing.obj
 0001:0003f338       ??$parse_command_line@D@@YAXPADPAPAD0PAI2@Z 10040338 f   libucrt:argv_parsing.obj
 0001:0003f50d       ??$common_get_or_create_environment_nolock@_W@@YAPAPA_WXZ 1004050d f   libucrt:environment_initialization.obj
 0001:0003f53c       ??$common_initialize_environment_nolock@D@@YAHXZ 1004053c f   libucrt:environment_initialization.obj
 0001:0003f595       ??$common_initialize_environment_nolock@_W@@YAHXZ 10040595 f   libucrt:environment_initialization.obj
 0001:0003f5e9       ??$create_environment@D@@YAQAPADQAD@Z 100405e9 f   libucrt:environment_initialization.obj
 0001:0003f6ba       ??$create_environment@_W@@YAQAPA_WQA_W@Z 100406ba f   libucrt:environment_initialization.obj
 0001:0003f7b4       ??$free_environment@_W@@YAXQAPA_W@Z 100407b4 f   libucrt:environment_initialization.obj
 0001:0003f7b4       ??$free_environment@D@@YAXQAPAD@Z 100407b4 f   libucrt:environment_initialization.obj
 0001:0003f7e3       ??$initialize_environment_by_cloning_nolock@_W@@YAHXZ 100407e3 f   libucrt:environment_initialization.obj
 0001:0003f89c       ??$uninitialize_environment_internal@D@@YAXAAPAPAD@Z 1004089c f   libucrt:environment_initialization.obj
 0001:0003f8b7       ??$uninitialize_environment_internal@_W@@YAXAAPAPA_W@Z 100408b7 f   libucrt:environment_initialization.obj
 0001:0003fa24       ??R<lambda_275893d493268fdec8709772e3fcec0e>@@QBEHXZ 10040a24 f   libucrt:onexit.obj
 0001:0003fb44       ??R<lambda_4e60a939b0d047cfe11ddc22648dfba9>@@QBEHXZ 10040b44 f   libucrt:onexit.obj
 0001:0003fd19       _initialize_global_variables 10040d19 f   libucrt:initialization.obj
 0001:0003fd2b       _initialize_c              10040d2b f   libucrt:initialization.obj
 0001:0003fd45       _uninitialize_global_state_isolation 10040d45 f   libucrt:initialization.obj
 0001:0003fd45       _report_memory_leaks       10040d45 f   libucrt:initialization.obj
 0001:0003fd45       _initialize_global_state_isolation 10040d45 f   libucrt:initialization.obj
 0001:0003fd45       _initialize_environment    10040d45 f   libucrt:initialization.obj
 0001:0003fd45       _uninitialize_c            10040d45 f   libucrt:initialization.obj
 0001:0003fd48       _uninitialize_environment  10040d48 f   libucrt:initialization.obj
 0001:0003fd50       _initialize_pointers       10040d50 f   libucrt:initialization.obj
 0001:0003fd8d       _uninitialize_vcruntime    10040d8d f   libucrt:initialization.obj
 0001:0003fd96       _uninitialize_allocated_memory 10040d96 f   libucrt:initialization.obj
 0001:0003fe92       ?_strupr_s_l_stat@@YAHQADIQAU__crt_locale_pointers@@@Z 10040e92 f   libucrt:strupr.obj
 0001:000410a8       ??$common_tox_l@$1?internal_isupper_l@@YA_NHQAU__crt_locale_pointers@@@Z$1?internal_map_lower@@YAHH0@Z@@YAHHKQAU__crt_locale_pointers@@@Z 100420a8 f   libucrt:tolower_toupper.obj
 0001:000411f2       ?internal_isupper_l@@YA_NHQAU__crt_locale_pointers@@@Z 100421f2 f   libucrt:tolower_toupper.obj
 0001:00041a0c       ?construct_ptd@@YAXQAU__acrt_ptd@@QAPAU__crt_locale_data@@@Z 10042a0c f   libucrt:per_thread_data.obj
 0001:00041a85       ?destroy_fls@@YGXPAX@Z     10042a85 f   libucrt:per_thread_data.obj
 0001:00041aa6       ?destroy_ptd@@YAXQAU__acrt_ptd@@@Z 10042aa6 f   libucrt:per_thread_data.obj
 0001:00041b4f       ?replace_current_thread_locale_nolock@@YAXQAU__acrt_ptd@@QAU__crt_locale_data@@@Z 10042b4f f   libucrt:per_thread_data.obj
 0001:00041df9       ?fp_format_a@@YAHQBNPADIQADIH_NIQAU__crt_locale_pointers@@@Z 10042df9 f   libucrt:cvt.obj
 0001:000420fc       ?fp_format_e@@YAHQBNQADI1IH_NIQAU__crt_locale_pointers@@@Z 100430fc f   libucrt:cvt.obj
 0001:00042197       ?fp_format_e_internal@@YAHQADIH_NIQAU_strflt@@1QAU__crt_locale_pointers@@@Z 10043197 f   libucrt:cvt.obj
 0001:000422e2       ?fp_format_f@@YAHQBNQADI1IHQAU__crt_locale_pointers@@@Z 100432e2 f   libucrt:cvt.obj
 0001:0004236f       ?fp_format_f_internal@@YAHQADIHQAU_strflt@@_NQAU__crt_locale_pointers@@@Z 1004336f f   libucrt:cvt.obj
 0001:00042446       ?fp_format_g@@YAHQBNQADI1IH_NIQAU__crt_locale_pointers@@@Z 10043446 f   libucrt:cvt.obj
 0001:0004250e       ?fp_format_nan_or_infinity@@YAHW4__acrt_fp_class@@_NPADI1@Z 1004350e f   libucrt:cvt.obj
 0001:00042606       ?shift_bytes@@YAXQADI0H@Z  10043606 f   libucrt:cvt.obj
 0001:00042933       ?initialize_inherited_file_handles_nolock@@YAXXZ 10043933 f   libucrt:ioinit.obj
 0001:000429e9       ?initialize_stdio_handles_nolock@@YAXXZ 100439e9 f   libucrt:ioinit.obj
 0001:00042c1f       ?find_or_allocate_unused_stream_nolock@@YA?AV__crt_stdio_stream@@XZ 10043c1f f   libucrt:stream.obj
 0001:00042f26       ??$common_openfile@_W@@YAPAU_iobuf@@QB_W0HV__crt_stdio_stream@@@Z 10043f26 f   libucrt:openfile.obj
 0001:0004332e       ?get_global_action_nolock@@YAPAP6AXH@ZH@Z 1004432e f   libucrt:signal.obj
 0001:00043370       ?siglookup@@YAPAU__crt_signal_action_t@@HQAU1@@Z 10044370 f   libucrt:signal.obj
 0001:00043729       ??$common_tcsncpy_s@D@@YAHQADIQBDI@Z 10044729 f   libucrt:strncpy_s.obj
 0001:000437e5       ?try_get_CompareStringEx@@YAP6GHPB_WK0H0HPAU_nlsversioninfo@@PAXJ@ZXZ 100447e5 f   libucrt:winapi_thunks.obj
 0001:000437ff       ?try_get_function@@YAPAXW4function_id@?A0x352e5c4b@@QBDQBW4module_id@2@2@Z 100447ff f   libucrt:winapi_thunks.obj
 0001:0004389b       ?try_get_module@@YAPAUHINSTANCE__@@W4module_id@?A0x352e5c4b@@@Z 1004489b f   libucrt:winapi_thunks.obj
 0001:00043dfc       ??$translate_text_mode_nolock@D@@YAHHQADI@Z 10044dfc f   libucrt:read.obj
 0001:00043f53       ??$translate_text_mode_nolock@_W@@YAHHQA_WI@Z 10044f53 f   libucrt:read.obj
 0001:00044113       ?translate_ansi_or_utf8_nolock@@YAHHQADIQA_WI@Z 10045113 f   libucrt:read.obj
 0001:00044263       ?translate_utf16_from_console_nolock@@YAHHQA_WI@Z 10045263 f   libucrt:read.obj
 0001:000447ac       ??$common_refill_and_read_nolock@D@@YAHV__crt_stdio_stream@@@Z 100457ac f   libucrt:_filbuf.obj
 0001:00044938       ??$common_lseek@J@@YAJHJH@Z 10045938 f   libucrt:lseek.obj
 0001:00044a23       ??$common_lseek@_J@@YA_JH_JH@Z 10045a23 f   libucrt:lseek.obj
 0001:00044b28       ??$common_lseek_nolock@J@@YAJHJH@Z 10045b28 f   libucrt:lseek.obj
 0001:00044b7f       ??$common_lseek_nolock@_J@@YA_JH_JH@Z 10045b7f f   libucrt:lseek.obj
 0001:00044bfd       ?common_lseek_do_seek_nolock@@YAJQAXJH@Z 10045bfd f   libucrt:lseek.obj
 0001:0004506b       ??$common_getpath@_W@@YAPA_WQB_WQA_WI@Z 1004606b f   libucrt:getpath.obj
 0001:00045545       ??$common_fdopen@_W@@YAPAU_iobuf@@HQB_W@Z 10046545 f   libucrt:fdopen.obj
 0001:00045777       ?write_double_translated_ansi_nolock@@YA?AUwrite_result@?A0x47fa6670@@HQBDI@Z 10046777 f   libucrt:write.obj
 0001:0004592a       ?write_double_translated_unicode_nolock@@YA?AUwrite_result@?A0x47fa6670@@QBDI@Z 1004692a f   libucrt:write.obj
 0001:00045997       ?write_requires_double_translation_nolock@@YA_NH@Z 10046997 f   libucrt:write.obj
 0001:00045a0d       ?write_text_ansi_nolock@@YA?AUwrite_result@?A0x47fa6670@@HQBDI@Z 10046a0d f   libucrt:write.obj
 0001:00045aec       ?write_text_utf16le_nolock@@YA?AUwrite_result@?A0x47fa6670@@HQBDI@Z 10046aec f   libucrt:write.obj
 0001:00045bda       ?write_text_utf8_nolock@@YA?AUwrite_result@?A0x47fa6670@@HQBDI@Z 10046bda f   libucrt:write.obj
 0001:00045ffe       ??$common_flush_and_write_nolock@D@@YAHHV__crt_stdio_stream@@@Z 10046ffe f   libucrt:_flsbuf.obj
 0001:0004610f       ??$write_buffer_nolock@D@@YA_NDV__crt_stdio_stream@@@Z 1004710f f   libucrt:_flsbuf.obj
 0001:000461e6       ??$common_xtox@_KD@@YAH_KQADII_N@Z 100471e6 f   libucrt:xtoa.obj
 0001:00046288       ??$common_xtox_s@_KD@@YAH_KQADII_N@Z 10047288 f   libucrt:xtoa.obj
 0001:000463e1       ??$common_sopen_dispatch@D@@YAHQBDHHHQAHH@Z 100473e1 f   libucrt:open.obj
 0001:000464ad       ??$common_sopen_dispatch@_W@@YAHQB_WHHHQAHH@Z 100474ad f   libucrt:open.obj
 0001:00046579       ?configure_text_mode@@YAHHUfile_options@?A0x704126de@@HAAW4__crt_lowio_text_mode@@@Z 10047579 f   libucrt:open.obj
 0001:000467c6       ?create_file@@YAPAXQB_WQAU_SECURITY_ATTRIBUTES@@Ufile_options@?A0x704126de@@@Z 100477c6 f   libucrt:open.obj
 0001:000467eb       ?decode_open_create_flags@@YAKH@Z 100477eb f   libucrt:open.obj
 0001:0004685b       ?decode_options@@YA?AUfile_options@?A0x704126de@@HHH@Z 1004785b f   libucrt:open.obj
 0001:000469d7       ?truncate_ctrl_z_if_present@@YAHH@Z 100479d7 f   libucrt:open.obj
 0001:0004716e       ??$common_spawnv@_W@@YAHHQB_WQBQB_W1@Z 1004816e f   libucrt:spawnv.obj
 0001:00047378       ??$execute_command@_W@@YAHHQB_WQBQB_W1@Z 10048378 f   libucrt:spawnv.obj
 0001:000475a4       ??R<lambda_5056f36f92c185fae794536d1ce2027b>@@QBE_NXZ 100485a4 f   libucrt:spawnv.obj
 0001:000476ef       ??$common_spawnvp@_W@@YAHHQB_WQBQB_W1@Z 100486ef f   libucrt:spawnvp.obj
 0001:000479e3       ?<helper_func_cdecl>@<lambda_62bb7ecb46d0a77b591a051c43eb5ad1>@@CAHPBX0@Z 100489e3 f   libucrt:argv_wildcards.obj
 0001:000479fb       ??$common_expand_argv_wildcards@D@@YAHQAPADQAPAPAD@Z 100489fb f   libucrt:argv_wildcards.obj
 0001:00047b8b       ??$copy_and_add_argument_to_buffer@D@@YAHQBD0IAAV?$argument_list@D@?A0xb0e4b824@@@Z 10048b8b f   libucrt:argv_wildcards.obj
 0001:00047c21       ??$expand_argument_wildcards@D@@YAHQAD0AAV?$argument_list@D@?A0xb0e4b824@@@Z 10048c21 f   libucrt:argv_wildcards.obj
 0001:00047efc       ??R<lambda_ad1ced32f4ac17aa236e5ef05d6b3b7c>@@QBEXXZ 10048efc f   libucrt:mbctype.obj
 0001:00047fc0       ?CPtoLocaleName@@YAPB_WH@Z 10048fc0 f   libucrt:mbctype.obj
 0001:00047ffe       ?getSystemCP@@YAHH@Z       10048ffe f   libucrt:mbctype.obj
 0001:00048071       ?setSBCS@@YAXPAU__crt_multibyte_data@@@Z 10049071 f   libucrt:mbctype.obj
 0001:000480d6       ?setSBUpLow@@YAXPAU__crt_multibyte_data@@@Z 100490d6 f   libucrt:mbctype.obj
 0001:0004826a       ?setmbcp_internal@@YAHH_N@Z 1004926a f   libucrt:mbctype.obj
 0001:0004861c       ?x_ismbbtype_l@@YAHPAU__crt_locale_pointers@@IHH@Z 1004961c f   libucrt:ismbbyte.obj
 0001:000486a6       ?find_end_of_double_null_terminated_sequence@@YAPB_WQB_W@Z 100496a6 f   libucrt:get_environment_from_os.obj
 0001:000487b0       ??$common_set_variable_in_environment_nolock@_W@@YAHQA_WH@Z 100497b0 f   libucrt:setenv.obj
 0001:000489ed       ??$copy_environment@_W@@YAPAPA_WQAPA_W@Z 100499ed f   libucrt:setenv.obj
 0001:00048aab       ??$find_in_environment_nolock@_W@@YAHQB_WI@Z 10049aab f   libucrt:setenv.obj
 0001:00048d49       ?__acrt_LCMapStringA_stat@@YAHPAU__crt_locale_pointers@@PB_WKPBDHPADHHH@Z 10049d49 f   libucrt:lcmapstringa.obj
 0001:0004a9c0       ?free_crt_array_internal@@YAXQAPBXI@Z 1004b9c0 f   libucrt:inittime.obj
 0001:0004b21e       ?GetTableIndexFromLocaleName@@YAHPB_W@Z 1004c21e f   libucrt:lcidtoname_downlevel.obj
 0001:0004b77a       ___get_abstract_control_sse2 1004c77a f   libucrt:_fenvutils.obj
 0001:0004b7f7       ___get_abstract_control_x87 1004c7f7 f   libucrt:_fenvutils.obj
 0001:0004b86a       ___get_machine_control     1004c86a f   libucrt:_fenvutils.obj
 0001:0004b8db       ___get_machine_control_sse2 1004c8db f   libucrt:_fenvutils.obj
 0001:0004b95b       ___get_machine_status_sse2 1004c95b f   libucrt:_fenvutils.obj
 0001:0004b9bc       ___get_machine_status_x87  1004c9bc f   libucrt:_fenvutils.obj
 0001:0004bc70       ??$construct_command_line@_W@@YAHQBQB_WQAPA_W@Z 1004cc70 f   libucrt:cenvarg.obj
 0001:0004bd5b       ??$construct_environment_block@_W@@YAHQBQB_WQAPA_W@Z 1004cd5b f   libucrt:cenvarg.obj
 0001:0004c018       ??R<lambda_48d6eb5163ce2d6448ba1bf257f3e514>@@QBE_NXZ 1004d018 f   libucrt:cenvarg.obj
 0001:0004c05e       ??R<lambda_dd1c267fe327b8eb9e23cfd134fb4af8>@@QBEPA_WXZ 1004d05e f   libucrt:cenvarg.obj
 0001:0004c130       ?shortsort@@YAXPAD0IP6AHPBX1@Z@Z 1004d130 f   libucrt:qsort.obj
 0001:0004c1d0       ?swap@@YAXPAD0I@Z          1004d1d0 f   libucrt:qsort.obj
 0001:0004c64e       ?initialize_multibyte@@YAHXZ 1004d64e f   libucrt:multibyte_initializer.obj
 0001:0004c730       $$000000                   1004d730     libucrt:log10.obj
 0001:0004c880       $$000000                   1004d880     libucrt:ceil_pentium4.obj
 0001:0004c9b0       $$000000                   1004d9b0     libucrt:_strnicm.obj
 0001:0004ca60       $$000000                   1004da60     libucrt:log10_pentium4.obj
 0001:0004ccf0       $$000000                   1004dcf0     libucrt:87tran.obj
 0001:0004cef0       $$000000                   1004def0     libucrt:87disp.obj
 0001:0004d0f0       $$000000                   1004e0f0     libucrt:common.obj
 0001:0004d280       $$000000                   1004e280     libucrt:genexcep.obj
 0001:0004e290       $$000000                   1004f290     LIBCMT:ulldvrm.obj
 0001:0004e330       $$000000                   1004f330     LIBCMT:_sehprolg4gs_.obj
 0001:0004e390       $$000000                   1004f390     LIBCMT:alloca16.obj
 0001:0004e3c0       $$000000                   1004f3c0     libvcruntime:memmove.obj
 0001:0004e624       TrailingUpVec              1004f624     libvcruntime:memmove.obj
 0001:0004e6d0       TrailingDownVec            1004f6d0     libvcruntime:memmove.obj
 0001:0004e938       __sehtable$?dllmain_crt_process_attach@@YAHQAUHINSTANCE__@@QAX@Z 1004f938     LIBCMT:dll_dllmain.obj
 0001:0004e958       __sehtable$?dllmain_crt_process_detach@@YAH_N@Z 1004f958     LIBCMT:dll_dllmain.obj
 0001:0004e978       __sehtable$?dllmain_dispatch@@YAHQAUHINSTANCE__@@KQAX@Z 1004f978     LIBCMT:dll_dllmain.obj
 0001:0004e998       __sehtable$___scrt_is_nonwritable_in_current_image 1004f998     LIBCMT:utility.obj
 0001:0004e9b8       __sehtable$??$?RV<lambda_db08b09ef7aa9d4f8620ce68402612bc>@@AAV<lambda_4f2c1eaeead2a5fc776db5b62ea0fb9b>@@V<lambda_3ae262bc35d4ba6a3825c4f6bcaaf95c>@@@?$__crt_seh_guarded_call@H@@QAEH$$QAV<lambda_db08b09ef7aa9d4f8620ce68402612bc>@@AAV<lambda_4f2c1eaeead2a5fc776db5b62ea0fb9b>@@$$QAV<lambda_3ae262bc35d4ba6a3825c4f6bcaaf95c>@@@Z 1004f9b8     libucrt:output.obj
 0001:0004e9d8       __sehtable$??$common_fsopen@_W@@YAPAU_iobuf@@QB_W0H@Z 1004f9d8     libucrt:fopen.obj
 0001:0004e9f8       __sehtable$_fclose         1004f9f8     libucrt:fclose.obj
 0001:0004ea18       __sehtable$??$common_freopen@_W@@YAHQAPAU_iobuf@@QB_W1V__crt_stdio_stream@@H@Z 1004fa18     libucrt:freopen.obj
 0001:0004ea38       __sehtable$_fread_s        1004fa38     libucrt:fread.obj
 0001:0004ea58       __sehtable$_fgetc          1004fa58     libucrt:fgetc.obj
 0001:0004ea78       __sehtable$_rewind         1004fa78     libucrt:rewind.obj
 0001:0004ea98       __sehtable$_ungetc         1004fa98     libucrt:ungetc.obj
 0001:0004eab8       __sehtable$__pclose        1004fab8     libucrt:popen.obj
 0001:0004ead8       __sehtable$??$common_popen@_W@@YAPAU_iobuf@@QB_W0@Z 1004fad8     libucrt:popen.obj
 0001:0004eaf8       __sehtable$_clearerr_s     1004faf8     libucrt:clearerr.obj
 0001:0004eb18       __sehtable$_fflush         1004fb18     libucrt:fflush.obj
 0001:0004eb38       __sehtable$_common_flush_all 1004fb38     libucrt:fflush.obj
 0001:0004eb60       __sehtable$??$common_fgets@D@@YAPADQADHV__crt_stdio_stream@@@Z 1004fb60     libucrt:fgets.obj
 0001:0004eb80       __sehtable$?common_fseek@@YAHV__crt_stdio_stream@@_JH@Z 1004fb80     libucrt:fseek.obj
 0001:0004eba0       __sehtable$??$common_ftell@J@@YAJV__crt_stdio_stream@@@Z 1004fba0     libucrt:ftell.obj
 0001:0004ebc0       __sehtable$??$?RV<lambda_11b4f7b0d3157825a5656a18eba1ae27>@@AAV<lambda_b51c0495177f500e782686251704ae76>@@V<lambda_cf89b47920b5017557bfe891e78aca36>@@@?$__crt_seh_guarded_call@I@@QAEI$$QAV<lambda_11b4f7b0d3157825a5656a18eba1ae27>@@AAV<lambda_b51c0495177f500e782686251704ae76>@@$$QAV<lambda_cf89b47920b5017557bfe891e78aca36>@@@Z 1004fbc0     libucrt:fwrite.obj
 0001:0004ebe0       __sehtable$??$?RV<lambda_d92cfe8357b99225085016881b624cb0>@@AAV<lambda_b721fa326cdb32351d23dfa67958c160>@@V<lambda_42d75b0848218ec137fa420c8ba9fdf9>@@@?$__crt_seh_guarded_call@H@@QAEH$$QAV<lambda_d92cfe8357b99225085016881b624cb0>@@AAV<lambda_b721fa326cdb32351d23dfa67958c160>@@$$QAV<lambda_42d75b0848218ec137fa420c8ba9fdf9>@@@Z 1004fbe0     libucrt:setvbuf.obj
 0001:0004ec00       __sehtable$?common_tmpfile_nolock@@YAHQAPAU_iobuf@@H@Z 1004fc00     libucrt:tmpfile.obj
 0001:0004ec20       __sehtable$?common_tmpfile@@YAHQAPAU_iobuf@@H@Z 1004fc20     libucrt:tmpfile.obj
 0001:0004ec40       __sehtable$??$?RV<lambda_948e0c831b1eafdf53315a00da3ad7eb>@@AAV<lambda_d82aded7e80d0a2836af81596bef263e>@@V<lambda_9cb36f98846f17dfe48cc7d4c6a6fede>@@@?$__crt_seh_guarded_call@H@@QAEH$$QAV<lambda_948e0c831b1eafdf53315a00da3ad7eb>@@AAV<lambda_d82aded7e80d0a2836af81596bef263e>@@$$QAV<lambda_9cb36f98846f17dfe48cc7d4c6a6fede>@@@Z 1004fc40     libucrt:input.obj
 0001:0004ec60       __sehtable$??$common_getenv@_W@@YAPA_WQB_W@Z 1004fc60     libucrt:getenv.obj
 0001:0004ec80       __sehtable$??$common_dupenv_s@_W@@YAHQAPA_WQAIQB_WHQBDH@Z 1004fc80     libucrt:getenv.obj
 0001:0004eca0       __sehtable$?common_exit@@YAXHW4_crt_exit_cleanup_mode@@W4_crt_exit_return_mode@@@Z 1004fca0     libucrt:exit.obj
 0001:0004ecc8       __sehtable$??$?RV<lambda_800076c951b434888f4765a74a194fcc>@@AAV<lambda_4e60a939b0d047cfe11ddc22648dfba9>@@V<lambda_6dbb1268764f43b569ce7b67e331d33a>@@@?$__crt_seh_guarded_call@H@@QAEH$$QAV<lambda_800076c951b434888f4765a74a194fcc>@@AAV<lambda_4e60a939b0d047cfe11ddc22648dfba9>@@$$QAV<lambda_6dbb1268764f43b569ce7b67e331d33a>@@@Z 1004fcc8     libucrt:onexit.obj
 0001:0004ece8       __sehtable$??$?RV<lambda_995298e7d72eb4c2aab26c0585b3abe5>@@AAV<lambda_275893d493268fdec8709772e3fcec0e>@@V<lambda_293819299cbf9a7022e18b56a874bb5c>@@@?$__crt_seh_guarded_call@H@@QAEH$$QAV<lambda_995298e7d72eb4c2aab26c0585b3abe5>@@AAV<lambda_275893d493268fdec8709772e3fcec0e>@@$$QAV<lambda_293819299cbf9a7022e18b56a874bb5c>@@@Z 1004fce8     libucrt:onexit.obj
 0001:0004ed08       __sehtable$_terminate      1004fd08     libucrt:terminate.obj
 0001:0004ed28       __sehtable$??$?RV<lambda_9df27f884b057bc3edfc946cb5b7cf47>@@AAV<lambda_e69574bed617af4e071282c136b37893>@@V<lambda_cc0d902bcbbeb830f749456577db4721>@@@?$__crt_seh_guarded_call@X@@QAEX$$QAV<lambda_9df27f884b057bc3edfc946cb5b7cf47>@@AAV<lambda_e69574bed617af4e071282c136b37893>@@$$QAV<lambda_cc0d902bcbbeb830f749456577db4721>@@@Z 1004fd28     libucrt:per_thread_data.obj
 0001:0004ed48       __sehtable$??$?RV<lambda_3518db117f0e7cdb002338c5d3c47b6c>@@AAV<lambda_b2ea41f6bbb362cd97d94c6828d90b61>@@V<lambda_abdedf541bb04549bc734292b4a045d4>@@@?$__crt_seh_guarded_call@X@@QAEX$$QAV<lambda_3518db117f0e7cdb002338c5d3c47b6c>@@AAV<lambda_b2ea41f6bbb362cd97d94c6828d90b61>@@$$QAV<lambda_abdedf541bb04549bc734292b4a045d4>@@@Z 1004fd48     libucrt:per_thread_data.obj
 0001:0004ed68       __sehtable$??$?RV<lambda_51b6e8b1eb166f2a3faf91f424b38130>@@AAV<lambda_6250bd4b2a391816dd638c3bf72b0bcb>@@V<lambda_0b5a4a3e68152e1d9b943535f5f47bed>@@@?$__crt_seh_guarded_call@X@@QAEX$$QAV<lambda_51b6e8b1eb166f2a3faf91f424b38130>@@AAV<lambda_6250bd4b2a391816dd638c3bf72b0bcb>@@$$QAV<lambda_0b5a4a3e68152e1d9b943535f5f47bed>@@@Z 1004fd68     libucrt:per_thread_data.obj
 0001:0004ed88       __sehtable$??$?RV<lambda_5b71d36f03204c0beab531769a5b5694>@@AAV<lambda_be2b3da3f62db62e9dad5dc70221a656>@@V<lambda_8f9ce462984622f9bf76b59e2aaaf805>@@@?$__crt_seh_guarded_call@X@@QAEX$$QAV<lambda_5b71d36f03204c0beab531769a5b5694>@@AAV<lambda_be2b3da3f62db62e9dad5dc70221a656>@@$$QAV<lambda_8f9ce462984622f9bf76b59e2aaaf805>@@@Z 1004fd88     libucrt:per_thread_data.obj
 0001:0004eda8       __sehtable$___acrt_uninitialize_locale 1004fda8     libucrt:wsetlocale.obj
 0001:0004edc8       __sehtable$___acrt_initialize_lowio 1004fdc8     libucrt:ioinit.obj
 0001:0004ede8       __sehtable$?__acrt_stdio_allocate_stream@@YA?AV__crt_stdio_stream@@XZ 1004fde8     libucrt:stream.obj
 0001:0004ee08       __sehtable$??$?RV<lambda_123407a5e2ac06da108355a851863b7a>@@AAV<lambda_2fe9b910cf3cbf4a0ab98a02ba45b3ec>@@V<lambda_ae55bdf541ad94d75914d381c370e64d>@@@?$__crt_seh_guarded_call@H@@QAEH$$QAV<lambda_123407a5e2ac06da108355a851863b7a>@@AAV<lambda_2fe9b910cf3cbf4a0ab98a02ba45b3ec>@@$$QAV<lambda_ae55bdf541ad94d75914d381c370e64d>@@@Z 1004fe08     libucrt:close.obj
 0001:0004ee28       __sehtable$_raise          1004fe28     libucrt:signal.obj
 0001:0004ee48       __sehtable$??$?RV<lambda_a048d3beccc847880fc8490e18b82769>@@AAV<lambda_ec61778202f4f5fc7e7711acc23c3bca>@@V<lambda_f7496a158712204296dd6628a163878e>@@@?$__crt_seh_guarded_call@P6AXH@Z@@QAEP6AXH@Z$$QAV<lambda_a048d3beccc847880fc8490e18b82769>@@AAV<lambda_ec61778202f4f5fc7e7711acc23c3bca>@@$$QAV<lambda_f7496a158712204296dd6628a163878e>@@@Z 1004fe48     libucrt:signal.obj
 0001:0004ee68       __sehtable$___set_fpsr_sse2 1004fe68     libucrt:fpctrl.obj
 0001:0004ee88       __sehtable$__fcloseall     1004fe88     libucrt:closeall.obj
 0001:0004eea8       __sehtable$__read          1004fea8     libucrt:read.obj
 0001:0004eec8       __sehtable$??$common_lseek@J@@YAJHJH@Z 1004fec8     libucrt:lseek.obj
 0001:0004eee8       __sehtable$??$common_lseek@_J@@YA_JH_JH@Z 1004fee8     libucrt:lseek.obj
 0001:0004ef08       __sehtable$__pipe          1004ff08     libucrt:pipe.obj
 0001:0004ef30       __sehtable$??$common_fdopen@_W@@YAPAU_iobuf@@HQB_W@Z 1004ff30     libucrt:fdopen.obj
 0001:0004ef50       __sehtable$??$?RV<lambda_61cee617f5178ae960314fd4d05640a0>@@AAV<lambda_6978c1fb23f02e42e1d9e99668cc68aa>@@V<lambda_9cd88cf8ad10232537feb2133f08c833>@@@?$__crt_seh_guarded_call@H@@QAEH$$QAV<lambda_61cee617f5178ae960314fd4d05640a0>@@AAV<lambda_6978c1fb23f02e42e1d9e99668cc68aa>@@$$QAV<lambda_9cd88cf8ad10232537feb2133f08c833>@@@Z 1004ff50     libucrt:commit.obj
 0001:0004ef70       __sehtable$__write         1004ff70     libucrt:write.obj
 0001:0004ef90       __sehtable$??$common_sopen_dispatch@D@@YAHQBDHHHQAHH@Z 1004ff90     libucrt:open.obj
 0001:0004efb0       __sehtable$??$common_sopen_dispatch@_W@@YAHQB_WHHHQAHH@Z 1004ffb0     libucrt:open.obj
 0001:0004efd0       __sehtable$__rmtmp         1004ffd0     libucrt:rmtmp.obj
 0001:0004eff8       __sehtable$??$?RV<lambda_eee62cb4a147bfbb98180ad682ce6e17>@@AAV<lambda_5056f36f92c185fae794536d1ce2027b>@@V<lambda_57c77e0e75d6a1e6f8ecaa6bd26c2518>@@@?$__crt_seh_guarded_call@_N@@QAE_N$$QAV<lambda_eee62cb4a147bfbb98180ad682ce6e17>@@AAV<lambda_5056f36f92c185fae794536d1ce2027b>@@$$QAV<lambda_57c77e0e75d6a1e6f8ecaa6bd26c2518>@@@Z 1004fff8     libucrt:spawnv.obj
 0001:0004f018       __sehtable$___acrt_update_thread_multibyte_data 10050018     libucrt:mbctype.obj
 0001:0004f038       __sehtable$??$?RV<lambda_978dc153c237d78434369da87b74ff60>@@AAV<lambda_ad1ced32f4ac17aa236e5ef05d6b3b7c>@@V<lambda_4a8533e2866a575feecb8298ce776b0d>@@@?$__crt_seh_guarded_call@X@@QAEX$$QAV<lambda_978dc153c237d78434369da87b74ff60>@@AAV<lambda_ad1ced32f4ac17aa236e5ef05d6b3b7c>@@$$QAV<lambda_4a8533e2866a575feecb8298ce776b0d>@@@Z 10050038     libucrt:mbctype.obj
 0001:0004f058       __sehtable$__query_new_handler 10050058     libucrt:new_handler.obj
 0001:0004f078       __sehtable$___acrt_update_thread_locale_data 10050078     libucrt:locale_refcounting.obj
 0001:0004f098       __sehtable$__alloc_osfhnd  10050098     libucrt:osfinfo.obj
 0001:0004f0b8       __sehtable$___acrt_lowio_ensure_fh_exists 100500b8     libucrt:osfinfo.obj
 0001:0004f0d8       __sehtable$__IsNonwritableInCurrentImage 100500d8     LIBCMT:pesect.obj
 0001:0004f100       .edata                     10050100     luafar3.exp
 0001:0004f128       rgpv                       10050128     luafar3.exp
 0001:0004f1d0       rgszName                   100501d0     luafar3.exp
 0001:0004f278       rgwOrd                     10050278     luafar3.exp
 0001:0004f2cc       szName                     100502cc     luafar3.exp
 0001:0004f2d8       $N00001                    100502d8     luafar3.exp
 0001:0004f2e3       $N00002                    100502e3     luafar3.exp
 0001:0004f2f3       $N00003                    100502f3     luafar3.exp
 0001:0004f301       $N00004                    10050301     luafar3.exp
 0001:0004f30c       $N00005                    1005030c     luafar3.exp
 0001:0004f319       $N00006                    10050319     luafar3.exp
 0001:0004f328       $N00007                    10050328     luafar3.exp
 0001:0004f333       $N00008                    10050333     luafar3.exp
 0001:0004f33d       $N00009                    1005033d     luafar3.exp
 0001:0004f348       $N00010                    10050348     luafar3.exp
 0001:0004f35b       $N00011                    1005035b     luafar3.exp
 0001:0004f36b       $N00012                    1005036b     luafar3.exp
 0001:0004f37d       $N00013                    1005037d     luafar3.exp
 0001:0004f391       $N00014                    10050391     luafar3.exp
 0001:0004f39d       $N00015                    1005039d     luafar3.exp
 0001:0004f3ac       $N00016                    100503ac     luafar3.exp
 0001:0004f3bd       $N00017                    100503bd     luafar3.exp
 0001:0004f3cd       $N00018                    100503cd     luafar3.exp
 0001:0004f3e1       $N00019                    100503e1     luafar3.exp
 0001:0004f3f2       $N00020                    100503f2     luafar3.exp
 0001:0004f3fa       $N00021                    100503fa     luafar3.exp
 0001:0004f40b       $N00022                    1005040b     luafar3.exp
 0001:0004f41c       $N00023                    1005041c     luafar3.exp
 0001:0004f428       $N00024                    10050428     luafar3.exp
 0001:0004f439       $N00025                    10050439     luafar3.exp
 0001:0004f44a       $N00026                    1005044a     luafar3.exp
 0001:0004f455       $N00027                    10050455     luafar3.exp
 0001:0004f45d       $N00028                    1005045d     luafar3.exp
 0001:0004f474       $N00029                    10050474     luafar3.exp
 0001:0004f48a       $N00030                    1005048a     luafar3.exp
 0001:0004f4a0       $N00031                    100504a0     luafar3.exp
 0001:0004f4b6       $N00032                    100504b6     luafar3.exp
 0001:0004f4c8       $N00033                    100504c8     luafar3.exp
 0001:0004f4db       $N00034                    100504db     luafar3.exp
 0001:0004f4f0       $N00035                    100504f0     luafar3.exp
 0001:0004f505       $N00036                    10050505     luafar3.exp
 0001:0004f51c       $N00037                    1005051c     luafar3.exp
 0001:0004f532       $N00038                    10050532     luafar3.exp
 0001:0004f53e       $N00039                    1005053e     luafar3.exp
 0001:0004f552       $N00040                    10050552     luafar3.exp
 0001:0004f563       $N00041                    10050563     luafar3.exp
 0001:0004f573       $N00042                    10050573     luafar3.exp
 0002:00000f20       ?names@?5??LF_InitLuaState1@@9@9 10051f20     service.obj
 0002:00000f30       _pageMap                   10051f30     slnudata.obj
 0002:00002630       _groupMap                  10053630     slnudata.obj
 0002:000043e0       _groups                    100553e0     slnudata.obj
 0002:000045e0       _pageMap                   100555e0     slnunico.obj
 0002:00005ce0       _groupMap                  10056ce0     slnunico.obj
 0002:00007a90       _groups                    10058a90     slnunico.obj
 0002:00007cc0       ?__vcrt_flsindex@@3KA      10058cc0     libvcruntime:per_thread_data.obj
 0002:00007ce0       _errno_no_memory           10058ce0     libucrt:errno.obj
 0002:00007ce4       _doserrno_no_memory        10058ce4     libucrt:errno.obj
 0002:00007d94       ___acrt_flsindex           10058d94     libucrt:per_thread_data.obj
 0002:00007e90       ?__DAZ_ENABLED@?1??__set_fpsr_sse2@@9@9 10058e90     libucrt:fpctrl.obj
 0002:00007f9c       ___rgctypeflag             10058f9c     libucrt:mbctype.obj
 0002:00007fa0       ___rgcode_page_info        10058fa0     libucrt:mbctype.obj
 0002:00008530       _luaopen_bit               10059530     service.obj
 0002:00008534       _luaopen_ffi               10059534     service.obj
 0002:00008538       _luaopen_jit               10059538     service.obj
 0002:0000853c       ?Function@?1??EncodePointerWrapper@@9@4@4Q6GPAXPAX@ZA 1005953c     vc_crt_fix_impl.obj
 0002:00008540       ?$S1@?1??EncodePointerWrapper@@9@4@4IA 10059540     vc_crt_fix_impl.obj
 0002:00008544       ?Function@?1??DecodePointerWrapper@@9@4@4Q6GPAXPAX@ZA 10059544     vc_crt_fix_impl.obj
 0002:00008548       ?$S2@?1??DecodePointerWrapper@@9@4@4IA 10059548     vc_crt_fix_impl.obj
 0002:0000854c       ?Function@?1??GetModuleHandleExWWrapper@@9@12@4Q6GHKPB_WPAPAUHINSTANCE__@@@ZA 1005954c     vc_crt_fix_impl.obj
 0002:00008550       ?$S3@?1??GetModuleHandleExWWrapper@@9@12@4IA 10059550     vc_crt_fix_impl.obj
 0002:00008554       ?Function@?1??InitializeSListHeadWrapper@@9@4@4Q6GXPAT_SLIST_HEADER@@@ZA 10059554     vc_crt_fix_impl.obj
 0002:00008558       ?$S4@?1??InitializeSListHeadWrapper@@9@4@4IA 10059558     vc_crt_fix_impl.obj
 0002:0000855c       ?Function@?1??InterlockedFlushSListWrapper@@9@4@4Q6GPAU_SINGLE_LIST_ENTRY@@PAT_SLIST_HEADER@@@ZA 1005955c     vc_crt_fix_impl.obj
 0002:00008560       ?$S5@?1??InterlockedFlushSListWrapper@@9@4@4IA 10059560     vc_crt_fix_impl.obj
 0002:00008564       ?Function@?1??InterlockedPopEntrySListWrapper@@9@4@4Q6GPAU_SINGLE_LIST_ENTRY@@PAT_SLIST_HEADER@@@ZA 10059564     vc_crt_fix_impl.obj
 0002:00008568       ?$S6@?1??InterlockedPopEntrySListWrapper@@9@4@4IA 10059568     vc_crt_fix_impl.obj
 0002:0000856c       ?Function@?1??InterlockedPushEntrySListWrapper@@9@8@4Q6GPAU_SINGLE_LIST_ENTRY@@PAT_SLIST_HEADER@@PAU2@@ZA 1005956c     vc_crt_fix_impl.obj
 0002:00008570       ?$S7@?1??InterlockedPushEntrySListWrapper@@9@8@4IA 10059570     vc_crt_fix_impl.obj
 0002:00008574       ?Function@?1??InterlockedPushListSListExWrapper@@9@16@4Q6GPAU_SINGLE_LIST_ENTRY@@PAT_SLIST_HEADER@@PAU2@1K@ZA 10059574     vc_crt_fix_impl.obj
 0002:00008578       ?$S8@?1??InterlockedPushListSListExWrapper@@9@16@4IA 10059578     vc_crt_fix_impl.obj
 0002:0000857c       ?Function@?1??RtlFirstEntrySListWrapper@@9@4@4Q6GPAU_SINGLE_LIST_ENTRY@@PAT_SLIST_HEADER@@@ZA 1005957c     vc_crt_fix_impl.obj
 0002:00008580       ?$S9@?1??RtlFirstEntrySListWrapper@@9@4@4IA 10059580     vc_crt_fix_impl.obj
 0002:00008584       ?Function@?1??QueryDepthSListWrapper@@9@4@4Q6GGPAT_SLIST_HEADER@@@ZA 10059584     vc_crt_fix_impl.obj
 0002:00008588       ?$S10@?1??QueryDepthSListWrapper@@9@4@4IA 10059588     vc_crt_fix_impl.obj
 0002:0000858c       ?__proc_attached@@3HA      1005958c     LIBCMT:dll_dllmain.obj
 0002:000085a0       ?module_local_atexit_table@@3U_onexit_table_t@@A 100595a0     LIBCMT:utility.obj
 0002:000085ac       ?module_local_at_quick_exit_table@@3U_onexit_table_t@@A 100595ac     LIBCMT:utility.obj
 0002:000085b8       ?is_initialized_as_dll@@3_NA 100595b8     LIBCMT:utility.obj
 0002:000085d0       _GS_ExceptionRecord        100595d0     LIBCMT:gs_report.obj
 0002:00008620       _GS_ContextRecord          10059620     LIBCMT:gs_report.obj
 0002:000088ec       ?__vcrt_startup_thread_ptd@@3U__vcrt_ptd@@A 100598ec     libvcruntime:per_thread_data.obj
 0002:00008914       ___vcrt_lock_table         10059914     libvcruntime:locks.obj
 0002:0000892c       ___vcrt_locks_initialized  1005992c     libvcruntime:locks.obj
 0002:00008930       ?module_handles@@3PAPAUHINSTANCE__@@A 10059930     libvcruntime:winapi_downlevel.obj
 0002:00008940       ?encoded_function_pointers@@3PAPAXA 10059940     libvcruntime:winapi_downlevel.obj
 0002:00008990       ?heap@@3V_HeapManager@@A   10059990     libvcruntime:undname.obj
 0002:000089b0       ___idtabsiz                100599b0     libucrt:popen.obj
 0002:000089b4       ___idpairs                 100599b4     libucrt:popen.obj
 0002:000089b8       _narrow_tmpfile_buffer_pointers 100599b8     libucrt:tmpfile.obj
 0002:000089c4       _wide_tmpfile_buffer_pointers 100599c4     libucrt:tmpfile.obj
 0002:000089d0       _c_termination_complete    100599d0     libucrt:exit.obj
 0002:000089d4       _thread_local_exit_callback_func 100599d4     libucrt:exit.obj
 0002:000089d8       ?c_exit_complete@?5??common_exit@@YAXHW4_crt_exit_cleanup_mode@@W4_crt_exit_return_mode@@@Z@4_NA 100599d8     libucrt:exit.obj
 0002:000089e0       ?program_name@?5???$common_configure_argv@D@@YAHW4_crt_argv_mode@@@Z@4PADA 100599e0     libucrt:argv_parsing.obj
 0002:00008b10       ___acrt_invalid_parameter_handler 10059b10     libucrt:invalid_parameter.obj
 0002:00008b14       _enable_percent_n          10059b14     libucrt:printf_count_output.obj
 0002:00008d2c       _ctrlc_action              10059d2c     libucrt:signal.obj
 0002:00008d30       _ctrlbreak_action          10059d30     libucrt:signal.obj
 0002:00008d34       _abort_action              10059d34     libucrt:signal.obj
 0002:00008d38       _term_action               10059d38     libucrt:signal.obj
 0002:00008d40       _module_handles            10059d40     libucrt:winapi_thunks.obj
 0002:00008d90       _encoded_function_pointers 10059d90     libucrt:winapi_thunks.obj
 0002:00008e10       ?state_cache@?1??__acrt_is_packaged_app@@9@4JA 10059e10     libucrt:winapi_thunks.obj
 0002:00008e18       ___acrt_lock_table         10059e18     libucrt:locks.obj
 0002:00008f50       ___acrt_locks_initialized  10059f50     libucrt:locks.obj
 0002:00008f70       _fSystemSet                10059f70     libucrt:mbctype.obj
 0002:00008f74       ?initialized@?1??__acrt_initialize_multibyte@@9@4_NA 10059f74     libucrt:mbctype.obj
 0002:00008f94       ___acrt_new_handler        10059f94     libucrt:new_handler.obj
 0002:00008f98       _user_matherr              10059f98     libucrt:matherr.obj
 0002:00008f9c       ___acrt_global_new_mode    10059f9c     libucrt:new_mode.obj
 0002:00008fac       ___acrt_app_type           10059fac     libucrt:report_runtime_error.obj
 0002:00008fb8       __pmatherr_set             10059fb8     libucrt:libm_error.obj
 0003:00000b04       .idata$6                   1005ab04     kernel32:KERNEL32.dll
 0003:00000b20       .idata$6                   1005ab20     user32:USER32.dll
 0003:00000bc4       .idata$6                   1005abc4     advapi32:ADVAPI32.dll
 0003:00000bf6       .idata$6                   1005abf6     shell32:SHELL32.dll
 0003:0000118e       .idata$6                   1005b18e     lua51:lua51.dll
 0003:000011da       .idata$6                   1005b1da     rpcrt4:RPCRT4.dll
 0004:00000000       __guard_fids____dcrt_uninitialize_environments_nolock 1005c000     libucrt:environment_initialization.obj
 0004:00000008       __guard_fids__             1005c008     libucrt:initialization.obj
 0004:00000068       __guard_fids____acrt_initialize_ptd 1005c068     libucrt:per_thread_data.obj
 0004:0000006c       __guard_fids__             1005c06c     libucrt:stdio_initializer.obj
 0004:00000070       __guard_fids__             1005c070     libucrt:stdio_initializer.obj
 0004:00000074       __guard_fids_??$expand_argument_wildcards@D@@YAHQAD0AAV?$argument_list@D@?A0xb0e4b824@@@Z 1005c074     libucrt:argv_wildcards.obj
 0004:00000078       __guard_fids__             1005c078     libucrt:locale_initializer.obj
 0004:0000007c       __guard_fids__             1005c07c     libucrt:tmpfile_initializer.obj
 0004:00000080       __guard_fids__             1005c080     libucrt:multibyte_initializer.obj
 0004:00000084       __guard_fids____libm_error_support 1005c084     libucrt:libm_error.obj
 0004:00000088       __guard_fids__             1005c088     libucrt:console_output_initializer.obj
 0004:0000008c       __guard_fids__             1005c08c     libucrt:sse2_initializer.obj
 0004:00000090       __guard_fids_?dllmain_crt_process_attach@@YAHQAUHINSTANCE__@@QAX@Z 1005c090     LIBCMT:dll_dllmain.obj
 0004:00000098       __guard_fids_?dllmain_dispatch@@YAHQAUHINSTANCE__@@KQAX@Z 1005c098     LIBCMT:dll_dllmain.obj
 0004:0000009c       __guard_fids__             1005c09c     LIBCMT:guard_support.obj
 0004:000000a0       __guard_fids____vcrt_initialize_ptd 1005c0a0     libvcruntime:per_thread_data.obj
 0005:00000060       $R000000                   1005d060     luafar3.res
